 diamond_support

 Timestamp is 5c762214 (Wed Feb 27 12:37:24 2019)

 Preferred load address is 10000000

 Start         Length     Name                   Class
 0001:00000000 00005aa8H .text$di                CODE
 0001:00005ab0 0001450eH .text$mn                CODE
 0001:00019fc0 00004f04H .text$x                 CODE
 0001:0001eed0 000010cbH .text$yd                CODE
 0002:00000000 00000834H .idata$5                DATA
 0002:00000834 00000004H .CRT$XCA                DATA
 0002:00000838 00000358H .CRT$XCU                DATA
 0002:00000b90 00000004H .CRT$XCZ                DATA
 0002:00000b94 00000004H .CRT$XIA                DATA
 0002:00000b98 00000004H .CRT$XIAA               DATA
 0002:00000b9c 00000004H .CRT$XIC                DATA
 0002:00000ba0 00000004H .CRT$XIZ                DATA
 0002:00000bb0 00002a10H .rdata                  DATA
 0002:000035c0 00000078H .rdata$debug            DATA
 0002:00003638 00001204H .rdata$r                DATA
 0002:00004840 00000478H .rdata$sxdata           DATA
 0002:00004cb8 00000004H .rtc$IAA                DATA
 0002:00004cbc 00000004H .rtc$IZZ                DATA
 0002:00004cc0 00000004H .rtc$TAA                DATA
 0002:00004cc4 00000004H .rtc$TZZ                DATA
 0002:00004cc8 000054fcH .xdata$x                DATA
 0002:0000a1d0 00000058H .edata                  DATA
 0002:0000a228 00000104H .idata$2                DATA
 0002:0000a32c 00000014H .idata$3                DATA
 0002:0000a340 00000834H .idata$4                DATA
 0002:0000ab74 00006f28H .idata$6                DATA
 0003:00000000 000000f4H .data                   DATA
 0003:000000f8 00000968H .data$r                 DATA
 0003:00000a60 000009c4H .bss                    DATA
 0004:00000000 00000058H .rsrc$01                DATA
 0004:00000060 00000180H .rsrc$02                DATA

  Address         Publics by Value              Rva+Base       Lib:Object

 0000:00000000       ___guard_fids_table        00000000     <absolute>
 0000:00000000       ___guard_flags             00000000     <absolute>
 0000:00000000       ___guard_fids_count        00000000     <absolute>
 0000:00000000       __except_list              00000000     <absolute>
 0000:0000011e       ___safe_se_handler_count   0000011e     <absolute>
 0000:00009876       __fltused                  00009876     <absolute>
 0000:00009876       __ldused                   00009876     <absolute>
 0000:00000000       ___ImageBase               10000000     <linker-defined>
 0001:00005ab0       ??$_Allocate@D@std@@YAPADIPAD@Z 10006ab0 f i DiamondBuildPrompter.obj
 0001:00005ae0       ??$addressof@D@std@@YAPADAAD@Z 10006ae0 f i DiamondBuildPrompter.obj
 0001:00005af0       ??$atomic@H@?$QAtomicOpsBySize@$03@@CAPAJPAH@Z 10006af0 f i DiamondBuildPrompter.obj
 0001:00005b00       ??$construct@PADAAPAD@?$_Wrap_alloc@V?$allocator@D@std@@@std@@QAEXPAPADAAPAD@Z 10006b00 f i DiamondBuildPrompter.obj
 0001:00005b20       ??$construct@PADAAPAD@?$allocator@D@std@@QAEXPAPADAAPAD@Z 10006b20 f i DiamondBuildPrompter.obj
 0001:00005b40       ??$construct@PADAAPAD@?$allocator_traits@V?$allocator@D@std@@@std@@SAXAAV?$allocator@D@1@PAPADAAPAD@Z 10006b40 f i DiamondBuildPrompter.obj
 0001:00005b60       ??$deref@H@?$QAtomicOpsBySize@$03@@SA_NAAH@Z 10006b60 f i DiamondBuildPrompter.obj
 0001:00005b80       ??$destroy@PAD@?$_Wrap_alloc@V?$allocator@D@std@@@std@@QAEXPAPAD@Z 10006b80 f i DiamondBuildPrompter.obj
 0001:00005b90       ??$destroy@PAD@?$allocator@D@std@@QAEXPAPAD@Z 10006b90 f i DiamondBuildPrompter.obj
 0001:00005ba0       ??$destroy@PAD@?$allocator_traits@V?$allocator@D@std@@@std@@SAXAAV?$allocator@D@1@PAPAD@Z 10006ba0 f i DiamondBuildPrompter.obj
 0001:00005bb0       ??$forward@AAPAD@std@@YAAAPADAAPAD@Z 10006bb0 f i DiamondBuildPrompter.obj
 0001:00005bc0       ??$load@H@?$QGenericAtomicOps@U?$QAtomicOpsBySize@$03@@@@SAHABH@Z 10006bc0 f i DiamondBuildPrompter.obj
 0001:00005bd0       ??$ref@H@?$QAtomicOpsBySize@$03@@SA_NAAH@Z 10006bd0 f i DiamondBuildPrompter.obj
 0001:00005bf0       ??0?$PrompterBase@VDiamondBuildPrompter@LocalWorkflow@U2@@@U2@@QAE@PAVActor@Workflow@1@_N@Z 10006bf0 f i DiamondBuildPrompter.obj
 0001:00005c20       ??0?$QForeachContainer@V?$QList@PAVPort@Workflow@U2@@@@@@QAE@ABV?$QList@PAVPort@Workflow@U2@@@@@Z 10006c20 f i DiamondBuildPrompter.obj
 0001:00005c60       ??0?$QList@PAVPort@Workflow@U2@@@@QAE@ABV0@@Z 10006c60 f i DiamondBuildPrompter.obj
 0001:00005d20       ??0?$_String_alloc@$0A@U?$_String_base_types@DV?$allocator@D@std@@@std@@@std@@QAE@ABV?$allocator@D@1@@Z 10006d20 f i DiamondBuildPrompter.obj
 0001:00005d40       ??0?$_String_val@U?$_Simple_types@D@std@@@std@@QAE@XZ 10006d40 f i DiamondBuildPrompter.obj
 0001:00005d60       ??0?$_Wrap_alloc@V?$allocator@D@std@@@std@@QAE@XZ 10006d60 f i DiamondBuildPrompter.obj
 0001:00005d70       ??0?$allocator@D@std@@QAE@XZ 10006d70 f i DiamondBuildPrompter.obj
 0001:00005d80       ??0?$basic_string@DU?$char_traits@D@std@@V?$allocator@D@2@@std@@QAE@PBD@Z 10006d80 f i DiamondBuildPrompter.obj
 0001:00005de0       ??0DiamondBuildPrompter@LocalWorkflow@U2@@QAE@PAVActor@Workflow@2@@Z 10006de0 f   DiamondBuildPrompter.obj
 0001:00005e10       ??0QLatin1Char@@QAE@D@Z    10006e10 f i DiamondBuildPrompter.obj
 0001:00005e20       ??0_Generic_error_category@std@@QAE@XZ 10006e20 f i DiamondBuildPrompter.obj
 0001:00005e30       ??0_Ignore@std@@QAE@XZ     10006e30 f i DiamondBuildPrompter.obj
 0001:00005e40       ??0_Iostream_error_category@std@@QAE@XZ 10006e40 f i DiamondBuildPrompter.obj
 0001:00005e50       ??0_System_error_category@std@@QAE@XZ 10006e50 f i DiamondBuildPrompter.obj
 0001:00005e60       ??0const_iterator@?$QList@PAVPort@Workflow@U2@@@@QAE@PAUNode@1@@Z 10006e60 f i DiamondBuildPrompter.obj
 0001:00005e70       ??0error_category@std@@QAE@XZ 10006e70 f i DiamondBuildPrompter.obj
 0001:00005e80       ??0error_condition@std@@QAE@HABVerror_category@1@@Z 10006e80 f i DiamondBuildPrompter.obj
 0001:00005ea0       ??1?$PrompterBase@VDiamondBuildPrompter@LocalWorkflow@U2@@@U2@@UAE@XZ 10006ea0 f i DiamondBuildPrompter.obj
 0001:00005eb0       ??1?$QForeachContainer@V?$QList@PAVPort@Workflow@U2@@@@@@QAE@XZ 10006eb0 f i DiamondBuildPrompter.obj
 0001:00005ee0       ??1?$QList@PAVPort@Workflow@U2@@@@QAE@XZ 10006ee0 f i DiamondBuildPrompter.obj
 0001:00005f10       ??1?$basic_string@DU?$char_traits@D@std@@V?$allocator@D@2@@std@@QAE@XZ 10006f10 f i DiamondBuildPrompter.obj
 0001:00005f40       ??1DiamondBuildPrompter@LocalWorkflow@U2@@UAE@XZ 10006f40 f i DiamondBuildPrompter.obj
 0001:00005f50       ??1_Generic_error_category@std@@UAE@XZ 10006f50 f i DiamondBuildPrompter.obj
 0001:00005f60       ??1_Iostream_error_category@std@@UAE@XZ 10006f60 f i DiamondBuildPrompter.obj
 0001:00005f70       ??1_System_error_category@std@@UAE@XZ 10006f70 f i DiamondBuildPrompter.obj
 0001:00005f80       ??1error_category@std@@UAE@XZ 10006f80 f i DiamondBuildPrompter.obj
 0001:00005f90       ??2@YAPAXIPAX@Z            10006f90 f i DiamondBuildPrompter.obj
 0001:00005fa0       ??3@YAXPAX0@Z              10006fa0 f i DiamondBuildPrompter.obj
 0001:00005fb0       ??8error_category@std@@QBE_NABV01@@Z 10006fb0 f i DiamondBuildPrompter.obj
 0001:00005fc0       ??8error_condition@std@@QBE_NABV01@@Z 10006fc0 f i DiamondBuildPrompter.obj
 0001:00005fe0       ??9const_iterator@?$QList@PAVPort@Workflow@U2@@@@QBE_NABV01@@Z 10006fe0 f i DiamondBuildPrompter.obj
 0001:00006000       ??Dconst_iterator@?$QList@PAVPort@Workflow@U2@@@@QBEABQAVPort@Workflow@U2@@XZ 10007000 f i DiamondBuildPrompter.obj
 0001:00006010       ??Econst_iterator@?$QList@PAVPort@Workflow@U2@@@@QAEAAV01@XZ 10007010 f i DiamondBuildPrompter.obj
 0001:00006016       ??_E?$PrompterBase@VDiamondBuildPrompter@LocalWorkflow@U2@@@U2@@WM@AEPAXI@Z 10007016 f i DiamondBuildPrompter.obj
 0001:0000601e       ??_EDiamondBuildPrompter@LocalWorkflow@U2@@WM@AEPAXI@Z 1000701e f i DiamondBuildPrompter.obj
 0001:00006030       ??_E?$PrompterBase@VDiamondBuildPrompter@LocalWorkflow@U2@@@U2@@UAEPAXI@Z 10007030 f i DiamondBuildPrompter.obj
 0001:00006030       ??_G?$PrompterBase@VDiamondBuildPrompter@LocalWorkflow@U2@@@U2@@UAEPAXI@Z 10007030 f i DiamondBuildPrompter.obj
 0001:00006060       ??_GDiamondBuildPrompter@LocalWorkflow@U2@@UAEPAXI@Z 10007060 f i DiamondBuildPrompter.obj
 0001:00006060       ??_EDiamondBuildPrompter@LocalWorkflow@U2@@UAEPAXI@Z 10007060 f i DiamondBuildPrompter.obj
 0001:00006090       ??_E_Generic_error_category@std@@UAEPAXI@Z 10007090 f i DiamondBuildPrompter.obj
 0001:00006090       ??_G_Generic_error_category@std@@UAEPAXI@Z 10007090 f i DiamondBuildPrompter.obj
 0001:000060c0       ??_E_Iostream_error_category@std@@UAEPAXI@Z 100070c0 f i DiamondBuildPrompter.obj
 0001:000060c0       ??_G_Iostream_error_category@std@@UAEPAXI@Z 100070c0 f i DiamondBuildPrompter.obj
 0001:000060f0       ??_G_System_error_category@std@@UAEPAXI@Z 100070f0 f i DiamondBuildPrompter.obj
 0001:000060f0       ??_E_System_error_category@std@@UAEPAXI@Z 100070f0 f i DiamondBuildPrompter.obj
 0001:00006120       ??_Gerror_category@std@@UAEPAXI@Z 10007120 f i DiamondBuildPrompter.obj
 0001:00006120       ??_Eerror_category@std@@UAEPAXI@Z 10007120 f i DiamondBuildPrompter.obj
 0001:00006150       ?_Copy@?$basic_string@DU?$char_traits@D@std@@V?$allocator@D@2@@std@@QAEXII@Z 10007150 f i DiamondBuildPrompter.obj
 0001:000062a0       ?_Eos@?$basic_string@DU?$char_traits@D@std@@V?$allocator@D@2@@std@@QAEXI@Z 100072a0 f i DiamondBuildPrompter.obj
 0001:000062d0       ?_Getal@?$_String_alloc@$0A@U?$_String_base_types@DV?$allocator@D@std@@@std@@@std@@QBE?AU?$_Wrap_alloc@V?$allocator@D@std@@@2@XZ 100072d0 f i DiamondBuildPrompter.obj
 0001:000062e0       ?_Grow@?$basic_string@DU?$char_traits@D@std@@V?$allocator@D@2@@std@@QAE_NI_N@Z 100072e0 f i DiamondBuildPrompter.obj
 0001:00006390       ?_Inside@?$basic_string@DU?$char_traits@D@std@@V?$allocator@D@2@@std@@QAE_NPBD@Z 10007390 f i DiamondBuildPrompter.obj
 0001:000063d0       ?_Myptr@?$_String_val@U?$_Simple_types@D@std@@@std@@QAEPADXZ 100073d0 f i DiamondBuildPrompter.obj
 0001:000063e0       ?_Myptr@?$_String_val@U?$_Simple_types@D@std@@@std@@QBEPBDXZ 100073e0 f i DiamondBuildPrompter.obj
 0001:000063f0       ?_Tidy@?$basic_string@DU?$char_traits@D@std@@V?$allocator@D@2@@std@@QAEX_NI@Z 100073f0 f i DiamondBuildPrompter.obj
 0001:00006440       ?_Xlen@?$basic_string@DU?$char_traits@D@std@@V?$allocator@D@2@@std@@QBEXXZ 10007440 f i DiamondBuildPrompter.obj
 0001:00006450       ?_Xran@?$basic_string@DU?$char_traits@D@std@@V?$allocator@D@2@@std@@QBEXXZ 10007450 f i DiamondBuildPrompter.obj
 0001:00006460       ?allocate@?$_Wrap_alloc@V?$allocator@D@std@@@std@@QAEPADI@Z 10007460 f i DiamondBuildPrompter.obj
 0001:00006490       ?allocate@?$allocator@D@std@@QAEPADI@Z 10007490 f i DiamondBuildPrompter.obj
 0001:000064c0       ?assign@?$basic_string@DU?$char_traits@D@std@@V?$allocator@D@2@@std@@QAEAAV12@ABV12@II@Z 100074c0 f i DiamondBuildPrompter.obj
 0001:000065e0       ?assign@?$basic_string@DU?$char_traits@D@std@@V?$allocator@D@2@@std@@QAEAAV12@PBD@Z 100075e0 f i DiamondBuildPrompter.obj
 0001:00006620       ?assign@?$basic_string@DU?$char_traits@D@std@@V?$allocator@D@2@@std@@QAEAAV12@PBDI@Z 10007620 f i DiamondBuildPrompter.obj
 0001:00006720       ?assign@?$char_traits@D@std@@SAXAADABD@Z 10007720 f i DiamondBuildPrompter.obj
 0001:00006730       ?begin@?$QList@PAVPort@Workflow@U2@@@@QBE?AVconst_iterator@1@XZ 10007730 f i DiamondBuildPrompter.obj
 0001:00006750       ?category@error_code@std@@QBEABVerror_category@2@XZ 10007750 f i DiamondBuildPrompter.obj
 0001:00006760       ?category@error_condition@std@@QBEABVerror_category@2@XZ 10007760 f i DiamondBuildPrompter.obj
 0001:00006770       ?composeRichDoc@DiamondBuildPrompter@LocalWorkflow@U2@@EAE?AVQString@@XZ 10007770 f   DiamondBuildPrompter.obj
 0001:000068a0       ?copy@?$char_traits@D@std@@SAPADPADPBDI@Z 100078a0 f i DiamondBuildPrompter.obj
 0001:000068c0       ?createDescription@?$PrompterBase@VDiamondBuildPrompter@LocalWorkflow@U2@@@U2@@UAEPAVActorDocument@Workflow@2@PAVActor@42@@Z 100078c0 f i DiamondBuildPrompter.obj
 0001:00006b60       ?dealloc@?$QList@PAVPort@Workflow@U2@@@@AAEXPAUData@QListData@@@Z 10007b60 f i DiamondBuildPrompter.obj
 0001:00006b80       ?deallocate@?$_Wrap_alloc@V?$allocator@D@std@@@std@@QAEXPADI@Z 10007b80 f i DiamondBuildPrompter.obj
 0001:00006ba0       ?deallocate@?$allocator@D@std@@QAEXPADI@Z 10007ba0 f i DiamondBuildPrompter.obj
 0001:00006bc0       ?default_error_condition@_System_error_category@std@@UBE?AVerror_condition@2@H@Z 10007bc0 f i DiamondBuildPrompter.obj
 0001:00006c00       ?default_error_condition@error_category@std@@UBE?AVerror_condition@2@H@Z 10007c00 f i DiamondBuildPrompter.obj
 0001:00006c20       ?deref@?$QBasicAtomicInteger@H@@QAE_NXZ 10007c20 f i DiamondBuildPrompter.obj
 0001:00006c30       ?deref@RefCount@QtPrivate@@QAE_NXZ 10007c30 f i DiamondBuildPrompter.obj
 0001:00006c50       ?end@?$QList@PAVPort@Workflow@U2@@@@QBE?AVconst_iterator@1@XZ 10007c50 f i DiamondBuildPrompter.obj
 0001:00006c70       ?equivalent@error_category@std@@UBE_NABVerror_code@2@H@Z 10007c70 f i DiamondBuildPrompter.obj
 0001:00006c90       ?equivalent@error_category@std@@UBE_NHABVerror_condition@2@@Z 10007c90 f i DiamondBuildPrompter.obj
 0001:00006cd0       ?erase@?$basic_string@DU?$char_traits@D@std@@V?$allocator@D@2@@std@@QAEAAV12@I@Z 10007cd0 f i DiamondBuildPrompter.obj
 0001:00006d10       ?erase@?$basic_string@DU?$char_traits@D@std@@V?$allocator@D@2@@std@@QAEAAV12@II@Z 10007d10 f i DiamondBuildPrompter.obj
 0001:00006db0       ?generic_category@std@@YAABVerror_category@1@XZ 10007db0 f i DiamondBuildPrompter.obj
 0001:00006dc0       ?length@?$char_traits@D@std@@SAIPBD@Z 10007dc0 f i DiamondBuildPrompter.obj
 0001:00006de0       ?load@?$QBasicAtomicInteger@H@@QBEHXZ 10007de0 f i DiamondBuildPrompter.obj
 0001:00006df0       ?max_size@?$_Wrap_alloc@V?$allocator@D@std@@@std@@QBEIXZ 10007df0 f i DiamondBuildPrompter.obj
 0001:00006e00       ?max_size@?$allocator@D@std@@QBEIXZ 10007e00 f i DiamondBuildPrompter.obj
 0001:00006e10       ?max_size@?$allocator_traits@V?$allocator@D@std@@@std@@SAIABV?$allocator@D@2@@Z 10007e10 f i DiamondBuildPrompter.obj
 0001:00006e20       ?max_size@?$basic_string@DU?$char_traits@D@std@@V?$allocator@D@2@@std@@QBEIXZ 10007e20 f i DiamondBuildPrompter.obj
 0001:00006e30       ?message@_Generic_error_category@std@@UBE?AV?$basic_string@DU?$char_traits@D@std@@V?$allocator@D@2@@2@H@Z 10007e30 f i DiamondBuildPrompter.obj
 0001:00006eb0       ?message@_Iostream_error_category@std@@UBE?AV?$basic_string@DU?$char_traits@D@std@@V?$allocator@D@2@@2@H@Z 10007eb0 f i DiamondBuildPrompter.obj
 0001:00006f00       ?message@_System_error_category@std@@UBE?AV?$basic_string@DU?$char_traits@D@std@@V?$allocator@D@2@@2@H@Z 10007f00 f i DiamondBuildPrompter.obj
 0001:00006f80       ?move@?$char_traits@D@std@@SAPADPADPBDI@Z 10007f80 f i DiamondBuildPrompter.obj
 0001:00006fa0       ?name@_Generic_error_category@std@@UBEPBDXZ 10007fa0 f i DiamondBuildPrompter.obj
 0001:00006fb0       ?name@_Iostream_error_category@std@@UBEPBDXZ 10007fb0 f i DiamondBuildPrompter.obj
 0001:00006fc0       ?name@_System_error_category@std@@UBEPBDXZ 10007fc0 f i DiamondBuildPrompter.obj
 0001:00006fd0       ?node_copy@?$QList@PAVPort@Workflow@U2@@@@AAEXPAUNode@1@00@Z 10007fd0 f i DiamondBuildPrompter.obj
 0001:00007000       ?node_destruct@?$QList@PAVPort@Workflow@U2@@@@AAEXPAUNode@1@0@Z 10008000 f i DiamondBuildPrompter.obj
 0001:00007010       ?ref@?$QBasicAtomicInteger@H@@QAE_NXZ 10008010 f i DiamondBuildPrompter.obj
 0001:00007030       ?ref@RefCount@QtPrivate@@QAE_NXZ 10008030 f i DiamondBuildPrompter.obj
 0001:00007050       ?size@?$basic_string@DU?$char_traits@D@std@@V?$allocator@D@2@@std@@QBEIXZ 10008050 f i DiamondBuildPrompter.obj
 0001:00007060       ?system_category@std@@YAABVerror_category@1@XZ 10008060 f i DiamondBuildPrompter.obj
 0001:00007070       ?t@Node@?$QList@PAVPort@Workflow@U2@@@@QAEAAPAVPort@Workflow@U2@@XZ 10008070 f i DiamondBuildPrompter.obj
 0001:00007080       ?tr@DiamondBuildPrompter@LocalWorkflow@U2@@SA?AVQString@@PBD0H@Z 10008080 f i DiamondBuildPrompter.obj
 0001:000070b0       ?value@error_code@std@@QBEHXZ 100080b0 f i DiamondBuildPrompter.obj
 0001:000070c0       ?value@error_condition@std@@QBEHXZ 100080c0 f i DiamondBuildPrompter.obj
 0001:000070d0       _hypot                     100080d0 f i DiamondBuildPrompter.obj
 0001:00007100       ??0?$QFlags@W4TaskFlag@U2@@@@QAE@VQFlag@@@Z 10008100 f i DiamondBuildTask.obj
 0001:00007110       ??0?$QFlags@W4TaskFlag@U2@@@@QAE@W4TaskFlag@U2@@@Z 10008110 f i DiamondBuildTask.obj
 0001:00007120       ??0?$QHash@VQString@@UQHashDummyValue@@@@QAE@XZ 10008120 f i DiamondBuildTask.obj
 0001:00007130       ??0?$QList@PAVTask@U2@@@@QAE@$$QAV0@@Z 10008130 f i DiamondBuildTask.obj
 0001:00007150       ??0?$QList@PAVTask@U2@@@@QAE@XZ 10008150 f i DiamondBuildTask.obj
 0001:00007160       ??0?$QList@VQString@@@@QAE@ABV0@@Z 10008160 f i DiamondBuildTask.obj
 0001:00007220       ??0?$QList@VQString@@@@QAE@XZ 10008220 f i DiamondBuildTask.obj
 0001:00007230       ??0?$QSet@VQString@@@@QAE@XZ 10008230 f i DiamondBuildTask.obj
 0001:00007240       ??0DiamondBuildTask@U2@@QAE@ABUDiamondBuildTaskSettings@1@@Z 10008240 f   DiamondBuildTask.obj
 0001:000073e0       ??0DiamondBuildTaskSettings@U2@@QAE@ABU01@@Z 100083e0 f i DiamondBuildTask.obj
 0001:00007470       ??0QFlag@@QAE@H@Z          10008470 f i DiamondBuildTask.obj
 0001:00007480       ??0QStringList@@QAE@ABV0@@Z 10008480 f i DiamondBuildTask.obj
 0001:000074a0       ??0QStringList@@QAE@XZ     100084a0 f i DiamondBuildTask.obj
 0001:000074b0       ??1?$QHash@VQString@@UQHashDummyValue@@@@QAE@XZ 100084b0 f i DiamondBuildTask.obj
 0001:000074e0       ??1?$QHashNode@VQString@@UQHashDummyValue@@@@QAE@XZ 100084e0 f i DiamondBuildTask.obj
 0001:000074f0       ??1?$QList@PAVTask@U2@@@@QAE@XZ 100084f0 f i DiamondBuildTask.obj
 0001:00007520       ??1?$QList@VQString@@@@QAE@XZ 10008520 f i DiamondBuildTask.obj
 0001:00007580       ??1?$QSet@VQString@@@@QAE@XZ 10008580 f i DiamondBuildTask.obj
 0001:000075b0       ??1DiamondBuildTask@U2@@UAE@XZ 100085b0 f i DiamondBuildTask.obj
 0001:00007650       ??1DiamondBuildTaskSettings@U2@@QAE@XZ 10008650 f i DiamondBuildTask.obj
 0001:000076d0       ??1QStringList@@QAE@XZ     100086d0 f i DiamondBuildTask.obj
 0001:000076e0       ??6?$QList@PAVTask@U2@@@@QAEAAV0@ABQAVTask@U2@@@Z 100086e0 f i DiamondBuildTask.obj
 0001:00007700       ??6QStringList@@QAEAAV0@ABVQString@@@Z 10008700 f i DiamondBuildTask.obj
 0001:00007720       ??BQFlag@@QBEHXZ           10008720 f i DiamondBuildTask.obj
 0001:00007730       ??H@YA?BVQString@@ABV0@PBD@Z 10008730 f i DiamondBuildTask.obj
 0001:000077d0       ??U?$QFlags@W4TaskFlag@U2@@@@QBE?AV0@W4TaskFlag@U2@@@Z 100087d0 f i DiamondBuildTask.obj
 0001:000077f0       ??_G?$QHashNode@VQString@@UQHashDummyValue@@@@QAEPAXI@Z 100087f0 f i DiamondBuildTask.obj
 0001:00007820       ??_GDiamondBuildTask@U2@@UAEPAXI@Z 10008820 f i DiamondBuildTask.obj
 0001:00007820       ??_EDiamondBuildTask@U2@@UAEPAXI@Z 10008820 f i DiamondBuildTask.obj
 0001:00007850       ??_GExternalToolLogParser@U2@@UAEPAXI@Z 10008850 f i DiamondBuildTask.obj
 0001:00007850       ??_EExternalToolLogParser@U2@@UAEPAXI@Z 10008850 f i DiamondBuildTask.obj
 0001:00007880       ??_EExternalToolRunTask@U2@@UAEPAXI@Z 10008880 f i DiamondBuildTask.obj
 0001:00007880       ??_GExternalToolRunTask@U2@@UAEPAXI@Z 10008880 f i DiamondBuildTask.obj
 0001:000078b0       ??_GQString@@QAEPAXI@Z     100088b0 f i DiamondBuildTask.obj
 0001:000078e0       ?append@?$QList@PAVTask@U2@@@@QAEXABQAVTask@U2@@@Z 100088e0 f i DiamondBuildTask.obj
 0001:00007970       ?append@?$QList@VQString@@@@QAEXABVQString@@@Z 10008970 f i DiamondBuildTask.obj
 0001:00007a60       ?checkSettings@DiamondBuildTask@U2@@AAEXXZ 10008a60 f   DiamondBuildTask.obj
 0001:00007b90       ?concrete@?$QHash@VQString@@UQHashDummyValue@@@@CAPAU?$QHashNode@VQString@@UQHashDummyValue@@@@PAUNode@QHashData@@@Z 10008b90 f i DiamondBuildTask.obj
 0001:00007ba0       ?dealloc@?$QList@PAVTask@U2@@@@AAEXPAUData@QListData@@@Z 10008ba0 f i DiamondBuildTask.obj
 0001:00007bc0       ?dealloc@?$QList@VQString@@@@AAEXPAUData@QListData@@@Z 10008bc0 f i DiamondBuildTask.obj
 0001:00007c00       ?deleteNode2@?$QHash@VQString@@UQHashDummyValue@@@@CAXPAUNode@QHashData@@@Z 10008c00 f i DiamondBuildTask.obj
 0001:00007c10       ?detach_helper_grow@?$QList@PAVTask@U2@@@@AAEPAUNode@1@HH@Z 10008c10 f i DiamondBuildTask.obj
 0001:00007d20       ?detach_helper_grow@?$QList@VQString@@@@AAEPAUNode@1@HH@Z 10008d20 f i DiamondBuildTask.obj
 0001:00007ea0       ?freeData@?$QHash@VQString@@UQHashDummyValue@@@@AAEXPAUQHashData@@@Z 10008ea0 f i DiamondBuildTask.obj
 0001:00007ec0       ?getArguments@DiamondBuildTask@U2@@ABE?AVQStringList@@ABVQString@@@Z 10008ec0 f   DiamondBuildTask.obj
 0001:00008040       ?getDatabaseUrl@DiamondBuildTask@U2@@QBE?BVQString@@XZ 10009040 f   DiamondBuildTask.obj
 0001:00008070       ?isEmpty@?$QList@VQString@@@@QBE_NXZ 10009070 f i DiamondBuildTask.obj
 0001:00008080       ?isShared@RefCount@QtPrivate@@QBE_NXZ 10009080 f i DiamondBuildTask.obj
 0001:000080a0       ?node_construct@?$QList@PAVTask@U2@@@@AAEXPAUNode@1@ABQAVTask@U2@@@Z 100090a0 f i DiamondBuildTask.obj
 0001:000080c0       ?node_construct@?$QList@VQString@@@@AAEXPAUNode@1@ABVQString@@@Z 100090c0 f i DiamondBuildTask.obj
 0001:00008110       ?node_copy@?$QList@PAVTask@U2@@@@AAEXPAUNode@1@00@Z 10009110 f i DiamondBuildTask.obj
 0001:00008140       ?node_copy@?$QList@VQString@@@@AAEXPAUNode@1@00@Z 10009140 f i DiamondBuildTask.obj
 0001:000081e0       ?node_destruct@?$QList@PAVTask@U2@@@@AAEXPAUNode@1@0@Z 100091e0 f i DiamondBuildTask.obj
 0001:000081f0       ?node_destruct@?$QList@PAVTask@U2@@@@AAEXPAUNode@1@@Z 100091f0 f i DiamondBuildTask.obj
 0001:00008200       ?node_destruct@?$QList@VQString@@@@AAEXPAUNode@1@0@Z 10009200 f i DiamondBuildTask.obj
 0001:00008230       ?node_destruct@?$QList@VQString@@@@AAEXPAUNode@1@@Z 10009230 f i DiamondBuildTask.obj
 0001:00008240       ?onSubTaskFinished@DiamondBuildTask@U2@@EAE?AV?$QList@PAVTask@U2@@@@PAVTask@2@@Z 10009240 f   DiamondBuildTask.obj
 0001:00008480       ?prepare@DiamondBuildTask@U2@@EAEXXZ 10009480 f   DiamondBuildTask.obj
 0001:000085d0       ?tr@DiamondBuildTask@U2@@SA?AVQString@@PBD0H@Z 100095d0 f i DiamondBuildTask.obj
 0001:00008600       ??6?$QList@VWorkflowNotification@U2@@@@QAEAAV0@ABVWorkflowNotification@U2@@@Z 10009600 f i DiamondBuildValidator.obj
 0001:00008620       ??_GWorkflowNotification@U2@@QAEPAXI@Z 10009620 f i DiamondBuildValidator.obj
 0001:00008650       ?append@?$QList@VWorkflowNotification@U2@@@@QAEXABVWorkflowNotification@U2@@@Z 10009650 f i DiamondBuildValidator.obj
 0001:00008730       ?dealloc@?$QList@VWorkflowNotification@U2@@@@AAEXPAUData@QListData@@@Z 10009730 f i DiamondBuildValidator.obj
 0001:00008790       ?detach_helper_grow@?$QList@VWorkflowNotification@U2@@@@AAEPAUNode@1@HH@Z 10009790 f i DiamondBuildValidator.obj
 0001:000088e0       ?node_construct@?$QList@VWorkflowNotification@U2@@@@AAEXPAUNode@1@ABVWorkflowNotification@U2@@@Z 100098e0 f i DiamondBuildValidator.obj
 0001:00008960       ?node_copy@?$QList@VWorkflowNotification@U2@@@@AAEXPAUNode@1@00@Z 10009960 f i DiamondBuildValidator.obj
 0001:00008a30       ?node_destruct@?$QList@VWorkflowNotification@U2@@@@AAEXPAUNode@1@0@Z 10009a30 f i DiamondBuildValidator.obj
 0001:00008a70       ?node_destruct@?$QList@VWorkflowNotification@U2@@@@AAEXPAUNode@1@@Z 10009a70 f i DiamondBuildValidator.obj
 0001:00008aa0       ?tr@DiamondBuildValidator@Workflow@U2@@SA?AVQString@@PBD0H@Z 10009aa0 f i DiamondBuildValidator.obj
 0001:00008ad0       ?validate@DiamondBuildValidator@Workflow@U2@@UBE_NPBVActor@23@AAV?$QList@VWorkflowNotification@U2@@@@ABV?$QMap@VQString@@V1@@@@Z 10009ad0 f   DiamondBuildValidator.obj
 0001:00008af0       ?validateTaxonomy@DiamondBuildValidator@Workflow@U2@@ABE_NPBVActor@23@AAV?$QList@VWorkflowNotification@U2@@@@@Z 10009af0 f   DiamondBuildValidator.obj
 0001:00008df0       ??$acquireMemoryFence@H@?$QGenericAtomicOps@U?$QAtomicOpsBySize@$03@@@@SAXABH@Z 10009df0 f i DiamondBuildWorker.obj
 0001:00008e00       ??$getAttributeValue@V?$QList@VDataset@U2@@@@@Attribute@U2@@QBE?AV?$QList@VDataset@U2@@@@PAVWorkflowContext@Workflow@1@@Z 10009e00 f i DiamondBuildWorker.obj
 0001:00008e20       ??$getAttributeValue@VQString@@@Attribute@U2@@QBE?AVQString@@PAVWorkflowContext@Workflow@1@@Z 10009e20 f i DiamondBuildWorker.obj
 0001:000091b0       ??$getAttributeValueWithoutScript@V?$QList@VDataset@U2@@@@@Attribute@U2@@QBE?AV?$QList@VDataset@U2@@@@XZ 1000a1b0 f i DiamondBuildWorker.obj
 0001:000091d0       ??$getAttributeValueWithoutScript@VQString@@@Attribute@U2@@QBE?AVQString@@XZ 1000a1d0 f i DiamondBuildWorker.obj
 0001:000091f0       ??$getValue@V?$QList@VDataset@U2@@@@@BaseWorker@LocalWorkflow@U2@@IBE?AV?$QList@VDataset@U2@@@@ABVQString@@@Z 1000a1f0 f i DiamondBuildWorker.obj
 0001:00009240       ??$getValue@VQString@@@BaseWorker@LocalWorkflow@U2@@IBE?AVQString@@ABV3@@Z 1000a240 f i DiamondBuildWorker.obj
 0001:00009350       ??$loadAcquire@H@?$QGenericAtomicOps@U?$QAtomicOpsBySize@$03@@@@SAHABH@Z 1000a350 f i DiamondBuildWorker.obj
 0001:00009360       ??$orderedMemoryFence@H@?$QGenericAtomicOps@U?$QAtomicOpsBySize@$03@@@@SAXABH@Z 1000a360 f i DiamondBuildWorker.obj
 0001:00009370       ??$qMapLessThanKey@VDescriptor@U2@@@@YA_NABVDescriptor@U2@@0@Z 1000a370 f i DiamondBuildWorker.obj
 0001:00009390       ??$qMapLessThanKey@VQString@@@@YA_NABVQString@@0@Z 1000a390 f i DiamondBuildWorker.obj
 0001:000093a0       ??$qMetaTypeId@V?$QList@VDataset@U2@@@@@@YAHXZ 1000a3a0 f i DiamondBuildWorker.obj
 0001:000093b0       ??$qMetaTypeId@VQString@@@@YAHXZ 1000a3b0 f i DiamondBuildWorker.obj
 0001:000093c0       ??$qRegisterMetaType@V?$QList@VDataset@U2@@@@@@YAHPBDPAV?$QList@VDataset@U2@@@@W4DefinedType@?$MetaTypeDefinedHelper@V?$QList@VDataset@U2@@@@$00@QtPrivate@@@Z 1000a3c0 f i DiamondBuildWorker.obj
 0001:00009480       ??$qRegisterNormalizedMetaType@V?$QList@VDataset@U2@@@@@@YAHABVQByteArray@@PAV?$QList@VDataset@U2@@@@W4DefinedType@?$MetaTypeDefinedHelper@V?$QList@VDataset@U2@@@@$00@QtPrivate@@@Z 1000a480 f i DiamondBuildWorker.obj
 0001:000094e0       ??$qobject_cast@PAVDiamondBuildTask@U2@@@@YAPAVDiamondBuildTask@U2@@PAVQObject@@@Z 1000a4e0 f i DiamondBuildWorker.obj
 0001:00009500       ??$qvariant_cast@V?$QList@VDataset@U2@@@@@@YA?AV?$QList@VDataset@U2@@@@ABVQVariant@@@Z 1000a500 f i DiamondBuildWorker.obj
 0001:00009520       ??$qvariant_cast@VQString@@@@YA?AVQString@@ABVQVariant@@@Z 1000a520 f i DiamondBuildWorker.obj
 0001:00009540       ??$releaseMemoryFence@H@?$QGenericAtomicOps@U?$QAtomicOpsBySize@$03@@@@SAXABH@Z 1000a540 f i DiamondBuildWorker.obj
 0001:00009550       ??$storeRelease@HH@?$QGenericAtomicOps@U?$QAtomicOpsBySize@$03@@@@SAXAAHH@Z 1000a550 f i DiamondBuildWorker.obj
 0001:00009560       ??$value@V?$QList@VDataset@U2@@@@@QVariant@@QBE?AV?$QList@VDataset@U2@@@@XZ 1000a560 f i DiamondBuildWorker.obj
 0001:00009580       ??$value@VQString@@@QVariant@@QBE?AVQString@@XZ 1000a580 f i DiamondBuildWorker.obj
 0001:000095a0       ??0?$QFlags@W4TypeFlag@QMetaType@@@@QAE@VQFlag@@@Z 1000a5a0 f i DiamondBuildWorker.obj
 0001:000095b0       ??0?$QForeachContainer@V?$QList@PAVURLContainer@U2@@@@@@QAE@ABV?$QList@PAVURLContainer@U2@@@@@Z 1000a5b0 f i DiamondBuildWorker.obj
 0001:000095f0       ??0?$QForeachContainer@V?$QList@VDescriptor@U2@@@@@@QAE@ABV?$QList@VDescriptor@U2@@@@@Z 1000a5f0 f i DiamondBuildWorker.obj
 0001:00009630       ??0?$QList@PAVURLContainer@U2@@@@QAE@ABV0@@Z 1000a630 f i DiamondBuildWorker.obj
 0001:000096f0       ??0?$QList@VDataset@U2@@@@QAE@$$QAV0@@Z 1000a6f0 f i DiamondBuildWorker.obj
 0001:00009710       ??0?$QList@VDataset@U2@@@@QAE@ABV0@@Z 1000a710 f i DiamondBuildWorker.obj
 0001:000097d0       ??0?$QList@VDataset@U2@@@@QAE@XZ 1000a7d0 f i DiamondBuildWorker.obj
 0001:000097e0       ??0?$QList@VDescriptor@U2@@@@QAE@$$QAV0@@Z 1000a7e0 f i DiamondBuildWorker.obj
 0001:00009800       ??0?$QList@VDescriptor@U2@@@@QAE@ABV0@@Z 1000a800 f i DiamondBuildWorker.obj
 0001:000098c0       ??0?$QList@VDescriptor@U2@@@@QAE@XZ 1000a8c0 f i DiamondBuildWorker.obj
 0001:000098d0       ??0?$QMap@VQString@@VQScriptValue@@@@QAE@XZ 1000a8d0 f i DiamondBuildWorker.obj
 0001:000098e0       ??0?$QMap@VQString@@VQVariant@@@@QAE@XZ 1000a8e0 f i DiamondBuildWorker.obj
 0001:000098f0       ??0DiamondBuildTaskSettings@U2@@QAE@XZ 1000a8f0 f i DiamondBuildWorker.obj
 0001:00009970       ??0DiamondBuildWorker@LocalWorkflow@U2@@QAE@PAVActor@Workflow@2@@Z 1000a970 f   DiamondBuildWorker.obj
 0001:000099b0       ??0QStringList@@QAE@ABVQString@@@Z 1000a9b0 f i DiamondBuildWorker.obj
 0001:00009a10       ??0const_iterator@?$QList@PAVURLContainer@U2@@@@QAE@PAUNode@1@@Z 1000aa10 f i DiamondBuildWorker.obj
 0001:00009a20       ??0const_iterator@?$QList@VDescriptor@U2@@@@QAE@PAUNode@1@@Z 1000aa20 f i DiamondBuildWorker.obj
 0001:00009a30       ??0const_iterator@?$QMap@VDescriptor@U2@@VQVariant@@@@QAE@PBU?$QMapNode@VDescriptor@U2@@VQVariant@@@@@Z 1000aa30 f i DiamondBuildWorker.obj
 0001:00009a40       ??0iterator@?$QMap@VQString@@VQScriptValue@@@@QAE@PAU?$QMapNode@VQString@@VQScriptValue@@@@@Z 1000aa40 f i DiamondBuildWorker.obj
 0001:00009a50       ??0iterator@?$QMap@VQString@@VQVariant@@@@QAE@PAU?$QMapNode@VQString@@VQVariant@@@@@Z 1000aa50 f i DiamondBuildWorker.obj
 0001:00009a60       ??1?$QExplicitlySharedDataPointer@VDataType@U2@@@@QAE@XZ 1000aa60 f i DiamondBuildWorker.obj
 0001:00009a80       ??1?$QForeachContainer@V?$QList@PAVURLContainer@U2@@@@@@QAE@XZ 1000aa80 f i DiamondBuildWorker.obj
 0001:00009ab0       ??1?$QForeachContainer@V?$QList@VDescriptor@U2@@@@@@QAE@XZ 1000aab0 f i DiamondBuildWorker.obj
 0001:00009ae0       ??1?$QList@PAVExternalToolListener@U2@@@@QAE@XZ 1000aae0 f i DiamondBuildWorker.obj
 0001:00009b10       ??1?$QList@PAVURLContainer@U2@@@@QAE@XZ 1000ab10 f i DiamondBuildWorker.obj
 0001:00009b40       ??1?$QList@VDataset@U2@@@@QAE@XZ 1000ab40 f i DiamondBuildWorker.obj
 0001:00009b70       ??1?$QList@VDescriptor@U2@@@@QAE@XZ 1000ab70 f i DiamondBuildWorker.obj
 0001:00009ba0       ??1?$QMap@VQString@@VQScriptValue@@@@QAE@XZ 1000aba0 f i DiamondBuildWorker.obj
 0001:00009bf0       ??1?$QMap@VQString@@VQVariant@@@@QAE@XZ 1000abf0 f i DiamondBuildWorker.obj
 0001:00009c40       ??1DiamondBuildWorker@LocalWorkflow@U2@@UAE@XZ 1000ac40 f i DiamondBuildWorker.obj
 0001:00009c50       ??8const_iterator@?$QMap@VDescriptor@U2@@VQVariant@@@@QBE_NABV01@@Z 1000ac50 f i DiamondBuildWorker.obj
 0001:00009c70       ??9const_iterator@?$QList@PAVURLContainer@U2@@@@QBE_NABV01@@Z 1000ac70 f i DiamondBuildWorker.obj
 0001:00009c90       ??9const_iterator@?$QList@VDescriptor@U2@@@@QBE_NABV01@@Z 1000ac90 f i DiamondBuildWorker.obj
 0001:00009cb0       ??9const_iterator@?$QMap@VDescriptor@U2@@VQVariant@@@@QBE_NABV01@@Z 1000acb0 f i DiamondBuildWorker.obj
 0001:00009cd0       ??A?$QMap@VQString@@VQScriptValue@@@@QAEAAVQScriptValue@@ABVQString@@@Z 1000acd0 f i DiamondBuildWorker.obj
 0001:00009da0       ??A?$QMap@VQString@@VQVariant@@@@QAEAAVQVariant@@ABVQString@@@Z 1000ada0 f i DiamondBuildWorker.obj
 0001:00009e70       ??Dconst_iterator@?$QList@PAVURLContainer@U2@@@@QBEABQAVURLContainer@U2@@XZ 1000ae70 f i DiamondBuildWorker.obj
 0001:00009e80       ??Dconst_iterator@?$QList@VDescriptor@U2@@@@QBEABVDescriptor@U2@@XZ 1000ae80 f i DiamondBuildWorker.obj
 0001:00009e90       ??Diterator@?$QMap@VQString@@VQScriptValue@@@@QBEAAVQScriptValue@@XZ 1000ae90 f i DiamondBuildWorker.obj
 0001:00009ea0       ??Diterator@?$QMap@VQString@@VQVariant@@@@QBEAAVQVariant@@XZ 1000aea0 f i DiamondBuildWorker.obj
 0001:00009eb0       ??Econst_iterator@?$QList@PAVURLContainer@U2@@@@QAEAAV01@XZ 1000aeb0 f i DiamondBuildWorker.obj
 0001:00009ec0       ??Econst_iterator@?$QList@VDescriptor@U2@@@@QAEAAV01@XZ 1000aec0 f i DiamondBuildWorker.obj
 0001:00009ed0       ??Econst_iterator@?$QMap@VDescriptor@U2@@VQVariant@@@@QAEAAV01@XZ 1000aed0 f i DiamondBuildWorker.obj
 0001:00009ef0       ??H@YA?BVQString@@ABV0@0@Z 1000aef0 f i DiamondBuildWorker.obj
 0001:00009f60       ??_5?$QFlags@W4TypeFlag@QMetaType@@@@QAEAAV0@W4TypeFlag@QMetaType@@@Z 1000af60 f i DiamondBuildWorker.obj
 0001:00009f6e       ??_EDiamondBuildWorker@LocalWorkflow@U2@@W7AEPAXI@Z 1000af6e f i DiamondBuildWorker.obj
 0001:00009f76       ??_EDiamondBuildWorker@LocalWorkflow@U2@@WBA@AEPAXI@Z 1000af76 f i DiamondBuildWorker.obj
 0001:00009f80       ??_G?$QList@VDataset@U2@@@@QAEPAXI@Z 1000af80 f i DiamondBuildWorker.obj
 0001:00009fc0       ??_GDataset@U2@@QAEPAXI@Z  1000afc0 f i DiamondBuildWorker.obj
 0001:00009ff0       ??_EDescriptor@U2@@UAEPAXI@Z 1000aff0 f i DiamondBuildWorker.obj
 0001:00009ff0       ??_GDescriptor@U2@@UAEPAXI@Z 1000aff0 f i DiamondBuildWorker.obj
 0001:0000a020       ??_GDiamondBuildWorker@LocalWorkflow@U2@@UAEPAXI@Z 1000b020 f i DiamondBuildWorker.obj
 0001:0000a020       ??_EDiamondBuildWorker@LocalWorkflow@U2@@UAEPAXI@Z 1000b020 f i DiamondBuildWorker.obj
 0001:0000a050       ??_EFailTask@U2@@UAEPAXI@Z 1000b050 f i DiamondBuildWorker.obj
 0001:0000a050       ??_GFailTask@U2@@UAEPAXI@Z 1000b050 f i DiamondBuildWorker.obj
 0001:0000a080       ??_GQScriptValue@@QAEPAXI@Z 1000b080 f i DiamondBuildWorker.obj
 0001:0000a0b0       ??_GQVariant@@QAEPAXI@Z    1000b0b0 f i DiamondBuildWorker.obj
 0001:0000a0e0       ??_GTaskSignalMapper@U2@@UAEPAXI@Z 1000b0e0 f i DiamondBuildWorker.obj
 0001:0000a0e0       ??_ETaskSignalMapper@U2@@UAEPAXI@Z 1000b0e0 f i DiamondBuildWorker.obj
 0001:0000a110       ?Construct@?$QMetaTypeFunctionHelper@V?$QList@VDataset@U2@@@@$00@QtMetaTypePrivate@@SAPAXPAXPBX@Z 1000b110 f i DiamondBuildWorker.obj
 0001:0000a1a0       ?Create@?$QMetaTypeFunctionHelper@V?$QList@VDataset@U2@@@@$00@QtMetaTypePrivate@@SAPAXPBX@Z 1000b1a0 f i DiamondBuildWorker.obj
 0001:0000a240       ?Delete@?$QMetaTypeFunctionHelper@V?$QList@VDataset@U2@@@@$00@QtMetaTypePrivate@@SAXPAX@Z 1000b240 f i DiamondBuildWorker.obj
 0001:0000a280       ?Destruct@?$QMetaTypeFunctionHelper@V?$QList@VDataset@U2@@@@$00@QtMetaTypePrivate@@SAXPAX@Z 1000b280 f i DiamondBuildWorker.obj
 0001:0000a2b0       ?append@?$QList@VDescriptor@U2@@@@QAEXABVDescriptor@U2@@@Z 1000b2b0 f i DiamondBuildWorker.obj
 0001:0000a3a0       ?at@?$QList@VDataset@U2@@@@QBEABVDataset@U2@@H@Z 1000b3a0 f i DiamondBuildWorker.obj
 0001:0000a3c0       ?begin@?$QList@PAVURLContainer@U2@@@@QBE?AVconst_iterator@1@XZ 1000b3c0 f i DiamondBuildWorker.obj
 0001:0000a3e0       ?begin@?$QList@VDescriptor@U2@@@@QBE?AVconst_iterator@1@XZ 1000b3e0 f i DiamondBuildWorker.obj
 0001:0000a400       ?begin@?$QMap@VDescriptor@U2@@VQVariant@@@@QBE?AVconst_iterator@1@XZ 1000b400 f i DiamondBuildWorker.obj
 0001:0000a420       ?begin@?$QMapData@VDescriptor@U2@@VQVariant@@@@QAEPAU?$QMapNode@VDescriptor@U2@@VQVariant@@@@XZ 1000b420 f i DiamondBuildWorker.obj
 0001:0000a430       ?cleanup@DiamondBuildWorker@LocalWorkflow@U2@@UAEXXZ 1000b430 f   DiamondBuildWorker.obj
 0001:0000a440       ?copy@?$QMapNode@VQString@@VQScriptValue@@@@QBEPAU1@PAU?$QMapData@VQString@@VQScriptValue@@@@@Z 1000b440 f i DiamondBuildWorker.obj
 0001:0000a4d0       ?copy@?$QMapNode@VQString@@VQVariant@@@@QBEPAU1@PAU?$QMapData@VQString@@VQVariant@@@@@Z 1000b4d0 f i DiamondBuildWorker.obj
 0001:0000a560       ?create@?$QMapData@VQString@@VQScriptValue@@@@SAPAU1@XZ 1000b560 f i DiamondBuildWorker.obj
 0001:0000a570       ?create@?$QMapData@VQString@@VQVariant@@@@SAPAU1@XZ 1000b570 f i DiamondBuildWorker.obj
 0001:0000a580       ?createNode@?$QMapData@VQString@@VQScriptValue@@@@QAEPAU?$QMapNode@VQString@@VQScriptValue@@@@ABVQString@@ABVQScriptValue@@PAU2@_N@Z 1000b580 f i DiamondBuildWorker.obj
 0001:0000a640       ?createNode@?$QMapData@VQString@@VQVariant@@@@QAEPAU?$QMapNode@VQString@@VQVariant@@@@ABVQString@@ABVQVariant@@PAU2@_N@Z 1000b640 f i DiamondBuildWorker.obj
 0001:0000a700       ?dealloc@?$QList@PAVExternalToolListener@U2@@@@AAEXPAUData@QListData@@@Z 1000b700 f i DiamondBuildWorker.obj
 0001:0000a720       ?dealloc@?$QList@PAVURLContainer@U2@@@@AAEXPAUData@QListData@@@Z 1000b720 f i DiamondBuildWorker.obj
 0001:0000a740       ?dealloc@?$QList@VDataset@U2@@@@AAEXPAUData@QListData@@@Z 1000b740 f i DiamondBuildWorker.obj
 0001:0000a7a0       ?dealloc@?$QList@VDescriptor@U2@@@@AAEXPAUData@QListData@@@Z 1000b7a0 f i DiamondBuildWorker.obj
 0001:0000a7f0       ?destroy@?$QMapData@VQString@@VQScriptValue@@@@QAEXXZ 1000b7f0 f i DiamondBuildWorker.obj
 0001:0000a820       ?destroy@?$QMapData@VQString@@VQVariant@@@@QAEXXZ 1000b820 f i DiamondBuildWorker.obj
 0001:0000a850       ?destroySubTree@?$QMapNode@VQString@@VQScriptValue@@@@QAEXXZ 1000b850 f i DiamondBuildWorker.obj
 0001:0000a890       ?destroySubTree@?$QMapNode@VQString@@VQVariant@@@@QAEXXZ 1000b890 f i DiamondBuildWorker.obj
 0001:0000a8d0       ?detach@?$QMap@VQString@@VQScriptValue@@@@QAEXXZ 1000b8d0 f i DiamondBuildWorker.obj
 0001:0000a8f0       ?detach@?$QMap@VQString@@VQVariant@@@@QAEXXZ 1000b8f0 f i DiamondBuildWorker.obj
 0001:0000a910       ?detach_helper@?$QList@VDescriptor@U2@@@@AAEXH@Z 1000b910 f i DiamondBuildWorker.obj
 0001:0000a9e0       ?detach_helper@?$QMap@VQString@@VQScriptValue@@@@AAEXXZ 1000b9e0 f i DiamondBuildWorker.obj
 0001:0000aa60       ?detach_helper@?$QMap@VQString@@VQVariant@@@@AAEXXZ 1000ba60 f i DiamondBuildWorker.obj
 0001:0000aae0       ?detach_helper_grow@?$QList@VDescriptor@U2@@@@AAEPAUNode@1@HH@Z 1000bae0 f i DiamondBuildWorker.obj
 0001:0000ac30       ?end@?$QList@PAVURLContainer@U2@@@@QBE?AVconst_iterator@1@XZ 1000bc30 f i DiamondBuildWorker.obj
 0001:0000ac50       ?end@?$QList@VDescriptor@U2@@@@QBE?AVconst_iterator@1@XZ 1000bc50 f i DiamondBuildWorker.obj
 0001:0000ac70       ?end@?$QMap@VDescriptor@U2@@VQVariant@@@@QBE?AVconst_iterator@1@XZ 1000bc70 f i DiamondBuildWorker.obj
 0001:0000ac90       ?end@?$QMapData@VDescriptor@U2@@VQVariant@@@@QAEPAU?$QMapNode@VDescriptor@U2@@VQVariant@@@@XZ 1000bc90 f i DiamondBuildWorker.obj
 0001:0000aca0       ?end@?$QMapData@VQString@@VQScriptValue@@@@QAEPAU?$QMapNode@VQString@@VQScriptValue@@@@XZ 1000bca0 f i DiamondBuildWorker.obj
 0001:0000acb0       ?end@?$QMapData@VQString@@VQVariant@@@@QAEPAU?$QMapNode@VQString@@VQVariant@@@@XZ 1000bcb0 f i DiamondBuildWorker.obj
 0001:0000acc0       ?findNode@?$QMapData@VDescriptor@U2@@VQVariant@@@@QBEPAU?$QMapNode@VDescriptor@U2@@VQVariant@@@@ABVDescriptor@U2@@@Z 1000bcc0 f i DiamondBuildWorker.obj
 0001:0000ad00       ?findNode@?$QMapData@VQString@@PAVIntegralBus@Workflow@U2@@@@QBEPAU?$QMapNode@VQString@@PAVIntegralBus@Workflow@U2@@@@ABVQString@@@Z 1000bd00 f i DiamondBuildWorker.obj
 0001:0000ad40       ?findNode@?$QMapData@VQString@@VQScriptValue@@@@QBEPAU?$QMapNode@VQString@@VQScriptValue@@@@ABVQString@@@Z 1000bd40 f i DiamondBuildWorker.obj
 0001:0000ad80       ?findNode@?$QMapData@VQString@@VQVariant@@@@QBEPAU?$QMapNode@VQString@@VQVariant@@@@ABVQString@@@Z 1000bd80 f i DiamondBuildWorker.obj
 0001:0000adc0       ?first@?$QList@VDataset@U2@@@@QBEABVDataset@U2@@XZ 1000bdc0 f i DiamondBuildWorker.obj
 0001:0000add0       ?getSettings@DiamondBuildWorker@LocalWorkflow@U2@@AAE?AUDiamondBuildTaskSettings@3@AAVU2OpStatus@3@@Z 1000bdd0 f   DiamondBuildWorker.obj
 0001:0000b560       ?init@DiamondBuildWorker@LocalWorkflow@U2@@UAEXXZ 1000c560 f   DiamondBuildWorker.obj
 0001:0000b720       ?insert@?$QMap@VQString@@VQScriptValue@@@@QAE?AViterator@1@ABVQString@@ABVQScriptValue@@@Z 1000c720 f i DiamondBuildWorker.obj
 0001:0000b7e0       ?insert@?$QMap@VQString@@VQVariant@@@@QAE?AViterator@1@ABVQString@@ABVQVariant@@@Z 1000c7e0 f i DiamondBuildWorker.obj
 0001:0000b8a0       ?invoke@?$MetaTypeInvoker@U?$QVariantValueHelper@V?$QList@VDataset@U2@@@@@QtPrivate@@ABVQVariant@@V?$QList@VDataset@U2@@@@@QtPrivate@@SA?AV?$QList@VDataset@U2@@@@ABVQVariant@@@Z 1000c8a0 f i DiamondBuildWorker.obj
 0001:0000b8c0       ?invoke@?$MetaTypeInvoker@U?$QVariantValueHelper@VQString@@@QtPrivate@@ABVQVariant@@VQString@@@QtPrivate@@SA?AVQString@@ABVQVariant@@@Z 1000c8c0 f i DiamondBuildWorker.obj
 0001:0000b8e0       ?isEmpty@?$QList@VDataset@U2@@@@QBE_NXZ 1000c8e0 f i DiamondBuildWorker.obj
 0001:0000b8f0       ?key@const_iterator@?$QMap@VDescriptor@U2@@VQVariant@@@@QBEABVDescriptor@U2@@XZ 1000c8f0 f i DiamondBuildWorker.obj
 0001:0000b900       ?leftNode@?$QMapNode@VDescriptor@U2@@VQVariant@@@@QBEPAU1@XZ 1000c900 f i DiamondBuildWorker.obj
 0001:0000b910       ?leftNode@?$QMapNode@VQString@@PAVIntegralBus@Workflow@U2@@@@QBEPAU1@XZ 1000c910 f i DiamondBuildWorker.obj
 0001:0000b920       ?leftNode@?$QMapNode@VQString@@VQScriptValue@@@@QBEPAU1@XZ 1000c920 f i DiamondBuildWorker.obj
 0001:0000b930       ?leftNode@?$QMapNode@VQString@@VQVariant@@@@QBEPAU1@XZ 1000c930 f i DiamondBuildWorker.obj
 0001:0000b940       ?loadAcquire@?$QBasicAtomicInteger@H@@QBEHXZ 1000c940 f i DiamondBuildWorker.obj
 0001:0000b950       ?lowerBound@?$QMapNode@VDescriptor@U2@@VQVariant@@@@QAEPAU1@ABVDescriptor@U2@@@Z 1000c950 f i DiamondBuildWorker.obj
 0001:0000b990       ?lowerBound@?$QMapNode@VQString@@PAVIntegralBus@Workflow@U2@@@@QAEPAU1@ABVQString@@@Z 1000c990 f i DiamondBuildWorker.obj
 0001:0000b9d0       ?lowerBound@?$QMapNode@VQString@@VQScriptValue@@@@QAEPAU1@ABVQString@@@Z 1000c9d0 f i DiamondBuildWorker.obj
 0001:0000ba10       ?lowerBound@?$QMapNode@VQString@@VQVariant@@@@QAEPAU1@ABVQString@@@Z 1000ca10 f i DiamondBuildWorker.obj
 0001:0000ba50       ?metaType@?$QVariantValueHelper@V?$QList@VDataset@U2@@@@@QtPrivate@@SA?AV?$QList@VDataset@U2@@@@ABVQVariant@@@Z 1000ca50 f i DiamondBuildWorker.obj
 0001:0000bb40       ?metaType@?$QVariantValueHelper@VQString@@@QtPrivate@@SA?AVQString@@ABVQVariant@@@Z 1000cb40 f i DiamondBuildWorker.obj
 0001:0000bc00       ?nextNode@?$QMapNode@VDescriptor@U2@@VQVariant@@@@QBEPBU1@XZ 1000cc00 f i DiamondBuildWorker.obj
 0001:0000bc10       ?node_construct@?$QList@VDescriptor@U2@@@@AAEXPAUNode@1@ABVDescriptor@U2@@@Z 1000cc10 f i DiamondBuildWorker.obj
 0001:0000bca0       ?node_copy@?$QList@PAVURLContainer@U2@@@@AAEXPAUNode@1@00@Z 1000cca0 f i DiamondBuildWorker.obj
 0001:0000bcd0       ?node_copy@?$QList@VDataset@U2@@@@AAEXPAUNode@1@00@Z 1000ccd0 f i DiamondBuildWorker.obj
 0001:0000bda0       ?node_copy@?$QList@VDescriptor@U2@@@@AAEXPAUNode@1@00@Z 1000cda0 f i DiamondBuildWorker.obj
 0001:0000be70       ?node_destruct@?$QList@PAVExternalToolListener@U2@@@@AAEXPAUNode@1@0@Z 1000ce70 f i DiamondBuildWorker.obj
 0001:0000be80       ?node_destruct@?$QList@PAVURLContainer@U2@@@@AAEXPAUNode@1@0@Z 1000ce80 f i DiamondBuildWorker.obj
 0001:0000be90       ?node_destruct@?$QList@VDataset@U2@@@@AAEXPAUNode@1@0@Z 1000ce90 f i DiamondBuildWorker.obj
 0001:0000bed0       ?node_destruct@?$QList@VDescriptor@U2@@@@AAEXPAUNode@1@0@Z 1000ced0 f i DiamondBuildWorker.obj
 0001:0000bf00       ?node_destruct@?$QList@VDescriptor@U2@@@@AAEXPAUNode@1@@Z 1000cf00 f i DiamondBuildWorker.obj
 0001:0000bf20       ?qt_metatype_id@?$QMetaTypeId2@V?$QList@VDataset@U2@@@@@@SAHXZ 1000cf20 f i DiamondBuildWorker.obj
 0001:0000bf30       ?qt_metatype_id@?$QMetaTypeId2@VQString@@@@SAHXZ 1000cf30 f i DiamondBuildWorker.obj
 0001:0000bf40       ?qt_metatype_id@?$QMetaTypeId@V?$QList@VDataset@U2@@@@@@SAHXZ 1000cf40 f i DiamondBuildWorker.obj
 0001:0000bfe0       ?qt_metatype_id@?$QMetaTypeIdHelper@V?$QList@VDataset@U2@@@@$00@QtPrivate@@SAHXZ 1000cfe0 f i DiamondBuildWorker.obj
 0001:0000bff0       ?qt_noop@@YAXXZ            1000cff0 f i DiamondBuildWorker.obj
 0001:0000c000       ?registerConverter@?$AssociativeContainerConverterHelper@V?$QList@VDataset@U2@@@@$0A@@QtPrivate@@SA_NH@Z 1000d000 f i DiamondBuildWorker.obj
 0001:0000c010       ?registerConverter@?$IsPair@V?$QList@VDataset@U2@@@@@QtPrivate@@SA_NH@Z 1000d010 f i DiamondBuildWorker.obj
 0001:0000c020       ?registerConverter@?$MetaTypeSmartPointerHelper@V?$QList@VDataset@U2@@@@X@QtPrivate@@SA_NH@Z 1000d020 f i DiamondBuildWorker.obj
 0001:0000c030       ?registerConverter@?$ValueTypeIsMetaType@V?$QList@VDataset@U2@@@@$0A@@QtPrivate@@SA_NH@Z 1000d030 f i DiamondBuildWorker.obj
 0001:0000c040       ?reserve@?$QList@VDescriptor@U2@@@@QAEXH@Z 1000d040 f i DiamondBuildWorker.obj
 0001:0000c070       ?rightNode@?$QMapNode@VDescriptor@U2@@VQVariant@@@@QBEPAU1@XZ 1000d070 f i DiamondBuildWorker.obj
 0001:0000c080       ?rightNode@?$QMapNode@VQString@@PAVIntegralBus@Workflow@U2@@@@QBEPAU1@XZ 1000d080 f i DiamondBuildWorker.obj
 0001:0000c090       ?rightNode@?$QMapNode@VQString@@VQScriptValue@@@@QBEPAU1@XZ 1000d090 f i DiamondBuildWorker.obj
 0001:0000c0a0       ?rightNode@?$QMapNode@VQString@@VQVariant@@@@QBEPAU1@XZ 1000d0a0 f i DiamondBuildWorker.obj
 0001:0000c0b0       ?root@?$QMapData@VDescriptor@U2@@VQVariant@@@@QBEPAU?$QMapNode@VDescriptor@U2@@VQVariant@@@@XZ 1000d0b0 f i DiamondBuildWorker.obj
 0001:0000c0c0       ?root@?$QMapData@VQString@@PAVIntegralBus@Workflow@U2@@@@QBEPAU?$QMapNode@VQString@@PAVIntegralBus@Workflow@U2@@@@XZ 1000d0c0 f i DiamondBuildWorker.obj
 0001:0000c0d0       ?root@?$QMapData@VQString@@VQScriptValue@@@@QBEPAU?$QMapNode@VQString@@VQScriptValue@@@@XZ 1000d0d0 f i DiamondBuildWorker.obj
 0001:0000c0e0       ?root@?$QMapData@VQString@@VQVariant@@@@QBEPAU?$QMapNode@VQString@@VQVariant@@@@XZ 1000d0e0 f i DiamondBuildWorker.obj
 0001:0000c0f0       ?size@?$QMap@VDescriptor@U2@@VQVariant@@@@QBEHXZ 1000d0f0 f i DiamondBuildWorker.obj
 0001:0000c100       ?sl_taskFinished@DiamondBuildWorker@LocalWorkflow@U2@@AAEXPAVTask@3@@Z 1000d100 f   DiamondBuildWorker.obj
 0001:0000c310       ?storeRelease@?$QBasicAtomicInteger@H@@QAEXH@Z 1000d310 f i DiamondBuildWorker.obj
 0001:0000c320       ?t@Node@?$QList@PAVURLContainer@U2@@@@QAEAAPAVURLContainer@U2@@XZ 1000d320 f i DiamondBuildWorker.obj
 0001:0000c330       ?t@Node@?$QList@VDataset@U2@@@@QAEAAVDataset@U2@@XZ 1000d330 f i DiamondBuildWorker.obj
 0001:0000c340       ?t@Node@?$QList@VDescriptor@U2@@@@QAEAAVDescriptor@U2@@XZ 1000d340 f i DiamondBuildWorker.obj
 0001:0000c350       ?tick@DiamondBuildWorker@LocalWorkflow@U2@@UAEPAVTask@3@XZ 1000d350 f   DiamondBuildWorker.obj
 0001:0000c550       ?tr@DiamondBuildWorker@LocalWorkflow@U2@@SA?AVQString@@PBD0H@Z 1000d550 f i DiamondBuildWorker.obj
 0001:0000c580       ?uniqueKeys@?$QMap@VDescriptor@U2@@VQVariant@@@@QBE?AV?$QList@VDescriptor@U2@@@@XZ 1000d580 f i DiamondBuildWorker.obj
 0001:0000c680       ?value@?$MetaObjectForType@V?$QList@VDataset@U2@@@@$0A@@QtPrivate@@SAPBUQMetaObject@@XZ 1000d680 f i DiamondBuildWorker.obj
 0001:0000c690       ?value@?$QMap@VDescriptor@U2@@VQVariant@@@@QBE?BVQVariant@@ABVDescriptor@U2@@ABV2@@Z 1000d690 f i DiamondBuildWorker.obj
 0001:0000c6f0       ?value@?$QMap@VQString@@PAVIntegralBus@Workflow@U2@@@@QBEQAVIntegralBus@Workflow@U2@@ABVQString@@ABQAV234@@Z 1000d6f0 f i DiamondBuildWorker.obj
 0001:0000c740       ??$_Move@AAPAVDataType@U2@@@std@@YA$$QAPAVDataType@U2@@AAPAV12@@Z 1000d740 f i DiamondBuildWorkerFactory.obj
 0001:0000c750       ??$qSwap@PAVDataType@U2@@@@YAXAAPAVDataType@U2@@0@Z 1000d750 f i DiamondBuildWorkerFactory.obj
 0001:0000c770       ??$swap@PAVDataType@U2@@@std@@YAXAAPAVDataType@U2@@0@Z 1000d770 f i DiamondBuildWorkerFactory.obj
 0001:0000c790       ??0?$QExplicitlySharedDataPointer@VDataType@U2@@@@QAE@ABV0@@Z 1000d790 f i DiamondBuildWorkerFactory.obj
 0001:0000c7b0       ??0?$QExplicitlySharedDataPointer@VDataType@U2@@@@QAE@PAVDataType@U2@@@Z 1000d7b0 f i DiamondBuildWorkerFactory.obj
 0001:0000c7d0       ??0?$QExplicitlySharedDataPointer@VDataType@U2@@@@QAE@XZ 1000d7d0 f i DiamondBuildWorkerFactory.obj
 0001:0000c7e0       ??0?$QFlags@W4Option@URLDelegate@U2@@@@QAE@VQFlag@@@Z 1000d7e0 f i DiamondBuildWorkerFactory.obj
 0001:0000c7f0       ??0?$QFlags@W4Option@URLDelegate@U2@@@@QAE@W4Option@URLDelegate@U2@@@Z 1000d7f0 f i DiamondBuildWorkerFactory.obj
 0001:0000c800       ??0?$QList@PAVAttribute@U2@@@@QAE@XZ 1000d800 f i DiamondBuildWorkerFactory.obj
 0001:0000c810       ??0?$QList@PAVPortDescriptor@Workflow@U2@@@@QAE@XZ 1000d810 f i DiamondBuildWorkerFactory.obj
 0001:0000c820       ??0?$QMap@VDescriptor@U2@@V?$QExplicitlySharedDataPointer@VDataType@U2@@@@@@QAE@XZ 1000d820 f i DiamondBuildWorkerFactory.obj
 0001:0000c830       ??0?$QMap@VQString@@PAVPropertyDelegate@U2@@@@QAE@XZ 1000d830 f i DiamondBuildWorkerFactory.obj
 0001:0000c840       ??0DiamondBuildValidator@Workflow@U2@@QAE@XZ 1000d840 f i DiamondBuildWorkerFactory.obj
 0001:0000c850       ??0DiamondBuildWorkerFactory@LocalWorkflow@U2@@QAE@XZ 1000d850 f   DiamondBuildWorkerFactory.obj
 0001:0000c870       ??0iterator@?$QMap@VDescriptor@U2@@V?$QExplicitlySharedDataPointer@VDataType@U2@@@@@@QAE@PAU?$QMapNode@VDescriptor@U2@@V?$QExplicitlySharedDataPointer@VDataType@U2@@@@@@@Z 1000d870 f i DiamondBuildWorkerFactory.obj
 0001:0000c880       ??0iterator@?$QMap@VQString@@PAVPropertyDelegate@U2@@@@QAE@PAU?$QMapNode@VQString@@PAVPropertyDelegate@U2@@@@@Z 1000d880 f i DiamondBuildWorkerFactory.obj
 0001:0000c890       ??1?$QList@PAVAttribute@U2@@@@QAE@XZ 1000d890 f i DiamondBuildWorkerFactory.obj
 0001:0000c8c0       ??1?$QList@PAVPortDescriptor@Workflow@U2@@@@QAE@XZ 1000d8c0 f i DiamondBuildWorkerFactory.obj
 0001:0000c8f0       ??1?$QMap@VDescriptor@U2@@V?$QExplicitlySharedDataPointer@VDataType@U2@@@@@@QAE@XZ 1000d8f0 f i DiamondBuildWorkerFactory.obj
 0001:0000c940       ??1?$QMap@VQString@@PAVPropertyDelegate@U2@@@@QAE@XZ 1000d940 f i DiamondBuildWorkerFactory.obj
 0001:0000c9b0       ??1DiamondBuildValidator@Workflow@U2@@UAE@XZ 1000d9b0 f i DiamondBuildWorkerFactory.obj
 0001:0000c9c0       ??1DiamondBuildWorkerFactory@LocalWorkflow@U2@@UAE@XZ 1000d9c0 f i DiamondBuildWorkerFactory.obj
 0001:0000c9d0       ??4?$QExplicitlySharedDataPointer@VDataType@U2@@@@QAEAAV0@$$QAV0@@Z 1000d9d0 f i DiamondBuildWorkerFactory.obj
 0001:0000c9f0       ??4?$QExplicitlySharedDataPointer@VDataType@U2@@@@QAEAAV0@ABV0@@Z 1000d9f0 f i DiamondBuildWorkerFactory.obj
 0001:0000ca40       ??6?$QList@PAVAttribute@U2@@@@QAEAAV0@ABQAVAttribute@U2@@@Z 1000da40 f i DiamondBuildWorkerFactory.obj
 0001:0000ca60       ??6?$QList@PAVPortDescriptor@Workflow@U2@@@@QAEAAV0@ABQAVPortDescriptor@Workflow@U2@@@Z 1000da60 f i DiamondBuildWorkerFactory.obj
 0001:0000ca80       ??A?$QMap@VDescriptor@U2@@V?$QExplicitlySharedDataPointer@VDataType@U2@@@@@@QAEAAV?$QExplicitlySharedDataPointer@VDataType@U2@@@@ABVDescriptor@U2@@@Z 1000da80 f i DiamondBuildWorkerFactory.obj
 0001:0000cb40       ??A?$QMap@VQString@@PAVPropertyDelegate@U2@@@@QAEAAPAVPropertyDelegate@U2@@ABVQString@@@Z 1000db40 f i DiamondBuildWorkerFactory.obj
 0001:0000cbc0       ??Diterator@?$QMap@VDescriptor@U2@@V?$QExplicitlySharedDataPointer@VDataType@U2@@@@@@QBEAAV?$QExplicitlySharedDataPointer@VDataType@U2@@@@XZ 1000dbc0 f i DiamondBuildWorkerFactory.obj
 0001:0000cbd0       ??Diterator@?$QMap@VQString@@PAVPropertyDelegate@U2@@@@QBEAAPAVPropertyDelegate@U2@@XZ 1000dbd0 f i DiamondBuildWorkerFactory.obj
 0001:0000cbe0       ??U?$QFlags@W4Option@URLDelegate@U2@@@@QBE?AV0@W4Option@URLDelegate@U2@@@Z 1000dbe0 f i DiamondBuildWorkerFactory.obj
 0001:0000cc00       ??U@YA?AV?$QFlags@W4Option@URLDelegate@U2@@@@W4Option@URLDelegate@U2@@0@Z 1000dc00 f i DiamondBuildWorkerFactory.obj
 0001:0000cc10       ??_EDiamondBuildWorkerFactory@LocalWorkflow@U2@@W7AEPAXI@Z 1000dc10 f i DiamondBuildWorkerFactory.obj
 0001:0000cc20       ??_G?$QExplicitlySharedDataPointer@VDataType@U2@@@@QAEPAXI@Z 1000dc20 f i DiamondBuildWorkerFactory.obj
 0001:0000cc60       ??_EAttribute@U2@@UAEPAXI@Z 1000dc60 f i DiamondBuildWorkerFactory.obj
 0001:0000cc60       ??_GAttribute@U2@@UAEPAXI@Z 1000dc60 f i DiamondBuildWorkerFactory.obj
 0001:0000cc90       ??_EDelegateEditor@U2@@UAEPAXI@Z 1000dc90 f i DiamondBuildWorkerFactory.obj
 0001:0000cc90       ??_GDelegateEditor@U2@@UAEPAXI@Z 1000dc90 f i DiamondBuildWorkerFactory.obj
 0001:0000ccc0       ??_GDiamondBuildValidator@Workflow@U2@@UAEPAXI@Z 1000dcc0 f i DiamondBuildWorkerFactory.obj
 0001:0000ccc0       ??_EDiamondBuildValidator@Workflow@U2@@UAEPAXI@Z 1000dcc0 f i DiamondBuildWorkerFactory.obj
 0001:0000ccf0       ??_EDiamondBuildWorkerFactory@LocalWorkflow@U2@@UAEPAXI@Z 1000dcf0 f i DiamondBuildWorkerFactory.obj
 0001:0000ccf0       ??_GDiamondBuildWorkerFactory@LocalWorkflow@U2@@UAEPAXI@Z 1000dcf0 f i DiamondBuildWorkerFactory.obj
 0001:0000cd20       ??_GGenomicLibraryDelegate@LocalWorkflow@U2@@UAEPAXI@Z 1000dd20 f i DiamondBuildWorkerFactory.obj
 0001:0000cd20       ??_EGenomicLibraryDelegate@LocalWorkflow@U2@@UAEPAXI@Z 1000dd20 f i DiamondBuildWorkerFactory.obj
 0001:0000cd50       ??_EIntegralBusActorPrototype@Workflow@U2@@UAEPAXI@Z 1000dd50 f i DiamondBuildWorkerFactory.obj
 0001:0000cd50       ??_GIntegralBusActorPrototype@Workflow@U2@@UAEPAXI@Z 1000dd50 f i DiamondBuildWorkerFactory.obj
 0001:0000cd80       ??_GMapDataType@U2@@UAEPAXI@Z 1000dd80 f i DiamondBuildWorkerFactory.obj
 0001:0000cd80       ??_EMapDataType@U2@@UAEPAXI@Z 1000dd80 f i DiamondBuildWorkerFactory.obj
 0001:0000cdb0       ??_EPortDescriptor@Workflow@U2@@UAEPAXI@Z 1000ddb0 f i DiamondBuildWorkerFactory.obj
 0001:0000cdb0       ??_GPortDescriptor@Workflow@U2@@UAEPAXI@Z 1000ddb0 f i DiamondBuildWorkerFactory.obj
 0001:0000cde0       ??_EURLDelegate@U2@@UAEPAXI@Z 1000dde0 f i DiamondBuildWorkerFactory.obj
 0001:0000cde0       ??_GURLDelegate@U2@@UAEPAXI@Z 1000dde0 f i DiamondBuildWorkerFactory.obj
 0001:0000ce10       ?append@?$QList@PAVAttribute@U2@@@@QAEXABQAVAttribute@U2@@@Z 1000de10 f i DiamondBuildWorkerFactory.obj
 0001:0000cea0       ?append@?$QList@PAVPortDescriptor@Workflow@U2@@@@QAEXABQAVPortDescriptor@Workflow@U2@@@Z 1000dea0 f i DiamondBuildWorkerFactory.obj
 0001:0000cf30       ?cleanup@DiamondBuildWorkerFactory@LocalWorkflow@U2@@SAXXZ 1000df30 f   DiamondBuildWorkerFactory.obj
 0001:0000cf80       ?copy@?$QMapNode@VDescriptor@U2@@V?$QExplicitlySharedDataPointer@VDataType@U2@@@@@@QBEPAU1@PAU?$QMapData@VDescriptor@U2@@V?$QExplicitlySharedDataPointer@VDataType@U2@@@@@@@Z 1000df80 f i DiamondBuildWorkerFactory.obj
 0001:0000d010       ?copy@?$QMapNode@VQString@@PAVPropertyDelegate@U2@@@@QBEPAU1@PAU?$QMapData@VQString@@PAVPropertyDelegate@U2@@@@@Z 1000e010 f i DiamondBuildWorkerFactory.obj
 0001:0000d0a0       ?create@?$QMapData@VDescriptor@U2@@V?$QExplicitlySharedDataPointer@VDataType@U2@@@@@@SAPAU1@XZ 1000e0a0 f i DiamondBuildWorkerFactory.obj
 0001:0000d0b0       ?create@?$QMapData@VQString@@PAVPropertyDelegate@U2@@@@SAPAU1@XZ 1000e0b0 f i DiamondBuildWorkerFactory.obj
 0001:0000d0c0       ?createNode@?$QMapData@VDescriptor@U2@@V?$QExplicitlySharedDataPointer@VDataType@U2@@@@@@QAEPAU?$QMapNode@VDescriptor@U2@@V?$QExplicitlySharedDataPointer@VDataType@U2@@@@@@ABVDescriptor@U2@@ABV?$QExplicitlySharedDataPointer@VDataType@U2@@@@PAU2@_N@Z 1000e0c0 f i DiamondBuildWorkerFactory.obj
 0001:0000d180       ?createNode@?$QMapData@VQString@@PAVPropertyDelegate@U2@@@@QAEPAU?$QMapNode@VQString@@PAVPropertyDelegate@U2@@@@ABVQString@@ABQAVPropertyDelegate@U2@@PAU2@_N@Z 1000e180 f i DiamondBuildWorkerFactory.obj
 0001:0000d220       ?createWorker@DiamondBuildWorkerFactory@LocalWorkflow@U2@@UAEPAVWorker@Workflow@3@PAVActor@53@@Z 1000e220 f   DiamondBuildWorkerFactory.obj
 0001:0000d290       ?dealloc@?$QList@PAVAttribute@U2@@@@AAEXPAUData@QListData@@@Z 1000e290 f i DiamondBuildWorkerFactory.obj
 0001:0000d2b0       ?dealloc@?$QList@PAVPortDescriptor@Workflow@U2@@@@AAEXPAUData@QListData@@@Z 1000e2b0 f i DiamondBuildWorkerFactory.obj
 0001:0000d2d0       ?destroy@?$QMapData@VDescriptor@U2@@V?$QExplicitlySharedDataPointer@VDataType@U2@@@@@@QAEXXZ 1000e2d0 f i DiamondBuildWorkerFactory.obj
 0001:0000d300       ?destroy@?$QMapData@VQString@@PAVPropertyDelegate@U2@@@@QAEXXZ 1000e300 f i DiamondBuildWorkerFactory.obj
 0001:0000d350       ?destroySubTree@?$QMapNode@VDescriptor@U2@@V?$QExplicitlySharedDataPointer@VDataType@U2@@@@@@QAEXXZ 1000e350 f i DiamondBuildWorkerFactory.obj
 0001:0000d3a0       ?destroySubTree@?$QMapNode@VQString@@PAVPropertyDelegate@U2@@@@QAEXXZ 1000e3a0 f i DiamondBuildWorkerFactory.obj
 0001:0000d3d0       ?detach@?$QMap@VDescriptor@U2@@V?$QExplicitlySharedDataPointer@VDataType@U2@@@@@@QAEXXZ 1000e3d0 f i DiamondBuildWorkerFactory.obj
 0001:0000d3f0       ?detach@?$QMap@VQString@@PAVPropertyDelegate@U2@@@@QAEXXZ 1000e3f0 f i DiamondBuildWorkerFactory.obj
 0001:0000d410       ?detach_helper@?$QMap@VDescriptor@U2@@V?$QExplicitlySharedDataPointer@VDataType@U2@@@@@@AAEXXZ 1000e410 f i DiamondBuildWorkerFactory.obj
 0001:0000d490       ?detach_helper@?$QMap@VQString@@PAVPropertyDelegate@U2@@@@AAEXXZ 1000e490 f i DiamondBuildWorkerFactory.obj
 0001:0000d540       ?detach_helper_grow@?$QList@PAVAttribute@U2@@@@AAEPAUNode@1@HH@Z 1000e540 f i DiamondBuildWorkerFactory.obj
 0001:0000d650       ?detach_helper_grow@?$QList@PAVPortDescriptor@Workflow@U2@@@@AAEPAUNode@1@HH@Z 1000e650 f i DiamondBuildWorkerFactory.obj
 0001:0000d760       ?end@?$QMapData@VDescriptor@U2@@V?$QExplicitlySharedDataPointer@VDataType@U2@@@@@@QAEPAU?$QMapNode@VDescriptor@U2@@V?$QExplicitlySharedDataPointer@VDataType@U2@@@@@@XZ 1000e760 f i DiamondBuildWorkerFactory.obj
 0001:0000d770       ?end@?$QMapData@VQString@@PAVPropertyDelegate@U2@@@@QAEPAU?$QMapNode@VQString@@PAVPropertyDelegate@U2@@@@XZ 1000e770 f i DiamondBuildWorkerFactory.obj
 0001:0000d780       ?findNode@?$QMapData@VDescriptor@U2@@V?$QExplicitlySharedDataPointer@VDataType@U2@@@@@@QBEPAU?$QMapNode@VDescriptor@U2@@V?$QExplicitlySharedDataPointer@VDataType@U2@@@@@@ABVDescriptor@U2@@@Z 1000e780 f i DiamondBuildWorkerFactory.obj
 0001:0000d7c0       ?findNode@?$QMapData@VQString@@PAVPropertyDelegate@U2@@@@QBEPAU?$QMapNode@VQString@@PAVPropertyDelegate@U2@@@@ABVQString@@@Z 1000e7c0 f i DiamondBuildWorkerFactory.obj
 0001:0000d800       ?init@DiamondBuildWorkerFactory@LocalWorkflow@U2@@SAXXZ 1000e800 f   DiamondBuildWorkerFactory.obj
 0001:0000e0e0       ?insert@?$QMap@VDescriptor@U2@@V?$QExplicitlySharedDataPointer@VDataType@U2@@@@@@QAE?AViterator@1@ABVDescriptor@U2@@ABV?$QExplicitlySharedDataPointer@VDataType@U2@@@@@Z 1000f0e0 f i DiamondBuildWorkerFactory.obj
 0001:0000e1e0       ?insert@?$QMap@VQString@@PAVPropertyDelegate@U2@@@@QAE?AViterator@1@ABVQString@@ABQAVPropertyDelegate@U2@@@Z 1000f1e0 f i DiamondBuildWorkerFactory.obj
 0001:0000e2a0       ?leftNode@?$QMapNode@VDescriptor@U2@@V?$QExplicitlySharedDataPointer@VDataType@U2@@@@@@QBEPAU1@XZ 1000f2a0 f i DiamondBuildWorkerFactory.obj
 0001:0000e2b0       ?leftNode@?$QMapNode@VQString@@PAVPropertyDelegate@U2@@@@QBEPAU1@XZ 1000f2b0 f i DiamondBuildWorkerFactory.obj
 0001:0000e2c0       ?lowerBound@?$QMapNode@VDescriptor@U2@@V?$QExplicitlySharedDataPointer@VDataType@U2@@@@@@QAEPAU1@ABVDescriptor@U2@@@Z 1000f2c0 f i DiamondBuildWorkerFactory.obj
 0001:0000e300       ?lowerBound@?$QMapNode@VQString@@PAVPropertyDelegate@U2@@@@QAEPAU1@ABVQString@@@Z 1000f300 f i DiamondBuildWorkerFactory.obj
 0001:0000e340       ?node_construct@?$QList@PAVAttribute@U2@@@@AAEXPAUNode@1@ABQAVAttribute@U2@@@Z 1000f340 f i DiamondBuildWorkerFactory.obj
 0001:0000e360       ?node_construct@?$QList@PAVPortDescriptor@Workflow@U2@@@@AAEXPAUNode@1@ABQAVPortDescriptor@Workflow@U2@@@Z 1000f360 f i DiamondBuildWorkerFactory.obj
 0001:0000e380       ?node_copy@?$QList@PAVAttribute@U2@@@@AAEXPAUNode@1@00@Z 1000f380 f i DiamondBuildWorkerFactory.obj
 0001:0000e3b0       ?node_copy@?$QList@PAVPortDescriptor@Workflow@U2@@@@AAEXPAUNode@1@00@Z 1000f3b0 f i DiamondBuildWorkerFactory.obj
 0001:0000e3e0       ?node_destruct@?$QList@PAVAttribute@U2@@@@AAEXPAUNode@1@0@Z 1000f3e0 f i DiamondBuildWorkerFactory.obj
 0001:0000e3f0       ?node_destruct@?$QList@PAVAttribute@U2@@@@AAEXPAUNode@1@@Z 1000f3f0 f i DiamondBuildWorkerFactory.obj
 0001:0000e400       ?node_destruct@?$QList@PAVPortDescriptor@Workflow@U2@@@@AAEXPAUNode@1@0@Z 1000f400 f i DiamondBuildWorkerFactory.obj
 0001:0000e410       ?node_destruct@?$QList@PAVPortDescriptor@Workflow@U2@@@@AAEXPAUNode@1@@Z 1000f410 f i DiamondBuildWorkerFactory.obj
 0001:0000e420       ?rightNode@?$QMapNode@VDescriptor@U2@@V?$QExplicitlySharedDataPointer@VDataType@U2@@@@@@QBEPAU1@XZ 1000f420 f i DiamondBuildWorkerFactory.obj
 0001:0000e430       ?rightNode@?$QMapNode@VQString@@PAVPropertyDelegate@U2@@@@QBEPAU1@XZ 1000f430 f i DiamondBuildWorkerFactory.obj
 0001:0000e440       ?root@?$QMapData@VDescriptor@U2@@V?$QExplicitlySharedDataPointer@VDataType@U2@@@@@@QBEPAU?$QMapNode@VDescriptor@U2@@V?$QExplicitlySharedDataPointer@VDataType@U2@@@@@@XZ 1000f440 f i DiamondBuildWorkerFactory.obj
 0001:0000e450       ?root@?$QMapData@VQString@@PAVPropertyDelegate@U2@@@@QBEPAU?$QMapNode@VQString@@PAVPropertyDelegate@U2@@@@XZ 1000f450 f i DiamondBuildWorkerFactory.obj
 0001:0000e460       ??0?$PrompterBase@VDiamondClassifyPrompter@LocalWorkflow@U2@@@U2@@QAE@PAVActor@Workflow@1@_N@Z 1000f460 f i DiamondClassifyPrompter.obj
 0001:0000e490       ??0DiamondClassifyPrompter@LocalWorkflow@U2@@QAE@PAVActor@Workflow@2@@Z 1000f490 f   DiamondClassifyPrompter.obj
 0001:0000e4c0       ??1?$PrompterBase@VDiamondClassifyPrompter@LocalWorkflow@U2@@@U2@@UAE@XZ 1000f4c0 f i DiamondClassifyPrompter.obj
 0001:0000e4d0       ??1DiamondClassifyPrompter@LocalWorkflow@U2@@UAE@XZ 1000f4d0 f i DiamondClassifyPrompter.obj
 0001:0000e4d6       ??_E?$PrompterBase@VDiamondClassifyPrompter@LocalWorkflow@U2@@@U2@@WM@AEPAXI@Z 1000f4d6 f i DiamondClassifyPrompter.obj
 0001:0000e4de       ??_EDiamondClassifyPrompter@LocalWorkflow@U2@@WM@AEPAXI@Z 1000f4de f i DiamondClassifyPrompter.obj
 0001:0000e4f0       ??_G?$PrompterBase@VDiamondClassifyPrompter@LocalWorkflow@U2@@@U2@@UAEPAXI@Z 1000f4f0 f i DiamondClassifyPrompter.obj
 0001:0000e4f0       ??_E?$PrompterBase@VDiamondClassifyPrompter@LocalWorkflow@U2@@@U2@@UAEPAXI@Z 1000f4f0 f i DiamondClassifyPrompter.obj
 0001:0000e520       ??_EDiamondClassifyPrompter@LocalWorkflow@U2@@UAEPAXI@Z 1000f520 f i DiamondClassifyPrompter.obj
 0001:0000e520       ??_GDiamondClassifyPrompter@LocalWorkflow@U2@@UAEPAXI@Z 1000f520 f i DiamondClassifyPrompter.obj
 0001:0000e550       ?composeRichDoc@DiamondClassifyPrompter@LocalWorkflow@U2@@EAE?AVQString@@XZ 1000f550 f   DiamondClassifyPrompter.obj
 0001:0000e6e0       ?createDescription@?$PrompterBase@VDiamondClassifyPrompter@LocalWorkflow@U2@@@U2@@UAEPAVActorDocument@Workflow@2@PAVActor@42@@Z 1000f6e0 f i DiamondClassifyPrompter.obj
 0001:0000e980       ?tr@DiamondClassifyPrompter@LocalWorkflow@U2@@SA?AVQString@@PBD0H@Z 1000f980 f i DiamondClassifyPrompter.obj
 0001:0000e9b0       ??0?$QFlags@W4OpenModeFlag@QIODevice@@@@QAE@W4OpenModeFlag@QIODevice@@@Z 1000f9b0 f i DiamondClassifyTask.obj
 0001:0000e9c0       ??0?$QMap@VQString@@I@@QAE@XZ 1000f9c0 f i DiamondClassifyTask.obj
 0001:0000e9d0       ??0DiamondClassifyTask@U2@@QAE@ABUDiamondClassifyTaskSettings@1@@Z 1000f9d0 f   DiamondClassifyTask.obj
 0001:0000eb30       ??0DiamondClassifyTaskSettings@U2@@QAE@ABU01@@Z 1000fb30 f i DiamondClassifyTask.obj
 0001:0000ec40       ??0DiamondClassifyTaskSettings@U2@@QAE@XZ 1000fc40 f   DiamondClassifyTask.obj
 0001:0000ed30       ??0iterator@?$QMap@VQString@@I@@QAE@PAU?$QMapNode@VQString@@I@@@Z 1000fd30 f i DiamondClassifyTask.obj
 0001:0000ed40       ??1?$QList@VQByteArray@@@@QAE@XZ 1000fd40 f i DiamondClassifyTask.obj
 0001:0000eda0       ??1?$QMap@VQString@@I@@QAE@XZ 1000fda0 f i DiamondClassifyTask.obj
 0001:0000ee10       ??1DiamondClassifyTask@U2@@UAE@XZ 1000fe10 f i DiamondClassifyTask.obj
 0001:0000ee80       ??1DiamondClassifyTaskSettings@U2@@QAE@XZ 1000fe80 f i DiamondClassifyTask.obj
 0001:0000ef30       ??A?$QList@VQByteArray@@@@QAEAAVQByteArray@@H@Z 1000ff30 f i DiamondClassifyTask.obj
 0001:0000ef60       ??_EDiamondClassifyTask@U2@@UAEPAXI@Z 1000ff60 f i DiamondClassifyTask.obj
 0001:0000ef60       ??_GDiamondClassifyTask@U2@@UAEPAXI@Z 1000ff60 f i DiamondClassifyTask.obj
 0001:0000efe0       ??_GQByteArray@@QAEPAXI@Z  1000ffe0 f i DiamondClassifyTask.obj
 0001:0000f010       ?checkSettings@DiamondClassifyTask@U2@@AAEXXZ 10010010 f   DiamondClassifyTask.obj
 0001:0000f1e0       ?contains@?$QMap@VQString@@I@@QBE_NABVQString@@@Z 100101e0 f i DiamondClassifyTask.obj
 0001:0000f220       ?copy@?$QMapNode@VQString@@I@@QBEPAU1@PAU?$QMapData@VQString@@I@@@Z 10010220 f i DiamondClassifyTask.obj
 0001:0000f2b0       ?create@?$QMapData@VQString@@I@@SAPAU1@XZ 100102b0 f i DiamondClassifyTask.obj
 0001:0000f2c0       ?createNode@?$QMapData@VQString@@I@@QAEPAU?$QMapNode@VQString@@I@@ABVQString@@ABIPAU2@_N@Z 100102c0 f i DiamondClassifyTask.obj
 0001:0000f360       ?dealloc@?$QList@VQByteArray@@@@AAEXPAUData@QListData@@@Z 10010360 f i DiamondClassifyTask.obj
 0001:0000f3a0       ?destroy@?$QMapData@VQString@@I@@QAEXXZ 100103a0 f i DiamondClassifyTask.obj
 0001:0000f3f0       ?destroySubTree@?$QMapNode@VQString@@I@@QAEXXZ 100103f0 f i DiamondClassifyTask.obj
 0001:0000f420       ?detach@?$QList@VQByteArray@@@@QAEXXZ 10010420 f i DiamondClassifyTask.obj
 0001:0000f440       ?detach@?$QMap@VQString@@I@@QAEXXZ 10010440 f i DiamondClassifyTask.obj
 0001:0000f460       ?detach_helper@?$QList@VQByteArray@@@@AAEXH@Z 10010460 f i DiamondClassifyTask.obj
 0001:0000f550       ?detach_helper@?$QList@VQByteArray@@@@AAEXXZ 10010550 f i DiamondClassifyTask.obj
 0001:0000f560       ?detach_helper@?$QMap@VQString@@I@@AAEXXZ 10010560 f i DiamondClassifyTask.obj
 0001:0000f610       ?end@?$QMapData@VQString@@I@@QAEPAU?$QMapNode@VQString@@I@@XZ 10010610 f i DiamondClassifyTask.obj
 0001:0000f620       ?findNode@?$QMapData@VQString@@I@@QBEPAU?$QMapNode@VQString@@I@@ABVQString@@@Z 10010620 f i DiamondClassifyTask.obj
 0001:0000f660       ?getArguments@DiamondClassifyTask@U2@@ABE?AVQStringList@@XZ 10010660 f   DiamondClassifyTask.obj
 0001:0000fcd0       ?getClassificationUrl@DiamondClassifyTask@U2@@QBEABVQString@@XZ 10010cd0 f   DiamondClassifyTask.obj
 0001:0000fce0       ?getParsedReport@DiamondClassifyTask@U2@@QBEABV?$QMap@VQString@@I@@XZ 10010ce0 f   DiamondClassifyTask.obj
 0001:0000fcf0       ?insert@?$QMap@VQString@@I@@QAE?AViterator@1@ABVQString@@ABI@Z 10010cf0 f i DiamondClassifyTask.obj
 0001:0000fdb0       ?leftNode@?$QMapNode@VQString@@I@@QBEPAU1@XZ 10010db0 f i DiamondClassifyTask.obj
 0001:0000fdc0       ?lowerBound@?$QMapNode@VQString@@I@@QAEPAU1@ABVQString@@@Z 10010dc0 f i DiamondClassifyTask.obj
 0001:0000fe00       ?node_copy@?$QList@VQByteArray@@@@AAEXPAUNode@1@00@Z 10010e00 f i DiamondClassifyTask.obj
 0001:0000fea0       ?node_destruct@?$QList@VQByteArray@@@@AAEXPAUNode@1@0@Z 10010ea0 f i DiamondClassifyTask.obj
 0001:0000fed0       ?prepare@DiamondClassifyTask@U2@@EAEXXZ 10010ed0 f   DiamondClassifyTask.obj
 0001:00010060       ?rightNode@?$QMapNode@VQString@@I@@QBEPAU1@XZ 10011060 f i DiamondClassifyTask.obj
 0001:00010070       ?root@?$QMapData@VQString@@I@@QBEPAU?$QMapNode@VQString@@I@@XZ 10011070 f i DiamondClassifyTask.obj
 0001:00010080       ?run@DiamondClassifyTask@U2@@EAEXXZ 10011080 f   DiamondClassifyTask.obj
 0001:000104b0       ?size@?$QList@VQByteArray@@@@QBEHXZ 100114b0 f i DiamondClassifyTask.obj
 0001:000104c0       ?t@Node@?$QList@VQByteArray@@@@QAEAAVQByteArray@@XZ 100114c0 f i DiamondClassifyTask.obj
 0001:000104d0       ?tr@DiamondClassifyTask@U2@@SA?AVQString@@PBD0H@Z 100114d0 f i DiamondClassifyTask.obj
 0001:00010500       ??$?0V?$QMap@VQString@@I@@@QAssociativeIterableImpl@QtMetaTypePrivate@@QAE@PBV?$QMap@VQString@@I@@@Z 10011500 f i DiamondClassifyWorker.obj
 0001:00010570       ??$_Advance@Vconst_iterator@?$QMap@VQString@@I@@H@std@@YAXAAVconst_iterator@?$QMap@VQString@@I@@HUbidirectional_iterator_tag@0@@Z 10011570 f i DiamondClassifyWorker.obj
 0001:000105b0       ??$_Distance2@Vconst_iterator@?$QMap@VQString@@I@@H@std@@YAXVconst_iterator@?$QMap@VQString@@I@@0AAHUbidirectional_iterator_tag@0@@Z 100115b0 f i DiamondClassifyWorker.obj
 0001:000105e0       ??$_Iter_cat@Vconst_iterator@?$QMap@VQString@@I@@@std@@YA?AUbidirectional_iterator_tag@0@ABVconst_iterator@?$QMap@VQString@@I@@@Z 100115e0 f i DiamondClassifyWorker.obj
 0001:000105f0       ??$advance@Vconst_iterator@?$QMap@VQString@@I@@H@std@@YAXAAVconst_iterator@?$QMap@VQString@@I@@H@Z 100115f0 f i DiamondClassifyWorker.obj
 0001:00010630       ??$advanceImpl@V?$QMap@VQString@@I@@@QAssociativeIterableImpl@QtMetaTypePrivate@@SAXPAPAXH@Z 10011630 f i DiamondClassifyWorker.obj
 0001:00010670       ??$beginImpl@V?$QMap@VQString@@I@@@QAssociativeIterableImpl@QtMetaTypePrivate@@SAXPBXPAPAX@Z 10011670 f i DiamondClassifyWorker.obj
 0001:000106b0       ??$distance@Vconst_iterator@?$QMap@VQString@@I@@@std@@YAHVconst_iterator@?$QMap@VQString@@I@@0@Z 100116b0 f i DiamondClassifyWorker.obj
 0001:000106e0       ??$endImpl@V?$QMap@VQString@@I@@@QAssociativeIterableImpl@QtMetaTypePrivate@@SAXPBXPAPAX@Z 100116e0 f i DiamondClassifyWorker.obj
 0001:00010710       ??$findImpl@V?$QMap@VQString@@I@@@QAssociativeIterableImpl@QtMetaTypePrivate@@SAXPBX0PAPAX@Z 10011710 f i DiamondClassifyWorker.obj
 0001:00010770       ??$fromValue@V?$QMap@VQString@@I@@@QVariant@@SA?AV0@ABV?$QMap@VQString@@I@@@Z 10011770 f i DiamondClassifyWorker.obj
 0001:00010790       ??$getAttributeValue@H@Attribute@U2@@QBEHPAVWorkflowContext@Workflow@1@@Z 10011790 f i DiamondClassifyWorker.obj
 0001:00010b60       ??$getAttributeValue@I@Attribute@U2@@QBEIPAVWorkflowContext@Workflow@1@@Z 10011b60 f i DiamondClassifyWorker.obj
 0001:00010bb0       ??$getAttributeValue@N@Attribute@U2@@QBENPAVWorkflowContext@Workflow@1@@Z 10011bb0 f i DiamondClassifyWorker.obj
 0001:00010c20       ??$getAttributeValueWithoutScript@H@Attribute@U2@@QBEHXZ 10011c20 f i DiamondClassifyWorker.obj
 0001:00010c60       ??$getAttributeValueWithoutScript@I@Attribute@U2@@QBEIXZ 10011c60 f i DiamondClassifyWorker.obj
 0001:00010ca0       ??$getAttributeValueWithoutScript@N@Attribute@U2@@QBENXZ 10011ca0 f i DiamondClassifyWorker.obj
 0001:00010d10       ??$getKeyImpl@V?$QMap@VQString@@I@@@QAssociativeIterableImpl@QtMetaTypePrivate@@SA?AUVariantData@1@PBQAXHI@Z 10011d10 f i DiamondClassifyWorker.obj
 0001:00010d30       ??$getValue@H@BaseWorker@LocalWorkflow@U2@@IBEHABVQString@@@Z 10011d30 f i DiamondClassifyWorker.obj
 0001:00010d60       ??$getValue@I@BaseWorker@LocalWorkflow@U2@@IBEIABVQString@@@Z 10011d60 f i DiamondClassifyWorker.obj
 0001:00010dc0       ??$getValue@N@BaseWorker@LocalWorkflow@U2@@IBENABVQString@@@Z 10011dc0 f i DiamondClassifyWorker.obj
 0001:00010e50       ??$getValueImpl@V?$QMap@VQString@@I@@@QAssociativeIterableImpl@QtMetaTypePrivate@@SA?AUVariantData@1@PBQAXHI@Z 10011e50 f i DiamondClassifyWorker.obj
 0001:00010e70       ??$qMetaTypeId@H@@YAHXZ    10011e70 f i DiamondClassifyWorker.obj
 0001:00010e80       ??$qMetaTypeId@I@@YAHXZ    10011e80 f i DiamondClassifyWorker.obj
 0001:00010e90       ??$qMetaTypeId@N@@YAHXZ    10011e90 f i DiamondClassifyWorker.obj
 0001:00010ea0       ??$qMetaTypeId@V?$QMap@VQString@@I@@@@YAHXZ 10011ea0 f i DiamondClassifyWorker.obj
 0001:00010eb0       ??$qMetaTypeId@VQAssociativeIterableImpl@QtMetaTypePrivate@@@@YAHXZ 10011eb0 f i DiamondClassifyWorker.obj
 0001:00010ec0       ??$qRegisterMetaType@V?$QMap@VQString@@I@@@@YAHPBDPAV?$QMap@VQString@@I@@W4DefinedType@?$MetaTypeDefinedHelper@V?$QMap@VQString@@I@@$00@QtPrivate@@@Z 10011ec0 f i DiamondClassifyWorker.obj
 0001:00010f30       ??$qRegisterMetaType@VQAssociativeIterableImpl@QtMetaTypePrivate@@@@YAHPBDPAVQAssociativeIterableImpl@QtMetaTypePrivate@@W4DefinedType@?$MetaTypeDefinedHelper@VQAssociativeIterableImpl@QtMetaTypePrivate@@$00@QtPrivate@@@Z 10011f30 f i DiamondClassifyWorker.obj
 0001:00010ff0       ??$qRegisterNormalizedMetaType@V?$QMap@VQString@@I@@@@YAHABVQByteArray@@PAV?$QMap@VQString@@I@@W4DefinedType@?$MetaTypeDefinedHelper@V?$QMap@VQString@@I@@$00@QtPrivate@@@Z 10011ff0 f i DiamondClassifyWorker.obj
 0001:00011060       ??$qRegisterNormalizedMetaType@VQAssociativeIterableImpl@QtMetaTypePrivate@@@@YAHABVQByteArray@@PAVQAssociativeIterableImpl@QtMetaTypePrivate@@W4DefinedType@?$MetaTypeDefinedHelper@VQAssociativeIterableImpl@QtMetaTypePrivate@@$00@QtPrivate@@@Z 10012060 f i DiamondClassifyWorker.obj
 0001:000110c0       ??$qVariantFromValue@V?$QMap@VQString@@I@@@@YA?AVQVariant@@ABV?$QMap@VQString@@I@@@Z 100120c0 f i DiamondClassifyWorker.obj
 0001:000110f0       ??$qobject_cast@PAVDiamondClassifyTask@U2@@@@YAPAVDiamondClassifyTask@U2@@PAVQObject@@@Z 100120f0 f i DiamondClassifyWorker.obj
 0001:00011110       ??$qvariant_cast@H@@YAHABVQVariant@@@Z 10012110 f i DiamondClassifyWorker.obj
 0001:00011150       ??$qvariant_cast@I@@YAIABVQVariant@@@Z 10012150 f i DiamondClassifyWorker.obj
 0001:00011190       ??$qvariant_cast@N@@YANABVQVariant@@@Z 10012190 f i DiamondClassifyWorker.obj
 0001:00011200       ??$sizeImpl@V?$QMap@VQString@@I@@@QAssociativeIterableImpl@QtMetaTypePrivate@@SAHPBX@Z 10012200 f i DiamondClassifyWorker.obj
 0001:00011240       ??$value@H@QVariant@@QBEHXZ 10012240 f i DiamondClassifyWorker.obj
 0001:00011280       ??$value@I@QVariant@@QBEIXZ 10012280 f i DiamondClassifyWorker.obj
 0001:000112c0       ??$value@N@QVariant@@QBENXZ 100122c0 f i DiamondClassifyWorker.obj
 0001:00011320       ??0?$ConverterFunctor@V?$QMap@VQString@@I@@VQAssociativeIterableImpl@QtMetaTypePrivate@@U?$QAssociativeIterableConvertFunctor@V?$QMap@VQString@@I@@@3@@QtPrivate@@QAE@U?$QAssociativeIterableConvertFunctor@V?$QMap@VQString@@I@@@QtMetaTypePrivate@@@Z 10012320 f i DiamondClassifyWorker.obj
 0001:00011330       ??0?$QMap@VQString@@I@@QAE@ABV0@@Z 10012330 f i DiamondClassifyWorker.obj
 0001:000113a0       ??0AbstractConverterFunction@QtPrivate@@QAE@P6A_NPBU01@PBXPAX@Z@Z 100123a0 f i DiamondClassifyWorker.obj
 0001:000113b0       ??0DiamondClassifyWorker@LocalWorkflow@U2@@QAE@PAVActor@Workflow@2@@Z 100123b0 f   DiamondClassifyWorker.obj
 0001:000113f0       ??0QAssociativeIterableImpl@QtMetaTypePrivate@@QAE@XZ 100123f0 f i DiamondClassifyWorker.obj
 0001:00011460       ??0VariantData@QtMetaTypePrivate@@QAE@HPBXI@Z 10012460 f i DiamondClassifyWorker.obj
 0001:00011480       ??0const_iterator@?$QMap@VQString@@I@@QAE@PBU?$QMapNode@VQString@@I@@@Z 10012480 f i DiamondClassifyWorker.obj
 0001:00011490       ??0const_iterator@?$QMap@VQString@@I@@QAE@XZ 10012490 f i DiamondClassifyWorker.obj
 0001:000114a0       ??1?$ConverterFunctor@V?$QMap@VQString@@I@@VQAssociativeIterableImpl@QtMetaTypePrivate@@U?$QAssociativeIterableConvertFunctor@V?$QMap@VQString@@I@@@3@@QtPrivate@@QAE@XZ 100124a0 f i DiamondClassifyWorker.obj
 0001:000114c0       ??1DiamondClassifyWorker@LocalWorkflow@U2@@UAE@XZ 100124c0 f i DiamondClassifyWorker.obj
 0001:000114d0       ??8const_iterator@?$QMap@VQString@@I@@QBE_NABV01@@Z 100124d0 f i DiamondClassifyWorker.obj
 0001:000114f0       ??9const_iterator@?$QMap@VQString@@I@@QBE_NABV01@@Z 100124f0 f i DiamondClassifyWorker.obj
 0001:00011510       ??Econst_iterator@?$QMap@VQString@@I@@QAEAAV01@XZ 10012510 f i DiamondClassifyWorker.obj
 0001:00011530       ??Fconst_iterator@?$QMap@VQString@@I@@QAEAAV01@XZ 10012530 f i DiamondClassifyWorker.obj
 0001:00011550       ??R?$QAssociativeIterableConvertFunctor@V?$QMap@VQString@@I@@@QtMetaTypePrivate@@QBE?AVQAssociativeIterableImpl@1@ABV?$QMap@VQString@@I@@@Z 10012550 f i DiamondClassifyWorker.obj
 0001:00011565       ??_EDiamondClassifyWorker@LocalWorkflow@U2@@W7AEPAXI@Z 10012565 f i DiamondClassifyWorker.obj
 0001:0001156d       ??_EDiamondClassifyWorker@LocalWorkflow@U2@@WBA@AEPAXI@Z 1001256d f i DiamondClassifyWorker.obj
 0001:00011580       ??_G?$QMap@VQString@@I@@QAEPAXI@Z 10012580 f i DiamondClassifyWorker.obj
 0001:000115b0       ??_GDiamondClassifyWorker@LocalWorkflow@U2@@UAEPAXI@Z 100125b0 f i DiamondClassifyWorker.obj
 0001:000115b0       ??_EDiamondClassifyWorker@LocalWorkflow@U2@@UAEPAXI@Z 100125b0 f i DiamondClassifyWorker.obj
 0001:000115e0       ?Construct@?$QMetaTypeFunctionHelper@V?$QMap@VQString@@I@@$00@QtMetaTypePrivate@@SAPAXPAXPBX@Z 100125e0 f i DiamondClassifyWorker.obj
 0001:00011670       ?Construct@?$QMetaTypeFunctionHelper@VQAssociativeIterableImpl@QtMetaTypePrivate@@$00@QtMetaTypePrivate@@SAPAXPAXPBX@Z 10012670 f i DiamondClassifyWorker.obj
 0001:000116c0       ?Create@?$QMetaTypeFunctionHelper@V?$QMap@VQString@@I@@$00@QtMetaTypePrivate@@SAPAXPBX@Z 100126c0 f i DiamondClassifyWorker.obj
 0001:00011760       ?Create@?$QMetaTypeFunctionHelper@VQAssociativeIterableImpl@QtMetaTypePrivate@@$00@QtMetaTypePrivate@@SAPAXPBX@Z 10012760 f i DiamondClassifyWorker.obj
 0001:000117c0       ?Delete@?$QMetaTypeFunctionHelper@V?$QMap@VQString@@I@@$00@QtMetaTypePrivate@@SAXPAX@Z 100127c0 f i DiamondClassifyWorker.obj
 0001:000117e0       ?Delete@?$QMetaTypeFunctionHelper@VQAssociativeIterableImpl@QtMetaTypePrivate@@$00@QtMetaTypePrivate@@SAXPAX@Z 100127e0 f i DiamondClassifyWorker.obj
 0001:000117f0       ?Destruct@?$QMetaTypeFunctionHelper@V?$QMap@VQString@@I@@$00@QtMetaTypePrivate@@SAXPAX@Z 100127f0 f i DiamondClassifyWorker.obj
 0001:00011800       ?Destruct@?$QMetaTypeFunctionHelper@VQAssociativeIterableImpl@QtMetaTypePrivate@@$00@QtMetaTypePrivate@@SAXPAX@Z 10012800 f i DiamondClassifyWorker.obj
 0001:00011810       ?assign@?$IteratorOwnerCommon@Vconst_iterator@?$QMap@VQString@@I@@@QtMetaTypePrivate@@SAXPAPAXPBQAX@Z 10012810 f i DiamondClassifyWorker.obj
 0001:00011840       ?assign@?$IteratorOwnerCommon@Vconst_iterator@?$QMap@VQString@@I@@@QtMetaTypePrivate@@SAXPAPAXVconst_iterator@?$QMap@VQString@@I@@@Z 10012840 f i DiamondClassifyWorker.obj
 0001:00011870       ?begin@?$QMap@VQString@@I@@QBE?AVconst_iterator@1@XZ 10012870 f i DiamondClassifyWorker.obj
 0001:00011890       ?begin@?$QMapData@VQString@@I@@QAEPAU?$QMapNode@VQString@@I@@XZ 10012890 f i DiamondClassifyWorker.obj
 0001:000118a0       ?cleanup@DiamondClassifyWorker@LocalWorkflow@U2@@UAEXXZ 100128a0 f   DiamondClassifyWorker.obj
 0001:000118b0       ?constFind@?$QMap@VQString@@I@@QBE?AVconst_iterator@1@ABVQString@@@Z 100128b0 f i DiamondClassifyWorker.obj
 0001:00011900       ?convert@?$ConverterFunctor@V?$QMap@VQString@@I@@VQAssociativeIterableImpl@QtMetaTypePrivate@@U?$QAssociativeIterableConvertFunctor@V?$QMap@VQString@@I@@@3@@QtPrivate@@SA_NPBUAbstractConverterFunction@2@PBXPAX@Z 10012900 f i DiamondClassifyWorker.obj
 0001:00011950       ?destroy@?$IteratorOwnerCommon@Vconst_iterator@?$QMap@VQString@@I@@@QtMetaTypePrivate@@SAXPAPAX@Z 10012950 f i DiamondClassifyWorker.obj
 0001:00011970       ?end@?$QMap@VQString@@I@@QBE?AVconst_iterator@1@XZ 10012970 f i DiamondClassifyWorker.obj
 0001:00011990       ?equal@?$IteratorOwnerCommon@Vconst_iterator@?$QMap@VQString@@I@@@QtMetaTypePrivate@@SA_NPBQAX0@Z 10012990 f i DiamondClassifyWorker.obj
 0001:000119b0       ?find@?$QMap@VQString@@I@@QBE?AVconst_iterator@1@ABVQString@@@Z 100129b0 f i DiamondClassifyWorker.obj
 0001:00011a00       ?getKey@?$AssociativeContainerAccessor@V?$QMap@VQString@@I@@$00@QtMetaTypePrivate@@SAABVQString@@ABVconst_iterator@?$QMap@VQString@@I@@@Z 10012a00 f i DiamondClassifyWorker.obj
 0001:00011a10       ?getSettings@DiamondClassifyWorker@LocalWorkflow@U2@@AAE?AUDiamondClassifyTaskSettings@3@AAVU2OpStatus@3@@Z 10012a10 f   DiamondClassifyWorker.obj
 0001:00012120       ?getValue@?$AssociativeContainerAccessor@V?$QMap@VQString@@I@@$00@QtMetaTypePrivate@@SAABIABVconst_iterator@?$QMap@VQString@@I@@@Z 10013120 f i DiamondClassifyWorker.obj
 0001:00012130       ?init@DiamondClassifyWorker@LocalWorkflow@U2@@UAEXXZ 10013130 f   DiamondClassifyWorker.obj
 0001:000124b0       ?invoke@?$MetaTypeInvoker@U?$QVariantValueHelper@H@QtPrivate@@ABVQVariant@@H@QtPrivate@@SAHABVQVariant@@@Z 100134b0 f i DiamondClassifyWorker.obj
 0001:000124f0       ?invoke@?$MetaTypeInvoker@U?$QVariantValueHelper@I@QtPrivate@@ABVQVariant@@I@QtPrivate@@SAIABVQVariant@@@Z 100134f0 f i DiamondClassifyWorker.obj
 0001:00012530       ?invoke@?$MetaTypeInvoker@U?$QVariantValueHelper@N@QtPrivate@@ABVQVariant@@N@QtPrivate@@SANABVQVariant@@@Z 10013530 f i DiamondClassifyWorker.obj
 0001:000125a0       ?key@const_iterator@?$QMap@VQString@@I@@QBEABVQString@@XZ 100135a0 f i DiamondClassifyWorker.obj
 0001:000125b0       ?metaType@?$QVariantValueHelper@H@QtPrivate@@SAHABVQVariant@@@Z 100135b0 f i DiamondClassifyWorker.obj
 0001:000125f0       ?metaType@?$QVariantValueHelper@I@QtPrivate@@SAIABVQVariant@@@Z 100135f0 f i DiamondClassifyWorker.obj
 0001:00012630       ?metaType@?$QVariantValueHelper@N@QtPrivate@@SANABVQVariant@@@Z 10013630 f i DiamondClassifyWorker.obj
 0001:00012680       ?nextNode@?$QMapNode@VQString@@I@@QBEPBU1@XZ 10013680 f i DiamondClassifyWorker.obj
 0001:00012690       ?previousNode@?$QMapNode@VQString@@I@@QBEPBU1@XZ 10013690 f i DiamondClassifyWorker.obj
 0001:000126a0       ?qt_metatype_id@?$QMetaTypeId2@H@@SAHXZ 100136a0 f i DiamondClassifyWorker.obj
 0001:000126b0       ?qt_metatype_id@?$QMetaTypeId2@I@@SAHXZ 100136b0 f i DiamondClassifyWorker.obj
 0001:000126c0       ?qt_metatype_id@?$QMetaTypeId2@N@@SAHXZ 100136c0 f i DiamondClassifyWorker.obj
 0001:000126d0       ?qt_metatype_id@?$QMetaTypeId2@V?$QMap@VQString@@I@@@@SAHXZ 100136d0 f i DiamondClassifyWorker.obj
 0001:000126e0       ?qt_metatype_id@?$QMetaTypeId2@VQAssociativeIterableImpl@QtMetaTypePrivate@@@@SAHXZ 100136e0 f i DiamondClassifyWorker.obj
 0001:000126f0       ?qt_metatype_id@?$QMetaTypeId@V?$QMap@VQString@@I@@@@SAHXZ 100136f0 f i DiamondClassifyWorker.obj
 0001:000127a0       ?qt_metatype_id@?$QMetaTypeId@VQAssociativeIterableImpl@QtMetaTypePrivate@@@@SAHXZ 100137a0 f i DiamondClassifyWorker.obj
 0001:00012840       ?qt_metatype_id@?$QMetaTypeIdHelper@V?$QMap@VQString@@I@@$00@QtPrivate@@SAHXZ 10013840 f i DiamondClassifyWorker.obj
 0001:00012850       ?qt_metatype_id@?$QMetaTypeIdHelper@VQAssociativeIterableImpl@QtMetaTypePrivate@@$00@QtPrivate@@SAHXZ 10013850 f i DiamondClassifyWorker.obj
 0001:00012860       ?registerConverter@?$AssociativeContainerConverterHelper@VQAssociativeIterableImpl@QtMetaTypePrivate@@$0A@@QtPrivate@@SA_NH@Z 10013860 f i DiamondClassifyWorker.obj
 0001:00012870       ?registerConverter@?$AssociativeValueTypeIsMetaType@V?$QMap@VQString@@I@@$00@QtPrivate@@SA_NH@Z 10013870 f i DiamondClassifyWorker.obj
 0001:000128e0       ?registerConverter@?$IsPair@V?$QMap@VQString@@I@@@QtPrivate@@SA_NH@Z 100138e0 f i DiamondClassifyWorker.obj
 0001:000128f0       ?registerConverter@?$IsPair@VQAssociativeIterableImpl@QtMetaTypePrivate@@@QtPrivate@@SA_NH@Z 100138f0 f i DiamondClassifyWorker.obj
 0001:00012900       ?registerConverter@?$MetaTypeSmartPointerHelper@V?$QMap@VQString@@I@@X@QtPrivate@@SA_NH@Z 10013900 f i DiamondClassifyWorker.obj
 0001:00012910       ?registerConverter@?$MetaTypeSmartPointerHelper@VQAssociativeIterableImpl@QtMetaTypePrivate@@X@QtPrivate@@SA_NH@Z 10013910 f i DiamondClassifyWorker.obj
 0001:00012920       ?registerConverter@?$SequentialContainerConverterHelper@V?$QMap@VQString@@I@@$0A@@QtPrivate@@SA_NH@Z 10013920 f i DiamondClassifyWorker.obj
 0001:00012930       ?registerConverter@?$SequentialContainerConverterHelper@VQAssociativeIterableImpl@QtMetaTypePrivate@@$0A@@QtPrivate@@SA_NH@Z 10013930 f i DiamondClassifyWorker.obj
 0001:00012940       ?size@?$QMap@VQString@@I@@QBEHXZ 10013940 f i DiamondClassifyWorker.obj
 0001:00012950       ?sl_taskFinished@DiamondClassifyWorker@LocalWorkflow@U2@@AAEXPAVTask@3@@Z 10013950 f   DiamondClassifyWorker.obj
 0001:00012bf0       ?tick@DiamondClassifyWorker@LocalWorkflow@U2@@UAEPAVTask@3@XZ 10013bf0 f   DiamondClassifyWorker.obj
 0001:00012e00       ?tr@DiamondClassifyWorker@LocalWorkflow@U2@@SA?AVQString@@PBD0H@Z 10013e00 f i DiamondClassifyWorker.obj
 0001:00012e30       ?value@?$MetaObjectForType@V?$QMap@VQString@@I@@$0A@@QtPrivate@@SAPBUQMetaObject@@XZ 10013e30 f i DiamondClassifyWorker.obj
 0001:00012e40       ?value@?$MetaObjectForType@VQAssociativeIterableImpl@QtMetaTypePrivate@@$0A@@QtPrivate@@SAPBUQMetaObject@@XZ 10013e40 f i DiamondClassifyWorker.obj
 0001:00012e50       ?value@const_iterator@?$QMap@VQString@@I@@QBEABIXZ 10013e50 f i DiamondClassifyWorker.obj
 0001:00012e60       ??$?0VQString@@H@?$QPair@VQString@@VQVariant@@@@QAE@$$QAU?$QPair@VQString@@H@@@Z 10013e60 f i DiamondClassifyWorkerFactory.obj
 0001:00012ec0       ??$?0VQString@@V0@@?$QPair@VQString@@VQVariant@@@@QAE@$$QAU?$QPair@VQString@@V1@@@@Z 10013ec0 f i DiamondClassifyWorkerFactory.obj
 0001:00012f20       ??$qMakePair@VQString@@H@@YA?AU?$QPair@VQString@@H@@ABVQString@@ABH@Z 10013f20 f i DiamondClassifyWorkerFactory.obj
 0001:00012f50       ??$qMakePair@VQString@@V1@@@YA?AU?$QPair@VQString@@V1@@@ABVQString@@0@Z 10013f50 f i DiamondClassifyWorkerFactory.obj
 0001:00012fb0       ??0?$QFlags@W4Flag@Attribute@U2@@@@QAE@VQFlag@@@Z 10013fb0 f i DiamondClassifyWorkerFactory.obj
 0001:00012fc0       ??0?$QFlags@W4Flag@Attribute@U2@@@@QAE@W4Flag@Attribute@U2@@@Z 10013fc0 f i DiamondClassifyWorkerFactory.obj
 0001:00012fd0       ??0?$QForeachContainer@V?$QList@PAVDNATranslation@U2@@@@@@QAE@ABV?$QList@PAVDNATranslation@U2@@@@@Z 10013fd0 f i DiamondClassifyWorkerFactory.obj
 0001:00013010       ??0?$QList@PAVDNATranslation@U2@@@@QAE@ABV0@@Z 10014010 f i DiamondClassifyWorkerFactory.obj
 0001:000130d0       ??0?$QList@U?$QPair@VQString@@V1@@@@@QAE@XZ 100140d0 f i DiamondClassifyWorkerFactory.obj
 0001:000130e0       ??0?$QList@U?$QPair@VQString@@VQVariant@@@@@@QAE@XZ 100140e0 f i DiamondClassifyWorkerFactory.obj
 0001:000130f0       ??0?$QPair@VQString@@H@@QAE@ABVQString@@ABH@Z 100140f0 f i DiamondClassifyWorkerFactory.obj
 0001:00013110       ??0?$QPair@VQString@@V1@@@QAE@ABU0@@Z 10014110 f i DiamondClassifyWorkerFactory.obj
 0001:00013170       ??0?$QPair@VQString@@V1@@@QAE@ABVQString@@0@Z 10014170 f i DiamondClassifyWorkerFactory.obj
 0001:000131d0       ??0?$QPair@VQString@@VQVariant@@@@QAE@ABU0@@Z 100141d0 f i DiamondClassifyWorkerFactory.obj
 0001:00013230       ??0DiamondClassifyWorkerFactory@LocalWorkflow@U2@@QAE@XZ 10014230 f   DiamondClassifyWorkerFactory.obj
 0001:00013250       ??0const_iterator@?$QList@PAVDNATranslation@U2@@@@QAE@PAUNode@1@@Z 10014250 f i DiamondClassifyWorkerFactory.obj
 0001:00013260       ??1?$QForeachContainer@V?$QList@PAVDNATranslation@U2@@@@@@QAE@XZ 10014260 f i DiamondClassifyWorkerFactory.obj
 0001:00013290       ??1?$QList@PAVDNATranslation@U2@@@@QAE@XZ 10014290 f i DiamondClassifyWorkerFactory.obj
 0001:000132c0       ??1?$QList@U?$QPair@VQString@@V1@@@@@QAE@XZ 100142c0 f i DiamondClassifyWorkerFactory.obj
 0001:00013310       ??1?$QList@U?$QPair@VQString@@VQVariant@@@@@@QAE@XZ 10014310 f i DiamondClassifyWorkerFactory.obj
 0001:00013360       ??1?$QPair@VQString@@H@@QAE@XZ 10014360 f i DiamondClassifyWorkerFactory.obj
 0001:00013370       ??1?$QPair@VQString@@V1@@@QAE@XZ 10014370 f i DiamondClassifyWorkerFactory.obj
 0001:000133d0       ??1?$QPair@VQString@@VQVariant@@@@QAE@XZ 100143d0 f i DiamondClassifyWorkerFactory.obj
 0001:00013430       ??1DiamondClassifyWorkerFactory@LocalWorkflow@U2@@UAE@XZ 10014430 f i DiamondClassifyWorkerFactory.obj
 0001:00013440       ??6?$QList@U?$QPair@VQString@@V1@@@@@QAEAAV0@ABU?$QPair@VQString@@V1@@@@Z 10014440 f i DiamondClassifyWorkerFactory.obj
 0001:00013460       ??9const_iterator@?$QList@PAVDNATranslation@U2@@@@QBE_NABV01@@Z 10014460 f i DiamondClassifyWorkerFactory.obj
 0001:00013480       ??Dconst_iterator@?$QList@PAVDNATranslation@U2@@@@QBEABQAVDNATranslation@U2@@XZ 10014480 f i DiamondClassifyWorkerFactory.obj
 0001:00013490       ??Econst_iterator@?$QList@PAVDNATranslation@U2@@@@QAEAAV01@XZ 10014490 f i DiamondClassifyWorkerFactory.obj
 0001:000134a0       ??U?$QFlags@W4Flag@Attribute@U2@@@@QBE?AV0@W4Flag@Attribute@U2@@@Z 100144a0 f i DiamondClassifyWorkerFactory.obj
 0001:000134c0       ??U@YA?AV?$QFlags@W4Flag@Attribute@U2@@@@W4Flag@Attribute@U2@@0@Z 100144c0 f i DiamondClassifyWorkerFactory.obj
 0001:000134d0       ??_EDiamondClassifyWorkerFactory@LocalWorkflow@U2@@W7AEPAXI@Z 100144d0 f i DiamondClassifyWorkerFactory.obj
 0001:000134e0       ??_G?$QPair@VQString@@V1@@@QAEPAXI@Z 100144e0 f i DiamondClassifyWorkerFactory.obj
 0001:00013550       ??_G?$QPair@VQString@@VQVariant@@@@QAEPAXI@Z 10014550 f i DiamondClassifyWorkerFactory.obj
 0001:000135c0       ??_EComboBoxDelegate@U2@@UAEPAXI@Z 100145c0 f i DiamondClassifyWorkerFactory.obj
 0001:000135c0       ??_GComboBoxDelegate@U2@@UAEPAXI@Z 100145c0 f i DiamondClassifyWorkerFactory.obj
 0001:000135f0       ??_EDatabaseDelegate@LocalWorkflow@U2@@UAEPAXI@Z 100145f0 f i DiamondClassifyWorkerFactory.obj
 0001:000135f0       ??_GDatabaseDelegate@LocalWorkflow@U2@@UAEPAXI@Z 100145f0 f i DiamondClassifyWorkerFactory.obj
 0001:00013620       ??_EDiamondClassifyWorkerFactory@LocalWorkflow@U2@@UAEPAXI@Z 10014620 f i DiamondClassifyWorkerFactory.obj
 0001:00013620       ??_GDiamondClassifyWorkerFactory@LocalWorkflow@U2@@UAEPAXI@Z 10014620 f i DiamondClassifyWorkerFactory.obj
 0001:00013650       ??_EDoubleSpinBoxDelegate@U2@@UAEPAXI@Z 10014650 f i DiamondClassifyWorkerFactory.obj
 0001:00013650       ??_GDoubleSpinBoxDelegate@U2@@UAEPAXI@Z 10014650 f i DiamondClassifyWorkerFactory.obj
 0001:00013680       ??_ESpinBoxDelegate@U2@@UAEPAXI@Z 10014680 f i DiamondClassifyWorkerFactory.obj
 0001:00013680       ??_GSpinBoxDelegate@U2@@UAEPAXI@Z 10014680 f i DiamondClassifyWorkerFactory.obj
 0001:000136b0       ?append@?$QList@U?$QPair@VQString@@V1@@@@@QAEXABU?$QPair@VQString@@V1@@@@Z 100146b0 f i DiamondClassifyWorkerFactory.obj
 0001:00013740       ?append@?$QList@U?$QPair@VQString@@VQVariant@@@@@@QAEXABU?$QPair@VQString@@VQVariant@@@@@Z 10014740 f i DiamondClassifyWorkerFactory.obj
 0001:000137d0       ?begin@?$QList@PAVDNATranslation@U2@@@@QBE?AVconst_iterator@1@XZ 100147d0 f i DiamondClassifyWorkerFactory.obj
 0001:000137f0       ?cleanup@DiamondClassifyWorkerFactory@LocalWorkflow@U2@@SAXXZ 100147f0 f   DiamondClassifyWorkerFactory.obj
 0001:00013840       ?createWorker@DiamondClassifyWorkerFactory@LocalWorkflow@U2@@UAEPAVWorker@Workflow@3@PAVActor@53@@Z 10014840 f   DiamondClassifyWorkerFactory.obj
 0001:000138b0       ?dealloc@?$QList@PAVDNATranslation@U2@@@@AAEXPAUData@QListData@@@Z 100148b0 f i DiamondClassifyWorkerFactory.obj
 0001:000138d0       ?dealloc@?$QList@U?$QPair@VQString@@V1@@@@@AAEXPAUData@QListData@@@Z 100148d0 f i DiamondClassifyWorkerFactory.obj
 0001:00013900       ?dealloc@?$QList@U?$QPair@VQString@@VQVariant@@@@@@AAEXPAUData@QListData@@@Z 10014900 f i DiamondClassifyWorkerFactory.obj
 0001:00013930       ?detach_helper_grow@?$QList@U?$QPair@VQString@@V1@@@@@AAEPAUNode@1@HH@Z 10014930 f i DiamondClassifyWorkerFactory.obj
 0001:00013aa0       ?detach_helper_grow@?$QList@U?$QPair@VQString@@VQVariant@@@@@@AAEPAUNode@1@HH@Z 10014aa0 f i DiamondClassifyWorkerFactory.obj
 0001:00013c10       ?end@?$QList@PAVDNATranslation@U2@@@@QBE?AVconst_iterator@1@XZ 10014c10 f i DiamondClassifyWorkerFactory.obj
 0001:00013c30       ?init@DiamondClassifyWorkerFactory@LocalWorkflow@U2@@SAXXZ 10014c30 f   DiamondClassifyWorkerFactory.obj
 0001:000171b0       ?max@?$numeric_limits@H@std@@SAHXZ 100181b0 f i DiamondClassifyWorkerFactory.obj
 0001:000171c0       ?node_construct@?$QList@U?$QPair@VQString@@V1@@@@@AAEXPAUNode@1@ABU?$QPair@VQString@@V1@@@@Z 100181c0 f i DiamondClassifyWorkerFactory.obj
 0001:00017250       ?node_construct@?$QList@U?$QPair@VQString@@VQVariant@@@@@@AAEXPAUNode@1@ABU?$QPair@VQString@@VQVariant@@@@@Z 10018250 f i DiamondClassifyWorkerFactory.obj
 0001:000172e0       ?node_copy@?$QList@PAVDNATranslation@U2@@@@AAEXPAUNode@1@00@Z 100182e0 f i DiamondClassifyWorkerFactory.obj
 0001:00017310       ?node_copy@?$QList@U?$QPair@VQString@@V1@@@@@AAEXPAUNode@1@00@Z 10018310 f i DiamondClassifyWorkerFactory.obj
 0001:00017410       ?node_copy@?$QList@U?$QPair@VQString@@VQVariant@@@@@@AAEXPAUNode@1@00@Z 10018410 f i DiamondClassifyWorkerFactory.obj
 0001:00017510       ?node_destruct@?$QList@PAVDNATranslation@U2@@@@AAEXPAUNode@1@0@Z 10018510 f i DiamondClassifyWorkerFactory.obj
 0001:00017520       ?node_destruct@?$QList@U?$QPair@VQString@@V1@@@@@AAEXPAUNode@1@0@Z 10018520 f i DiamondClassifyWorkerFactory.obj
 0001:000175a0       ?node_destruct@?$QList@U?$QPair@VQString@@V1@@@@@AAEXPAUNode@1@@Z 100185a0 f i DiamondClassifyWorkerFactory.obj
 0001:00017610       ?node_destruct@?$QList@U?$QPair@VQString@@VQVariant@@@@@@AAEXPAUNode@1@0@Z 10018610 f i DiamondClassifyWorkerFactory.obj
 0001:00017690       ?node_destruct@?$QList@U?$QPair@VQString@@VQVariant@@@@@@AAEXPAUNode@1@@Z 10018690 f i DiamondClassifyWorkerFactory.obj
 0001:00017700       ?t@Node@?$QList@PAVDNATranslation@U2@@@@QAEAAPAVDNATranslation@U2@@XZ 10018700 f i DiamondClassifyWorkerFactory.obj
 0001:00017710       ??0DiamondSupport@U2@@QAE@ABVQString@@@Z 10018710 f   DiamondSupport.obj
 0001:00017860       ??1DiamondSupport@U2@@UAE@XZ 10018860 f i DiamondSupport.obj
 0001:00017870       ??_GDiamondSupport@U2@@UAEPAXI@Z 10018870 f i DiamondSupport.obj
 0001:00017870       ??_EDiamondSupport@U2@@UAEPAXI@Z 10018870 f i DiamondSupport.obj
 0001:000178a0       ?tr@DiamondSupport@U2@@SA?AVQString@@PBD0H@Z 100188a0 f i DiamondSupport.obj
 0001:000178d0       ??0DiamondSupportPlugin@U2@@QAE@XZ 100188d0 f   DiamondSupportPlugin.obj
 0001:00017980       ??1DiamondSupportPlugin@U2@@UAE@XZ 10018980 f   DiamondSupportPlugin.obj
 0001:000179f0       ??_GDiamondSupportPlugin@U2@@UAEPAXI@Z 100189f0 f i DiamondSupportPlugin.obj
 0001:000179f0       ??_EDiamondSupportPlugin@U2@@UAEPAXI@Z 100189f0 f i DiamondSupportPlugin.obj
 0001:00017a70       _ugene_plugin_init         10018a70 f   DiamondSupportPlugin.obj
 0001:00017a90       ??0GenomesPreparationTask@U2@@QAE@ABVQStringList@@ABVQString@@@Z 10018a90 f   GenomesPreparationTask.obj
 0001:00017ba0       ??1GenomesPreparationTask@U2@@UAE@XZ 10018ba0 f i GenomesPreparationTask.obj
 0001:00017c10       ??_EGenomesPreparationTask@U2@@UAEPAXI@Z 10018c10 f i GenomesPreparationTask.obj
 0001:00017c10       ??_GGenomesPreparationTask@U2@@UAEPAXI@Z 10018c10 f i GenomesPreparationTask.obj
 0001:00017c90       ?at@?$QList@VQString@@@@QBEABVQString@@H@Z 10018c90 f i GenomesPreparationTask.obj
 0001:00017cb0       ?count@?$QList@VQString@@@@QBEHXZ 10018cb0 f i GenomesPreparationTask.obj
 0001:00017cc0       ?first@?$QList@VQString@@@@QBEABVQString@@XZ 10018cc0 f i GenomesPreparationTask.obj
 0001:00017cd0       ?getPreparedGenomesFileUrl@GenomesPreparationTask@U2@@QBEABVQString@@XZ 10018cd0 f   GenomesPreparationTask.obj
 0001:00017ce0       ?run@GenomesPreparationTask@U2@@EAEXXZ 10018ce0 f   GenomesPreparationTask.obj
 0001:00017f00       ?t@Node@?$QList@VQString@@@@QAEAAVQString@@XZ 10018f00 f i GenomesPreparationTask.obj
 0001:00017f10       ?tr@GenomesPreparationTask@U2@@SA?AVQString@@PBD0H@Z 10018f10 f i GenomesPreparationTask.obj
 0001:00017f40       ??C?$QScopedPointer@VQObjectData@@U?$QScopedPointerDeleter@VQObjectData@@@@@@QBEPAVQObjectData@@XZ 10018f40 f i moc_DiamondBuildPrompter.obj
 0001:00017f50       ?metaObject@DiamondBuildPrompter@LocalWorkflow@U2@@UBEPBUQMetaObject@@XZ 10018f50 f   moc_DiamondBuildPrompter.obj
 0001:00017f70       ?qt_metacall@DiamondBuildPrompter@LocalWorkflow@U2@@UAEHW4Call@QMetaObject@@HPAPAX@Z 10018f70 f   moc_DiamondBuildPrompter.obj
 0001:00017f80       ?qt_metacast@DiamondBuildPrompter@LocalWorkflow@U2@@UAEPAXPBD@Z 10018f80 f   moc_DiamondBuildPrompter.obj
 0001:00017fe0       ?qt_static_metacall@DiamondBuildPrompter@LocalWorkflow@U2@@CAXPAVQObject@@W4Call@QMetaObject@@HPAPAX@Z 10018fe0 f   moc_DiamondBuildPrompter.obj
 0001:00017ff0       ?metaObject@DiamondBuildTask@U2@@UBEPBUQMetaObject@@XZ 10018ff0 f   moc_DiamondBuildTask.obj
 0001:00018010       ?qt_metacall@DiamondBuildTask@U2@@UAEHW4Call@QMetaObject@@HPAPAX@Z 10019010 f   moc_DiamondBuildTask.obj
 0001:00018020       ?qt_metacast@DiamondBuildTask@U2@@UAEPAXPBD@Z 10019020 f   moc_DiamondBuildTask.obj
 0001:00018080       ?qt_static_metacall@DiamondBuildTask@U2@@CAXPAVQObject@@W4Call@QMetaObject@@HPAPAX@Z 10019080 f   moc_DiamondBuildTask.obj
 0001:00018090       ??$qMetaTypeId@PAVTask@U2@@@@YAHXZ 10019090 f i moc_DiamondBuildWorker.obj
 0001:000180a0       ??$qRegisterMetaType@PAVTask@U2@@@@YAHXZ 100190a0 f i moc_DiamondBuildWorker.obj
 0001:000180b0       ??$qRegisterNormalizedMetaType@PAVTask@U2@@@@YAHABVQByteArray@@PAPAVTask@U2@@W4DefinedType@?$MetaTypeDefinedHelper@PAVTask@U2@@$00@QtPrivate@@@Z 100190b0 f i moc_DiamondBuildWorker.obj
 0001:00018110       ?Construct@?$QMetaTypeFunctionHelper@PAVTask@U2@@$00@QtMetaTypePrivate@@SAPAXPAXPBX@Z 10019110 f i moc_DiamondBuildWorker.obj
 0001:00018140       ?Create@?$QMetaTypeFunctionHelper@PAVTask@U2@@$00@QtMetaTypePrivate@@SAPAXPBX@Z 10019140 f i moc_DiamondBuildWorker.obj
 0001:00018180       ?Delete@?$QMetaTypeFunctionHelper@PAVTask@U2@@$00@QtMetaTypePrivate@@SAXPAX@Z 10019180 f i moc_DiamondBuildWorker.obj
 0001:00018190       ?Destruct@?$QMetaTypeFunctionHelper@PAVTask@U2@@$00@QtMetaTypePrivate@@SAXPAX@Z 10019190 f i moc_DiamondBuildWorker.obj
 0001:000181a0       ?metaObject@DiamondBuildWorker@LocalWorkflow@U2@@UBEPBUQMetaObject@@XZ 100191a0 f   moc_DiamondBuildWorker.obj
 0001:000181c0       ?qt_metacall@DiamondBuildWorker@LocalWorkflow@U2@@UAEHW4Call@QMetaObject@@HPAPAX@Z 100191c0 f   moc_DiamondBuildWorker.obj
 0001:00018220       ?qt_metacast@DiamondBuildWorker@LocalWorkflow@U2@@UAEPAXPBD@Z 10019220 f   moc_DiamondBuildWorker.obj
 0001:00018280       ?qt_metatype_id@?$QMetaTypeId2@PAVTask@U2@@@@SAHXZ 10019280 f i moc_DiamondBuildWorker.obj
 0001:00018290       ?qt_metatype_id@?$QMetaTypeIdHelper@PAVTask@U2@@$00@QtPrivate@@SAHXZ 10019290 f i moc_DiamondBuildWorker.obj
 0001:000182a0       ?qt_metatype_id@?$QMetaTypeIdQObject@PAVTask@U2@@$00@@SAHXZ 100192a0 f i moc_DiamondBuildWorker.obj
 0001:00018380       ?qt_static_metacall@DiamondBuildWorker@LocalWorkflow@U2@@CAXPAVQObject@@W4Call@QMetaObject@@HPAPAX@Z 10019380 f   moc_DiamondBuildWorker.obj
 0001:000183e0       ?registerConverter@?$AssociativeContainerConverterHelper@PAVTask@U2@@$0A@@QtPrivate@@SA_NH@Z 100193e0 f i moc_DiamondBuildWorker.obj
 0001:000183f0       ?registerConverter@?$IsPair@PAVTask@U2@@@QtPrivate@@SA_NH@Z 100193f0 f i moc_DiamondBuildWorker.obj
 0001:00018400       ?registerConverter@?$MetaTypeSmartPointerHelper@PAVTask@U2@@X@QtPrivate@@SA_NH@Z 10019400 f i moc_DiamondBuildWorker.obj
 0001:00018410       ?registerConverter@?$SequentialContainerConverterHelper@PAVTask@U2@@$0A@@QtPrivate@@SA_NH@Z 10019410 f i moc_DiamondBuildWorker.obj
 0001:00018420       ?value@?$MetaObjectForType@PAVTask@U2@@$00@QtPrivate@@SAPBUQMetaObject@@XZ 10019420 f i moc_DiamondBuildWorker.obj
 0001:00018430       ?metaObject@DiamondClassifyPrompter@LocalWorkflow@U2@@UBEPBUQMetaObject@@XZ 10019430 f   moc_DiamondClassifyPrompter.obj
 0001:00018450       ?qt_metacall@DiamondClassifyPrompter@LocalWorkflow@U2@@UAEHW4Call@QMetaObject@@HPAPAX@Z 10019450 f   moc_DiamondClassifyPrompter.obj
 0001:00018460       ?qt_metacast@DiamondClassifyPrompter@LocalWorkflow@U2@@UAEPAXPBD@Z 10019460 f   moc_DiamondClassifyPrompter.obj
 0001:000184c0       ?qt_static_metacall@DiamondClassifyPrompter@LocalWorkflow@U2@@CAXPAVQObject@@W4Call@QMetaObject@@HPAPAX@Z 100194c0 f   moc_DiamondClassifyPrompter.obj
 0001:000184d0       ?metaObject@DiamondClassifyTask@U2@@UBEPBUQMetaObject@@XZ 100194d0 f   moc_DiamondClassifyTask.obj
 0001:000184f0       ?qt_metacall@DiamondClassifyTask@U2@@UAEHW4Call@QMetaObject@@HPAPAX@Z 100194f0 f   moc_DiamondClassifyTask.obj
 0001:00018500       ?qt_metacast@DiamondClassifyTask@U2@@UAEPAXPBD@Z 10019500 f   moc_DiamondClassifyTask.obj
 0001:00018560       ?qt_static_metacall@DiamondClassifyTask@U2@@CAXPAVQObject@@W4Call@QMetaObject@@HPAPAX@Z 10019560 f   moc_DiamondClassifyTask.obj
 0001:00018570       ?metaObject@DiamondClassifyWorker@LocalWorkflow@U2@@UBEPBUQMetaObject@@XZ 10019570 f   moc_DiamondClassifyWorker.obj
 0001:00018590       ?qt_metacall@DiamondClassifyWorker@LocalWorkflow@U2@@UAEHW4Call@QMetaObject@@HPAPAX@Z 10019590 f   moc_DiamondClassifyWorker.obj
 0001:000185f0       ?qt_metacast@DiamondClassifyWorker@LocalWorkflow@U2@@UAEPAXPBD@Z 100195f0 f   moc_DiamondClassifyWorker.obj
 0001:00018650       ?qt_static_metacall@DiamondClassifyWorker@LocalWorkflow@U2@@CAXPAVQObject@@W4Call@QMetaObject@@HPAPAX@Z 10019650 f   moc_DiamondClassifyWorker.obj
 0001:000186b0       ?metaObject@DiamondSupport@U2@@UBEPBUQMetaObject@@XZ 100196b0 f   moc_DiamondSupport.obj
 0001:000186d0       ?qt_metacall@DiamondSupport@U2@@UAEHW4Call@QMetaObject@@HPAPAX@Z 100196d0 f   moc_DiamondSupport.obj
 0001:000186e0       ?qt_metacast@DiamondSupport@U2@@UAEPAXPBD@Z 100196e0 f   moc_DiamondSupport.obj
 0001:00018740       ?qt_static_metacall@DiamondSupport@U2@@CAXPAVQObject@@W4Call@QMetaObject@@HPAPAX@Z 10019740 f   moc_DiamondSupport.obj
 0001:00018750       ?metaObject@DiamondSupportPlugin@U2@@UBEPBUQMetaObject@@XZ 10019750 f   moc_DiamondSupportPlugin.obj
 0001:00018770       ?qt_metacall@DiamondSupportPlugin@U2@@UAEHW4Call@QMetaObject@@HPAPAX@Z 10019770 f   moc_DiamondSupportPlugin.obj
 0001:00018780       ?qt_metacast@DiamondSupportPlugin@U2@@UAEPAXPBD@Z 10019780 f   moc_DiamondSupportPlugin.obj
 0001:000187e0       ?qt_static_metacall@DiamondSupportPlugin@U2@@CAXPAVQObject@@W4Call@QMetaObject@@HPAPAX@Z 100197e0 f   moc_DiamondSupportPlugin.obj
 0001:000187f0       ?metaObject@GenomesPreparationTask@U2@@UBEPBUQMetaObject@@XZ 100197f0 f   moc_GenomesPreparationTask.obj
 0001:00018810       ?qt_metacall@GenomesPreparationTask@U2@@UAEHW4Call@QMetaObject@@HPAPAX@Z 10019810 f   moc_GenomesPreparationTask.obj
 0001:00018820       ?qt_metacast@GenomesPreparationTask@U2@@UAEPAXPBD@Z 10019820 f   moc_GenomesPreparationTask.obj
 0001:00018880       ?qt_static_metacall@GenomesPreparationTask@U2@@CAXPAVQObject@@W4Call@QMetaObject@@HPAPAX@Z 10019880 f   moc_GenomesPreparationTask.obj
 0001:00018882       ??0GenomicLibraryDelegate@LocalWorkflow@U2@@QAE@PAVQObject@@@Z 10019882 f   ngs_reads_classification:ngs_reads_classification.dll
 0001:00018888       ?clone@GenomicLibraryDelegate@LocalWorkflow@U2@@UAEPAVPropertyDelegate@3@XZ 10019888 f   ngs_reads_classification:ngs_reads_classification.dll
 0001:0001888e       ?createEditor@GenomicLibraryDelegate@LocalWorkflow@U2@@UBEPAVQWidget@@PAV4@ABVQStyleOptionViewItem@@ABVQModelIndex@@@Z 1001988e f   ngs_reads_classification:ngs_reads_classification.dll
 0001:00018894       ?createWizardWidget@GenomicLibraryDelegate@LocalWorkflow@U2@@UBEPAVPropertyWidget@3@AAVU2OpStatus@3@PAVQWidget@@@Z 10019894 f   ngs_reads_classification:ngs_reads_classification.dll
 0001:0001889a       ?getDisplayValue@GenomicLibraryDelegate@LocalWorkflow@U2@@UBE?AVQVariant@@ABV4@@Z 1001989a f   ngs_reads_classification:ngs_reads_classification.dll
 0001:000188a0       ?metaObject@GenomicLibraryDelegate@LocalWorkflow@U2@@UBEPBUQMetaObject@@XZ 100198a0 f   ngs_reads_classification:ngs_reads_classification.dll
 0001:000188a6       ?qt_metacall@GenomicLibraryDelegate@LocalWorkflow@U2@@UAEHW4Call@QMetaObject@@HPAPAX@Z 100198a6 f   ngs_reads_classification:ngs_reads_classification.dll
 0001:000188ac       ?qt_metacast@GenomicLibraryDelegate@LocalWorkflow@U2@@UAEPAXPBD@Z 100198ac f   ngs_reads_classification:ngs_reads_classification.dll
 0001:000188b2       ?setEditorData@GenomicLibraryDelegate@LocalWorkflow@U2@@UBEXPAVQWidget@@ABVQModelIndex@@@Z 100198b2 f   ngs_reads_classification:ngs_reads_classification.dll
 0001:000188b8       ?setModelData@GenomicLibraryDelegate@LocalWorkflow@U2@@UBEXPAVQWidget@@PAVQAbstractItemModel@@ABVQModelIndex@@@Z 100198b8 f   ngs_reads_classification:ngs_reads_classification.dll
 0001:000188be       ?getBaseFileNameWithSuffixes@NgsReadsClassificationUtils@U2@@SA?AVQString@@ABV3@ABVQStringList@@0_N@Z 100198be f   ngs_reads_classification:ngs_reads_classification.dll
 0001:000188c4       ?countClassified@NgsReadsClassificationUtils@U2@@SAHABV?$QMap@VQString@@I@@@Z 100198c4 f   ngs_reads_classification:ngs_reads_classification.dll
 0001:000188ca       ?TAXONOMY_CLASSIFICATION_SLOT@TaxonomySupport@LocalWorkflow@U2@@SA?BVDescriptor@3@XZ 100198ca f   ngs_reads_classification:ngs_reads_classification.dll
 0001:000188d0       ?TAXONOMY_CLASSIFICATION_TYPE@TaxonomySupport@LocalWorkflow@U2@@SA?AV?$QExplicitlySharedDataPointer@VDataType@U2@@@@XZ 100198d0 f   ngs_reads_classification:ngs_reads_classification.dll
 0001:000188d6       ??0DatabaseDelegate@LocalWorkflow@U2@@QAE@ABVQString@@0ABV?$QList@U?$QPair@VQString@@V1@@@@@0_N@Z 100198d6 f   ngs_reads_classification:ngs_reads_classification.dll
 0001:000188dc       ??1DatabaseDelegate@LocalWorkflow@U2@@UAE@XZ 100198dc f   ngs_reads_classification:ngs_reads_classification.dll
 0001:000188e2       ?update@DatabaseDelegate@LocalWorkflow@U2@@UAEXXZ 100198e2 f   ngs_reads_classification:ngs_reads_classification.dll
 0001:000188e8       ??0Logger@U2@@QAE@ABVQString@@@Z 100198e8 f   U2Core:U2Core.dll
 0001:000188ee       ??1Logger@U2@@UAE@XZ       100198ee f   U2Core:U2Core.dll
 0001:000188f4       ??1GCounter@U2@@UAE@XZ     100198f4 f   U2Core:U2Core.dll
 0001:000188fa       ??0GReportableCounter@U2@@QAE@ABVQString@@0N@Z 100198fa f   U2Core:U2Core.dll
 0001:00018900       ??1SimpleEventCounter@U2@@UAE@XZ 10019900 f   U2Core:U2Core.dll
 0001:00018906       ?rollFileName@GUrlUtils@U2@@SA?AVQString@@ABV3@ABV?$QSet@VQString@@@@@Z 10019906 f   U2Core:U2Core.dll
 0001:0001890c       ?addSubTask@Task@U2@@QAEXPAV12@@Z 1001990c f   U2Core:U2Core.dll
 0001:00018912       ?setError@Task@U2@@QAEXABVQString@@@Z 10019912 f   U2Core:U2Core.dll
 0001:00018918       ??0ExternalToolRunTask@U2@@QAE@ABVQString@@ABVQStringList@@PAVExternalToolLogParser@1@010_N@Z 10019918 f   U2Core:U2Core.dll
 0001:0001891e       ??1ExternalToolRunTask@U2@@UAE@XZ 1001991e f   U2Core:U2Core.dll
 0001:00018924       ??0ExternalToolSupportTask@U2@@QAE@ABVQString@@V?$QFlags@W4TaskFlag@U2@@@@@Z 10019924 f   U2Core:U2Core.dll
 0001:0001892a       ??1ExternalToolSupportTask@U2@@UAE@XZ 1001992a f   U2Core:U2Core.dll
 0001:00018930       ??0ExternalToolLogParser@U2@@QAE@XZ 10019930 f   U2Core:U2Core.dll
 0001:00018936       ??1ExternalToolLogParser@U2@@UAE@XZ 10019936 f   U2Core:U2Core.dll
 0001:0001893c       ?cleanup@Task@U2@@UAEXXZ   1001993c f   U2Core:U2Core.dll
 0001:00018942       ?generateReport@Task@U2@@UBE?AVQString@@XZ 10019942 f   U2Core:U2Core.dll
 0001:00018948       ?getNumParallelSubtasks@Task@U2@@UBEHXZ 10019948 f   U2Core:U2Core.dll
 0001:0001894e       ?getParentTask@Task@U2@@UBEPAV12@XZ 1001994e f   U2Core:U2Core.dll
 0001:00018954       ?getProgress@ExternalToolLogParser@U2@@UAEHXZ 10019954 f   U2Core:U2Core.dll
 0001:0001895a       ?getSubtaskWithErrors@Task@U2@@UBEPAV12@XZ 1001995a f   U2Core:U2Core.dll
 0001:00018960       ?getTaskId@Task@U2@@UBE_JXZ 10019960 f   U2Core:U2Core.dll
 0001:00018966       ?getTopLevelParentTask@Task@U2@@UAEPAV12@XZ 10019966 f   U2Core:U2Core.dll
 0001:0001896c       ?getWarnings@Task@U2@@UBE?AVQStringList@@XZ 1001996c f   U2Core:U2Core.dll
 0001:00018972       ?hasSubtasksWithErrors@Task@U2@@UBE_NXZ 10019972 f   U2Core:U2Core.dll
 0001:00018978       ?hasWarning@Task@U2@@UBE_NXZ 10019978 f   U2Core:U2Core.dll
 0001:0001897e       ?isError@ExternalToolLogParser@U2@@MBE_NABVQString@@@Z 1001997e f   U2Core:U2Core.dll
 0001:00018984       ?isNotificationReport@Task@U2@@UBE_NXZ 10019984 f   U2Core:U2Core.dll
 0001:0001898a       ?isReportingEnabled@Task@U2@@UBE_NXZ 1001998a f   U2Core:U2Core.dll
 0001:00018990       ?isReportingSupported@Task@U2@@UBE_NXZ 10019990 f   U2Core:U2Core.dll
 0001:00018996       ?isTopLevelTask@Task@U2@@UBE_NXZ 10019996 f   U2Core:U2Core.dll
 0001:0001899c       ?metaObject@ExternalToolLogParser@U2@@UBEPBUQMetaObject@@XZ 1001999c f   U2Core:U2Core.dll
 0001:000189a2       ?metaObject@ExternalToolRunTask@U2@@UBEPBUQMetaObject@@XZ 100199a2 f   U2Core:U2Core.dll
 0001:000189a8       ?onSubTaskFinished@Task@U2@@MAE?AV?$QList@PAVTask@U2@@@@PAV12@@Z 100199a8 f   U2Core:U2Core.dll
 0001:000189ae       ?parseErrOutput@ExternalToolLogParser@U2@@UAEXABVQString@@@Z 100199ae f   U2Core:U2Core.dll
 0001:000189b4       ?parseOutput@ExternalToolLogParser@U2@@UAEXABVQString@@@Z 100199b4 f   U2Core:U2Core.dll
 0001:000189ba       ?prepare@Task@U2@@UAEXXZ   100199ba f   U2Core:U2Core.dll
 0001:000189c0       ?processErrLine@ExternalToolLogParser@U2@@MAEXABVQString@@@Z 100199c0 f   U2Core:U2Core.dll
 0001:000189c6       ?processLine@ExternalToolLogParser@U2@@MAEXABVQString@@@Z 100199c6 f   U2Core:U2Core.dll
 0001:000189cc       ?propagateSubtaskError@Task@U2@@UAE_NXZ 100199cc f   U2Core:U2Core.dll
 0001:000189d2       ?qt_metacall@ExternalToolLogParser@U2@@UAEHW4Call@QMetaObject@@HPAPAX@Z 100199d2 f   U2Core:U2Core.dll
 0001:000189d8       ?qt_metacall@ExternalToolRunTask@U2@@UAEHW4Call@QMetaObject@@HPAPAX@Z 100199d8 f   U2Core:U2Core.dll
 0001:000189de       ?qt_metacast@ExternalToolLogParser@U2@@UAEPAXPBD@Z 100199de f   U2Core:U2Core.dll
 0001:000189e4       ?qt_metacast@ExternalToolRunTask@U2@@UAEPAXPBD@Z 100199e4 f   U2Core:U2Core.dll
 0001:000189ea       ?report@Task@U2@@UAE?AW4ReportResult@12@XZ 100199ea f   U2Core:U2Core.dll
 0001:000189f0       ?run@ExternalToolRunTask@U2@@UAEXXZ 100199f0 f   U2Core:U2Core.dll
 0001:000189f6       ?run@Task@U2@@UAEXXZ       100199f6 f   U2Core:U2Core.dll
 0001:000189fc       ?setCollectChildrensWarningsFlag@Task@U2@@UAEX_N@Z 100199fc f   U2Core:U2Core.dll
 0001:00018a02       ?setLastError@ExternalToolLogParser@U2@@MAEXABVQString@@@Z 10019a02 f   U2Core:U2Core.dll
 0001:00018a08       ?setListenerForHelper@ExternalToolSupportTask@U2@@MAEXPAVExternalToolRunTaskHelper@2@H@Z 10019a08 f   U2Core:U2Core.dll
 0001:00018a0e       ?setListenerForTask@ExternalToolSupportTask@U2@@MAEXPAVExternalToolRunTask@2@H@Z 10019a0e f   U2Core:U2Core.dll
 0001:00018a14       ?setNoAutoDelete@Task@U2@@UAEX_N@Z 10019a14 f   U2Core:U2Core.dll
 0001:00018a1a       ?setNotificationReport@Task@U2@@UAEX_N@Z 10019a1a f   U2Core:U2Core.dll
 0001:00018a20       ?setReportingEnabled@Task@U2@@UAEX_N@Z 10019a20 f   U2Core:U2Core.dll
 0001:00018a26       ?setReportingSupported@Task@U2@@UAEX_N@Z 10019a26 f   U2Core:U2Core.dll
 0001:00018a2c       ?getDataPathRegistry@AppContext@U2@@SAPAVU2DataPathRegistry@2@XZ 10019a2c f   U2Core:U2Core.dll
 0001:00018a32       ?isValid@U2DataPath@U2@@QBE_NXZ 10019a32 f   U2Core:U2Core.dll
 0001:00018a38       ?getPathByName@U2DataPath@U2@@QBE?AVQString@@ABV3@@Z 10019a38 f   U2Core:U2Core.dll
 0001:00018a3e       ?getDataPathByName@U2DataPathRegistry@U2@@QAEPAVU2DataPath@2@ABVQString@@@Z 10019a3e f   U2Core:U2Core.dll
 0001:00018a44       ?error@Logger@U2@@QAEXABVQString@@@Z 10019a44 f   U2Core:U2Core.dll
 0001:00018a4a       ?isCoR@U2OpStatus@U2@@UBE_NXZ 10019a4a f   U2Core:U2Core.dll
 0001:00018a50       ??0TaskStateInfo@U2@@QAE@XZ 10019a50 f   U2Core:U2Core.dll
 0001:00018a56       ?getError@TaskStateInfo@U2@@UBE?AVQString@@XZ 10019a56 f   U2Core:U2Core.dll
 0001:00018a5c       ?setError@TaskStateInfo@U2@@UAEXABVQString@@@Z 10019a5c f   U2Core:U2Core.dll
 0001:00018a62       ??1TaskStateInfo@U2@@UAE@XZ 10019a62 f   U2Core:U2Core.dll
 0001:00018a68       ?hasError@Task@U2@@QBE_NXZ 10019a68 f   U2Core:U2Core.dll
 0001:00018a6e       ??0FailTask@U2@@QAE@ABVQString@@@Z 10019a6e f   U2Core:U2Core.dll
 0001:00018a74       ??1FailTask@U2@@UAE@XZ     10019a74 f   U2Core:U2Core.dll
 0001:00018a7a       ??0GUrl@U2@@QAE@ABVQString@@@Z 10019a7a f   U2Core:U2Core.dll
 0001:00018a80       ??1GUrl@U2@@QAE@XZ         10019a80 f   U2Core:U2Core.dll
 0001:00018a86       ?createWorkingDir@FileAndDirectoryUtils@U2@@SA?AVQString@@ABV3@H00@Z 10019a86 f   U2Core:U2Core.dll
 0001:00018a8c       ?ensureFileExt@GUrlUtils@U2@@SA?AVGUrl@2@ABV32@ABVQStringList@@@Z 10019a8c f   U2Core:U2Core.dll
 0001:00018a92       ?rollFileName@GUrlUtils@U2@@SA?AVQString@@ABV3@0ABV?$QSet@VQString@@@@@Z 10019a92 f   U2Core:U2Core.dll
 0001:00018a98       ?createDirectory@GUrlUtils@U2@@SA?AVQString@@ABV3@0AAVU2OpStatus@2@@Z 10019a98 f   U2Core:U2Core.dll
 0001:00018a9e       ??0TaskSignalMapper@U2@@QAE@PAVTask@1@@Z 10019a9e f   U2Core:U2Core.dll
 0001:00018aa4       ?getError@U2OpStatusImpl@U2@@UBE?AVQString@@XZ 10019aa4 f   U2Core:U2Core.dll
 0001:00018aaa       ??0U2OpStatus2Log@U2@@QAE@W4LogLevel@1@@Z 10019aaa f   U2Core:U2Core.dll
 0001:00018ab0       ??1U2OpStatus2Log@U2@@UAE@XZ 10019ab0 f   U2Core:U2Core.dll
 0001:00018ab6       ?addListeners@ExternalToolSupportTask@U2@@QAEXABV?$QList@PAVExternalToolListener@U2@@@@@Z 10019ab6 f   U2Core:U2Core.dll
 0001:00018abc       ?runScript@ScriptTask@U2@@SA?AVQScriptValue@@PAVQScriptEngine@@ABV?$QMap@VQString@@VQScriptValue@@@@ABVQString@@AAVTaskStateInfo@2@@Z 10019abc f   U2Core:U2Core.dll
 0001:00018ac2       ?metaObject@FailTask@U2@@UBEPBUQMetaObject@@XZ 10019ac2 f   U2Core:U2Core.dll
 0001:00018ac8       ?metaObject@TaskSignalMapper@U2@@UBEPBUQMetaObject@@XZ 10019ac8 f   U2Core:U2Core.dll
 0001:00018ace       ?qt_metacall@FailTask@U2@@UAEHW4Call@QMetaObject@@HPAPAX@Z 10019ace f   U2Core:U2Core.dll
 0001:00018ad4       ?qt_metacall@TaskSignalMapper@U2@@UAEHW4Call@QMetaObject@@HPAPAX@Z 10019ad4 f   U2Core:U2Core.dll
 0001:00018ada       ?qt_metacast@FailTask@U2@@UAEPAXPBD@Z 10019ada f   U2Core:U2Core.dll
 0001:00018ae0       ?qt_metacast@TaskSignalMapper@U2@@UAEPAXPBD@Z 10019ae0 f   U2Core:U2Core.dll
 0001:00018ae6       ?getDNATranslationRegistry@AppContext@U2@@SAPAVDNATranslationRegistry@2@XZ 10019ae6 f   U2Core:U2Core.dll
 0001:00018aec       ?lookupTranslation@DNATranslationRegistry@U2@@QAEPAVDNATranslation@2@ABVQString@@@Z 10019aec f   U2Core:U2Core.dll
 0001:00018af2       ?trace@Logger@U2@@QAEXABVQString@@@Z 10019af2 f   U2Core:U2Core.dll
 0001:00018af8       ?info@Logger@U2@@QAEXABVQString@@@Z 10019af8 f   U2Core:U2Core.dll
 0001:00018afe       ?getAppSettings@AppContext@U2@@SAPAVAppSettings@2@XZ 10019afe f   U2Core:U2Core.dll
 0001:00018b04       ?getDNAAlphabetRegistry@AppContext@U2@@SAPAVDNAAlphabetRegistry@2@XZ 10019b04 f   U2Core:U2Core.dll
 0001:00018b0a       ?NUCL_DNA_DEFAULT@BaseDNAAlphabetIds@U2@@SA?BVQString@@XZ 10019b0a f   U2Core:U2Core.dll
 0001:00018b10       ?lookupTranslation@DNATranslationRegistry@U2@@QAE?AV?$QList@PAVDNATranslation@U2@@@@PBVDNAAlphabet@2@W4DNATranslationType@2@@Z 10019b10 f   U2Core:U2Core.dll
 0001:00018b16       ??0ExternalTool@U2@@QAE@VQString@@0@Z 10019b16 f   U2Core:U2Core.dll
 0001:00018b1c       ??1ExternalTool@U2@@UAE@XZ 10019b1c f   U2Core:U2Core.dll
 0001:00018b22       ?getAdditionalParameters@ExternalTool@U2@@UAEXABVQString@@@Z 10019b22 f   U2Core:U2Core.dll
 0001:00018b28       ?getAdditionalPaths@ExternalTool@U2@@UBE?AVQStringList@@XZ 10019b28 f   U2Core:U2Core.dll
 0001:00018b2e       ?getToolRunnerAdditionalOptions@ExternalTool@U2@@UAE?BVQStringList@@XZ 10019b2e f   U2Core:U2Core.dll
 0001:00018b34       ?performAdditionalChecks@ExternalTool@U2@@UAEXABVQString@@@Z 10019b34 f   U2Core:U2Core.dll
 0001:00018b3a       ?getExternalToolRegistry@AppContext@U2@@SAPAVExternalToolRegistry@2@XZ 10019b3a f   U2Core:U2Core.dll
 0001:00018b40       ?registerEntry@ExternalToolRegistry@U2@@QAE_NPAVExternalTool@2@@Z 10019b40 f   U2Core:U2Core.dll
 0001:00018b46       ?unregisterEntry@ExternalToolRegistry@U2@@QAEXABVQString@@@Z 10019b46 f   U2Core:U2Core.dll
 0001:00018b4c       ??0Plugin@U2@@QAE@ABVQString@@0_NW4PluginState@1@@Z 10019b4c f   U2Core:U2Core.dll
 0001:00018b52       ??1Plugin@U2@@UAE@XZ       10019b52 f   U2Core:U2Core.dll
 0001:00018b58       ?errorOpeningFileWrite@L10N@U2@@SA?AVQString@@ABVGUrl@2@@Z 10019b58 f   U2Core:U2Core.dll
 0001:00018b5e       ?errorWritingFile@L10N@U2@@SA?AVQString@@ABVGUrl@2@@Z 10019b5e f   U2Core:U2Core.dll
 0001:00018b64       ??0Task@U2@@QAE@ABVQString@@V?$QFlags@W4TaskFlag@U2@@@@@Z 10019b64 f   U2Core:U2Core.dll
 0001:00018b6a       ??1Task@U2@@UAE@XZ         10019b6a f   U2Core:U2Core.dll
 0001:00018b70       ?qt_metacast@Task@U2@@UAEPAXPBD@Z 10019b70 f   U2Core:U2Core.dll
 0001:00018b76       ?qt_metacall@Task@U2@@UAEHW4Call@QMetaObject@@HPAPAX@Z 10019b76 f   U2Core:U2Core.dll
 0001:00018b7c       ?qt_metacast@ExternalTool@U2@@UAEPAXPBD@Z 10019b7c f   U2Core:U2Core.dll
 0001:00018b82       ?qt_metacall@ExternalTool@U2@@UAEHW4Call@QMetaObject@@HPAPAX@Z 10019b82 f   U2Core:U2Core.dll
 0001:00018b88       ?qt_metacast@Plugin@U2@@UAEPAXPBD@Z 10019b88 f   U2Core:U2Core.dll
 0001:00018b8e       ?qt_metacall@Plugin@U2@@UAEHW4Call@QMetaObject@@HPAPAX@Z 10019b8e f   U2Core:U2Core.dll
 0001:00018b94       ??0StreamSequenceReader@U2@@QAE@XZ 10019b94 f   U2Formats:U2Formats.dll
 0001:00018b9a       ??1StreamSequenceReader@U2@@UAE@XZ 10019b9a f   U2Formats:U2Formats.dll
 0001:00018ba0       ?init@StreamSequenceReader@U2@@QAE_NABVQStringList@@@Z 10019ba0 f   U2Formats:U2Formats.dll
 0001:00018ba6       ?hasNext@StreamSequenceReader@U2@@QAE_NXZ 10019ba6 f   U2Formats:U2Formats.dll
 0001:00018bac       ?getErrorMessage@StreamSequenceReader@U2@@QAE?AVQString@@XZ 10019bac f   U2Formats:U2Formats.dll
 0001:00018bb2       ?getNextSequenceObject@StreamSequenceReader@U2@@QAEPAVDNASequence@2@XZ 10019bb2 f   U2Formats:U2Formats.dll
 0001:00018bb8       ??1StreamShortReadWriter@U2@@UAE@XZ 10019bb8 f   U2Formats:U2Formats.dll
 0001:00018bbe       ?init@StreamShortReadWriter@U2@@QAE_NABVGUrl@2@@Z 10019bbe f   U2Formats:U2Formats.dll
 0001:00018bc4       ?writeNextSequence@StreamShortReadWriter@U2@@QAE_NABVDNASequence@2@@Z 10019bc4 f   U2Formats:U2Formats.dll
 0001:00018bca       ??0StreamGzippedShortReadWriter@U2@@QAE@XZ 10019bca f   U2Formats:U2Formats.dll
 0001:00018bd0       ??1StreamGzippedShortReadWriter@U2@@UAE@XZ 10019bd0 f   U2Formats:U2Formats.dll
 0001:00018bd6       ?prepareFileFilter@DialogUtils@U2@@SA?AVQString@@ABV3@ABVQStringList@@_N1@Z 10019bd6 f   U2Gui:U2Gui.dll
 0001:00018bdc       ?prepareDocumentsFileFilter@DialogUtils@U2@@SA?AVQString@@ABV3@_NABVQStringList@@@Z 10019bdc f   U2Gui:U2Gui.dll
 0001:00018be2       ?getInputPorts@Actor@Workflow@U2@@QBE?AV?$QList@PAVPort@Workflow@U2@@@@XZ 10019be2 f   U2Lang:U2Lang.dll
 0001:00018be8       ?getOutputPorts@Actor@Workflow@U2@@QBE?AV?$QList@PAVPort@Workflow@U2@@@@XZ 10019be8 f   U2Lang:U2Lang.dll
 0001:00018bee       ??0PrompterBaseImpl@U2@@QAE@PAVActor@Workflow@1@@Z 10019bee f   U2Lang:U2Lang.dll
 0001:00018bf4       ?getURL@PrompterBaseImpl@U2@@QAE?AVQString@@ABV3@PA_N00@Z 10019bf4 f   U2Lang:U2Lang.dll
 0001:00018bfa       ?getHyperlink@PrompterBaseImpl@U2@@SA?AVQString@@ABV3@0@Z 10019bfa f   U2Lang:U2Lang.dll
 0001:00018c00       ??1PrompterBaseImpl@U2@@UAE@XZ 10019c00 f   U2Lang:U2Lang.dll
 0001:00018c06       ?metaObject@PrompterBaseImpl@U2@@UBEPBUQMetaObject@@XZ 10019c06 f   U2Lang:U2Lang.dll
 0001:00018c0c       ?qt_metacall@PrompterBaseImpl@U2@@UAEHW4Call@QMetaObject@@HPAPAX@Z 10019c0c f   U2Lang:U2Lang.dll
 0001:00018c12       ?qt_metacast@PrompterBaseImpl@U2@@UAEPAXPBD@Z 10019c12 f   U2Lang:U2Lang.dll
 0001:00018c18       ?sl_actorModified@PrompterBaseImpl@U2@@MAEXXZ 10019c18 f   U2Lang:U2Lang.dll
 0001:00018c1e       ?update@PrompterBaseImpl@U2@@UAEXABV?$QMap@VQString@@VQVariant@@@@@Z 10019c1e f   U2Lang:U2Lang.dll
 0001:00018c24       ??0WorkflowNotification@U2@@QAE@ABVQString@@00@Z 10019c24 f   U2Lang:U2Lang.dll
 0001:00018c2a       ??1WorkflowNotification@U2@@QAE@XZ 10019c2a f   U2Lang:U2Lang.dll
 0001:00018c30       ??0WorkflowNotification@U2@@QAE@ABV01@@Z 10019c30 f   U2Lang:U2Lang.dll
 0001:00018c36       ?getId@Actor@Workflow@U2@@QBE?AVQString@@XZ 10019c36 f   U2Lang:U2Lang.dll
 0001:00018c3c       ??1Descriptor@U2@@UAE@XZ   10019c3c f   U2Lang:U2Lang.dll
 0001:00018c42       ?getId@Descriptor@U2@@QBE?AVQString@@XZ 10019c42 f   U2Lang:U2Lang.dll
 0001:00018c48       ??0Descriptor@U2@@QAE@ABV01@@Z 10019c48 f   U2Lang:U2Lang.dll
 0001:00018c4e       ?URL_SLOT@BaseSlots@Workflow@U2@@SA?BVDescriptor@3@XZ 10019c4e f   U2Lang:U2Lang.dll
 0001:00018c54       ??0Dataset@U2@@QAE@ABV01@@Z 10019c54 f   U2Lang:U2Lang.dll
 0001:00018c5a       ??1Dataset@U2@@QAE@XZ      10019c5a f   U2Lang:U2Lang.dll
 0001:00018c60       ?getUrls@Dataset@U2@@QBE?AV?$QList@PAVURLContainer@U2@@@@XZ 10019c60 f   U2Lang:U2Lang.dll
 0001:00018c66       ?initEngine@WorkflowScriptLibrary@U2@@SAXPAVWorkflowScriptEngine@2@@Z 10019c66 f   U2Lang:U2Lang.dll
 0001:00018c6c       ??0MessageMetadata@U2@@QAE@ABVQString@@@Z 10019c6c f   U2Lang:U2Lang.dll
 0001:00018c72       ?getId@MessageMetadata@U2@@QBEHXZ 10019c72 f   U2Lang:U2Lang.dll
 0001:00018c78       ??1MessageMetadata@U2@@QAE@XZ 10019c78 f   U2Lang:U2Lang.dll
 0001:00018c7e       ?put@MessageMetadataStorage@U2@@QAEXABVMessageMetadata@2@@Z 10019c7e f   U2Lang:U2Lang.dll
 0001:00018c84       ?getMonitor@WorkflowContext@Workflow@U2@@QAEPAVWorkflowMonitor@23@XZ 10019c84 f   U2Lang:U2Lang.dll
 0001:00018c8a       ?workingDir@WorkflowContext@Workflow@U2@@QBE?AVQString@@XZ 10019c8a f   U2Lang:U2Lang.dll
 0001:00018c90       ?absolutePath@WorkflowContext@Workflow@U2@@QBE?AVQString@@ABV4@@Z 10019c90 f   U2Lang:U2Lang.dll
 0001:00018c96       ?getMetadataStorage@WorkflowContext@Workflow@U2@@QAEAAVMessageMetadataStorage@3@XZ 10019c96 f   U2Lang:U2Lang.dll
 0001:00018c9c       ??0WorkflowScriptEngine@U2@@QAE@PAVWorkflowContext@Workflow@1@@Z 10019c9c f   U2Lang:U2Lang.dll
 0001:00018ca2       ??1WorkflowScriptEngine@U2@@UAE@XZ 10019ca2 f   U2Lang:U2Lang.dll
 0001:00018ca8       ?isEmpty@AttributeScript@U2@@QBE_NXZ 10019ca8 f   U2Lang:U2Lang.dll
 0001:00018cae       ?getScriptText@AttributeScript@U2@@QBEABVQString@@XZ 10019cae f   U2Lang:U2Lang.dll
 0001:00018cb4       ?getScriptVars@AttributeScript@U2@@QBEABV?$QMap@VDescriptor@U2@@VQVariant@@@@XZ 10019cb4 f   U2Lang:U2Lang.dll
 0001:00018cba       ??0Message@Workflow@U2@@QAE@V?$QExplicitlySharedDataPointer@VDataType@U2@@@@ABVQVariant@@H@Z 10019cba f   U2Lang:U2Lang.dll
 0001:00018cc0       ??1Message@Workflow@U2@@QAE@XZ 10019cc0 f   U2Lang:U2Lang.dll
 0001:00018cc6       ?addOutputFile@WorkflowMonitor@Workflow@U2@@QAEXABVQString@@0_N@Z 10019cc6 f   U2Lang:U2Lang.dll
 0001:00018ccc       ?isOutUrlAttribute@RFSUtils@U2@@SA_NPAVAttribute@2@PAVActor@Workflow@2@AA_N@Z 10019ccc f   U2Lang:U2Lang.dll
 0001:00018cd2       ?getBusType@IntegralBus@Workflow@U2@@QBE?AV?$QExplicitlySharedDataPointer@VDataType@U2@@@@XZ 10019cd2 f   U2Lang:U2Lang.dll
 0001:00018cd8       ??0BaseWorker@LocalWorkflow@U2@@QAE@PAVActor@Workflow@2@_N@Z 10019cd8 f   U2Lang:U2Lang.dll
 0001:00018cde       ??1BaseWorker@LocalWorkflow@U2@@UAE@XZ 10019cde f   U2Lang:U2Lang.dll
 0001:00018ce4       ?createLogListeners@BaseWorker@LocalWorkflow@U2@@QAE?AV?$QList@PAVExternalToolListener@U2@@@@H@Z 10019ce4 f   U2Lang:U2Lang.dll
 0001:00018cea       ?addCommunication@BaseWorker@LocalWorkflow@U2@@UAE_NABVQString@@PAVCommunicationChannel@Workflow@3@@Z 10019cea f   U2Lang:U2Lang.dll
 0001:00018cf0       ?canTaskBeCanceled@BaseWorker@LocalWorkflow@U2@@MBE_NPAVTask@3@@Z 10019cf0 f   U2Lang:U2Lang.dll
 0001:00018cf6       ?getActorId@BaseWorker@LocalWorkflow@U2@@UBE?AVQString@@XZ 10019cf6 f   U2Lang:U2Lang.dll
 0001:00018cfc       ?getCommunication@BaseWorker@LocalWorkflow@U2@@UAEPAVCommunicationChannel@Workflow@3@ABVQString@@@Z 10019cfc f   U2Lang:U2Lang.dll
 0001:00018d02       ?getMessageAndSetupScriptValues@BaseWorker@LocalWorkflow@U2@@UAE?AVMessage@Workflow@3@PAVCommunicationChannel@53@@Z 10019d02 f   U2Lang:U2Lang.dll
 0001:00018d08       ?getOutputFiles@BaseWorker@LocalWorkflow@U2@@UAE?AVQStringList@@XZ 10019d08 f   U2Lang:U2Lang.dll
 0001:00018d0e       ?isDone@BaseWorker@LocalWorkflow@U2@@UBE_NXZ 10019d0e f   U2Lang:U2Lang.dll
 0001:00018d14       ?isReady@BaseWorker@LocalWorkflow@U2@@UBE_NXZ 10019d14 f   U2Lang:U2Lang.dll
 0001:00018d1a       ?setDone@BaseWorker@LocalWorkflow@U2@@UAEXXZ 10019d1a f   U2Lang:U2Lang.dll
 0001:00018d20       ??0Descriptor@U2@@QAE@ABVQString@@00@Z 10019d20 f   U2Lang:U2Lang.dll
 0001:00018d26       ??0Descriptor@U2@@QAE@ABVQString@@@Z 10019d26 f   U2Lang:U2Lang.dll
 0001:00018d2c       ??0MapDataType@U2@@QAE@ABVDescriptor@1@ABV?$QMap@VDescriptor@U2@@V?$QExplicitlySharedDataPointer@VDataType@U2@@@@@@@Z 10019d2c f   U2Lang:U2Lang.dll
 0001:00018d32       ??1MapDataType@U2@@UAE@XZ  10019d32 f   U2Lang:U2Lang.dll
 0001:00018d38       ??0Attribute@U2@@QAE@ABVDescriptor@1@V?$QExplicitlySharedDataPointer@VDataType@U2@@@@_NABVQVariant@@@Z 10019d38 f   U2Lang:U2Lang.dll
 0001:00018d3e       ??1Attribute@U2@@UAE@XZ    10019d3e f   U2Lang:U2Lang.dll
 0001:00018d44       ??1PropertyDelegate@U2@@UAE@XZ 10019d44 f   U2Lang:U2Lang.dll
 0001:00018d4a       ??0DelegateTags@U2@@QAE@PAVQObject@@@Z 10019d4a f   U2Lang:U2Lang.dll
 0001:00018d50       ?set@DelegateTags@U2@@QAEXABVQString@@ABVQVariant@@@Z 10019d50 f   U2Lang:U2Lang.dll
 0001:00018d56       ??1DelegateTags@U2@@UAE@XZ 10019d56 f   U2Lang:U2Lang.dll
 0001:00018d5c       ??0PortDescriptor@Workflow@U2@@QAE@ABVDescriptor@2@V?$QExplicitlySharedDataPointer@VDataType@U2@@@@_N2I@Z 10019d5c f   U2Lang:U2Lang.dll
 0001:00018d62       ??1PortDescriptor@Workflow@U2@@UAE@XZ 10019d62 f   U2Lang:U2Lang.dll
 0001:00018d68       ??0ActorPrototype@Workflow@U2@@QAE@ABVDescriptor@2@ABV?$QList@PAVPortDescriptor@Workflow@U2@@@@ABV?$QList@PAVAttribute@U2@@@@@Z 10019d68 f   U2Lang:U2Lang.dll
 0001:00018d6e       ??1ActorPrototype@Workflow@U2@@UAE@XZ 10019d6e f   U2Lang:U2Lang.dll
 0001:00018d74       ?setEditor@ActorPrototype@Workflow@U2@@QAEXPAVConfigurationEditor@3@@Z 10019d74 f   U2Lang:U2Lang.dll
 0001:00018d7a       ?setValidator@ActorPrototype@Workflow@U2@@QAEXPAVConfigurationValidator@3@@Z 10019d7a f   U2Lang:U2Lang.dll
 0001:00018d80       ?setPrompter@ActorPrototype@Workflow@U2@@QAEXPAVPrompter@23@@Z 10019d80 f   U2Lang:U2Lang.dll
 0001:00018d86       ?addExternalTool@ActorPrototype@Workflow@U2@@QAEXABVQString@@0@Z 10019d86 f   U2Lang:U2Lang.dll
 0001:00018d8c       ?registerProto@ActorPrototypeRegistry@Workflow@U2@@QAEXABVDescriptor@3@PAVActorPrototype@23@@Z 10019d8c f   U2Lang:U2Lang.dll
 0001:00018d92       ?unregisterProto@ActorPrototypeRegistry@Workflow@U2@@QAEPAVActorPrototype@23@ABVQString@@@Z 10019d92 f   U2Lang:U2Lang.dll
 0001:00018d98       ?STRING_TYPE@BaseTypes@U2@@SA?AV?$QExplicitlySharedDataPointer@VDataType@U2@@@@XZ 10019d98 f   U2Lang:U2Lang.dll
 0001:00018d9e       ?URL_DATASETS_TYPE@BaseTypes@U2@@SA?AV?$QExplicitlySharedDataPointer@VDataType@U2@@@@XZ 10019d9e f   U2Lang:U2Lang.dll
 0001:00018da4       ?getInstance@WorkflowEnv@Workflow@U2@@KAPAV123@XZ 10019da4 f   U2Lang:U2Lang.dll
 0001:00018daa       ??0DomainFactory@Workflow@U2@@QAE@ABVQString@@@Z 10019daa f   U2Lang:U2Lang.dll
 0001:00018db0       ??1DomainFactory@Workflow@U2@@UAE@XZ 10019db0 f   U2Lang:U2Lang.dll
 0001:00018db6       ?clone@Attribute@U2@@UAEPAV12@XZ 10019db6 f   U2Lang:U2Lang.dll
 0001:00018dbc       ?createConnection@DomainFactory@Workflow@U2@@UAEPAVCommunicationChannel@23@PAVLink@23@@Z 10019dbc f   U2Lang:U2Lang.dll
 0001:00018dc2       ?createInstance@ActorPrototype@Workflow@U2@@UAEPAVActor@23@ABVQString@@PAVAttributeScript@3@ABV?$QMap@VQString@@VQVariant@@@@@Z 10019dc2 f   U2Lang:U2Lang.dll
 0001:00018dc8       ?createPort@IntegralBusActorPrototype@Workflow@U2@@UAEPAVPort@23@ABVPortDescriptor@23@PAVActor@23@@Z 10019dc8 f   U2Lang:U2Lang.dll
 0001:00018dce       ?createScheduler@DomainFactory@Workflow@U2@@UAEPAVScheduler@23@PAVSchema@23@@Z 10019dce f   U2Lang:U2Lang.dll
 0001:00018dd4       ?destroy@DomainFactory@Workflow@U2@@UAEXPAVScheduler@23@PAVSchema@23@@Z 10019dd4 f   U2Lang:U2Lang.dll
 0001:00018dda       ?getAllDescriptors@MapDataType@U2@@UBE?AV?$QList@VDescriptor@U2@@@@XZ 10019dda f   U2Lang:U2Lang.dll
 0001:00018de0       ?getAllEntries@?$IdRegistry@VDomainFactory@Workflow@U2@@@U2@@UBE?AV?$QList@PAVDomainFactory@Workflow@U2@@@@XZ 10019de0 f   U2Lang:U2Lang.dll
 0001:00018de6       ?getAllIds@?$IdRegistry@VDomainFactory@Workflow@U2@@@U2@@UBE?AV?$QList@VQString@@@@XZ 10019de6 f   U2Lang:U2Lang.dll
 0001:00018dec       ?getAttributePureValue@Attribute@U2@@UBEABVQVariant@@XZ 10019dec f   U2Lang:U2Lang.dll
 0001:00018df2       ?getById@?$IdRegistry@VDomainFactory@Workflow@U2@@@U2@@UAEPAVDomainFactory@Workflow@2@ABVQString@@@Z 10019df2 f   U2Lang:U2Lang.dll
 0001:00018df8       ?getDatatypeByDescriptor@MapDataType@U2@@UBE?AV?$QExplicitlySharedDataPointer@VDataType@U2@@@@ABVDescriptor@2@@Z 10019df8 f   U2Lang:U2Lang.dll
 0001:00018dfe       ?getDatatypesMap@MapDataType@U2@@UBE?AV?$QMap@VDescriptor@U2@@V?$QExplicitlySharedDataPointer@VDataType@U2@@@@@@XZ 10019dfe f   U2Lang:U2Lang.dll
 0001:00018e04       ?getDefaultPureValue@Attribute@U2@@UBEABVQVariant@@XZ 10019e04 f   U2Lang:U2Lang.dll
 0001:00018e0a       ?getGroup@Attribute@U2@@UAE?AW4AttributeGroup@2@XZ 10019e0a f   U2Lang:U2Lang.dll
 0001:00018e10       ?getItems@PropertyDelegate@U2@@UBEXAAV?$QMap@VQString@@VQVariant@@@@@Z 10019e10 f   U2Lang:U2Lang.dll
 0001:00018e16       ?getType@PortDescriptor@Workflow@U2@@UBE?AV?$QExplicitlySharedDataPointer@VDataType@U2@@@@XZ 10019e16 f   U2Lang:U2Lang.dll
 0001:00018e1c       ?getWidget@ConfigurationEditor@U2@@UAEPAVQWidget@@XZ 10019e1c f   U2Lang:U2Lang.dll
 0001:00018e22       ?isAcceptableDrop@ActorPrototype@Workflow@U2@@UBE_NPBVQMimeData@@PAV?$QMap@VQString@@VQVariant@@@@@Z 10019e22 f   U2Lang:U2Lang.dll
 0001:00018e28       ?isDefaultValue@Attribute@U2@@UBE_NXZ 10019e28 f   U2Lang:U2Lang.dll
 0001:00018e2e       ?isEmpty@Attribute@U2@@UBE_NXZ 10019e2e f   U2Lang:U2Lang.dll
 0001:00018e34       ?isEmpty@ConfigurationEditor@U2@@UBE_NXZ 10019e34 f   U2Lang:U2Lang.dll
 0001:00018e3a       ?kind@MapDataType@U2@@UBE?AW4Kind@DataType@2@XZ 10019e3a f   U2Lang:U2Lang.dll
 0001:00018e40       ?registerEntry@?$IdRegistry@VDomainFactory@Workflow@U2@@@U2@@UAE_NPAVDomainFactory@Workflow@2@@Z 10019e40 f   U2Lang:U2Lang.dll
 0001:00018e46       ?setAttributeValue@Attribute@U2@@UAEXABVQVariant@@@Z 10019e46 f   U2Lang:U2Lang.dll
 0001:00018e4c       ?setVisibleSlot@PortDescriptor@Workflow@U2@@UAEXABVQString@@_N@Z 10019e4c f   U2Lang:U2Lang.dll
 0001:00018e52       ?type@PropertyDelegate@U2@@UBE?AW4Type@12@XZ 10019e52 f   U2Lang:U2Lang.dll
 0001:00018e58       ?unregisterEntry@?$IdRegistry@VDomainFactory@Workflow@U2@@@U2@@UAEPAVDomainFactory@Workflow@2@ABVQString@@@Z 10019e58 f   U2Lang:U2Lang.dll
 0001:00018e5e       ?update@PropertyDelegate@U2@@UAEXXZ 10019e5e f   U2Lang:U2Lang.dll
 0001:00018e64       ?updateActorIds@Attribute@U2@@UAEXABV?$QMap@VQString@@V1@@@@Z 10019e64 f   U2Lang:U2Lang.dll
 0001:00018e6a       ?validate@ActorValidator@Workflow@U2@@UBE_NPBVConfiguration@3@AAV?$QList@VWorkflowNotification@U2@@@@@Z 10019e6a f   U2Lang:U2Lang.dll
 0001:00018e70       ?validate@Attribute@U2@@UAE_NAAV?$QList@VWorkflowNotification@U2@@@@@Z 10019e70 f   U2Lang:U2Lang.dll
 0001:00018e76       ?getProducersOrUnset@PrompterBaseImpl@U2@@QAE?AVQString@@ABV3@0@Z 10019e76 f   U2Lang:U2Lang.dll
 0001:00018e7c       ?getFileUrl@MessageMetadata@U2@@QBEABVQString@@XZ 10019e7c f   U2Lang:U2Lang.dll
 0001:00018e82       ?get@MessageMetadataStorage@U2@@QBE?AVMessageMetadata@2@H@Z 10019e82 f   U2Lang:U2Lang.dll
 0001:00018e88       ?getData@Message@Workflow@U2@@QBE?AVQVariant@@XZ 10019e88 f   U2Lang:U2Lang.dll
 0001:00018e8e       ?getMetadataId@Message@Workflow@U2@@QBEHXZ 10019e8e f   U2Lang:U2Lang.dll
 0001:00018e94       ?addInfo@WorkflowMonitor@Workflow@U2@@QAEXABVQString@@00@Z 10019e94 f   U2Lang:U2Lang.dll
 0001:00018e9a       ??0Attribute@U2@@QAE@ABVDescriptor@1@V?$QExplicitlySharedDataPointer@VDataType@U2@@@@V?$QFlags@W4Flag@Attribute@U2@@@@ABVQVariant@@@Z 10019e9a f   U2Lang:U2Lang.dll
 0001:00018ea0       ?NUM_TYPE@BaseTypes@U2@@SA?AV?$QExplicitlySharedDataPointer@VDataType@U2@@@@XZ 10019ea0 f   U2Lang:U2Lang.dll
 0001:00018ea6       ?qt_metacast@BaseWorker@LocalWorkflow@U2@@UAEPAXPBD@Z 10019ea6 f   U2Lang:U2Lang.dll
 0001:00018eac       ?qt_metacall@BaseWorker@LocalWorkflow@U2@@UAEHW4Call@QMetaObject@@HPAPAX@Z 10019eac f   U2Lang:U2Lang.dll
 0001:00018eb2       ??0DelegateEditor@U2@@QAE@ABV?$QMap@VQString@@PAVPropertyDelegate@U2@@@@@Z 10019eb2 f   U2Designer:U2Designer.dll
 0001:00018eb8       ??1DelegateEditor@U2@@UAE@XZ 10019eb8 f   U2Designer:U2Designer.dll
 0001:00018ebe       ??0URLDelegate@U2@@QAE@ABVDelegateTags@1@ABVQString@@ABV?$QFlags@W4Option@URLDelegate@U2@@@@PAVQObject@@@Z 10019ebe f   U2Designer:U2Designer.dll
 0001:00018ec4       ??1URLDelegate@U2@@UAE@XZ  10019ec4 f   U2Designer:U2Designer.dll
 0001:00018eca       ?addDelegate@DelegateEditor@U2@@UAEXPAVPropertyDelegate@2@ABVQString@@@Z 10019eca f   U2Designer:U2Designer.dll
 0001:00018ed0       ?clone@DelegateEditor@U2@@UAEPAVConfigurationEditor@2@XZ 10019ed0 f   U2Designer:U2Designer.dll
 0001:00018ed6       ?clone@URLDelegate@U2@@UAEPAVPropertyDelegate@2@XZ 10019ed6 f   U2Designer:U2Designer.dll
 0001:00018edc       ?commit@DelegateEditor@U2@@UAEXXZ 10019edc f   U2Designer:U2Designer.dll
 0001:00018ee2       ?createEditor@URLDelegate@U2@@UBEPAVQWidget@@PAV3@ABVQStyleOptionViewItem@@ABVQModelIndex@@@Z 10019ee2 f   U2Designer:U2Designer.dll
 0001:00018ee8       ?createWizardWidget@URLDelegate@U2@@UBEPAVPropertyWidget@2@AAVU2OpStatus@2@PAVQWidget@@@Z 10019ee8 f   U2Designer:U2Designer.dll
 0001:00018eee       ?getDelegate@DelegateEditor@U2@@UAEPAVPropertyDelegate@2@ABVQString@@@Z 10019eee f   U2Designer:U2Designer.dll
 0001:00018ef4       ?getDisplayValue@URLDelegate@U2@@UBE?AVQVariant@@ABV3@@Z 10019ef4 f   U2Designer:U2Designer.dll
 0001:00018efa       ?metaObject@DelegateEditor@U2@@UBEPBUQMetaObject@@XZ 10019efa f   U2Designer:U2Designer.dll
 0001:00018f00       ?metaObject@URLDelegate@U2@@UBEPBUQMetaObject@@XZ 10019f00 f   U2Designer:U2Designer.dll
 0001:00018f06       ?qt_metacall@DelegateEditor@U2@@UAEHW4Call@QMetaObject@@HPAPAX@Z 10019f06 f   U2Designer:U2Designer.dll
 0001:00018f0c       ?qt_metacall@URLDelegate@U2@@UAEHW4Call@QMetaObject@@HPAPAX@Z 10019f0c f   U2Designer:U2Designer.dll
 0001:00018f12       ?qt_metacast@DelegateEditor@U2@@UAEPAXPBD@Z 10019f12 f   U2Designer:U2Designer.dll
 0001:00018f18       ?qt_metacast@URLDelegate@U2@@UAEPAXPBD@Z 10019f18 f   U2Designer:U2Designer.dll
 0001:00018f1e       ?removeDelegate@DelegateEditor@U2@@UAEPAVPropertyDelegate@2@ABVQString@@@Z 10019f1e f   U2Designer:U2Designer.dll
 0001:00018f24       ?setEditorData@URLDelegate@U2@@UBEXPAVQWidget@@ABVQModelIndex@@@Z 10019f24 f   U2Designer:U2Designer.dll
 0001:00018f2a       ?setModelData@URLDelegate@U2@@UBEXPAVQWidget@@PAVQAbstractItemModel@@ABVQModelIndex@@@Z 10019f2a f   U2Designer:U2Designer.dll
 0001:00018f30       ?type@URLDelegate@U2@@UBE?AW4Type@PropertyDelegate@2@XZ 10019f30 f   U2Designer:U2Designer.dll
 0001:00018f36       ?updateDelegate@DelegateEditor@U2@@UAEXABVQString@@@Z 10019f36 f   U2Designer:U2Designer.dll
 0001:00018f3c       ?updateDelegates@DelegateEditor@U2@@UAEXXZ 10019f3c f   U2Designer:U2Designer.dll
 0001:00018f42       ??0URLDelegate@U2@@QAE@ABVDelegateTags@1@ABVQString@@_N22PAVQObject@@2@Z 10019f42 f   U2Designer:U2Designer.dll
 0001:00018f48       ??0SpinBoxDelegate@U2@@QAE@ABV?$QMap@VQString@@VQVariant@@@@PAVQObject@@@Z 10019f48 f   U2Designer:U2Designer.dll
 0001:00018f4e       ??1SpinBoxDelegate@U2@@UAE@XZ 10019f4e f   U2Designer:U2Designer.dll
 0001:00018f54       ??0DoubleSpinBoxDelegate@U2@@QAE@ABV?$QMap@VQString@@VQVariant@@@@PAVQObject@@@Z 10019f54 f   U2Designer:U2Designer.dll
 0001:00018f5a       ??1DoubleSpinBoxDelegate@U2@@UAE@XZ 10019f5a f   U2Designer:U2Designer.dll
 0001:00018f60       ??0ComboBoxDelegate@U2@@QAE@ABV?$QMap@VQString@@VQVariant@@@@PAVQObject@@@Z 10019f60 f   U2Designer:U2Designer.dll
 0001:00018f66       ??0ComboBoxDelegate@U2@@QAE@ABV?$QList@U?$QPair@VQString@@VQVariant@@@@@@PAVQObject@@@Z 10019f66 f   U2Designer:U2Designer.dll
 0001:00018f6c       ??1ComboBoxDelegate@U2@@UAE@XZ 10019f6c f   U2Designer:U2Designer.dll
 0001:00018f72       ?clone@ComboBoxDelegate@U2@@UAEPAVPropertyDelegate@2@XZ 10019f72 f   U2Designer:U2Designer.dll
 0001:00018f78       ?clone@DoubleSpinBoxDelegate@U2@@UAEPAVPropertyDelegate@2@XZ 10019f78 f   U2Designer:U2Designer.dll
 0001:00018f7e       ?clone@SpinBoxDelegate@U2@@UAEPAVPropertyDelegate@2@XZ 10019f7e f   U2Designer:U2Designer.dll
 0001:00018f84       ?createEditor@ComboBoxDelegate@U2@@UBEPAVQWidget@@PAV3@ABVQStyleOptionViewItem@@ABVQModelIndex@@@Z 10019f84 f   U2Designer:U2Designer.dll
 0001:00018f8a       ?createEditor@DoubleSpinBoxDelegate@U2@@UBEPAVQWidget@@PAV3@ABVQStyleOptionViewItem@@ABVQModelIndex@@@Z 10019f8a f   U2Designer:U2Designer.dll
 0001:00018f90       ?createEditor@SpinBoxDelegate@U2@@UBEPAVQWidget@@PAV3@ABVQStyleOptionViewItem@@ABVQModelIndex@@@Z 10019f90 f   U2Designer:U2Designer.dll
 0001:00018f96       ?createWizardWidget@ComboBoxDelegate@U2@@UBEPAVPropertyWidget@2@AAVU2OpStatus@2@PAVQWidget@@@Z 10019f96 f   U2Designer:U2Designer.dll
 0001:00018f9c       ?createWizardWidget@DoubleSpinBoxDelegate@U2@@UBEPAVPropertyWidget@2@AAVU2OpStatus@2@PAVQWidget@@@Z 10019f9c f   U2Designer:U2Designer.dll
 0001:00018fa2       ?createWizardWidget@SpinBoxDelegate@U2@@UBEPAVPropertyWidget@2@AAVU2OpStatus@2@PAVQWidget@@@Z 10019fa2 f   U2Designer:U2Designer.dll
 0001:00018fa8       ?getDisplayValue@ComboBoxDelegate@U2@@UBE?AVQVariant@@ABV3@@Z 10019fa8 f   U2Designer:U2Designer.dll
 0001:00018fae       ?getDisplayValue@DoubleSpinBoxDelegate@U2@@UBE?AVQVariant@@ABV3@@Z 10019fae f   U2Designer:U2Designer.dll
 0001:00018fb4       ?getDisplayValue@SpinBoxDelegate@U2@@UBE?AVQVariant@@ABV3@@Z 10019fb4 f   U2Designer:U2Designer.dll
 0001:00018fba       ?getItems@ComboBoxDelegate@U2@@UBEXAAV?$QMap@VQString@@VQVariant@@@@@Z 10019fba f   U2Designer:U2Designer.dll
 0001:00018fc0       ?getItems@DoubleSpinBoxDelegate@U2@@UBEXAAV?$QMap@VQString@@VQVariant@@@@@Z 10019fc0 f   U2Designer:U2Designer.dll
 0001:00018fc6       ?getItems@SpinBoxDelegate@U2@@UBEXAAV?$QMap@VQString@@VQVariant@@@@@Z 10019fc6 f   U2Designer:U2Designer.dll
 0001:00018fcc       ?metaObject@ComboBoxDelegate@U2@@UBEPBUQMetaObject@@XZ 10019fcc f   U2Designer:U2Designer.dll
 0001:00018fd2       ?metaObject@DoubleSpinBoxDelegate@U2@@UBEPBUQMetaObject@@XZ 10019fd2 f   U2Designer:U2Designer.dll
 0001:00018fd8       ?metaObject@SpinBoxDelegate@U2@@UBEPBUQMetaObject@@XZ 10019fd8 f   U2Designer:U2Designer.dll
 0001:00018fde       ?qt_metacall@ComboBoxDelegate@U2@@UAEHW4Call@QMetaObject@@HPAPAX@Z 10019fde f   U2Designer:U2Designer.dll
 0001:00018fe4       ?qt_metacall@DoubleSpinBoxDelegate@U2@@UAEHW4Call@QMetaObject@@HPAPAX@Z 10019fe4 f   U2Designer:U2Designer.dll
 0001:00018fea       ?qt_metacall@SpinBoxDelegate@U2@@UAEHW4Call@QMetaObject@@HPAPAX@Z 10019fea f   U2Designer:U2Designer.dll
 0001:00018ff0       ?qt_metacast@ComboBoxDelegate@U2@@UAEPAXPBD@Z 10019ff0 f   U2Designer:U2Designer.dll
 0001:00018ff6       ?qt_metacast@DoubleSpinBoxDelegate@U2@@UAEPAXPBD@Z 10019ff6 f   U2Designer:U2Designer.dll
 0001:00018ffe       ?qt_metacast@SpinBoxDelegate@U2@@UAEPAXPBD@Z 10019ffe f   U2Designer:U2Designer.dll
 0001:00019004       ?setEditorData@ComboBoxDelegate@U2@@UBEXPAVQWidget@@ABVQModelIndex@@@Z 1001a004 f   U2Designer:U2Designer.dll
 0001:0001900a       ?setEditorData@DoubleSpinBoxDelegate@U2@@UBEXPAVQWidget@@ABVQModelIndex@@@Z 1001a00a f   U2Designer:U2Designer.dll
 0001:00019010       ?setEditorData@SpinBoxDelegate@U2@@UBEXPAVQWidget@@ABVQModelIndex@@@Z 1001a010 f   U2Designer:U2Designer.dll
 0001:00019016       ?setModelData@ComboBoxDelegate@U2@@UBEXPAVQWidget@@PAVQAbstractItemModel@@ABVQModelIndex@@@Z 1001a016 f   U2Designer:U2Designer.dll
 0001:0001901c       ?setModelData@DoubleSpinBoxDelegate@U2@@UBEXPAVQWidget@@PAVQAbstractItemModel@@ABVQModelIndex@@@Z 1001a01c f   U2Designer:U2Designer.dll
 0001:00019022       ?setModelData@SpinBoxDelegate@U2@@UBEXPAVQWidget@@PAVQAbstractItemModel@@ABVQModelIndex@@@Z 1001a022 f   U2Designer:U2Designer.dll
 0001:00019028       ?destroyEditor@QAbstractItemDelegate@@UBEXPAVQWidget@@ABVQModelIndex@@@Z 1001a028 f   Qt5Widgets:Qt5Widgets.dll
 0001:0001902e       ?drawCheck@QItemDelegate@@MBEXPAVQPainter@@ABVQStyleOptionViewItem@@ABVQRect@@W4CheckState@Qt@@@Z 1001a02e f   Qt5Widgets:Qt5Widgets.dll
 0001:00019034       ?drawDecoration@QItemDelegate@@MBEXPAVQPainter@@ABVQStyleOptionViewItem@@ABVQRect@@ABVQPixmap@@@Z 1001a034 f   Qt5Widgets:Qt5Widgets.dll
 0001:0001903a       ?drawDisplay@QItemDelegate@@MBEXPAVQPainter@@ABVQStyleOptionViewItem@@ABVQRect@@ABVQString@@@Z 1001a03a f   Qt5Widgets:Qt5Widgets.dll
 0001:00019040       ?drawFocus@QItemDelegate@@MBEXPAVQPainter@@ABVQStyleOptionViewItem@@ABVQRect@@@Z 1001a040 f   Qt5Widgets:Qt5Widgets.dll
 0001:00019046       ?editorEvent@QItemDelegate@@MAE_NPAVQEvent@@PAVQAbstractItemModel@@ABVQStyleOptionViewItem@@ABVQModelIndex@@@Z 1001a046 f   Qt5Widgets:Qt5Widgets.dll
 0001:0001904c       ?eventFilter@QItemDelegate@@MAE_NPAVQObject@@PAVQEvent@@@Z 1001a04c f   Qt5Widgets:Qt5Widgets.dll
 0001:00019052       ?helpEvent@QAbstractItemDelegate@@UAE_NPAVQHelpEvent@@PAVQAbstractItemView@@ABVQStyleOptionViewItem@@ABVQModelIndex@@@Z 1001a052 f   Qt5Widgets:Qt5Widgets.dll
 0001:00019058       ?paint@QItemDelegate@@UBEXPAVQPainter@@ABVQStyleOptionViewItem@@ABVQModelIndex@@@Z 1001a058 f   Qt5Widgets:Qt5Widgets.dll
 0001:0001905e       ?paintingRoles@QAbstractItemDelegate@@UBE?AV?$QVector@H@@XZ 1001a05e f   Qt5Widgets:Qt5Widgets.dll
 0001:00019064       ?sizeHint@QItemDelegate@@UBE?AVQSize@@ABVQStyleOptionViewItem@@ABVQModelIndex@@@Z 1001a064 f   Qt5Widgets:Qt5Widgets.dll
 0001:0001906a       ?updateEditorGeometry@QItemDelegate@@UBEXPAVQWidget@@ABVQStyleOptionViewItem@@ABVQModelIndex@@@Z 1001a06a f   Qt5Widgets:Qt5Widgets.dll
 0001:00019070       ?clear@QTextDocument@@UAEXXZ 1001a070 f   Qt5Gui:Qt5Gui.dll
 0001:00019076       ?createObject@QTextDocument@@MAEPAVQTextObject@@ABVQTextFormat@@@Z 1001a076 f   Qt5Gui:Qt5Gui.dll
 0001:0001907c       ?loadResource@QTextDocument@@MAE?AVQVariant@@HABVQUrl@@@Z 1001a07c f   Qt5Gui:Qt5Gui.dll
 0001:00019082       ??0QScriptValue@@QAE@XZ    1001a082 f   Qt5Script:Qt5Script.dll
 0001:00019088       ??1QScriptValue@@QAE@XZ    1001a088 f   Qt5Script:Qt5Script.dll
 0001:0001908e       ??0QScriptValue@@QAE@ABV0@@Z 1001a08e f   Qt5Script:Qt5Script.dll
 0001:00019094       ??4QScriptValue@@QAEAAV0@ABV0@@Z 1001a094 f   Qt5Script:Qt5Script.dll
 0001:0001909a       ?isString@QScriptValue@@QBE_NXZ 1001a09a f   Qt5Script:Qt5Script.dll
 0001:000190a0       ?toString@QScriptValue@@QBE?AVQString@@XZ 1001a0a0 f   Qt5Script:Qt5Script.dll
 0001:000190a6       ??1QScriptEngine@@UAE@XZ   1001a0a6 f   Qt5Script:Qt5Script.dll
 0001:000190ac       ?newVariant@QScriptEngine@@QAE?AVQScriptValue@@ABVQVariant@@@Z 1001a0ac f   Qt5Script:Qt5Script.dll
 0001:000190b2       ?isNumber@QScriptValue@@QBE_NXZ 1001a0b2 f   Qt5Script:Qt5Script.dll
 0001:000190b8       ?toInt32@QScriptValue@@QBEHXZ 1001a0b8 f   Qt5Script:Qt5Script.dll
 0001:000190be       ?tr@QMetaObject@@QBE?AVQString@@PBD0H@Z 1001a0be f   Qt5Core:Qt5Core.dll
 0001:000190c4       ??1Connection@QMetaObject@@QAE@XZ 1001a0c4 f   Qt5Core:Qt5Core.dll
 0001:000190ca       ??0QChar@@QAE@UQLatin1Char@@@Z 1001a0ca f   Qt5Core:Qt5Core.dll
 0001:000190d0       ??1QString@@QAE@XZ         1001a0d0 f   Qt5Core:Qt5Core.dll
 0001:000190d6       ?arg@QString@@QBE?AV1@ABV1@HVQChar@@@Z 1001a0d6 f   Qt5Core:Qt5Core.dll
 0001:000190dc       ?fromAscii_helper@QString@@CAPAU?$QTypedArrayData@G@@PBDH@Z 1001a0dc f   Qt5Core:Qt5Core.dll
 0001:000190e2       ?detach@QListData@@QAEPAUData@1@H@Z 1001a0e2 f   Qt5Core:Qt5Core.dll
 0001:000190e8       ?dispose@QListData@@SAXPAUData@1@@Z 1001a0e8 f   Qt5Core:Qt5Core.dll
 0001:000190ee       ?connect@QObject@@QBE?AVConnection@QMetaObject@@PBV1@PBD1W4ConnectionType@Qt@@@Z 1001a0ee f   Qt5Core:Qt5Core.dll
 0001:000190f4       ?childEvent@QObject@@MAEXPAVQChildEvent@@@Z 1001a0f4 f   Qt5Core:Qt5Core.dll
 0001:000190fa       ?connectNotify@QObject@@MAEXABVQMetaMethod@@@Z 1001a0fa f   Qt5Core:Qt5Core.dll
 0001:00019100       ?customEvent@QObject@@MAEXPAVQEvent@@@Z 1001a100 f   Qt5Core:Qt5Core.dll
 0001:00019106       ?disconnectNotify@QObject@@MAEXABVQMetaMethod@@@Z 1001a106 f   Qt5Core:Qt5Core.dll
 0001:0001910c       ?event@QObject@@UAE_NPAVQEvent@@@Z 1001a10c f   Qt5Core:Qt5Core.dll
 0001:00019112       ?eventFilter@QObject@@UAE_NPAV1@PAVQEvent@@@Z 1001a112 f   Qt5Core:Qt5Core.dll
 0001:00019118       ?timerEvent@QObject@@MAEXPAVQTimerEvent@@@Z 1001a118 f   Qt5Core:Qt5Core.dll
 0001:0001911e       ?detach_grow@QListData@@QAEPAUData@1@PAHH@Z 1001a11e f   Qt5Core:Qt5Core.dll
 0001:00019124       ?append@QListData@@QAEPAPAXXZ 1001a124 f   Qt5Core:Qt5Core.dll
 0001:0001912a       ??0QString@@QAE@XZ         1001a12a f   Qt5Core:Qt5Core.dll
 0001:00019130       ??0QString@@QAE@ABV0@@Z    1001a130 f   Qt5Core:Qt5Core.dll
 0001:00019136       ?append@QString@@QAEAAV1@ABV1@@Z 1001a136 f   Qt5Core:Qt5Core.dll
 0001:0001913c       ?fromUtf8@QString@@SA?AV1@PBDH@Z 1001a13c f   Qt5Core:Qt5Core.dll
 0001:00019142       ?free_helper@QHashData@@QAEXP6AXPAUNode@1@@Z@Z 1001a142 f   Qt5Core:Qt5Core.dll
 0001:00019148       ?translate@QCoreApplication@@SA?AVQString@@PBD00H@Z 1001a148 f   Qt5Core:Qt5Core.dll
 0001:0001914e       ?cast@QMetaObject@@QBEPAVQObject@@PAV2@@Z 1001a14e f   Qt5Core:Qt5Core.dll
 0001:00019154       ?normalizedType@QMetaObject@@SA?AVQByteArray@@PBD@Z 1001a154 f   Qt5Core:Qt5Core.dll
 0001:0001915a       ??1QByteArray@@QAE@XZ      1001a15a f   Qt5Core:Qt5Core.dll
 0001:00019160       ??4QString@@QAEAAV0@ABV0@@Z 1001a160 f   Qt5Core:Qt5Core.dll
 0001:00019166       ??0QString@@QAE@$$QAV0@@Z  1001a166 f   Qt5Core:Qt5Core.dll
 0001:0001916c       ??4QString@@QAEAAV0@$$QAV0@@Z 1001a16c f   Qt5Core:Qt5Core.dll
 0001:00019172       ?arg@QString@@QBE?AV1@HHHVQChar@@@Z 1001a172 f   Qt5Core:Qt5Core.dll
 0001:00019178       ??M@YA_NABVQString@@0@Z    1001a178 f   Qt5Core:Qt5Core.dll
 0001:0001917e       ?realloc@QListData@@QAEXH@Z 1001a17e f   Qt5Core:Qt5Core.dll
 0001:00019184       ?registerNormalizedType@QMetaType@@SAHABVQByteArray@@P6AXPAX@ZP6APAXPBX@Z2P6APAX13@ZHV?$QFlags@W4TypeFlag@QMetaType@@@@PBUQMetaObject@@@Z 1001a184 f   Qt5Core:Qt5Core.dll
 0001:0001918a       ?registerNormalizedTypedef@QMetaType@@SAHABVQByteArray@@H@Z 1001a18a f   Qt5Core:Qt5Core.dll
 0001:00019190       ??1QObject@@UAE@XZ         1001a190 f   Qt5Core:Qt5Core.dll
 0001:00019196       ?nextNode@QMapNodeBase@@QBEPBU1@XZ 1001a196 f   Qt5Core:Qt5Core.dll
 0001:0001919c       ?freeNodeAndRebalance@QMapDataBase@@QAEXPAUQMapNodeBase@@@Z 1001a19c f   Qt5Core:Qt5Core.dll
 0001:000191a2       ?recalcMostLeftNode@QMapDataBase@@QAEXXZ 1001a1a2 f   Qt5Core:Qt5Core.dll
 0001:000191a8       ?createNode@QMapDataBase@@QAEPAUQMapNodeBase@@HHPAU2@_N@Z 1001a1a8 f   Qt5Core:Qt5Core.dll
 0001:000191ae       ?freeTree@QMapDataBase@@QAEXPAUQMapNodeBase@@H@Z 1001a1ae f   Qt5Core:Qt5Core.dll
 0001:000191b4       ?createData@QMapDataBase@@SAPAU1@XZ 1001a1b4 f   Qt5Core:Qt5Core.dll
 0001:000191ba       ?freeData@QMapDataBase@@SAXPAU1@@Z 1001a1ba f   Qt5Core:Qt5Core.dll
 0001:000191c0       ??0QVariant@@QAE@XZ        1001a1c0 f   Qt5Core:Qt5Core.dll
 0001:000191c6       ??1QVariant@@QAE@XZ        1001a1c6 f   Qt5Core:Qt5Core.dll
 0001:000191cc       ??0QVariant@@QAE@ABV0@@Z   1001a1cc f   Qt5Core:Qt5Core.dll
 0001:000191d2       ??0QVariant@@QAE@ABVQString@@@Z 1001a1d2 f   Qt5Core:Qt5Core.dll
 0001:000191d8       ??0QVariant@@QAE@ABV?$QMap@VQString@@VQVariant@@@@@Z 1001a1d8 f   Qt5Core:Qt5Core.dll
 0001:000191de       ??4QVariant@@QAEAAV0@ABV0@@Z 1001a1de f   Qt5Core:Qt5Core.dll
 0001:000191e4       ??4QVariant@@QAEAAV0@$$QAV0@@Z 1001a1e4 f   Qt5Core:Qt5Core.dll
 0001:000191ea       ?userType@QVariant@@QBEHXZ 1001a1ea f   Qt5Core:Qt5Core.dll
 0001:000191f0       ?constData@QVariant@@QBEPBXXZ 1001a1f0 f   Qt5Core:Qt5Core.dll
 0001:000191f6       ?convert@QVariant@@QBE_NHPAX@Z 1001a1f6 f   Qt5Core:Qt5Core.dll
 0001:000191fc       ??0QByteArray@@QAE@XZ      1001a1fc f   Qt5Core:Qt5Core.dll
 0001:00019202       ??0QByteArray@@QAE@ABV0@@Z 1001a202 f   Qt5Core:Qt5Core.dll
 0001:00019208       ??4QByteArray@@QAEAAV0@$$QAV0@@Z 1001a208 f   Qt5Core:Qt5Core.dll
 0001:0001920e       ?split@QByteArray@@QBE?AV?$QList@VQByteArray@@@@D@Z 1001a20e f   Qt5Core:Qt5Core.dll
 0001:00019214       ?toUInt@QByteArray@@QBEIPA_NH@Z 1001a214 f   Qt5Core:Qt5Core.dll
 0001:0001921a       ?arg@QString@@QBE?AV1@IHHVQChar@@@Z 1001a21a f   Qt5Core:Qt5Core.dll
 0001:00019220       ?compare@QString@@QBEHABV1@W4CaseSensitivity@Qt@@@Z 1001a220 f   Qt5Core:Qt5Core.dll
 0001:00019226       ?number@QString@@SA?AV1@HH@Z 1001a226 f   Qt5Core:Qt5Core.dll
 0001:0001922c       ?number@QString@@SA?AV1@IH@Z 1001a22c f   Qt5Core:Qt5Core.dll
 0001:00019232       ?number@QString@@SA?AV1@NDH@Z 1001a232 f   Qt5Core:Qt5Core.dll
 0001:00019238       ??0QString@@QAE@ABVQByteArray@@@Z 1001a238 f   Qt5Core:Qt5Core.dll
 0001:0001923e       ?readLine@QIODevice@@QAE?AVQByteArray@@_J@Z 1001a23e f   Qt5Core:Qt5Core.dll
 0001:00019244       ?close@QFileDevice@@UAEXXZ 1001a244 f   Qt5Core:Qt5Core.dll
 0001:0001924a       ??0QFile@@QAE@ABVQString@@@Z 1001a24a f   Qt5Core:Qt5Core.dll
 0001:00019250       ??1QFile@@UAE@XZ           1001a250 f   Qt5Core:Qt5Core.dll
 0001:00019256       ?open@QFile@@UAE_NV?$QFlags@W4OpenModeFlag@QIODevice@@@@@Z 1001a256 f   Qt5Core:Qt5Core.dll
 0001:0001925c       ?hasRegisteredConverterFunction@QMetaType@@SA_NHH@Z 1001a25c f   Qt5Core:Qt5Core.dll
 0001:00019262       ?registerConverterFunction@QMetaType@@SA_NPBUAbstractConverterFunction@QtPrivate@@HH@Z 1001a262 f   Qt5Core:Qt5Core.dll
 0001:00019268       ?unregisterConverterFunction@QMetaType@@SAXHH@Z 1001a268 f   Qt5Core:Qt5Core.dll
 0001:0001926e       ?previousNode@QMapNodeBase@@QBEPBU1@XZ 1001a26e f   Qt5Core:Qt5Core.dll
 0001:00019274       ??0QVariant@@QAE@HPBXI@Z   1001a274 f   Qt5Core:Qt5Core.dll
 0001:0001927a       ?toString@QVariant@@QBE?AVQString@@XZ 1001a27a f   Qt5Core:Qt5Core.dll
 0001:00019280       ?toMap@QVariant@@QBE?AV?$QMap@VQString@@VQVariant@@@@XZ 1001a280 f   Qt5Core:Qt5Core.dll
 0001:00019286       ?mid@QString@@QBE?AV1@HH@Z 1001a286 f   Qt5Core:Qt5Core.dll
 0001:0001928c       ?toInt@QString@@QBEHPA_NH@Z 1001a28c f   Qt5Core:Qt5Core.dll
 0001:00019292       ?idealThreadCount@QThread@@SAHXZ 1001a292 f   Qt5Core:Qt5Core.dll
 0001:00019298       ??0QVariant@@QAE@H@Z       1001a298 f   Qt5Core:Qt5Core.dll
 0001:0001929e       ??0QVariant@@QAE@N@Z       1001a29e f   Qt5Core:Qt5Core.dll
 0001:000192a4       ??0QVariant@@QAE@PBD@Z     1001a2a4 f   Qt5Core:Qt5Core.dll
 0001:000192aa       ??4QString@@QAEAAV0@PBD@Z  1001a2aa f   Qt5Core:Qt5Core.dll
 0001:000192b0       ??0QRegExp@@QAE@ABVQString@@W4CaseSensitivity@Qt@@W4PatternSyntax@0@@Z 1001a2b0 f   Qt5Core:Qt5Core.dll
 0001:000192b6       ??1QRegExp@@QAE@XZ         1001a2b6 f   Qt5Core:Qt5Core.dll
 0001:000192bc       ??4QRegExp@@QAEAAV0@$$QAV0@@Z 1001a2bc f   Qt5Core:Qt5Core.dll
 0001:000192c2       ?tr@QObject@@SA?AVQString@@PBD0H@Z 1001a2c2 f   Qt5Core:Qt5Core.dll
 0001:000192c8       ?dynamicMetaObject@QObjectData@@QBEPAUQMetaObject@@XZ 1001a2c8 f   Qt5Core:Qt5Core.dll
 0001:000192ce       ?className@QMetaObject@@QBEPBDXZ 1001a2ce f   Qt5Core:Qt5Core.dll
 0001:000192d4       ?reserve@QByteArray@@QAEXH@Z 1001a2d4 f   Qt5Core:Qt5Core.dll
 0001:000192da       ?append@QByteArray@@QAEAAV1@D@Z 1001a2da f   Qt5Core:Qt5Core.dll
 0001:000192e0       ?append@QByteArray@@QAEAAV1@PBD@Z 1001a2e0 f   Qt5Core:Qt5Core.dll
 0001:000192e6       ?_Xbad_alloc@std@@YAXXZ    1001a2e6 f   msvcprt:MSVCP120.dll
 0001:000192ec       ?_Xlength_error@std@@YAXPBD@Z 1001a2ec f   msvcprt:MSVCP120.dll
 0001:000192f2       ?_Xout_of_range@std@@YAXPBD@Z 1001a2f2 f   msvcprt:MSVCP120.dll
 0001:000192f8       ?_Syserror_map@std@@YAPBDH@Z 1001a2f8 f   msvcprt:MSVCP120.dll
 0001:000192fe       ?_Winerror_map@std@@YAPBDH@Z 1001a2fe f   msvcprt:MSVCP120.dll
 0001:00019304       __purecall                 1001a304 f   MSVCRT:MSVCR120.dll
 0001:0001930a       ??2@YAPAXI@Z               1001a30a f   MSVCRT:MSVCR120.dll
 0001:00019310       ??3@YAXPAX@Z               1001a310 f   MSVCRT:MSVCR120.dll
 0001:00019316       ___atonexitinit            1001a316 f   MSVCRT:atonexit.obj
 0001:00019352       __onexit                   1001a352 f   MSVCRT:atonexit.obj
 0001:000193fb       _atexit                    1001a3fb f   MSVCRT:atonexit.obj
 0001:00019410       _memmove                   1001a410 f   MSVCRT:MSVCR120.dll
 0001:00019416       __hypot                    1001a416 f   MSVCRT:MSVCR120.dll
 0001:0001941c       @__security_check_cookie@4 1001a41c f   MSVCRT:secchk.obj
 0001:0001942c       __CxxThrowException@8      1001a42c f   MSVCRT:MSVCR120.dll
 0001:00019432       ___CxxFrameHandler3        1001a432 f   MSVCRT:MSVCR120.dll
 0001:00019438       _memcpy                    1001a438 f   MSVCRT:MSVCR120.dll
 0001:0001943e       ??0type_info@@AAE@ABV0@@Z  1001a43e f   MSVCRT:ti_inst.obj
 0001:00019449       ??4type_info@@AAEAAV0@ABV0@@Z 1001a449 f   MSVCRT:ti_inst.obj
 0001:0001944e       ??_Etype_info@@UAEPAXI@Z   1001a44e f i MSVCRT:ti_inst.obj
 0001:000194ec       _NtCurrentTeb              1001a4ec f i MSVCRT:crtdll.obj
 0001:000194f3       __CRT_INIT@12              1001a4f3 f   MSVCRT:crtdll.obj
 0001:000196ea       __DllMainCRTStartup@12     1001a6ea f   MSVCRT:crtdll.obj
 0001:00019840       __lock                     1001a840 f   MSVCRT:MSVCR120.dll
 0001:00019846       __unlock                   1001a846 f   MSVCRT:MSVCR120.dll
 0001:0001984c       __calloc_crt               1001a84c f   MSVCRT:MSVCR120.dll
 0001:00019852       ___dllonexit               1001a852 f   MSVCRT:MSVCR120.dll
 0001:00019860       __SEH_prolog4              1001a860 f   MSVCRT:sehprolg4.obj
 0001:000198a5       __SEH_epilog4              1001a8a5 f   MSVCRT:sehprolg4.obj
 0001:000198b9       __except_handler4          1001a8b9 f   MSVCRT:chandler4gs.obj
 0001:000198dc       ___raise_securityfailure   1001a8dc f   MSVCRT:gs_report.obj
 0001:00019919       ___report_gsfailure        1001a919 f   MSVCRT:gs_report.obj
 0001:00019a14       ___report_rangecheckfailure 1001aa14 f   MSVCRT:gs_report.obj
 0001:00019a20       ___report_securityfailure  1001aa20 f   MSVCRT:gs_report.obj
 0001:00019af0       ___report_securityfailureEx 1001aaf0 f   MSVCRT:gs_report.obj
 0001:00019c06       ??_M@YGXPAXIHP6EX0@Z@Z     1001ac06 f   MSVCRT:ehvecdtr.obj
 0001:00019c8e       ?__ArrayUnwind@@YGXPAXIHP6EX0@Z@Z 1001ac8e f   MSVCRT:ehvecdtr.obj
 0001:00019cec       ??1type_info@@UAE@XZ       1001acec f   MSVCRT:MSVCR120.dll
 0001:00019cf2       ___CppXcptFilter           1001acf2 f   MSVCRT:MSVCR120.dll
 0001:00019cf8       __amsg_exit                1001acf8 f   MSVCRT:MSVCR120.dll
 0001:00019d00       __FindPESection            1001ad00 f   MSVCRT:pesect.obj
 0001:00019d50       __IsNonwritableInCurrentImage 1001ad50 f   MSVCRT:pesect.obj
 0001:00019e10       __ValidateImageBase        1001ae10 f   MSVCRT:pesect.obj
 0001:00019e42       _free                      1001ae42 f   MSVCRT:MSVCR120.dll
 0001:00019e48       ___security_init_cookie    1001ae48 f   MSVCRT:gs_support.obj
 0001:00019ee4       _DllMain@12                1001aee4 f   MSVCRT:dllmain.obj
 0001:00019f06       __malloc_crt               1001af06 f   MSVCRT:MSVCR120.dll
 0001:00019f0c       __RTC_Initialize           1001af0c f   MSVCRT:initsect.obj
 0001:00019f2c       __RTC_Terminate            1001af2c f   MSVCRT:initsect.obj
 0001:00019f4c       __initterm                 1001af4c f   MSVCRT:MSVCR120.dll
 0001:00019f52       __initterm_e               1001af52 f   MSVCRT:MSVCR120.dll
 0001:00019f58       ___clean_type_info_names   1001af58 f   MSVCRT:tncleanup.obj
 0001:00019f64       __except_handler4_common   1001af64 f   MSVCRT:MSVCR120.dll
 0001:00019f6a       __crt_debugger_hook        1001af6a f   MSVCRT:MSVCR120.dll
 0001:00019f70       ___crtUnhandledException   1001af70 f   MSVCRT:MSVCR120.dll
 0001:00019f76       ___crtTerminateProcess     1001af76 f   MSVCRT:MSVCR120.dll
 0001:00019f7c       ?terminate@@YAXXZ          1001af7c f   MSVCRT:MSVCR120.dll
 0001:00019f82       ___clean_type_info_names_internal 1001af82 f   MSVCRT:MSVCR120.dll
 0001:00019f88       _EncodePointer@4           1001af88 f   kernel32:KERNEL32.dll
 0001:00019f8e       _DecodePointer@4           1001af8e f   kernel32:KERNEL32.dll
 0001:00019f94       _IsDebuggerPresent@0       1001af94 f   kernel32:KERNEL32.dll
 0001:00019f9a       _IsProcessorFeaturePresent@4 1001af9a f   kernel32:KERNEL32.dll
 0001:00019fa0       _QueryPerformanceCounter@4 1001afa0 f   kernel32:KERNEL32.dll
 0001:00019fa6       _GetCurrentProcessId@0     1001afa6 f   kernel32:KERNEL32.dll
 0001:00019fac       _GetCurrentThreadId@0      1001afac f   kernel32:KERNEL32.dll
 0001:00019fb2       _GetSystemTimeAsFileTime@4 1001afb2 f   kernel32:KERNEL32.dll
 0001:00019fb8       _DisableThreadLibraryCalls@4 1001afb8 f   kernel32:KERNEL32.dll
 0001:0001f5b0       ??__Ff@?4??registerConverter@?$AssociativeValueTypeIsMetaType@V?$QMap@VQString@@I@@$00@QtPrivate@@SA_NH@Z@YAXXZ 100205b0 f i DiamondClassifyWorker.obj
 0002:00000000       __imp__DisableThreadLibraryCalls@4 10021000     kernel32:KERNEL32.dll
 0002:00000004       __imp__GetSystemTimeAsFileTime@4 10021004     kernel32:KERNEL32.dll
 0002:00000008       __imp__GetCurrentThreadId@0 10021008     kernel32:KERNEL32.dll
 0002:0000000c       __imp__GetCurrentProcessId@0 1002100c     kernel32:KERNEL32.dll
 0002:00000010       __imp__QueryPerformanceCounter@4 10021010     kernel32:KERNEL32.dll
 0002:00000014       __imp__IsProcessorFeaturePresent@4 10021014     kernel32:KERNEL32.dll
 0002:00000018       __imp__IsDebuggerPresent@0 10021018     kernel32:KERNEL32.dll
 0002:0000001c       __imp__DecodePointer@4     1002101c     kernel32:KERNEL32.dll
 0002:00000020       __imp__EncodePointer@4     10021020     kernel32:KERNEL32.dll
 0002:00000024       \177KERNEL32_NULL_THUNK_DATA 10021024     kernel32:KERNEL32.dll
 0002:00000028       __imp_?_Xlength_error@std@@YAXPBD@Z 10021028     msvcprt:MSVCP120.dll
 0002:0000002c       __imp_?_Xout_of_range@std@@YAXPBD@Z 1002102c     msvcprt:MSVCP120.dll
 0002:00000030       __imp_?_Syserror_map@std@@YAPBDH@Z 10021030     msvcprt:MSVCP120.dll
 0002:00000034       __imp_?_Winerror_map@std@@YAPBDH@Z 10021034     msvcprt:MSVCP120.dll
 0002:00000038       __imp_?_Xbad_alloc@std@@YAXXZ 10021038     msvcprt:MSVCP120.dll
 0002:0000003c       \177MSVCP120_NULL_THUNK_DATA 1002103c     msvcprt:MSVCP120.dll
 0002:00000040       __imp___initterm_e         10021040     MSVCRT:MSVCR120.dll
 0002:00000044       __imp___initterm           10021044     MSVCRT:MSVCR120.dll
 0002:00000048       __imp___malloc_crt         10021048     MSVCRT:MSVCR120.dll
 0002:0000004c       __imp__free                1002104c     MSVCRT:MSVCR120.dll
 0002:00000050       __imp___except_handler4_common 10021050     MSVCRT:MSVCR120.dll
 0002:00000054       __imp____CppXcptFilter     10021054     MSVCRT:MSVCR120.dll
 0002:00000058       __imp_??1type_info@@UAE@XZ 10021058     MSVCRT:MSVCR120.dll
 0002:0000005c       __imp___onexit             1002105c     MSVCRT:MSVCR120.dll
 0002:00000060       __imp____dllonexit         10021060     MSVCRT:MSVCR120.dll
 0002:00000064       __imp___calloc_crt         10021064     MSVCRT:MSVCR120.dll
 0002:00000068       __imp___unlock             10021068     MSVCRT:MSVCR120.dll
 0002:0000006c       __imp___lock               1002106c     MSVCRT:MSVCR120.dll
 0002:00000070       __imp____CxxFrameHandler3  10021070     MSVCRT:MSVCR120.dll
 0002:00000074       __imp___CxxThrowException@8 10021074     MSVCRT:MSVCR120.dll
 0002:00000078       __imp___hypot              10021078     MSVCRT:MSVCR120.dll
 0002:0000007c       __imp__memmove             1002107c     MSVCRT:MSVCR120.dll
 0002:00000080       __imp_??3@YAXPAX@Z         10021080     MSVCRT:MSVCR120.dll
 0002:00000084       __imp_??2@YAPAXI@Z         10021084     MSVCRT:MSVCR120.dll
 0002:00000088       __imp___purecall           10021088     MSVCRT:MSVCR120.dll
 0002:0000008c       __imp___crt_debugger_hook  1002108c     MSVCRT:MSVCR120.dll
 0002:00000090       __imp____crtUnhandledException 10021090     MSVCRT:MSVCR120.dll
 0002:00000094       __imp____crtTerminateProcess 10021094     MSVCRT:MSVCR120.dll
 0002:00000098       __imp_?terminate@@YAXXZ    10021098     MSVCRT:MSVCR120.dll
 0002:0000009c       __imp____clean_type_info_names_internal 1002109c     MSVCRT:MSVCR120.dll
 0002:000000a0       __imp___amsg_exit          100210a0     MSVCRT:MSVCR120.dll
 0002:000000a4       __imp__memcpy              100210a4     MSVCRT:MSVCR120.dll
 0002:000000a8       \177MSVCR120_NULL_THUNK_DATA 100210a8     MSVCRT:MSVCR120.dll
 0002:000000ac       __imp_?className@QMetaObject@@QBEPBDXZ 100210ac     Qt5Core:Qt5Core.dll
 0002:000000b0       __imp_?reserve@QByteArray@@QAEXH@Z 100210b0     Qt5Core:Qt5Core.dll
 0002:000000b4       __imp_?append@QByteArray@@QAEAAV1@D@Z 100210b4     Qt5Core:Qt5Core.dll
 0002:000000b8       __imp_?append@QByteArray@@QAEAAV1@PBD@Z 100210b8     Qt5Core:Qt5Core.dll
 0002:000000bc       __imp_?tr@QObject@@SA?AVQString@@PBD0H@Z 100210bc     Qt5Core:Qt5Core.dll
 0002:000000c0       __imp_??4QRegExp@@QAEAAV0@$$QAV0@@Z 100210c0     Qt5Core:Qt5Core.dll
 0002:000000c4       __imp_??1QRegExp@@QAE@XZ   100210c4     Qt5Core:Qt5Core.dll
 0002:000000c8       __imp_??0QRegExp@@QAE@ABVQString@@W4CaseSensitivity@Qt@@W4PatternSyntax@0@@Z 100210c8     Qt5Core:Qt5Core.dll
 0002:000000cc       __imp_??4QString@@QAEAAV0@PBD@Z 100210cc     Qt5Core:Qt5Core.dll
 0002:000000d0       __imp_??0QVariant@@QAE@PBD@Z 100210d0     Qt5Core:Qt5Core.dll
 0002:000000d4       __imp_??0QVariant@@QAE@N@Z 100210d4     Qt5Core:Qt5Core.dll
 0002:000000d8       __imp_??0QVariant@@QAE@H@Z 100210d8     Qt5Core:Qt5Core.dll
 0002:000000dc       __imp_?idealThreadCount@QThread@@SAHXZ 100210dc     Qt5Core:Qt5Core.dll
 0002:000000e0       __imp_?toInt@QString@@QBEHPA_NH@Z 100210e0     Qt5Core:Qt5Core.dll
 0002:000000e4       __imp_?mid@QString@@QBE?AV1@HH@Z 100210e4     Qt5Core:Qt5Core.dll
 0002:000000e8       __imp_?toMap@QVariant@@QBE?AV?$QMap@VQString@@VQVariant@@@@XZ 100210e8     Qt5Core:Qt5Core.dll
 0002:000000ec       __imp_?toString@QVariant@@QBE?AVQString@@XZ 100210ec     Qt5Core:Qt5Core.dll
 0002:000000f0       __imp_??0QVariant@@QAE@HPBXI@Z 100210f0     Qt5Core:Qt5Core.dll
 0002:000000f4       __imp_?previousNode@QMapNodeBase@@QBEPBU1@XZ 100210f4     Qt5Core:Qt5Core.dll
 0002:000000f8       __imp_?unregisterConverterFunction@QMetaType@@SAXHH@Z 100210f8     Qt5Core:Qt5Core.dll
 0002:000000fc       __imp_?registerConverterFunction@QMetaType@@SA_NPBUAbstractConverterFunction@QtPrivate@@HH@Z 100210fc     Qt5Core:Qt5Core.dll
 0002:00000100       __imp_?hasRegisteredConverterFunction@QMetaType@@SA_NHH@Z 10021100     Qt5Core:Qt5Core.dll
 0002:00000104       __imp_?open@QFile@@UAE_NV?$QFlags@W4OpenModeFlag@QIODevice@@@@@Z 10021104     Qt5Core:Qt5Core.dll
 0002:00000108       __imp_??1QFile@@UAE@XZ     10021108     Qt5Core:Qt5Core.dll
 0002:0000010c       __imp_??0QFile@@QAE@ABVQString@@@Z 1002110c     Qt5Core:Qt5Core.dll
 0002:00000110       __imp_?close@QFileDevice@@UAEXXZ 10021110     Qt5Core:Qt5Core.dll
 0002:00000114       __imp_?readLine@QIODevice@@QAE?AVQByteArray@@_J@Z 10021114     Qt5Core:Qt5Core.dll
 0002:00000118       __imp_?tr@QMetaObject@@QBE?AVQString@@PBD0H@Z 10021118     Qt5Core:Qt5Core.dll
 0002:0000011c       __imp_??1Connection@QMetaObject@@QAE@XZ 1002111c     Qt5Core:Qt5Core.dll
 0002:00000120       __imp_??0QChar@@QAE@UQLatin1Char@@@Z 10021120     Qt5Core:Qt5Core.dll
 0002:00000124       __imp_??1QString@@QAE@XZ   10021124     Qt5Core:Qt5Core.dll
 0002:00000128       __imp_?arg@QString@@QBE?AV1@ABV1@HVQChar@@@Z 10021128     Qt5Core:Qt5Core.dll
 0002:0000012c       __imp_?fromAscii_helper@QString@@CAPAU?$QTypedArrayData@G@@PBDH@Z 1002112c     Qt5Core:Qt5Core.dll
 0002:00000130       __imp_?detach@QListData@@QAEPAUData@1@H@Z 10021130     Qt5Core:Qt5Core.dll
 0002:00000134       __imp_?dispose@QListData@@SAXPAUData@1@@Z 10021134     Qt5Core:Qt5Core.dll
 0002:00000138       __imp_?connect@QObject@@QBE?AVConnection@QMetaObject@@PBV1@PBD1W4ConnectionType@Qt@@@Z 10021138     Qt5Core:Qt5Core.dll
 0002:0000013c       __imp_?childEvent@QObject@@MAEXPAVQChildEvent@@@Z 1002113c     Qt5Core:Qt5Core.dll
 0002:00000140       __imp_?connectNotify@QObject@@MAEXABVQMetaMethod@@@Z 10021140     Qt5Core:Qt5Core.dll
 0002:00000144       __imp_?customEvent@QObject@@MAEXPAVQEvent@@@Z 10021144     Qt5Core:Qt5Core.dll
 0002:00000148       __imp_?disconnectNotify@QObject@@MAEXABVQMetaMethod@@@Z 10021148     Qt5Core:Qt5Core.dll
 0002:0000014c       __imp_?event@QObject@@UAE_NPAVQEvent@@@Z 1002114c     Qt5Core:Qt5Core.dll
 0002:00000150       __imp_?eventFilter@QObject@@UAE_NPAV1@PAVQEvent@@@Z 10021150     Qt5Core:Qt5Core.dll
 0002:00000154       __imp_?timerEvent@QObject@@MAEXPAVQTimerEvent@@@Z 10021154     Qt5Core:Qt5Core.dll
 0002:00000158       __imp_?detach_grow@QListData@@QAEPAUData@1@PAHH@Z 10021158     Qt5Core:Qt5Core.dll
 0002:0000015c       __imp_?append@QListData@@QAEPAPAXXZ 1002115c     Qt5Core:Qt5Core.dll
 0002:00000160       __imp_??0QString@@QAE@XZ   10021160     Qt5Core:Qt5Core.dll
 0002:00000164       __imp_??0QString@@QAE@ABV0@@Z 10021164     Qt5Core:Qt5Core.dll
 0002:00000168       __imp_?append@QString@@QAEAAV1@ABV1@@Z 10021168     Qt5Core:Qt5Core.dll
 0002:0000016c       __imp_?fromUtf8@QString@@SA?AV1@PBDH@Z 1002116c     Qt5Core:Qt5Core.dll
 0002:00000170       __imp_?free_helper@QHashData@@QAEXP6AXPAUNode@1@@Z@Z 10021170     Qt5Core:Qt5Core.dll
 0002:00000174       __imp_?shared_null@QListData@@2UData@1@B 10021174     Qt5Core:Qt5Core.dll
 0002:00000178       __imp_?shared_null@QHashData@@2U1@B 10021178     Qt5Core:Qt5Core.dll
 0002:0000017c       __imp_?translate@QCoreApplication@@SA?AVQString@@PBD00H@Z 1002117c     Qt5Core:Qt5Core.dll
 0002:00000180       __imp_?cast@QMetaObject@@QBEPAVQObject@@PAV2@@Z 10021180     Qt5Core:Qt5Core.dll
 0002:00000184       __imp_?normalizedType@QMetaObject@@SA?AVQByteArray@@PBD@Z 10021184     Qt5Core:Qt5Core.dll
 0002:00000188       __imp_??1QByteArray@@QAE@XZ 10021188     Qt5Core:Qt5Core.dll
 0002:0000018c       __imp_??4QString@@QAEAAV0@ABV0@@Z 1002118c     Qt5Core:Qt5Core.dll
 0002:00000190       __imp_??0QString@@QAE@$$QAV0@@Z 10021190     Qt5Core:Qt5Core.dll
 0002:00000194       __imp_??4QString@@QAEAAV0@$$QAV0@@Z 10021194     Qt5Core:Qt5Core.dll
 0002:00000198       __imp_?arg@QString@@QBE?AV1@HHHVQChar@@@Z 10021198     Qt5Core:Qt5Core.dll
 0002:0000019c       __imp_??M@YA_NABVQString@@0@Z 1002119c     Qt5Core:Qt5Core.dll
 0002:000001a0       __imp_?realloc@QListData@@QAEXH@Z 100211a0     Qt5Core:Qt5Core.dll
 0002:000001a4       __imp_?registerNormalizedType@QMetaType@@SAHABVQByteArray@@P6AXPAX@ZP6APAXPBX@Z2P6APAX13@ZHV?$QFlags@W4TypeFlag@QMetaType@@@@PBUQMetaObject@@@Z 100211a4     Qt5Core:Qt5Core.dll
 0002:000001a8       __imp_?registerNormalizedTypedef@QMetaType@@SAHABVQByteArray@@H@Z 100211a8     Qt5Core:Qt5Core.dll
 0002:000001ac       __imp_??1QObject@@UAE@XZ   100211ac     Qt5Core:Qt5Core.dll
 0002:000001b0       __imp_?nextNode@QMapNodeBase@@QBEPBU1@XZ 100211b0     Qt5Core:Qt5Core.dll
 0002:000001b4       __imp_?freeNodeAndRebalance@QMapDataBase@@QAEXPAUQMapNodeBase@@@Z 100211b4     Qt5Core:Qt5Core.dll
 0002:000001b8       __imp_?recalcMostLeftNode@QMapDataBase@@QAEXXZ 100211b8     Qt5Core:Qt5Core.dll
 0002:000001bc       __imp_?createNode@QMapDataBase@@QAEPAUQMapNodeBase@@HHPAU2@_N@Z 100211bc     Qt5Core:Qt5Core.dll
 0002:000001c0       __imp_?freeTree@QMapDataBase@@QAEXPAUQMapNodeBase@@H@Z 100211c0     Qt5Core:Qt5Core.dll
 0002:000001c4       __imp_?createData@QMapDataBase@@SAPAU1@XZ 100211c4     Qt5Core:Qt5Core.dll
 0002:000001c8       __imp_?freeData@QMapDataBase@@SAXPAU1@@Z 100211c8     Qt5Core:Qt5Core.dll
 0002:000001cc       __imp_??0QVariant@@QAE@XZ  100211cc     Qt5Core:Qt5Core.dll
 0002:000001d0       __imp_??1QVariant@@QAE@XZ  100211d0     Qt5Core:Qt5Core.dll
 0002:000001d4       __imp_??0QVariant@@QAE@ABV0@@Z 100211d4     Qt5Core:Qt5Core.dll
 0002:000001d8       __imp_??0QVariant@@QAE@ABVQString@@@Z 100211d8     Qt5Core:Qt5Core.dll
 0002:000001dc       __imp_??0QVariant@@QAE@ABV?$QMap@VQString@@VQVariant@@@@@Z 100211dc     Qt5Core:Qt5Core.dll
 0002:000001e0       __imp_??4QVariant@@QAEAAV0@ABV0@@Z 100211e0     Qt5Core:Qt5Core.dll
 0002:000001e4       __imp_??4QVariant@@QAEAAV0@$$QAV0@@Z 100211e4     Qt5Core:Qt5Core.dll
 0002:000001e8       __imp_?userType@QVariant@@QBEHXZ 100211e8     Qt5Core:Qt5Core.dll
 0002:000001ec       __imp_?constData@QVariant@@QBEPBXXZ 100211ec     Qt5Core:Qt5Core.dll
 0002:000001f0       __imp_?convert@QVariant@@QBE_NHPAX@Z 100211f0     Qt5Core:Qt5Core.dll
 0002:000001f4       __imp_?shared_null@QMapDataBase@@2U1@B 100211f4     Qt5Core:Qt5Core.dll
 0002:000001f8       __imp_??0QByteArray@@QAE@XZ 100211f8     Qt5Core:Qt5Core.dll
 0002:000001fc       __imp_??0QByteArray@@QAE@ABV0@@Z 100211fc     Qt5Core:Qt5Core.dll
 0002:00000200       __imp_??4QByteArray@@QAEAAV0@$$QAV0@@Z 10021200     Qt5Core:Qt5Core.dll
 0002:00000204       __imp_?split@QByteArray@@QBE?AV?$QList@VQByteArray@@@@D@Z 10021204     Qt5Core:Qt5Core.dll
 0002:00000208       __imp_?toUInt@QByteArray@@QBEIPA_NH@Z 10021208     Qt5Core:Qt5Core.dll
 0002:0000020c       __imp_?arg@QString@@QBE?AV1@IHHVQChar@@@Z 1002120c     Qt5Core:Qt5Core.dll
 0002:00000210       __imp_?compare@QString@@QBEHABV1@W4CaseSensitivity@Qt@@@Z 10021210     Qt5Core:Qt5Core.dll
 0002:00000214       __imp_?number@QString@@SA?AV1@HH@Z 10021214     Qt5Core:Qt5Core.dll
 0002:00000218       __imp_?number@QString@@SA?AV1@IH@Z 10021218     Qt5Core:Qt5Core.dll
 0002:0000021c       __imp_?number@QString@@SA?AV1@NDH@Z 1002121c     Qt5Core:Qt5Core.dll
 0002:00000220       __imp_??0QString@@QAE@ABVQByteArray@@@Z 10021220     Qt5Core:Qt5Core.dll
 0002:00000224       __imp_?dynamicMetaObject@QObjectData@@QBEPAUQMetaObject@@XZ 10021224     Qt5Core:Qt5Core.dll
 0002:00000228       \177Qt5Core_NULL_THUNK_DATA 10021228     Qt5Core:Qt5Core.dll
 0002:0000022c       __imp_?clear@QTextDocument@@UAEXXZ 1002122c     Qt5Gui:Qt5Gui.dll
 0002:00000230       __imp_?createObject@QTextDocument@@MAEPAVQTextObject@@ABVQTextFormat@@@Z 10021230     Qt5Gui:Qt5Gui.dll
 0002:00000234       __imp_?loadResource@QTextDocument@@MAE?AVQVariant@@HABVQUrl@@@Z 10021234     Qt5Gui:Qt5Gui.dll
 0002:00000238       \177Qt5Gui_NULL_THUNK_DATA 10021238     Qt5Gui:Qt5Gui.dll
 0002:0000023c       __imp_?toString@QScriptValue@@QBE?AVQString@@XZ 1002123c     Qt5Script:Qt5Script.dll
 0002:00000240       __imp_?isString@QScriptValue@@QBE_NXZ 10021240     Qt5Script:Qt5Script.dll
 0002:00000244       __imp_??4QScriptValue@@QAEAAV0@ABV0@@Z 10021244     Qt5Script:Qt5Script.dll
 0002:00000248       __imp_??0QScriptValue@@QAE@ABV0@@Z 10021248     Qt5Script:Qt5Script.dll
 0002:0000024c       __imp_??1QScriptValue@@QAE@XZ 1002124c     Qt5Script:Qt5Script.dll
 0002:00000250       __imp_??0QScriptValue@@QAE@XZ 10021250     Qt5Script:Qt5Script.dll
 0002:00000254       __imp_??1QScriptEngine@@UAE@XZ 10021254     Qt5Script:Qt5Script.dll
 0002:00000258       __imp_?newVariant@QScriptEngine@@QAE?AVQScriptValue@@ABVQVariant@@@Z 10021258     Qt5Script:Qt5Script.dll
 0002:0000025c       __imp_?isNumber@QScriptValue@@QBE_NXZ 1002125c     Qt5Script:Qt5Script.dll
 0002:00000260       __imp_?toInt32@QScriptValue@@QBEHXZ 10021260     Qt5Script:Qt5Script.dll
 0002:00000264       \177Qt5Script_NULL_THUNK_DATA 10021264     Qt5Script:Qt5Script.dll
 0002:00000268       __imp_?updateEditorGeometry@QItemDelegate@@UBEXPAVQWidget@@ABVQStyleOptionViewItem@@ABVQModelIndex@@@Z 10021268     Qt5Widgets:Qt5Widgets.dll
 0002:0000026c       __imp_?paintingRoles@QAbstractItemDelegate@@UBE?AV?$QVector@H@@XZ 1002126c     Qt5Widgets:Qt5Widgets.dll
 0002:00000270       __imp_?paint@QItemDelegate@@UBEXPAVQPainter@@ABVQStyleOptionViewItem@@ABVQModelIndex@@@Z 10021270     Qt5Widgets:Qt5Widgets.dll
 0002:00000274       __imp_?helpEvent@QAbstractItemDelegate@@UAE_NPAVQHelpEvent@@PAVQAbstractItemView@@ABVQStyleOptionViewItem@@ABVQModelIndex@@@Z 10021274     Qt5Widgets:Qt5Widgets.dll
 0002:00000278       __imp_?eventFilter@QItemDelegate@@MAE_NPAVQObject@@PAVQEvent@@@Z 10021278     Qt5Widgets:Qt5Widgets.dll
 0002:0000027c       __imp_?editorEvent@QItemDelegate@@MAE_NPAVQEvent@@PAVQAbstractItemModel@@ABVQStyleOptionViewItem@@ABVQModelIndex@@@Z 1002127c     Qt5Widgets:Qt5Widgets.dll
 0002:00000280       __imp_?drawFocus@QItemDelegate@@MBEXPAVQPainter@@ABVQStyleOptionViewItem@@ABVQRect@@@Z 10021280     Qt5Widgets:Qt5Widgets.dll
 0002:00000284       __imp_?drawDisplay@QItemDelegate@@MBEXPAVQPainter@@ABVQStyleOptionViewItem@@ABVQRect@@ABVQString@@@Z 10021284     Qt5Widgets:Qt5Widgets.dll
 0002:00000288       __imp_?drawDecoration@QItemDelegate@@MBEXPAVQPainter@@ABVQStyleOptionViewItem@@ABVQRect@@ABVQPixmap@@@Z 10021288     Qt5Widgets:Qt5Widgets.dll
 0002:0000028c       __imp_?drawCheck@QItemDelegate@@MBEXPAVQPainter@@ABVQStyleOptionViewItem@@ABVQRect@@W4CheckState@Qt@@@Z 1002128c     Qt5Widgets:Qt5Widgets.dll
 0002:00000290       __imp_?destroyEditor@QAbstractItemDelegate@@UBEXPAVQWidget@@ABVQModelIndex@@@Z 10021290     Qt5Widgets:Qt5Widgets.dll
 0002:00000294       __imp_?sizeHint@QItemDelegate@@UBE?AVQSize@@ABVQStyleOptionViewItem@@ABVQModelIndex@@@Z 10021294     Qt5Widgets:Qt5Widgets.dll
 0002:00000298       \177Qt5Widgets_NULL_THUNK_DATA 10021298     Qt5Widgets:Qt5Widgets.dll
 0002:0000029c       __imp_??0ExternalToolLogParser@U2@@QAE@XZ 1002129c     U2Core:U2Core.dll
 0002:000002a0       __imp_??1ExternalToolSupportTask@U2@@UAE@XZ 100212a0     U2Core:U2Core.dll
 0002:000002a4       __imp_??0ExternalToolSupportTask@U2@@QAE@ABVQString@@V?$QFlags@W4TaskFlag@U2@@@@@Z 100212a4     U2Core:U2Core.dll
 0002:000002a8       __imp_??1ExternalToolRunTask@U2@@UAE@XZ 100212a8     U2Core:U2Core.dll
 0002:000002ac       __imp_??0ExternalToolRunTask@U2@@QAE@ABVQString@@ABVQStringList@@PAVExternalToolLogParser@1@010_N@Z 100212ac     U2Core:U2Core.dll
 0002:000002b0       __imp_?setError@Task@U2@@QAEXABVQString@@@Z 100212b0     U2Core:U2Core.dll
 0002:000002b4       __imp_?addSubTask@Task@U2@@QAEXPAV12@@Z 100212b4     U2Core:U2Core.dll
 0002:000002b8       __imp_?rollFileName@GUrlUtils@U2@@SA?AVQString@@ABV3@ABV?$QSet@VQString@@@@@Z 100212b8     U2Core:U2Core.dll
 0002:000002bc       __imp_??1SimpleEventCounter@U2@@UAE@XZ 100212bc     U2Core:U2Core.dll
 0002:000002c0       __imp_??0GReportableCounter@U2@@QAE@ABVQString@@0N@Z 100212c0     U2Core:U2Core.dll
 0002:000002c4       __imp_??1GCounter@U2@@UAE@XZ 100212c4     U2Core:U2Core.dll
 0002:000002c8       __imp_??1Logger@U2@@UAE@XZ 100212c8     U2Core:U2Core.dll
 0002:000002cc       __imp_?staticMetaObject@Plugin@U2@@2UQMetaObject@@B 100212cc     U2Core:U2Core.dll
 0002:000002d0       __imp_?qt_metacall@Plugin@U2@@UAEHW4Call@QMetaObject@@HPAPAX@Z 100212d0     U2Core:U2Core.dll
 0002:000002d4       __imp_?qt_metacast@Plugin@U2@@UAEPAXPBD@Z 100212d4     U2Core:U2Core.dll
 0002:000002d8       __imp_?staticMetaObject@ExternalTool@U2@@2UQMetaObject@@B 100212d8     U2Core:U2Core.dll
 0002:000002dc       __imp_?qt_metacall@ExternalTool@U2@@UAEHW4Call@QMetaObject@@HPAPAX@Z 100212dc     U2Core:U2Core.dll
 0002:000002e0       __imp_?qt_metacast@ExternalTool@U2@@UAEPAXPBD@Z 100212e0     U2Core:U2Core.dll
 0002:000002e4       __imp_?staticMetaObject@Task@U2@@2UQMetaObject@@B 100212e4     U2Core:U2Core.dll
 0002:000002e8       __imp_?qt_metacall@Task@U2@@UAEHW4Call@QMetaObject@@HPAPAX@Z 100212e8     U2Core:U2Core.dll
 0002:000002ec       __imp_?qt_metacast@Task@U2@@UAEPAXPBD@Z 100212ec     U2Core:U2Core.dll
 0002:000002f0       __imp_??1Task@U2@@UAE@XZ   100212f0     U2Core:U2Core.dll
 0002:000002f4       __imp_??0Task@U2@@QAE@ABVQString@@V?$QFlags@W4TaskFlag@U2@@@@@Z 100212f4     U2Core:U2Core.dll
 0002:000002f8       __imp_?errorWritingFile@L10N@U2@@SA?AVQString@@ABVGUrl@2@@Z 100212f8     U2Core:U2Core.dll
 0002:000002fc       __imp_?errorOpeningFileWrite@L10N@U2@@SA?AVQString@@ABVGUrl@2@@Z 100212fc     U2Core:U2Core.dll
 0002:00000300       __imp_??1Plugin@U2@@UAE@XZ 10021300     U2Core:U2Core.dll
 0002:00000304       __imp_??0Plugin@U2@@QAE@ABVQString@@0_NW4PluginState@1@@Z 10021304     U2Core:U2Core.dll
 0002:00000308       __imp_?unregisterEntry@ExternalToolRegistry@U2@@QAEXABVQString@@@Z 10021308     U2Core:U2Core.dll
 0002:0000030c       __imp_?registerEntry@ExternalToolRegistry@U2@@QAE_NPAVExternalTool@2@@Z 1002130c     U2Core:U2Core.dll
 0002:00000310       __imp_?getExternalToolRegistry@AppContext@U2@@SAPAVExternalToolRegistry@2@XZ 10021310     U2Core:U2Core.dll
 0002:00000314       __imp_?performAdditionalChecks@ExternalTool@U2@@UAEXABVQString@@@Z 10021314     U2Core:U2Core.dll
 0002:00000318       __imp_?getToolRunnerAdditionalOptions@ExternalTool@U2@@UAE?BVQStringList@@XZ 10021318     U2Core:U2Core.dll
 0002:0000031c       __imp_?getAdditionalPaths@ExternalTool@U2@@UBE?AVQStringList@@XZ 1002131c     U2Core:U2Core.dll
 0002:00000320       __imp_?getAdditionalParameters@ExternalTool@U2@@UAEXABVQString@@@Z 10021320     U2Core:U2Core.dll
 0002:00000324       __imp_??1ExternalTool@U2@@UAE@XZ 10021324     U2Core:U2Core.dll
 0002:00000328       __imp_??0ExternalTool@U2@@QAE@VQString@@0@Z 10021328     U2Core:U2Core.dll
 0002:0000032c       __imp_?PLAIN_TEXT@BaseDocumentFormats@U2@@2VQString@@B 1002132c     U2Core:U2Core.dll
 0002:00000330       __imp_?lookupTranslation@DNATranslationRegistry@U2@@QAE?AV?$QList@PAVDNATranslation@U2@@@@PBVDNAAlphabet@2@W4DNATranslationType@2@@Z 10021330     U2Core:U2Core.dll
 0002:00000334       __imp_?NUCL_DNA_DEFAULT@BaseDNAAlphabetIds@U2@@SA?BVQString@@XZ 10021334     U2Core:U2Core.dll
 0002:00000338       __imp_?getDNAAlphabetRegistry@AppContext@U2@@SAPAVDNAAlphabetRegistry@2@XZ 10021338     U2Core:U2Core.dll
 0002:0000033c       __imp_?getAppSettings@AppContext@U2@@SAPAVAppSettings@2@XZ 1002133c     U2Core:U2Core.dll
 0002:00000340       __imp_?info@Logger@U2@@QAEXABVQString@@@Z 10021340     U2Core:U2Core.dll
 0002:00000344       __imp_?trace@Logger@U2@@QAEXABVQString@@@Z 10021344     U2Core:U2Core.dll
 0002:00000348       __imp_?lookupTranslation@DNATranslationRegistry@U2@@QAEPAVDNATranslation@2@ABVQString@@@Z 10021348     U2Core:U2Core.dll
 0002:0000034c       __imp_?getDNATranslationRegistry@AppContext@U2@@SAPAVDNATranslationRegistry@2@XZ 1002134c     U2Core:U2Core.dll
 0002:00000350       __imp_?qt_metacast@TaskSignalMapper@U2@@UAEPAXPBD@Z 10021350     U2Core:U2Core.dll
 0002:00000354       __imp_?qt_metacast@FailTask@U2@@UAEPAXPBD@Z 10021354     U2Core:U2Core.dll
 0002:00000358       __imp_?qt_metacall@TaskSignalMapper@U2@@UAEHW4Call@QMetaObject@@HPAPAX@Z 10021358     U2Core:U2Core.dll
 0002:0000035c       __imp_?qt_metacall@FailTask@U2@@UAEHW4Call@QMetaObject@@HPAPAX@Z 1002135c     U2Core:U2Core.dll
 0002:00000360       __imp_?metaObject@TaskSignalMapper@U2@@UBEPBUQMetaObject@@XZ 10021360     U2Core:U2Core.dll
 0002:00000364       __imp_?metaObject@FailTask@U2@@UBEPBUQMetaObject@@XZ 10021364     U2Core:U2Core.dll
 0002:00000368       __imp_?runScript@ScriptTask@U2@@SA?AVQScriptValue@@PAVQScriptEngine@@ABV?$QMap@VQString@@VQScriptValue@@@@ABVQString@@AAVTaskStateInfo@2@@Z 10021368     U2Core:U2Core.dll
 0002:0000036c       __imp_?addListeners@ExternalToolSupportTask@U2@@QAEXABV?$QList@PAVExternalToolListener@U2@@@@@Z 1002136c     U2Core:U2Core.dll
 0002:00000370       __imp_??1U2OpStatus2Log@U2@@UAE@XZ 10021370     U2Core:U2Core.dll
 0002:00000374       __imp_??0U2OpStatus2Log@U2@@QAE@W4LogLevel@1@@Z 10021374     U2Core:U2Core.dll
 0002:00000378       __imp_?getError@U2OpStatusImpl@U2@@UBE?AVQString@@XZ 10021378     U2Core:U2Core.dll
 0002:0000037c       __imp_??0TaskSignalMapper@U2@@QAE@PAVTask@1@@Z 1002137c     U2Core:U2Core.dll
 0002:00000380       __imp_?createDirectory@GUrlUtils@U2@@SA?AVQString@@ABV3@0AAVU2OpStatus@2@@Z 10021380     U2Core:U2Core.dll
 0002:00000384       __imp_?rollFileName@GUrlUtils@U2@@SA?AVQString@@ABV3@0ABV?$QSet@VQString@@@@@Z 10021384     U2Core:U2Core.dll
 0002:00000388       __imp_?ensureFileExt@GUrlUtils@U2@@SA?AVGUrl@2@ABV32@ABVQStringList@@@Z 10021388     U2Core:U2Core.dll
 0002:0000038c       __imp_?createWorkingDir@FileAndDirectoryUtils@U2@@SA?AVQString@@ABV3@H00@Z 1002138c     U2Core:U2Core.dll
 0002:00000390       __imp_??1GUrl@U2@@QAE@XZ   10021390     U2Core:U2Core.dll
 0002:00000394       __imp_??0GUrl@U2@@QAE@ABVQString@@@Z 10021394     U2Core:U2Core.dll
 0002:00000398       __imp_??1FailTask@U2@@UAE@XZ 10021398     U2Core:U2Core.dll
 0002:0000039c       __imp_??0FailTask@U2@@QAE@ABVQString@@@Z 1002139c     U2Core:U2Core.dll
 0002:000003a0       __imp_?hasError@Task@U2@@QBE_NXZ 100213a0     U2Core:U2Core.dll
 0002:000003a4       __imp_??1TaskStateInfo@U2@@UAE@XZ 100213a4     U2Core:U2Core.dll
 0002:000003a8       __imp_?setError@TaskStateInfo@U2@@UAEXABVQString@@@Z 100213a8     U2Core:U2Core.dll
 0002:000003ac       __imp_?getError@TaskStateInfo@U2@@UBE?AVQString@@XZ 100213ac     U2Core:U2Core.dll
 0002:000003b0       __imp_??0TaskStateInfo@U2@@QAE@XZ 100213b0     U2Core:U2Core.dll
 0002:000003b4       __imp_?isCoR@U2OpStatus@U2@@UBE_NXZ 100213b4     U2Core:U2Core.dll
 0002:000003b8       __imp_?error@Logger@U2@@QAEXABVQString@@@Z 100213b8     U2Core:U2Core.dll
 0002:000003bc       __imp_?getDataPathByName@U2DataPathRegistry@U2@@QAEPAVU2DataPath@2@ABVQString@@@Z 100213bc     U2Core:U2Core.dll
 0002:000003c0       __imp_?getPathByName@U2DataPath@U2@@QBE?AVQString@@ABV3@@Z 100213c0     U2Core:U2Core.dll
 0002:000003c4       __imp_?isValid@U2DataPath@U2@@QBE_NXZ 100213c4     U2Core:U2Core.dll
 0002:000003c8       __imp_?getDataPathRegistry@AppContext@U2@@SAPAVU2DataPathRegistry@2@XZ 100213c8     U2Core:U2Core.dll
 0002:000003cc       __imp_??_7SimpleEventCounter@U2@@6B@ 100213cc     U2Core:U2Core.dll
 0002:000003d0       __imp_?setReportingSupported@Task@U2@@UAEX_N@Z 100213d0     U2Core:U2Core.dll
 0002:000003d4       __imp_?setReportingEnabled@Task@U2@@UAEX_N@Z 100213d4     U2Core:U2Core.dll
 0002:000003d8       __imp_?setNotificationReport@Task@U2@@UAEX_N@Z 100213d8     U2Core:U2Core.dll
 0002:000003dc       __imp_??1ExternalToolLogParser@U2@@UAE@XZ 100213dc     U2Core:U2Core.dll
 0002:000003e0       __imp_?setNoAutoDelete@Task@U2@@UAEX_N@Z 100213e0     U2Core:U2Core.dll
 0002:000003e4       __imp_?setListenerForTask@ExternalToolSupportTask@U2@@MAEXPAVExternalToolRunTask@2@H@Z 100213e4     U2Core:U2Core.dll
 0002:000003e8       __imp_?setListenerForHelper@ExternalToolSupportTask@U2@@MAEXPAVExternalToolRunTaskHelper@2@H@Z 100213e8     U2Core:U2Core.dll
 0002:000003ec       __imp_?setLastError@ExternalToolLogParser@U2@@MAEXABVQString@@@Z 100213ec     U2Core:U2Core.dll
 0002:000003f0       __imp_?setCollectChildrensWarningsFlag@Task@U2@@UAEX_N@Z 100213f0     U2Core:U2Core.dll
 0002:000003f4       __imp_?run@Task@U2@@UAEXXZ 100213f4     U2Core:U2Core.dll
 0002:000003f8       __imp_?run@ExternalToolRunTask@U2@@UAEXXZ 100213f8     U2Core:U2Core.dll
 0002:000003fc       __imp_?report@Task@U2@@UAE?AW4ReportResult@12@XZ 100213fc     U2Core:U2Core.dll
 0002:00000400       __imp_?qt_metacast@ExternalToolRunTask@U2@@UAEPAXPBD@Z 10021400     U2Core:U2Core.dll
 0002:00000404       __imp_?qt_metacast@ExternalToolLogParser@U2@@UAEPAXPBD@Z 10021404     U2Core:U2Core.dll
 0002:00000408       __imp_?qt_metacall@ExternalToolRunTask@U2@@UAEHW4Call@QMetaObject@@HPAPAX@Z 10021408     U2Core:U2Core.dll
 0002:0000040c       __imp_?qt_metacall@ExternalToolLogParser@U2@@UAEHW4Call@QMetaObject@@HPAPAX@Z 1002140c     U2Core:U2Core.dll
 0002:00000410       __imp_?propagateSubtaskError@Task@U2@@UAE_NXZ 10021410     U2Core:U2Core.dll
 0002:00000414       __imp_?processLine@ExternalToolLogParser@U2@@MAEXABVQString@@@Z 10021414     U2Core:U2Core.dll
 0002:00000418       __imp_?processErrLine@ExternalToolLogParser@U2@@MAEXABVQString@@@Z 10021418     U2Core:U2Core.dll
 0002:0000041c       __imp_?prepare@Task@U2@@UAEXXZ 1002141c     U2Core:U2Core.dll
 0002:00000420       __imp_?parseOutput@ExternalToolLogParser@U2@@UAEXABVQString@@@Z 10021420     U2Core:U2Core.dll
 0002:00000424       __imp_?parseErrOutput@ExternalToolLogParser@U2@@UAEXABVQString@@@Z 10021424     U2Core:U2Core.dll
 0002:00000428       __imp_?onSubTaskFinished@Task@U2@@MAE?AV?$QList@PAVTask@U2@@@@PAV12@@Z 10021428     U2Core:U2Core.dll
 0002:0000042c       __imp_?metaObject@ExternalToolRunTask@U2@@UBEPBUQMetaObject@@XZ 1002142c     U2Core:U2Core.dll
 0002:00000430       __imp_??0Logger@U2@@QAE@ABVQString@@@Z 10021430     U2Core:U2Core.dll
 0002:00000434       __imp_?metaObject@ExternalToolLogParser@U2@@UBEPBUQMetaObject@@XZ 10021434     U2Core:U2Core.dll
 0002:00000438       __imp_?isTopLevelTask@Task@U2@@UBE_NXZ 10021438     U2Core:U2Core.dll
 0002:0000043c       __imp_?isReportingSupported@Task@U2@@UBE_NXZ 1002143c     U2Core:U2Core.dll
 0002:00000440       __imp_?isReportingEnabled@Task@U2@@UBE_NXZ 10021440     U2Core:U2Core.dll
 0002:00000444       __imp_?isNotificationReport@Task@U2@@UBE_NXZ 10021444     U2Core:U2Core.dll
 0002:00000448       __imp_?isError@ExternalToolLogParser@U2@@MBE_NABVQString@@@Z 10021448     U2Core:U2Core.dll
 0002:0000044c       __imp_?hasWarning@Task@U2@@UBE_NXZ 1002144c     U2Core:U2Core.dll
 0002:00000450       __imp_?hasSubtasksWithErrors@Task@U2@@UBE_NXZ 10021450     U2Core:U2Core.dll
 0002:00000454       __imp_?getWarnings@Task@U2@@UBE?AVQStringList@@XZ 10021454     U2Core:U2Core.dll
 0002:00000458       __imp_?getTopLevelParentTask@Task@U2@@UAEPAV12@XZ 10021458     U2Core:U2Core.dll
 0002:0000045c       __imp_?getTaskId@Task@U2@@UBE_JXZ 1002145c     U2Core:U2Core.dll
 0002:00000460       __imp_?getSubtaskWithErrors@Task@U2@@UBEPAV12@XZ 10021460     U2Core:U2Core.dll
 0002:00000464       __imp_?getProgress@ExternalToolLogParser@U2@@UAEHXZ 10021464     U2Core:U2Core.dll
 0002:00000468       __imp_?getParentTask@Task@U2@@UBEPAV12@XZ 10021468     U2Core:U2Core.dll
 0002:0000046c       __imp_?getNumParallelSubtasks@Task@U2@@UBEHXZ 1002146c     U2Core:U2Core.dll
 0002:00000470       __imp_?generateReport@Task@U2@@UBE?AVQString@@XZ 10021470     U2Core:U2Core.dll
 0002:00000474       __imp_?cleanup@Task@U2@@UAEXXZ 10021474     U2Core:U2Core.dll
 0002:00000478       \177U2Core_NULL_THUNK_DATA 10021478     U2Core:U2Core.dll
 0002:0000047c       __imp_??0DoubleSpinBoxDelegate@U2@@QAE@ABV?$QMap@VQString@@VQVariant@@@@PAVQObject@@@Z 1002147c     U2Designer:U2Designer.dll
 0002:00000480       __imp_?setModelData@SpinBoxDelegate@U2@@UBEXPAVQWidget@@PAVQAbstractItemModel@@ABVQModelIndex@@@Z 10021480     U2Designer:U2Designer.dll
 0002:00000484       __imp_?setModelData@DoubleSpinBoxDelegate@U2@@UBEXPAVQWidget@@PAVQAbstractItemModel@@ABVQModelIndex@@@Z 10021484     U2Designer:U2Designer.dll
 0002:00000488       __imp_?setModelData@ComboBoxDelegate@U2@@UBEXPAVQWidget@@PAVQAbstractItemModel@@ABVQModelIndex@@@Z 10021488     U2Designer:U2Designer.dll
 0002:0000048c       __imp_?setEditorData@SpinBoxDelegate@U2@@UBEXPAVQWidget@@ABVQModelIndex@@@Z 1002148c     U2Designer:U2Designer.dll
 0002:00000490       __imp_?setEditorData@DoubleSpinBoxDelegate@U2@@UBEXPAVQWidget@@ABVQModelIndex@@@Z 10021490     U2Designer:U2Designer.dll
 0002:00000494       __imp_?setEditorData@ComboBoxDelegate@U2@@UBEXPAVQWidget@@ABVQModelIndex@@@Z 10021494     U2Designer:U2Designer.dll
 0002:00000498       __imp_?qt_metacast@SpinBoxDelegate@U2@@UAEPAXPBD@Z 10021498     U2Designer:U2Designer.dll
 0002:0000049c       __imp_??0DelegateEditor@U2@@QAE@ABV?$QMap@VQString@@PAVPropertyDelegate@U2@@@@@Z 1002149c     U2Designer:U2Designer.dll
 0002:000004a0       __imp_??1DelegateEditor@U2@@UAE@XZ 100214a0     U2Designer:U2Designer.dll
 0002:000004a4       __imp_??0URLDelegate@U2@@QAE@ABVDelegateTags@1@ABVQString@@ABV?$QFlags@W4Option@URLDelegate@U2@@@@PAVQObject@@@Z 100214a4     U2Designer:U2Designer.dll
 0002:000004a8       __imp_??1URLDelegate@U2@@UAE@XZ 100214a8     U2Designer:U2Designer.dll
 0002:000004ac       __imp_?addDelegate@DelegateEditor@U2@@UAEXPAVPropertyDelegate@2@ABVQString@@@Z 100214ac     U2Designer:U2Designer.dll
 0002:000004b0       __imp_?clone@DelegateEditor@U2@@UAEPAVConfigurationEditor@2@XZ 100214b0     U2Designer:U2Designer.dll
 0002:000004b4       __imp_?clone@URLDelegate@U2@@UAEPAVPropertyDelegate@2@XZ 100214b4     U2Designer:U2Designer.dll
 0002:000004b8       __imp_?commit@DelegateEditor@U2@@UAEXXZ 100214b8     U2Designer:U2Designer.dll
 0002:000004bc       __imp_?createEditor@URLDelegate@U2@@UBEPAVQWidget@@PAV3@ABVQStyleOptionViewItem@@ABVQModelIndex@@@Z 100214bc     U2Designer:U2Designer.dll
 0002:000004c0       __imp_?createWizardWidget@URLDelegate@U2@@UBEPAVPropertyWidget@2@AAVU2OpStatus@2@PAVQWidget@@@Z 100214c0     U2Designer:U2Designer.dll
 0002:000004c4       __imp_?getDelegate@DelegateEditor@U2@@UAEPAVPropertyDelegate@2@ABVQString@@@Z 100214c4     U2Designer:U2Designer.dll
 0002:000004c8       __imp_?getDisplayValue@URLDelegate@U2@@UBE?AVQVariant@@ABV3@@Z 100214c8     U2Designer:U2Designer.dll
 0002:000004cc       __imp_?metaObject@DelegateEditor@U2@@UBEPBUQMetaObject@@XZ 100214cc     U2Designer:U2Designer.dll
 0002:000004d0       __imp_?metaObject@URLDelegate@U2@@UBEPBUQMetaObject@@XZ 100214d0     U2Designer:U2Designer.dll
 0002:000004d4       __imp_?qt_metacall@DelegateEditor@U2@@UAEHW4Call@QMetaObject@@HPAPAX@Z 100214d4     U2Designer:U2Designer.dll
 0002:000004d8       __imp_?qt_metacall@URLDelegate@U2@@UAEHW4Call@QMetaObject@@HPAPAX@Z 100214d8     U2Designer:U2Designer.dll
 0002:000004dc       __imp_?qt_metacast@DelegateEditor@U2@@UAEPAXPBD@Z 100214dc     U2Designer:U2Designer.dll
 0002:000004e0       __imp_?qt_metacast@URLDelegate@U2@@UAEPAXPBD@Z 100214e0     U2Designer:U2Designer.dll
 0002:000004e4       __imp_?removeDelegate@DelegateEditor@U2@@UAEPAVPropertyDelegate@2@ABVQString@@@Z 100214e4     U2Designer:U2Designer.dll
 0002:000004e8       __imp_?setEditorData@URLDelegate@U2@@UBEXPAVQWidget@@ABVQModelIndex@@@Z 100214e8     U2Designer:U2Designer.dll
 0002:000004ec       __imp_?setModelData@URLDelegate@U2@@UBEXPAVQWidget@@PAVQAbstractItemModel@@ABVQModelIndex@@@Z 100214ec     U2Designer:U2Designer.dll
 0002:000004f0       __imp_?type@URLDelegate@U2@@UBE?AW4Type@PropertyDelegate@2@XZ 100214f0     U2Designer:U2Designer.dll
 0002:000004f4       __imp_?updateDelegate@DelegateEditor@U2@@UAEXABVQString@@@Z 100214f4     U2Designer:U2Designer.dll
 0002:000004f8       __imp_?updateDelegates@DelegateEditor@U2@@UAEXXZ 100214f8     U2Designer:U2Designer.dll
 0002:000004fc       __imp_??0URLDelegate@U2@@QAE@ABVDelegateTags@1@ABVQString@@_N22PAVQObject@@2@Z 100214fc     U2Designer:U2Designer.dll
 0002:00000500       __imp_??0SpinBoxDelegate@U2@@QAE@ABV?$QMap@VQString@@VQVariant@@@@PAVQObject@@@Z 10021500     U2Designer:U2Designer.dll
 0002:00000504       __imp_??1SpinBoxDelegate@U2@@UAE@XZ 10021504     U2Designer:U2Designer.dll
 0002:00000508       __imp_??1DoubleSpinBoxDelegate@U2@@UAE@XZ 10021508     U2Designer:U2Designer.dll
 0002:0000050c       __imp_??0ComboBoxDelegate@U2@@QAE@ABV?$QMap@VQString@@VQVariant@@@@PAVQObject@@@Z 1002150c     U2Designer:U2Designer.dll
 0002:00000510       __imp_??0ComboBoxDelegate@U2@@QAE@ABV?$QList@U?$QPair@VQString@@VQVariant@@@@@@PAVQObject@@@Z 10021510     U2Designer:U2Designer.dll
 0002:00000514       __imp_??1ComboBoxDelegate@U2@@UAE@XZ 10021514     U2Designer:U2Designer.dll
 0002:00000518       __imp_?clone@ComboBoxDelegate@U2@@UAEPAVPropertyDelegate@2@XZ 10021518     U2Designer:U2Designer.dll
 0002:0000051c       __imp_?clone@DoubleSpinBoxDelegate@U2@@UAEPAVPropertyDelegate@2@XZ 1002151c     U2Designer:U2Designer.dll
 0002:00000520       __imp_?clone@SpinBoxDelegate@U2@@UAEPAVPropertyDelegate@2@XZ 10021520     U2Designer:U2Designer.dll
 0002:00000524       __imp_?createEditor@ComboBoxDelegate@U2@@UBEPAVQWidget@@PAV3@ABVQStyleOptionViewItem@@ABVQModelIndex@@@Z 10021524     U2Designer:U2Designer.dll
 0002:00000528       __imp_?createEditor@DoubleSpinBoxDelegate@U2@@UBEPAVQWidget@@PAV3@ABVQStyleOptionViewItem@@ABVQModelIndex@@@Z 10021528     U2Designer:U2Designer.dll
 0002:0000052c       __imp_?createEditor@SpinBoxDelegate@U2@@UBEPAVQWidget@@PAV3@ABVQStyleOptionViewItem@@ABVQModelIndex@@@Z 1002152c     U2Designer:U2Designer.dll
 0002:00000530       __imp_?createWizardWidget@ComboBoxDelegate@U2@@UBEPAVPropertyWidget@2@AAVU2OpStatus@2@PAVQWidget@@@Z 10021530     U2Designer:U2Designer.dll
 0002:00000534       __imp_?createWizardWidget@DoubleSpinBoxDelegate@U2@@UBEPAVPropertyWidget@2@AAVU2OpStatus@2@PAVQWidget@@@Z 10021534     U2Designer:U2Designer.dll
 0002:00000538       __imp_?createWizardWidget@SpinBoxDelegate@U2@@UBEPAVPropertyWidget@2@AAVU2OpStatus@2@PAVQWidget@@@Z 10021538     U2Designer:U2Designer.dll
 0002:0000053c       __imp_?getDisplayValue@ComboBoxDelegate@U2@@UBE?AVQVariant@@ABV3@@Z 1002153c     U2Designer:U2Designer.dll
 0002:00000540       __imp_?getDisplayValue@DoubleSpinBoxDelegate@U2@@UBE?AVQVariant@@ABV3@@Z 10021540     U2Designer:U2Designer.dll
 0002:00000544       __imp_?getDisplayValue@SpinBoxDelegate@U2@@UBE?AVQVariant@@ABV3@@Z 10021544     U2Designer:U2Designer.dll
 0002:00000548       __imp_?getItems@ComboBoxDelegate@U2@@UBEXAAV?$QMap@VQString@@VQVariant@@@@@Z 10021548     U2Designer:U2Designer.dll
 0002:0000054c       __imp_?getItems@DoubleSpinBoxDelegate@U2@@UBEXAAV?$QMap@VQString@@VQVariant@@@@@Z 1002154c     U2Designer:U2Designer.dll
 0002:00000550       __imp_?getItems@SpinBoxDelegate@U2@@UBEXAAV?$QMap@VQString@@VQVariant@@@@@Z 10021550     U2Designer:U2Designer.dll
 0002:00000554       __imp_?metaObject@ComboBoxDelegate@U2@@UBEPBUQMetaObject@@XZ 10021554     U2Designer:U2Designer.dll
 0002:00000558       __imp_?metaObject@DoubleSpinBoxDelegate@U2@@UBEPBUQMetaObject@@XZ 10021558     U2Designer:U2Designer.dll
 0002:0000055c       __imp_?metaObject@SpinBoxDelegate@U2@@UBEPBUQMetaObject@@XZ 1002155c     U2Designer:U2Designer.dll
 0002:00000560       __imp_?qt_metacall@ComboBoxDelegate@U2@@UAEHW4Call@QMetaObject@@HPAPAX@Z 10021560     U2Designer:U2Designer.dll
 0002:00000564       __imp_?qt_metacall@DoubleSpinBoxDelegate@U2@@UAEHW4Call@QMetaObject@@HPAPAX@Z 10021564     U2Designer:U2Designer.dll
 0002:00000568       __imp_?qt_metacall@SpinBoxDelegate@U2@@UAEHW4Call@QMetaObject@@HPAPAX@Z 10021568     U2Designer:U2Designer.dll
 0002:0000056c       __imp_?qt_metacast@ComboBoxDelegate@U2@@UAEPAXPBD@Z 1002156c     U2Designer:U2Designer.dll
 0002:00000570       __imp_?qt_metacast@DoubleSpinBoxDelegate@U2@@UAEPAXPBD@Z 10021570     U2Designer:U2Designer.dll
 0002:00000574       \177U2Designer_NULL_THUNK_DATA 10021574     U2Designer:U2Designer.dll
 0002:00000578       __imp_?init@StreamShortReadWriter@U2@@QAE_NABVGUrl@2@@Z 10021578     U2Formats:U2Formats.dll
 0002:0000057c       __imp_??1StreamShortReadWriter@U2@@UAE@XZ 1002157c     U2Formats:U2Formats.dll
 0002:00000580       __imp_?getNextSequenceObject@StreamSequenceReader@U2@@QAEPAVDNASequence@2@XZ 10021580     U2Formats:U2Formats.dll
 0002:00000584       __imp_?getErrorMessage@StreamSequenceReader@U2@@QAE?AVQString@@XZ 10021584     U2Formats:U2Formats.dll
 0002:00000588       __imp_?hasNext@StreamSequenceReader@U2@@QAE_NXZ 10021588     U2Formats:U2Formats.dll
 0002:0000058c       __imp_?init@StreamSequenceReader@U2@@QAE_NABVQStringList@@@Z 1002158c     U2Formats:U2Formats.dll
 0002:00000590       __imp_??0StreamSequenceReader@U2@@QAE@XZ 10021590     U2Formats:U2Formats.dll
 0002:00000594       __imp_?writeNextSequence@StreamShortReadWriter@U2@@QAE_NABVDNASequence@2@@Z 10021594     U2Formats:U2Formats.dll
 0002:00000598       __imp_??0StreamGzippedShortReadWriter@U2@@QAE@XZ 10021598     U2Formats:U2Formats.dll
 0002:0000059c       __imp_??1StreamGzippedShortReadWriter@U2@@UAE@XZ 1002159c     U2Formats:U2Formats.dll
 0002:000005a0       __imp_??1StreamSequenceReader@U2@@UAE@XZ 100215a0     U2Formats:U2Formats.dll
 0002:000005a4       \177U2Formats_NULL_THUNK_DATA 100215a4     U2Formats:U2Formats.dll
 0002:000005a8       __imp_?prepareFileFilter@DialogUtils@U2@@SA?AVQString@@ABV3@ABVQStringList@@_N1@Z 100215a8     U2Gui:U2Gui.dll
 0002:000005ac       __imp_?prepareDocumentsFileFilter@DialogUtils@U2@@SA?AVQString@@ABV3@_NABVQStringList@@@Z 100215ac     U2Gui:U2Gui.dll
 0002:000005b0       \177U2Gui_NULL_THUNK_DATA  100215b0     U2Gui:U2Gui.dll
 0002:000005b4       __imp_?getProducersOrUnset@PrompterBaseImpl@U2@@QAE?AVQString@@ABV3@0@Z 100215b4     U2Lang:U2Lang.dll
 0002:000005b8       __imp_?ID@LocalDomainFactory@LocalWorkflow@U2@@2VQString@@B 100215b8     U2Lang:U2Lang.dll
 0002:000005bc       __imp_??_7ActorValidator@Workflow@U2@@6B@ 100215bc     U2Lang:U2Lang.dll
 0002:000005c0       __imp_??_7ConfigurationValidator@U2@@6B@ 100215c0     U2Lang:U2Lang.dll
 0002:000005c4       __imp_?FILTER@DelegateTags@U2@@2VQString@@B 100215c4     U2Lang:U2Lang.dll
 0002:000005c8       __imp_?validate@Attribute@U2@@UAE_NAAV?$QList@VWorkflowNotification@U2@@@@@Z 100215c8     U2Lang:U2Lang.dll
 0002:000005cc       __imp_?validate@ActorValidator@Workflow@U2@@UBE_NPBVConfiguration@3@AAV?$QList@VWorkflowNotification@U2@@@@@Z 100215cc     U2Lang:U2Lang.dll
 0002:000005d0       __imp_?updateActorIds@Attribute@U2@@UAEXABV?$QMap@VQString@@V1@@@@Z 100215d0     U2Lang:U2Lang.dll
 0002:000005d4       __imp_?update@PropertyDelegate@U2@@UAEXXZ 100215d4     U2Lang:U2Lang.dll
 0002:000005d8       __imp_?unregisterEntry@?$IdRegistry@VDomainFactory@Workflow@U2@@@U2@@UAEPAVDomainFactory@Workflow@2@ABVQString@@@Z 100215d8     U2Lang:U2Lang.dll
 0002:000005dc       __imp_?setVisibleSlot@PortDescriptor@Workflow@U2@@UAEXABVQString@@_N@Z 100215dc     U2Lang:U2Lang.dll
 0002:000005e0       __imp_?setAttributeValue@Attribute@U2@@UAEXABVQVariant@@@Z 100215e0     U2Lang:U2Lang.dll
 0002:000005e4       __imp_?registerEntry@?$IdRegistry@VDomainFactory@Workflow@U2@@@U2@@UAE_NPAVDomainFactory@Workflow@2@@Z 100215e4     U2Lang:U2Lang.dll
 0002:000005e8       __imp_?kind@MapDataType@U2@@UBE?AW4Kind@DataType@2@XZ 100215e8     U2Lang:U2Lang.dll
 0002:000005ec       __imp_?isEmpty@ConfigurationEditor@U2@@UBE_NXZ 100215ec     U2Lang:U2Lang.dll
 0002:000005f0       __imp_?isEmpty@Attribute@U2@@UBE_NXZ 100215f0     U2Lang:U2Lang.dll
 0002:000005f4       __imp_?isDefaultValue@Attribute@U2@@UBE_NXZ 100215f4     U2Lang:U2Lang.dll
 0002:000005f8       __imp_?isAcceptableDrop@ActorPrototype@Workflow@U2@@UBE_NPBVQMimeData@@PAV?$QMap@VQString@@VQVariant@@@@@Z 100215f8     U2Lang:U2Lang.dll
 0002:000005fc       __imp_?getWidget@ConfigurationEditor@U2@@UAEPAVQWidget@@XZ 100215fc     U2Lang:U2Lang.dll
 0002:00000600       __imp_?getType@PortDescriptor@Workflow@U2@@UBE?AV?$QExplicitlySharedDataPointer@VDataType@U2@@@@XZ 10021600     U2Lang:U2Lang.dll
 0002:00000604       __imp_?getItems@PropertyDelegate@U2@@UBEXAAV?$QMap@VQString@@VQVariant@@@@@Z 10021604     U2Lang:U2Lang.dll
 0002:00000608       __imp_?getGroup@Attribute@U2@@UAE?AW4AttributeGroup@2@XZ 10021608     U2Lang:U2Lang.dll
 0002:0000060c       __imp_?getDefaultPureValue@Attribute@U2@@UBEABVQVariant@@XZ 1002160c     U2Lang:U2Lang.dll
 0002:00000610       __imp_?getDatatypesMap@MapDataType@U2@@UBE?AV?$QMap@VDescriptor@U2@@V?$QExplicitlySharedDataPointer@VDataType@U2@@@@@@XZ 10021610     U2Lang:U2Lang.dll
 0002:00000614       __imp_?getDatatypeByDescriptor@MapDataType@U2@@UBE?AV?$QExplicitlySharedDataPointer@VDataType@U2@@@@ABVDescriptor@2@@Z 10021614     U2Lang:U2Lang.dll
 0002:00000618       __imp_?getMetadataId@Message@Workflow@U2@@QBEHXZ 10021618     U2Lang:U2Lang.dll
 0002:0000061c       __imp_?getAttributePureValue@Attribute@U2@@UBEABVQVariant@@XZ 1002161c     U2Lang:U2Lang.dll
 0002:00000620       __imp_?getAllIds@?$IdRegistry@VDomainFactory@Workflow@U2@@@U2@@UBE?AV?$QList@VQString@@@@XZ 10021620     U2Lang:U2Lang.dll
 0002:00000624       __imp_?getAllEntries@?$IdRegistry@VDomainFactory@Workflow@U2@@@U2@@UBE?AV?$QList@PAVDomainFactory@Workflow@U2@@@@XZ 10021624     U2Lang:U2Lang.dll
 0002:00000628       __imp_?getAllDescriptors@MapDataType@U2@@UBE?AV?$QList@VDescriptor@U2@@@@XZ 10021628     U2Lang:U2Lang.dll
 0002:0000062c       __imp_?createScheduler@DomainFactory@Workflow@U2@@UAEPAVScheduler@23@PAVSchema@23@@Z 1002162c     U2Lang:U2Lang.dll
 0002:00000630       __imp_?createPort@IntegralBusActorPrototype@Workflow@U2@@UAEPAVPort@23@ABVPortDescriptor@23@PAVActor@23@@Z 10021630     U2Lang:U2Lang.dll
 0002:00000634       __imp_?createInstance@ActorPrototype@Workflow@U2@@UAEPAVActor@23@ABVQString@@PAVAttributeScript@3@ABV?$QMap@VQString@@VQVariant@@@@@Z 10021634     U2Lang:U2Lang.dll
 0002:00000638       __imp_?createConnection@DomainFactory@Workflow@U2@@UAEPAVCommunicationChannel@23@PAVLink@23@@Z 10021638     U2Lang:U2Lang.dll
 0002:0000063c       __imp_?clone@Attribute@U2@@UAEPAV12@XZ 1002163c     U2Lang:U2Lang.dll
 0002:00000640       __imp_??1DomainFactory@Workflow@U2@@UAE@XZ 10021640     U2Lang:U2Lang.dll
 0002:00000644       __imp_??0DomainFactory@Workflow@U2@@QAE@ABVQString@@@Z 10021644     U2Lang:U2Lang.dll
 0002:00000648       __imp_?getInstance@WorkflowEnv@Workflow@U2@@KAPAV123@XZ 10021648     U2Lang:U2Lang.dll
 0002:0000064c       __imp_?URL_DATASETS_TYPE@BaseTypes@U2@@SA?AV?$QExplicitlySharedDataPointer@VDataType@U2@@@@XZ 1002164c     U2Lang:U2Lang.dll
 0002:00000650       __imp_?STRING_TYPE@BaseTypes@U2@@SA?AV?$QExplicitlySharedDataPointer@VDataType@U2@@@@XZ 10021650     U2Lang:U2Lang.dll
 0002:00000654       __imp_?unregisterProto@ActorPrototypeRegistry@Workflow@U2@@QAEPAVActorPrototype@23@ABVQString@@@Z 10021654     U2Lang:U2Lang.dll
 0002:00000658       __imp_?registerProto@ActorPrototypeRegistry@Workflow@U2@@QAEXABVDescriptor@3@PAVActorPrototype@23@@Z 10021658     U2Lang:U2Lang.dll
 0002:0000065c       __imp_?addExternalTool@ActorPrototype@Workflow@U2@@QAEXABVQString@@0@Z 1002165c     U2Lang:U2Lang.dll
 0002:00000660       __imp_?setPrompter@ActorPrototype@Workflow@U2@@QAEXPAVPrompter@23@@Z 10021660     U2Lang:U2Lang.dll
 0002:00000664       __imp_?setValidator@ActorPrototype@Workflow@U2@@QAEXPAVConfigurationValidator@3@@Z 10021664     U2Lang:U2Lang.dll
 0002:00000668       __imp_?setEditor@ActorPrototype@Workflow@U2@@QAEXPAVConfigurationEditor@3@@Z 10021668     U2Lang:U2Lang.dll
 0002:0000066c       __imp_??1ActorPrototype@Workflow@U2@@UAE@XZ 1002166c     U2Lang:U2Lang.dll
 0002:00000670       __imp_??0ActorPrototype@Workflow@U2@@QAE@ABVDescriptor@2@ABV?$QList@PAVPortDescriptor@Workflow@U2@@@@ABV?$QList@PAVAttribute@U2@@@@@Z 10021670     U2Lang:U2Lang.dll
 0002:00000674       __imp_??1PortDescriptor@Workflow@U2@@UAE@XZ 10021674     U2Lang:U2Lang.dll
 0002:00000678       __imp_??0PortDescriptor@Workflow@U2@@QAE@ABVDescriptor@2@V?$QExplicitlySharedDataPointer@VDataType@U2@@@@_N2I@Z 10021678     U2Lang:U2Lang.dll
 0002:0000067c       __imp_??1DelegateTags@U2@@UAE@XZ 1002167c     U2Lang:U2Lang.dll
 0002:00000680       __imp_?set@DelegateTags@U2@@QAEXABVQString@@ABVQVariant@@@Z 10021680     U2Lang:U2Lang.dll
 0002:00000684       __imp_??0DelegateTags@U2@@QAE@PAVQObject@@@Z 10021684     U2Lang:U2Lang.dll
 0002:00000688       __imp_??1PropertyDelegate@U2@@UAE@XZ 10021688     U2Lang:U2Lang.dll
 0002:0000068c       __imp_??1Attribute@U2@@UAE@XZ 1002168c     U2Lang:U2Lang.dll
 0002:00000690       __imp_??0Attribute@U2@@QAE@ABVDescriptor@1@V?$QExplicitlySharedDataPointer@VDataType@U2@@@@_NABVQVariant@@@Z 10021690     U2Lang:U2Lang.dll
 0002:00000694       __imp_?getFileUrl@MessageMetadata@U2@@QBEABVQString@@XZ 10021694     U2Lang:U2Lang.dll
 0002:00000698       __imp_??0MapDataType@U2@@QAE@ABVDescriptor@1@ABV?$QMap@VDescriptor@U2@@V?$QExplicitlySharedDataPointer@VDataType@U2@@@@@@@Z 10021698     U2Lang:U2Lang.dll
 0002:0000069c       __imp_??0Descriptor@U2@@QAE@ABVQString@@@Z 1002169c     U2Lang:U2Lang.dll
 0002:000006a0       __imp_??0Descriptor@U2@@QAE@ABVQString@@00@Z 100216a0     U2Lang:U2Lang.dll
 0002:000006a4       __imp_?setDone@BaseWorker@LocalWorkflow@U2@@UAEXXZ 100216a4     U2Lang:U2Lang.dll
 0002:000006a8       __imp_?isReady@BaseWorker@LocalWorkflow@U2@@UBE_NXZ 100216a8     U2Lang:U2Lang.dll
 0002:000006ac       __imp_?isDone@BaseWorker@LocalWorkflow@U2@@UBE_NXZ 100216ac     U2Lang:U2Lang.dll
 0002:000006b0       __imp_?getOutputFiles@BaseWorker@LocalWorkflow@U2@@UAE?AVQStringList@@XZ 100216b0     U2Lang:U2Lang.dll
 0002:000006b4       __imp_?getMessageAndSetupScriptValues@BaseWorker@LocalWorkflow@U2@@UAE?AVMessage@Workflow@3@PAVCommunicationChannel@53@@Z 100216b4     U2Lang:U2Lang.dll
 0002:000006b8       __imp_?getCommunication@BaseWorker@LocalWorkflow@U2@@UAEPAVCommunicationChannel@Workflow@3@ABVQString@@@Z 100216b8     U2Lang:U2Lang.dll
 0002:000006bc       __imp_?getActorId@BaseWorker@LocalWorkflow@U2@@UBE?AVQString@@XZ 100216bc     U2Lang:U2Lang.dll
 0002:000006c0       __imp_?canTaskBeCanceled@BaseWorker@LocalWorkflow@U2@@MBE_NPAVTask@3@@Z 100216c0     U2Lang:U2Lang.dll
 0002:000006c4       __imp_?addCommunication@BaseWorker@LocalWorkflow@U2@@UAE_NABVQString@@PAVCommunicationChannel@Workflow@3@@Z 100216c4     U2Lang:U2Lang.dll
 0002:000006c8       __imp_?createLogListeners@BaseWorker@LocalWorkflow@U2@@QAE?AV?$QList@PAVExternalToolListener@U2@@@@H@Z 100216c8     U2Lang:U2Lang.dll
 0002:000006cc       __imp_??1BaseWorker@LocalWorkflow@U2@@UAE@XZ 100216cc     U2Lang:U2Lang.dll
 0002:000006d0       __imp_??0BaseWorker@LocalWorkflow@U2@@QAE@PAVActor@Workflow@2@_N@Z 100216d0     U2Lang:U2Lang.dll
 0002:000006d4       __imp_?getBusType@IntegralBus@Workflow@U2@@QBE?AV?$QExplicitlySharedDataPointer@VDataType@U2@@@@XZ 100216d4     U2Lang:U2Lang.dll
 0002:000006d8       __imp_?isOutUrlAttribute@RFSUtils@U2@@SA_NPAVAttribute@2@PAVActor@Workflow@2@AA_N@Z 100216d8     U2Lang:U2Lang.dll
 0002:000006dc       __imp_?addOutputFile@WorkflowMonitor@Workflow@U2@@QAEXABVQString@@0_N@Z 100216dc     U2Lang:U2Lang.dll
 0002:000006e0       __imp_??1Message@Workflow@U2@@QAE@XZ 100216e0     U2Lang:U2Lang.dll
 0002:000006e4       __imp_??0Message@Workflow@U2@@QAE@V?$QExplicitlySharedDataPointer@VDataType@U2@@@@ABVQVariant@@H@Z 100216e4     U2Lang:U2Lang.dll
 0002:000006e8       __imp_?getScriptVars@AttributeScript@U2@@QBEABV?$QMap@VDescriptor@U2@@VQVariant@@@@XZ 100216e8     U2Lang:U2Lang.dll
 0002:000006ec       __imp_?getScriptText@AttributeScript@U2@@QBEABVQString@@XZ 100216ec     U2Lang:U2Lang.dll
 0002:000006f0       __imp_?isEmpty@AttributeScript@U2@@QBE_NXZ 100216f0     U2Lang:U2Lang.dll
 0002:000006f4       __imp_??1WorkflowScriptEngine@U2@@UAE@XZ 100216f4     U2Lang:U2Lang.dll
 0002:000006f8       __imp_??0WorkflowScriptEngine@U2@@QAE@PAVWorkflowContext@Workflow@1@@Z 100216f8     U2Lang:U2Lang.dll
 0002:000006fc       __imp_?getMetadataStorage@WorkflowContext@Workflow@U2@@QAEAAVMessageMetadataStorage@3@XZ 100216fc     U2Lang:U2Lang.dll
 0002:00000700       __imp_?absolutePath@WorkflowContext@Workflow@U2@@QBE?AVQString@@ABV4@@Z 10021700     U2Lang:U2Lang.dll
 0002:00000704       __imp_?workingDir@WorkflowContext@Workflow@U2@@QBE?AVQString@@XZ 10021704     U2Lang:U2Lang.dll
 0002:00000708       __imp_?getMonitor@WorkflowContext@Workflow@U2@@QAEPAVWorkflowMonitor@23@XZ 10021708     U2Lang:U2Lang.dll
 0002:0000070c       __imp_?put@MessageMetadataStorage@U2@@QAEXABVMessageMetadata@2@@Z 1002170c     U2Lang:U2Lang.dll
 0002:00000710       __imp_??1MessageMetadata@U2@@QAE@XZ 10021710     U2Lang:U2Lang.dll
 0002:00000714       __imp_?getId@MessageMetadata@U2@@QBEHXZ 10021714     U2Lang:U2Lang.dll
 0002:00000718       __imp_??0MessageMetadata@U2@@QAE@ABVQString@@@Z 10021718     U2Lang:U2Lang.dll
 0002:0000071c       __imp_?initEngine@WorkflowScriptLibrary@U2@@SAXPAVWorkflowScriptEngine@2@@Z 1002171c     U2Lang:U2Lang.dll
 0002:00000720       __imp_?getUrls@Dataset@U2@@QBE?AV?$QList@PAVURLContainer@U2@@@@XZ 10021720     U2Lang:U2Lang.dll
 0002:00000724       __imp_??1Dataset@U2@@QAE@XZ 10021724     U2Lang:U2Lang.dll
 0002:00000728       __imp_??0Dataset@U2@@QAE@ABV01@@Z 10021728     U2Lang:U2Lang.dll
 0002:0000072c       __imp_?URL_SLOT@BaseSlots@Workflow@U2@@SA?BVDescriptor@3@XZ 1002172c     U2Lang:U2Lang.dll
 0002:00000730       __imp_??0Descriptor@U2@@QAE@ABV01@@Z 10021730     U2Lang:U2Lang.dll
 0002:00000734       __imp_?getId@Descriptor@U2@@QBE?AVQString@@XZ 10021734     U2Lang:U2Lang.dll
 0002:00000738       __imp_??1Descriptor@U2@@UAE@XZ 10021738     U2Lang:U2Lang.dll
 0002:0000073c       __imp_?U2_ERROR@WorkflowNotification@U2@@2VQString@@B 1002173c     U2Lang:U2Lang.dll
 0002:00000740       __imp_?getId@Actor@Workflow@U2@@QBE?AVQString@@XZ 10021740     U2Lang:U2Lang.dll
 0002:00000744       __imp_??0WorkflowNotification@U2@@QAE@ABV01@@Z 10021744     U2Lang:U2Lang.dll
 0002:00000748       __imp_??1WorkflowNotification@U2@@QAE@XZ 10021748     U2Lang:U2Lang.dll
 0002:0000074c       __imp_??0WorkflowNotification@U2@@QAE@ABVQString@@00@Z 1002174c     U2Lang:U2Lang.dll
 0002:00000750       __imp_?update@PrompterBaseImpl@U2@@UAEXABV?$QMap@VQString@@VQVariant@@@@@Z 10021750     U2Lang:U2Lang.dll
 0002:00000754       __imp_?sl_actorModified@PrompterBaseImpl@U2@@MAEXXZ 10021754     U2Lang:U2Lang.dll
 0002:00000758       __imp_?qt_metacast@PrompterBaseImpl@U2@@UAEPAXPBD@Z 10021758     U2Lang:U2Lang.dll
 0002:0000075c       __imp_?qt_metacall@PrompterBaseImpl@U2@@UAEHW4Call@QMetaObject@@HPAPAX@Z 1002175c     U2Lang:U2Lang.dll
 0002:00000760       __imp_?metaObject@PrompterBaseImpl@U2@@UBEPBUQMetaObject@@XZ 10021760     U2Lang:U2Lang.dll
 0002:00000764       __imp_??1PrompterBaseImpl@U2@@UAE@XZ 10021764     U2Lang:U2Lang.dll
 0002:00000768       __imp_?getHyperlink@PrompterBaseImpl@U2@@SA?AVQString@@ABV3@0@Z 10021768     U2Lang:U2Lang.dll
 0002:0000076c       __imp_?getURL@PrompterBaseImpl@U2@@QAE?AVQString@@ABV3@PA_N00@Z 1002176c     U2Lang:U2Lang.dll
 0002:00000770       __imp_??0PrompterBaseImpl@U2@@QAE@PAVActor@Workflow@1@@Z 10021770     U2Lang:U2Lang.dll
 0002:00000774       __imp_?getOutputPorts@Actor@Workflow@U2@@QBE?AV?$QList@PAVPort@Workflow@U2@@@@XZ 10021774     U2Lang:U2Lang.dll
 0002:00000778       __imp_?getInputPorts@Actor@Workflow@U2@@QBE?AV?$QList@PAVPort@Workflow@U2@@@@XZ 10021778     U2Lang:U2Lang.dll
 0002:0000077c       __imp_?get@MessageMetadataStorage@U2@@QBE?AVMessageMetadata@2@H@Z 1002177c     U2Lang:U2Lang.dll
 0002:00000780       __imp_??1MapDataType@U2@@UAE@XZ 10021780     U2Lang:U2Lang.dll
 0002:00000784       __imp_?getData@Message@Workflow@U2@@QBE?AVQVariant@@XZ 10021784     U2Lang:U2Lang.dll
 0002:00000788       __imp_?addInfo@WorkflowMonitor@Workflow@U2@@QAEXABVQString@@00@Z 10021788     U2Lang:U2Lang.dll
 0002:0000078c       __imp_?U2_INFO@WorkflowNotification@U2@@2VQString@@B 1002178c     U2Lang:U2Lang.dll
 0002:00000790       __imp_??0Attribute@U2@@QAE@ABVDescriptor@1@V?$QExplicitlySharedDataPointer@VDataType@U2@@@@V?$QFlags@W4Flag@Attribute@U2@@@@ABVQVariant@@@Z 10021790     U2Lang:U2Lang.dll
 0002:00000794       __imp_?staticMetaObject@BaseWorker@LocalWorkflow@U2@@2UQMetaObject@@B 10021794     U2Lang:U2Lang.dll
 0002:00000798       __imp_?qt_metacall@BaseWorker@LocalWorkflow@U2@@UAEHW4Call@QMetaObject@@HPAPAX@Z 10021798     U2Lang:U2Lang.dll
 0002:0000079c       __imp_?qt_metacast@BaseWorker@LocalWorkflow@U2@@UAEPAXPBD@Z 1002179c     U2Lang:U2Lang.dll
 0002:000007a0       __imp_?staticMetaObject@PrompterBaseImpl@U2@@2UQMetaObject@@B 100217a0     U2Lang:U2Lang.dll
 0002:000007a4       __imp_?FORMAT@DelegateTags@U2@@2VQString@@B 100217a4     U2Lang:U2Lang.dll
 0002:000007a8       __imp_?PLACEHOLDER_TEXT@DelegateTags@U2@@2VQString@@B 100217a8     U2Lang:U2Lang.dll
 0002:000007ac       __imp_?getById@?$IdRegistry@VDomainFactory@Workflow@U2@@@U2@@UAEPAVDomainFactory@Workflow@2@ABVQString@@@Z 100217ac     U2Lang:U2Lang.dll
 0002:000007b0       __imp_?NUM_TYPE@BaseTypes@U2@@SA?AV?$QExplicitlySharedDataPointer@VDataType@U2@@@@XZ 100217b0     U2Lang:U2Lang.dll
 0002:000007b4       __imp_?type@PropertyDelegate@U2@@UBE?AW4Type@12@XZ 100217b4     U2Lang:U2Lang.dll
 0002:000007b8       __imp_?destroy@DomainFactory@Workflow@U2@@UAEXPAVScheduler@23@PAVSchema@23@@Z 100217b8     U2Lang:U2Lang.dll
 0002:000007bc       \177U2Lang_NULL_THUNK_DATA 100217bc     U2Lang:U2Lang.dll
 0002:000007c0       __imp_?WORKFLOW_CLASSIFY_TOOL_ID@NgsReadsClassificationPlugin@U2@@2VQString@@B 100217c0     ngs_reads_classification:ngs_reads_classification.dll
 0002:000007c4       __imp_?DIAMOND_UNIPROT_90_DATABASE_ITEM_ID@NgsReadsClassificationPlugin@U2@@2VQString@@B 100217c4     ngs_reads_classification:ngs_reads_classification.dll
 0002:000007c8       __imp_?DIAMOND_UNIPROT_90_DATABASE_DATA_ID@NgsReadsClassificationPlugin@U2@@2VQString@@B 100217c8     ngs_reads_classification:ngs_reads_classification.dll
 0002:000007cc       __imp_?DIAMOND_UNIPROT_50_DATABASE_ITEM_ID@NgsReadsClassificationPlugin@U2@@2VQString@@B 100217cc     ngs_reads_classification:ngs_reads_classification.dll
 0002:000007d0       __imp_?DIAMOND_UNIPROT_50_DATABASE_DATA_ID@NgsReadsClassificationPlugin@U2@@2VQString@@B 100217d0     ngs_reads_classification:ngs_reads_classification.dll
 0002:000007d4       __imp_?update@DatabaseDelegate@LocalWorkflow@U2@@UAEXXZ 100217d4     ngs_reads_classification:ngs_reads_classification.dll
 0002:000007d8       __imp_??1DatabaseDelegate@LocalWorkflow@U2@@UAE@XZ 100217d8     ngs_reads_classification:ngs_reads_classification.dll
 0002:000007dc       __imp_??0DatabaseDelegate@LocalWorkflow@U2@@QAE@ABVQString@@0ABV?$QList@U?$QPair@VQString@@V1@@@@@0_N@Z 100217dc     ngs_reads_classification:ngs_reads_classification.dll
 0002:000007e0       __imp_?TAXONOMY_CLASSIFICATION_TYPE@TaxonomySupport@LocalWorkflow@U2@@SA?AV?$QExplicitlySharedDataPointer@VDataType@U2@@@@XZ 100217e0     ngs_reads_classification:ngs_reads_classification.dll
 0002:000007e4       __imp_?TAXONOMY_CLASSIFICATION_SLOT@TaxonomySupport@LocalWorkflow@U2@@SA?BVDescriptor@3@XZ 100217e4     ngs_reads_classification:ngs_reads_classification.dll
 0002:000007e8       __imp_?CLASSIFICATION_SUFFIX@NgsReadsClassificationUtils@U2@@2VQString@@B 100217e8     ngs_reads_classification:ngs_reads_classification.dll
 0002:000007ec       __imp_?TAXONOMY_CLASSIFICATION_SLOT_ID@TaxonomySupport@LocalWorkflow@U2@@2VQString@@B 100217ec     ngs_reads_classification:ngs_reads_classification.dll
 0002:000007f0       __imp_?countClassified@NgsReadsClassificationUtils@U2@@SAHABV?$QMap@VQString@@I@@@Z 100217f0     ngs_reads_classification:ngs_reads_classification.dll
 0002:000007f4       __imp_?getBaseFileNameWithSuffixes@NgsReadsClassificationUtils@U2@@SA?AVQString@@ABV3@ABVQStringList@@0_N@Z 100217f4     ngs_reads_classification:ngs_reads_classification.dll
 0002:000007f8       __imp_?WORKFLOW_ELEMENTS_GROUP@NgsReadsClassificationPlugin@U2@@2VQString@@B 100217f8     ngs_reads_classification:ngs_reads_classification.dll
 0002:000007fc       __imp_?setModelData@GenomicLibraryDelegate@LocalWorkflow@U2@@UBEXPAVQWidget@@PAVQAbstractItemModel@@ABVQModelIndex@@@Z 100217fc     ngs_reads_classification:ngs_reads_classification.dll
 0002:00000800       __imp_?setEditorData@GenomicLibraryDelegate@LocalWorkflow@U2@@UBEXPAVQWidget@@ABVQModelIndex@@@Z 10021800     ngs_reads_classification:ngs_reads_classification.dll
 0002:00000804       __imp_?qt_metacast@GenomicLibraryDelegate@LocalWorkflow@U2@@UAEPAXPBD@Z 10021804     ngs_reads_classification:ngs_reads_classification.dll
 0002:00000808       __imp_?qt_metacall@GenomicLibraryDelegate@LocalWorkflow@U2@@UAEHW4Call@QMetaObject@@HPAPAX@Z 10021808     ngs_reads_classification:ngs_reads_classification.dll
 0002:0000080c       __imp_?metaObject@GenomicLibraryDelegate@LocalWorkflow@U2@@UBEPBUQMetaObject@@XZ 1002180c     ngs_reads_classification:ngs_reads_classification.dll
 0002:00000810       __imp_?getDisplayValue@GenomicLibraryDelegate@LocalWorkflow@U2@@UBE?AVQVariant@@ABV4@@Z 10021810     ngs_reads_classification:ngs_reads_classification.dll
 0002:00000814       __imp_?createWizardWidget@GenomicLibraryDelegate@LocalWorkflow@U2@@UBEPAVPropertyWidget@3@AAVU2OpStatus@3@PAVQWidget@@@Z 10021814     ngs_reads_classification:ngs_reads_classification.dll
 0002:00000818       __imp_?createEditor@GenomicLibraryDelegate@LocalWorkflow@U2@@UBEPAVQWidget@@PAV4@ABVQStyleOptionViewItem@@ABVQModelIndex@@@Z 10021818     ngs_reads_classification:ngs_reads_classification.dll
 0002:0000081c       __imp_?clone@GenomicLibraryDelegate@LocalWorkflow@U2@@UAEPAVPropertyDelegate@3@XZ 1002181c     ngs_reads_classification:ngs_reads_classification.dll
 0002:00000820       __imp_??0GenomicLibraryDelegate@LocalWorkflow@U2@@QAE@PAVQObject@@@Z 10021820     ngs_reads_classification:ngs_reads_classification.dll
 0002:00000824       __imp_?TAXON_PROT_ACCESSION_2_TAXID_ITEM_ID@NgsReadsClassificationPlugin@U2@@2VQString@@B 10021824     ngs_reads_classification:ngs_reads_classification.dll
 0002:00000828       __imp_?TAXON_NODES_ITEM_ID@NgsReadsClassificationPlugin@U2@@2VQString@@B 10021828     ngs_reads_classification:ngs_reads_classification.dll
 0002:0000082c       __imp_?TAXONOMY_DATA_ID@NgsReadsClassificationPlugin@U2@@2VQString@@B 1002182c     ngs_reads_classification:ngs_reads_classification.dll
 0002:00000830       \177ngs_reads_classification_NULL_THUNK_DATA 10021830     ngs_reads_classification:ngs_reads_classification.dll
 0002:00000834       ___xc_a                    10021834     MSVCRT:cinitexe.obj
 0002:00000b90       ___xc_z                    10021b90     MSVCRT:cinitexe.obj
 0002:00000b94       ___xi_a                    10021b94     MSVCRT:cinitexe.obj
 0002:00000ba0       ___xi_z                    10021ba0     MSVCRT:cinitexe.obj
 0002:00000be8       ??_C@_00CNPNBAHC@?$AA@     10021be8     DiamondBuildPrompter.obj
 0002:00000bf0       ??_7error_category@std@@6B@ 10021bf0     DiamondBuildPrompter.obj
 0002:00000c0c       ??_7_Generic_error_category@std@@6B@ 10021c0c     DiamondBuildPrompter.obj
 0002:00000c24       ??_C@_07DCLBNMLN@generic?$AA@ 10021c24     DiamondBuildPrompter.obj
 0002:00000c2c       ??_C@_0O@BFJCFAAK@unknown?5error?$AA@ 10021c2c     DiamondBuildPrompter.obj
 0002:00000c40       ??_7_Iostream_error_category@std@@6B@ 10021c40     DiamondBuildPrompter.obj
 0002:00000c58       ??_C@_08LLGCOLLL@iostream?$AA@ 10021c58     DiamondBuildPrompter.obj
 0002:00000c64       ??_C@_0BG@PADBLCHM@iostream?5stream?5error?$AA@ 10021c64     DiamondBuildPrompter.obj
 0002:00000c80       ??_7_System_error_category@std@@6B@ 10021c80     DiamondBuildPrompter.obj
 0002:00000c98       ??_C@_06FHFOAHML@system?$AA@ 10021c98     DiamondBuildPrompter.obj
 0002:00000ca0       ??_C@_0L@JLHNEGIN@Algorithms?$AA@ 10021ca0     DiamondBuildPrompter.obj
 0002:00000cac       ??_C@_07PGLPGHFC@Console?$AA@ 10021cac     DiamondBuildPrompter.obj
 0002:00000cb4       ??_C@_0O@BOFHOPCF@Core?5Services?$AA@ 10021cb4     DiamondBuildPrompter.obj
 0002:00000cc4       ??_C@_0N@PPADAKBM@Input?1Output?$AA@ 10021cc4     DiamondBuildPrompter.obj
 0002:00000cd4       ??_C@_0M@KPPBKPKK@Performance?$AA@ 10021cd4     DiamondBuildPrompter.obj
 0002:00000ce0       ??_C@_07BFDHHBBI@Scripts?$AA@ 10021ce0     DiamondBuildPrompter.obj
 0002:00000ce8       ??_C@_05EEGKELMG@Tasks?$AA@ 10021ce8     DiamondBuildPrompter.obj
 0002:00000cf0       ??_C@_0P@NIIOBHGA@User?5Interface?$AA@ 10021cf0     DiamondBuildPrompter.obj
 0002:00000d00       ??_C@_0N@JINCGGMN@User?5Actions?$AA@ 10021d00     DiamondBuildPrompter.obj
 0002:00000d14       ??_7?$PrompterBase@VDiamondBuildPrompter@LocalWorkflow@U2@@@U2@@6BActorDocument@Workflow@1@@ 10021d14     DiamondBuildPrompter.obj
 0002:00000d5c       ??_7?$PrompterBase@VDiamondBuildPrompter@LocalWorkflow@U2@@@U2@@6BPrompter@Workflow@1@@ 10021d5c     DiamondBuildPrompter.obj
 0002:00000d68       ??_7DiamondBuildPrompter@LocalWorkflow@U2@@6BActorDocument@Workflow@2@@ 10021d68     DiamondBuildPrompter.obj
 0002:00000db0       ??_7DiamondBuildPrompter@LocalWorkflow@U2@@6BPrompter@Workflow@2@@ 10021db0     DiamondBuildPrompter.obj
 0002:00000db8       ??_C@_0CO@FECPPJED@Use?5custom?5data?5to?5build?5?$CF1?5DIAM@ 10021db8     DiamondBuildPrompter.obj
 0002:00000de8       ??_C@_0BE@LGBLLFOL@1sl_actorModified?$CI?$CJ?$AA@ 10021de8     DiamondBuildPrompter.obj
 0002:00000dfc       ??_C@_0BD@FGIDJNMI@2si_labelChanged?$CI?$CJ?$AA@ 10021dfc     DiamondBuildPrompter.obj
 0002:00000e10       ??_C@_0P@DIBOLHGA@2si_modified?$CI?$CJ?$AA@ 10021e10     DiamondBuildPrompter.obj
 0002:00000e20       ??_C@_0BC@HBGBGNIM@2bindingChanged?$CI?$CJ?$AA@ 10021e20     DiamondBuildPrompter.obj
 0002:00000e34       ??_C@_0BA@JFNIOLAK@string?5too?5long?$AA@ 10021e34     DiamondBuildPrompter.obj
 0002:00000e44       ??_C@_0BI@CFPLBAOH@invalid?5string?5position?$AA@ 10021e44     DiamondBuildPrompter.obj
 0002:00000e64       ??_SExternalToolRunTask@U2@@6B@ 10021e64     DiamondBuildTask.obj
 0002:00000ef4       ??_SExternalToolLogParser@U2@@6B@ 10021ef4     DiamondBuildTask.obj
 0002:00000f40       ??_7DiamondBuildTask@U2@@6B@ 10021f40     DiamondBuildTask.obj
 0002:00000fd4       ??_C@_0BH@OFECGMDJ@Build?5DIAMOND?5database?$AA@ 10021fd4     DiamondBuildTask.obj
 0002:00000fec       ??_C@_0BB@JKHAOHNM@DiamondBuildTask?$AA@ 10021fec     DiamondBuildTask.obj
 0002:00001000       ??_C@_0BI@LGIPEFEA@?1prepared_genomes?4fa?4gz?$AA@ 10022000     DiamondBuildTask.obj
 0002:00001018       ??_C@_0BN@GHDCPDMM@Result?5database?5URL?5is?5empty?$AA@ 10022018     DiamondBuildTask.obj
 0002:00001038       ??_C@_0DD@NEMKMAKL@There?5is?5no?5input?5files?5to?5build@ 10022038     DiamondBuildTask.obj
 0002:0000106c       ??_C@_0BH@KIPCGCFI@Taxon?5map?5URL?5is?5empty?$AA@ 1002206c     DiamondBuildTask.obj
 0002:00001084       ??_C@_0BJ@KHDBPMIM@Taxon?5nodes?5URL?5is?5empty?$AA@ 10022084     DiamondBuildTask.obj
 0002:000010a0       ??_C@_06LBFFPKOP@makedb?$AA@ 100220a0     DiamondBuildTask.obj
 0002:000010a8       ??_C@_04OOKMCCDC@?9?9in?$AA@ 100220a8     DiamondBuildTask.obj
 0002:000010b0       ??_C@_02DBLKFNPN@?9d?$AA@  100220b0     DiamondBuildTask.obj
 0002:000010b4       ??_C@_0L@HNJMCLIP@?9?9taxonmap?$AA@ 100220b4     DiamondBuildTask.obj
 0002:000010c0       ??_C@_0N@LMHGCPKB@?9?9taxonnodes?$AA@ 100220c0     DiamondBuildTask.obj
 0002:000010d0       __real@3ff0000000000000    100220d0     DiamondBuildTask.obj
 0002:000010d8       ??_C@_0BG@GDOLLAJJ@DiamondBuildValidator?$AA@ 100220d8     DiamondBuildValidator.obj
 0002:000010f0       ??_C@_0BL@PLINAGHB@U2DataPathRegistry?5is?5NULL?$AA@ 100220f0     DiamondBuildValidator.obj
 0002:0000110c       ??_C@_0DK@FGLPPHNF@Taxonomy?5classification?5data?5fro@ 1002210c     DiamondBuildValidator.obj
 0002:00001148       ??_C@_0EL@ENMJCHGK@Taxonomy?5classification?5data?5fro@ 10022148     DiamondBuildValidator.obj
 0002:0000119c       ??_SFailTask@U2@@6B@       1002219c     DiamondBuildWorker.obj
 0002:0000122c       ??_STaskSignalMapper@U2@@6B@ 1002222c     DiamondBuildWorker.obj
 0002:0000125c       ??_SDescriptor@U2@@6B@     1002225c     DiamondBuildWorker.obj
 0002:00001260       ??_C@_0BD@FOHBGHEI@QList?$DMU2?3?3Dataset?$DO?$AA@ 10022260     DiamondBuildWorker.obj
 0002:00001274       ??_C@_0BF@COKBMJP@Script?5task?5canceled?$AA@ 10022274     DiamondBuildWorker.obj
 0002:00001290       ??_7DiamondBuildWorker@LocalWorkflow@U2@@6BQObject@@@ 10022290     DiamondBuildWorker.obj
 0002:000012d4       ??_7DiamondBuildWorker@LocalWorkflow@U2@@6BWorker@Workflow@2@@ 100222d4     DiamondBuildWorker.obj
 0002:000012f0       ??_7DiamondBuildWorker@LocalWorkflow@U2@@6BCommunicationSubject@Workflow@2@@ 100222f0     DiamondBuildWorker.obj
 0002:000012fc       ??_C@_0O@FNOJHKLA@diamond_build?$AA@ 100222fc     DiamondBuildWorker.obj
 0002:0000130c       ??_C@_0CK@IGBIANDN@Trying?5to?5recover?5from?5error?3?5?$CF1@ 1002230c     DiamondBuildWorker.obj
 0002:00001338       ??_C@_0BK@LMMJOEHE@Port?5with?5id?5?8?$CF1?8?5is?5NULL?$AA@ 10022338     DiamondBuildWorker.obj
 0002:00001354       ??_C@_0BL@PEBOIBDC@src?2DiamondBuildWorker?4cpp?$AA@ 10022354     DiamondBuildWorker.obj
 0002:00001370       ??_C@_0BJ@JJNIMNNJ@1sl_taskFinished?$CITask?5?$CK?$CJ?$AA@ 10022370     DiamondBuildWorker.obj
 0002:0000138c       ??_C@_0BJ@DHBKDAMN@2si_taskFinished?$CITask?5?$CK?$CJ?$AA@ 1002238c     DiamondBuildWorker.obj
 0002:000013a8       ??_C@_09DMOIMEE@Dataset?51?$AA@ 100223a8     DiamondBuildWorker.obj
 0002:000013b4       ??_C@_04NPPLLODI@dmnd?$AA@ 100223b4     DiamondBuildWorker.obj
 0002:000013bc       ??_C@_01IDAFKMJL@_?$AA@    100223bc     DiamondBuildWorker.obj
 0002:000013c4       ??_SMapDataType@U2@@6B@    100223c4     DiamondBuildWorkerFactory.obj
 0002:000013dc       ??_SAttribute@U2@@6B@      100223dc     DiamondBuildWorkerFactory.obj
 0002:0000140c       ??_SDelegateEditor@U2@@6B@ 1002240c     DiamondBuildWorkerFactory.obj
 0002:00001464       ??_SURLDelegate@U2@@6B@    10022464     DiamondBuildWorkerFactory.obj
 0002:000014e4       ??_SPortDescriptor@Workflow@U2@@6B@ 100224e4     DiamondBuildWorkerFactory.obj
 0002:000014f4       ??_SIntegralBusActorPrototype@Workflow@U2@@6B@ 100224f4     DiamondBuildWorkerFactory.obj
 0002:00001508       ??_7DiamondBuildValidator@Workflow@U2@@6B@ 10022508     DiamondBuildWorkerFactory.obj
 0002:00001518       ??_7DiamondBuildWorkerFactory@LocalWorkflow@U2@@6B?$IdRegistry@VDomainFactory@Workflow@U2@@@2@@ 10022518     DiamondBuildWorkerFactory.obj
 0002:00001544       ??_7DiamondBuildWorkerFactory@LocalWorkflow@U2@@6BDescriptor@2@@ 10022544     DiamondBuildWorkerFactory.obj
 0002:0000154c       ??_SGenomicLibraryDelegate@LocalWorkflow@U2@@6B@ 1002254c     DiamondBuildWorkerFactory.obj
 0002:000015c8       ??_C@_0O@CGBOLLLC@diamond?9build?$AA@ 100225c8     DiamondBuildWorkerFactory.obj
 0002:000015d8       ??_C@_03KEJHNBPP@out?$AA@  100225d8     DiamondBuildWorkerFactory.obj
 0002:000015dc       ??_C@_08PBOCEOLL@database?$AA@ 100225dc     DiamondBuildWorkerFactory.obj
 0002:000015e8       ??_C@_0BA@GJNMLPPF@genomic?9library?$AA@ 100225e8     DiamondBuildWorkerFactory.obj
 0002:000015f8       ??_C@_0M@FOOCJNHH@Output?5URL?4?$AA@ 100225f8     DiamondBuildWorkerFactory.obj
 0002:00001604       ??_C@_0L@OALCHELH@Output?5URL?$AA@ 10022604     DiamondBuildWorkerFactory.obj
 0002:00001610       ??_C@_0CC@MDEIGEIG@URL?5to?5the?5DIAMOND?5database?5file@ 10022610     DiamondBuildWorkerFactory.obj
 0002:00001634       ??_C@_0BI@GJBIOAEE@Output?5DIAMOND?5database?$AA@ 10022634     DiamondBuildWorkerFactory.obj
 0002:0000164c       ??_C@_04HKKABCEL@?9out?$AA@ 1002264c     DiamondBuildWorkerFactory.obj
 0002:00001658       ??_C@_0ED@DKKEAINM@A?5name?5of?5the?5binary?5DIAMOND?5dat@ 10022658     DiamondBuildWorkerFactory.obj
 0002:0000169c       ??_C@_08HDBDMMBI@Database?$AA@ 1002269c     DiamondBuildWorkerFactory.obj
 0002:000016a8       ??_C@_0DD@KOJHFLAJ@Genomes?5that?5should?5be?5used?5to?5b@ 100226a8     DiamondBuildWorkerFactory.obj
 0002:000016dc       ??_C@_0BA@IPKMCDNP@Genomic?5library?$AA@ 100226dc     DiamondBuildWorkerFactory.obj
 0002:000016ec       ??_C@_0BB@OMGPHPEF@DIAMOND?5database?$AA@ 100226ec     DiamondBuildWorkerFactory.obj
 0002:00001700       ??_C@_0BB@EMIKDEND@diamond?1database?$AA@ 10022700     DiamondBuildWorkerFactory.obj
 0002:00001714       ??_C@_0DM@LLKPIOHM@Build?5a?5DIAMOND?5formatted?5databa@ 10022714     DiamondBuildWorkerFactory.obj
 0002:00001750       ??_C@_0BH@GHLDOOJK@Build?5DIAMOND?5Database?$AA@ 10022750     DiamondBuildWorkerFactory.obj
 0002:0000176c       ??_7?$PrompterBase@VDiamondClassifyPrompter@LocalWorkflow@U2@@@U2@@6BActorDocument@Workflow@1@@ 1002276c     DiamondClassifyPrompter.obj
 0002:000017b4       ??_7?$PrompterBase@VDiamondClassifyPrompter@LocalWorkflow@U2@@@U2@@6BPrompter@Workflow@1@@ 100227b4     DiamondClassifyPrompter.obj
 0002:000017c0       ??_7DiamondClassifyPrompter@LocalWorkflow@U2@@6BActorDocument@Workflow@2@@ 100227c0     DiamondClassifyPrompter.obj
 0002:00001808       ??_7DiamondClassifyPrompter@LocalWorkflow@U2@@6BPrompter@Workflow@2@@ 10022808     DiamondClassifyPrompter.obj
 0002:00001810       ??_C@_0EB@PDCLDOO@Classify?5sequences?5from?5?$DMu?$DO?$CF1?$DM?1u@ 10022810     DiamondClassifyPrompter.obj
 0002:00001854       ??_C@_07DLHCIBDH@default?$AA@ 10022854     DiamondClassifyTask.obj
 0002:00001860       ??_7DiamondClassifyTask@U2@@6B@ 10022860     DiamondClassifyTask.obj
 0002:000018f4       ??_C@_05IGNOIJHB@ultra?$AA@ 100228f4     DiamondClassifyTask.obj
 0002:000018fc       ??_C@_04DGANLAON@high?$AA@ 100228fc     DiamondClassifyTask.obj
 0002:00001904       ??_C@_08LHCHCHBK@BLOSUM45?$AA@ 10022904     DiamondClassifyTask.obj
 0002:00001910       ??_C@_08MLJCLJGI@BLOSUM50?$AA@ 10022910     DiamondClassifyTask.obj
 0002:0000191c       ??_C@_08PLOCGFLD@BLOSUM62?$AA@ 1002291c     DiamondClassifyTask.obj
 0002:00001928       ??_C@_08MDEKCKDL@BLOSUM80?$AA@ 10022928     DiamondClassifyTask.obj
 0002:00001934       ??_C@_08MCIIEAAM@BLOSUM90?$AA@ 10022934     DiamondClassifyTask.obj
 0002:00001940       ??_C@_06ICOFKNKF@PAM250?$AA@ 10022940     DiamondClassifyTask.obj
 0002:00001948       ??_C@_05LADMGCFE@PAM70?$AA@ 10022948     DiamondClassifyTask.obj
 0002:00001950       ??_C@_05LHDFMKII@PAM30?$AA@ 10022950     DiamondClassifyTask.obj
 0002:00001958       ??_C@_03FPDHAOMG@102?$AA@  10022958     DiamondClassifyTask.obj
 0002:0000195c       ??_C@_0CA@IJLLKBEJ@Classify?5sequences?5with?5DIAMOND?$AA@ 1002295c     DiamondClassifyTask.obj
 0002:0000197c       ??_C@_0BE@CHOIECLJ@DiamondClassifyTask?$AA@ 1002297c     DiamondClassifyTask.obj
 0002:00001990       ??_C@_0CG@IHMCOLO@Cannot?5open?5classification?5repor@ 10022990     DiamondClassifyTask.obj
 0002:000019b8       ??_C@_0CE@HGOFAKPG@Found?5Diamond?5classification?3?5?$CF1@ 100229b8     DiamondClassifyTask.obj
 0002:000019e0       ??_C@_0EO@GBJCHADO@Duplicate?5sequence?5name?5?8?$CF1?8?5hav@ 100229e0     DiamondClassifyTask.obj
 0002:00001a30       ??_C@_0BL@BANFFFNO@Broken?5Diamond?5report?5?3?5?$CF1?$AA@ 10022a30     DiamondClassifyTask.obj
 0002:00001a4c       ??_C@_0BD@HKKHAEBH@Reads?5URL?5is?5empty?$AA@ 10022a4c     DiamondClassifyTask.obj
 0002:00001a60       ??_C@_0BO@GAADBEEH@DIAMOND?5database?5URL?5is?5empty?$AA@ 10022a60     DiamondClassifyTask.obj
 0002:00001a80       ??_C@_0CE@PKDJHHAD@DIAMOND?5classification?5URL?5is?5em@ 10022a80     DiamondClassifyTask.obj
 0002:00001aa4       ??_C@_0BB@CAFAIHNA@NCBI?9GenBank?5?$CD?$CF1?$AA@ 10022aa4     DiamondClassifyTask.obj
 0002:00001ab8       ??_C@_0BJ@HKONGBAF@Invalid?5genetic?5code?3?5?$CF1?$AA@ 10022ab8     DiamondClassifyTask.obj
 0002:00001ad4       ??_C@_06GIEKNAJB@blastx?$AA@ 10022ad4     DiamondClassifyTask.obj
 0002:00001adc       ??_C@_02DIMDPHP@?9f?$AA@   10022adc     DiamondClassifyTask.obj
 0002:00001ae0       ??_C@_02GAPLLOJ@?9q?$AA@   10022ae0     DiamondClassifyTask.obj
 0002:00001ae4       ??_C@_02NCEOIEDG@?9o?$AA@  10022ae4     DiamondClassifyTask.obj
 0002:00001ae8       ??_C@_0M@HBKGIIAN@?9?9sensitive?$AA@ 10022ae8     DiamondClassifyTask.obj
 0002:00001af4       ??_C@_0BB@GJEKBDOC@?9?9more?9sensitive?$AA@ 10022af4     DiamondClassifyTask.obj
 0002:00001b08       ??_C@_0CI@IHGOGFFN@Unknown?5sensitivity?5value?3?5?$CF1?0?5i@ 10022b08     DiamondClassifyTask.obj
 0002:00001b30       ??_C@_05EELHGBCB@?9?9top?$AA@ 10022b30     DiamondClassifyTask.obj
 0002:00001b38       ??_C@_08EMHGCFLB@?9?9matrix?$AA@ 10022b38     DiamondClassifyTask.obj
 0002:00001b44       ??_C@_02CIKBGMLM@?9e?$AA@  10022b44     DiamondClassifyTask.obj
 0002:00001b48       ??_C@_02GHOAPKHL@?9b?$AA@  10022b48     DiamondClassifyTask.obj
 0002:00001b4c       ??_C@_02BPBEIKKI@?9p?$AA@  10022b4c     DiamondClassifyTask.obj
 0002:00001b50       ??_C@_0BA@BNMBNFCI@?9?9query?9gencode?$AA@ 10022b50     DiamondClassifyTask.obj
 0002:00001b60       ??_C@_02JGAIBLNN@?9F?$AA@  10022b60     DiamondClassifyTask.obj
 0002:00001b64       ??_C@_09OMJKJGMN@?9?9gapopen?$AA@ 10022b64     DiamondClassifyTask.obj
 0002:00001b70       ??_C@_0M@OGECNPHB@?9?9gapextend?$AA@ 10022b70     DiamondClassifyTask.obj
 0002:00001b7c       ??_C@_0P@GEBFNBFJ@?9?9index?9chunks?$AA@ 10022b7c     DiamondClassifyTask.obj
 0002:00001b90       __xmm@40000000000000003f50624dd2f1a9fc 10022b90     DiamondClassifyTask.obj
 0002:00001ba0       ??_C@_0CM@ICPJCNAJ@QtMetaTypePrivate?3?3QAssociativeI@ 10022ba0     DiamondClassifyWorker.obj
 0002:00001bcc       ??_C@_0DA@ENPGIFBJ@U2?3?3LocalWorkflow?3?3TaxonomyClass@ 10022bcc     DiamondClassifyWorker.obj
 0002:00001c00       ??_7DiamondClassifyWorker@LocalWorkflow@U2@@6BQObject@@@ 10022c00     DiamondClassifyWorker.obj
 0002:00001c44       ??_7DiamondClassifyWorker@LocalWorkflow@U2@@6BWorker@Workflow@2@@ 10022c44     DiamondClassifyWorker.obj
 0002:00001c60       ??_7DiamondClassifyWorker@LocalWorkflow@U2@@6BCommunicationSubject@Workflow@2@@ 10022c60     DiamondClassifyWorker.obj
 0002:00001c6c       ??_C@_07FCMFEHDO@diamond?$AA@ 10022c6c     DiamondClassifyWorker.obj
 0002:00001c74       ??_C@_0BO@JGIHHBDI@src?2DiamondClassifyWorker?4cpp?$AA@ 10022c74     DiamondClassifyWorker.obj
 0002:00001c94       ??_C@_0DF@GPCBDEIK@There?5were?5?$CF1?5input?5reads?0?5?$CF2?5re@ 10022c94     DiamondClassifyWorker.obj
 0002:00001ccc       ??_C@_0P@FKJGJMFL@DIAMOND_?$CF1?4txt?$AA@ 10022ccc     DiamondClassifyWorker.obj
 0002:00001cdc       ??_C@_03CLFHJCDC@txt?$AA@  10022cdc     DiamondClassifyWorker.obj
 0002:00001ce0       ??_C@_07KPJIPLLK@DIAMOND?$AA@ 10022ce0     DiamondClassifyWorker.obj
 0002:00001ce8       ??_C@_01KMDKNFGN@?1?$AA@   10022ce8     DiamondClassifyWorker.obj
 0002:00001cf0       __real@0000000000000000    10022cf0     DiamondClassifyWorker.obj
 0002:00001cfc       ??_SSpinBoxDelegate@U2@@6B@ 10022cfc     DiamondClassifyWorkerFactory.obj
 0002:00001d7c       ??_SDoubleSpinBoxDelegate@U2@@6B@ 10022d7c     DiamondClassifyWorkerFactory.obj
 0002:00001dfc       ??_SComboBoxDelegate@U2@@6B@ 10022dfc     DiamondClassifyWorkerFactory.obj
 0002:00001e7c       ??_7DiamondClassifyWorkerFactory@LocalWorkflow@U2@@6B?$IdRegistry@VDomainFactory@Workflow@U2@@@2@@ 10022e7c     DiamondClassifyWorkerFactory.obj
 0002:00001ea8       ??_7DiamondClassifyWorkerFactory@LocalWorkflow@U2@@6BDescriptor@2@@ 10022ea8     DiamondClassifyWorkerFactory.obj
 0002:00001eb4       ??_SDatabaseDelegate@LocalWorkflow@U2@@6B@ 10022eb4     DiamondClassifyWorkerFactory.obj
 0002:00001f30       ??_C@_0BB@KIENCGBE@diamond?9classify?$AA@ 10022f30     DiamondClassifyWorkerFactory.obj
 0002:00001f44       ??_C@_02LMMGJAGL@in?$AA@   10022f44     DiamondClassifyWorkerFactory.obj
 0002:00001f48       ??_C@_0L@LGHLPLD@reads?9url1?$AA@ 10022f48     DiamondClassifyWorkerFactory.obj
 0002:00001f54       ??_C@_0L@HPPLHBN@input?9data?$AA@ 10022f54     DiamondClassifyWorkerFactory.obj
 0002:00001f60       ??_C@_0N@IPJCHDGG@genetic?9code?$AA@ 10022f60     DiamondClassifyWorkerFactory.obj
 0002:00001f70       ??_C@_0P@OJHJNHMJ@sensitive?9mode?$AA@ 10022f70     DiamondClassifyWorkerFactory.obj
 0002:00001f80       ??_C@_0BK@MCLNLPDM@top?9alignments?9percentage?$AA@ 10022f80     DiamondClassifyWorkerFactory.obj
 0002:00001f9c       ??_C@_0M@CFLABEHO@frame?9shift?$AA@ 10022f9c     DiamondClassifyWorkerFactory.obj
 0002:00001fa8       ??_C@_07OONFBLNG@e?9value?$AA@ 10022fa8     DiamondClassifyWorkerFactory.obj
 0002:00001fb0       ??_C@_06CGNOPMBC@matrix?$AA@ 10022fb0     DiamondClassifyWorkerFactory.obj
 0002:00001fb8       ??_C@_08KPNAGODI@gap?9open?$AA@ 10022fb8     DiamondClassifyWorkerFactory.obj
 0002:00001fc4       ??_C@_0L@DMOPPDON@gap?9extend?$AA@ 10022fc4     DiamondClassifyWorkerFactory.obj
 0002:00001fd0       ??_C@_07NFPADACG@threads?$AA@ 10022fd0     DiamondClassifyWorkerFactory.obj
 0002:00001fd8       ??_C@_0L@BJGDCDM@block?9size?$AA@ 10022fd8     DiamondClassifyWorkerFactory.obj
 0002:00001fe4       ??_C@_0N@LCOHNACN@index?9chunks?$AA@ 10022fe4     DiamondClassifyWorkerFactory.obj
 0002:00001ff4       ??_C@_0L@JDEFPCKN@output?9url?$AA@ 10022ff4     DiamondClassifyWorkerFactory.obj
 0002:00002000       ??_C@_0L@BOLLAKIP@Input?5URL?4?$AA@ 10023000     DiamondClassifyWorkerFactory.obj
 0002:0000200c       ??_C@_09GGCOOKFN@Input?5URL?$AA@ 1002300c     DiamondClassifyWorkerFactory.obj
 0002:00002018       ??_C@_0MP@GLIMJGBD@URL?$CIs?$CJ?5to?5FASTQ?5or?5FASTA?5file?$CIs?$CJ@ 10023018     DiamondClassifyWorkerFactory.obj
 0002:000020e8       ??_C@_0BA@GLOOOALC@Input?5sequences?$AA@ 100230e8     DiamondClassifyWorkerFactory.obj
 0002:000020f8       ??_C@_0FC@HELOHFGJ@A?5list?5of?5sequence?5names?5with?5th@ 100230f8     DiamondClassifyWorkerFactory.obj
 0002:0000214c       ??_C@_0BH@EMLHPCJO@DIAMOND?5Classification?$AA@ 1002314c     DiamondClassifyWorkerFactory.obj
 0002:00002164       ??_C@_03DAJLOBIG@?9in?$AA@ 10023164     DiamondClassifyWorkerFactory.obj
 0002:00002168       ??_C@_0CG@NOLPFNDI@Input?5a?5binary?5DIAMOND?5database?5@ 10023168     DiamondClassifyWorkerFactory.obj
 0002:00002190       ??_C@_0EI@BCEHCGKM@Genetic?5code?5used?5for?5translatio@ 10023190     DiamondClassifyWorkerFactory.obj
 0002:000021d8       ??_C@_0N@IAHCCLEN@Genetic?5code?$AA@ 100231d8     DiamondClassifyWorkerFactory.obj
 0002:000021e8       ??_C@_0OO@PIMDAMMI@The?5sensitive?5modes?5?$CI?9?9sensitive@ 100231e8     DiamondClassifyWorkerFactory.obj
 0002:000022d8       ??_C@_0P@NNCCPKIJ@Sensitive?5mode?$AA@ 100232d8     DiamondClassifyWorkerFactory.obj
 0002:000022e8       ??_C@_0BLL@JHNJDMJ@DIAMOND?5uses?5the?5lowest?5common?5a@ 100232e8     DiamondClassifyWorkerFactory.obj
 0002:000024a4       ??_C@_0BK@EIFBAGAC@Top?5alignments?5percentage?$AA@ 100234a4     DiamondClassifyWorkerFactory.obj
 0002:000024c0       ??_C@_0BAI@FNGJLAG@Penalty?5for?5frameshift?5in?5DNA?9vs@ 100234c0     DiamondClassifyWorkerFactory.obj
 0002:000025c8       ??_C@_0L@OEJCHLNP@Frameshift?$AA@ 100235c8     DiamondClassifyWorkerFactory.obj
 0002:000025d4       ??_C@_0DN@HNENFFOE@Maximum?5expected?5value?5to?5report@ 100235d4     DiamondClassifyWorkerFactory.obj
 0002:00002614       ??_C@_0P@PLHGLICP@Expected?5value?$AA@ 10023614     DiamondClassifyWorkerFactory.obj
 0002:00002624       ??_C@_0BL@MEGMFHCG@Scoring?5matrix?5?$CI?9?9matrix?$CJ?4?$AA@ 10023624     DiamondClassifyWorkerFactory.obj
 0002:00002640       ??_C@_06OJGDMFIO@Matrix?$AA@ 10023640     DiamondClassifyWorkerFactory.obj
 0002:00002648       ??_C@_0BO@BHBMEHHP@Gap?5open?5penalty?5?$CI?9?9gapopen?$CJ?4?$AA@ 10023648     DiamondClassifyWorkerFactory.obj
 0002:00002668       ??_C@_0BB@EJMHCDJH@Gap?5open?5penalty?$AA@ 10023668     DiamondClassifyWorkerFactory.obj
 0002:0000267c       ??_C@_0CF@LAOMGCOE@Gap?5extension?5penalty?5?$CI?9?9gapexte@ 1002367c     DiamondClassifyWorkerFactory.obj
 0002:000026a4       ??_C@_0BG@FCHIHJMG@Gap?5extension?5penalty?$AA@ 100236a4     DiamondClassifyWorkerFactory.obj
 0002:000026bc       ??_C@_0CC@BOFOJCJF@Number?5of?5CPU?5threads?5?$CI?9?9treads?$CJ@ 100236bc     DiamondClassifyWorkerFactory.obj
 0002:000026e0       ??_C@_0BC@GJADDMKB@Number?5of?5threads?$AA@ 100236e0     DiamondClassifyWorkerFactory.obj
 0002:000026f8       ??_C@_0BFJ@PPFJGLFP@Block?5size?5in?5billions?5of?5sequen@ 100236f8     DiamondClassifyWorkerFactory.obj
 0002:00002854       ??_C@_0L@DLJEKODF@Block?5size?$AA@ 10023854     DiamondClassifyWorkerFactory.obj
 0002:00002860       ??_C@_0BBM@EGGMMGBO@The?5number?5of?5chunks?5for?5process@ 10023860     DiamondClassifyWorkerFactory.obj
 0002:0000297c       ??_C@_0N@JKJMIOAJ@Index?5chunks?$AA@ 1002397c     DiamondClassifyWorkerFactory.obj
 0002:00002990       ??_C@_0BBG@NEHKFCPM@Specify?5the?5output?5file?5name?4?$DMbr@ 10023990     DiamondClassifyWorkerFactory.obj
 0002:00002aa8       ??_C@_0M@LEIJPAKP@Output?5file?$AA@ 10023aa8     DiamondClassifyWorkerFactory.obj
 0002:00002ab4       ??_C@_0CA@BBFPBJKD@Classify?5tool?4?5Hidden?5attribute?$AA@ 10023ab4     DiamondClassifyWorkerFactory.obj
 0002:00002ad4       ??_C@_0BA@EAHCLEBK@NCBI?9GenBank?5?$CD1?$AA@ 10023ad4     DiamondClassifyWorkerFactory.obj
 0002:00002ae4       ??_C@_07MCAEODGB@Default?$AA@ 10023ae4     DiamondClassifyWorkerFactory.obj
 0002:00002aec       ??_C@_09GNDCDNAC@Sensitive?$AA@ 10023aec     DiamondClassifyWorkerFactory.obj
 0002:00002af8       ??_C@_0P@BGEPDKON@More?5sensitive?$AA@ 10023af8     DiamondClassifyWorkerFactory.obj
 0002:00002b08       ??_C@_07CCOEHHFD@minimum?$AA@ 10023b08     DiamondClassifyWorkerFactory.obj
 0002:00002b10       ??_C@_07MEIENILC@maximum?$AA@ 10023b10     DiamondClassifyWorkerFactory.obj
 0002:00002b18       ??_C@_06EMCDFPCG@suffix?$AA@ 10023b18     DiamondClassifyWorkerFactory.obj
 0002:00002b20       ??_C@_01FGNFDNOH@?$CF?$AA@ 10023b20     DiamondClassifyWorkerFactory.obj
 0002:00002b24       ??_C@_0BB@HBOHNBEB@specialValueText?$AA@ 10023b24     DiamondClassifyWorkerFactory.obj
 0002:00002b38       ??_C@_07DKFOHFAF@Skipped?$AA@ 10023b38     DiamondClassifyWorkerFactory.obj
 0002:00002b40       ??_C@_0L@HOCHOMFK@singleStep?$AA@ 10023b40     DiamondClassifyWorkerFactory.obj
 0002:00002b4c       ??_C@_08LCDAKGCH@decimals?$AA@ 10023b4c     DiamondClassifyWorkerFactory.obj
 0002:00002b58       ??_C@_04LBDCJOFB@Auto?$AA@ 10023b58     DiamondClassifyWorkerFactory.obj
 0002:00002b60       ??_C@_0P@NCLDGEAH@diamond?1output?$AA@ 10023b60     DiamondClassifyWorkerFactory.obj
 0002:00002b70       ??_C@_0BJD@IODJKAPJ@In?5general?0?5DIAMOND?5is?5a?5sequenc@ 10023b70     DiamondClassifyWorkerFactory.obj
 0002:00002d04       ??_C@_0CA@ILFOKNNB@Classify?5Sequences?5with?5DIAMOND?$AA@ 10023d04     DiamondClassifyWorkerFactory.obj
 0002:00002d28       __real@3f50624dd2f1a9fc    10023d28     DiamondClassifyWorkerFactory.obj
 0002:00002d30       __real@3fb999999999999a    10023d30     DiamondClassifyWorkerFactory.obj
 0002:00002d38       __real@3fe0000000000000    10023d38     DiamondClassifyWorkerFactory.obj
 0002:00002d44       ??_7DiamondSupport@U2@@6B@ 10023d44     DiamondSupport.obj
 0002:00002d80       ??_C@_09GAJKMFCA@?9?9version?$AA@ 10023d80     DiamondSupport.obj
 0002:00002d8c       ??_C@_0BB@JIMMFALI@diamond?5version?5?$AA@ 10023d8c     DiamondSupport.obj
 0002:00002da0       ??_C@_0CA@OCKABKJG@diamond?5version?5?$CI?2d?$CL?2?4?2d?$CL?2?4?2d?$CL?$CJ?$AA@ 10023da0     DiamondSupport.obj
 0002:00002dc0       ??_C@_0MD@EOFPGGIK@In?5general?0?5DIAMOND?5is?5a?5sequenc@ 10023dc0     DiamondSupport.obj
 0002:00002e88       ??_7DiamondSupportPlugin@U2@@6B@ 10023e88     DiamondSupportPlugin.obj
 0002:00002eb4       ??_C@_0BO@JOCDNLDN@DIAMOND?5external?5tool?5support?$AA@ 10023eb4     DiamondSupportPlugin.obj
 0002:00002ed8       ??_C@_0LM@EFAFEHIO@The?5plugin?5supports?5DIAMOND?3?5a?5s@ 10023ed8     DiamondSupportPlugin.obj
 0002:00002f98       ??_7GenomesPreparationTask@U2@@6B@ 10023f98     GenomesPreparationTask.obj
 0002:00003024       ??_C@_0BE@ENCNMNOD@Genomes?5preparation?$AA@ 10024024     GenomesPreparationTask.obj
 0002:00003038       ??_C@_0BJ@ELJNNO@Genomes?5URLs?5are?5not?5set?$AA@ 10024038     GenomesPreparationTask.obj
 0002:00003054       ??_C@_0CM@BOHEBGM@File?5URL?5to?5write?5prepared?5genom@ 10024054     GenomesPreparationTask.obj
 0002:0000354c       ?value@?$integral_constant@_N$0A@@std@@2_NB 1002454c     MSVCRT:ti_inst.obj
 0002:0000354d       ?value@?$integral_constant@_N$00@std@@2_NB 1002454d     MSVCRT:ti_inst.obj
 0002:00003554       ??_7type_info@@6B@         10024554     MSVCRT:ti_inst.obj
 0002:00003558       __pRawDllMain              10024558     MSVCRT:crtdll.obj
 0002:00003558       __pDefaultRawDllMain       10024558     MSVCRT:crtdll.obj
 0002:00003564       ?ProcessDetach@NativeDll@<CrtImplementationDetails>@@0IB 10024564     MSVCRT:initsect.obj
 0002:00003568       ?ProcessAttach@NativeDll@<CrtImplementationDetails>@@0IB 10024568     MSVCRT:initsect.obj
 0002:0000356c       ?ThreadAttach@NativeDll@<CrtImplementationDetails>@@0IB 1002456c     MSVCRT:initsect.obj
 0002:00003570       ?ThreadDetach@NativeDll@<CrtImplementationDetails>@@0IB 10024570     MSVCRT:initsect.obj
 0002:00003574       ?ProcessVerifier@NativeDll@<CrtImplementationDetails>@@0IB 10024574     MSVCRT:initsect.obj
 0002:00003578       __load_config_used         10024578     MSVCRT:loadcfg.obj
 0002:00003638       ??_R4error_category@std@@6B@ 10024638     DiamondBuildPrompter.obj
 0002:0000364c       ??_R3error_category@std@@8 1002464c     DiamondBuildPrompter.obj
 0002:0000365c       ??_R2error_category@std@@8 1002465c     DiamondBuildPrompter.obj
 0002:00003664       ??_R1A@?0A@EA@error_category@std@@8 10024664     DiamondBuildPrompter.obj
 0002:00003680       ??_R4_Generic_error_category@std@@6B@ 10024680     DiamondBuildPrompter.obj
 0002:00003694       ??_R3_Generic_error_category@std@@8 10024694     DiamondBuildPrompter.obj
 0002:000036a4       ??_R2_Generic_error_category@std@@8 100246a4     DiamondBuildPrompter.obj
 0002:000036b0       ??_R1A@?0A@EA@_Generic_error_category@std@@8 100246b0     DiamondBuildPrompter.obj
 0002:000036cc       ??_R4_Iostream_error_category@std@@6B@ 100246cc     DiamondBuildPrompter.obj
 0002:000036e0       ??_R3_Iostream_error_category@std@@8 100246e0     DiamondBuildPrompter.obj
 0002:000036f0       ??_R2_Iostream_error_category@std@@8 100246f0     DiamondBuildPrompter.obj
 0002:00003700       ??_R1A@?0A@EA@_Iostream_error_category@std@@8 10024700     DiamondBuildPrompter.obj
 0002:0000371c       ??_R4_System_error_category@std@@6B@ 1002471c     DiamondBuildPrompter.obj
 0002:00003730       ??_R3_System_error_category@std@@8 10024730     DiamondBuildPrompter.obj
 0002:00003740       ??_R2_System_error_category@std@@8 10024740     DiamondBuildPrompter.obj
 0002:00003750       ??_R1A@?0A@EA@_System_error_category@std@@8 10024750     DiamondBuildPrompter.obj
 0002:0000376c       ??_R1A@?0A@EA@QObject@@8   1002476c     DiamondBuildPrompter.obj
 0002:00003788       ??_R3QObject@@8            10024788     DiamondBuildPrompter.obj
 0002:00003798       ??_R2QObject@@8            10024798     DiamondBuildPrompter.obj
 0002:000037a0       ??_R4DiamondBuildPrompter@LocalWorkflow@U2@@6BActorDocument@Workflow@2@@ 100247a0     DiamondBuildPrompter.obj
 0002:000037b4       ??_R3DiamondBuildPrompter@LocalWorkflow@U2@@8 100247b4     DiamondBuildPrompter.obj
 0002:000037c4       ??_R2DiamondBuildPrompter@LocalWorkflow@U2@@8 100247c4     DiamondBuildPrompter.obj
 0002:000037e4       ??_R1A@?0A@EA@DiamondBuildPrompter@LocalWorkflow@U2@@8 100247e4     DiamondBuildPrompter.obj
 0002:00003800       ??_R1A@?0A@EA@?$PrompterBase@VDiamondBuildPrompter@LocalWorkflow@U2@@@U2@@8 10024800     DiamondBuildPrompter.obj
 0002:0000381c       ??_R3?$PrompterBase@VDiamondBuildPrompter@LocalWorkflow@U2@@@U2@@8 1002481c     DiamondBuildPrompter.obj
 0002:0000382c       ??_R2?$PrompterBase@VDiamondBuildPrompter@LocalWorkflow@U2@@@U2@@8 1002482c     DiamondBuildPrompter.obj
 0002:00003848       ??_R1A@?0A@EA@PrompterBaseImpl@U2@@8 10024848     DiamondBuildPrompter.obj
 0002:00003864       ??_R3PrompterBaseImpl@U2@@8 10024864     DiamondBuildPrompter.obj
 0002:00003874       ??_R2PrompterBaseImpl@U2@@8 10024874     DiamondBuildPrompter.obj
 0002:0000388c       ??_R1A@?0A@EA@ActorDocument@Workflow@U2@@8 1002488c     DiamondBuildPrompter.obj
 0002:000038a8       ??_R3ActorDocument@Workflow@U2@@8 100248a8     DiamondBuildPrompter.obj
 0002:000038b8       ??_R2ActorDocument@Workflow@U2@@8 100248b8     DiamondBuildPrompter.obj
 0002:000038c8       ??_R1A@?0A@EA@QTextDocument@@8 100248c8     DiamondBuildPrompter.obj
 0002:000038e4       ??_R3QTextDocument@@8      100248e4     DiamondBuildPrompter.obj
 0002:000038f4       ??_R2QTextDocument@@8      100248f4     DiamondBuildPrompter.obj
 0002:00003900       ??_R1M@?0A@EA@Prompter@Workflow@U2@@8 10024900     DiamondBuildPrompter.obj
 0002:0000391c       ??_R3Prompter@Workflow@U2@@8 1002491c     DiamondBuildPrompter.obj
 0002:0000392c       ??_R2Prompter@Workflow@U2@@8 1002492c     DiamondBuildPrompter.obj
 0002:00003934       ??_R1A@?0A@EA@Prompter@Workflow@U2@@8 10024934     DiamondBuildPrompter.obj
 0002:00003950       ??_R4DiamondBuildPrompter@LocalWorkflow@U2@@6BPrompter@Workflow@2@@ 10024950     DiamondBuildPrompter.obj
 0002:00003964       ??_R4?$PrompterBase@VDiamondBuildPrompter@LocalWorkflow@U2@@@U2@@6BActorDocument@Workflow@1@@ 10024964     DiamondBuildPrompter.obj
 0002:00003978       ??_R4?$PrompterBase@VDiamondBuildPrompter@LocalWorkflow@U2@@@U2@@6BPrompter@Workflow@1@@ 10024978     DiamondBuildPrompter.obj
 0002:0000398c       ??_R4ExternalToolLogParser@U2@@6B@ 1002498c     DiamondBuildTask.obj
 0002:000039a0       ??_R3ExternalToolLogParser@U2@@8 100249a0     DiamondBuildTask.obj
 0002:000039b0       ??_R2ExternalToolLogParser@U2@@8 100249b0     DiamondBuildTask.obj
 0002:000039bc       ??_R1A@?0A@EA@ExternalToolLogParser@U2@@8 100249bc     DiamondBuildTask.obj
 0002:000039d8       ??_R4ExternalToolRunTask@U2@@6B@ 100249d8     DiamondBuildTask.obj
 0002:000039ec       ??_R3ExternalToolRunTask@U2@@8 100249ec     DiamondBuildTask.obj
 0002:000039fc       ??_R2ExternalToolRunTask@U2@@8 100249fc     DiamondBuildTask.obj
 0002:00003a0c       ??_R1A@?0A@EA@ExternalToolRunTask@U2@@8 10024a0c     DiamondBuildTask.obj
 0002:00003a28       ??_R1A@?0A@EA@Task@U2@@8   10024a28     DiamondBuildTask.obj
 0002:00003a44       ??_R3Task@U2@@8            10024a44     DiamondBuildTask.obj
 0002:00003a54       ??_R2Task@U2@@8            10024a54     DiamondBuildTask.obj
 0002:00003a60       ??_R4DiamondBuildTask@U2@@6B@ 10024a60     DiamondBuildTask.obj
 0002:00003a74       ??_R3DiamondBuildTask@U2@@8 10024a74     DiamondBuildTask.obj
 0002:00003a84       ??_R2DiamondBuildTask@U2@@8 10024a84     DiamondBuildTask.obj
 0002:00003a98       ??_R1A@?0A@EA@DiamondBuildTask@U2@@8 10024a98     DiamondBuildTask.obj
 0002:00003ab4       ??_R1A@?0A@EA@ExternalToolSupportTask@U2@@8 10024ab4     DiamondBuildTask.obj
 0002:00003ad0       ??_R3ExternalToolSupportTask@U2@@8 10024ad0     DiamondBuildTask.obj
 0002:00003ae0       ??_R2ExternalToolSupportTask@U2@@8 10024ae0     DiamondBuildTask.obj
 0002:00003af0       ??_R4FailTask@U2@@6B@      10024af0     DiamondBuildWorker.obj
 0002:00003b04       ??_R3FailTask@U2@@8        10024b04     DiamondBuildWorker.obj
 0002:00003b14       ??_R2FailTask@U2@@8        10024b14     DiamondBuildWorker.obj
 0002:00003b24       ??_R1A@?0A@EA@FailTask@U2@@8 10024b24     DiamondBuildWorker.obj
 0002:00003b40       ??_R4TaskSignalMapper@U2@@6B@ 10024b40     DiamondBuildWorker.obj
 0002:00003b54       ??_R3TaskSignalMapper@U2@@8 10024b54     DiamondBuildWorker.obj
 0002:00003b64       ??_R2TaskSignalMapper@U2@@8 10024b64     DiamondBuildWorker.obj
 0002:00003b70       ??_R1A@?0A@EA@TaskSignalMapper@U2@@8 10024b70     DiamondBuildWorker.obj
 0002:00003b8c       ??_R4Descriptor@U2@@6B@    10024b8c     DiamondBuildWorker.obj
 0002:00003ba0       ??_R3Descriptor@U2@@8      10024ba0     DiamondBuildWorker.obj
 0002:00003bb0       ??_R2Descriptor@U2@@8      10024bb0     DiamondBuildWorker.obj
 0002:00003bb8       ??_R1A@?0A@EA@Descriptor@U2@@8 10024bb8     DiamondBuildWorker.obj
 0002:00003bd4       ??_R4DiamondBuildWorker@LocalWorkflow@U2@@6BQObject@@@ 10024bd4     DiamondBuildWorker.obj
 0002:00003be8       ??_R3DiamondBuildWorker@LocalWorkflow@U2@@8 10024be8     DiamondBuildWorker.obj
 0002:00003bf8       ??_R2DiamondBuildWorker@LocalWorkflow@U2@@8 10024bf8     DiamondBuildWorker.obj
 0002:00003c10       ??_R1A@?0A@EA@DiamondBuildWorker@LocalWorkflow@U2@@8 10024c10     DiamondBuildWorker.obj
 0002:00003c2c       ??_R1A@?0A@EA@BaseWorker@LocalWorkflow@U2@@8 10024c2c     DiamondBuildWorker.obj
 0002:00003c48       ??_R3BaseWorker@LocalWorkflow@U2@@8 10024c48     DiamondBuildWorker.obj
 0002:00003c58       ??_R2BaseWorker@LocalWorkflow@U2@@8 10024c58     DiamondBuildWorker.obj
 0002:00003c6c       ??_R17?0A@EA@Worker@Workflow@U2@@8 10024c6c     DiamondBuildWorker.obj
 0002:00003c88       ??_R3Worker@Workflow@U2@@8 10024c88     DiamondBuildWorker.obj
 0002:00003c98       ??_R2Worker@Workflow@U2@@8 10024c98     DiamondBuildWorker.obj
 0002:00003ca0       ??_R1A@?0A@EA@Worker@Workflow@U2@@8 10024ca0     DiamondBuildWorker.obj
 0002:00003cbc       ??_R1BA@?0A@EA@CommunicationSubject@Workflow@U2@@8 10024cbc     DiamondBuildWorker.obj
 0002:00003cd8       ??_R3CommunicationSubject@Workflow@U2@@8 10024cd8     DiamondBuildWorker.obj
 0002:00003ce8       ??_R2CommunicationSubject@Workflow@U2@@8 10024ce8     DiamondBuildWorker.obj
 0002:00003cf0       ??_R1A@?0A@EA@CommunicationSubject@Workflow@U2@@8 10024cf0     DiamondBuildWorker.obj
 0002:00003d0c       ??_R4DiamondBuildWorker@LocalWorkflow@U2@@6BWorker@Workflow@2@@ 10024d0c     DiamondBuildWorker.obj
 0002:00003d20       ??_R4DiamondBuildWorker@LocalWorkflow@U2@@6BCommunicationSubject@Workflow@2@@ 10024d20     DiamondBuildWorker.obj
 0002:00003d34       ??_R4MapDataType@U2@@6B@   10024d34     DiamondBuildWorkerFactory.obj
 0002:00003d48       ??_R3MapDataType@U2@@8     10024d48     DiamondBuildWorkerFactory.obj
 0002:00003d58       ??_R2MapDataType@U2@@8     10024d58     DiamondBuildWorkerFactory.obj
 0002:00003d6c       ??_R1A@?0A@EA@MapDataType@U2@@8 10024d6c     DiamondBuildWorkerFactory.obj
 0002:00003d88       ??_R1A@?0A@EA@DataType@U2@@8 10024d88     DiamondBuildWorkerFactory.obj
 0002:00003da4       ??_R3DataType@U2@@8        10024da4     DiamondBuildWorkerFactory.obj
 0002:00003db4       ??_R2DataType@U2@@8        10024db4     DiamondBuildWorkerFactory.obj
 0002:00003dc4       ??_R1BA@?0A@EA@QSharedData@@8 10024dc4     DiamondBuildWorkerFactory.obj
 0002:00003de0       ??_R3QSharedData@@8        10024de0     DiamondBuildWorkerFactory.obj
 0002:00003df0       ??_R2QSharedData@@8        10024df0     DiamondBuildWorkerFactory.obj
 0002:00003df8       ??_R1A@?0A@EA@QSharedData@@8 10024df8     DiamondBuildWorkerFactory.obj
 0002:00003e14       ??_R4Attribute@U2@@6B@     10024e14     DiamondBuildWorkerFactory.obj
 0002:00003e28       ??_R3Attribute@U2@@8       10024e28     DiamondBuildWorkerFactory.obj
 0002:00003e38       ??_R2Attribute@U2@@8       10024e38     DiamondBuildWorkerFactory.obj
 0002:00003e44       ??_R1A@?0A@EA@Attribute@U2@@8 10024e44     DiamondBuildWorkerFactory.obj
 0002:00003e60       ??_R3ConfigurationEditor@U2@@8 10024e60     DiamondBuildWorkerFactory.obj
 0002:00003e70       ??_R2ConfigurationEditor@U2@@8 10024e70     DiamondBuildWorkerFactory.obj
 0002:00003e7c       ??_R1A@?0A@EA@ConfigurationEditor@U2@@8 10024e7c     DiamondBuildWorkerFactory.obj
 0002:00003e98       ??_R4DelegateEditor@U2@@6B@ 10024e98     DiamondBuildWorkerFactory.obj
 0002:00003eac       ??_R3DelegateEditor@U2@@8  10024eac     DiamondBuildWorkerFactory.obj
 0002:00003ebc       ??_R2DelegateEditor@U2@@8  10024ebc     DiamondBuildWorkerFactory.obj
 0002:00003ecc       ??_R1A@?0A@EA@DelegateEditor@U2@@8 10024ecc     DiamondBuildWorkerFactory.obj
 0002:00003ee8       ??_R4URLDelegate@U2@@6B@   10024ee8     DiamondBuildWorkerFactory.obj
 0002:00003efc       ??_R3URLDelegate@U2@@8     10024efc     DiamondBuildWorkerFactory.obj
 0002:00003f0c       ??_R2URLDelegate@U2@@8     10024f0c     DiamondBuildWorkerFactory.obj
 0002:00003f24       ??_R1A@?0A@EA@URLDelegate@U2@@8 10024f24     DiamondBuildWorkerFactory.obj
 0002:00003f40       ??_R1A@?0A@EA@PropertyDelegate@U2@@8 10024f40     DiamondBuildWorkerFactory.obj
 0002:00003f5c       ??_R3PropertyDelegate@U2@@8 10024f5c     DiamondBuildWorkerFactory.obj
 0002:00003f6c       ??_R2PropertyDelegate@U2@@8 10024f6c     DiamondBuildWorkerFactory.obj
 0002:00003f80       ??_R1A@?0A@EA@QItemDelegate@@8 10024f80     DiamondBuildWorkerFactory.obj
 0002:00003f9c       ??_R3QItemDelegate@@8      10024f9c     DiamondBuildWorkerFactory.obj
 0002:00003fac       ??_R2QItemDelegate@@8      10024fac     DiamondBuildWorkerFactory.obj
 0002:00003fbc       ??_R1A@?0A@EA@QAbstractItemDelegate@@8 10024fbc     DiamondBuildWorkerFactory.obj
 0002:00003fd8       ??_R3QAbstractItemDelegate@@8 10024fd8     DiamondBuildWorkerFactory.obj
 0002:00003fe8       ??_R2QAbstractItemDelegate@@8 10024fe8     DiamondBuildWorkerFactory.obj
 0002:00003ff4       ??_R4PortDescriptor@Workflow@U2@@6B@ 10024ff4     DiamondBuildWorkerFactory.obj
 0002:00004008       ??_R3PortDescriptor@Workflow@U2@@8 10025008     DiamondBuildWorkerFactory.obj
 0002:00004018       ??_R2PortDescriptor@Workflow@U2@@8 10025018     DiamondBuildWorkerFactory.obj
 0002:00004024       ??_R1A@?0A@EA@PortDescriptor@Workflow@U2@@8 10025024     DiamondBuildWorkerFactory.obj
 0002:00004040       ??_R17?0A@EA@Descriptor@U2@@8 10025040     DiamondBuildWorkerFactory.obj
 0002:0000405c       ??_R4IntegralBusActorPrototype@Workflow@U2@@6B@ 1002505c     DiamondBuildWorkerFactory.obj
 0002:00004070       ??_R3IntegralBusActorPrototype@Workflow@U2@@8 10025070     DiamondBuildWorkerFactory.obj
 0002:00004080       ??_R2IntegralBusActorPrototype@Workflow@U2@@8 10025080     DiamondBuildWorkerFactory.obj
 0002:00004094       ??_R1A@?0A@EA@IntegralBusActorPrototype@Workflow@U2@@8 10025094     DiamondBuildWorkerFactory.obj
 0002:000040b0       ??_R1A@?0A@EA@ActorPrototype@Workflow@U2@@8 100250b0     DiamondBuildWorkerFactory.obj
 0002:000040cc       ??_R3ActorPrototype@Workflow@U2@@8 100250cc     DiamondBuildWorkerFactory.obj
 0002:000040dc       ??_R2ActorPrototype@Workflow@U2@@8 100250dc     DiamondBuildWorkerFactory.obj
 0002:000040ec       ??_R1A@?0A@EA@VisualDescriptor@U2@@8 100250ec     DiamondBuildWorkerFactory.obj
 0002:00004108       ??_R3VisualDescriptor@U2@@8 10025108     DiamondBuildWorkerFactory.obj
 0002:00004118       ??_R2VisualDescriptor@U2@@8 10025118     DiamondBuildWorkerFactory.obj
 0002:00004124       ??_R4DiamondBuildValidator@Workflow@U2@@6B@ 10025124     DiamondBuildWorkerFactory.obj
 0002:00004138       ??_R3DiamondBuildValidator@Workflow@U2@@8 10025138     DiamondBuildWorkerFactory.obj
 0002:00004148       ??_R2DiamondBuildValidator@Workflow@U2@@8 10025148     DiamondBuildWorkerFactory.obj
 0002:00004158       ??_R1A@?0A@EA@DiamondBuildValidator@Workflow@U2@@8 10025158     DiamondBuildWorkerFactory.obj
 0002:00004174       ??_R1A@?0A@EA@ActorValidator@Workflow@U2@@8 10025174     DiamondBuildWorkerFactory.obj
 0002:00004190       ??_R3ActorValidator@Workflow@U2@@8 10025190     DiamondBuildWorkerFactory.obj
 0002:000041a0       ??_R2ActorValidator@Workflow@U2@@8 100251a0     DiamondBuildWorkerFactory.obj
 0002:000041ac       ??_R1A@?0A@EA@ConfigurationValidator@U2@@8 100251ac     DiamondBuildWorkerFactory.obj
 0002:000041c8       ??_R3ConfigurationValidator@U2@@8 100251c8     DiamondBuildWorkerFactory.obj
 0002:000041d8       ??_R2ConfigurationValidator@U2@@8 100251d8     DiamondBuildWorkerFactory.obj
 0002:000041e0       ??_R4DiamondBuildWorkerFactory@LocalWorkflow@U2@@6B?$IdRegistry@VDomainFactory@Workflow@U2@@@2@@ 100251e0     DiamondBuildWorkerFactory.obj
 0002:000041f4       ??_R3DiamondBuildWorkerFactory@LocalWorkflow@U2@@8 100251f4     DiamondBuildWorkerFactory.obj
 0002:00004204       ??_R2DiamondBuildWorkerFactory@LocalWorkflow@U2@@8 10025204     DiamondBuildWorkerFactory.obj
 0002:00004218       ??_R1A@?0A@EA@DiamondBuildWorkerFactory@LocalWorkflow@U2@@8 10025218     DiamondBuildWorkerFactory.obj
 0002:00004234       ??_R1A@?0A@EA@DomainFactory@Workflow@U2@@8 10025234     DiamondBuildWorkerFactory.obj
 0002:00004250       ??_R3DomainFactory@Workflow@U2@@8 10025250     DiamondBuildWorkerFactory.obj
 0002:00004260       ??_R2DomainFactory@Workflow@U2@@8 10025260     DiamondBuildWorkerFactory.obj
 0002:00004270       ??_R1A@?0A@EA@?$IdRegistry@VDomainFactory@Workflow@U2@@@U2@@8 10025270     DiamondBuildWorkerFactory.obj
 0002:0000428c       ??_R3?$IdRegistry@VDomainFactory@Workflow@U2@@@U2@@8 1002528c     DiamondBuildWorkerFactory.obj
 0002:0000429c       ??_R2?$IdRegistry@VDomainFactory@Workflow@U2@@@U2@@8 1002529c     DiamondBuildWorkerFactory.obj
 0002:000042a4       ??_R4DiamondBuildWorkerFactory@LocalWorkflow@U2@@6BDescriptor@2@@ 100252a4     DiamondBuildWorkerFactory.obj
 0002:000042b8       ??_R4GenomicLibraryDelegate@LocalWorkflow@U2@@6B@ 100252b8     DiamondBuildWorkerFactory.obj
 0002:000042cc       ??_R3GenomicLibraryDelegate@LocalWorkflow@U2@@8 100252cc     DiamondBuildWorkerFactory.obj
 0002:000042dc       ??_R2GenomicLibraryDelegate@LocalWorkflow@U2@@8 100252dc     DiamondBuildWorkerFactory.obj
 0002:000042f4       ??_R1A@?0A@EA@GenomicLibraryDelegate@LocalWorkflow@U2@@8 100252f4     DiamondBuildWorkerFactory.obj
 0002:00004310       ??_R4DiamondClassifyPrompter@LocalWorkflow@U2@@6BActorDocument@Workflow@2@@ 10025310     DiamondClassifyPrompter.obj
 0002:00004324       ??_R3DiamondClassifyPrompter@LocalWorkflow@U2@@8 10025324     DiamondClassifyPrompter.obj
 0002:00004334       ??_R2DiamondClassifyPrompter@LocalWorkflow@U2@@8 10025334     DiamondClassifyPrompter.obj
 0002:00004354       ??_R1A@?0A@EA@DiamondClassifyPrompter@LocalWorkflow@U2@@8 10025354     DiamondClassifyPrompter.obj
 0002:00004370       ??_R1A@?0A@EA@?$PrompterBase@VDiamondClassifyPrompter@LocalWorkflow@U2@@@U2@@8 10025370     DiamondClassifyPrompter.obj
 0002:0000438c       ??_R3?$PrompterBase@VDiamondClassifyPrompter@LocalWorkflow@U2@@@U2@@8 1002538c     DiamondClassifyPrompter.obj
 0002:0000439c       ??_R2?$PrompterBase@VDiamondClassifyPrompter@LocalWorkflow@U2@@@U2@@8 1002539c     DiamondClassifyPrompter.obj
 0002:000043b8       ??_R4DiamondClassifyPrompter@LocalWorkflow@U2@@6BPrompter@Workflow@2@@ 100253b8     DiamondClassifyPrompter.obj
 0002:000043cc       ??_R4?$PrompterBase@VDiamondClassifyPrompter@LocalWorkflow@U2@@@U2@@6BActorDocument@Workflow@1@@ 100253cc     DiamondClassifyPrompter.obj
 0002:000043e0       ??_R4?$PrompterBase@VDiamondClassifyPrompter@LocalWorkflow@U2@@@U2@@6BPrompter@Workflow@1@@ 100253e0     DiamondClassifyPrompter.obj
 0002:000043f4       ??_R4DiamondClassifyTask@U2@@6B@ 100253f4     DiamondClassifyTask.obj
 0002:00004408       ??_R3DiamondClassifyTask@U2@@8 10025408     DiamondClassifyTask.obj
 0002:00004418       ??_R2DiamondClassifyTask@U2@@8 10025418     DiamondClassifyTask.obj
 0002:0000442c       ??_R1A@?0A@EA@DiamondClassifyTask@U2@@8 1002542c     DiamondClassifyTask.obj
 0002:00004448       ??_R4DiamondClassifyWorker@LocalWorkflow@U2@@6BQObject@@@ 10025448     DiamondClassifyWorker.obj
 0002:0000445c       ??_R3DiamondClassifyWorker@LocalWorkflow@U2@@8 1002545c     DiamondClassifyWorker.obj
 0002:0000446c       ??_R2DiamondClassifyWorker@LocalWorkflow@U2@@8 1002546c     DiamondClassifyWorker.obj
 0002:00004484       ??_R1A@?0A@EA@DiamondClassifyWorker@LocalWorkflow@U2@@8 10025484     DiamondClassifyWorker.obj
 0002:000044a0       ??_R4DiamondClassifyWorker@LocalWorkflow@U2@@6BWorker@Workflow@2@@ 100254a0     DiamondClassifyWorker.obj
 0002:000044b4       ??_R4DiamondClassifyWorker@LocalWorkflow@U2@@6BCommunicationSubject@Workflow@2@@ 100254b4     DiamondClassifyWorker.obj
 0002:000044c8       ??_R4SpinBoxDelegate@U2@@6B@ 100254c8     DiamondClassifyWorkerFactory.obj
 0002:000044dc       ??_R3SpinBoxDelegate@U2@@8 100254dc     DiamondClassifyWorkerFactory.obj
 0002:000044ec       ??_R2SpinBoxDelegate@U2@@8 100254ec     DiamondClassifyWorkerFactory.obj
 0002:00004504       ??_R1A@?0A@EA@SpinBoxDelegate@U2@@8 10025504     DiamondClassifyWorkerFactory.obj
 0002:00004520       ??_R4DoubleSpinBoxDelegate@U2@@6B@ 10025520     DiamondClassifyWorkerFactory.obj
 0002:00004534       ??_R3DoubleSpinBoxDelegate@U2@@8 10025534     DiamondClassifyWorkerFactory.obj
 0002:00004544       ??_R2DoubleSpinBoxDelegate@U2@@8 10025544     DiamondClassifyWorkerFactory.obj
 0002:0000455c       ??_R1A@?0A@EA@DoubleSpinBoxDelegate@U2@@8 1002555c     DiamondClassifyWorkerFactory.obj
 0002:00004578       ??_R4ComboBoxDelegate@U2@@6B@ 10025578     DiamondClassifyWorkerFactory.obj
 0002:0000458c       ??_R3ComboBoxDelegate@U2@@8 1002558c     DiamondClassifyWorkerFactory.obj
 0002:0000459c       ??_R2ComboBoxDelegate@U2@@8 1002559c     DiamondClassifyWorkerFactory.obj
 0002:000045b4       ??_R1A@?0A@EA@ComboBoxDelegate@U2@@8 100255b4     DiamondClassifyWorkerFactory.obj
 0002:000045d0       ??_R4DiamondClassifyWorkerFactory@LocalWorkflow@U2@@6B?$IdRegistry@VDomainFactory@Workflow@U2@@@2@@ 100255d0     DiamondClassifyWorkerFactory.obj
 0002:000045e4       ??_R3DiamondClassifyWorkerFactory@LocalWorkflow@U2@@8 100255e4     DiamondClassifyWorkerFactory.obj
 0002:000045f4       ??_R2DiamondClassifyWorkerFactory@LocalWorkflow@U2@@8 100255f4     DiamondClassifyWorkerFactory.obj
 0002:00004608       ??_R1A@?0A@EA@DiamondClassifyWorkerFactory@LocalWorkflow@U2@@8 10025608     DiamondClassifyWorkerFactory.obj
 0002:00004624       ??_R4DiamondClassifyWorkerFactory@LocalWorkflow@U2@@6BDescriptor@2@@ 10025624     DiamondClassifyWorkerFactory.obj
 0002:00004638       ??_R4DatabaseDelegate@LocalWorkflow@U2@@6B@ 10025638     DiamondClassifyWorkerFactory.obj
 0002:0000464c       ??_R3DatabaseDelegate@LocalWorkflow@U2@@8 1002564c     DiamondClassifyWorkerFactory.obj
 0002:0000465c       ??_R2DatabaseDelegate@LocalWorkflow@U2@@8 1002565c     DiamondClassifyWorkerFactory.obj
 0002:00004678       ??_R1A@?0A@EA@DatabaseDelegate@LocalWorkflow@U2@@8 10025678     DiamondClassifyWorkerFactory.obj
 0002:00004694       ??_R4DiamondSupport@U2@@6B@ 10025694     DiamondSupport.obj
 0002:000046a8       ??_R3DiamondSupport@U2@@8  100256a8     DiamondSupport.obj
 0002:000046b8       ??_R2DiamondSupport@U2@@8  100256b8     DiamondSupport.obj
 0002:000046c8       ??_R1A@?0A@EA@DiamondSupport@U2@@8 100256c8     DiamondSupport.obj
 0002:000046e4       ??_R1A@?0A@EA@ExternalTool@U2@@8 100256e4     DiamondSupport.obj
 0002:00004700       ??_R3ExternalTool@U2@@8    10025700     DiamondSupport.obj
 0002:00004710       ??_R2ExternalTool@U2@@8    10025710     DiamondSupport.obj
 0002:0000471c       ??_R4DiamondSupportPlugin@U2@@6B@ 1002571c     DiamondSupportPlugin.obj
 0002:00004730       ??_R3DiamondSupportPlugin@U2@@8 10025730     DiamondSupportPlugin.obj
 0002:00004740       ??_R2DiamondSupportPlugin@U2@@8 10025740     DiamondSupportPlugin.obj
 0002:00004750       ??_R1A@?0A@EA@DiamondSupportPlugin@U2@@8 10025750     DiamondSupportPlugin.obj
 0002:0000476c       ??_R1A@?0A@EA@Plugin@U2@@8 1002576c     DiamondSupportPlugin.obj
 0002:00004788       ??_R3Plugin@U2@@8          10025788     DiamondSupportPlugin.obj
 0002:00004798       ??_R2Plugin@U2@@8          10025798     DiamondSupportPlugin.obj
 0002:000047a4       ??_R4GenomesPreparationTask@U2@@6B@ 100257a4     GenomesPreparationTask.obj
 0002:000047b8       ??_R3GenomesPreparationTask@U2@@8 100257b8     GenomesPreparationTask.obj
 0002:000047c8       ??_R2GenomesPreparationTask@U2@@8 100257c8     GenomesPreparationTask.obj
 0002:000047d8       ??_R1A@?0A@EA@GenomesPreparationTask@U2@@8 100257d8     GenomesPreparationTask.obj
 0002:000047f4       ??_R4type_info@@6B@        100257f4     MSVCRT:ti_inst.obj
 0002:00004808       ??_R3type_info@@8          10025808     MSVCRT:ti_inst.obj
 0002:00004818       ??_R2type_info@@8          10025818     MSVCRT:ti_inst.obj
 0002:00004820       ??_R1A@?0A@EA@type_info@@8 10025820     MSVCRT:ti_inst.obj
 0002:00004840       ___safe_se_handler_table   10025840     <linker-defined>
 0002:00004cb8       ___rtc_iaa                 10025cb8     MSVCRT:initsect.obj
 0002:00004cbc       ___rtc_izz                 10025cbc     MSVCRT:initsect.obj
 0002:00004cc0       ___rtc_taa                 10025cc0     MSVCRT:initsect.obj
 0002:00004cc4       ___rtc_tzz                 10025cc4     MSVCRT:initsect.obj
 0002:0000a228       __IMPORT_DESCRIPTOR_ngs_reads_classification 1002b228     ngs_reads_classification:ngs_reads_classification.dll
 0002:0000a23c       __IMPORT_DESCRIPTOR_U2Core 1002b23c     U2Core:U2Core.dll
 0002:0000a250       __IMPORT_DESCRIPTOR_U2Formats 1002b250     U2Formats:U2Formats.dll
 0002:0000a264       __IMPORT_DESCRIPTOR_U2Gui  1002b264     U2Gui:U2Gui.dll
 0002:0000a278       __IMPORT_DESCRIPTOR_U2Lang 1002b278     U2Lang:U2Lang.dll
 0002:0000a28c       __IMPORT_DESCRIPTOR_U2Designer 1002b28c     U2Designer:U2Designer.dll
 0002:0000a2a0       __IMPORT_DESCRIPTOR_Qt5Widgets 1002b2a0     Qt5Widgets:Qt5Widgets.dll
 0002:0000a2b4       __IMPORT_DESCRIPTOR_Qt5Gui 1002b2b4     Qt5Gui:Qt5Gui.dll
 0002:0000a2c8       __IMPORT_DESCRIPTOR_Qt5Script 1002b2c8     Qt5Script:Qt5Script.dll
 0002:0000a2dc       __IMPORT_DESCRIPTOR_Qt5Core 1002b2dc     Qt5Core:Qt5Core.dll
 0002:0000a2f0       __IMPORT_DESCRIPTOR_MSVCP120 1002b2f0     msvcprt:MSVCP120.dll
 0002:0000a304       __IMPORT_DESCRIPTOR_MSVCR120 1002b304     MSVCRT:MSVCR120.dll
 0002:0000a318       __IMPORT_DESCRIPTOR_KERNEL32 1002b318     kernel32:KERNEL32.dll
 0002:0000a32c       __NULL_IMPORT_DESCRIPTOR   1002b32c     ngs_reads_classification:ngs_reads_classification.dll
 0003:00000000       ?_Generic_object@?$_Error_objects@H@std@@2V_Generic_error_category@2@A 10033000     DiamondBuildPrompter.obj
 0003:00000004       ?_Iostream_object@?$_Error_objects@H@std@@2V_Iostream_error_category@2@A 10033004     DiamondBuildPrompter.obj
 0003:00000008       ?_System_object@?$_Error_objects@H@std@@2V_System_error_category@2@A 10033008     DiamondBuildPrompter.obj
 0003:0000000c       ?staticMetaObject@DiamondBuildPrompter@LocalWorkflow@U2@@2UQMetaObject@@B 1003300c     moc_DiamondBuildPrompter.obj
 0003:00000024       ?staticMetaObject@DiamondBuildTask@U2@@2UQMetaObject@@B 10033024     moc_DiamondBuildTask.obj
 0003:0000003c       ?staticMetaObject@DiamondBuildWorker@LocalWorkflow@U2@@2UQMetaObject@@B 1003303c     moc_DiamondBuildWorker.obj
 0003:00000054       ?staticMetaObject@DiamondClassifyPrompter@LocalWorkflow@U2@@2UQMetaObject@@B 10033054     moc_DiamondClassifyPrompter.obj
 0003:0000006c       ?staticMetaObject@DiamondClassifyTask@U2@@2UQMetaObject@@B 1003306c     moc_DiamondClassifyTask.obj
 0003:00000084       ?staticMetaObject@DiamondClassifyWorker@LocalWorkflow@U2@@2UQMetaObject@@B 10033084     moc_DiamondClassifyWorker.obj
 0003:0000009c       ?staticMetaObject@DiamondSupport@U2@@2UQMetaObject@@B 1003309c     moc_DiamondSupport.obj
 0003:000000b4       ?staticMetaObject@DiamondSupportPlugin@U2@@2UQMetaObject@@B 100330b4     moc_DiamondSupportPlugin.obj
 0003:000000cc       ?staticMetaObject@GenomesPreparationTask@U2@@2UQMetaObject@@B 100330cc     moc_GenomesPreparationTask.obj
 0003:000000e4       ___security_cookie         100330e4     MSVCRT:gs_cookie.obj
 0003:000000e8       ___security_cookie_complement 100330e8     MSVCRT:gs_cookie.obj
 0003:000000f0       ___native_dllmain_reason   100330f0     MSVCRT:natstart.obj
 0003:000000f8       ??_R0?AVerror_category@std@@@8 100330f8     DiamondBuildPrompter.obj
 0003:0000011c       ??_R0?AV_Generic_error_category@std@@@8 1003311c     DiamondBuildPrompter.obj
 0003:00000148       ??_R0?AV_Iostream_error_category@std@@@8 10033148     DiamondBuildPrompter.obj
 0003:00000174       ??_R0?AV_System_error_category@std@@@8 10033174     DiamondBuildPrompter.obj
 0003:000001a0       ??_R0?AVQObject@@@8        100331a0     DiamondBuildPrompter.obj
 0003:000001b8       ??_R0?AVDiamondBuildPrompter@LocalWorkflow@U2@@@8 100331b8     DiamondBuildPrompter.obj
 0003:000001f0       ??_R0?AV?$PrompterBase@VDiamondBuildPrompter@LocalWorkflow@U2@@@U2@@@8 100331f0     DiamondBuildPrompter.obj
 0003:0000023c       ??_R0?AVPrompterBaseImpl@U2@@@8 1003323c     DiamondBuildPrompter.obj
 0003:00000260       ??_R0?AVActorDocument@Workflow@U2@@@8 10033260     DiamondBuildPrompter.obj
 0003:00000288       ??_R0?AVQTextDocument@@@8  10033288     DiamondBuildPrompter.obj
 0003:000002a4       ??_R0?AVPrompter@Workflow@U2@@@8 100332a4     DiamondBuildPrompter.obj
 0003:000002c8       ??_R0?AVExternalToolLogParser@U2@@@8 100332c8     DiamondBuildTask.obj
 0003:000002f0       ??_R0?AVExternalToolRunTask@U2@@@8 100332f0     DiamondBuildTask.obj
 0003:00000318       ??_R0?AVTask@U2@@@8        10033318     DiamondBuildTask.obj
 0003:00000330       ??_R0?AVDiamondBuildTask@U2@@@8 10033330     DiamondBuildTask.obj
 0003:00000354       ??_R0?AVExternalToolSupportTask@U2@@@8 10033354     DiamondBuildTask.obj
 0003:00000380       ??_R0?AVFailTask@U2@@@8    10033380     DiamondBuildWorker.obj
 0003:0000039c       ??_R0?AVTaskSignalMapper@U2@@@8 1003339c     DiamondBuildWorker.obj
 0003:000003c0       ??_R0?AVDescriptor@U2@@@8  100333c0     DiamondBuildWorker.obj
 0003:000003dc       ??_R0?AVDiamondBuildWorker@LocalWorkflow@U2@@@8 100333dc     DiamondBuildWorker.obj
 0003:00000410       ??_R0?AVBaseWorker@LocalWorkflow@U2@@@8 10033410     DiamondBuildWorker.obj
 0003:0000043c       ??_R0?AVWorker@Workflow@U2@@@8 1003343c     DiamondBuildWorker.obj
 0003:00000460       ??_R0?AVCommunicationSubject@Workflow@U2@@@8 10033460     DiamondBuildWorker.obj
 0003:00000490       ??_R0?AVMapDataType@U2@@@8 10033490     DiamondBuildWorkerFactory.obj
 0003:000004b0       ??_R0?AVDataType@U2@@@8    100334b0     DiamondBuildWorkerFactory.obj
 0003:000004cc       ??_R0?AVQSharedData@@@8    100334cc     DiamondBuildWorkerFactory.obj
 0003:000004e8       ??_R0?AVAttribute@U2@@@8   100334e8     DiamondBuildWorkerFactory.obj
 0003:00000504       ??_R0?AVConfigurationEditor@U2@@@8 10033504     DiamondBuildWorkerFactory.obj
 0003:0000052c       ??_R0?AVDelegateEditor@U2@@@8 1003352c     DiamondBuildWorkerFactory.obj
 0003:0000054c       ??_R0?AVURLDelegate@U2@@@8 1003354c     DiamondBuildWorkerFactory.obj
 0003:0000056c       ??_R0?AVPropertyDelegate@U2@@@8 1003356c     DiamondBuildWorkerFactory.obj
 0003:00000590       ??_R0?AVQItemDelegate@@@8  10033590     DiamondBuildWorkerFactory.obj
 0003:000005ac       ??_R0?AVQAbstractItemDelegate@@@8 100335ac     DiamondBuildWorkerFactory.obj
 0003:000005d0       ??_R0?AVPortDescriptor@Workflow@U2@@@8 100335d0     DiamondBuildWorkerFactory.obj
 0003:000005fc       ??_R0?AVIntegralBusActorPrototype@Workflow@U2@@@8 100335fc     DiamondBuildWorkerFactory.obj
 0003:00000630       ??_R0?AVActorPrototype@Workflow@U2@@@8 10033630     DiamondBuildWorkerFactory.obj
 0003:0000065c       ??_R0?AVVisualDescriptor@U2@@@8 1003365c     DiamondBuildWorkerFactory.obj
 0003:00000680       ??_R0?AVDiamondBuildValidator@Workflow@U2@@@8 10033680     DiamondBuildWorkerFactory.obj
 0003:000006b0       ??_R0?AVActorValidator@Workflow@U2@@@8 100336b0     DiamondBuildWorkerFactory.obj
 0003:000006dc       ??_R0?AVConfigurationValidator@U2@@@8 100336dc     DiamondBuildWorkerFactory.obj
 0003:00000704       ??_R0?AVDiamondBuildWorkerFactory@LocalWorkflow@U2@@@8 10033704     DiamondBuildWorkerFactory.obj
 0003:00000740       ??_R0?AVDomainFactory@Workflow@U2@@@8 10033740     DiamondBuildWorkerFactory.obj
 0003:00000768       ??_R0?AV?$IdRegistry@VDomainFactory@Workflow@U2@@@U2@@@8 10033768     DiamondBuildWorkerFactory.obj
 0003:000007a4       ??_R0?AVGenomicLibraryDelegate@LocalWorkflow@U2@@@8 100337a4     DiamondBuildWorkerFactory.obj
 0003:000007dc       ??_R0?AVDiamondClassifyPrompter@LocalWorkflow@U2@@@8 100337dc     DiamondClassifyPrompter.obj
 0003:00000818       ??_R0?AV?$PrompterBase@VDiamondClassifyPrompter@LocalWorkflow@U2@@@U2@@@8 10033818     DiamondClassifyPrompter.obj
 0003:00000864       ??_R0?AVDiamondClassifyTask@U2@@@8 10033864     DiamondClassifyTask.obj
 0003:0000088c       ??_R0?AVDiamondClassifyWorker@LocalWorkflow@U2@@@8 1003388c     DiamondClassifyWorker.obj
 0003:000008c4       ??_R0?AVSpinBoxDelegate@U2@@@8 100338c4     DiamondClassifyWorkerFactory.obj
 0003:000008e8       ??_R0?AVDoubleSpinBoxDelegate@U2@@@8 100338e8     DiamondClassifyWorkerFactory.obj
 0003:00000910       ??_R0?AVComboBoxDelegate@U2@@@8 10033910     DiamondClassifyWorkerFactory.obj
 0003:00000934       ??_R0?AVDiamondClassifyWorkerFactory@LocalWorkflow@U2@@@8 10033934     DiamondClassifyWorkerFactory.obj
 0003:00000970       ??_R0?AVDatabaseDelegate@LocalWorkflow@U2@@@8 10033970     DiamondClassifyWorkerFactory.obj
 0003:000009a0       ??_R0?AVDiamondSupport@U2@@@8 100339a0     DiamondSupport.obj
 0003:000009c0       ??_R0?AVExternalTool@U2@@@8 100339c0     DiamondSupport.obj
 0003:000009e0       ??_R0?AVDiamondSupportPlugin@U2@@@8 100339e0     DiamondSupportPlugin.obj
 0003:00000a08       ??_R0?AVPlugin@U2@@@8      10033a08     DiamondSupportPlugin.obj
 0003:00000a20       ??_R0?AVGenomesPreparationTask@U2@@@8 10033a20     GenomesPreparationTask.obj
 0003:00000a48       ??_R0?AVtype_info@@@8      10033a48     MSVCRT:ti_inst.obj
 0003:00000aac       ?id@?$num_put@DV?$back_insert_iterator@V?$basic_string@DU?$char_traits@D@std@@V?$allocator@D@2@@std@@@std@@@std@@2V0locale@2@A 10033aac     DiamondBuildPrompter.obj
 0003:00000ab0       ?id@?$num_put@_WV?$back_insert_iterator@V?$basic_string@_WU?$char_traits@_W@std@@V?$allocator@_W@2@@std@@@std@@@std@@2V0locale@2@A 10033ab0     DiamondBuildPrompter.obj
 0003:00000ba4       ?DIAMOND_BUILD_DIR@DiamondBuildWorker@LocalWorkflow@U2@@0VQString@@B 10033ba4     DiamondBuildWorker.obj
 0003:00000bc8       ?metatype_id@?1??qt_metatype_id@?$QMetaTypeId@V?$QList@VDataset@U2@@@@@@SAHXZ@4V?$QBasicAtomicInteger@H@@A 10033bc8     DiamondBuildWorker.obj
 0003:00000bf8       ?ACTOR_ID@DiamondBuildWorkerFactory@LocalWorkflow@U2@@2VQString@@B 10033bf8     DiamondBuildWorkerFactory.obj
 0003:00000bfc       ?OUTPUT_PORT_ID@DiamondBuildWorkerFactory@LocalWorkflow@U2@@2VQString@@B 10033bfc     DiamondBuildWorkerFactory.obj
 0003:00000c18       ?DATABASE_ATTR_ID@DiamondBuildWorkerFactory@LocalWorkflow@U2@@2VQString@@B 10033c18     DiamondBuildWorkerFactory.obj
 0003:00000c24       ?GENOMIC_LIBRARY_ATTR_ID@DiamondBuildWorkerFactory@LocalWorkflow@U2@@2VQString@@B 10033c24     DiamondBuildWorkerFactory.obj
 0003:00000c80       ?SENSITIVE_ULTRA@DiamondClassifyTaskSettings@U2@@2VQString@@B 10033c80     DiamondClassifyTask.obj
 0003:00000c8c       ?BLOSUM50@DiamondClassifyTaskSettings@U2@@2VQString@@B 10033c8c     DiamondClassifyTask.obj
 0003:00000ca8       ?BLOSUM80@DiamondClassifyTaskSettings@U2@@2VQString@@B 10033ca8     DiamondClassifyTask.obj
 0003:00000cbc       ?SENSITIVE_DEFAULT@DiamondClassifyTaskSettings@U2@@2VQString@@B 10033cbc     DiamondClassifyTask.obj
 0003:00000cc0       ?BLOSUM62@DiamondClassifyTaskSettings@U2@@2VQString@@B 10033cc0     DiamondClassifyTask.obj
 0003:00000cc4       ?SENSITIVE_HIGH@DiamondClassifyTaskSettings@U2@@2VQString@@B 10033cc4     DiamondClassifyTask.obj
 0003:00000cd0       ?BLOSUM45@DiamondClassifyTaskSettings@U2@@2VQString@@B 10033cd0     DiamondClassifyTask.obj
 0003:00000cd4       ?PAM70@DiamondClassifyTaskSettings@U2@@2VQString@@B 10033cd4     DiamondClassifyTask.obj
 0003:00000ce0       ?BLOSUM90@DiamondClassifyTaskSettings@U2@@2VQString@@B 10033ce0     DiamondClassifyTask.obj
 0003:00000ce4       ?PAM30@DiamondClassifyTaskSettings@U2@@2VQString@@B 10033ce4     DiamondClassifyTask.obj
 0003:00000ce8       ?TAXONOMIC_CLASSIFICATION_OUTPUT_FORMAT@DiamondClassifyTask@U2@@0VQString@@B 10033ce8     DiamondClassifyTask.obj
 0003:00000cec       ?PAM250@DiamondClassifyTaskSettings@U2@@2VQString@@B 10033cec     DiamondClassifyTask.obj
 0003:00000d68       ?DIAMOND_DIR@DiamondClassifyWorker@LocalWorkflow@U2@@0VQString@@B 10033d68     DiamondClassifyWorker.obj
 0003:00000d6c       ?metatype_id@?1??qt_metatype_id@?$QMetaTypeId@VQAssociativeIterableImpl@QtMetaTypePrivate@@@@SAHXZ@4V?$QBasicAtomicInteger@H@@A 10033d6c     DiamondClassifyWorker.obj
 0003:00000d70       ?metatype_id@?1??qt_metatype_id@?$QMetaTypeId@V?$QMap@VQString@@I@@@@SAHXZ@4V?$QBasicAtomicInteger@H@@A 10033d70     DiamondClassifyWorker.obj
 0003:00000d74       ?f@?4??registerConverter@?$AssociativeValueTypeIsMetaType@V?$QMap@VQString@@I@@$00@QtPrivate@@SA_NH@Z@4U?$ConverterFunctor@V?$QMap@VQString@@I@@VQAssociativeIterableImpl@QtMetaTypePrivate@@U?$QAssociativeIterableConvertFunctor@V?$QMap@VQString@@I@@@3@@3@B 10033d74     DiamondClassifyWorker.obj
 0003:00000d7c       ??_B?4??registerConverter@?$AssociativeValueTypeIsMetaType@V?$QMap@VQString@@I@@$00@QtPrivate@@SA_NH@Z@54 10033d7c     DiamondClassifyWorker.obj
 0003:00000d84       ?OUTPUT_PORT_ID@DiamondClassifyWorkerFactory@LocalWorkflow@U2@@2VQString@@B 10033d84     DiamondClassifyWorkerFactory.obj
 0003:00000d88       ?CHUNKS_ATTR_ID@DiamondClassifyWorkerFactory@LocalWorkflow@U2@@2VQString@@B 10033d88     DiamondClassifyWorkerFactory.obj
 0003:00000d8c       ?ACTOR_ID@DiamondClassifyWorkerFactory@LocalWorkflow@U2@@2VQString@@B 10033d8c     DiamondClassifyWorkerFactory.obj
 0003:00000d90       ?MATRIX_ATTR_ID@DiamondClassifyWorkerFactory@LocalWorkflow@U2@@2VQString@@B 10033d90     DiamondClassifyWorkerFactory.obj
 0003:00000d94       ?OUTPUT_URL_ATTR_ID@DiamondClassifyWorkerFactory@LocalWorkflow@U2@@2VQString@@B 10033d94     DiamondClassifyWorkerFactory.obj
 0003:00000dc0       ?DATABASE_ATTR_ID@DiamondClassifyWorkerFactory@LocalWorkflow@U2@@2VQString@@B 10033dc0     DiamondClassifyWorkerFactory.obj
 0003:00000dc4       ?TOP_ALIGNMENTS_PERCENTAGE_ATTR_ID@DiamondClassifyWorkerFactory@LocalWorkflow@U2@@2VQString@@B 10033dc4     DiamondClassifyWorkerFactory.obj
 0003:00000dc8       ?THREADS_ATTR_ID@DiamondClassifyWorkerFactory@LocalWorkflow@U2@@2VQString@@B 10033dc8     DiamondClassifyWorkerFactory.obj
 0003:00000dcc       ?GO_PEN_ATTR_ID@DiamondClassifyWorkerFactory@LocalWorkflow@U2@@2VQString@@B 10033dcc     DiamondClassifyWorkerFactory.obj
 0003:00000dd0       ?FSHIFT_ATTR_ID@DiamondClassifyWorkerFactory@LocalWorkflow@U2@@2VQString@@B 10033dd0     DiamondClassifyWorkerFactory.obj
 0003:00000de4       ?GENCODE_ATTR_ID@DiamondClassifyWorkerFactory@LocalWorkflow@U2@@2VQString@@B 10033de4     DiamondClassifyWorkerFactory.obj
 0003:00000df0       ?INPUT_SLOT@DiamondClassifyWorkerFactory@LocalWorkflow@U2@@2VQString@@B 10033df0     DiamondClassifyWorkerFactory.obj
 0003:00000dfc       ?WORKFLOW_CLASSIFY_TOOL_DIAMOND@DiamondClassifyWorkerFactory@LocalWorkflow@U2@@2VQString@@B 10033dfc     DiamondClassifyWorkerFactory.obj
 0003:00000e00       ?SENSITIVE_ATTR_ID@DiamondClassifyWorkerFactory@LocalWorkflow@U2@@2VQString@@B 10033e00     DiamondClassifyWorkerFactory.obj
 0003:00000e04       ?INPUT_PORT_ID@DiamondClassifyWorkerFactory@LocalWorkflow@U2@@2VQString@@B 10033e04     DiamondClassifyWorkerFactory.obj
 0003:00000e08       ?EVALUE_ATTR_ID@DiamondClassifyWorkerFactory@LocalWorkflow@U2@@2VQString@@B 10033e08     DiamondClassifyWorkerFactory.obj
 0003:00000e0c       ?INPUT_DATA_ATTR_ID@DiamondClassifyWorkerFactory@LocalWorkflow@U2@@2VQString@@B 10033e0c     DiamondClassifyWorkerFactory.obj
 0003:00000e10       ?GE_PEN_ATTR_ID@DiamondClassifyWorkerFactory@LocalWorkflow@U2@@2VQString@@B 10033e10     DiamondClassifyWorkerFactory.obj
 0003:00000e14       ?BSIZE_ATTR_ID@DiamondClassifyWorkerFactory@LocalWorkflow@U2@@2VQString@@B 10033e14     DiamondClassifyWorkerFactory.obj
 0003:00000e1c       ?TOOL_NAME@DiamondSupport@U2@@2VQString@@B 10033e1c     DiamondSupport.obj
 0003:00000e5c       ?PLUGIN_NAME@DiamondSupportPlugin@U2@@2VQString@@B 10033e5c     DiamondSupportPlugin.obj
 0003:00000e70       ?PLUGIN_DESCRIPRION@DiamondSupportPlugin@U2@@2VQString@@B 10033e70     DiamondSupportPlugin.obj
 0003:00000fa4       ?metatype_id@?1??qt_metatype_id@?$QMetaTypeIdQObject@PAVTask@U2@@$00@@SAHXZ@4V?$QBasicAtomicInteger@H@@A 10033fa4     moc_DiamondBuildWorker.obj
 0003:00001408       ?__type_info_root_node@@3U__type_info_node@@A 10034408     MSVCRT:tncleanup.obj
 0003:00001410       ___native_startup_lock     10034410     <common>
 0003:00001414       ___native_startup_state    10034414     <common>
 0003:00001418       ___dyn_tls_init_callback   10034418     <common>
 0003:0000141c       ___onexitend               1003441c     <common>
 0003:00001420       ___onexitbegin             10034420     <common>

 entry point at        0001:000196ea

 Static symbols

 0000:fffc5000       .debug$S                   10000000     MSVCRT:MSVCR120.dll
 0000:fffc5000       .debug$S                   10000000     MSVCRT:MSVCR120.dll
 0000:fffc5000       .debug$S                   10000000     MSVCRT:MSVCR120.dll
 0000:fffc5000       .debug$S                   10000000     MSVCRT:MSVCR120.dll
 0000:fffc5000       .debug$S                   10000000     MSVCRT:MSVCR120.dll
 0000:fffc5000       .debug$S                   10000000     MSVCRT:MSVCR120.dll
 0000:fffc5000       .debug$S                   10000000     MSVCRT:MSVCR120.dll
 0000:fffc5000       .debug$S                   10000000     MSVCRT:MSVCR120.dll
 0000:fffc5000       .debug$S                   10000000     MSVCRT:MSVCR120.dll
 0002:fffdf000       __catchsym$??0?$QList@VQString@@@@QAE@ABV0@@Z$2 10000000     GenomesPreparationTask.obj
 0000:fffc5000       .debug$S                   10000000     MSVCRT:MSVCR120.dll
 0002:fffdf000       __catchsym$?_Copy@?$basic_string@DU?$char_traits@D@std@@V?$allocator@D@2@@std@@QAEXII@Z$5 10000000     DiamondBuildValidator.obj
 0000:fffc5000       .debug$S                   10000000     MSVCRT:MSVCR120.dll
 0002:fffdf000       ?_Generic_object$initializer$@?$_Error_objects@H@std@@2P6AXXZA 10000000     DiamondBuildValidator.obj
 0000:fffc5000       .debug$S                   10000000     MSVCRT:MSVCR120.dll
 0002:fffdf000       ?_Iostream_object$initializer$@?$_Error_objects@H@std@@2P6AXXZA 10000000     DiamondBuildValidator.obj
 0000:fffc5000       .debug$S                   10000000     MSVCRT:MSVCR120.dll
 0002:fffdf000       ?_System_object$initializer$@?$_Error_objects@H@std@@2P6AXXZA 10000000     DiamondBuildValidator.obj
 0000:fffc5000       .debug$S                   10000000     MSVCRT:MSVCR120.dll
 0002:fffdf000       ?_System_object$initializer$@?$_Error_objects@H@std@@2P6AXXZA 10000000     DiamondClassifyWorkerFactory.obj
 0000:fffc5000       .debug$S                   10000000     MSVCRT:MSVCR120.dll
 0002:fffdf000       ?_Iostream_object$initializer$@?$_Error_objects@H@std@@2P6AXXZA 10000000     DiamondClassifyWorkerFactory.obj
 0000:fffc5000       .debug$S                   10000000     MSVCRT:MSVCR120.dll
 0002:fffdf000       ?_Generic_object$initializer$@?$_Error_objects@H@std@@2P6AXXZA 10000000     DiamondClassifyWorkerFactory.obj
 0000:fffc5000       .debug$S                   10000000     MSVCRT:MSVCR120.dll
 0001:fffff000       __ehhandler$?_Copy@?$basic_string@DU?$char_traits@D@std@@V?$allocator@D@2@@std@@QAEXII@Z 10000000 f   DiamondClassifyWorker.obj
 0000:fffc5000       .debug$S                   10000000     MSVCRT:MSVCR120.dll
 0001:fffff000       __unwindfunclet$??H@YA?BVQString@@ABV0@0@Z$0 10000000 f   DiamondClassifyWorker.obj
 0001:fffff000       __unwindfunclet$??H@YA?BVQString@@ABV0@PBD@Z$0 10000000 f   DiamondClassifyWorker.obj
 0000:fffc5000       .debug$S                   10000000     MSVCRT:MSVCR120.dll
 0001:fffff000       __ehhandler$?_Copy@?$basic_string@DU?$char_traits@D@std@@V?$allocator@D@2@@std@@QAEXII@Z 10000000 f   DiamondBuildTask.obj
 0000:fffc5000       .debug$S                   10000000     MSVCRT:MSVCR120.dll
 0002:fffdf000       __catchsym$?createNode@?$QMapData@VQString@@PAVPropertyDelegate@U2@@@@QAEPAU?$QMapNode@VQString@@PAVPropertyDelegate@U2@@@@ABVQString@@ABQAVPropertyDelegate@U2@@PAU2@_N@Z$5 10000000     DiamondClassifyWorkerFactory.obj
 0000:fffc5000       .debug$S                   10000000     MSVCRT:MSVCR120.dll
 0001:fffff000       __ehhandler$?_Copy@?$basic_string@DU?$char_traits@D@std@@V?$allocator@D@2@@std@@QAEXII@Z 10000000 f   moc_GenomesPreparationTask.obj
 0002:fffdf000       __catchsym$?_Copy@?$basic_string@DU?$char_traits@D@std@@V?$allocator@D@2@@std@@QAEXII@Z$5 10000000     DiamondClassifyPrompter.obj
 0002:fffdf000       __catchsym$?createNode@?$QMapData@VDescriptor@U2@@V?$QExplicitlySharedDataPointer@VDataType@U2@@@@@@QAEPAU?$QMapNode@VDescriptor@U2@@V?$QExplicitlySharedDataPointer@VDataType@U2@@@@@@ABVDescriptor@U2@@ABV?$QExplicitlySharedDataPointer@VDataType@U2@@@@PAU2@_N@Z$6 10000000     DiamondClassifyWorkerFactory.obj
 0002:fffdf000       __catchsym$?node_copy@?$QList@VQString@@@@AAEXPAUNode@1@00@Z$6 10000000     GenomesPreparationTask.obj
 0002:fffdf000       __catchsym$?createNode@?$QMapData@VQString@@VQVariant@@@@QAEPAU?$QMapNode@VQString@@VQVariant@@@@ABVQString@@ABVQVariant@@PAU2@_N@Z$7 10000000     DiamondClassifyWorkerFactory.obj
 0001:fffff000       __unwindfunclet$?node_copy@?$QList@VQString@@@@AAEXPAUNode@1@00@Z$5 10000000 f   DiamondBuildWorker.obj
 0002:fffdf000       __catchsym$??0?$QList@PAVPort@Workflow@U2@@@@QAE@ABV0@@Z$2 10000000     DiamondClassifyPrompter.obj
 0002:fffdf000       __catchsym$?detach_helper_grow@?$QList@PAVPortDescriptor@Workflow@U2@@@@AAEPAUNode@1@HH@Z$5 10000000     DiamondClassifyWorkerFactory.obj
 0001:fffff000       __unwindfunclet$?node_construct@?$QList@VQString@@@@AAEXPAUNode@1@ABVQString@@@Z$1 10000000 f   DiamondBuildWorker.obj
 0000:fffc5000       .debug$S                   10000000     U2Core:U2Core.dll
 0002:fffdf000       __catchsym$?append@?$QList@PAVPortDescriptor@Workflow@U2@@@@QAEXABQAVPortDescriptor@Workflow@U2@@@Z$6 10000000     DiamondClassifyWorkerFactory.obj
 0000:fffc5000       .debug$S                   10000000     U2Core:U2Core.dll
 0001:fffff000       __ehhandler$?detach_helper_grow@?$QList@VQString@@@@AAEPAUNode@1@HH@Z 10000000 f   DiamondBuildWorker.obj
 0002:fffdf000       __catchsym$?detach_helper_grow@?$QList@PAVAttribute@U2@@@@AAEPAUNode@1@HH@Z$5 10000000     DiamondClassifyWorkerFactory.obj
 0001:fffff000       __unwindfunclet$?append@?$QList@VQString@@@@QAEXABVQString@@@Z$7 10000000 f   DiamondBuildWorker.obj
 0001:fffff000       __unwindfunclet$??0DiamondBuildTaskSettings@U2@@QAE@ABU01@@Z$0 10000000 f   DiamondBuildWorker.obj
 0002:fffdf000       __catchsym$?append@?$QList@PAVAttribute@U2@@@@QAEXABQAVAttribute@U2@@@Z$6 10000000     DiamondClassifyWorkerFactory.obj
 0000:fffc5000       .debug$S                   10000000     U2Core:U2Core.dll
 0002:fffdf000       __unwindtable$??A?$QMap@VDescriptor@U2@@V?$QExplicitlySharedDataPointer@VDataType@U2@@@@@@QAEAAV?$QExplicitlySharedDataPointer@VDataType@U2@@@@ABVDescriptor@U2@@@Z 10000000     DiamondClassifyWorkerFactory.obj
 0001:fffff000       __ehhandler$??0?$QList@VQString@@@@QAE@ABV0@@Z 10000000 f   DiamondBuildWorker.obj
 0000:fffc5000       .debug$S                   10000000     U2Core:U2Core.dll
 0002:fffdf000       ?_Generic_object$initializer$@?$_Error_objects@H@std@@2P6AXXZA 10000000     DiamondClassifyPrompter.obj
 0002:fffdf000       __catchsym$?_Copy@?$basic_string@DU?$char_traits@D@std@@V?$allocator@D@2@@std@@QAEXII@Z$5 10000000     DiamondBuildTask.obj
 0002:fffdf000       ?_Generic_object$initializer$@?$_Error_objects@H@std@@2P6AXXZA 10000000     DiamondBuildTask.obj
 0002:fffdf000       ?_Iostream_object$initializer$@?$_Error_objects@H@std@@2P6AXXZA 10000000     DiamondClassifyPrompter.obj
 0002:fffdf000       __catchsym$?_Copy@?$basic_string@DU?$char_traits@D@std@@V?$allocator@D@2@@std@@QAEXII@Z$5 10000000     moc_GenomesPreparationTask.obj
 0000:fffc5000       .debug$S                   10000000     MSVCRT:MSVCR120.dll
 0000:fffc5000       .debug$S                   10000000     MSVCRT:MSVCR120.dll
 0000:fffc5000       .debug$S                   10000000     MSVCRT:MSVCR120.dll
 0000:fffc5000       .debug$S                   10000000     MSVCRT:MSVCR120.dll
 0000:fffc5000       .debug$S                   10000000     MSVCRT:MSVCR120.dll
 0002:fffdf000       __unwindtable$??A?$QMap@VQString@@VQVariant@@@@QAEAAVQVariant@@ABVQString@@@Z 10000000     DiamondClassifyWorkerFactory.obj
 0002:fffdf000       ?_System_object$initializer$@?$_Error_objects@H@std@@2P6AXXZA 10000000     DiamondClassifyPrompter.obj
 0002:fffdf000       __unwindtable$??H@YA?BVQString@@ABV0@PBD@Z 10000000     DiamondClassifyWorkerFactory.obj
 0000:fffc5000       .debug$S                   10000000     U2Core:U2Core.dll
 0000:fffc5000       .debug$S                   10000000     msvcprt:MSVCP120.dll
 0000:fffc5000       .debug$S                   10000000     msvcprt:MSVCP120.dll
 0000:fffc5000       .debug$S                   10000000     msvcprt:MSVCP120.dll
 0000:fffc5000       .debug$S                   10000000     msvcprt:MSVCP120.dll
 0000:fffc5000       .debug$S                   10000000     msvcprt:MSVCP120.dll
 0000:fffc5000       .debug$S                   10000000     kernel32:KERNEL32.dll
 0000:fffc5000       .debug$S                   10000000     kernel32:KERNEL32.dll
 0000:fffc5000       .debug$S                   10000000     kernel32:KERNEL32.dll
 0000:fffc5000       .debug$S                   10000000     kernel32:KERNEL32.dll
 0000:fffc5000       .debug$S                   10000000     kernel32:KERNEL32.dll
 0000:fffc5000       .debug$S                   10000000     kernel32:KERNEL32.dll
 0000:fffc5000       .debug$S                   10000000     kernel32:KERNEL32.dll
 0000:fffc5000       .debug$S                   10000000     kernel32:KERNEL32.dll
 0000:fffc5000       .debug$S                   10000000     kernel32:KERNEL32.dll
 0000:fffc5000       .debug$S                   10000000     Qt5Core:Qt5Core.dll
 0000:fffc5000       .debug$S                   10000000     Qt5Core:Qt5Core.dll
 0000:fffc5000       .debug$S                   10000000     Qt5Core:Qt5Core.dll
 0000:fffc5000       .debug$S                   10000000     Qt5Core:Qt5Core.dll
 0000:fffc5000       .debug$S                   10000000     Qt5Core:Qt5Core.dll
 0000:fffc5000       .debug$S                   10000000     Qt5Core:Qt5Core.dll
 0000:fffc5000       .debug$S                   10000000     Qt5Core:Qt5Core.dll
 0000:fffc5000       .debug$S                   10000000     Qt5Core:Qt5Core.dll
 0000:fffc5000       .debug$S                   10000000     Qt5Core:Qt5Core.dll
 0000:fffc5000       .debug$S                   10000000     Qt5Core:Qt5Core.dll
 0000:fffc5000       .debug$S                   10000000     Qt5Core:Qt5Core.dll
 0000:fffc5000       .debug$S                   10000000     Qt5Core:Qt5Core.dll
 0000:fffc5000       .debug$S                   10000000     Qt5Core:Qt5Core.dll
 0000:fffc5000       .debug$S                   10000000     Qt5Core:Qt5Core.dll
 0000:fffc5000       .debug$S                   10000000     Qt5Core:Qt5Core.dll
 0000:fffc5000       .debug$S                   10000000     Qt5Core:Qt5Core.dll
 0000:fffc5000       .debug$S                   10000000     Qt5Core:Qt5Core.dll
 0000:fffc5000       .debug$S                   10000000     Qt5Core:Qt5Core.dll
 0002:fffdf000       ?_Generic_object$initializer$@?$_Error_objects@H@std@@2P6AXXZA 10000000     moc_GenomesPreparationTask.obj
 0002:fffdf000       ?_Iostream_object$initializer$@?$_Error_objects@H@std@@2P6AXXZA 10000000     moc_GenomesPreparationTask.obj
 0002:fffdf000       ?_System_object$initializer$@?$_Error_objects@H@std@@2P6AXXZA 10000000     moc_GenomesPreparationTask.obj
 0000:fffc5000       .debug$S                   10000000     Qt5Core:Qt5Core.dll
 0000:fffc5000       .debug$S                   10000000     Qt5Core:Qt5Core.dll
 0002:fffdf000       __catchsym$?_Copy@?$basic_string@DU?$char_traits@D@std@@V?$allocator@D@2@@std@@QAEXII@Z$5 10000000     DiamondClassifyWorkerFactory.obj
 0000:fffc5000       .debug$S                   10000000     U2Core:U2Core.dll
 0000:fffc5000       .debug$S                   10000000     Qt5Core:Qt5Core.dll
 0001:fffff000       __unwindfunclet$?createNode@?$QMapData@VQString@@PAVPropertyDelegate@U2@@@@QAEPAU?$QMapNode@VQString@@PAVPropertyDelegate@U2@@@@ABVQString@@ABQAVPropertyDelegate@U2@@PAU2@_N@Z$4 10000000 f   DiamondClassifyWorkerFactory.obj
 0000:fffc5000       .debug$S                   10000000     Qt5Core:Qt5Core.dll
 0001:fffff000       __unwindfunclet$?createNode@?$QMapData@VDescriptor@U2@@V?$QExplicitlySharedDataPointer@VDataType@U2@@@@@@QAEPAU?$QMapNode@VDescriptor@U2@@V?$QExplicitlySharedDataPointer@VDataType@U2@@@@@@ABVDescriptor@U2@@ABV?$QExplicitlySharedDataPointer@VDataType@U2@@@@PAU2@_N@Z$4 10000000 f   DiamondClassifyWorkerFactory.obj
 0000:fffc5000       .debug$S                   10000000     Qt5Core:Qt5Core.dll
 0001:fffff000       __ehhandler$?_Copy@?$basic_string@DU?$char_traits@D@std@@V?$allocator@D@2@@std@@QAEXII@Z 10000000 f   moc_DiamondSupportPlugin.obj
 0001:fffff000       __unwindfunclet$?createNode@?$QMapData@VQString@@VQVariant@@@@QAEPAU?$QMapNode@VQString@@VQVariant@@@@ABVQString@@ABVQVariant@@PAU2@_N@Z$4 10000000 f   DiamondClassifyWorkerFactory.obj
 0001:fffff000       __unwindfunclet$?append@?$QList@VQString@@@@QAEXABVQString@@@Z$7 10000000 f   DiamondClassifyWorker.obj
 0001:fffff000       __ehhandler$?detach_helper_grow@?$QList@VQString@@@@AAEPAUNode@1@HH@Z 10000000 f   DiamondClassifyWorker.obj
 0001:fffff000       __unwindfunclet$?node_construct@?$QList@VQString@@@@AAEXPAUNode@1@ABVQString@@@Z$1 10000000 f   DiamondClassifyWorker.obj
 0001:fffff000       __unwindfunclet$?node_copy@?$QList@VQString@@@@AAEXPAUNode@1@00@Z$5 10000000 f   DiamondClassifyWorker.obj
 0000:fffc5000       .debug$S                   10000000     U2Core:U2Core.dll
 0002:fffdf000       __catchsym$?_Copy@?$basic_string@DU?$char_traits@D@std@@V?$allocator@D@2@@std@@QAEXII@Z$5 10000000     moc_DiamondSupportPlugin.obj
 0000:fffc5000       .debug$S                   10000000     Qt5Core:Qt5Core.dll
 0000:fffc5000       .debug$S                   10000000     Qt5Core:Qt5Core.dll
 0000:fffc5000       .debug$S                   10000000     Qt5Core:Qt5Core.dll
 0000:fffc5000       .debug$S                   10000000     Qt5Core:Qt5Core.dll
 0000:fffc5000       .debug$S                   10000000     Qt5Core:Qt5Core.dll
 0002:fffdf000       ?_Generic_object$initializer$@?$_Error_objects@H@std@@2P6AXXZA 10000000     moc_DiamondSupportPlugin.obj
 0002:fffdf000       ?_Iostream_object$initializer$@?$_Error_objects@H@std@@2P6AXXZA 10000000     moc_DiamondSupportPlugin.obj
 0002:fffdf000       ?_System_object$initializer$@?$_Error_objects@H@std@@2P6AXXZA 10000000     moc_DiamondSupportPlugin.obj
 0000:fffc5000       .debug$S                   10000000     Qt5Core:Qt5Core.dll
 0000:fffc5000       .debug$S                   10000000     Qt5Core:Qt5Core.dll
 0000:fffc5000       .debug$S                   10000000     U2Core:U2Core.dll
 0001:fffff000       __unwindfunclet$??A?$QMap@VQString@@VQVariant@@@@QAEAAVQVariant@@ABVQString@@@Z$0 10000000 f   DiamondClassifyWorker.obj
 0000:fffc5000       .debug$S                   10000000     Qt5Core:Qt5Core.dll
 0001:fffff000       __ehhandler$??0?$QList@VDescriptor@U2@@@@QAE@ABV0@@Z 10000000 f   DiamondClassifyWorker.obj
 0000:fffc5000       .debug$S                   10000000     Qt5Core:Qt5Core.dll
 0000:fffc5000       .debug$S                   10000000     U2Core:U2Core.dll
 0000:fffc5000       .debug$S                   10000000     Qt5Core:Qt5Core.dll
 0001:fffff000       __ehhandler$?_Copy@?$basic_string@DU?$char_traits@D@std@@V?$allocator@D@2@@std@@QAEXII@Z 10000000 f   moc_DiamondSupport.obj
 0001:fffff000       __unwindfunclet$?append@?$QList@VDescriptor@U2@@@@QAEXABVDescriptor@U2@@@Z$6 10000000 f   DiamondClassifyWorker.obj
 0001:fffff000       __ehhandler$?detach_helper_grow@?$QList@VDescriptor@U2@@@@AAEPAUNode@1@HH@Z 10000000 f   DiamondClassifyWorker.obj
 0001:fffff000       __ehhandler$?detach_helper@?$QList@VDescriptor@U2@@@@AAEXH@Z 10000000 f   DiamondClassifyWorker.obj
 0000:fffc5000       .debug$S                   10000000     U2Core:U2Core.dll
 0001:fffff000       __unwindfunclet$?node_construct@?$QList@VDescriptor@U2@@@@AAEXPAUNode@1@ABVDescriptor@U2@@@Z$0 10000000 f   DiamondClassifyWorker.obj
 0000:fffc5000       .debug$S                   10000000     U2Core:U2Core.dll
 0002:fffdf000       __catchsym$?_Copy@?$basic_string@DU?$char_traits@D@std@@V?$allocator@D@2@@std@@QAEXII@Z$5 10000000     moc_DiamondSupport.obj
 0000:fffc5000       .debug$S                   10000000     Qt5Core:Qt5Core.dll
 0000:fffc5000       .debug$S                   10000000     Qt5Core:Qt5Core.dll
 0000:fffc5000       .debug$S                   10000000     Qt5Core:Qt5Core.dll
 0000:fffc5000       .debug$S                   10000000     Qt5Core:Qt5Core.dll
 0000:fffc5000       .debug$S                   10000000     Qt5Core:Qt5Core.dll
 0002:fffdf000       ?_Generic_object$initializer$@?$_Error_objects@H@std@@2P6AXXZA 10000000     moc_DiamondSupport.obj
 0002:fffdf000       ?_Iostream_object$initializer$@?$_Error_objects@H@std@@2P6AXXZA 10000000     moc_DiamondSupport.obj
 0002:fffdf000       ?_System_object$initializer$@?$_Error_objects@H@std@@2P6AXXZA 10000000     moc_DiamondSupport.obj
 0000:fffc5000       .debug$S                   10000000     Qt5Core:Qt5Core.dll
 0000:fffc5000       .debug$S                   10000000     Qt5Core:Qt5Core.dll
 0000:fffc5000       .debug$S                   10000000     U2Core:U2Core.dll
 0000:fffc5000       .debug$S                   10000000     Qt5Core:Qt5Core.dll
 0001:fffff000       __unwindfunclet$?node_copy@?$QList@VDescriptor@U2@@@@AAEXPAUNode@1@00@Z$4 10000000 f   DiamondClassifyWorker.obj
 0000:fffc5000       .debug$S                   10000000     Qt5Core:Qt5Core.dll
 0000:fffc5000       .debug$S                   10000000     U2Core:U2Core.dll
 0000:fffc5000       .debug$S                   10000000     Qt5Core:Qt5Core.dll
 0001:fffff000       __unwindfunclet$??A?$QMap@VQString@@VQScriptValue@@@@QAEAAVQScriptValue@@ABVQString@@@Z$0 10000000 f   DiamondClassifyWorker.obj
 0000:fffc5000       .debug$S                   10000000     Qt5Core:Qt5Core.dll
 0001:fffff000       __unwindfunclet$?uniqueKeys@?$QMap@VDescriptor@U2@@VQVariant@@@@QBE?AV?$QList@VDescriptor@U2@@@@XZ$1 10000000 f   DiamondClassifyWorker.obj
 0000:fffc5000       .debug$S                   10000000     Qt5Core:Qt5Core.dll
 0001:fffff000       __unwindfunclet$??$getAttributeValue@VQString@@@Attribute@U2@@QBE?AVQString@@PAVWorkflowContext@Workflow@1@@Z$0 10000000 f   DiamondClassifyWorker.obj
 0000:fffc5000       .debug$S                   10000000     Qt5Core:Qt5Core.dll
 0001:fffff000       __unwindfunclet$??$getValue@VQString@@@BaseWorker@LocalWorkflow@U2@@IBE?AVQString@@ABV3@@Z$0 10000000 f   DiamondClassifyWorker.obj
 0000:fffc5000       .debug$S                   10000000     Qt5Core:Qt5Core.dll
 0001:fffff000       __unwindfunclet$??1DiamondClassifyTaskSettings@U2@@QAE@XZ$0 10000000 f   DiamondClassifyWorker.obj
 0000:fffc5000       .debug$S                   10000000     Qt5Core:Qt5Core.dll
 0000:fffc5000       .debug$S                   10000000     U2Core:U2Core.dll
 0000:fffc5000       .debug$S                   10000000     Qt5Core:Qt5Core.dll
 0001:fffff000       __unwindfunclet$??0DiamondClassifyTaskSettings@U2@@QAE@ABU01@@Z$0 10000000 f   DiamondClassifyWorker.obj
 0000:fffc5000       .debug$S                   10000000     U2Core:U2Core.dll
 0000:fffc5000       .debug$S                   10000000     Qt5Core:Qt5Core.dll
 0001:fffff000       __unwindfunclet$?createNode@?$QMapData@VQString@@VQVariant@@@@QAEPAU?$QMapNode@VQString@@VQVariant@@@@ABVQString@@ABVQVariant@@PAU2@_N@Z$4 10000000 f   DiamondClassifyWorker.obj
 0000:fffc5000       .debug$S                   10000000     Qt5Core:Qt5Core.dll
 0001:fffff000       __unwindfunclet$?createNode@?$QMapData@VQString@@VQScriptValue@@@@QAEPAU?$QMapNode@VQString@@VQScriptValue@@@@ABVQString@@ABVQScriptValue@@PAU2@_N@Z$4 10000000 f   DiamondClassifyWorker.obj
 0000:fffc5000       .debug$S                   10000000     Qt5Core:Qt5Core.dll
 0001:fffff000       __ehhandler$?_Copy@?$basic_string@DU?$char_traits@D@std@@V?$allocator@D@2@@std@@QAEXII@Z 10000000 f   moc_DiamondClassifyWorker.obj
 0001:fffff000       __unwindfunclet$?createNode@?$QMapData@VQString@@I@@QAEPAU?$QMapNode@VQString@@I@@ABVQString@@ABIPAU2@_N@Z$4 10000000 f   DiamondClassifyWorker.obj
 0001:fffff000       __unwindfunclet$?metaType@?$QVariantValueHelper@VQString@@@QtPrivate@@SA?AVQString@@ABVQVariant@@@Z$0 10000000 f   DiamondClassifyWorker.obj
 0000:fffc5000       .debug$S                   10000000     U2Core:U2Core.dll
 0001:fffff000       __ehhandler$?_Copy@?$basic_string@DU?$char_traits@D@std@@V?$allocator@D@2@@std@@QAEXII@Z 10000000 f   DiamondBuildWorker.obj
 0002:fffdf000       __catchsym$?_Copy@?$basic_string@DU?$char_traits@D@std@@V?$allocator@D@2@@std@@QAEXII@Z$5 10000000     DiamondClassifyWorker.obj
 0000:fffc5000       .debug$S                   10000000     U2Core:U2Core.dll
 0002:fffdf000       __unwindtable$??H@YA?BVQString@@ABV0@0@Z 10000000     DiamondClassifyWorker.obj
 0000:fffc5000       .debug$S                   10000000     U2Core:U2Core.dll
 0002:fffdf000       __unwindtable$??H@YA?BVQString@@ABV0@PBD@Z 10000000     DiamondClassifyWorker.obj
 0000:fffc5000       .debug$S                   10000000     U2Core:U2Core.dll
 0002:fffdf000       __catchsym$?append@?$QList@VQString@@@@QAEXABVQString@@@Z$13 10000000     DiamondClassifyWorker.obj
 0000:fffc5000       .debug$S                   10000000     U2Core:U2Core.dll
 0002:fffdf000       __catchsym$?detach_helper_grow@?$QList@VQString@@@@AAEPAUNode@1@HH@Z$5 10000000     DiamondClassifyWorker.obj
 0001:fffff000       __ehhandler$?_Copy@?$basic_string@DU?$char_traits@D@std@@V?$allocator@D@2@@std@@QAEXII@Z 10000000 f   DiamondBuildWorkerFactory.obj
 0002:fffdf000       __unwindtable$?node_construct@?$QList@VQString@@@@AAEXPAUNode@1@ABVQString@@@Z 10000000     DiamondClassifyWorker.obj
 0000:fffc5000       .debug$S                   10000000     U2Core:U2Core.dll
 0002:fffdf000       __catchsym$?node_copy@?$QList@VQString@@@@AAEXPAUNode@1@00@Z$6 10000000     DiamondClassifyWorker.obj
 0002:fffdf000       ?_System_object$initializer$@?$_Error_objects@H@std@@2P6AXXZA 10000000     DiamondBuildWorkerFactory.obj
 0002:fffdf000       ?_Iostream_object$initializer$@?$_Error_objects@H@std@@2P6AXXZA 10000000     DiamondBuildWorkerFactory.obj
 0002:fffdf000       ?_Generic_object$initializer$@?$_Error_objects@H@std@@2P6AXXZA 10000000     DiamondBuildWorkerFactory.obj
 0000:fffc5000       .debug$S                   10000000     U2Core:U2Core.dll
 0001:fffff000       __unwindfunclet$?qt_metatype_id@?$QMetaTypeIdQObject@PAVTask@U2@@$00@@SAHXZ$0 10000000 f   moc_DiamondClassifyWorker.obj
 0000:fffc5000       .debug$S                   10000000     U2Core:U2Core.dll
 0002:fffdf000       __unwindtable$??A?$QMap@VQString@@VQVariant@@@@QAEAAVQVariant@@ABVQString@@@Z 10000000     DiamondClassifyWorker.obj
 0001:fffff000       __unwindfunclet$??H@YA?BVQString@@ABV0@PBD@Z$0 10000000 f   DiamondBuildWorkerFactory.obj
 0000:fffc5000       .debug$S                   10000000     U2Core:U2Core.dll
 0002:fffdf000       __catchsym$?_Copy@?$basic_string@DU?$char_traits@D@std@@V?$allocator@D@2@@std@@QAEXII@Z$5 10000000     moc_DiamondClassifyWorker.obj
 0000:fffc5000       .debug$S                   10000000     Qt5Core:Qt5Core.dll
 0000:fffc5000       .debug$S                   10000000     Qt5Core:Qt5Core.dll
 0000:fffc5000       .debug$S                   10000000     Qt5Core:Qt5Core.dll
 0000:fffc5000       .debug$S                   10000000     Qt5Core:Qt5Core.dll
 0000:fffc5000       .debug$S                   10000000     Qt5Core:Qt5Core.dll
 0000:fffc5000       .debug$S                   10000000     Qt5Core:Qt5Core.dll
 0000:fffc5000       .debug$S                   10000000     Qt5Core:Qt5Core.dll
 0000:fffc5000       .debug$S                   10000000     Qt5Core:Qt5Core.dll
 0000:fffc5000       .debug$S                   10000000     Qt5Core:Qt5Core.dll
 0000:fffc5000       .debug$S                   10000000     Qt5Core:Qt5Core.dll
 0000:fffc5000       .debug$S                   10000000     Qt5Core:Qt5Core.dll
 0000:fffc5000       .debug$S                   10000000     Qt5Core:Qt5Core.dll
 0000:fffc5000       .debug$S                   10000000     Qt5Core:Qt5Core.dll
 0000:fffc5000       .debug$S                   10000000     Qt5Core:Qt5Core.dll
 0000:fffc5000       .debug$S                   10000000     Qt5Core:Qt5Core.dll
 0000:fffc5000       .debug$S                   10000000     Qt5Core:Qt5Core.dll
 0000:fffc5000       .debug$S                   10000000     Qt5Core:Qt5Core.dll
 0000:fffc5000       .debug$S                   10000000     Qt5Core:Qt5Core.dll
 0001:fffff000       __unwindfunclet$?node_copy@?$QList@VQString@@@@AAEXPAUNode@1@00@Z$5 10000000 f   GenomesPreparationTask.obj
 0002:fffdf000       __unwindtable$?qt_metatype_id@?$QMetaTypeIdQObject@PAVTask@U2@@$00@@SAHXZ 10000000     moc_DiamondClassifyWorker.obj
 0000:fffc5000       .debug$S                   10000000     Qt5Core:Qt5Core.dll
 0000:fffc5000       .debug$S                   10000000     Qt5Core:Qt5Core.dll
 0000:fffc5000       .debug$S                   10000000     Qt5Core:Qt5Core.dll
 0000:fffc5000       .debug$S                   10000000     Qt5Core:Qt5Core.dll
 0000:fffc5000       .debug$S                   10000000     Qt5Core:Qt5Core.dll
 0000:fffc5000       .debug$S                   10000000     Qt5Core:Qt5Core.dll
 0000:fffc5000       .debug$S                   10000000     Qt5Core:Qt5Core.dll
 0000:fffc5000       .debug$S                   10000000     Qt5Core:Qt5Core.dll
 0000:fffc5000       .debug$S                   10000000     Qt5Core:Qt5Core.dll
 0000:fffc5000       .debug$S                   10000000     Qt5Core:Qt5Core.dll
 0000:fffc5000       .debug$S                   10000000     Qt5Core:Qt5Core.dll
 0000:fffc5000       .debug$S                   10000000     Qt5Core:Qt5Core.dll
 0000:fffc5000       .debug$S                   10000000     Qt5Core:Qt5Core.dll
 0000:fffc5000       .debug$S                   10000000     Qt5Core:Qt5Core.dll
 0000:fffc5000       .debug$S                   10000000     Qt5Core:Qt5Core.dll
 0000:fffc5000       .debug$S                   10000000     Qt5Core:Qt5Core.dll
 0000:fffc5000       .debug$S                   10000000     Qt5Core:Qt5Core.dll
 0000:fffc5000       .debug$S                   10000000     Qt5Core:Qt5Core.dll
 0000:fffc5000       .debug$S                   10000000     Qt5Core:Qt5Core.dll
 0000:fffc5000       .debug$S                   10000000     Qt5Core:Qt5Core.dll
 0000:fffc5000       .debug$S                   10000000     Qt5Core:Qt5Core.dll
 0000:fffc5000       .debug$S                   10000000     Qt5Core:Qt5Core.dll
 0000:fffc5000       .debug$S                   10000000     Qt5Core:Qt5Core.dll
 0002:fffdf000       ?_Generic_object$initializer$@?$_Error_objects@H@std@@2P6AXXZA 10000000     moc_DiamondClassifyWorker.obj
 0002:fffdf000       ?_Iostream_object$initializer$@?$_Error_objects@H@std@@2P6AXXZA 10000000     moc_DiamondClassifyWorker.obj
 0002:fffdf000       ?_System_object$initializer$@?$_Error_objects@H@std@@2P6AXXZA 10000000     moc_DiamondClassifyWorker.obj
 0000:fffc5000       .debug$S                   10000000     Qt5Core:Qt5Core.dll
 0000:fffc5000       .debug$S                   10000000     Qt5Core:Qt5Core.dll
 0002:fffdf000       __catchsym$??0?$QList@VDescriptor@U2@@@@QAE@ABV0@@Z$2 10000000     DiamondClassifyWorker.obj
 0000:fffc5000       .debug$S                   10000000     Qt5Script:Qt5Script.dll
 0000:fffc5000       .debug$S                   10000000     U2Core:U2Core.dll
 0000:fffc5000       .debug$S                   10000000     Qt5Script:Qt5Script.dll
 0002:fffdf000       __catchsym$?append@?$QList@VDescriptor@U2@@@@QAEXABVDescriptor@U2@@@Z$9 10000000     DiamondClassifyWorker.obj
 0000:fffc5000       .debug$S                   10000000     Qt5Script:Qt5Script.dll
 0000:fffc5000       .debug$S                   10000000     U2Core:U2Core.dll
 0000:fffc5000       .debug$S                   10000000     Qt5Script:Qt5Script.dll
 0002:fffdf000       __catchsym$?detach_helper_grow@?$QList@VDescriptor@U2@@@@AAEPAUNode@1@HH@Z$5 10000000     DiamondClassifyWorker.obj
 0000:fffc5000       .debug$S                   10000000     Qt5Script:Qt5Script.dll
 0000:fffc5000       .debug$S                   10000000     U2Core:U2Core.dll
 0000:fffc5000       .debug$S                   10000000     Qt5Script:Qt5Script.dll
 0002:fffdf000       __catchsym$?detach_helper@?$QList@VDescriptor@U2@@@@AAEXH@Z$2 10000000     DiamondClassifyWorker.obj
 0000:fffc5000       .debug$S                   10000000     Qt5Script:Qt5Script.dll
 0001:fffff000       __ehhandler$??0?$QList@VQString@@@@QAE@ABV0@@Z 10000000 f   GenomesPreparationTask.obj
 0000:fffc5000       .debug$S                   10000000     Qt5Script:Qt5Script.dll
 0002:fffdf000       __unwindtable$?node_construct@?$QList@VDescriptor@U2@@@@AAEXPAUNode@1@ABVDescriptor@U2@@@Z 10000000     DiamondClassifyWorker.obj
 0000:fffc5000       .debug$S                   10000000     Qt5Script:Qt5Script.dll
 0000:fffc5000       .debug$S                   10000000     U2Core:U2Core.dll
 0002:fffdf000       __catchsym$?node_copy@?$QList@VDescriptor@U2@@@@AAEXPAUNode@1@00@Z$6 10000000     DiamondClassifyWorker.obj
 0000:fffc5000       .debug$S                   10000000     Qt5Script:Qt5Script.dll
 0000:fffc5000       .debug$S                   10000000     U2Core:U2Core.dll
 0000:fffc5000       .debug$S                   10000000     Qt5Gui:Qt5Gui.dll
 0002:fffdf000       __unwindtable$??A?$QMap@VQString@@VQScriptValue@@@@QAEAAVQScriptValue@@ABVQString@@@Z 10000000     DiamondClassifyWorker.obj
 0000:fffc5000       .debug$S                   10000000     Qt5Gui:Qt5Gui.dll
 0001:fffff000       __ehhandler$?_Copy@?$basic_string@DU?$char_traits@D@std@@V?$allocator@D@2@@std@@QAEXII@Z 10000000 f   moc_DiamondClassifyTask.obj
 0001:fffff000       __ehhandler$?_Copy@?$basic_string@DU?$char_traits@D@std@@V?$allocator@D@2@@std@@QAEXII@Z 10000000 f   GenomesPreparationTask.obj
 0002:fffdf000       __unwindtable$?uniqueKeys@?$QMap@VDescriptor@U2@@VQVariant@@@@QBE?AV?$QList@VDescriptor@U2@@@@XZ 10000000     DiamondClassifyWorker.obj
 0002:fffdf000       __ehfuncinfo$??$getAttributeValue@VQString@@@Attribute@U2@@QBE?AVQString@@PAVWorkflowContext@Workflow@1@@Z 10000000     DiamondClassifyWorker.obj
 0000:fffc5000       .debug$S                   10000000     U2Core:U2Core.dll
 0002:fffdf000       __unwindtable$??$getValue@VQString@@@BaseWorker@LocalWorkflow@U2@@IBE?AVQString@@ABV3@@Z 10000000     DiamondClassifyWorker.obj
 0002:fffdf000       __ehfuncinfo$??1DiamondClassifyTaskSettings@U2@@QAE@XZ 10000000     DiamondClassifyWorker.obj
 0002:fffdf000       __ehfuncinfo$??0DiamondClassifyTaskSettings@U2@@QAE@ABU01@@Z 10000000     DiamondClassifyWorker.obj
 0000:fffc5000       .debug$S                   10000000     U2Core:U2Core.dll
 0002:fffdf000       __catchsym$?createNode@?$QMapData@VQString@@VQVariant@@@@QAEPAU?$QMapNode@VQString@@VQVariant@@@@ABVQString@@ABVQVariant@@PAU2@_N@Z$7 10000000     DiamondClassifyWorker.obj
 0000:fffc5000       .debug$S                   10000000     U2Core:U2Core.dll
 0002:fffdf000       __catchsym$?createNode@?$QMapData@VQString@@VQScriptValue@@@@QAEPAU?$QMapNode@VQString@@VQScriptValue@@@@ABVQString@@ABVQScriptValue@@PAU2@_N@Z$7 10000000     DiamondClassifyWorker.obj
 0000:fffc5000       .debug$S                   10000000     U2Core:U2Core.dll
 0002:fffdf000       __catchsym$?createNode@?$QMapData@VQString@@I@@QAEPAU?$QMapNode@VQString@@I@@ABVQString@@ABIPAU2@_N@Z$5 10000000     DiamondClassifyWorker.obj
 0000:fffc5000       .debug$S                   10000000     U2Core:U2Core.dll
 0002:fffdf000       __unwindtable$?metaType@?$QVariantValueHelper@VQString@@@QtPrivate@@SA?AVQString@@ABVQVariant@@@Z 10000000     DiamondClassifyWorker.obj
 0001:fffff000       __ehhandler$?_Copy@?$basic_string@DU?$char_traits@D@std@@V?$allocator@D@2@@std@@QAEXII@Z 10000000 f   DiamondBuildValidator.obj
 0002:fffdf000       ?_Generic_object$initializer$@?$_Error_objects@H@std@@2P6AXXZA 10000000     DiamondClassifyWorker.obj
 0002:fffdf000       ?_Iostream_object$initializer$@?$_Error_objects@H@std@@2P6AXXZA 10000000     DiamondClassifyWorker.obj
 0002:fffdf000       ?_System_object$initializer$@?$_Error_objects@H@std@@2P6AXXZA 10000000     DiamondClassifyWorker.obj
 0002:fffdf000       ?_System_object$initializer$@?$_Error_objects@H@std@@2P6AXXZA 10000000     DiamondBuildWorker.obj
 0002:fffdf000       ?_Iostream_object$initializer$@?$_Error_objects@H@std@@2P6AXXZA 10000000     DiamondBuildWorker.obj
 0002:fffdf000       ?_Generic_object$initializer$@?$_Error_objects@H@std@@2P6AXXZA 10000000     DiamondBuildWorker.obj
 0002:fffdf000       __unwindtable$??0DiamondBuildTaskSettings@U2@@QAE@ABU01@@Z 10000000     DiamondBuildWorker.obj
 0000:fffc5000       .debug$S                   10000000     U2Core:U2Core.dll
 0002:fffdf000       __catchsym$?_Copy@?$basic_string@DU?$char_traits@D@std@@V?$allocator@D@2@@std@@QAEXII@Z$5 10000000     moc_DiamondClassifyTask.obj
 0000:fffc5000       .debug$S                   10000000     Qt5Gui:Qt5Gui.dll
 0000:fffc5000       .debug$S                   10000000     Qt5Widgets:Qt5Widgets.dll
 0000:fffc5000       .debug$S                   10000000     Qt5Widgets:Qt5Widgets.dll
 0000:fffc5000       .debug$S                   10000000     Qt5Widgets:Qt5Widgets.dll
 0000:fffc5000       .debug$S                   10000000     Qt5Widgets:Qt5Widgets.dll
 0000:fffc5000       .debug$S                   10000000     Qt5Widgets:Qt5Widgets.dll
 0000:fffc5000       .debug$S                   10000000     Qt5Widgets:Qt5Widgets.dll
 0000:fffc5000       .debug$S                   10000000     Qt5Widgets:Qt5Widgets.dll
 0000:fffc5000       .debug$S                   10000000     Qt5Widgets:Qt5Widgets.dll
 0000:fffc5000       .debug$S                   10000000     Qt5Widgets:Qt5Widgets.dll
 0000:fffc5000       .debug$S                   10000000     Qt5Widgets:Qt5Widgets.dll
 0000:fffc5000       .debug$S                   10000000     Qt5Widgets:Qt5Widgets.dll
 0000:fffc5000       .debug$S                   10000000     Qt5Widgets:Qt5Widgets.dll
 0000:fffc5000       .debug$S                   10000000     U2Designer:U2Designer.dll
 0000:fffc5000       .debug$S                   10000000     U2Designer:U2Designer.dll
 0000:fffc5000       .debug$S                   10000000     U2Designer:U2Designer.dll
 0000:fffc5000       .debug$S                   10000000     U2Designer:U2Designer.dll
 0000:fffc5000       .debug$S                   10000000     U2Designer:U2Designer.dll
 0000:fffc5000       .debug$S                   10000000     U2Designer:U2Designer.dll
 0000:fffc5000       .debug$S                   10000000     U2Designer:U2Designer.dll
 0000:fffc5000       .debug$S                   10000000     U2Designer:U2Designer.dll
 0000:fffc5000       .debug$S                   10000000     U2Designer:U2Designer.dll
 0000:fffc5000       .debug$S                   10000000     U2Designer:U2Designer.dll
 0000:fffc5000       .debug$S                   10000000     U2Designer:U2Designer.dll
 0000:fffc5000       .debug$S                   10000000     U2Designer:U2Designer.dll
 0000:fffc5000       .debug$S                   10000000     U2Designer:U2Designer.dll
 0000:fffc5000       .debug$S                   10000000     U2Designer:U2Designer.dll
 0000:fffc5000       .debug$S                   10000000     U2Designer:U2Designer.dll
 0000:fffc5000       .debug$S                   10000000     U2Designer:U2Designer.dll
 0000:fffc5000       .debug$S                   10000000     U2Designer:U2Designer.dll
 0000:fffc5000       .debug$S                   10000000     U2Designer:U2Designer.dll
 0000:fffc5000       .debug$S                   10000000     U2Designer:U2Designer.dll
 0000:fffc5000       .debug$S                   10000000     U2Designer:U2Designer.dll
 0000:fffc5000       .debug$S                   10000000     U2Designer:U2Designer.dll
 0000:fffc5000       .debug$S                   10000000     U2Designer:U2Designer.dll
 0000:fffc5000       .debug$S                   10000000     U2Designer:U2Designer.dll
 0000:fffc5000       .debug$S                   10000000     U2Designer:U2Designer.dll
 0000:fffc5000       .debug$S                   10000000     U2Designer:U2Designer.dll
 0000:fffc5000       .debug$S                   10000000     U2Designer:U2Designer.dll
 0000:fffc5000       .debug$S                   10000000     U2Designer:U2Designer.dll
 0000:fffc5000       .debug$S                   10000000     U2Designer:U2Designer.dll
 0002:fffdf000       ?_Generic_object$initializer$@?$_Error_objects@H@std@@2P6AXXZA 10000000     moc_DiamondClassifyTask.obj
 0002:fffdf000       ?_Iostream_object$initializer$@?$_Error_objects@H@std@@2P6AXXZA 10000000     moc_DiamondClassifyTask.obj
 0002:fffdf000       ?_System_object$initializer$@?$_Error_objects@H@std@@2P6AXXZA 10000000     moc_DiamondClassifyTask.obj
 0000:fffc5000       .debug$S                   10000000     U2Designer:U2Designer.dll
 0000:fffc5000       .debug$S                   10000000     U2Designer:U2Designer.dll
 0002:fffdf000       __unwindtable$??1DiamondBuildTaskSettings@U2@@QAE@XZ 10000000     DiamondBuildWorker.obj
 0000:fffc5000       .debug$S                   10000000     U2Designer:U2Designer.dll
 0002:fffdf000       __catchsym$?node_copy@?$QList@VQString@@@@AAEXPAUNode@1@00@Z$6 10000000     DiamondBuildWorker.obj
 0000:fffc5000       .debug$S                   10000000     U2Designer:U2Designer.dll
 0000:fffc5000       .debug$S                   10000000     U2Core:U2Core.dll
 0000:fffc5000       .debug$S                   10000000     U2Designer:U2Designer.dll
 0002:fffdf000       __unwindtable$?node_construct@?$QList@VQString@@@@AAEXPAUNode@1@ABVQString@@@Z 10000000     DiamondBuildWorker.obj
 0000:fffc5000       .debug$S                   10000000     U2Designer:U2Designer.dll
 0000:fffc5000       .debug$S                   10000000     U2Core:U2Core.dll
 0000:fffc5000       .debug$S                   10000000     U2Designer:U2Designer.dll
 0002:fffdf000       __catchsym$?detach_helper_grow@?$QList@VQString@@@@AAEPAUNode@1@HH@Z$5 10000000     DiamondBuildWorker.obj
 0000:fffc5000       .debug$S                   10000000     U2Designer:U2Designer.dll
 0001:fffff000       __ehhandler$?_Copy@?$basic_string@DU?$char_traits@D@std@@V?$allocator@D@2@@std@@QAEXII@Z 10000000 f   DiamondClassifyTask.obj
 0000:fffc5000       .debug$S                   10000000     U2Designer:U2Designer.dll
 0001:fffff000       __ehhandler$??0?$QList@VQString@@@@QAE@ABV0@@Z 10000000 f   DiamondClassifyTask.obj
 0000:fffc5000       .debug$S                   10000000     U2Designer:U2Designer.dll
 0001:fffff000       __unwindfunclet$?append@?$QList@VQString@@@@QAEXABVQString@@@Z$7 10000000 f   DiamondClassifyTask.obj
 0000:fffc5000       .debug$S                   10000000     U2Designer:U2Designer.dll
 0001:fffff000       __ehhandler$?detach_helper_grow@?$QList@PAVPortDescriptor@Workflow@U2@@@@AAEPAUNode@1@HH@Z 10000000 f   DiamondClassifyWorkerFactory.obj
 0001:fffff000       __ehhandler$?append@?$QList@PAVPortDescriptor@Workflow@U2@@@@QAEXABQAVPortDescriptor@Workflow@U2@@@Z 10000000 f   DiamondClassifyWorkerFactory.obj
 0000:fffc5000       .debug$S                   10000000     U2Designer:U2Designer.dll
 0001:fffff000       __ehhandler$?detach_helper_grow@?$QList@PAVAttribute@U2@@@@AAEPAUNode@1@HH@Z 10000000 f   DiamondClassifyWorkerFactory.obj
 0000:fffc5000       .debug$S                   10000000     U2Designer:U2Designer.dll
 0001:fffff000       __ehhandler$?append@?$QList@PAVAttribute@U2@@@@QAEXABQAVAttribute@U2@@@Z 10000000 f   DiamondClassifyWorkerFactory.obj
 0000:fffc5000       .debug$S                   10000000     U2Designer:U2Designer.dll
 0001:fffff000       __ehhandler$?_Copy@?$basic_string@DU?$char_traits@D@std@@V?$allocator@D@2@@std@@QAEXII@Z 10000000 f   moc_DiamondClassifyPrompter.obj
 0001:fffff000       __ehhandler$?detach_helper_grow@?$QList@VQString@@@@AAEPAUNode@1@HH@Z 10000000 f   DiamondClassifyTask.obj
 0001:fffff000       __unwindfunclet$?node_construct@?$QList@VQString@@@@AAEXPAUNode@1@ABVQString@@@Z$1 10000000 f   DiamondClassifyTask.obj
 0001:fffff000       __unwindfunclet$?node_copy@?$QList@VQString@@@@AAEXPAUNode@1@00@Z$5 10000000 f   DiamondClassifyTask.obj
 0001:fffff000       __unwindfunclet$??A?$QMap@VDescriptor@U2@@V?$QExplicitlySharedDataPointer@VDataType@U2@@@@@@QAEAAV?$QExplicitlySharedDataPointer@VDataType@U2@@@@ABVDescriptor@U2@@@Z$0 10000000 f   DiamondClassifyWorkerFactory.obj
 0000:fffc5000       .debug$S                   10000000     U2Core:U2Core.dll
 0000:fffc5000       .debug$S                   10000000     U2Core:U2Core.dll
 0002:fffdf000       __catchsym$?_Copy@?$basic_string@DU?$char_traits@D@std@@V?$allocator@D@2@@std@@QAEXII@Z$5 10000000     DiamondClassifyTask.obj
 0000:fffc5000       .debug$S                   10000000     U2Core:U2Core.dll
 0002:fffdf000       __catchsym$?append@?$QList@VQString@@@@QAEXABVQString@@@Z$13 10000000     DiamondBuildWorker.obj
 0000:fffc5000       .debug$S                   10000000     U2Core:U2Core.dll
 0000:fffc5000       .debug$S                   10000000     U2Core:U2Core.dll
 0002:fffdf000       __catchsym$??0?$QList@VQString@@@@QAE@ABV0@@Z$2 10000000     DiamondClassifyTask.obj
 0000:fffc5000       .debug$S                   10000000     U2Core:U2Core.dll
 0002:fffdf000       __catchsym$?append@?$QList@VQString@@@@QAEXABVQString@@@Z$13 10000000     DiamondClassifyTask.obj
 0001:fffff000       __unwindfunclet$??A?$QMap@VQString@@VQVariant@@@@QAEAAVQVariant@@ABVQString@@@Z$0 10000000 f   DiamondClassifyWorkerFactory.obj
 0000:fffc5000       .debug$S                   10000000     U2Core:U2Core.dll
 0001:fffff000       __unwindfunclet$??H@YA?BVQString@@ABV0@PBD@Z$0 10000000 f   DiamondClassifyWorkerFactory.obj
 0001:fffff000       __ehhandler$?_Copy@?$basic_string@DU?$char_traits@D@std@@V?$allocator@D@2@@std@@QAEXII@Z 10000000 f   DiamondClassifyWorkerFactory.obj
 0002:fffdf000       ?_Iostream_object$initializer$@?$_Error_objects@H@std@@2P6AXXZA 10000000     DiamondBuildTask.obj
 0002:fffdf000       ?_System_object$initializer$@?$_Error_objects@H@std@@2P6AXXZA 10000000     DiamondBuildTask.obj
 0000:fffc5000       .debug$S                   10000000     U2Core:U2Core.dll
 0002:fffdf000       __catchsym$?detach_helper_grow@?$QList@VQString@@@@AAEPAUNode@1@HH@Z$5 10000000     DiamondClassifyTask.obj
 0000:fffc5000       .debug$S                   10000000     U2Core:U2Core.dll
 0000:fffc5000       .debug$S                   10000000     U2Core:U2Core.dll
 0002:fffdf000       __catchsym$?_Copy@?$basic_string@DU?$char_traits@D@std@@V?$allocator@D@2@@std@@QAEXII@Z$5 10000000     moc_DiamondClassifyPrompter.obj
 0000:fffc5000       .debug$S                   10000000     U2Designer:U2Designer.dll
 0000:fffc5000       .debug$S                   10000000     U2Designer:U2Designer.dll
 0000:fffc5000       .debug$S                   10000000     U2Designer:U2Designer.dll
 0000:fffc5000       .debug$S                   10000000     U2Designer:U2Designer.dll
 0000:fffc5000       .debug$S                   10000000     U2Designer:U2Designer.dll
 0000:fffc5000       .debug$S                   10000000     U2Designer:U2Designer.dll
 0000:fffc5000       .debug$S                   10000000     U2Designer:U2Designer.dll
 0000:fffc5000       .debug$S                   10000000     U2Designer:U2Designer.dll
 0000:fffc5000       .debug$S                   10000000     U2Designer:U2Designer.dll
 0000:fffc5000       .debug$S                   10000000     U2Designer:U2Designer.dll
 0000:fffc5000       .debug$S                   10000000     U2Designer:U2Designer.dll
 0000:fffc5000       .debug$S                   10000000     U2Designer:U2Designer.dll
 0000:fffc5000       .debug$S                   10000000     U2Designer:U2Designer.dll
 0000:fffc5000       .debug$S                   10000000     U2Designer:U2Designer.dll
 0000:fffc5000       .debug$S                   10000000     U2Designer:U2Designer.dll
 0000:fffc5000       .debug$S                   10000000     U2Designer:U2Designer.dll
 0000:fffc5000       .debug$S                   10000000     U2Designer:U2Designer.dll
 0000:fffc5000       .debug$S                   10000000     U2Designer:U2Designer.dll
 0000:fffc5000       .debug$S                   10000000     U2Designer:U2Designer.dll
 0000:fffc5000       .debug$S                   10000000     U2Designer:U2Designer.dll
 0000:fffc5000       .debug$S                   10000000     U2Lang:U2Lang.dll
 0000:fffc5000       .debug$S                   10000000     U2Lang:U2Lang.dll
 0000:fffc5000       .debug$S                   10000000     U2Lang:U2Lang.dll
 0000:fffc5000       .debug$S                   10000000     U2Lang:U2Lang.dll
 0000:fffc5000       .debug$S                   10000000     U2Lang:U2Lang.dll
 0000:fffc5000       .debug$S                   10000000     U2Lang:U2Lang.dll
 0000:fffc5000       .debug$S                   10000000     U2Lang:U2Lang.dll
 0000:fffc5000       .debug$S                   10000000     U2Lang:U2Lang.dll
 0000:fffc5000       .debug$S                   10000000     U2Lang:U2Lang.dll
 0000:fffc5000       .debug$S                   10000000     U2Lang:U2Lang.dll
 0000:fffc5000       .debug$S                   10000000     U2Lang:U2Lang.dll
 0000:fffc5000       .debug$S                   10000000     U2Lang:U2Lang.dll
 0000:fffc5000       .debug$S                   10000000     U2Lang:U2Lang.dll
 0000:fffc5000       .debug$S                   10000000     U2Lang:U2Lang.dll
 0000:fffc5000       .debug$S                   10000000     U2Lang:U2Lang.dll
 0000:fffc5000       .debug$S                   10000000     U2Lang:U2Lang.dll
 0000:fffc5000       .debug$S                   10000000     U2Lang:U2Lang.dll
 0000:fffc5000       .debug$S                   10000000     U2Lang:U2Lang.dll
 0000:fffc5000       .debug$S                   10000000     U2Lang:U2Lang.dll
 0000:fffc5000       .debug$S                   10000000     U2Lang:U2Lang.dll
 0000:fffc5000       .debug$S                   10000000     U2Lang:U2Lang.dll
 0002:fffdf000       ?_Generic_object$initializer$@?$_Error_objects@H@std@@2P6AXXZA 10000000     moc_DiamondClassifyPrompter.obj
 0002:fffdf000       ?_Iostream_object$initializer$@?$_Error_objects@H@std@@2P6AXXZA 10000000     moc_DiamondClassifyPrompter.obj
 0002:fffdf000       ?_System_object$initializer$@?$_Error_objects@H@std@@2P6AXXZA 10000000     moc_DiamondClassifyPrompter.obj
 0000:fffc5000       .debug$S                   10000000     U2Lang:U2Lang.dll
 0000:fffc5000       .debug$S                   10000000     U2Lang:U2Lang.dll
 0002:fffdf000       __unwindtable$?node_construct@?$QList@VQString@@@@AAEXPAUNode@1@ABVQString@@@Z 10000000     DiamondClassifyTask.obj
 0000:fffc5000       .debug$S                   10000000     U2Lang:U2Lang.dll
 0000:fffc5000       .debug$S                   10000000     U2Core:U2Core.dll
 0000:fffc5000       .debug$S                   10000000     U2Lang:U2Lang.dll
 0002:fffdf000       __catchsym$?node_copy@?$QList@VQString@@@@AAEXPAUNode@1@00@Z$6 10000000     DiamondClassifyTask.obj
 0000:fffc5000       .debug$S                   10000000     U2Lang:U2Lang.dll
 0002:fffdf000       ?_System_object$initializer$@?$_Error_objects@H@std@@2P6AXXZA 10000000     DiamondSupport.obj
 0000:fffc5000       .debug$S                   10000000     U2Lang:U2Lang.dll
 0002:fffdf000       ?_Iostream_object$initializer$@?$_Error_objects@H@std@@2P6AXXZA 10000000     DiamondSupport.obj
 0000:fffc5000       .debug$S                   10000000     U2Lang:U2Lang.dll
 0002:fffdf000       ?_Generic_object$initializer$@?$_Error_objects@H@std@@2P6AXXZA 10000000     DiamondSupport.obj
 0000:fffc5000       .debug$S                   10000000     U2Lang:U2Lang.dll
 0002:fffdf000       __catchsym$?node_copy@?$QList@VQString@@@@AAEXPAUNode@1@00@Z$6 10000000     DiamondSupport.obj
 0000:fffc5000       .debug$S                   10000000     U2Lang:U2Lang.dll
 0000:fffc5000       .debug$S                   10000000     U2Core:U2Core.dll
 0000:fffc5000       .debug$S                   10000000     U2Lang:U2Lang.dll
 0002:fffdf000       __unwindtable$?node_construct@?$QList@VQString@@@@AAEXPAUNode@1@ABVQString@@@Z 10000000     DiamondSupport.obj
 0000:fffc5000       .debug$S                   10000000     U2Lang:U2Lang.dll
 0000:fffc5000       .debug$S                   10000000     U2Core:U2Core.dll
 0002:fffdf000       __catchsym$?detach_helper_grow@?$QList@VQString@@@@AAEPAUNode@1@HH@Z$5 10000000     DiamondSupport.obj
 0000:fffc5000       .debug$S                   10000000     U2Lang:U2Lang.dll
 0000:fffc5000       .debug$S                   10000000     U2Core:U2Core.dll
 0000:fffc5000       .debug$S                   10000000     U2Lang:U2Lang.dll
 0002:fffdf000       __catchsym$?append@?$QList@VQString@@@@QAEXABVQString@@@Z$13 10000000     DiamondSupport.obj
 0000:fffc5000       .debug$S                   10000000     U2Lang:U2Lang.dll
 0001:fffff000       __ehhandler$?_Copy@?$basic_string@DU?$char_traits@D@std@@V?$allocator@D@2@@std@@QAEXII@Z 10000000 f   moc_DiamondBuildWorker.obj
 0000:fffc5000       .debug$S                   10000000     U2Core:U2Core.dll
 0002:fffdf000       __catchsym$?_Copy@?$basic_string@DU?$char_traits@D@std@@V?$allocator@D@2@@std@@QAEXII@Z$5 10000000     DiamondSupport.obj
 0000:fffc5000       .debug$S                   10000000     U2Core:U2Core.dll
 0002:fffdf000       __catchsym$??0?$QList@VQString@@@@QAE@ABV0@@Z$2 10000000     DiamondBuildWorker.obj
 0002:fffdf000       ?_System_object$initializer$@?$_Error_objects@H@std@@2P6AXXZA 10000000     moc_DiamondBuildPrompter.obj
 0002:fffdf000       __catchsym$?_Copy@?$basic_string@DU?$char_traits@D@std@@V?$allocator@D@2@@std@@QAEXII@Z$5 10000000     DiamondBuildWorker.obj
 0002:fffdf000       ?_Iostream_object$initializer$@?$_Error_objects@H@std@@2P6AXXZA 10000000     moc_DiamondBuildPrompter.obj
 0001:fffff000       __unwindfunclet$??1DiamondBuildTaskSettings@U2@@QAE@XZ$0 10000000 f   DiamondBuildWorker.obj
 0002:fffdf000       ?_Generic_object$initializer$@?$_Error_objects@H@std@@2P6AXXZA 10000000     moc_DiamondBuildPrompter.obj
 0001:fffff000       __unwindfunclet$?node_copy@?$QList@VQString@@@@AAEXPAUNode@1@00@Z$5 10000000 f   DiamondSupport.obj
 0002:fffdf000       __unwindtable$??0QStringList@@QAE@ABVQString@@@Z 10000000     DiamondBuildWorkerFactory.obj
 0000:fffc5000       .debug$S                   10000000     U2Core:U2Core.dll
 0002:fffdf000       __catchsym$?node_copy@?$QList@VQString@@@@AAEXPAUNode@1@00@Z$6 10000000     DiamondBuildWorkerFactory.obj
 0000:fffc5000       .debug$S                   10000000     U2Core:U2Core.dll
 0001:fffff000       __unwindfunclet$?node_construct@?$QList@VQString@@@@AAEXPAUNode@1@ABVQString@@@Z$1 10000000 f   DiamondSupport.obj
 0001:fffff000       __ehhandler$?detach_helper_grow@?$QList@VQString@@@@AAEPAUNode@1@HH@Z 10000000 f   DiamondSupport.obj
 0002:fffdf000       __unwindtable$?node_construct@?$QList@VQString@@@@AAEXPAUNode@1@ABVQString@@@Z 10000000     DiamondBuildWorkerFactory.obj
 0000:fffc5000       .debug$S                   10000000     U2Core:U2Core.dll
 0002:fffdf000       __catchsym$?detach_helper_grow@?$QList@VQString@@@@AAEPAUNode@1@HH@Z$5 10000000     DiamondBuildWorkerFactory.obj
 0000:fffc5000       .debug$S                   10000000     U2Core:U2Core.dll
 0001:fffff000       __unwindfunclet$?append@?$QList@VQString@@@@QAEXABVQString@@@Z$7 10000000 f   DiamondSupport.obj
 0001:fffff000       __ehhandler$?_Copy@?$basic_string@DU?$char_traits@D@std@@V?$allocator@D@2@@std@@QAEXII@Z 10000000 f   DiamondSupport.obj
 0002:fffdf000       ?_System_object$initializer$@?$_Error_objects@H@std@@2P6AXXZA 10000000     DiamondSupportPlugin.obj
 0002:fffdf000       ?_Iostream_object$initializer$@?$_Error_objects@H@std@@2P6AXXZA 10000000     DiamondSupportPlugin.obj
 0002:fffdf000       ?_Generic_object$initializer$@?$_Error_objects@H@std@@2P6AXXZA 10000000     DiamondSupportPlugin.obj
 0000:fffc5000       .debug$S                   10000000     U2Core:U2Core.dll
 0002:fffdf000       __catchsym$?_Copy@?$basic_string@DU?$char_traits@D@std@@V?$allocator@D@2@@std@@QAEXII@Z$5 10000000     moc_DiamondBuildWorker.obj
 0000:fffc5000       .debug$S                   10000000     U2Lang:U2Lang.dll
 0000:fffc5000       .debug$S                   10000000     U2Lang:U2Lang.dll
 0000:fffc5000       .debug$S                   10000000     U2Lang:U2Lang.dll
 0000:fffc5000       .debug$S                   10000000     U2Lang:U2Lang.dll
 0000:fffc5000       .debug$S                   10000000     U2Lang:U2Lang.dll
 0000:fffc5000       .debug$S                   10000000     U2Lang:U2Lang.dll
 0000:fffc5000       .debug$S                   10000000     U2Lang:U2Lang.dll
 0000:fffc5000       .debug$S                   10000000     U2Lang:U2Lang.dll
 0000:fffc5000       .debug$S                   10000000     U2Lang:U2Lang.dll
 0000:fffc5000       .debug$S                   10000000     U2Lang:U2Lang.dll
 0000:fffc5000       .debug$S                   10000000     U2Lang:U2Lang.dll
 0000:fffc5000       .debug$S                   10000000     U2Lang:U2Lang.dll
 0000:fffc5000       .debug$S                   10000000     U2Lang:U2Lang.dll
 0000:fffc5000       .debug$S                   10000000     U2Lang:U2Lang.dll
 0000:fffc5000       .debug$S                   10000000     U2Lang:U2Lang.dll
 0000:fffc5000       .debug$S                   10000000     U2Lang:U2Lang.dll
 0000:fffc5000       .debug$S                   10000000     U2Lang:U2Lang.dll
 0000:fffc5000       .debug$S                   10000000     U2Lang:U2Lang.dll
 0000:fffc5000       .debug$S                   10000000     U2Lang:U2Lang.dll
 0000:fffc5000       .debug$S                   10000000     U2Lang:U2Lang.dll
 0000:fffc5000       .debug$S                   10000000     U2Lang:U2Lang.dll
 0000:fffc5000       .debug$S                   10000000     U2Lang:U2Lang.dll
 0000:fffc5000       .debug$S                   10000000     U2Lang:U2Lang.dll
 0000:fffc5000       .debug$S                   10000000     U2Lang:U2Lang.dll
 0000:fffc5000       .debug$S                   10000000     U2Lang:U2Lang.dll
 0000:fffc5000       .debug$S                   10000000     U2Lang:U2Lang.dll
 0000:fffc5000       .debug$S                   10000000     U2Lang:U2Lang.dll
 0000:fffc5000       .debug$S                   10000000     U2Lang:U2Lang.dll
 0000:fffc5000       .debug$S                   10000000     U2Lang:U2Lang.dll
 0000:fffc5000       .debug$S                   10000000     U2Lang:U2Lang.dll
 0000:fffc5000       .debug$S                   10000000     U2Lang:U2Lang.dll
 0000:fffc5000       .debug$S                   10000000     U2Lang:U2Lang.dll
 0000:fffc5000       .debug$S                   10000000     U2Lang:U2Lang.dll
 0000:fffc5000       .debug$S                   10000000     U2Lang:U2Lang.dll
 0000:fffc5000       .debug$S                   10000000     U2Lang:U2Lang.dll
 0000:fffc5000       .debug$S                   10000000     U2Lang:U2Lang.dll
 0000:fffc5000       .debug$S                   10000000     U2Lang:U2Lang.dll
 0000:fffc5000       .debug$S                   10000000     U2Lang:U2Lang.dll
 0000:fffc5000       .debug$S                   10000000     U2Lang:U2Lang.dll
 0000:fffc5000       .debug$S                   10000000     U2Lang:U2Lang.dll
 0000:fffc5000       .debug$S                   10000000     U2Lang:U2Lang.dll
 0000:fffc5000       .debug$S                   10000000     U2Lang:U2Lang.dll
 0000:fffc5000       .debug$S                   10000000     U2Lang:U2Lang.dll
 0002:fffdf000       ?_Generic_object$initializer$@?$_Error_objects@H@std@@2P6AXXZA 10000000     moc_DiamondBuildWorker.obj
 0002:fffdf000       ?_Iostream_object$initializer$@?$_Error_objects@H@std@@2P6AXXZA 10000000     moc_DiamondBuildWorker.obj
 0002:fffdf000       ?_System_object$initializer$@?$_Error_objects@H@std@@2P6AXXZA 10000000     moc_DiamondBuildWorker.obj
 0000:fffc5000       .debug$S                   10000000     U2Lang:U2Lang.dll
 0000:fffc5000       .debug$S                   10000000     U2Lang:U2Lang.dll
 0000:fffc5000       .debug$S                   10000000     ngs_reads_classification:ngs_reads_classification.dll
 0000:fffc5000       .debug$S                   10000000     U2Lang:U2Lang.dll
 0000:fffc5000       .debug$S                   10000000     ngs_reads_classification:ngs_reads_classification.dll
 0000:fffc5000       .debug$S                   10000000     U2Lang:U2Lang.dll
 0000:fffc5000       .debug$S                   10000000     ngs_reads_classification:ngs_reads_classification.dll
 0000:fffc5000       .debug$S                   10000000     U2Lang:U2Lang.dll
 0000:fffc5000       .debug$S                   10000000     ngs_reads_classification:ngs_reads_classification.dll
 0000:fffc5000       .debug$S                   10000000     U2Lang:U2Lang.dll
 0000:fffc5000       .debug$S                   10000000     ngs_reads_classification:ngs_reads_classification.dll
 0000:fffc5000       .debug$S                   10000000     U2Lang:U2Lang.dll
 0000:fffc5000       .debug$S                   10000000     ngs_reads_classification:ngs_reads_classification.dll
 0000:fffc5000       .debug$S                   10000000     U2Lang:U2Lang.dll
 0000:fffc5000       .debug$S                   10000000     ngs_reads_classification:ngs_reads_classification.dll
 0000:fffc5000       .debug$S                   10000000     U2Lang:U2Lang.dll
 0000:fffc5000       .debug$S                   10000000     ngs_reads_classification:ngs_reads_classification.dll
 0000:fffc5000       .debug$S                   10000000     U2Lang:U2Lang.dll
 0000:fffc5000       .debug$S                   10000000     ngs_reads_classification:ngs_reads_classification.dll
 0000:fffc5000       .debug$S                   10000000     U2Lang:U2Lang.dll
 0000:fffc5000       .debug$S                   10000000     ngs_reads_classification:ngs_reads_classification.dll
 0000:fffc5000       .debug$S                   10000000     ngs_reads_classification:ngs_reads_classification.dll
 0000:fffc5000       .debug$S                   10000000     U2Lang:U2Lang.dll
 0000:fffc5000       .debug$S                   10000000     ngs_reads_classification:ngs_reads_classification.dll
 0000:fffc5000       .debug$S                   10000000     U2Lang:U2Lang.dll
 0000:fffc5000       .debug$S                   10000000     ngs_reads_classification:ngs_reads_classification.dll
 0000:fffc5000       .debug$S                   10000000     U2Lang:U2Lang.dll
 0001:fffff000       __ehhandler$?_Copy@?$basic_string@DU?$char_traits@D@std@@V?$allocator@D@2@@std@@QAEXII@Z 10000000 f   moc_DiamondBuildTask.obj
 0000:fffc5000       .debug$S                   10000000     ngs_reads_classification:ngs_reads_classification.dll
 0000:fffc5000       .debug$S                   10000000     ngs_reads_classification:ngs_reads_classification.dll
 0000:fffc5000       .debug$S                   10000000     ngs_reads_classification:ngs_reads_classification.dll
 0002:fffdf000       __catchsym$?append@?$QList@VQString@@@@QAEXABVQString@@@Z$13 10000000     DiamondBuildWorkerFactory.obj
 0000:fffc5000       .debug$S                   10000000     U2Core:U2Core.dll
 0000:fffc5000       .debug$S                   10000000     ngs_reads_classification:ngs_reads_classification.dll
 0000:fffc5000       .debug$S                   10000000     ngs_reads_classification:ngs_reads_classification.dll
 0000:fffc5000       .debug$S                   10000000     ngs_reads_classification:ngs_reads_classification.dll
 0002:fffdf000       __unwindtable$??H@YA?BVQString@@ABV0@PBD@Z 10000000     DiamondBuildWorkerFactory.obj
 0000:fffc5000       .debug$S                   10000000     U2Core:U2Core.dll
 0002:fffdf000       __catchsym$?_Copy@?$basic_string@DU?$char_traits@D@std@@V?$allocator@D@2@@std@@QAEXII@Z$5 10000000     DiamondBuildWorkerFactory.obj
 0000:fffc5000       .debug$S                   10000000     U2Core:U2Core.dll
 0000:fffc5000       .debug$S                   10000000     ngs_reads_classification:ngs_reads_classification.dll
 0000:fffc5000       .debug$S                   10000000     ngs_reads_classification:ngs_reads_classification.dll
 0000:fffc5000       .debug$S                   10000000     ngs_reads_classification:ngs_reads_classification.dll
 0000:fffc5000       .debug$S                   10000000     ngs_reads_classification:ngs_reads_classification.dll
 0000:fffc5000       .debug$S                   10000000     ngs_reads_classification:ngs_reads_classification.dll
 0000:fffc5000       .debug$S                   10000000     ngs_reads_classification:ngs_reads_classification.dll
 0000:fffc5000       .debug$S                   10000000     ngs_reads_classification:ngs_reads_classification.dll
 0000:fffc5000       .debug$S                   10000000     ngs_reads_classification:ngs_reads_classification.dll
 0000:fffc5000       .debug$S                   10000000     ngs_reads_classification:ngs_reads_classification.dll
 0002:fffdf000       __catchsym$?_Copy@?$basic_string@DU?$char_traits@D@std@@V?$allocator@D@2@@std@@QAEXII@Z$5 10000000     DiamondSupportPlugin.obj
 0000:fffc5000       .debug$S                   10000000     U2Core:U2Core.dll
 0000:fffc5000       .debug$S                   10000000     U2Core:U2Core.dll
 0002:fffdf000       __catchsym$?_Copy@?$basic_string@DU?$char_traits@D@std@@V?$allocator@D@2@@std@@QAEXII@Z$5 10000000     moc_DiamondBuildTask.obj
 0000:fffc5000       .debug$S                   10000000     U2Lang:U2Lang.dll
 0000:fffc5000       .debug$S                   10000000     U2Lang:U2Lang.dll
 0000:fffc5000       .debug$S                   10000000     U2Lang:U2Lang.dll
 0000:fffc5000       .debug$S                   10000000     U2Lang:U2Lang.dll
 0000:fffc5000       .debug$S                   10000000     U2Lang:U2Lang.dll
 0000:fffc5000       .debug$S                   10000000     U2Lang:U2Lang.dll
 0000:fffc5000       .debug$S                   10000000     U2Lang:U2Lang.dll
 0000:fffc5000       .debug$S                   10000000     U2Lang:U2Lang.dll
 0000:fffc5000       .debug$S                   10000000     U2Lang:U2Lang.dll
 0000:fffc5000       .debug$S                   10000000     U2Lang:U2Lang.dll
 0000:fffc5000       .debug$S                   10000000     U2Lang:U2Lang.dll
 0000:fffc5000       .debug$S                   10000000     U2Lang:U2Lang.dll
 0000:fffc5000       .debug$S                   10000000     U2Lang:U2Lang.dll
 0000:fffc5000       .debug$S                   10000000     U2Lang:U2Lang.dll
 0000:fffc5000       .debug$S                   10000000     U2Lang:U2Lang.dll
 0000:fffc5000       .debug$S                   10000000     U2Lang:U2Lang.dll
 0000:fffc5000       .debug$S                   10000000     U2Lang:U2Lang.dll
 0000:fffc5000       .debug$S                   10000000     U2Lang:U2Lang.dll
 0000:fffc5000       .debug$S                   10000000     U2Lang:U2Lang.dll
 0000:fffc5000       .debug$S                   10000000     U2Lang:U2Lang.dll
 0000:fffc5000       .debug$S                   10000000     U2Lang:U2Lang.dll
 0000:fffc5000       .debug$S                   10000000     U2Lang:U2Lang.dll
 0000:fffc5000       .debug$S                   10000000     U2Lang:U2Lang.dll
 0000:fffc5000       .debug$S                   10000000     U2Lang:U2Lang.dll
 0000:fffc5000       .debug$S                   10000000     U2Lang:U2Lang.dll
 0000:fffc5000       .debug$S                   10000000     U2Lang:U2Lang.dll
 0000:fffc5000       .debug$S                   10000000     U2Lang:U2Lang.dll
 0000:fffc5000       .debug$S                   10000000     U2Lang:U2Lang.dll
 0000:fffc5000       .debug$S                   10000000     U2Lang:U2Lang.dll
 0000:fffc5000       .debug$S                   10000000     U2Lang:U2Lang.dll
 0000:fffc5000       .debug$S                   10000000     U2Lang:U2Lang.dll
 0000:fffc5000       .debug$S                   10000000     U2Lang:U2Lang.dll
 0000:fffc5000       .debug$S                   10000000     U2Lang:U2Lang.dll
 0000:fffc5000       .debug$S                   10000000     U2Lang:U2Lang.dll
 0000:fffc5000       .debug$S                   10000000     U2Lang:U2Lang.dll
 0000:fffc5000       .debug$S                   10000000     U2Lang:U2Lang.dll
 0000:fffc5000       .debug$S                   10000000     U2Lang:U2Lang.dll
 0000:fffc5000       .debug$S                   10000000     U2Lang:U2Lang.dll
 0000:fffc5000       .debug$S                   10000000     U2Gui:U2Gui.dll
 0000:fffc5000       .debug$S                   10000000     U2Gui:U2Gui.dll
 0000:fffc5000       .debug$S                   10000000     U2Formats:U2Formats.dll
 0002:fffdf000       ?_Generic_object$initializer$@?$_Error_objects@H@std@@2P6AXXZA 10000000     moc_DiamondBuildTask.obj
 0002:fffdf000       ?_Iostream_object$initializer$@?$_Error_objects@H@std@@2P6AXXZA 10000000     moc_DiamondBuildTask.obj
 0002:fffdf000       ?_System_object$initializer$@?$_Error_objects@H@std@@2P6AXXZA 10000000     moc_DiamondBuildTask.obj
 0000:fffc5000       .debug$S                   10000000     U2Formats:U2Formats.dll
 0000:fffc5000       .debug$S                   10000000     U2Formats:U2Formats.dll
 0002:fffdf000       ?_Generic_object$initializer$@?$_Error_objects@H@std@@2P6AXXZA 10000000     DiamondClassifyTask.obj
 0000:fffc5000       .debug$S                   10000000     U2Formats:U2Formats.dll
 0002:fffdf000       ?_Iostream_object$initializer$@?$_Error_objects@H@std@@2P6AXXZA 10000000     DiamondClassifyTask.obj
 0000:fffc5000       .debug$S                   10000000     U2Formats:U2Formats.dll
 0002:fffdf000       ?_System_object$initializer$@?$_Error_objects@H@std@@2P6AXXZA 10000000     DiamondClassifyTask.obj
 0000:fffc5000       .debug$S                   10000000     U2Formats:U2Formats.dll
 0001:fffff000       __ehhandler$?_Copy@?$basic_string@DU?$char_traits@D@std@@V?$allocator@D@2@@std@@QAEXII@Z 10000000 f   DiamondClassifyPrompter.obj
 0000:fffc5000       .debug$S                   10000000     U2Formats:U2Formats.dll
 0001:fffff000       __ehhandler$??0?$QList@PAVPort@Workflow@U2@@@@QAE@ABV0@@Z 10000000 f   DiamondClassifyPrompter.obj
 0000:fffc5000       .debug$S                   10000000     U2Formats:U2Formats.dll
 0001:fffff000       __ehhandler$?_Copy@?$basic_string@DU?$char_traits@D@std@@V?$allocator@D@2@@std@@QAEXII@Z 10000000 f   DiamondSupportPlugin.obj
 0000:fffc5000       .debug$S                   10000000     U2Formats:U2Formats.dll
 0000:fffc5000       .debug$S                   10000000     U2Core:U2Core.dll
 0000:fffc5000       .debug$S                   10000000     U2Formats:U2Formats.dll
 0000:fffc5000       .debug$S                   10000000     U2Core:U2Core.dll
 0000:fffc5000       .debug$S                   10000000     U2Formats:U2Formats.dll
 0000:fffc5000       .debug$S                   10000000     U2Core:U2Core.dll
 0000:fffc5000       .debug$S                   10000000     U2Core:U2Core.dll
 0000:fffc5000       .debug$S                   10000000     U2Core:U2Core.dll
 0000:fffc5000       .debug$S                   10000000     U2Core:U2Core.dll
 0000:fffc5000       .debug$S                   10000000     U2Core:U2Core.dll
 0000:fffc5000       .debug$S                   10000000     U2Core:U2Core.dll
 0000:fffc5000       .debug$S                   10000000     U2Core:U2Core.dll
 0000:fffc5000       .debug$S                   10000000     U2Core:U2Core.dll
 0000:fffc5000       .debug$S                   10000000     U2Core:U2Core.dll
 0001:fffff000       __ehhandler$?_Copy@?$basic_string@DU?$char_traits@D@std@@V?$allocator@D@2@@std@@QAEXII@Z 10000000 f   moc_DiamondBuildPrompter.obj
 0000:fffc5000       .debug$S                   10000000     U2Core:U2Core.dll
 0000:fffc5000       .debug$S                   10000000     U2Core:U2Core.dll
 0000:fffc5000       .debug$S                   10000000     U2Core:U2Core.dll
 0000:fffc5000       .debug$S                   10000000     U2Core:U2Core.dll
 0000:fffc5000       .debug$S                   10000000     U2Core:U2Core.dll
 0001:fffff000       __unwindfunclet$??0QStringList@@QAE@ABVQString@@@Z$0 10000000 f   DiamondBuildWorkerFactory.obj
 0000:fffc5000       .debug$S                   10000000     U2Core:U2Core.dll
 0001:fffff000       __unwindfunclet$?node_copy@?$QList@VQString@@@@AAEXPAUNode@1@00@Z$5 10000000 f   DiamondBuildWorkerFactory.obj
 0000:fffc5000       .debug$S                   10000000     U2Core:U2Core.dll
 0000:fffc5000       .debug$S                   10000000     U2Core:U2Core.dll
 0001:fffff000       __unwindfunclet$?node_construct@?$QList@VQString@@@@AAEXPAUNode@1@ABVQString@@@Z$1 10000000 f   DiamondBuildWorkerFactory.obj
 0002:fffdf000       ?_System_object$initializer$@?$_Error_objects@H@std@@2P6AXXZA 10000000     GenomesPreparationTask.obj
 0002:fffdf000       ?_Iostream_object$initializer$@?$_Error_objects@H@std@@2P6AXXZA 10000000     GenomesPreparationTask.obj
 0002:fffdf000       ?_Generic_object$initializer$@?$_Error_objects@H@std@@2P6AXXZA 10000000     GenomesPreparationTask.obj
 0001:fffff000       __ehhandler$?detach_helper_grow@?$QList@VQString@@@@AAEPAUNode@1@HH@Z 10000000 f   DiamondBuildWorkerFactory.obj
 0000:fffc5000       .debug$S                   10000000     U2Core:U2Core.dll
 0001:fffff000       __unwindfunclet$?append@?$QList@VQString@@@@QAEXABVQString@@@Z$7 10000000 f   DiamondBuildWorkerFactory.obj
 0000:fffc5000       .debug$S                   10000000     U2Core:U2Core.dll
 0000:fffc5000       .debug$S                   10000000     U2Core:U2Core.dll
 0000:fffc5000       .debug$S                   10000000     U2Core:U2Core.dll
 0000:fffc5000       .debug$S                   10000000     U2Core:U2Core.dll
 0000:fffc5000       .debug$S                   10000000     U2Core:U2Core.dll
 0000:fffc5000       .debug$S                   10000000     U2Core:U2Core.dll
 0000:fffc5000       .debug$S                   10000000     U2Core:U2Core.dll
 0002:fffdf000       __catchsym$?_Copy@?$basic_string@DU?$char_traits@D@std@@V?$allocator@D@2@@std@@QAEXII@Z$5 10000000     moc_DiamondBuildPrompter.obj
 0000:fffc5000       .debug$S                   10000000     U2Core:U2Core.dll
 0000:fffc5000       .debug$S                   10000000     U2Core:U2Core.dll
 0000:fffc5000       .debug$S                   10000000     U2Core:U2Core.dll
 0000:fffc5000       .debug$S                   10000000     U2Core:U2Core.dll
 0000:fffc5000       .debug$S                   10000000     U2Core:U2Core.dll
 0000:fffc5000       .debug$S                   10000000     U2Core:U2Core.dll
 0000:fffc5000       .debug$S                   10000000     U2Core:U2Core.dll
 0000:fffc5000       .debug$S                   10000000     U2Core:U2Core.dll
 0000:fffc5000       .debug$S                   10000000     U2Core:U2Core.dll
 0000:fffc5000       .debug$S                   10000000     U2Core:U2Core.dll
 0000:fffc5000       .debug$S                   10000000     U2Core:U2Core.dll
 0000:fffc5000       .debug$S                   10000000     U2Core:U2Core.dll
 0000:fffc5000       .debug$S                   10000000     U2Core:U2Core.dll
 0000:fffc5000       .debug$S                   10000000     U2Core:U2Core.dll
 0000:fffc5000       .debug$S                   10000000     U2Core:U2Core.dll
 0000:fffc5000       .debug$S                   10000000     U2Core:U2Core.dll
 0000:fffc5000       .debug$S                   10000000     U2Core:U2Core.dll
 0000:fffc5000       .debug$S                   10000000     U2Core:U2Core.dll
 0000:fffc5000       .debug$S                   10000000     U2Core:U2Core.dll
 0000:fffc5000       .debug$S                   10000000     U2Core:U2Core.dll
 0000:fffc5000       .debug$S                   10000000     U2Core:U2Core.dll
 0000:fffc5000       .debug$S                   10000000     U2Core:U2Core.dll
 0000:fffc5000       .debug$S                   10000000     U2Core:U2Core.dll
 0000:fffc5000       .debug$S                   10000000     U2Core:U2Core.dll
 0000:fffc5000       .debug$S                   10000000     U2Core:U2Core.dll
 0000:fffc5000       .debug$S                   10000000     U2Core:U2Core.dll
 0000:fffc5000       .debug$S                   10000000     U2Core:U2Core.dll
 0000:fffc5000       .debug$S                   10000000     U2Core:U2Core.dll
 0000:fffc5000       .debug$S                   10000000     U2Core:U2Core.dll
 0002:fffdf000       __catchsym$?_Copy@?$basic_string@DU?$char_traits@D@std@@V?$allocator@D@2@@std@@QAEXII@Z$5 10000000     GenomesPreparationTask.obj
 0001:fffff008       __ehhandler$??0QStringList@@QAE@ABVQString@@@Z 10000008 f   DiamondBuildWorkerFactory.obj
 0002:fffdf008       __ehfuncinfo$??A?$QMap@VDescriptor@U2@@V?$QExplicitlySharedDataPointer@VDataType@U2@@@@@@QAEAAV?$QExplicitlySharedDataPointer@VDataType@U2@@@@ABVDescriptor@U2@@@Z 10000008     DiamondClassifyWorkerFactory.obj
 0002:fffdf008       __ehfuncinfo$??A?$QMap@VQString@@VQVariant@@@@QAEAAVQVariant@@ABVQString@@@Z 10000008     DiamondClassifyWorkerFactory.obj
 0002:fffdf008       __ehfuncinfo$?uniqueKeys@?$QMap@VDescriptor@U2@@VQVariant@@@@QBE?AV?$QList@VDescriptor@U2@@@@XZ 10000008     DiamondClassifyWorker.obj
 0002:fffdf008       __ehfuncinfo$??A?$QMap@VQString@@VQScriptValue@@@@QAEAAVQScriptValue@@ABVQString@@@Z 10000008     DiamondClassifyWorker.obj
 0002:fffdf008       __ehfuncinfo$?qt_metatype_id@?$QMetaTypeIdQObject@PAVTask@U2@@$00@@SAHXZ 10000008     moc_DiamondClassifyWorker.obj
 0002:fffdf008       __ehfuncinfo$??0QStringList@@QAE@ABVQString@@@Z 10000008     DiamondBuildWorkerFactory.obj
 0002:fffdf008       __ehfuncinfo$??H@YA?BVQString@@ABV0@0@Z 10000008     DiamondClassifyWorker.obj
 0001:fffff008       __ehhandler$??A?$QMap@VDescriptor@U2@@V?$QExplicitlySharedDataPointer@VDataType@U2@@@@@@QAEAAV?$QExplicitlySharedDataPointer@VDataType@U2@@@@ABVDescriptor@U2@@@Z 10000008 f   DiamondClassifyWorkerFactory.obj
 0002:fffdf008       __ehfuncinfo$??A?$QMap@VQString@@VQVariant@@@@QAEAAVQVariant@@ABVQString@@@Z 10000008     DiamondClassifyWorker.obj
 0001:fffff009       __unwindfunclet$??1DiamondBuildTaskSettings@U2@@QAE@XZ$1 10000009 f   DiamondBuildWorker.obj
 0001:fffff009       __unwindfunclet$??1DiamondClassifyTaskSettings@U2@@QAE@XZ$1 10000009 f   DiamondClassifyWorker.obj
 0001:fffff009       __ehhandler$??A?$QMap@VQString@@VQScriptValue@@@@QAEAAVQScriptValue@@ABVQString@@@Z 10000009 f   DiamondClassifyWorker.obj
 0001:fffff009       __ehhandler$??A?$QMap@VQString@@VQVariant@@@@QAEAAVQVariant@@ABVQString@@@Z 10000009 f   DiamondClassifyWorker.obj
 0001:fffff009       __unwindfunclet$??0DiamondBuildTaskSettings@U2@@QAE@ABU01@@Z$1 10000009 f   DiamondBuildWorker.obj
 0001:fffff009       __ehhandler$?qt_metatype_id@?$QMetaTypeIdQObject@PAVTask@U2@@$00@@SAHXZ 10000009 f   moc_DiamondClassifyWorker.obj
 0001:fffff009       __unwindfunclet$??0DiamondClassifyTaskSettings@U2@@QAE@ABU01@@Z$1 10000009 f   DiamondClassifyWorker.obj
 0001:fffff009       __ehhandler$??A?$QMap@VQString@@VQVariant@@@@QAEAAVQVariant@@ABVQString@@@Z 10000009 f   DiamondClassifyWorkerFactory.obj
 0001:fffff00b       __ehhandler$?append@?$QList@VDescriptor@U2@@@@QAEXABVDescriptor@U2@@@Z 1000000b f   DiamondClassifyWorker.obj
 0001:fffff00b       __ehhandler$?node_copy@?$QList@VDescriptor@U2@@@@AAEXPAUNode@1@00@Z 1000000b f   DiamondClassifyWorker.obj
 0001:fffff00b       __ehhandler$?node_construct@?$QList@VDescriptor@U2@@@@AAEXPAUNode@1@ABVDescriptor@U2@@@Z 1000000b f   DiamondClassifyWorker.obj
 0002:fffdf010       __ehfuncinfo$?node_construct@?$QList@VQString@@@@AAEXPAUNode@1@ABVQString@@@Z 10000010     DiamondClassifyTask.obj
 0002:fffdf010       __catchsym$?detach_helper_grow@?$QList@VQString@@@@AAEPAUNode@1@HH@Z$4 10000010     DiamondClassifyTask.obj
 0002:fffdf010       __ehfuncinfo$?node_construct@?$QList@VQString@@@@AAEXPAUNode@1@ABVQString@@@Z 10000010     DiamondSupport.obj
 0002:fffdf010       __catchsym$?append@?$QList@VQString@@@@QAEXABVQString@@@Z$12 10000010     DiamondClassifyTask.obj
 0002:fffdf010       __unwindtable$??0?$QList@VQString@@@@QAE@ABV0@@Z 10000010     DiamondClassifyTask.obj
 0002:fffdf010       __catchsym$?append@?$QList@VQString@@@@QAEXABVQString@@@Z$12 10000010     DiamondBuildWorker.obj
 0002:fffdf010       __catchsym$?detach_helper_grow@?$QList@VQString@@@@AAEPAUNode@1@HH@Z$4 10000010     DiamondBuildWorker.obj
 0002:fffdf010       __catchsym$?_Copy@?$basic_string@DU?$char_traits@D@std@@V?$allocator@D@2@@std@@QAEXII@Z$4 10000010     DiamondClassifyTask.obj
 0002:fffdf010       __catchsym$?detach_helper_grow@?$QList@VQString@@@@AAEPAUNode@1@HH@Z$4 10000010     DiamondSupport.obj
 0002:fffdf010       __ehfuncinfo$?node_construct@?$QList@VQString@@@@AAEXPAUNode@1@ABVQString@@@Z 10000010     DiamondBuildWorker.obj
 0002:fffdf010       __tryblocktable$?node_copy@?$QList@VQString@@@@AAEXPAUNode@1@00@Z 10000010     DiamondBuildWorker.obj
 0002:fffdf010       __catchsym$?_Copy@?$basic_string@DU?$char_traits@D@std@@V?$allocator@D@2@@std@@QAEXII@Z$4 10000010     moc_DiamondClassifyTask.obj
 0002:fffdf010       __ehfuncinfo$?metaType@?$QVariantValueHelper@VQString@@@QtPrivate@@SA?AVQString@@ABVQVariant@@@Z 10000010     DiamondClassifyWorker.obj
 0002:fffdf010       __tryblocktable$?createNode@?$QMapData@VQString@@I@@QAEPAU?$QMapNode@VQString@@I@@ABVQString@@ABIPAU2@_N@Z 10000010     DiamondClassifyWorker.obj
 0002:fffdf010       __catchsym$?createNode@?$QMapData@VQString@@VQScriptValue@@@@QAEPAU?$QMapNode@VQString@@VQScriptValue@@@@ABVQString@@ABVQScriptValue@@PAU2@_N@Z$6 10000010     DiamondClassifyWorker.obj
 0002:fffdf010       __catchsym$?createNode@?$QMapData@VQString@@VQVariant@@@@QAEPAU?$QMapNode@VQString@@VQVariant@@@@ABVQString@@ABVQVariant@@PAU2@_N@Z$6 10000010     DiamondClassifyWorker.obj
 0002:fffdf010       __catchsym$?append@?$QList@VQString@@@@QAEXABVQString@@@Z$12 10000010     DiamondSupport.obj
 0002:fffdf010       __catchsym$?_Copy@?$basic_string@DU?$char_traits@D@std@@V?$allocator@D@2@@std@@QAEXII@Z$4 10000010     DiamondSupport.obj
 0002:fffdf010       __unwindtable$??0?$QList@VQString@@@@QAE@ABV0@@Z 10000010     DiamondBuildWorker.obj
 0002:fffdf010       __catchsym$?_Copy@?$basic_string@DU?$char_traits@D@std@@V?$allocator@D@2@@std@@QAEXII@Z$4 10000010     moc_DiamondClassifyPrompter.obj
 0002:fffdf010       __ehfuncinfo$?node_construct@?$QList@VDescriptor@U2@@@@AAEXPAUNode@1@ABVDescriptor@U2@@@Z 10000010     DiamondClassifyWorker.obj
 0002:fffdf010       __unwindtable$?detach_helper@?$QList@VDescriptor@U2@@@@AAEXH@Z 10000010     DiamondClassifyWorker.obj
 0002:fffdf010       __catchsym$?detach_helper_grow@?$QList@VDescriptor@U2@@@@AAEPAUNode@1@HH@Z$4 10000010     DiamondClassifyWorker.obj
 0002:fffdf010       __catchsym$?append@?$QList@VDescriptor@U2@@@@QAEXABVDescriptor@U2@@@Z$8 10000010     DiamondClassifyWorker.obj
 0002:fffdf010       __catchsym$?_Copy@?$basic_string@DU?$char_traits@D@std@@V?$allocator@D@2@@std@@QAEXII@Z$4 10000010     DiamondBuildWorker.obj
 0002:fffdf010       __catchsym$?_Copy@?$basic_string@DU?$char_traits@D@std@@V?$allocator@D@2@@std@@QAEXII@Z$4 10000010     moc_DiamondClassifyWorker.obj
 0002:fffdf010       __unwindtable$??0?$QList@VDescriptor@U2@@@@QAE@ABV0@@Z 10000010     DiamondClassifyWorker.obj
 0002:fffdf010       __tryblocktable$?node_copy@?$QList@VQString@@@@AAEXPAUNode@1@00@Z 10000010     DiamondBuildWorkerFactory.obj
 0002:fffdf010       __ehfuncinfo$?node_construct@?$QList@VQString@@@@AAEXPAUNode@1@ABVQString@@@Z 10000010     DiamondBuildWorkerFactory.obj
 0002:fffdf010       __tryblocktable$?node_copy@?$QList@VQString@@@@AAEXPAUNode@1@00@Z 10000010     DiamondClassifyWorker.obj
 0002:fffdf010       __ehfuncinfo$?node_construct@?$QList@VQString@@@@AAEXPAUNode@1@ABVQString@@@Z 10000010     DiamondClassifyWorker.obj
 0002:fffdf010       __catchsym$?detach_helper_grow@?$QList@VQString@@@@AAEPAUNode@1@HH@Z$4 10000010     DiamondClassifyWorker.obj
 0002:fffdf010       __catchsym$?append@?$QList@VQString@@@@QAEXABVQString@@@Z$12 10000010     DiamondClassifyWorker.obj
 0002:fffdf010       __ehfuncinfo$??H@YA?BVQString@@ABV0@PBD@Z 10000010     DiamondClassifyWorker.obj
 0002:fffdf010       __catchsym$?detach_helper_grow@?$QList@VQString@@@@AAEPAUNode@1@HH@Z$4 10000010     DiamondBuildWorkerFactory.obj
 0002:fffdf010       __catchsym$?_Copy@?$basic_string@DU?$char_traits@D@std@@V?$allocator@D@2@@std@@QAEXII@Z$4 10000010     DiamondClassifyWorker.obj
 0002:fffdf010       __catchsym$?_Copy@?$basic_string@DU?$char_traits@D@std@@V?$allocator@D@2@@std@@QAEXII@Z$4 10000010     moc_DiamondBuildWorker.obj
 0002:fffdf010       __catchsym$?append@?$QList@VQString@@@@QAEXABVQString@@@Z$12 10000010     DiamondBuildWorkerFactory.obj
 0002:fffdf010       __ehfuncinfo$??H@YA?BVQString@@ABV0@PBD@Z 10000010     DiamondBuildWorkerFactory.obj
 0002:fffdf010       __tryblocktable$?node_copy@?$QList@VQString@@@@AAEXPAUNode@1@00@Z 10000010     DiamondClassifyTask.obj
 0002:fffdf010       __catchsym$?_Copy@?$basic_string@DU?$char_traits@D@std@@V?$allocator@D@2@@std@@QAEXII@Z$4 10000010     moc_DiamondSupport.obj
 0002:fffdf010       __tryblocktable$?node_copy@?$QList@VDescriptor@U2@@@@AAEXPAUNode@1@00@Z 10000010     DiamondClassifyWorker.obj
 0002:fffdf010       __tryblocktable$?node_copy@?$QList@VQString@@@@AAEXPAUNode@1@00@Z 10000010     DiamondSupport.obj
 0002:fffdf010       __catchsym$?_Copy@?$basic_string@DU?$char_traits@D@std@@V?$allocator@D@2@@std@@QAEXII@Z$4 10000010     DiamondBuildWorkerFactory.obj
 0002:fffdf010       __catchsym$?_Copy@?$basic_string@DU?$char_traits@D@std@@V?$allocator@D@2@@std@@QAEXII@Z$4 10000010     moc_DiamondSupportPlugin.obj
 0002:fffdf010       __catchsym$?_Copy@?$basic_string@DU?$char_traits@D@std@@V?$allocator@D@2@@std@@QAEXII@Z$4 10000010     DiamondClassifyWorkerFactory.obj
 0002:fffdf010       __ehfuncinfo$??H@YA?BVQString@@ABV0@PBD@Z 10000010     DiamondClassifyWorkerFactory.obj
 0002:fffdf010       __catchsym$?_Copy@?$basic_string@DU?$char_traits@D@std@@V?$allocator@D@2@@std@@QAEXII@Z$4 10000010     DiamondSupportPlugin.obj
 0002:fffdf010       __catchsym$?_Copy@?$basic_string@DU?$char_traits@D@std@@V?$allocator@D@2@@std@@QAEXII@Z$4 10000010     moc_GenomesPreparationTask.obj
 0002:fffdf010       __catchsym$?_Copy@?$basic_string@DU?$char_traits@D@std@@V?$allocator@D@2@@std@@QAEXII@Z$4 10000010     DiamondBuildTask.obj
 0002:fffdf010       __catchsym$?_Copy@?$basic_string@DU?$char_traits@D@std@@V?$allocator@D@2@@std@@QAEXII@Z$4 10000010     moc_DiamondBuildTask.obj
 0002:fffdf010       __tryblocktable$?append@?$QList@PAVAttribute@U2@@@@QAEXABQAVAttribute@U2@@@Z 10000010     DiamondClassifyWorkerFactory.obj
 0002:fffdf010       __catchsym$?detach_helper_grow@?$QList@PAVAttribute@U2@@@@AAEPAUNode@1@HH@Z$4 10000010     DiamondClassifyWorkerFactory.obj
 0002:fffdf010       __ehfuncinfo$??$getValue@VQString@@@BaseWorker@LocalWorkflow@U2@@IBE?AVQString@@ABV3@@Z 10000010     DiamondClassifyWorker.obj
 0002:fffdf010       __tryblocktable$?append@?$QList@PAVPortDescriptor@Workflow@U2@@@@QAEXABQAVPortDescriptor@Workflow@U2@@@Z 10000010     DiamondClassifyWorkerFactory.obj
 0002:fffdf010       __catchsym$?detach_helper_grow@?$QList@PAVPortDescriptor@Workflow@U2@@@@AAEPAUNode@1@HH@Z$4 10000010     DiamondClassifyWorkerFactory.obj
 0002:fffdf010       __catchsym$?createNode@?$QMapData@VQString@@VQVariant@@@@QAEPAU?$QMapNode@VQString@@VQVariant@@@@ABVQString@@ABVQVariant@@PAU2@_N@Z$6 10000010     DiamondClassifyWorkerFactory.obj
 0002:fffdf010       __tryblocktable$?createNode@?$QMapData@VDescriptor@U2@@V?$QExplicitlySharedDataPointer@VDataType@U2@@@@@@QAEPAU?$QMapNode@VDescriptor@U2@@V?$QExplicitlySharedDataPointer@VDataType@U2@@@@@@ABVDescriptor@U2@@ABV?$QExplicitlySharedDataPointer@VDataType@U2@@@@PAU2@_N@Z 10000010     DiamondClassifyWorkerFactory.obj
 0002:fffdf010       __unwindtable$??0?$QList@PAVPort@Workflow@U2@@@@QAE@ABV0@@Z 10000010     DiamondClassifyPrompter.obj
 0002:fffdf010       __tryblocktable$?node_copy@?$QList@VQString@@@@AAEXPAUNode@1@00@Z 10000010     GenomesPreparationTask.obj
 0002:fffdf010       __tryblocktable$?createNode@?$QMapData@VQString@@PAVPropertyDelegate@U2@@@@QAEPAU?$QMapNode@VQString@@PAVPropertyDelegate@U2@@@@ABVQString@@ABQAVPropertyDelegate@U2@@PAU2@_N@Z 10000010     DiamondClassifyWorkerFactory.obj
 0002:fffdf010       __catchsym$?_Copy@?$basic_string@DU?$char_traits@D@std@@V?$allocator@D@2@@std@@QAEXII@Z$4 10000010     DiamondClassifyPrompter.obj
 0002:fffdf010       __catchsym$?_Copy@?$basic_string@DU?$char_traits@D@std@@V?$allocator@D@2@@std@@QAEXII@Z$4 10000010     DiamondBuildValidator.obj
 0002:fffdf010       __unwindtable$??0?$QList@VQString@@@@QAE@ABV0@@Z 10000010     GenomesPreparationTask.obj
 0002:fffdf010       __catchsym$?_Copy@?$basic_string@DU?$char_traits@D@std@@V?$allocator@D@2@@std@@QAEXII@Z$4 10000010     moc_DiamondBuildPrompter.obj
 0002:fffdf010       __catchsym$?_Copy@?$basic_string@DU?$char_traits@D@std@@V?$allocator@D@2@@std@@QAEXII@Z$4 10000010     GenomesPreparationTask.obj
 0001:fffff011       __ehhandler$?node_copy@?$QList@VQString@@@@AAEXPAUNode@1@00@Z 10000011 f   GenomesPreparationTask.obj
 0001:fffff011       __unwindfunclet$?append@?$QList@VQString@@@@QAEXABVQString@@@Z$11 10000011 f   DiamondBuildWorkerFactory.obj
 0001:fffff011       __ehhandler$?node_copy@?$QList@VQString@@@@AAEXPAUNode@1@00@Z 10000011 f   DiamondClassifyTask.obj
 0001:fffff011       __ehhandler$?node_construct@?$QList@VQString@@@@AAEXPAUNode@1@ABVQString@@@Z 10000011 f   DiamondClassifyTask.obj
 0001:fffff011       __ehhandler$?node_construct@?$QList@VQString@@@@AAEXPAUNode@1@ABVQString@@@Z 10000011 f   DiamondBuildWorkerFactory.obj
 0001:fffff011       __ehhandler$?node_copy@?$QList@VQString@@@@AAEXPAUNode@1@00@Z 10000011 f   DiamondClassifyWorker.obj
 0001:fffff011       __ehhandler$?node_copy@?$QList@VQString@@@@AAEXPAUNode@1@00@Z 10000011 f   DiamondBuildWorkerFactory.obj
 0001:fffff011       __ehhandler$?node_construct@?$QList@VQString@@@@AAEXPAUNode@1@ABVQString@@@Z 10000011 f   DiamondClassifyWorker.obj
 0001:fffff011       __unwindfunclet$?append@?$QList@VQString@@@@QAEXABVQString@@@Z$11 10000011 f   DiamondClassifyWorker.obj
 0001:fffff011       __unwindfunclet$?append@?$QList@VQString@@@@QAEXABVQString@@@Z$11 10000011 f   DiamondSupport.obj
 0001:fffff011       __ehhandler$?node_construct@?$QList@VQString@@@@AAEXPAUNode@1@ABVQString@@@Z 10000011 f   DiamondSupport.obj
 0001:fffff011       __ehhandler$?node_copy@?$QList@VQString@@@@AAEXPAUNode@1@00@Z 10000011 f   DiamondSupport.obj
 0001:fffff011       __ehhandler$?node_construct@?$QList@VQString@@@@AAEXPAUNode@1@ABVQString@@@Z 10000011 f   DiamondBuildWorker.obj
 0001:fffff011       __ehhandler$?node_copy@?$QList@VQString@@@@AAEXPAUNode@1@00@Z 10000011 f   DiamondBuildWorker.obj
 0001:fffff011       __unwindfunclet$?append@?$QList@VQString@@@@QAEXABVQString@@@Z$11 10000011 f   DiamondBuildWorker.obj
 0001:fffff011       __unwindfunclet$?append@?$QList@VQString@@@@QAEXABVQString@@@Z$11 10000011 f   DiamondClassifyTask.obj
 0001:fffff014       __unwindfunclet$?createNode@?$QMapData@VQString@@VQVariant@@@@QAEPAU?$QMapNode@VQString@@VQVariant@@@@ABVQString@@ABVQVariant@@PAU2@_N@Z$5 10000014 f   DiamondClassifyWorker.obj
 0001:fffff014       __unwindfunclet$?createNode@?$QMapData@VQString@@VQScriptValue@@@@QAEPAU?$QMapNode@VQString@@VQScriptValue@@@@ABVQString@@ABVQScriptValue@@PAU2@_N@Z$5 10000014 f   DiamondClassifyWorker.obj
 0001:fffff014       __ehhandler$?createNode@?$QMapData@VDescriptor@U2@@V?$QExplicitlySharedDataPointer@VDataType@U2@@@@@@QAEPAU?$QMapNode@VDescriptor@U2@@V?$QExplicitlySharedDataPointer@VDataType@U2@@@@@@ABVDescriptor@U2@@ABV?$QExplicitlySharedDataPointer@VDataType@U2@@@@PAU2@_N@Z 10000014 f   DiamondClassifyWorkerFactory.obj
 0001:fffff014       __ehhandler$?createNode@?$QMapData@VQString@@I@@QAEPAU?$QMapNode@VQString@@I@@ABVQString@@ABIPAU2@_N@Z 10000014 f   DiamondClassifyWorker.obj
 0001:fffff014       __unwindfunclet$??0DiamondBuildTaskSettings@U2@@QAE@ABU01@@Z$2 10000014 f   DiamondBuildWorker.obj
 0001:fffff014       __unwindfunclet$?createNode@?$QMapData@VQString@@VQVariant@@@@QAEPAU?$QMapNode@VQString@@VQVariant@@@@ABVQString@@ABVQVariant@@PAU2@_N@Z$5 10000014 f   DiamondClassifyWorkerFactory.obj
 0001:fffff014       __unwindfunclet$??1DiamondBuildTaskSettings@U2@@QAE@XZ$2 10000014 f   DiamondBuildWorker.obj
 0001:fffff014       __ehhandler$?createNode@?$QMapData@VQString@@PAVPropertyDelegate@U2@@@@QAEPAU?$QMapNode@VQString@@PAVPropertyDelegate@U2@@@@ABVQString@@ABQAVPropertyDelegate@U2@@PAU2@_N@Z 10000014 f   DiamondClassifyWorkerFactory.obj
 0001:fffff015       __unwindfunclet$??1DiamondClassifyTaskSettings@U2@@QAE@XZ$2 10000015 f   DiamondClassifyWorker.obj
 0001:fffff015       __unwindfunclet$??0DiamondClassifyTaskSettings@U2@@QAE@ABU01@@Z$2 10000015 f   DiamondClassifyWorker.obj
 0001:fffff019       __ehhandler$?uniqueKeys@?$QMap@VDescriptor@U2@@VQVariant@@@@QBE?AV?$QList@VDescriptor@U2@@@@XZ 10000019 f   DiamondClassifyWorker.obj
 0001:fffff01a       __unwindfunclet$?metaType@?$QVariantValueHelper@VQString@@@QtPrivate@@SA?AVQString@@ABVQVariant@@@Z$1 1000001a f   DiamondClassifyWorker.obj
 0001:fffff01a       __ehhandler$??H@YA?BVQString@@ABV0@0@Z 1000001a f   DiamondClassifyWorker.obj
 0001:fffff01a       __unwindfunclet$??H@YA?BVQString@@ABV0@PBD@Z$1 1000001a f   DiamondClassifyWorkerFactory.obj
 0001:fffff01a       __unwindfunclet$??$getAttributeValue@VQString@@@Attribute@U2@@QBE?AVQString@@PAVWorkflowContext@Workflow@1@@Z$1 1000001a f   DiamondClassifyWorker.obj
 0001:fffff01a       __unwindfunclet$??H@YA?BVQString@@ABV0@PBD@Z$1 1000001a f   DiamondClassifyWorker.obj
 0001:fffff01a       __unwindfunclet$??$getValue@VQString@@@BaseWorker@LocalWorkflow@U2@@IBE?AVQString@@ABV3@@Z$1 1000001a f   DiamondClassifyWorker.obj
 0001:fffff01a       __unwindfunclet$??H@YA?BVQString@@ABV0@PBD@Z$1 1000001a f   DiamondBuildWorkerFactory.obj
 0002:fffdf020       __unwindtable$?detach_helper_grow@?$QList@VQString@@@@AAEPAUNode@1@HH@Z 10000020     DiamondSupport.obj
 0002:fffdf020       __unwindtable$?_Copy@?$basic_string@DU?$char_traits@D@std@@V?$allocator@D@2@@std@@QAEXII@Z 10000020     moc_DiamondSupport.obj
 0002:fffdf020       __unwindtable$?_Copy@?$basic_string@DU?$char_traits@D@std@@V?$allocator@D@2@@std@@QAEXII@Z 10000020     moc_DiamondClassifyTask.obj
 0002:fffdf020       __unwindtable$?_Copy@?$basic_string@DU?$char_traits@D@std@@V?$allocator@D@2@@std@@QAEXII@Z 10000020     GenomesPreparationTask.obj
 0002:fffdf020       __unwindtable$?_Copy@?$basic_string@DU?$char_traits@D@std@@V?$allocator@D@2@@std@@QAEXII@Z 10000020     moc_DiamondBuildWorker.obj
 0002:fffdf020       __unwindtable$?_Copy@?$basic_string@DU?$char_traits@D@std@@V?$allocator@D@2@@std@@QAEXII@Z 10000020     moc_DiamondSupportPlugin.obj
 0002:fffdf020       __unwindtable$?detach_helper_grow@?$QList@VQString@@@@AAEPAUNode@1@HH@Z 10000020     DiamondClassifyTask.obj
 0002:fffdf020       __ehfuncinfo$?createNode@?$QMapData@VQString@@VQScriptValue@@@@QAEPAU?$QMapNode@VQString@@VQScriptValue@@@@ABVQString@@ABVQScriptValue@@PAU2@_N@Z 10000020     DiamondClassifyWorker.obj
 0002:fffdf020       __unwindtable$?_Copy@?$basic_string@DU?$char_traits@D@std@@V?$allocator@D@2@@std@@QAEXII@Z 10000020     DiamondClassifyPrompter.obj
 0002:fffdf020       __ehfuncinfo$?append@?$QList@VQString@@@@QAEXABVQString@@@Z 10000020     DiamondBuildWorkerFactory.obj
 0002:fffdf020       __unwindtable$?_Copy@?$basic_string@DU?$char_traits@D@std@@V?$allocator@D@2@@std@@QAEXII@Z 10000020     DiamondBuildWorkerFactory.obj
 0002:fffdf020       __ehfuncinfo$?createNode@?$QMapData@VQString@@VQVariant@@@@QAEPAU?$QMapNode@VQString@@VQVariant@@@@ABVQString@@ABVQVariant@@PAU2@_N@Z 10000020     DiamondClassifyWorker.obj
 0002:fffdf020       __unwindtable$?_Copy@?$basic_string@DU?$char_traits@D@std@@V?$allocator@D@2@@std@@QAEXII@Z 10000020     moc_DiamondClassifyPrompter.obj
 0002:fffdf020       __tryblocktable$??0?$QList@VQString@@@@QAE@ABV0@@Z 10000020     GenomesPreparationTask.obj
 0002:fffdf020       __unwindtable$?detach_helper_grow@?$QList@VQString@@@@AAEPAUNode@1@HH@Z 10000020     DiamondBuildWorkerFactory.obj
 0002:fffdf020       __unwindtable$?_Copy@?$basic_string@DU?$char_traits@D@std@@V?$allocator@D@2@@std@@QAEXII@Z 10000020     moc_DiamondBuildTask.obj
 0002:fffdf020       __unwindtable$?_Copy@?$basic_string@DU?$char_traits@D@std@@V?$allocator@D@2@@std@@QAEXII@Z 10000020     DiamondSupportPlugin.obj
 0002:fffdf020       __unwindtable$?_Copy@?$basic_string@DU?$char_traits@D@std@@V?$allocator@D@2@@std@@QAEXII@Z 10000020     DiamondBuildWorker.obj
 0002:fffdf020       __tryblocktable$?detach_helper@?$QList@VDescriptor@U2@@@@AAEXH@Z 10000020     DiamondClassifyWorker.obj
 0002:fffdf020       __unwindtable$?_Copy@?$basic_string@DU?$char_traits@D@std@@V?$allocator@D@2@@std@@QAEXII@Z 10000020     DiamondClassifyTask.obj
 0002:fffdf020       __tryblocktable$??0?$QList@PAVPort@Workflow@U2@@@@QAE@ABV0@@Z 10000020     DiamondClassifyPrompter.obj
 0002:fffdf020       __unwindtable$?_Copy@?$basic_string@DU?$char_traits@D@std@@V?$allocator@D@2@@std@@QAEXII@Z 10000020     moc_DiamondBuildPrompter.obj
 0001:fffff020       __unwindfunclet$??0DiamondBuildTaskSettings@U2@@QAE@ABU01@@Z$3 10000020 f   DiamondBuildWorker.obj
 0001:fffff020       __unwindfunclet$??1DiamondBuildTaskSettings@U2@@QAE@XZ$3 10000020 f   DiamondBuildWorker.obj
 0002:fffdf020       __unwindtable$?detach_helper_grow@?$QList@VDescriptor@U2@@@@AAEPAUNode@1@HH@Z 10000020     DiamondClassifyWorker.obj
 0002:fffdf020       __unwindtable$?_Copy@?$basic_string@DU?$char_traits@D@std@@V?$allocator@D@2@@std@@QAEXII@Z 10000020     DiamondClassifyWorkerFactory.obj
 0002:fffdf020       __ehfuncinfo$??0DiamondBuildTaskSettings@U2@@QAE@ABU01@@Z 10000020     DiamondBuildWorker.obj
 0002:fffdf020       __ehfuncinfo$?append@?$QList@VDescriptor@U2@@@@QAEXABVDescriptor@U2@@@Z 10000020     DiamondClassifyWorker.obj
 0002:fffdf020       __tryblocktable$??0?$QList@VDescriptor@U2@@@@QAE@ABV0@@Z 10000020     DiamondClassifyWorker.obj
 0002:fffdf020       __ehfuncinfo$??1DiamondBuildTaskSettings@U2@@QAE@XZ 10000020     DiamondBuildWorker.obj
 0002:fffdf020       __ehfuncinfo$?append@?$QList@VQString@@@@QAEXABVQString@@@Z 10000020     DiamondBuildWorker.obj
 0002:fffdf020       __tryblocktable$??0?$QList@VQString@@@@QAE@ABV0@@Z 10000020     DiamondBuildWorker.obj
 0002:fffdf020       __unwindtable$?_Copy@?$basic_string@DU?$char_traits@D@std@@V?$allocator@D@2@@std@@QAEXII@Z 10000020     moc_GenomesPreparationTask.obj
 0002:fffdf020       __unwindtable$?_Copy@?$basic_string@DU?$char_traits@D@std@@V?$allocator@D@2@@std@@QAEXII@Z 10000020     moc_DiamondClassifyWorker.obj
 0002:fffdf020       __unwindtable$?_Copy@?$basic_string@DU?$char_traits@D@std@@V?$allocator@D@2@@std@@QAEXII@Z 10000020     DiamondBuildTask.obj
 0002:fffdf020       __unwindtable$?_Copy@?$basic_string@DU?$char_traits@D@std@@V?$allocator@D@2@@std@@QAEXII@Z 10000020     DiamondSupport.obj
 0002:fffdf020       __ehfuncinfo$?append@?$QList@VQString@@@@QAEXABVQString@@@Z 10000020     DiamondSupport.obj
 0002:fffdf020       __unwindtable$?detach_helper_grow@?$QList@VQString@@@@AAEPAUNode@1@HH@Z 10000020     DiamondClassifyWorker.obj
 0002:fffdf020       __ehfuncinfo$?createNode@?$QMapData@VQString@@VQVariant@@@@QAEPAU?$QMapNode@VQString@@VQVariant@@@@ABVQString@@ABVQVariant@@PAU2@_N@Z 10000020     DiamondClassifyWorkerFactory.obj
 0002:fffdf020       __ehfuncinfo$?append@?$QList@VQString@@@@QAEXABVQString@@@Z 10000020     DiamondClassifyTask.obj
 0002:fffdf020       __tryblocktable$??0?$QList@VQString@@@@QAE@ABV0@@Z 10000020     DiamondClassifyTask.obj
 0002:fffdf020       __unwindtable$?_Copy@?$basic_string@DU?$char_traits@D@std@@V?$allocator@D@2@@std@@QAEXII@Z 10000020     DiamondClassifyWorker.obj
 0002:fffdf020       __ehfuncinfo$?append@?$QList@VQString@@@@QAEXABVQString@@@Z 10000020     DiamondClassifyWorker.obj
 0002:fffdf020       __unwindtable$?detach_helper_grow@?$QList@PAVAttribute@U2@@@@AAEPAUNode@1@HH@Z 10000020     DiamondClassifyWorkerFactory.obj
 0002:fffdf020       __unwindtable$?detach_helper_grow@?$QList@PAVPortDescriptor@Workflow@U2@@@@AAEPAUNode@1@HH@Z 10000020     DiamondClassifyWorkerFactory.obj
 0002:fffdf020       __unwindtable$?_Copy@?$basic_string@DU?$char_traits@D@std@@V?$allocator@D@2@@std@@QAEXII@Z 10000020     DiamondBuildValidator.obj
 0002:fffdf020       __unwindtable$?detach_helper_grow@?$QList@VQString@@@@AAEPAUNode@1@HH@Z 10000020     DiamondBuildWorker.obj
 0001:fffff021       __unwindfunclet$??0DiamondClassifyTaskSettings@U2@@QAE@ABU01@@Z$3 10000021 f   DiamondClassifyWorker.obj
 0001:fffff021       __unwindfunclet$??1DiamondClassifyTaskSettings@U2@@QAE@XZ$3 10000021 f   DiamondClassifyWorker.obj
 0001:fffff022       __ehhandler$?append@?$QList@VQString@@@@QAEXABVQString@@@Z 10000022 f   DiamondClassifyWorker.obj
 0001:fffff022       __ehhandler$?append@?$QList@VQString@@@@QAEXABVQString@@@Z 10000022 f   DiamondBuildWorker.obj
 0001:fffff022       __ehhandler$?append@?$QList@VQString@@@@QAEXABVQString@@@Z 10000022 f   DiamondSupport.obj
 0001:fffff022       __ehhandler$?append@?$QList@VQString@@@@QAEXABVQString@@@Z 10000022 f   DiamondClassifyTask.obj
 0001:fffff022       __ehhandler$?append@?$QList@VQString@@@@QAEXABVQString@@@Z 10000022 f   DiamondBuildWorkerFactory.obj
 0001:fffff023       __ehhandler$??$getValue@VQString@@@BaseWorker@LocalWorkflow@U2@@IBE?AVQString@@ABV3@@Z 10000023 f   DiamondClassifyWorker.obj
 0001:fffff023       __unwindfunclet$??$getAttributeValue@VQString@@@Attribute@U2@@QBE?AVQString@@PAVWorkflowContext@Workflow@1@@Z$2 10000023 f   DiamondClassifyWorker.obj
 0001:fffff023       __ehhandler$?metaType@?$QVariantValueHelper@VQString@@@QtPrivate@@SA?AVQString@@ABVQVariant@@@Z 10000023 f   DiamondClassifyWorker.obj
 0001:fffff023       __ehhandler$??H@YA?BVQString@@ABV0@PBD@Z 10000023 f   DiamondBuildWorkerFactory.obj
 0001:fffff023       __ehhandler$??H@YA?BVQString@@ABV0@PBD@Z 10000023 f   DiamondClassifyWorker.obj
 0001:fffff023       __ehhandler$??H@YA?BVQString@@ABV0@PBD@Z 10000023 f   DiamondClassifyWorkerFactory.obj
 0002:fffdf024       __unwindtable$??$getAttributeValue@VQString@@@Attribute@U2@@QBE?AVQString@@PAVWorkflowContext@Workflow@1@@Z 10000024     DiamondClassifyWorker.obj
 0002:fffdf024       __ehfuncinfo$?append@?$QList@PAVPortDescriptor@Workflow@U2@@@@QAEXABQAVPortDescriptor@Workflow@U2@@@Z 10000024     DiamondClassifyWorkerFactory.obj
 0002:fffdf024       __ehfuncinfo$?node_copy@?$QList@VQString@@@@AAEXPAUNode@1@00@Z 10000024     DiamondClassifyWorker.obj
 0002:fffdf024       __ehfuncinfo$?createNode@?$QMapData@VQString@@I@@QAEPAU?$QMapNode@VQString@@I@@ABVQString@@ABIPAU2@_N@Z 10000024     DiamondClassifyWorker.obj
 0002:fffdf024       __ehfuncinfo$?node_copy@?$QList@VQString@@@@AAEXPAUNode@1@00@Z 10000024     DiamondSupport.obj
 0002:fffdf024       __unwindtable$??0DiamondClassifyTaskSettings@U2@@QAE@ABU01@@Z 10000024     DiamondClassifyWorker.obj
 0002:fffdf024       __ehfuncinfo$?createNode@?$QMapData@VDescriptor@U2@@V?$QExplicitlySharedDataPointer@VDataType@U2@@@@@@QAEPAU?$QMapNode@VDescriptor@U2@@V?$QExplicitlySharedDataPointer@VDataType@U2@@@@@@ABVDescriptor@U2@@ABV?$QExplicitlySharedDataPointer@VDataType@U2@@@@PAU2@_N@Z 10000024     DiamondClassifyWorkerFactory.obj
 0002:fffdf024       __unwindtable$??1DiamondClassifyTaskSettings@U2@@QAE@XZ 10000024     DiamondClassifyWorker.obj
 0002:fffdf024       __ehfuncinfo$?createNode@?$QMapData@VQString@@PAVPropertyDelegate@U2@@@@QAEPAU?$QMapNode@VQString@@PAVPropertyDelegate@U2@@@@ABVQString@@ABQAVPropertyDelegate@U2@@PAU2@_N@Z 10000024     DiamondClassifyWorkerFactory.obj
 0002:fffdf024       __ehfuncinfo$?node_copy@?$QList@VQString@@@@AAEXPAUNode@1@00@Z 10000024     GenomesPreparationTask.obj
 0002:fffdf024       __ehfuncinfo$?node_copy@?$QList@VQString@@@@AAEXPAUNode@1@00@Z 10000024     DiamondBuildWorker.obj
 0002:fffdf024       __ehfuncinfo$?node_copy@?$QList@VQString@@@@AAEXPAUNode@1@00@Z 10000024     DiamondBuildWorkerFactory.obj
 0002:fffdf024       __ehfuncinfo$?node_copy@?$QList@VDescriptor@U2@@@@AAEXPAUNode@1@00@Z 10000024     DiamondClassifyWorker.obj
 0002:fffdf024       __ehfuncinfo$?node_copy@?$QList@VQString@@@@AAEXPAUNode@1@00@Z 10000024     DiamondClassifyTask.obj
 0002:fffdf024       __ehfuncinfo$?append@?$QList@PAVAttribute@U2@@@@QAEXABQAVAttribute@U2@@@Z 10000024     DiamondClassifyWorkerFactory.obj
 0001:fffff028       __ehhandler$?createNode@?$QMapData@VQString@@VQVariant@@@@QAEPAU?$QMapNode@VQString@@VQVariant@@@@ABVQString@@ABVQVariant@@PAU2@_N@Z 10000028 f   DiamondClassifyWorkerFactory.obj
 0001:fffff028       __ehhandler$?createNode@?$QMapData@VQString@@VQVariant@@@@QAEPAU?$QMapNode@VQString@@VQVariant@@@@ABVQString@@ABVQVariant@@PAU2@_N@Z 10000028 f   DiamondClassifyWorker.obj
 0001:fffff028       __ehhandler$?createNode@?$QMapData@VQString@@VQScriptValue@@@@QAEPAU?$QMapNode@VQString@@VQScriptValue@@@@ABVQString@@ABVQScriptValue@@PAU2@_N@Z 10000028 f   DiamondClassifyWorker.obj
 0001:fffff02b       __unwindfunclet$??$getAttributeValue@VQString@@@Attribute@U2@@QBE?AVQString@@PAVWorkflowContext@Workflow@1@@Z$3 1000002b f   DiamondClassifyWorker.obj
 0001:fffff02c       __ehhandler$??1DiamondBuildTaskSettings@U2@@QAE@XZ 1000002c f   DiamondBuildWorker.obj
 0001:fffff02c       __ehhandler$??0DiamondBuildTaskSettings@U2@@QAE@ABU01@@Z 1000002c f   DiamondBuildWorker.obj
 0001:fffff02d       __unwindfunclet$??0DiamondClassifyTaskSettings@U2@@QAE@ABU01@@Z$4 1000002d f   DiamondClassifyWorker.obj
 0001:fffff02d       __unwindfunclet$??1DiamondClassifyTaskSettings@U2@@QAE@XZ$4 1000002d f   DiamondClassifyWorker.obj
 0001:fffff033       __unwindfunclet$??$getAttributeValue@VQString@@@Attribute@U2@@QBE?AVQString@@PAVWorkflowContext@Workflow@1@@Z$4 10000033 f   DiamondClassifyWorker.obj
 0002:fffdf034       __ehfuncinfo$??0?$QList@VQString@@@@QAE@ABV0@@Z 10000034     GenomesPreparationTask.obj
 0002:fffdf034       __ehfuncinfo$?detach_helper@?$QList@VDescriptor@U2@@@@AAEXH@Z 10000034     DiamondClassifyWorker.obj
 0002:fffdf034       __ehfuncinfo$??0?$QList@PAVPort@Workflow@U2@@@@QAE@ABV0@@Z 10000034     DiamondClassifyPrompter.obj
 0002:fffdf034       __ehfuncinfo$??0?$QList@VQString@@@@QAE@ABV0@@Z 10000034     DiamondClassifyTask.obj
 0002:fffdf034       __ehfuncinfo$??0?$QList@VQString@@@@QAE@ABV0@@Z 10000034     DiamondBuildWorker.obj
 0002:fffdf034       __ehfuncinfo$??0?$QList@VDescriptor@U2@@@@QAE@ABV0@@Z 10000034     DiamondClassifyWorker.obj
 0001:fffff039       __unwindfunclet$??1DiamondClassifyTaskSettings@U2@@QAE@XZ$5 10000039 f   DiamondClassifyWorker.obj
 0001:fffff039       __unwindfunclet$??0DiamondClassifyTaskSettings@U2@@QAE@ABU01@@Z$5 10000039 f   DiamondClassifyWorker.obj
 0001:fffff03b       __unwindfunclet$??$getAttributeValue@VQString@@@Attribute@U2@@QBE?AVQString@@PAVWorkflowContext@Workflow@1@@Z$5 1000003b f   DiamondClassifyWorker.obj
 0002:fffdf040       __ehfuncinfo$?_Copy@?$basic_string@DU?$char_traits@D@std@@V?$allocator@D@2@@std@@QAEXII@Z 10000040     moc_DiamondSupportPlugin.obj
 0002:fffdf040       __ehfuncinfo$?_Copy@?$basic_string@DU?$char_traits@D@std@@V?$allocator@D@2@@std@@QAEXII@Z 10000040     DiamondClassifyTask.obj
 0002:fffdf040       __ehfuncinfo$?_Copy@?$basic_string@DU?$char_traits@D@std@@V?$allocator@D@2@@std@@QAEXII@Z 10000040     moc_DiamondBuildTask.obj
 0002:fffdf040       __ehfuncinfo$?_Copy@?$basic_string@DU?$char_traits@D@std@@V?$allocator@D@2@@std@@QAEXII@Z 10000040     moc_GenomesPreparationTask.obj
 0002:fffdf040       __ehfuncinfo$?_Copy@?$basic_string@DU?$char_traits@D@std@@V?$allocator@D@2@@std@@QAEXII@Z 10000040     DiamondBuildWorkerFactory.obj
 0002:fffdf040       __ehfuncinfo$?_Copy@?$basic_string@DU?$char_traits@D@std@@V?$allocator@D@2@@std@@QAEXII@Z 10000040     moc_DiamondClassifyWorker.obj
 0002:fffdf040       __ehfuncinfo$?detach_helper_grow@?$QList@PAVAttribute@U2@@@@AAEPAUNode@1@HH@Z 10000040     DiamondClassifyWorkerFactory.obj
 0002:fffdf040       __ehfuncinfo$?_Copy@?$basic_string@DU?$char_traits@D@std@@V?$allocator@D@2@@std@@QAEXII@Z 10000040     moc_DiamondClassifyPrompter.obj
 0002:fffdf040       __ehfuncinfo$?detach_helper_grow@?$QList@VDescriptor@U2@@@@AAEPAUNode@1@HH@Z 10000040     DiamondClassifyWorker.obj
 0002:fffdf040       __ehfuncinfo$?_Copy@?$basic_string@DU?$char_traits@D@std@@V?$allocator@D@2@@std@@QAEXII@Z 10000040     DiamondSupportPlugin.obj
 0002:fffdf040       __ehfuncinfo$?detach_helper_grow@?$QList@VQString@@@@AAEPAUNode@1@HH@Z 10000040     DiamondBuildWorkerFactory.obj
 0002:fffdf040       __ehfuncinfo$?_Copy@?$basic_string@DU?$char_traits@D@std@@V?$allocator@D@2@@std@@QAEXII@Z 10000040     DiamondClassifyWorkerFactory.obj
 0002:fffdf040       __ehfuncinfo$?detach_helper_grow@?$QList@PAVPortDescriptor@Workflow@U2@@@@AAEPAUNode@1@HH@Z 10000040     DiamondClassifyWorkerFactory.obj
 0002:fffdf040       __ehfuncinfo$?_Copy@?$basic_string@DU?$char_traits@D@std@@V?$allocator@D@2@@std@@QAEXII@Z 10000040     moc_DiamondBuildPrompter.obj
 0002:fffdf040       __ehfuncinfo$?_Copy@?$basic_string@DU?$char_traits@D@std@@V?$allocator@D@2@@std@@QAEXII@Z 10000040     DiamondBuildTask.obj
 0002:fffdf040       __ehfuncinfo$?_Copy@?$basic_string@DU?$char_traits@D@std@@V?$allocator@D@2@@std@@QAEXII@Z 10000040     DiamondClassifyPrompter.obj
 0002:fffdf040       __ehfuncinfo$?_Copy@?$basic_string@DU?$char_traits@D@std@@V?$allocator@D@2@@std@@QAEXII@Z 10000040     moc_DiamondBuildWorker.obj
 0002:fffdf040       __ehfuncinfo$?_Copy@?$basic_string@DU?$char_traits@D@std@@V?$allocator@D@2@@std@@QAEXII@Z 10000040     DiamondClassifyWorker.obj
 0002:fffdf040       __ehfuncinfo$?_Copy@?$basic_string@DU?$char_traits@D@std@@V?$allocator@D@2@@std@@QAEXII@Z 10000040     GenomesPreparationTask.obj
 0002:fffdf040       __ehfuncinfo$?detach_helper_grow@?$QList@VQString@@@@AAEPAUNode@1@HH@Z 10000040     DiamondBuildWorker.obj
 0002:fffdf040       __ehfuncinfo$?_Copy@?$basic_string@DU?$char_traits@D@std@@V?$allocator@D@2@@std@@QAEXII@Z 10000040     DiamondBuildWorker.obj
 0002:fffdf040       __ehfuncinfo$?_Copy@?$basic_string@DU?$char_traits@D@std@@V?$allocator@D@2@@std@@QAEXII@Z 10000040     DiamondSupport.obj
 0002:fffdf040       __ehfuncinfo$?_Copy@?$basic_string@DU?$char_traits@D@std@@V?$allocator@D@2@@std@@QAEXII@Z 10000040     DiamondBuildValidator.obj
 0002:fffdf040       __ehfuncinfo$?detach_helper_grow@?$QList@VQString@@@@AAEPAUNode@1@HH@Z 10000040     DiamondSupport.obj
 0002:fffdf040       __ehfuncinfo$?_Copy@?$basic_string@DU?$char_traits@D@std@@V?$allocator@D@2@@std@@QAEXII@Z 10000040     moc_DiamondSupport.obj
 0002:fffdf040       __ehfuncinfo$?detach_helper_grow@?$QList@VQString@@@@AAEPAUNode@1@HH@Z 10000040     DiamondClassifyTask.obj
 0002:fffdf040       __ehfuncinfo$?detach_helper_grow@?$QList@VQString@@@@AAEPAUNode@1@HH@Z 10000040     DiamondClassifyWorker.obj
 0002:fffdf040       __ehfuncinfo$?_Copy@?$basic_string@DU?$char_traits@D@std@@V?$allocator@D@2@@std@@QAEXII@Z 10000040     moc_DiamondClassifyTask.obj
 0002:fffdf044       __tryblocktable$?append@?$QList@VQString@@@@QAEXABVQString@@@Z 10000044     DiamondClassifyWorker.obj
 0002:fffdf044       __tryblocktable$?createNode@?$QMapData@VQString@@VQVariant@@@@QAEPAU?$QMapNode@VQString@@VQVariant@@@@ABVQString@@ABVQVariant@@PAU2@_N@Z 10000044     DiamondClassifyWorkerFactory.obj
 0002:fffdf044       __tryblocktable$?append@?$QList@VQString@@@@QAEXABVQString@@@Z 10000044     DiamondBuildWorker.obj
 0002:fffdf044       __tryblocktable$?append@?$QList@VQString@@@@QAEXABVQString@@@Z 10000044     DiamondClassifyTask.obj
 0002:fffdf044       __tryblocktable$?createNode@?$QMapData@VQString@@VQScriptValue@@@@QAEPAU?$QMapNode@VQString@@VQScriptValue@@@@ABVQString@@ABVQScriptValue@@PAU2@_N@Z 10000044     DiamondClassifyWorker.obj
 0002:fffdf044       __tryblocktable$?createNode@?$QMapData@VQString@@VQVariant@@@@QAEPAU?$QMapNode@VQString@@VQVariant@@@@ABVQString@@ABVQVariant@@PAU2@_N@Z 10000044     DiamondClassifyWorker.obj
 0002:fffdf044       __tryblocktable$?append@?$QList@VQString@@@@QAEXABVQString@@@Z 10000044     DiamondBuildWorkerFactory.obj
 0002:fffdf044       __tryblocktable$?append@?$QList@VDescriptor@U2@@@@QAEXABVDescriptor@U2@@@Z 10000044     DiamondClassifyWorker.obj
 0001:fffff044       __unwindfunclet$??$getAttributeValue@VQString@@@Attribute@U2@@QBE?AVQString@@PAVWorkflowContext@Workflow@1@@Z$6 10000044 f   DiamondClassifyWorker.obj
 0002:fffdf044       __tryblocktable$?append@?$QList@VQString@@@@QAEXABVQString@@@Z 10000044     DiamondSupport.obj
 0001:fffff045       __unwindfunclet$??0DiamondClassifyTaskSettings@U2@@QAE@ABU01@@Z$6 10000045 f   DiamondClassifyWorker.obj
 0001:fffff045       __unwindfunclet$??1DiamondClassifyTaskSettings@U2@@QAE@XZ$6 10000045 f   DiamondClassifyWorker.obj
 0002:fffdf048       __unwindtable$?node_copy@?$QList@VQString@@@@AAEXPAUNode@1@00@Z 10000048     GenomesPreparationTask.obj
 0002:fffdf048       __unwindtable$?node_copy@?$QList@VQString@@@@AAEXPAUNode@1@00@Z 10000048     DiamondClassifyTask.obj
 0002:fffdf048       __unwindtable$?append@?$QList@PAVAttribute@U2@@@@QAEXABQAVAttribute@U2@@@Z 10000048     DiamondClassifyWorkerFactory.obj
 0002:fffdf048       __unwindtable$?createNode@?$QMapData@VDescriptor@U2@@V?$QExplicitlySharedDataPointer@VDataType@U2@@@@@@QAEPAU?$QMapNode@VDescriptor@U2@@V?$QExplicitlySharedDataPointer@VDataType@U2@@@@@@ABVDescriptor@U2@@ABV?$QExplicitlySharedDataPointer@VDataType@U2@@@@PAU2@_N@Z 10000048     DiamondClassifyWorkerFactory.obj
 0002:fffdf048       __unwindtable$?node_copy@?$QList@VQString@@@@AAEXPAUNode@1@00@Z 10000048     DiamondSupport.obj
 0002:fffdf048       __unwindtable$?node_copy@?$QList@VQString@@@@AAEXPAUNode@1@00@Z 10000048     DiamondBuildWorkerFactory.obj
 0002:fffdf048       __unwindtable$?createNode@?$QMapData@VQString@@I@@QAEPAU?$QMapNode@VQString@@I@@ABVQString@@ABIPAU2@_N@Z 10000048     DiamondClassifyWorker.obj
 0002:fffdf048       __unwindtable$?node_copy@?$QList@VQString@@@@AAEXPAUNode@1@00@Z 10000048     DiamondBuildWorker.obj
 0002:fffdf048       __unwindtable$?append@?$QList@PAVPortDescriptor@Workflow@U2@@@@QAEXABQAVPortDescriptor@Workflow@U2@@@Z 10000048     DiamondClassifyWorkerFactory.obj
 0002:fffdf048       __unwindtable$?node_copy@?$QList@VQString@@@@AAEXPAUNode@1@00@Z 10000048     DiamondClassifyWorker.obj
 0002:fffdf048       __unwindtable$?createNode@?$QMapData@VQString@@PAVPropertyDelegate@U2@@@@QAEPAU?$QMapNode@VQString@@PAVPropertyDelegate@U2@@@@ABVQString@@ABQAVPropertyDelegate@U2@@PAU2@_N@Z 10000048     DiamondClassifyWorkerFactory.obj
 0002:fffdf048       __unwindtable$?node_copy@?$QList@VDescriptor@U2@@@@AAEXPAUNode@1@00@Z 10000048     DiamondClassifyWorker.obj
 0001:fffff04d       __unwindfunclet$??$getAttributeValue@VQString@@@Attribute@U2@@QBE?AVQString@@PAVWorkflowContext@Workflow@1@@Z$7 1000004d f   DiamondClassifyWorker.obj
 0001:fffff051       __ehhandler$??1DiamondClassifyTaskSettings@U2@@QAE@XZ 10000051 f   DiamondClassifyWorker.obj
 0001:fffff051       __ehhandler$??0DiamondClassifyTaskSettings@U2@@QAE@ABU01@@Z 10000051 f   DiamondClassifyWorker.obj
 0001:fffff056       __unwindfunclet$??$getAttributeValue@VQString@@@Attribute@U2@@QBE?AVQString@@PAVWorkflowContext@Workflow@1@@Z$8 10000056 f   DiamondClassifyWorker.obj
 0001:fffff05f       __unwindfunclet$??$getAttributeValue@VQString@@@Attribute@U2@@QBE?AVQString@@PAVWorkflowContext@Workflow@1@@Z$9 1000005f f   DiamondClassifyWorker.obj
 0001:fffff062       __catch$?node_copy@?$QList@VQString@@@@AAEXPAUNode@1@00@Z$2 10000062 f   DiamondClassifyTask.obj
 0001:fffff062       __catch$?node_copy@?$QList@VQString@@@@AAEXPAUNode@1@00@Z$2 10000062 f   DiamondBuildWorkerFactory.obj
 0001:fffff062       __catch$?node_copy@?$QList@VQString@@@@AAEXPAUNode@1@00@Z$2 10000062 f   DiamondSupport.obj
 0001:fffff062       __catch$?node_copy@?$QList@VQString@@@@AAEXPAUNode@1@00@Z$2 10000062 f   DiamondClassifyWorker.obj
 0001:fffff062       __catch$?node_copy@?$QList@VQString@@@@AAEXPAUNode@1@00@Z$2 10000062 f   DiamondBuildWorker.obj
 0001:fffff062       __catch$?node_copy@?$QList@VQString@@@@AAEXPAUNode@1@00@Z$2 10000062 f   GenomesPreparationTask.obj
 0002:fffdf064       __tryblocktable$?detach_helper_grow@?$QList@VQString@@@@AAEPAUNode@1@HH@Z 10000064     DiamondBuildWorkerFactory.obj
 0002:fffdf064       __tryblocktable$?_Copy@?$basic_string@DU?$char_traits@D@std@@V?$allocator@D@2@@std@@QAEXII@Z 10000064     moc_DiamondBuildTask.obj
 0002:fffdf064       __tryblocktable$?_Copy@?$basic_string@DU?$char_traits@D@std@@V?$allocator@D@2@@std@@QAEXII@Z 10000064     DiamondSupportPlugin.obj
 0002:fffdf064       __tryblocktable$?_Copy@?$basic_string@DU?$char_traits@D@std@@V?$allocator@D@2@@std@@QAEXII@Z 10000064     moc_DiamondClassifyTask.obj
 0002:fffdf064       __tryblocktable$?_Copy@?$basic_string@DU?$char_traits@D@std@@V?$allocator@D@2@@std@@QAEXII@Z 10000064     DiamondClassifyWorker.obj
 0002:fffdf064       __tryblocktable$?_Copy@?$basic_string@DU?$char_traits@D@std@@V?$allocator@D@2@@std@@QAEXII@Z 10000064     moc_DiamondBuildWorker.obj
 0002:fffdf064       __tryblocktable$?detach_helper_grow@?$QList@VQString@@@@AAEPAUNode@1@HH@Z 10000064     DiamondClassifyWorker.obj
 0002:fffdf064       __tryblocktable$?_Copy@?$basic_string@DU?$char_traits@D@std@@V?$allocator@D@2@@std@@QAEXII@Z 10000064     DiamondClassifyTask.obj
 0002:fffdf064       __tryblocktable$?_Copy@?$basic_string@DU?$char_traits@D@std@@V?$allocator@D@2@@std@@QAEXII@Z 10000064     moc_DiamondSupportPlugin.obj
 0002:fffdf064       __tryblocktable$?detach_helper_grow@?$QList@PAVAttribute@U2@@@@AAEPAUNode@1@HH@Z 10000064     DiamondClassifyWorkerFactory.obj
 0002:fffdf064       __tryblocktable$?_Copy@?$basic_string@DU?$char_traits@D@std@@V?$allocator@D@2@@std@@QAEXII@Z 10000064     DiamondBuildWorker.obj
 0002:fffdf064       __tryblocktable$?detach_helper_grow@?$QList@VQString@@@@AAEPAUNode@1@HH@Z 10000064     DiamondClassifyTask.obj
 0002:fffdf064       __tryblocktable$?_Copy@?$basic_string@DU?$char_traits@D@std@@V?$allocator@D@2@@std@@QAEXII@Z 10000064     moc_DiamondClassifyWorker.obj
 0002:fffdf064       __tryblocktable$?_Copy@?$basic_string@DU?$char_traits@D@std@@V?$allocator@D@2@@std@@QAEXII@Z 10000064     GenomesPreparationTask.obj
 0002:fffdf064       __tryblocktable$?_Copy@?$basic_string@DU?$char_traits@D@std@@V?$allocator@D@2@@std@@QAEXII@Z 10000064     DiamondClassifyWorkerFactory.obj
 0002:fffdf064       __tryblocktable$?_Copy@?$basic_string@DU?$char_traits@D@std@@V?$allocator@D@2@@std@@QAEXII@Z 10000064     moc_GenomesPreparationTask.obj
 0002:fffdf064       __tryblocktable$?_Copy@?$basic_string@DU?$char_traits@D@std@@V?$allocator@D@2@@std@@QAEXII@Z 10000064     moc_DiamondSupport.obj
 0002:fffdf064       __tryblocktable$?_Copy@?$basic_string@DU?$char_traits@D@std@@V?$allocator@D@2@@std@@QAEXII@Z 10000064     DiamondBuildTask.obj
 0002:fffdf064       __tryblocktable$?_Copy@?$basic_string@DU?$char_traits@D@std@@V?$allocator@D@2@@std@@QAEXII@Z 10000064     DiamondClassifyPrompter.obj
 0002:fffdf064       __tryblocktable$?_Copy@?$basic_string@DU?$char_traits@D@std@@V?$allocator@D@2@@std@@QAEXII@Z 10000064     DiamondSupport.obj
 0002:fffdf064       __tryblocktable$?_Copy@?$basic_string@DU?$char_traits@D@std@@V?$allocator@D@2@@std@@QAEXII@Z 10000064     DiamondBuildValidator.obj
 0002:fffdf064       __tryblocktable$?_Copy@?$basic_string@DU?$char_traits@D@std@@V?$allocator@D@2@@std@@QAEXII@Z 10000064     moc_DiamondClassifyPrompter.obj
 0002:fffdf064       __tryblocktable$?detach_helper_grow@?$QList@VQString@@@@AAEPAUNode@1@HH@Z 10000064     DiamondSupport.obj
 0002:fffdf064       __tryblocktable$?detach_helper_grow@?$QList@VDescriptor@U2@@@@AAEPAUNode@1@HH@Z 10000064     DiamondClassifyWorker.obj
 0002:fffdf064       __tryblocktable$?_Copy@?$basic_string@DU?$char_traits@D@std@@V?$allocator@D@2@@std@@QAEXII@Z 10000064     DiamondBuildWorkerFactory.obj
 0002:fffdf064       __tryblocktable$?detach_helper_grow@?$QList@VQString@@@@AAEPAUNode@1@HH@Z 10000064     DiamondBuildWorker.obj
 0002:fffdf064       __tryblocktable$?_Copy@?$basic_string@DU?$char_traits@D@std@@V?$allocator@D@2@@std@@QAEXII@Z 10000064     moc_DiamondBuildPrompter.obj
 0002:fffdf064       __tryblocktable$?detach_helper_grow@?$QList@PAVPortDescriptor@Workflow@U2@@@@AAEPAUNode@1@HH@Z 10000064     DiamondClassifyWorkerFactory.obj
 0001:fffff068       __unwindfunclet$??$getAttributeValue@VQString@@@Attribute@U2@@QBE?AVQString@@PAVWorkflowContext@Workflow@1@@Z$10 10000068 f   DiamondClassifyWorker.obj
 0002:fffdf06c       __unwindtable$?append@?$QList@VQString@@@@QAEXABVQString@@@Z 1000006c     DiamondSupport.obj
 0002:fffdf06c       __unwindtable$?append@?$QList@VQString@@@@QAEXABVQString@@@Z 1000006c     DiamondBuildWorkerFactory.obj
 0002:fffdf06c       __unwindtable$?append@?$QList@VQString@@@@QAEXABVQString@@@Z 1000006c     DiamondBuildWorker.obj
 0002:fffdf06c       __unwindtable$?createNode@?$QMapData@VQString@@VQVariant@@@@QAEPAU?$QMapNode@VQString@@VQVariant@@@@ABVQString@@ABVQVariant@@PAU2@_N@Z 1000006c     DiamondClassifyWorker.obj
 0002:fffdf06c       __unwindtable$?append@?$QList@VDescriptor@U2@@@@QAEXABVDescriptor@U2@@@Z 1000006c     DiamondClassifyWorker.obj
 0002:fffdf06c       __unwindtable$?append@?$QList@VQString@@@@QAEXABVQString@@@Z 1000006c     DiamondClassifyTask.obj
 0002:fffdf06c       __unwindtable$?createNode@?$QMapData@VQString@@VQVariant@@@@QAEPAU?$QMapNode@VQString@@VQVariant@@@@ABVQString@@ABVQVariant@@PAU2@_N@Z 1000006c     DiamondClassifyWorkerFactory.obj
 0002:fffdf06c       __unwindtable$?createNode@?$QMapData@VQString@@VQScriptValue@@@@QAEPAU?$QMapNode@VQString@@VQScriptValue@@@@ABVQString@@ABVQScriptValue@@PAU2@_N@Z 1000006c     DiamondClassifyWorker.obj
 0002:fffdf06c       __unwindtable$?append@?$QList@VQString@@@@QAEXABVQString@@@Z 1000006c     DiamondClassifyWorker.obj
 0001:fffff071       __unwindfunclet$??$getAttributeValue@VQString@@@Attribute@U2@@QBE?AVQString@@PAVWorkflowContext@Workflow@1@@Z$11 10000071 f   DiamondClassifyWorker.obj
 0001:fffff07a       __unwindfunclet$??$getAttributeValue@VQString@@@Attribute@U2@@QBE?AVQString@@PAVWorkflowContext@Workflow@1@@Z$12 1000007a f   DiamondClassifyWorker.obj
 0001:fffff07d       __catch$?append@?$QList@VQString@@@@QAEXABVQString@@@Z$0 1000007d f   DiamondClassifyWorker.obj
 0001:fffff07d       __catch$?append@?$QList@VQString@@@@QAEXABVQString@@@Z$0 1000007d f   DiamondBuildWorkerFactory.obj
 0001:fffff07d       __catch$?append@?$QList@VQString@@@@QAEXABVQString@@@Z$0 1000007d f   DiamondBuildWorker.obj
 0001:fffff07d       __catch$?append@?$QList@VQString@@@@QAEXABVQString@@@Z$0 1000007d f   DiamondSupport.obj
 0001:fffff07d       __catch$?append@?$QList@VQString@@@@QAEXABVQString@@@Z$0 1000007d f   DiamondClassifyTask.obj
 0001:fffff083       __ehhandler$??$getAttributeValue@VQString@@@Attribute@U2@@QBE?AVQString@@PAVWorkflowContext@Workflow@1@@Z 10000083 f   DiamondClassifyWorker.obj
 0001:fffff085       __catch$?createNode@?$QMapData@VQString@@PAVPropertyDelegate@U2@@@@QAEPAU?$QMapNode@VQString@@PAVPropertyDelegate@U2@@@@ABVQString@@ABQAVPropertyDelegate@U2@@PAU2@_N@Z$2 10000085 f   DiamondClassifyWorkerFactory.obj
 0001:fffff085       __catch$?append@?$QList@PAVAttribute@U2@@@@QAEXABQAVAttribute@U2@@@Z$4 10000085 f   DiamondClassifyWorkerFactory.obj
 0001:fffff085       __catch$?append@?$QList@PAVPortDescriptor@Workflow@U2@@@@QAEXABQAVPortDescriptor@Workflow@U2@@@Z$4 10000085 f   DiamondClassifyWorkerFactory.obj
 0001:fffff085       __catch$?node_copy@?$QList@VDescriptor@U2@@@@AAEXPAUNode@1@00@Z$0 10000085 f   DiamondClassifyWorker.obj
 0001:fffff085       __catch$?createNode@?$QMapData@VQString@@I@@QAEPAU?$QMapNode@VQString@@I@@ABVQString@@ABIPAU2@_N@Z$2 10000085 f   DiamondClassifyWorker.obj
 0001:fffff08e       __catch$?createNode@?$QMapData@VQString@@VQVariant@@@@QAEPAU?$QMapNode@VQString@@VQVariant@@@@ABVQString@@ABVQVariant@@PAU2@_N@Z$0 1000008e f   DiamondClassifyWorker.obj
 0001:fffff08e       __catch$?createNode@?$QMapData@VQString@@VQScriptValue@@@@QAEPAU?$QMapNode@VQString@@VQScriptValue@@@@ABVQString@@ABVQScriptValue@@PAU2@_N@Z$0 1000008e f   DiamondClassifyWorker.obj
 0001:fffff08e       __catch$?createNode@?$QMapData@VQString@@VQVariant@@@@QAEPAU?$QMapNode@VQString@@VQVariant@@@@ABVQString@@ABVQVariant@@PAU2@_N@Z$0 1000008e f   DiamondClassifyWorkerFactory.obj
 0001:fffff096       __catch$?_Copy@?$basic_string@DU?$char_traits@D@std@@V?$allocator@D@2@@std@@QAEXII@Z$0 10000096 f   DiamondBuildWorkerFactory.obj
 0001:fffff096       __catch$?_Copy@?$basic_string@DU?$char_traits@D@std@@V?$allocator@D@2@@std@@QAEXII@Z$0 10000096 f   DiamondBuildValidator.obj
 0001:fffff096       __catch$?_Copy@?$basic_string@DU?$char_traits@D@std@@V?$allocator@D@2@@std@@QAEXII@Z$0 10000096 f   moc_DiamondBuildPrompter.obj
 0001:fffff096       __catch$?_Copy@?$basic_string@DU?$char_traits@D@std@@V?$allocator@D@2@@std@@QAEXII@Z$0 10000096 f   moc_DiamondClassifyWorker.obj
 0001:fffff096       __catch$?_Copy@?$basic_string@DU?$char_traits@D@std@@V?$allocator@D@2@@std@@QAEXII@Z$0 10000096 f   DiamondBuildWorker.obj
 0001:fffff096       __catch$?_Copy@?$basic_string@DU?$char_traits@D@std@@V?$allocator@D@2@@std@@QAEXII@Z$0 10000096 f   moc_DiamondSupportPlugin.obj
 0001:fffff096       __catch$?_Copy@?$basic_string@DU?$char_traits@D@std@@V?$allocator@D@2@@std@@QAEXII@Z$0 10000096 f   GenomesPreparationTask.obj
 0001:fffff096       __catch$?_Copy@?$basic_string@DU?$char_traits@D@std@@V?$allocator@D@2@@std@@QAEXII@Z$0 10000096 f   moc_DiamondClassifyPrompter.obj
 0001:fffff096       __catch$?_Copy@?$basic_string@DU?$char_traits@D@std@@V?$allocator@D@2@@std@@QAEXII@Z$0 10000096 f   DiamondClassifyWorker.obj
 0001:fffff096       __catch$?_Copy@?$basic_string@DU?$char_traits@D@std@@V?$allocator@D@2@@std@@QAEXII@Z$0 10000096 f   DiamondClassifyPrompter.obj
 0001:fffff096       __catch$?_Copy@?$basic_string@DU?$char_traits@D@std@@V?$allocator@D@2@@std@@QAEXII@Z$0 10000096 f   DiamondClassifyTask.obj
 0001:fffff096       __catch$?_Copy@?$basic_string@DU?$char_traits@D@std@@V?$allocator@D@2@@std@@QAEXII@Z$0 10000096 f   moc_DiamondSupport.obj
 0001:fffff096       __catch$?_Copy@?$basic_string@DU?$char_traits@D@std@@V?$allocator@D@2@@std@@QAEXII@Z$0 10000096 f   DiamondSupportPlugin.obj
 0001:fffff096       __catch$?_Copy@?$basic_string@DU?$char_traits@D@std@@V?$allocator@D@2@@std@@QAEXII@Z$0 10000096 f   DiamondSupport.obj
 0001:fffff096       __catch$?_Copy@?$basic_string@DU?$char_traits@D@std@@V?$allocator@D@2@@std@@QAEXII@Z$0 10000096 f   DiamondBuildTask.obj
 0001:fffff096       __catch$?_Copy@?$basic_string@DU?$char_traits@D@std@@V?$allocator@D@2@@std@@QAEXII@Z$0 10000096 f   DiamondClassifyWorkerFactory.obj
 0001:fffff096       __catch$?_Copy@?$basic_string@DU?$char_traits@D@std@@V?$allocator@D@2@@std@@QAEXII@Z$0 10000096 f   moc_DiamondClassifyTask.obj
 0001:fffff096       __catch$?_Copy@?$basic_string@DU?$char_traits@D@std@@V?$allocator@D@2@@std@@QAEXII@Z$0 10000096 f   moc_GenomesPreparationTask.obj
 0001:fffff096       __catch$?_Copy@?$basic_string@DU?$char_traits@D@std@@V?$allocator@D@2@@std@@QAEXII@Z$0 10000096 f   moc_DiamondBuildTask.obj
 0001:fffff096       __catch$?_Copy@?$basic_string@DU?$char_traits@D@std@@V?$allocator@D@2@@std@@QAEXII@Z$0 10000096 f   moc_DiamondBuildWorker.obj
 0001:fffff09d       __catch$?createNode@?$QMapData@VDescriptor@U2@@V?$QExplicitlySharedDataPointer@VDataType@U2@@@@@@QAEPAU?$QMapNode@VDescriptor@U2@@V?$QExplicitlySharedDataPointer@VDataType@U2@@@@@@ABVDescriptor@U2@@ABV?$QExplicitlySharedDataPointer@VDataType@U2@@@@PAU2@_N@Z$2 1000009d f   DiamondClassifyWorkerFactory.obj
 0001:fffff09e       __catch$??0?$QList@VQString@@@@QAE@ABV0@@Z$0 1000009e f   DiamondBuildWorker.obj
 0001:fffff09e       __catch$??0?$QList@PAVPort@Workflow@U2@@@@QAE@ABV0@@Z$0 1000009e f   DiamondClassifyPrompter.obj
 0001:fffff09e       __catch$??0?$QList@VQString@@@@QAE@ABV0@@Z$0 1000009e f   GenomesPreparationTask.obj
 0001:fffff09e       __catch$??0?$QList@VDescriptor@U2@@@@QAE@ABV0@@Z$0 1000009e f   DiamondClassifyWorker.obj
 0001:fffff09e       __catch$??0?$QList@VQString@@@@QAE@ABV0@@Z$0 1000009e f   DiamondClassifyTask.obj
 0001:fffff0a3       __catch$?createNode@?$QMapData@VQString@@VQVariant@@@@QAEPAU?$QMapNode@VQString@@VQVariant@@@@ABVQString@@ABVQVariant@@PAU2@_N@Z$2 100000a3 f   DiamondClassifyWorkerFactory.obj
 0001:fffff0a3       __catch$?createNode@?$QMapData@VQString@@VQVariant@@@@QAEPAU?$QMapNode@VQString@@VQVariant@@@@ABVQString@@ABVQVariant@@PAU2@_N@Z$2 100000a3 f   DiamondClassifyWorker.obj
 0001:fffff0a3       __catch$?createNode@?$QMapData@VQString@@VQScriptValue@@@@QAEPAU?$QMapNode@VQString@@VQScriptValue@@@@ABVQString@@ABVQScriptValue@@PAU2@_N@Z$2 100000a3 f   DiamondClassifyWorker.obj
 0001:fffff0aa       __catch$?detach_helper@?$QList@VDescriptor@U2@@@@AAEXH@Z$0 100000aa f   DiamondClassifyWorker.obj
 0001:fffff0ac       __catch$?append@?$QList@VDescriptor@U2@@@@QAEXABVDescriptor@U2@@@Z$0 100000ac f   DiamondClassifyWorker.obj
 0001:fffff0ac       __catch$?append@?$QList@VDescriptor@U2@@@@QAEXABVDescriptor@U2@@@Z$2 100000ac f   DiamondClassifyWorker.obj
 0001:fffff0ce       __catch$?append@?$QList@VQString@@@@QAEXABVQString@@@Z$4 100000ce f   DiamondBuildWorkerFactory.obj
 0001:fffff0ce       __catch$?append@?$QList@VQString@@@@QAEXABVQString@@@Z$4 100000ce f   DiamondClassifyTask.obj
 0001:fffff0ce       __catch$?append@?$QList@VQString@@@@QAEXABVQString@@@Z$4 100000ce f   DiamondBuildWorker.obj
 0001:fffff0ce       __catch$?append@?$QList@VQString@@@@QAEXABVQString@@@Z$4 100000ce f   DiamondClassifyWorker.obj
 0001:fffff0ce       __catch$?append@?$QList@VQString@@@@QAEXABVQString@@@Z$4 100000ce f   DiamondSupport.obj
 0001:fffff0d3       __catch$?_Copy@?$basic_string@DU?$char_traits@D@std@@V?$allocator@D@2@@std@@QAEXII@Z$1 100000d3 f   DiamondClassifyTask.obj
 0001:fffff0d3       __catch$?_Copy@?$basic_string@DU?$char_traits@D@std@@V?$allocator@D@2@@std@@QAEXII@Z$1 100000d3 f   DiamondClassifyPrompter.obj
 0001:fffff0d3       __catch$?_Copy@?$basic_string@DU?$char_traits@D@std@@V?$allocator@D@2@@std@@QAEXII@Z$1 100000d3 f   DiamondBuildWorker.obj
 0001:fffff0d3       __catch$?_Copy@?$basic_string@DU?$char_traits@D@std@@V?$allocator@D@2@@std@@QAEXII@Z$1 100000d3 f   moc_DiamondSupport.obj
 0001:fffff0d3       __catch$?_Copy@?$basic_string@DU?$char_traits@D@std@@V?$allocator@D@2@@std@@QAEXII@Z$1 100000d3 f   moc_GenomesPreparationTask.obj
 0001:fffff0d3       __catch$?_Copy@?$basic_string@DU?$char_traits@D@std@@V?$allocator@D@2@@std@@QAEXII@Z$1 100000d3 f   DiamondSupportPlugin.obj
 0001:fffff0d3       __catch$?_Copy@?$basic_string@DU?$char_traits@D@std@@V?$allocator@D@2@@std@@QAEXII@Z$1 100000d3 f   moc_DiamondBuildTask.obj
 0001:fffff0d3       __catch$?_Copy@?$basic_string@DU?$char_traits@D@std@@V?$allocator@D@2@@std@@QAEXII@Z$1 100000d3 f   moc_DiamondClassifyWorker.obj
 0001:fffff0d3       __catch$?_Copy@?$basic_string@DU?$char_traits@D@std@@V?$allocator@D@2@@std@@QAEXII@Z$1 100000d3 f   GenomesPreparationTask.obj
 0001:fffff0d3       __catch$?_Copy@?$basic_string@DU?$char_traits@D@std@@V?$allocator@D@2@@std@@QAEXII@Z$1 100000d3 f   moc_DiamondBuildWorker.obj
 0001:fffff0d3       __catch$?_Copy@?$basic_string@DU?$char_traits@D@std@@V?$allocator@D@2@@std@@QAEXII@Z$1 100000d3 f   moc_DiamondClassifyPrompter.obj
 0001:fffff0d3       __catch$?_Copy@?$basic_string@DU?$char_traits@D@std@@V?$allocator@D@2@@std@@QAEXII@Z$1 100000d3 f   moc_DiamondSupportPlugin.obj
 0001:fffff0d3       __catch$?_Copy@?$basic_string@DU?$char_traits@D@std@@V?$allocator@D@2@@std@@QAEXII@Z$1 100000d3 f   DiamondClassifyWorker.obj
 0001:fffff0d3       __catch$?_Copy@?$basic_string@DU?$char_traits@D@std@@V?$allocator@D@2@@std@@QAEXII@Z$1 100000d3 f   DiamondBuildValidator.obj
 0001:fffff0d3       __catch$?_Copy@?$basic_string@DU?$char_traits@D@std@@V?$allocator@D@2@@std@@QAEXII@Z$1 100000d3 f   DiamondSupport.obj
 0001:fffff0d3       __catch$?_Copy@?$basic_string@DU?$char_traits@D@std@@V?$allocator@D@2@@std@@QAEXII@Z$1 100000d3 f   DiamondBuildTask.obj
 0001:fffff0d3       __catch$?_Copy@?$basic_string@DU?$char_traits@D@std@@V?$allocator@D@2@@std@@QAEXII@Z$1 100000d3 f   DiamondClassifyWorkerFactory.obj
 0001:fffff0d3       __catch$?_Copy@?$basic_string@DU?$char_traits@D@std@@V?$allocator@D@2@@std@@QAEXII@Z$1 100000d3 f   DiamondBuildWorkerFactory.obj
 0001:fffff0d3       __catch$?_Copy@?$basic_string@DU?$char_traits@D@std@@V?$allocator@D@2@@std@@QAEXII@Z$1 100000d3 f   moc_DiamondClassifyTask.obj
 0001:fffff0d3       __catch$?_Copy@?$basic_string@DU?$char_traits@D@std@@V?$allocator@D@2@@std@@QAEXII@Z$1 100000d3 f   moc_DiamondBuildPrompter.obj
 0001:fffff0ef       __catch$?detach_helper_grow@?$QList@VDescriptor@U2@@@@AAEPAUNode@1@HH@Z$2 100000ef f   DiamondClassifyWorker.obj
 0001:fffff0f1       __catch$?detach_helper_grow@?$QList@PAVAttribute@U2@@@@AAEPAUNode@1@HH@Z$2 100000f1 f   DiamondClassifyWorkerFactory.obj
 0001:fffff0f1       __catch$?detach_helper_grow@?$QList@PAVPortDescriptor@Workflow@U2@@@@AAEPAUNode@1@HH@Z$0 100000f1 f   DiamondClassifyWorkerFactory.obj
 0001:fffff0f1       __catch$?detach_helper_grow@?$QList@PAVAttribute@U2@@@@AAEPAUNode@1@HH@Z$0 100000f1 f   DiamondClassifyWorkerFactory.obj
 0001:fffff0f1       __catch$?detach_helper_grow@?$QList@PAVPortDescriptor@Workflow@U2@@@@AAEPAUNode@1@HH@Z$2 100000f1 f   DiamondClassifyWorkerFactory.obj
 0001:fffff11e       __catch$?detach_helper_grow@?$QList@VQString@@@@AAEPAUNode@1@HH@Z$2 1000011e f   DiamondBuildWorker.obj
 0001:fffff11e       __catch$?detach_helper_grow@?$QList@VQString@@@@AAEPAUNode@1@HH@Z$2 1000011e f   DiamondBuildWorkerFactory.obj
 0001:fffff11e       __catch$?detach_helper_grow@?$QList@VQString@@@@AAEPAUNode@1@HH@Z$2 1000011e f   DiamondSupport.obj
 0001:fffff11e       __catch$?detach_helper_grow@?$QList@VQString@@@@AAEPAUNode@1@HH@Z$2 1000011e f   DiamondClassifyTask.obj
 0001:fffff11e       __catch$?detach_helper_grow@?$QList@VQString@@@@AAEPAUNode@1@HH@Z$2 1000011e f   DiamondClassifyWorker.obj
 0001:fffff12a       __catch$?detach_helper_grow@?$QList@VDescriptor@U2@@@@AAEPAUNode@1@HH@Z$0 1000012a f   DiamondClassifyWorker.obj
 0001:fffff159       __catch$?detach_helper_grow@?$QList@VQString@@@@AAEPAUNode@1@HH@Z$0 10000159 f   DiamondBuildWorker.obj
 0001:fffff159       __catch$?detach_helper_grow@?$QList@VQString@@@@AAEPAUNode@1@HH@Z$0 10000159 f   DiamondClassifyWorker.obj
 0001:fffff159       __catch$?detach_helper_grow@?$QList@VQString@@@@AAEPAUNode@1@HH@Z$0 10000159 f   DiamondBuildWorkerFactory.obj
 0001:fffff159       __catch$?detach_helper_grow@?$QList@VQString@@@@AAEPAUNode@1@HH@Z$0 10000159 f   DiamondSupport.obj
 0001:fffff159       __catch$?detach_helper_grow@?$QList@VQString@@@@AAEPAUNode@1@HH@Z$0 10000159 f   DiamondClassifyTask.obj
 0001:00000000       ??__E?_Generic_object@?$_Error_objects@H@std@@2V_Generic_error_category@2@A@@YAXXZ 10001000 f   DiamondBuildPrompter.obj
 0001:00000010       ??__E?_Iostream_object@?$_Error_objects@H@std@@2V_Iostream_error_category@2@A@@YAXXZ 10001010 f   DiamondBuildPrompter.obj
 0001:00000020       ??__E?_System_object@?$_Error_objects@H@std@@2V_System_error_category@2@A@@YAXXZ 10001020 f   DiamondBuildPrompter.obj
 0001:00000030       ??__EalgoLog@U2@@YAXXZ     10001030 f   DiamondBuildPrompter.obj
 0001:000000b0       ??__EcmdLog@U2@@YAXXZ      100010b0 f   DiamondBuildPrompter.obj
 0001:00000130       ??__EcoreLog@U2@@YAXXZ     10001130 f   DiamondBuildPrompter.obj
 0001:000001b0       ??__EioLog@U2@@YAXXZ       100011b0 f   DiamondBuildPrompter.obj
 0001:00000230       ??__EperfLog@U2@@YAXXZ     10001230 f   DiamondBuildPrompter.obj
 0001:000002b0       ??__EscriptLog@U2@@YAXXZ   100012b0 f   DiamondBuildPrompter.obj
 0001:00000330       ??__EtaskLog@U2@@YAXXZ     10001330 f   DiamondBuildPrompter.obj
 0001:000003b0       ??__EuiLog@U2@@YAXXZ       100013b0 f   DiamondBuildPrompter.obj
 0001:00000430       ??__EuserActLog@U2@@YAXXZ  10001430 f   DiamondBuildPrompter.obj
 0001:000004b0       ??__E?_Generic_object@?$_Error_objects@H@std@@2V_Generic_error_category@2@A@@YAXXZ 100014b0 f   DiamondBuildTask.obj
 0001:000004c0       ??__E?_Iostream_object@?$_Error_objects@H@std@@2V_Iostream_error_category@2@A@@YAXXZ 100014c0 f   DiamondBuildTask.obj
 0001:000004d0       ??__E?_System_object@?$_Error_objects@H@std@@2V_System_error_category@2@A@@YAXXZ 100014d0 f   DiamondBuildTask.obj
 0001:000004e0       ??__EalgoLog@U2@@YAXXZ     100014e0 f   DiamondBuildTask.obj
 0001:00000560       ??__EcmdLog@U2@@YAXXZ      10001560 f   DiamondBuildTask.obj
 0001:000005e0       ??__EcoreLog@U2@@YAXXZ     100015e0 f   DiamondBuildTask.obj
 0001:00000660       ??__EioLog@U2@@YAXXZ       10001660 f   DiamondBuildTask.obj
 0001:000006e0       ??__EperfLog@U2@@YAXXZ     100016e0 f   DiamondBuildTask.obj
 0001:00000760       ??__EscriptLog@U2@@YAXXZ   10001760 f   DiamondBuildTask.obj
 0001:000007e0       ??__EtaskLog@U2@@YAXXZ     100017e0 f   DiamondBuildTask.obj
 0001:00000860       ??__EuiLog@U2@@YAXXZ       10001860 f   DiamondBuildTask.obj
 0001:000008e0       ??__EuserActLog@U2@@YAXXZ  100018e0 f   DiamondBuildTask.obj
 0001:00000960       ??__E?_Generic_object@?$_Error_objects@H@std@@2V_Generic_error_category@2@A@@YAXXZ 10001960 f   DiamondBuildValidator.obj
 0001:00000970       ??__E?_Iostream_object@?$_Error_objects@H@std@@2V_Iostream_error_category@2@A@@YAXXZ 10001970 f   DiamondBuildValidator.obj
 0001:00000980       ??__E?_System_object@?$_Error_objects@H@std@@2V_System_error_category@2@A@@YAXXZ 10001980 f   DiamondBuildValidator.obj
 0001:00000990       ??__EalgoLog@U2@@YAXXZ     10001990 f   DiamondBuildValidator.obj
 0001:00000a10       ??__EcmdLog@U2@@YAXXZ      10001a10 f   DiamondBuildValidator.obj
 0001:00000a90       ??__EcoreLog@U2@@YAXXZ     10001a90 f   DiamondBuildValidator.obj
 0001:00000b10       ??__EioLog@U2@@YAXXZ       10001b10 f   DiamondBuildValidator.obj
 0001:00000b90       ??__EperfLog@U2@@YAXXZ     10001b90 f   DiamondBuildValidator.obj
 0001:00000c10       ??__EscriptLog@U2@@YAXXZ   10001c10 f   DiamondBuildValidator.obj
 0001:00000c90       ??__EtaskLog@U2@@YAXXZ     10001c90 f   DiamondBuildValidator.obj
 0001:00000d10       ??__EuiLog@U2@@YAXXZ       10001d10 f   DiamondBuildValidator.obj
 0001:00000d90       ??__EuserActLog@U2@@YAXXZ  10001d90 f   DiamondBuildValidator.obj
 0001:00000e10       ??__E?DIAMOND_BUILD_DIR@DiamondBuildWorker@LocalWorkflow@U2@@0VQString@@B@@YAXXZ 10001e10 f   DiamondBuildWorker.obj
 0001:00000e30       ??__E?_Generic_object@?$_Error_objects@H@std@@2V_Generic_error_category@2@A@@YAXXZ 10001e30 f   DiamondBuildWorker.obj
 0001:00000e40       ??__E?_Iostream_object@?$_Error_objects@H@std@@2V_Iostream_error_category@2@A@@YAXXZ 10001e40 f   DiamondBuildWorker.obj
 0001:00000e50       ??__E?_System_object@?$_Error_objects@H@std@@2V_System_error_category@2@A@@YAXXZ 10001e50 f   DiamondBuildWorker.obj
 0001:00000e60       ??__EalgoLog@U2@@YAXXZ     10001e60 f   DiamondBuildWorker.obj
 0001:00000ee0       ??__EcmdLog@U2@@YAXXZ      10001ee0 f   DiamondBuildWorker.obj
 0001:00000f60       ??__EcoreLog@U2@@YAXXZ     10001f60 f   DiamondBuildWorker.obj
 0001:00000fe0       ??__EioLog@U2@@YAXXZ       10001fe0 f   DiamondBuildWorker.obj
 0001:00001060       ??__EperfLog@U2@@YAXXZ     10002060 f   DiamondBuildWorker.obj
 0001:000010e0       ??__EscriptLog@U2@@YAXXZ   100020e0 f   DiamondBuildWorker.obj
 0001:00001160       ??__EtaskLog@U2@@YAXXZ     10002160 f   DiamondBuildWorker.obj
 0001:000011e0       ??__EuiLog@U2@@YAXXZ       100021e0 f   DiamondBuildWorker.obj
 0001:00001260       ??__EuserActLog@U2@@YAXXZ  10002260 f   DiamondBuildWorker.obj
 0001:000012e0       ??__E?ACTOR_ID@DiamondBuildWorkerFactory@LocalWorkflow@U2@@2VQString@@B@@YAXXZ 100022e0 f   DiamondBuildWorkerFactory.obj
 0001:00001300       ??__E?DATABASE_ATTR_ID@DiamondBuildWorkerFactory@LocalWorkflow@U2@@2VQString@@B@@YAXXZ 10002300 f   DiamondBuildWorkerFactory.obj
 0001:00001320       ??__E?GENOMIC_LIBRARY_ATTR_ID@DiamondBuildWorkerFactory@LocalWorkflow@U2@@2VQString@@B@@YAXXZ 10002320 f   DiamondBuildWorkerFactory.obj
 0001:00001340       ??__E?OUTPUT_PORT_ID@DiamondBuildWorkerFactory@LocalWorkflow@U2@@2VQString@@B@@YAXXZ 10002340 f   DiamondBuildWorkerFactory.obj
 0001:00001360       ??__E?_Generic_object@?$_Error_objects@H@std@@2V_Generic_error_category@2@A@@YAXXZ 10002360 f   DiamondBuildWorkerFactory.obj
 0001:00001370       ??__E?_Iostream_object@?$_Error_objects@H@std@@2V_Iostream_error_category@2@A@@YAXXZ 10002370 f   DiamondBuildWorkerFactory.obj
 0001:00001380       ??__E?_System_object@?$_Error_objects@H@std@@2V_System_error_category@2@A@@YAXXZ 10002380 f   DiamondBuildWorkerFactory.obj
 0001:00001390       ??__EalgoLog@U2@@YAXXZ     10002390 f   DiamondBuildWorkerFactory.obj
 0001:00001410       ??__EcmdLog@U2@@YAXXZ      10002410 f   DiamondBuildWorkerFactory.obj
 0001:00001490       ??__EcoreLog@U2@@YAXXZ     10002490 f   DiamondBuildWorkerFactory.obj
 0001:00001510       ??__EioLog@U2@@YAXXZ       10002510 f   DiamondBuildWorkerFactory.obj
 0001:00001590       ??__EperfLog@U2@@YAXXZ     10002590 f   DiamondBuildWorkerFactory.obj
 0001:00001610       ??__EscriptLog@U2@@YAXXZ   10002610 f   DiamondBuildWorkerFactory.obj
 0001:00001690       ??__EtaskLog@U2@@YAXXZ     10002690 f   DiamondBuildWorkerFactory.obj
 0001:00001710       ??__EuiLog@U2@@YAXXZ       10002710 f   DiamondBuildWorkerFactory.obj
 0001:00001790       ??__EuserActLog@U2@@YAXXZ  10002790 f   DiamondBuildWorkerFactory.obj
 0001:00001810       ??__E?_Generic_object@?$_Error_objects@H@std@@2V_Generic_error_category@2@A@@YAXXZ 10002810 f   DiamondClassifyPrompter.obj
 0001:00001820       ??__E?_Iostream_object@?$_Error_objects@H@std@@2V_Iostream_error_category@2@A@@YAXXZ 10002820 f   DiamondClassifyPrompter.obj
 0001:00001830       ??__E?_System_object@?$_Error_objects@H@std@@2V_System_error_category@2@A@@YAXXZ 10002830 f   DiamondClassifyPrompter.obj
 0001:00001840       ??__EalgoLog@U2@@YAXXZ     10002840 f   DiamondClassifyPrompter.obj
 0001:000018c0       ??__EcmdLog@U2@@YAXXZ      100028c0 f   DiamondClassifyPrompter.obj
 0001:00001940       ??__EcoreLog@U2@@YAXXZ     10002940 f   DiamondClassifyPrompter.obj
 0001:000019c0       ??__EioLog@U2@@YAXXZ       100029c0 f   DiamondClassifyPrompter.obj
 0001:00001a40       ??__EperfLog@U2@@YAXXZ     10002a40 f   DiamondClassifyPrompter.obj
 0001:00001ac0       ??__EscriptLog@U2@@YAXXZ   10002ac0 f   DiamondClassifyPrompter.obj
 0001:00001b40       ??__EtaskLog@U2@@YAXXZ     10002b40 f   DiamondClassifyPrompter.obj
 0001:00001bc0       ??__EuiLog@U2@@YAXXZ       10002bc0 f   DiamondClassifyPrompter.obj
 0001:00001c40       ??__EuserActLog@U2@@YAXXZ  10002c40 f   DiamondClassifyPrompter.obj
 0001:00001cc0       ??__E?BLOSUM45@DiamondClassifyTaskSettings@U2@@2VQString@@B@@YAXXZ 10002cc0 f   DiamondClassifyTask.obj
 0001:00001ce0       ??__E?BLOSUM50@DiamondClassifyTaskSettings@U2@@2VQString@@B@@YAXXZ 10002ce0 f   DiamondClassifyTask.obj
 0001:00001d00       ??__E?BLOSUM62@DiamondClassifyTaskSettings@U2@@2VQString@@B@@YAXXZ 10002d00 f   DiamondClassifyTask.obj
 0001:00001d20       ??__E?BLOSUM80@DiamondClassifyTaskSettings@U2@@2VQString@@B@@YAXXZ 10002d20 f   DiamondClassifyTask.obj
 0001:00001d40       ??__E?BLOSUM90@DiamondClassifyTaskSettings@U2@@2VQString@@B@@YAXXZ 10002d40 f   DiamondClassifyTask.obj
 0001:00001d60       ??__E?PAM250@DiamondClassifyTaskSettings@U2@@2VQString@@B@@YAXXZ 10002d60 f   DiamondClassifyTask.obj
 0001:00001d80       ??__E?PAM30@DiamondClassifyTaskSettings@U2@@2VQString@@B@@YAXXZ 10002d80 f   DiamondClassifyTask.obj
 0001:00001da0       ??__E?PAM70@DiamondClassifyTaskSettings@U2@@2VQString@@B@@YAXXZ 10002da0 f   DiamondClassifyTask.obj
 0001:00001dc0       ??__E?SENSITIVE_DEFAULT@DiamondClassifyTaskSettings@U2@@2VQString@@B@@YAXXZ 10002dc0 f   DiamondClassifyTask.obj
 0001:00001de0       ??__E?SENSITIVE_HIGH@DiamondClassifyTaskSettings@U2@@2VQString@@B@@YAXXZ 10002de0 f   DiamondClassifyTask.obj
 0001:00001e00       ??__E?SENSITIVE_ULTRA@DiamondClassifyTaskSettings@U2@@2VQString@@B@@YAXXZ 10002e00 f   DiamondClassifyTask.obj
 0001:00001e20       ??__E?TAXONOMIC_CLASSIFICATION_OUTPUT_FORMAT@DiamondClassifyTask@U2@@0VQString@@B@@YAXXZ 10002e20 f   DiamondClassifyTask.obj
 0001:00001e40       ??__E?_Generic_object@?$_Error_objects@H@std@@2V_Generic_error_category@2@A@@YAXXZ 10002e40 f   DiamondClassifyTask.obj
 0001:00001e50       ??__E?_Iostream_object@?$_Error_objects@H@std@@2V_Iostream_error_category@2@A@@YAXXZ 10002e50 f   DiamondClassifyTask.obj
 0001:00001e60       ??__E?_System_object@?$_Error_objects@H@std@@2V_System_error_category@2@A@@YAXXZ 10002e60 f   DiamondClassifyTask.obj
 0001:00001e70       ??__EalgoLog@U2@@YAXXZ     10002e70 f   DiamondClassifyTask.obj
 0001:00001ef0       ??__EcmdLog@U2@@YAXXZ      10002ef0 f   DiamondClassifyTask.obj
 0001:00001f70       ??__EcoreLog@U2@@YAXXZ     10002f70 f   DiamondClassifyTask.obj
 0001:00001ff0       ??__EioLog@U2@@YAXXZ       10002ff0 f   DiamondClassifyTask.obj
 0001:00002070       ??__EperfLog@U2@@YAXXZ     10003070 f   DiamondClassifyTask.obj
 0001:000020f0       ??__EscriptLog@U2@@YAXXZ   100030f0 f   DiamondClassifyTask.obj
 0001:00002170       ??__EtaskLog@U2@@YAXXZ     10003170 f   DiamondClassifyTask.obj
 0001:000021f0       ??__EuiLog@U2@@YAXXZ       100031f0 f   DiamondClassifyTask.obj
 0001:00002270       ??__EuserActLog@U2@@YAXXZ  10003270 f   DiamondClassifyTask.obj
 0001:000022f0       ??__E?DIAMOND_DIR@DiamondClassifyWorker@LocalWorkflow@U2@@0VQString@@B@@YAXXZ 100032f0 f   DiamondClassifyWorker.obj
 0001:00002310       ??__E?_Generic_object@?$_Error_objects@H@std@@2V_Generic_error_category@2@A@@YAXXZ 10003310 f   DiamondClassifyWorker.obj
 0001:00002320       ??__E?_Iostream_object@?$_Error_objects@H@std@@2V_Iostream_error_category@2@A@@YAXXZ 10003320 f   DiamondClassifyWorker.obj
 0001:00002330       ??__E?_System_object@?$_Error_objects@H@std@@2V_System_error_category@2@A@@YAXXZ 10003330 f   DiamondClassifyWorker.obj
 0001:00002340       ??__EalgoLog@U2@@YAXXZ     10003340 f   DiamondClassifyWorker.obj
 0001:000023c0       ??__EcmdLog@U2@@YAXXZ      100033c0 f   DiamondClassifyWorker.obj
 0001:00002440       ??__EcoreLog@U2@@YAXXZ     10003440 f   DiamondClassifyWorker.obj
 0001:000024c0       ??__EioLog@U2@@YAXXZ       100034c0 f   DiamondClassifyWorker.obj
 0001:00002540       ??__EperfLog@U2@@YAXXZ     10003540 f   DiamondClassifyWorker.obj
 0001:000025c0       ??__EscriptLog@U2@@YAXXZ   100035c0 f   DiamondClassifyWorker.obj
 0001:00002640       ??__EtaskLog@U2@@YAXXZ     10003640 f   DiamondClassifyWorker.obj
 0001:000026c0       ??__EuiLog@U2@@YAXXZ       100036c0 f   DiamondClassifyWorker.obj
 0001:00002740       ??__EuserActLog@U2@@YAXXZ  10003740 f   DiamondClassifyWorker.obj
 0001:000027c0       ??__E?ACTOR_ID@DiamondClassifyWorkerFactory@LocalWorkflow@U2@@2VQString@@B@@YAXXZ 100037c0 f   DiamondClassifyWorkerFactory.obj
 0001:000027e0       ??__E?BSIZE_ATTR_ID@DiamondClassifyWorkerFactory@LocalWorkflow@U2@@2VQString@@B@@YAXXZ 100037e0 f   DiamondClassifyWorkerFactory.obj
 0001:00002800       ??__E?CHUNKS_ATTR_ID@DiamondClassifyWorkerFactory@LocalWorkflow@U2@@2VQString@@B@@YAXXZ 10003800 f   DiamondClassifyWorkerFactory.obj
 0001:00002820       ??__E?DATABASE_ATTR_ID@DiamondClassifyWorkerFactory@LocalWorkflow@U2@@2VQString@@B@@YAXXZ 10003820 f   DiamondClassifyWorkerFactory.obj
 0001:00002840       ??__E?EVALUE_ATTR_ID@DiamondClassifyWorkerFactory@LocalWorkflow@U2@@2VQString@@B@@YAXXZ 10003840 f   DiamondClassifyWorkerFactory.obj
 0001:00002860       ??__E?FSHIFT_ATTR_ID@DiamondClassifyWorkerFactory@LocalWorkflow@U2@@2VQString@@B@@YAXXZ 10003860 f   DiamondClassifyWorkerFactory.obj
 0001:00002880       ??__E?GENCODE_ATTR_ID@DiamondClassifyWorkerFactory@LocalWorkflow@U2@@2VQString@@B@@YAXXZ 10003880 f   DiamondClassifyWorkerFactory.obj
 0001:000028a0       ??__E?GE_PEN_ATTR_ID@DiamondClassifyWorkerFactory@LocalWorkflow@U2@@2VQString@@B@@YAXXZ 100038a0 f   DiamondClassifyWorkerFactory.obj
 0001:000028c0       ??__E?GO_PEN_ATTR_ID@DiamondClassifyWorkerFactory@LocalWorkflow@U2@@2VQString@@B@@YAXXZ 100038c0 f   DiamondClassifyWorkerFactory.obj
 0001:000028e0       ??__E?INPUT_DATA_ATTR_ID@DiamondClassifyWorkerFactory@LocalWorkflow@U2@@2VQString@@B@@YAXXZ 100038e0 f   DiamondClassifyWorkerFactory.obj
 0001:00002900       ??__E?INPUT_PORT_ID@DiamondClassifyWorkerFactory@LocalWorkflow@U2@@2VQString@@B@@YAXXZ 10003900 f   DiamondClassifyWorkerFactory.obj
 0001:00002920       ??__E?INPUT_SLOT@DiamondClassifyWorkerFactory@LocalWorkflow@U2@@2VQString@@B@@YAXXZ 10003920 f   DiamondClassifyWorkerFactory.obj
 0001:00002940       ??__E?MATRIX_ATTR_ID@DiamondClassifyWorkerFactory@LocalWorkflow@U2@@2VQString@@B@@YAXXZ 10003940 f   DiamondClassifyWorkerFactory.obj
 0001:00002960       ??__E?OUTPUT_PORT_ID@DiamondClassifyWorkerFactory@LocalWorkflow@U2@@2VQString@@B@@YAXXZ 10003960 f   DiamondClassifyWorkerFactory.obj
 0001:00002980       ??__E?OUTPUT_URL_ATTR_ID@DiamondClassifyWorkerFactory@LocalWorkflow@U2@@2VQString@@B@@YAXXZ 10003980 f   DiamondClassifyWorkerFactory.obj
 0001:000029a0       ??__E?SENSITIVE_ATTR_ID@DiamondClassifyWorkerFactory@LocalWorkflow@U2@@2VQString@@B@@YAXXZ 100039a0 f   DiamondClassifyWorkerFactory.obj
 0001:000029c0       ??__E?THREADS_ATTR_ID@DiamondClassifyWorkerFactory@LocalWorkflow@U2@@2VQString@@B@@YAXXZ 100039c0 f   DiamondClassifyWorkerFactory.obj
 0001:000029e0       ??__E?TOP_ALIGNMENTS_PERCENTAGE_ATTR_ID@DiamondClassifyWorkerFactory@LocalWorkflow@U2@@2VQString@@B@@YAXXZ 100039e0 f   DiamondClassifyWorkerFactory.obj
 0001:00002a00       ??__E?WORKFLOW_CLASSIFY_TOOL_DIAMOND@DiamondClassifyWorkerFactory@LocalWorkflow@U2@@2VQString@@B@@YAXXZ 10003a00 f   DiamondClassifyWorkerFactory.obj
 0001:00002a20       ??__E?_Generic_object@?$_Error_objects@H@std@@2V_Generic_error_category@2@A@@YAXXZ 10003a20 f   DiamondClassifyWorkerFactory.obj
 0001:00002a30       ??__E?_Iostream_object@?$_Error_objects@H@std@@2V_Iostream_error_category@2@A@@YAXXZ 10003a30 f   DiamondClassifyWorkerFactory.obj
 0001:00002a40       ??__E?_System_object@?$_Error_objects@H@std@@2V_System_error_category@2@A@@YAXXZ 10003a40 f   DiamondClassifyWorkerFactory.obj
 0001:00002a50       ??__EalgoLog@U2@@YAXXZ     10003a50 f   DiamondClassifyWorkerFactory.obj
 0001:00002ad0       ??__EcmdLog@U2@@YAXXZ      10003ad0 f   DiamondClassifyWorkerFactory.obj
 0001:00002b50       ??__EcoreLog@U2@@YAXXZ     10003b50 f   DiamondClassifyWorkerFactory.obj
 0001:00002bd0       ??__EioLog@U2@@YAXXZ       10003bd0 f   DiamondClassifyWorkerFactory.obj
 0001:00002c50       ??__EperfLog@U2@@YAXXZ     10003c50 f   DiamondClassifyWorkerFactory.obj
 0001:00002cd0       ??__EscriptLog@U2@@YAXXZ   10003cd0 f   DiamondClassifyWorkerFactory.obj
 0001:00002d50       ??__EtaskLog@U2@@YAXXZ     10003d50 f   DiamondClassifyWorkerFactory.obj
 0001:00002dd0       ??__EuiLog@U2@@YAXXZ       10003dd0 f   DiamondClassifyWorkerFactory.obj
 0001:00002e50       ??__EuserActLog@U2@@YAXXZ  10003e50 f   DiamondClassifyWorkerFactory.obj
 0001:00002ed0       ??__E?TOOL_NAME@DiamondSupport@U2@@2VQString@@B@@YAXXZ 10003ed0 f   DiamondSupport.obj
 0001:00002ef0       ??__E?_Generic_object@?$_Error_objects@H@std@@2V_Generic_error_category@2@A@@YAXXZ 10003ef0 f   DiamondSupport.obj
 0001:00002f00       ??__E?_Iostream_object@?$_Error_objects@H@std@@2V_Iostream_error_category@2@A@@YAXXZ 10003f00 f   DiamondSupport.obj
 0001:00002f10       ??__E?_System_object@?$_Error_objects@H@std@@2V_System_error_category@2@A@@YAXXZ 10003f10 f   DiamondSupport.obj
 0001:00002f20       ??__E?PLUGIN_DESCRIPRION@DiamondSupportPlugin@U2@@2VQString@@B@@YAXXZ 10003f20 f   DiamondSupportPlugin.obj
 0001:00002f50       ??__E?PLUGIN_NAME@DiamondSupportPlugin@U2@@2VQString@@B@@YAXXZ 10003f50 f   DiamondSupportPlugin.obj
 0001:00002f80       ??__E?_Generic_object@?$_Error_objects@H@std@@2V_Generic_error_category@2@A@@YAXXZ 10003f80 f   DiamondSupportPlugin.obj
 0001:00002f90       ??__E?_Iostream_object@?$_Error_objects@H@std@@2V_Iostream_error_category@2@A@@YAXXZ 10003f90 f   DiamondSupportPlugin.obj
 0001:00002fa0       ??__E?_System_object@?$_Error_objects@H@std@@2V_System_error_category@2@A@@YAXXZ 10003fa0 f   DiamondSupportPlugin.obj
 0001:00002fb0       ??__EalgoLog@U2@@YAXXZ     10003fb0 f   DiamondSupportPlugin.obj
 0001:00003030       ??__EcmdLog@U2@@YAXXZ      10004030 f   DiamondSupportPlugin.obj
 0001:000030b0       ??__EcoreLog@U2@@YAXXZ     100040b0 f   DiamondSupportPlugin.obj
 0001:00003130       ??__EioLog@U2@@YAXXZ       10004130 f   DiamondSupportPlugin.obj
 0001:000031b0       ??__EperfLog@U2@@YAXXZ     100041b0 f   DiamondSupportPlugin.obj
 0001:00003230       ??__EscriptLog@U2@@YAXXZ   10004230 f   DiamondSupportPlugin.obj
 0001:000032b0       ??__EtaskLog@U2@@YAXXZ     100042b0 f   DiamondSupportPlugin.obj
 0001:00003330       ??__EuiLog@U2@@YAXXZ       10004330 f   DiamondSupportPlugin.obj
 0001:000033b0       ??__EuserActLog@U2@@YAXXZ  100043b0 f   DiamondSupportPlugin.obj
 0001:00003430       ??__E?_Generic_object@?$_Error_objects@H@std@@2V_Generic_error_category@2@A@@YAXXZ 10004430 f   GenomesPreparationTask.obj
 0001:00003440       ??__E?_Iostream_object@?$_Error_objects@H@std@@2V_Iostream_error_category@2@A@@YAXXZ 10004440 f   GenomesPreparationTask.obj
 0001:00003450       ??__E?_System_object@?$_Error_objects@H@std@@2V_System_error_category@2@A@@YAXXZ 10004450 f   GenomesPreparationTask.obj
 0001:00003460       ??__EalgoLog@U2@@YAXXZ     10004460 f   GenomesPreparationTask.obj
 0001:000034e0       ??__EcmdLog@U2@@YAXXZ      100044e0 f   GenomesPreparationTask.obj
 0001:00003560       ??__EcoreLog@U2@@YAXXZ     10004560 f   GenomesPreparationTask.obj
 0001:000035e0       ??__EioLog@U2@@YAXXZ       100045e0 f   GenomesPreparationTask.obj
 0001:00003660       ??__EperfLog@U2@@YAXXZ     10004660 f   GenomesPreparationTask.obj
 0001:000036e0       ??__EscriptLog@U2@@YAXXZ   100046e0 f   GenomesPreparationTask.obj
 0001:00003760       ??__EtaskLog@U2@@YAXXZ     10004760 f   GenomesPreparationTask.obj
 0001:000037e0       ??__EuiLog@U2@@YAXXZ       100047e0 f   GenomesPreparationTask.obj
 0001:00003860       ??__EuserActLog@U2@@YAXXZ  10004860 f   GenomesPreparationTask.obj
 0001:000038e0       ??__E?_Generic_object@?$_Error_objects@H@std@@2V_Generic_error_category@2@A@@YAXXZ 100048e0 f   moc_DiamondBuildPrompter.obj
 0001:000038f0       ??__E?_Iostream_object@?$_Error_objects@H@std@@2V_Iostream_error_category@2@A@@YAXXZ 100048f0 f   moc_DiamondBuildPrompter.obj
 0001:00003900       ??__E?_System_object@?$_Error_objects@H@std@@2V_System_error_category@2@A@@YAXXZ 10004900 f   moc_DiamondBuildPrompter.obj
 0001:00003910       ??__E?staticMetaObject@DiamondBuildPrompter@LocalWorkflow@U2@@2UQMetaObject@@B@@YAXXZ 10004910 f   moc_DiamondBuildPrompter.obj
 0001:00003920       ??__EalgoLog@U2@@YAXXZ     10004920 f   moc_DiamondBuildPrompter.obj
 0001:000039a0       ??__EcmdLog@U2@@YAXXZ      100049a0 f   moc_DiamondBuildPrompter.obj
 0001:00003a20       ??__EcoreLog@U2@@YAXXZ     10004a20 f   moc_DiamondBuildPrompter.obj
 0001:00003aa0       ??__EioLog@U2@@YAXXZ       10004aa0 f   moc_DiamondBuildPrompter.obj
 0001:00003b20       ??__EperfLog@U2@@YAXXZ     10004b20 f   moc_DiamondBuildPrompter.obj
 0001:00003ba0       ??__EscriptLog@U2@@YAXXZ   10004ba0 f   moc_DiamondBuildPrompter.obj
 0001:00003c20       ??__EtaskLog@U2@@YAXXZ     10004c20 f   moc_DiamondBuildPrompter.obj
 0001:00003ca0       ??__EuiLog@U2@@YAXXZ       10004ca0 f   moc_DiamondBuildPrompter.obj
 0001:00003d20       ??__EuserActLog@U2@@YAXXZ  10004d20 f   moc_DiamondBuildPrompter.obj
 0001:00003da0       ??__E?_Generic_object@?$_Error_objects@H@std@@2V_Generic_error_category@2@A@@YAXXZ 10004da0 f   moc_DiamondBuildTask.obj
 0001:00003db0       ??__E?_Iostream_object@?$_Error_objects@H@std@@2V_Iostream_error_category@2@A@@YAXXZ 10004db0 f   moc_DiamondBuildTask.obj
 0001:00003dc0       ??__E?_System_object@?$_Error_objects@H@std@@2V_System_error_category@2@A@@YAXXZ 10004dc0 f   moc_DiamondBuildTask.obj
 0001:00003dd0       ??__E?staticMetaObject@DiamondBuildTask@U2@@2UQMetaObject@@B@@YAXXZ 10004dd0 f   moc_DiamondBuildTask.obj
 0001:00003de0       ??__EalgoLog@U2@@YAXXZ     10004de0 f   moc_DiamondBuildTask.obj
 0001:00003e60       ??__EcmdLog@U2@@YAXXZ      10004e60 f   moc_DiamondBuildTask.obj
 0001:00003ee0       ??__EcoreLog@U2@@YAXXZ     10004ee0 f   moc_DiamondBuildTask.obj
 0001:00003f60       ??__EioLog@U2@@YAXXZ       10004f60 f   moc_DiamondBuildTask.obj
 0001:00003fe0       ??__EperfLog@U2@@YAXXZ     10004fe0 f   moc_DiamondBuildTask.obj
 0001:00004060       ??__EscriptLog@U2@@YAXXZ   10005060 f   moc_DiamondBuildTask.obj
 0001:000040e0       ??__EtaskLog@U2@@YAXXZ     100050e0 f   moc_DiamondBuildTask.obj
 0001:00004160       ??__EuiLog@U2@@YAXXZ       10005160 f   moc_DiamondBuildTask.obj
 0001:000041e0       ??__EuserActLog@U2@@YAXXZ  100051e0 f   moc_DiamondBuildTask.obj
 0001:00004260       ??__E?_Generic_object@?$_Error_objects@H@std@@2V_Generic_error_category@2@A@@YAXXZ 10005260 f   moc_DiamondBuildWorker.obj
 0001:00004270       ??__E?_Iostream_object@?$_Error_objects@H@std@@2V_Iostream_error_category@2@A@@YAXXZ 10005270 f   moc_DiamondBuildWorker.obj
 0001:00004280       ??__E?_System_object@?$_Error_objects@H@std@@2V_System_error_category@2@A@@YAXXZ 10005280 f   moc_DiamondBuildWorker.obj
 0001:00004290       ??__E?staticMetaObject@DiamondBuildWorker@LocalWorkflow@U2@@2UQMetaObject@@B@@YAXXZ 10005290 f   moc_DiamondBuildWorker.obj
 0001:000042a0       ??__EalgoLog@U2@@YAXXZ     100052a0 f   moc_DiamondBuildWorker.obj
 0001:00004320       ??__EcmdLog@U2@@YAXXZ      10005320 f   moc_DiamondBuildWorker.obj
 0001:000043a0       ??__EcoreLog@U2@@YAXXZ     100053a0 f   moc_DiamondBuildWorker.obj
 0001:00004420       ??__EioLog@U2@@YAXXZ       10005420 f   moc_DiamondBuildWorker.obj
 0001:000044a0       ??__EperfLog@U2@@YAXXZ     100054a0 f   moc_DiamondBuildWorker.obj
 0001:00004520       ??__EscriptLog@U2@@YAXXZ   10005520 f   moc_DiamondBuildWorker.obj
 0001:000045a0       ??__EtaskLog@U2@@YAXXZ     100055a0 f   moc_DiamondBuildWorker.obj
 0001:00004620       ??__EuiLog@U2@@YAXXZ       10005620 f   moc_DiamondBuildWorker.obj
 0001:000046a0       ??__EuserActLog@U2@@YAXXZ  100056a0 f   moc_DiamondBuildWorker.obj
 0001:00004720       ??__E?_Generic_object@?$_Error_objects@H@std@@2V_Generic_error_category@2@A@@YAXXZ 10005720 f   moc_DiamondClassifyPrompter.obj
 0001:00004730       ??__E?_Iostream_object@?$_Error_objects@H@std@@2V_Iostream_error_category@2@A@@YAXXZ 10005730 f   moc_DiamondClassifyPrompter.obj
 0001:00004740       ??__E?_System_object@?$_Error_objects@H@std@@2V_System_error_category@2@A@@YAXXZ 10005740 f   moc_DiamondClassifyPrompter.obj
 0001:00004750       ??__E?staticMetaObject@DiamondClassifyPrompter@LocalWorkflow@U2@@2UQMetaObject@@B@@YAXXZ 10005750 f   moc_DiamondClassifyPrompter.obj
 0001:00004760       ??__EalgoLog@U2@@YAXXZ     10005760 f   moc_DiamondClassifyPrompter.obj
 0001:000047e0       ??__EcmdLog@U2@@YAXXZ      100057e0 f   moc_DiamondClassifyPrompter.obj
 0001:00004860       ??__EcoreLog@U2@@YAXXZ     10005860 f   moc_DiamondClassifyPrompter.obj
 0001:000048e0       ??__EioLog@U2@@YAXXZ       100058e0 f   moc_DiamondClassifyPrompter.obj
 0001:00004960       ??__EperfLog@U2@@YAXXZ     10005960 f   moc_DiamondClassifyPrompter.obj
 0001:000049e0       ??__EscriptLog@U2@@YAXXZ   100059e0 f   moc_DiamondClassifyPrompter.obj
 0001:00004a60       ??__EtaskLog@U2@@YAXXZ     10005a60 f   moc_DiamondClassifyPrompter.obj
 0001:00004ae0       ??__EuiLog@U2@@YAXXZ       10005ae0 f   moc_DiamondClassifyPrompter.obj
 0001:00004b60       ??__EuserActLog@U2@@YAXXZ  10005b60 f   moc_DiamondClassifyPrompter.obj
 0001:00004be0       ??__E?_Generic_object@?$_Error_objects@H@std@@2V_Generic_error_category@2@A@@YAXXZ 10005be0 f   moc_DiamondClassifyTask.obj
 0001:00004bf0       ??__E?_Iostream_object@?$_Error_objects@H@std@@2V_Iostream_error_category@2@A@@YAXXZ 10005bf0 f   moc_DiamondClassifyTask.obj
 0001:00004c00       ??__E?_System_object@?$_Error_objects@H@std@@2V_System_error_category@2@A@@YAXXZ 10005c00 f   moc_DiamondClassifyTask.obj
 0001:00004c10       ??__E?staticMetaObject@DiamondClassifyTask@U2@@2UQMetaObject@@B@@YAXXZ 10005c10 f   moc_DiamondClassifyTask.obj
 0001:00004c20       ??__EalgoLog@U2@@YAXXZ     10005c20 f   moc_DiamondClassifyTask.obj
 0001:00004ca0       ??__EcmdLog@U2@@YAXXZ      10005ca0 f   moc_DiamondClassifyTask.obj
 0001:00004d20       ??__EcoreLog@U2@@YAXXZ     10005d20 f   moc_DiamondClassifyTask.obj
 0001:00004da0       ??__EioLog@U2@@YAXXZ       10005da0 f   moc_DiamondClassifyTask.obj
 0001:00004e20       ??__EperfLog@U2@@YAXXZ     10005e20 f   moc_DiamondClassifyTask.obj
 0001:00004ea0       ??__EscriptLog@U2@@YAXXZ   10005ea0 f   moc_DiamondClassifyTask.obj
 0001:00004f20       ??__EtaskLog@U2@@YAXXZ     10005f20 f   moc_DiamondClassifyTask.obj
 0001:00004fb0       ??__EuiLog@U2@@YAXXZ       10005fb0 f   moc_DiamondClassifyTask.obj
 0001:00005030       ??__EuserActLog@U2@@YAXXZ  10006030 f   moc_DiamondClassifyTask.obj
 0001:000050b0       ??__E?_Generic_object@?$_Error_objects@H@std@@2V_Generic_error_category@2@A@@YAXXZ 100060b0 f   moc_DiamondClassifyWorker.obj
 0001:000050c0       ??__E?_Iostream_object@?$_Error_objects@H@std@@2V_Iostream_error_category@2@A@@YAXXZ 100060c0 f   moc_DiamondClassifyWorker.obj
 0001:000050d0       ??__E?_System_object@?$_Error_objects@H@std@@2V_System_error_category@2@A@@YAXXZ 100060d0 f   moc_DiamondClassifyWorker.obj
 0001:000050e0       ??__E?staticMetaObject@DiamondClassifyWorker@LocalWorkflow@U2@@2UQMetaObject@@B@@YAXXZ 100060e0 f   moc_DiamondClassifyWorker.obj
 0001:000050f0       ??__EalgoLog@U2@@YAXXZ     100060f0 f   moc_DiamondClassifyWorker.obj
 0001:00005170       ??__EcmdLog@U2@@YAXXZ      10006170 f   moc_DiamondClassifyWorker.obj
 0001:000051f0       ??__EcoreLog@U2@@YAXXZ     100061f0 f   moc_DiamondClassifyWorker.obj
 0001:00005270       ??__EioLog@U2@@YAXXZ       10006270 f   moc_DiamondClassifyWorker.obj
 0001:000052f0       ??__EperfLog@U2@@YAXXZ     100062f0 f   moc_DiamondClassifyWorker.obj
 0001:00005370       ??__EscriptLog@U2@@YAXXZ   10006370 f   moc_DiamondClassifyWorker.obj
 0001:000053f0       ??__EtaskLog@U2@@YAXXZ     100063f0 f   moc_DiamondClassifyWorker.obj
 0001:00005470       ??__EuiLog@U2@@YAXXZ       10006470 f   moc_DiamondClassifyWorker.obj
 0001:000054f0       ??__EuserActLog@U2@@YAXXZ  100064f0 f   moc_DiamondClassifyWorker.obj
 0001:00005570       ??__E?_Generic_object@?$_Error_objects@H@std@@2V_Generic_error_category@2@A@@YAXXZ 10006570 f   moc_DiamondSupport.obj
 0001:00005580       ??__E?_Iostream_object@?$_Error_objects@H@std@@2V_Iostream_error_category@2@A@@YAXXZ 10006580 f   moc_DiamondSupport.obj
 0001:00005590       ??__E?_System_object@?$_Error_objects@H@std@@2V_System_error_category@2@A@@YAXXZ 10006590 f   moc_DiamondSupport.obj
 0001:000055a0       ??__E?staticMetaObject@DiamondSupport@U2@@2UQMetaObject@@B@@YAXXZ 100065a0 f   moc_DiamondSupport.obj
 0001:000055b0       ??__E?_Generic_object@?$_Error_objects@H@std@@2V_Generic_error_category@2@A@@YAXXZ 100065b0 f   moc_DiamondSupportPlugin.obj
 0001:000055c0       ??__E?_Iostream_object@?$_Error_objects@H@std@@2V_Iostream_error_category@2@A@@YAXXZ 100065c0 f   moc_DiamondSupportPlugin.obj
 0001:000055d0       ??__E?_System_object@?$_Error_objects@H@std@@2V_System_error_category@2@A@@YAXXZ 100065d0 f   moc_DiamondSupportPlugin.obj
 0001:000055e0       ??__E?staticMetaObject@DiamondSupportPlugin@U2@@2UQMetaObject@@B@@YAXXZ 100065e0 f   moc_DiamondSupportPlugin.obj
 0001:000055f0       ??__E?_Generic_object@?$_Error_objects@H@std@@2V_Generic_error_category@2@A@@YAXXZ 100065f0 f   moc_GenomesPreparationTask.obj
 0001:00005600       ??__E?_Iostream_object@?$_Error_objects@H@std@@2V_Iostream_error_category@2@A@@YAXXZ 10006600 f   moc_GenomesPreparationTask.obj
 0001:00005610       ??__E?_System_object@?$_Error_objects@H@std@@2V_System_error_category@2@A@@YAXXZ 10006610 f   moc_GenomesPreparationTask.obj
 0001:00005620       ??__E?staticMetaObject@GenomesPreparationTask@U2@@2UQMetaObject@@B@@YAXXZ 10006620 f   moc_GenomesPreparationTask.obj
 0001:00005630       ??__EalgoLog@U2@@YAXXZ     10006630 f   moc_GenomesPreparationTask.obj
 0001:000056b0       ??__EcmdLog@U2@@YAXXZ      100066b0 f   moc_GenomesPreparationTask.obj
 0001:00005730       ??__EcoreLog@U2@@YAXXZ     10006730 f   moc_GenomesPreparationTask.obj
 0001:000057b0       ??__EioLog@U2@@YAXXZ       100067b0 f   moc_GenomesPreparationTask.obj
 0001:00005830       ??__EperfLog@U2@@YAXXZ     10006830 f   moc_GenomesPreparationTask.obj
 0001:000058b0       ??__EscriptLog@U2@@YAXXZ   100068b0 f   moc_GenomesPreparationTask.obj
 0001:00005930       ??__EtaskLog@U2@@YAXXZ     10006930 f   moc_GenomesPreparationTask.obj
 0001:000059b0       ??__EuiLog@U2@@YAXXZ       100069b0 f   moc_GenomesPreparationTask.obj
 0001:00005a30       ??__EuserActLog@U2@@YAXXZ  10006a30 f   moc_GenomesPreparationTask.obj
 0001:00005cfe       __catch$??0?$QList@PAVPort@Workflow@U2@@@@QAE@ABV0@@Z$0 10006cfe f i DiamondBuildPrompter.obj
 0001:000061e6       __catch$?_Copy@?$basic_string@DU?$char_traits@D@std@@V?$allocator@D@2@@std@@QAEXII@Z$0 100071e6 f i DiamondBuildPrompter.obj
 0001:00006223       __catch$?_Copy@?$basic_string@DU?$char_traits@D@std@@V?$allocator@D@2@@std@@QAEXII@Z$1 10007223 f i DiamondBuildPrompter.obj
 0001:000071fe       __catch$??0?$QList@VQString@@@@QAE@ABV0@@Z$0 100081fe f i DiamondBuildTask.obj
 0001:00007965       __catch$?append@?$QList@PAVTask@U2@@@@QAEXABQAVTask@U2@@@Z$4 10008965 f i DiamondBuildTask.obj
 0001:000079ed       __catch$?append@?$QList@VQString@@@@QAEXABVQString@@@Z$0 100089ed f i DiamondBuildTask.obj
 0001:00007a3e       __catch$?append@?$QList@VQString@@@@QAEXABVQString@@@Z$4 10008a3e f i DiamondBuildTask.obj
 0001:00007d01       __catch$?detach_helper_grow@?$QList@PAVTask@U2@@@@AAEPAUNode@1@HH@Z$2 10008d01 f i DiamondBuildTask.obj
 0001:00007d01       __catch$?detach_helper_grow@?$QList@PAVTask@U2@@@@AAEPAUNode@1@HH@Z$0 10008d01 f i DiamondBuildTask.obj
 0001:00007e3e       __catch$?detach_helper_grow@?$QList@VQString@@@@AAEPAUNode@1@HH@Z$2 10008e3e f i DiamondBuildTask.obj
 0001:00007e79       __catch$?detach_helper_grow@?$QList@VQString@@@@AAEPAUNode@1@HH@Z$0 10008e79 f i DiamondBuildTask.obj
 0001:000081a2       __catch$?node_copy@?$QList@VQString@@@@AAEXPAUNode@1@00@Z$2 100091a2 f i DiamondBuildTask.obj
 0001:000086f0       __catch$?append@?$QList@VWorkflowNotification@U2@@@@QAEXABVWorkflowNotification@U2@@@Z$0 100096f0 f i DiamondBuildValidator.obj
 0001:000086f0       __catch$?append@?$QList@VWorkflowNotification@U2@@@@QAEXABVWorkflowNotification@U2@@@Z$2 100096f0 f i DiamondBuildValidator.obj
 0001:0000887f       __catch$?detach_helper_grow@?$QList@VWorkflowNotification@U2@@@@AAEPAUNode@1@HH@Z$2 1000987f f i DiamondBuildValidator.obj
 0001:000088ba       __catch$?detach_helper_grow@?$QList@VWorkflowNotification@U2@@@@AAEPAUNode@1@HH@Z$0 100098ba f i DiamondBuildValidator.obj
 0001:000089de       __catch$?node_copy@?$QList@VWorkflowNotification@U2@@@@AAEXPAUNode@1@00@Z$0 100099de f i DiamondBuildValidator.obj
 0001:000096ce       __catch$??0?$QList@PAVURLContainer@U2@@@@QAE@ABV0@@Z$0 1000a6ce f i DiamondBuildWorker.obj
 0001:000097ae       __catch$??0?$QList@VDataset@U2@@@@QAE@ABV0@@Z$0 1000a7ae f i DiamondBuildWorker.obj
 0001:0000989e       __catch$??0?$QList@VDescriptor@U2@@@@QAE@ABV0@@Z$0 1000a89e f i DiamondBuildWorker.obj
 0001:0000a35c       __catch$?append@?$QList@VDescriptor@U2@@@@QAEXABVDescriptor@U2@@@Z$0 1000b35c f i DiamondBuildWorker.obj
 0001:0000a35c       __catch$?append@?$QList@VDescriptor@U2@@@@QAEXABVDescriptor@U2@@@Z$2 1000b35c f i DiamondBuildWorker.obj
 0001:0000a60e       __catch$?createNode@?$QMapData@VQString@@VQScriptValue@@@@QAEPAU?$QMapNode@VQString@@VQScriptValue@@@@ABVQString@@ABVQScriptValue@@PAU2@_N@Z$0 1000b60e f i DiamondBuildWorker.obj
 0001:0000a623       __catch$?createNode@?$QMapData@VQString@@VQScriptValue@@@@QAEPAU?$QMapNode@VQString@@VQScriptValue@@@@ABVQString@@ABVQScriptValue@@PAU2@_N@Z$2 1000b623 f i DiamondBuildWorker.obj
 0001:0000a6ce       __catch$?createNode@?$QMapData@VQString@@VQVariant@@@@QAEPAU?$QMapNode@VQString@@VQVariant@@@@ABVQString@@ABVQVariant@@PAU2@_N@Z$0 1000b6ce f i DiamondBuildWorker.obj
 0001:0000a6e3       __catch$?createNode@?$QMapData@VQString@@VQVariant@@@@QAEPAU?$QMapNode@VQString@@VQVariant@@@@ABVQString@@ABVQVariant@@PAU2@_N@Z$2 1000b6e3 f i DiamondBuildWorker.obj
 0001:0000a9ba       __catch$?detach_helper@?$QList@VDescriptor@U2@@@@AAEXH@Z$0 1000b9ba f i DiamondBuildWorker.obj
 0001:0000abcf       __catch$?detach_helper_grow@?$QList@VDescriptor@U2@@@@AAEPAUNode@1@HH@Z$2 1000bbcf f i DiamondBuildWorker.obj
 0001:0000ac0a       __catch$?detach_helper_grow@?$QList@VDescriptor@U2@@@@AAEPAUNode@1@HH@Z$0 1000bc0a f i DiamondBuildWorker.obj
 0001:0000bd4e       __catch$?node_copy@?$QList@VDataset@U2@@@@AAEXPAUNode@1@00@Z$0 1000cd4e f i DiamondBuildWorker.obj
 0001:0000be25       __catch$?node_copy@?$QList@VDescriptor@U2@@@@AAEXPAUNode@1@00@Z$0 1000ce25 f i DiamondBuildWorker.obj
 0001:0000ce95       __catch$?append@?$QList@PAVAttribute@U2@@@@QAEXABQAVAttribute@U2@@@Z$4 1000de95 f i DiamondBuildWorkerFactory.obj
 0001:0000cf25       __catch$?append@?$QList@PAVPortDescriptor@Workflow@U2@@@@QAEXABQAVPortDescriptor@Workflow@U2@@@Z$4 1000df25 f i DiamondBuildWorkerFactory.obj
 0001:0000d15d       __catch$?createNode@?$QMapData@VDescriptor@U2@@V?$QExplicitlySharedDataPointer@VDataType@U2@@@@@@QAEPAU?$QMapNode@VDescriptor@U2@@V?$QExplicitlySharedDataPointer@VDataType@U2@@@@@@ABVDescriptor@U2@@ABV?$QExplicitlySharedDataPointer@VDataType@U2@@@@PAU2@_N@Z$2 1000e15d f i DiamondBuildWorkerFactory.obj
 0001:0000d205       __catch$?createNode@?$QMapData@VQString@@PAVPropertyDelegate@U2@@@@QAEPAU?$QMapNode@VQString@@PAVPropertyDelegate@U2@@@@ABVQString@@ABQAVPropertyDelegate@U2@@PAU2@_N@Z$2 1000e205 f i DiamondBuildWorkerFactory.obj
 0001:0000d631       __catch$?detach_helper_grow@?$QList@PAVAttribute@U2@@@@AAEPAUNode@1@HH@Z$2 1000e631 f i DiamondBuildWorkerFactory.obj
 0001:0000d631       __catch$?detach_helper_grow@?$QList@PAVAttribute@U2@@@@AAEPAUNode@1@HH@Z$0 1000e631 f i DiamondBuildWorkerFactory.obj
 0001:0000d741       __catch$?detach_helper_grow@?$QList@PAVPortDescriptor@Workflow@U2@@@@AAEPAUNode@1@HH@Z$0 1000e741 f i DiamondBuildWorkerFactory.obj
 0001:0000d741       __catch$?detach_helper_grow@?$QList@PAVPortDescriptor@Workflow@U2@@@@AAEPAUNode@1@HH@Z$2 1000e741 f i DiamondBuildWorkerFactory.obj
 0001:0000f345       __catch$?createNode@?$QMapData@VQString@@I@@QAEPAU?$QMapNode@VQString@@I@@ABVQString@@ABIPAU2@_N@Z$2 10010345 f i DiamondClassifyTask.obj
 0001:0000f531       __catch$?detach_helper@?$QList@VQByteArray@@@@AAEXH@Z$0 10010531 f i DiamondClassifyTask.obj
 0001:0000fe62       __catch$?node_copy@?$QList@VQByteArray@@@@AAEXPAUNode@1@00@Z$2 10010e62 f i DiamondClassifyTask.obj
 0001:000130ae       __catch$??0?$QList@PAVDNATranslation@U2@@@@QAE@ABV0@@Z$0 100140ae f i DiamondClassifyWorkerFactory.obj
 0001:00013702       __catch$?append@?$QList@U?$QPair@VQString@@V1@@@@@QAEXABU?$QPair@VQString@@V1@@@@Z$0 10014702 f i DiamondClassifyWorkerFactory.obj
 0001:00013702       __catch$?append@?$QList@U?$QPair@VQString@@V1@@@@@QAEXABU?$QPair@VQString@@V1@@@@Z$2 10014702 f i DiamondClassifyWorkerFactory.obj
 0001:00013792       __catch$?append@?$QList@U?$QPair@VQString@@VQVariant@@@@@@QAEXABU?$QPair@VQString@@VQVariant@@@@@Z$0 10014792 f i DiamondClassifyWorkerFactory.obj
 0001:00013792       __catch$?append@?$QList@U?$QPair@VQString@@VQVariant@@@@@@QAEXABU?$QPair@VQString@@VQVariant@@@@@Z$2 10014792 f i DiamondClassifyWorkerFactory.obj
 0001:00013a3c       __catch$?detach_helper_grow@?$QList@U?$QPair@VQString@@V1@@@@@AAEPAUNode@1@HH@Z$2 10014a3c f i DiamondClassifyWorkerFactory.obj
 0001:00013a77       __catch$?detach_helper_grow@?$QList@U?$QPair@VQString@@V1@@@@@AAEPAUNode@1@HH@Z$0 10014a77 f i DiamondClassifyWorkerFactory.obj
 0001:00013bac       __catch$?detach_helper_grow@?$QList@U?$QPair@VQString@@VQVariant@@@@@@AAEPAUNode@1@HH@Z$2 10014bac f i DiamondClassifyWorkerFactory.obj
 0001:00013be7       __catch$?detach_helper_grow@?$QList@U?$QPair@VQString@@VQVariant@@@@@@AAEPAUNode@1@HH@Z$0 10014be7 f i DiamondClassifyWorkerFactory.obj
 0001:000173ab       __catch$?node_copy@?$QList@U?$QPair@VQString@@V1@@@@@AAEXPAUNode@1@00@Z$0 100183ab f i DiamondClassifyWorkerFactory.obj
 0001:000174ab       __catch$?node_copy@?$QList@U?$QPair@VQString@@VQVariant@@@@@@AAEXPAUNode@1@00@Z$0 100184ab f i DiamondClassifyWorkerFactory.obj
 0001:000194a0       _pre_c_init                1001a4a0 f   MSVCRT:crtdll.obj
 0001:0001970d       ___DllMainCRTStartup       1001a70d f   MSVCRT:crtdll.obj
 0001:00019860       $$000000                   1001a860     MSVCRT:sehprolg4.obj
 0001:00019c75       ?ArrayUnwindFilter@@YAHPAU_EXCEPTION_POINTERS@@@Z 1001ac75 f   MSVCRT:ehvecdtr.obj
 0001:00019fc0       __ehhandler$??0?$QList@PAVPort@Workflow@U2@@@@QAE@ABV0@@Z 1001afc0 f   DiamondBuildPrompter.obj
 0001:00019fe0       __unwindfunclet$??__EalgoLog@U2@@YAXXZ$0 1001afe0 f   DiamondBuildPrompter.obj
 0001:00019fe9       __ehhandler$??__EalgoLog@U2@@YAXXZ 1001afe9 f   DiamondBuildPrompter.obj
 0001:0001a010       __unwindfunclet$??__EcmdLog@U2@@YAXXZ$0 1001b010 f   DiamondBuildPrompter.obj
 0001:0001a019       __ehhandler$??__EcmdLog@U2@@YAXXZ 1001b019 f   DiamondBuildPrompter.obj
 0001:0001a040       __unwindfunclet$??__EcoreLog@U2@@YAXXZ$0 1001b040 f   DiamondBuildPrompter.obj
 0001:0001a049       __ehhandler$??__EcoreLog@U2@@YAXXZ 1001b049 f   DiamondBuildPrompter.obj
 0001:0001a070       __unwindfunclet$??__EioLog@U2@@YAXXZ$0 1001b070 f   DiamondBuildPrompter.obj
 0001:0001a079       __ehhandler$??__EioLog@U2@@YAXXZ 1001b079 f   DiamondBuildPrompter.obj
 0001:0001a0a0       __unwindfunclet$??__EperfLog@U2@@YAXXZ$0 1001b0a0 f   DiamondBuildPrompter.obj
 0001:0001a0a9       __ehhandler$??__EperfLog@U2@@YAXXZ 1001b0a9 f   DiamondBuildPrompter.obj
 0001:0001a0d0       __unwindfunclet$??__EscriptLog@U2@@YAXXZ$0 1001b0d0 f   DiamondBuildPrompter.obj
 0001:0001a0d9       __ehhandler$??__EscriptLog@U2@@YAXXZ 1001b0d9 f   DiamondBuildPrompter.obj
 0001:0001a100       __unwindfunclet$??__EtaskLog@U2@@YAXXZ$0 1001b100 f   DiamondBuildPrompter.obj
 0001:0001a109       __ehhandler$??__EtaskLog@U2@@YAXXZ 1001b109 f   DiamondBuildPrompter.obj
 0001:0001a130       __unwindfunclet$??__EuiLog@U2@@YAXXZ$0 1001b130 f   DiamondBuildPrompter.obj
 0001:0001a139       __ehhandler$??__EuiLog@U2@@YAXXZ 1001b139 f   DiamondBuildPrompter.obj
 0001:0001a160       __unwindfunclet$??__EuserActLog@U2@@YAXXZ$0 1001b160 f   DiamondBuildPrompter.obj
 0001:0001a169       __ehhandler$??__EuserActLog@U2@@YAXXZ 1001b169 f   DiamondBuildPrompter.obj
 0001:0001a190       __ehhandler$?_Copy@?$basic_string@DU?$char_traits@D@std@@V?$allocator@D@2@@std@@QAEXII@Z 1001b190 f   DiamondBuildPrompter.obj
 0001:0001a1b0       __unwindfunclet$?composeRichDoc@DiamondBuildPrompter@LocalWorkflow@U2@@EAE?AVQString@@XZ$0 1001b1b0 f   DiamondBuildPrompter.obj
 0001:0001a1b9       __unwindfunclet$?composeRichDoc@DiamondBuildPrompter@LocalWorkflow@U2@@EAE?AVQString@@XZ$1 1001b1b9 f   DiamondBuildPrompter.obj
 0001:0001a1c2       __unwindfunclet$?composeRichDoc@DiamondBuildPrompter@LocalWorkflow@U2@@EAE?AVQString@@XZ$2 1001b1c2 f   DiamondBuildPrompter.obj
 0001:0001a1cb       __unwindfunclet$?composeRichDoc@DiamondBuildPrompter@LocalWorkflow@U2@@EAE?AVQString@@XZ$3 1001b1cb f   DiamondBuildPrompter.obj
 0001:0001a1d4       __unwindfunclet$?composeRichDoc@DiamondBuildPrompter@LocalWorkflow@U2@@EAE?AVQString@@XZ$4 1001b1d4 f   DiamondBuildPrompter.obj
 0001:0001a1dd       __unwindfunclet$?composeRichDoc@DiamondBuildPrompter@LocalWorkflow@U2@@EAE?AVQString@@XZ$5 1001b1dd f   DiamondBuildPrompter.obj
 0001:0001a1f7       __ehhandler$?composeRichDoc@DiamondBuildPrompter@LocalWorkflow@U2@@EAE?AVQString@@XZ 1001b1f7 f   DiamondBuildPrompter.obj
 0001:0001a220       __unwindfunclet$?createDescription@?$PrompterBase@VDiamondBuildPrompter@LocalWorkflow@U2@@@U2@@UAEPAVActorDocument@Workflow@2@PAVActor@42@@Z$0 1001b220 f   DiamondBuildPrompter.obj
 0001:0001a22b       __unwindfunclet$?createDescription@?$PrompterBase@VDiamondBuildPrompter@LocalWorkflow@U2@@@U2@@UAEPAVActorDocument@Workflow@2@PAVActor@42@@Z$3 1001b22b f   DiamondBuildPrompter.obj
 0001:0001a233       __unwindfunclet$?createDescription@?$PrompterBase@VDiamondBuildPrompter@LocalWorkflow@U2@@@U2@@UAEPAVActorDocument@Workflow@2@PAVActor@42@@Z$4 1001b233 f   DiamondBuildPrompter.obj
 0001:0001a23b       __unwindfunclet$?createDescription@?$PrompterBase@VDiamondBuildPrompter@LocalWorkflow@U2@@@U2@@UAEPAVActorDocument@Workflow@2@PAVActor@42@@Z$6 1001b23b f   DiamondBuildPrompter.obj
 0001:0001a243       __unwindfunclet$?createDescription@?$PrompterBase@VDiamondBuildPrompter@LocalWorkflow@U2@@@U2@@UAEPAVActorDocument@Workflow@2@PAVActor@42@@Z$7 1001b243 f   DiamondBuildPrompter.obj
 0001:0001a24b       __ehhandler$?createDescription@?$PrompterBase@VDiamondBuildPrompter@LocalWorkflow@U2@@@U2@@UAEPAVActorDocument@Workflow@2@PAVActor@42@@Z 1001b24b f   DiamondBuildPrompter.obj
 0001:0001a270       __ehhandler$??0?$QList@VQString@@@@QAE@ABV0@@Z 1001b270 f   DiamondBuildTask.obj
 0001:0001a290       __unwindfunclet$??0DiamondBuildTask@U2@@QAE@ABUDiamondBuildTaskSettings@1@@Z$0 1001b290 f   DiamondBuildTask.obj
 0001:0001a299       __unwindfunclet$??0DiamondBuildTask@U2@@QAE@ABUDiamondBuildTaskSettings@1@@Z$1 1001b299 f   DiamondBuildTask.obj
 0001:0001a2a2       __unwindfunclet$??0DiamondBuildTask@U2@@QAE@ABUDiamondBuildTaskSettings@1@@Z$7 1001b2a2 f   DiamondBuildTask.obj
 0001:0001a2ab       __unwindfunclet$??0DiamondBuildTask@U2@@QAE@ABUDiamondBuildTaskSettings@1@@Z$8 1001b2ab f   DiamondBuildTask.obj
 0001:0001a2b6       __unwindfunclet$??0DiamondBuildTask@U2@@QAE@ABUDiamondBuildTaskSettings@1@@Z$9 1001b2b6 f   DiamondBuildTask.obj
 0001:0001a2c2       __unwindfunclet$??0DiamondBuildTask@U2@@QAE@ABUDiamondBuildTaskSettings@1@@Z$10 1001b2c2 f   DiamondBuildTask.obj
 0001:0001a2ce       __unwindfunclet$??0DiamondBuildTask@U2@@QAE@ABUDiamondBuildTaskSettings@1@@Z$2 1001b2ce f   DiamondBuildTask.obj
 0001:0001a2dc       __unwindfunclet$??0DiamondBuildTask@U2@@QAE@ABUDiamondBuildTaskSettings@1@@Z$3 1001b2dc f   DiamondBuildTask.obj
 0001:0001a2ea       __unwindfunclet$??0DiamondBuildTask@U2@@QAE@ABUDiamondBuildTaskSettings@1@@Z$4 1001b2ea f   DiamondBuildTask.obj
 0001:0001a2f3       __unwindfunclet$??0DiamondBuildTask@U2@@QAE@ABUDiamondBuildTaskSettings@1@@Z$5 1001b2f3 f   DiamondBuildTask.obj
 0001:0001a2fc       __unwindfunclet$??0DiamondBuildTask@U2@@QAE@ABUDiamondBuildTaskSettings@1@@Z$6 1001b2fc f   DiamondBuildTask.obj
 0001:0001a305       __ehhandler$??0DiamondBuildTask@U2@@QAE@ABUDiamondBuildTaskSettings@1@@Z 1001b305 f   DiamondBuildTask.obj
 0001:0001a320       __unwindfunclet$??0DiamondBuildTaskSettings@U2@@QAE@ABU01@@Z$0 1001b320 f   DiamondBuildTask.obj
 0001:0001a329       __unwindfunclet$??0DiamondBuildTaskSettings@U2@@QAE@ABU01@@Z$1 1001b329 f   DiamondBuildTask.obj
 0001:0001a334       __unwindfunclet$??0DiamondBuildTaskSettings@U2@@QAE@ABU01@@Z$2 1001b334 f   DiamondBuildTask.obj
 0001:0001a340       __unwindfunclet$??0DiamondBuildTaskSettings@U2@@QAE@ABU01@@Z$3 1001b340 f   DiamondBuildTask.obj
 0001:0001a34c       __ehhandler$??0DiamondBuildTaskSettings@U2@@QAE@ABU01@@Z 1001b34c f   DiamondBuildTask.obj
 0001:0001a370       __unwindfunclet$??1DiamondBuildTask@U2@@UAE@XZ$0 1001b370 f   DiamondBuildTask.obj
 0001:0001a379       __unwindfunclet$??1DiamondBuildTask@U2@@UAE@XZ$2 1001b379 f   DiamondBuildTask.obj
 0001:0001a382       __unwindfunclet$??1DiamondBuildTask@U2@@UAE@XZ$3 1001b382 f   DiamondBuildTask.obj
 0001:0001a38d       __unwindfunclet$??1DiamondBuildTask@U2@@UAE@XZ$4 1001b38d f   DiamondBuildTask.obj
 0001:0001a399       __unwindfunclet$??1DiamondBuildTask@U2@@UAE@XZ$5 1001b399 f   DiamondBuildTask.obj
 0001:0001a3a5       __ehhandler$??1DiamondBuildTask@U2@@UAE@XZ 1001b3a5 f   DiamondBuildTask.obj
 0001:0001a3c0       __unwindfunclet$??1DiamondBuildTaskSettings@U2@@QAE@XZ$0 1001b3c0 f   DiamondBuildTask.obj
 0001:0001a3c9       __unwindfunclet$??1DiamondBuildTaskSettings@U2@@QAE@XZ$1 1001b3c9 f   DiamondBuildTask.obj
 0001:0001a3d4       __unwindfunclet$??1DiamondBuildTaskSettings@U2@@QAE@XZ$2 1001b3d4 f   DiamondBuildTask.obj
 0001:0001a3e0       __unwindfunclet$??1DiamondBuildTaskSettings@U2@@QAE@XZ$3 1001b3e0 f   DiamondBuildTask.obj
 0001:0001a3ec       __ehhandler$??1DiamondBuildTaskSettings@U2@@QAE@XZ 1001b3ec f   DiamondBuildTask.obj
 0001:0001a410       __unwindfunclet$??H@YA?BVQString@@ABV0@PBD@Z$0 1001b410 f   DiamondBuildTask.obj
 0001:0001a42a       __unwindfunclet$??H@YA?BVQString@@ABV0@PBD@Z$1 1001b42a f   DiamondBuildTask.obj
 0001:0001a433       __ehhandler$??H@YA?BVQString@@ABV0@PBD@Z 1001b433 f   DiamondBuildTask.obj
 0001:0001a450       __unwindfunclet$??__EalgoLog@U2@@YAXXZ$0 1001b450 f   DiamondBuildTask.obj
 0001:0001a459       __ehhandler$??__EalgoLog@U2@@YAXXZ 1001b459 f   DiamondBuildTask.obj
 0001:0001a480       __unwindfunclet$??__EcmdLog@U2@@YAXXZ$0 1001b480 f   DiamondBuildTask.obj
 0001:0001a489       __ehhandler$??__EcmdLog@U2@@YAXXZ 1001b489 f   DiamondBuildTask.obj
 0001:0001a4b0       __unwindfunclet$??__EcoreLog@U2@@YAXXZ$0 1001b4b0 f   DiamondBuildTask.obj
 0001:0001a4b9       __ehhandler$??__EcoreLog@U2@@YAXXZ 1001b4b9 f   DiamondBuildTask.obj
 0001:0001a4e0       __unwindfunclet$??__EioLog@U2@@YAXXZ$0 1001b4e0 f   DiamondBuildTask.obj
 0001:0001a4e9       __ehhandler$??__EioLog@U2@@YAXXZ 1001b4e9 f   DiamondBuildTask.obj
 0001:0001a510       __unwindfunclet$??__EperfLog@U2@@YAXXZ$0 1001b510 f   DiamondBuildTask.obj
 0001:0001a519       __ehhandler$??__EperfLog@U2@@YAXXZ 1001b519 f   DiamondBuildTask.obj
 0001:0001a540       __unwindfunclet$??__EscriptLog@U2@@YAXXZ$0 1001b540 f   DiamondBuildTask.obj
 0001:0001a549       __ehhandler$??__EscriptLog@U2@@YAXXZ 1001b549 f   DiamondBuildTask.obj
 0001:0001a570       __unwindfunclet$??__EtaskLog@U2@@YAXXZ$0 1001b570 f   DiamondBuildTask.obj
 0001:0001a579       __ehhandler$??__EtaskLog@U2@@YAXXZ 1001b579 f   DiamondBuildTask.obj
 0001:0001a5a0       __unwindfunclet$??__EuiLog@U2@@YAXXZ$0 1001b5a0 f   DiamondBuildTask.obj
 0001:0001a5a9       __ehhandler$??__EuiLog@U2@@YAXXZ 1001b5a9 f   DiamondBuildTask.obj
 0001:0001a5d0       __unwindfunclet$??__EuserActLog@U2@@YAXXZ$0 1001b5d0 f   DiamondBuildTask.obj
 0001:0001a5d9       __ehhandler$??__EuserActLog@U2@@YAXXZ 1001b5d9 f   DiamondBuildTask.obj
 0001:0001a600       __ehhandler$?append@?$QList@PAVTask@U2@@@@QAEXABQAVTask@U2@@@Z 1001b600 f   DiamondBuildTask.obj
 0001:0001a620       __unwindfunclet$?append@?$QList@VQString@@@@QAEXABVQString@@@Z$7 1001b620 f   DiamondBuildTask.obj
 0001:0001a631       __unwindfunclet$?append@?$QList@VQString@@@@QAEXABVQString@@@Z$11 1001b631 f   DiamondBuildTask.obj
 0001:0001a642       __ehhandler$?append@?$QList@VQString@@@@QAEXABVQString@@@Z 1001b642 f   DiamondBuildTask.obj
 0001:0001a660       __unwindfunclet$?checkSettings@DiamondBuildTask@U2@@AAEXXZ$0 1001b660 f   DiamondBuildTask.obj
 0001:0001a669       __unwindfunclet$?checkSettings@DiamondBuildTask@U2@@AAEXXZ$1 1001b669 f   DiamondBuildTask.obj
 0001:0001a672       __unwindfunclet$?checkSettings@DiamondBuildTask@U2@@AAEXXZ$2 1001b672 f   DiamondBuildTask.obj
 0001:0001a67b       __unwindfunclet$?checkSettings@DiamondBuildTask@U2@@AAEXXZ$3 1001b67b f   DiamondBuildTask.obj
 0001:0001a684       __ehhandler$?checkSettings@DiamondBuildTask@U2@@AAEXXZ 1001b684 f   DiamondBuildTask.obj
 0001:0001a6a0       __ehhandler$?detach_helper_grow@?$QList@PAVTask@U2@@@@AAEPAUNode@1@HH@Z 1001b6a0 f   DiamondBuildTask.obj
 0001:0001a6c0       __ehhandler$?detach_helper_grow@?$QList@VQString@@@@AAEPAUNode@1@HH@Z 1001b6c0 f   DiamondBuildTask.obj
 0001:0001a6e0       __unwindfunclet$?getArguments@DiamondBuildTask@U2@@ABE?AVQStringList@@ABVQString@@@Z$0 1001b6e0 f   DiamondBuildTask.obj
 0001:0001a6f9       __unwindfunclet$?getArguments@DiamondBuildTask@U2@@ABE?AVQStringList@@ABVQString@@@Z$1 1001b6f9 f   DiamondBuildTask.obj
 0001:0001a702       __unwindfunclet$?getArguments@DiamondBuildTask@U2@@ABE?AVQStringList@@ABVQString@@@Z$2 1001b702 f   DiamondBuildTask.obj
 0001:0001a70b       __unwindfunclet$?getArguments@DiamondBuildTask@U2@@ABE?AVQStringList@@ABVQString@@@Z$3 1001b70b f   DiamondBuildTask.obj
 0001:0001a714       __unwindfunclet$?getArguments@DiamondBuildTask@U2@@ABE?AVQStringList@@ABVQString@@@Z$4 1001b714 f   DiamondBuildTask.obj
 0001:0001a71d       __unwindfunclet$?getArguments@DiamondBuildTask@U2@@ABE?AVQStringList@@ABVQString@@@Z$5 1001b71d f   DiamondBuildTask.obj
 0001:0001a726       __ehhandler$?getArguments@DiamondBuildTask@U2@@ABE?AVQStringList@@ABVQString@@@Z 1001b726 f   DiamondBuildTask.obj
 0001:0001a750       __unwindfunclet$?node_construct@?$QList@VQString@@@@AAEXPAUNode@1@ABVQString@@@Z$1 1001b750 f   DiamondBuildTask.obj
 0001:0001a761       __ehhandler$?node_construct@?$QList@VQString@@@@AAEXPAUNode@1@ABVQString@@@Z 1001b761 f   DiamondBuildTask.obj
 0001:0001a780       __unwindfunclet$?node_copy@?$QList@VQString@@@@AAEXPAUNode@1@00@Z$5 1001b780 f   DiamondBuildTask.obj
 0001:0001a791       __ehhandler$?node_copy@?$QList@VQString@@@@AAEXPAUNode@1@00@Z 1001b791 f   DiamondBuildTask.obj
 0001:0001a7b0       __unwindfunclet$?onSubTaskFinished@DiamondBuildTask@U2@@EAE?AV?$QList@PAVTask@U2@@@@PAVTask@2@@Z$0 1001b7b0 f   DiamondBuildTask.obj
 0001:0001a7b8       __unwindfunclet$?onSubTaskFinished@DiamondBuildTask@U2@@EAE?AV?$QList@PAVTask@U2@@@@PAVTask@2@@Z$1 1001b7b8 f   DiamondBuildTask.obj
 0001:0001a7d1       __unwindfunclet$?onSubTaskFinished@DiamondBuildTask@U2@@EAE?AV?$QList@PAVTask@U2@@@@PAVTask@2@@Z$2 1001b7d1 f   DiamondBuildTask.obj
 0001:0001a7dc       __unwindfunclet$?onSubTaskFinished@DiamondBuildTask@U2@@EAE?AV?$QList@PAVTask@U2@@@@PAVTask@2@@Z$3 1001b7dc f   DiamondBuildTask.obj
 0001:0001a7f6       __unwindfunclet$?onSubTaskFinished@DiamondBuildTask@U2@@EAE?AV?$QList@PAVTask@U2@@@@PAVTask@2@@Z$4 1001b7f6 f   DiamondBuildTask.obj
 0001:0001a801       __unwindfunclet$?onSubTaskFinished@DiamondBuildTask@U2@@EAE?AV?$QList@PAVTask@U2@@@@PAVTask@2@@Z$5 1001b801 f   DiamondBuildTask.obj
 0001:0001a81b       __unwindfunclet$?onSubTaskFinished@DiamondBuildTask@U2@@EAE?AV?$QList@PAVTask@U2@@@@PAVTask@2@@Z$6 1001b81b f   DiamondBuildTask.obj
 0001:0001a834       __unwindfunclet$?onSubTaskFinished@DiamondBuildTask@U2@@EAE?AV?$QList@PAVTask@U2@@@@PAVTask@2@@Z$7 1001b834 f   DiamondBuildTask.obj
 0001:0001a84d       __ehhandler$?onSubTaskFinished@DiamondBuildTask@U2@@EAE?AV?$QList@PAVTask@U2@@@@PAVTask@2@@Z 1001b84d f   DiamondBuildTask.obj
 0001:0001a870       __unwindfunclet$?prepare@DiamondBuildTask@U2@@EAEXXZ$0 1001b870 f   DiamondBuildTask.obj
 0001:0001a87b       __unwindfunclet$?prepare@DiamondBuildTask@U2@@EAEXXZ$1 1001b87b f   DiamondBuildTask.obj
 0001:0001a894       __unwindfunclet$?prepare@DiamondBuildTask@U2@@EAEXXZ$2 1001b894 f   DiamondBuildTask.obj
 0001:0001a8ae       __unwindfunclet$?prepare@DiamondBuildTask@U2@@EAEXXZ$3 1001b8ae f   DiamondBuildTask.obj
 0001:0001a8c8       __ehhandler$?prepare@DiamondBuildTask@U2@@EAEXXZ 1001b8c8 f   DiamondBuildTask.obj
 0001:0001a8f0       __unwindfunclet$??__EalgoLog@U2@@YAXXZ$0 1001b8f0 f   DiamondBuildValidator.obj
 0001:0001a8f9       __ehhandler$??__EalgoLog@U2@@YAXXZ 1001b8f9 f   DiamondBuildValidator.obj
 0001:0001a920       __unwindfunclet$??__EcmdLog@U2@@YAXXZ$0 1001b920 f   DiamondBuildValidator.obj
 0001:0001a929       __ehhandler$??__EcmdLog@U2@@YAXXZ 1001b929 f   DiamondBuildValidator.obj
 0001:0001a950       __unwindfunclet$??__EcoreLog@U2@@YAXXZ$0 1001b950 f   DiamondBuildValidator.obj
 0001:0001a959       __ehhandler$??__EcoreLog@U2@@YAXXZ 1001b959 f   DiamondBuildValidator.obj
 0001:0001a980       __unwindfunclet$??__EioLog@U2@@YAXXZ$0 1001b980 f   DiamondBuildValidator.obj
 0001:0001a989       __ehhandler$??__EioLog@U2@@YAXXZ 1001b989 f   DiamondBuildValidator.obj
 0001:0001a9b0       __unwindfunclet$??__EperfLog@U2@@YAXXZ$0 1001b9b0 f   DiamondBuildValidator.obj
 0001:0001a9b9       __ehhandler$??__EperfLog@U2@@YAXXZ 1001b9b9 f   DiamondBuildValidator.obj
 0001:0001a9e0       __unwindfunclet$??__EscriptLog@U2@@YAXXZ$0 1001b9e0 f   DiamondBuildValidator.obj
 0001:0001a9e9       __ehhandler$??__EscriptLog@U2@@YAXXZ 1001b9e9 f   DiamondBuildValidator.obj
 0001:0001aa10       __unwindfunclet$??__EtaskLog@U2@@YAXXZ$0 1001ba10 f   DiamondBuildValidator.obj
 0001:0001aa19       __ehhandler$??__EtaskLog@U2@@YAXXZ 1001ba19 f   DiamondBuildValidator.obj
 0001:0001aa40       __unwindfunclet$??__EuiLog@U2@@YAXXZ$0 1001ba40 f   DiamondBuildValidator.obj
 0001:0001aa49       __ehhandler$??__EuiLog@U2@@YAXXZ 1001ba49 f   DiamondBuildValidator.obj
 0001:0001aa70       __unwindfunclet$??__EuserActLog@U2@@YAXXZ$0 1001ba70 f   DiamondBuildValidator.obj
 0001:0001aa79       __ehhandler$??__EuserActLog@U2@@YAXXZ 1001ba79 f   DiamondBuildValidator.obj
 0001:0001aaa0       __unwindfunclet$?append@?$QList@VWorkflowNotification@U2@@@@QAEXABVWorkflowNotification@U2@@@Z$6 1001baa0 f   DiamondBuildValidator.obj
 0001:0001aaab       __ehhandler$?append@?$QList@VWorkflowNotification@U2@@@@QAEXABVWorkflowNotification@U2@@@Z 1001baab f   DiamondBuildValidator.obj
 0001:0001aad0       __ehhandler$?detach_helper_grow@?$QList@VWorkflowNotification@U2@@@@AAEPAUNode@1@HH@Z 1001bad0 f   DiamondBuildValidator.obj
 0001:0001aaf0       __unwindfunclet$?node_construct@?$QList@VWorkflowNotification@U2@@@@AAEXPAUNode@1@ABVWorkflowNotification@U2@@@Z$0 1001baf0 f   DiamondBuildValidator.obj
 0001:0001aafb       __ehhandler$?node_construct@?$QList@VWorkflowNotification@U2@@@@AAEXPAUNode@1@ABVWorkflowNotification@U2@@@Z 1001bafb f   DiamondBuildValidator.obj
 0001:0001ab20       __unwindfunclet$?node_copy@?$QList@VWorkflowNotification@U2@@@@AAEXPAUNode@1@00@Z$4 1001bb20 f   DiamondBuildValidator.obj
 0001:0001ab2b       __ehhandler$?node_copy@?$QList@VWorkflowNotification@U2@@@@AAEXPAUNode@1@00@Z 1001bb2b f   DiamondBuildValidator.obj
 0001:0001ab50       __unwindfunclet$?validateTaxonomy@DiamondBuildValidator@Workflow@U2@@ABE_NPBVActor@23@AAV?$QList@VWorkflowNotification@U2@@@@@Z$0 1001bb50 f   DiamondBuildValidator.obj
 0001:0001ab59       __unwindfunclet$?validateTaxonomy@DiamondBuildValidator@Workflow@U2@@ABE_NPBVActor@23@AAV?$QList@VWorkflowNotification@U2@@@@@Z$1 1001bb59 f   DiamondBuildValidator.obj
 0001:0001ab62       __unwindfunclet$?validateTaxonomy@DiamondBuildValidator@Workflow@U2@@ABE_NPBVActor@23@AAV?$QList@VWorkflowNotification@U2@@@@@Z$2 1001bb62 f   DiamondBuildValidator.obj
 0001:0001ab6b       __unwindfunclet$?validateTaxonomy@DiamondBuildValidator@Workflow@U2@@ABE_NPBVActor@23@AAV?$QList@VWorkflowNotification@U2@@@@@Z$6 1001bb6b f   DiamondBuildValidator.obj
 0001:0001ab74       __unwindfunclet$?validateTaxonomy@DiamondBuildValidator@Workflow@U2@@ABE_NPBVActor@23@AAV?$QList@VWorkflowNotification@U2@@@@@Z$8 1001bb74 f   DiamondBuildValidator.obj
 0001:0001ab7d       __unwindfunclet$?validateTaxonomy@DiamondBuildValidator@Workflow@U2@@ABE_NPBVActor@23@AAV?$QList@VWorkflowNotification@U2@@@@@Z$9 1001bb7d f   DiamondBuildValidator.obj
 0001:0001ab86       __unwindfunclet$?validateTaxonomy@DiamondBuildValidator@Workflow@U2@@ABE_NPBVActor@23@AAV?$QList@VWorkflowNotification@U2@@@@@Z$10 1001bb86 f   DiamondBuildValidator.obj
 0001:0001ab8f       __unwindfunclet$?validateTaxonomy@DiamondBuildValidator@Workflow@U2@@ABE_NPBVActor@23@AAV?$QList@VWorkflowNotification@U2@@@@@Z$12 1001bb8f f   DiamondBuildValidator.obj
 0001:0001ab98       __unwindfunclet$?validateTaxonomy@DiamondBuildValidator@Workflow@U2@@ABE_NPBVActor@23@AAV?$QList@VWorkflowNotification@U2@@@@@Z$13 1001bb98 f   DiamondBuildValidator.obj
 0001:0001aba1       __unwindfunclet$?validateTaxonomy@DiamondBuildValidator@Workflow@U2@@ABE_NPBVActor@23@AAV?$QList@VWorkflowNotification@U2@@@@@Z$14 1001bba1 f   DiamondBuildValidator.obj
 0001:0001abaa       __unwindfunclet$?validateTaxonomy@DiamondBuildValidator@Workflow@U2@@ABE_NPBVActor@23@AAV?$QList@VWorkflowNotification@U2@@@@@Z$3 1001bbaa f   DiamondBuildValidator.obj
 0001:0001abb3       __unwindfunclet$?validateTaxonomy@DiamondBuildValidator@Workflow@U2@@ABE_NPBVActor@23@AAV?$QList@VWorkflowNotification@U2@@@@@Z$4 1001bbb3 f   DiamondBuildValidator.obj
 0001:0001abbc       __unwindfunclet$?validateTaxonomy@DiamondBuildValidator@Workflow@U2@@ABE_NPBVActor@23@AAV?$QList@VWorkflowNotification@U2@@@@@Z$5 1001bbbc f   DiamondBuildValidator.obj
 0001:0001abc5       __ehhandler$?validateTaxonomy@DiamondBuildValidator@Workflow@U2@@ABE_NPBVActor@23@AAV?$QList@VWorkflowNotification@U2@@@@@Z 1001bbc5 f   DiamondBuildValidator.obj
 0001:0001abe0       __unwindfunclet$??$getAttributeValue@VQString@@@Attribute@U2@@QBE?AVQString@@PAVWorkflowContext@Workflow@1@@Z$0 1001bbe0 f   DiamondBuildWorker.obj
 0001:0001abfa       __unwindfunclet$??$getAttributeValue@VQString@@@Attribute@U2@@QBE?AVQString@@PAVWorkflowContext@Workflow@1@@Z$1 1001bbfa f   DiamondBuildWorker.obj
 0001:0001ac03       __unwindfunclet$??$getAttributeValue@VQString@@@Attribute@U2@@QBE?AVQString@@PAVWorkflowContext@Workflow@1@@Z$2 1001bc03 f   DiamondBuildWorker.obj
 0001:0001ac0b       __unwindfunclet$??$getAttributeValue@VQString@@@Attribute@U2@@QBE?AVQString@@PAVWorkflowContext@Workflow@1@@Z$3 1001bc0b f   DiamondBuildWorker.obj
 0001:0001ac13       __unwindfunclet$??$getAttributeValue@VQString@@@Attribute@U2@@QBE?AVQString@@PAVWorkflowContext@Workflow@1@@Z$4 1001bc13 f   DiamondBuildWorker.obj
 0001:0001ac1b       __unwindfunclet$??$getAttributeValue@VQString@@@Attribute@U2@@QBE?AVQString@@PAVWorkflowContext@Workflow@1@@Z$5 1001bc1b f   DiamondBuildWorker.obj
 0001:0001ac24       __unwindfunclet$??$getAttributeValue@VQString@@@Attribute@U2@@QBE?AVQString@@PAVWorkflowContext@Workflow@1@@Z$6 1001bc24 f   DiamondBuildWorker.obj
 0001:0001ac2d       __unwindfunclet$??$getAttributeValue@VQString@@@Attribute@U2@@QBE?AVQString@@PAVWorkflowContext@Workflow@1@@Z$7 1001bc2d f   DiamondBuildWorker.obj
 0001:0001ac36       __unwindfunclet$??$getAttributeValue@VQString@@@Attribute@U2@@QBE?AVQString@@PAVWorkflowContext@Workflow@1@@Z$8 1001bc36 f   DiamondBuildWorker.obj
 0001:0001ac3f       __unwindfunclet$??$getAttributeValue@VQString@@@Attribute@U2@@QBE?AVQString@@PAVWorkflowContext@Workflow@1@@Z$9 1001bc3f f   DiamondBuildWorker.obj
 0001:0001ac48       __unwindfunclet$??$getAttributeValue@VQString@@@Attribute@U2@@QBE?AVQString@@PAVWorkflowContext@Workflow@1@@Z$10 1001bc48 f   DiamondBuildWorker.obj
 0001:0001ac51       __unwindfunclet$??$getAttributeValue@VQString@@@Attribute@U2@@QBE?AVQString@@PAVWorkflowContext@Workflow@1@@Z$11 1001bc51 f   DiamondBuildWorker.obj
 0001:0001ac5a       __unwindfunclet$??$getAttributeValue@VQString@@@Attribute@U2@@QBE?AVQString@@PAVWorkflowContext@Workflow@1@@Z$12 1001bc5a f   DiamondBuildWorker.obj
 0001:0001ac63       __ehhandler$??$getAttributeValue@VQString@@@Attribute@U2@@QBE?AVQString@@PAVWorkflowContext@Workflow@1@@Z 1001bc63 f   DiamondBuildWorker.obj
 0001:0001ac90       __unwindfunclet$??$getValue@VQString@@@BaseWorker@LocalWorkflow@U2@@IBE?AVQString@@ABV3@@Z$0 1001bc90 f   DiamondBuildWorker.obj
 0001:0001acaa       __unwindfunclet$??$getValue@VQString@@@BaseWorker@LocalWorkflow@U2@@IBE?AVQString@@ABV3@@Z$1 1001bcaa f   DiamondBuildWorker.obj
 0001:0001acb3       __ehhandler$??$getValue@VQString@@@BaseWorker@LocalWorkflow@U2@@IBE?AVQString@@ABV3@@Z 1001bcb3 f   DiamondBuildWorker.obj
 0001:0001acd0       __unwindfunclet$??$qRegisterMetaType@V?$QList@VDataset@U2@@@@@@YAHPBDPAV?$QList@VDataset@U2@@@@W4DefinedType@?$MetaTypeDefinedHelper@V?$QList@VDataset@U2@@@@$00@QtPrivate@@@Z$0 1001bcd0 f   DiamondBuildWorker.obj
 0001:0001acd9       __ehhandler$??$qRegisterMetaType@V?$QList@VDataset@U2@@@@@@YAHPBDPAV?$QList@VDataset@U2@@@@W4DefinedType@?$MetaTypeDefinedHelper@V?$QList@VDataset@U2@@@@$00@QtPrivate@@@Z 1001bcd9 f   DiamondBuildWorker.obj
 0001:0001ad00       __ehhandler$??0?$QList@PAVURLContainer@U2@@@@QAE@ABV0@@Z 1001bd00 f   DiamondBuildWorker.obj
 0001:0001ad20       __ehhandler$??0?$QList@VDataset@U2@@@@QAE@ABV0@@Z 1001bd20 f   DiamondBuildWorker.obj
 0001:0001ad40       __ehhandler$??0?$QList@VDescriptor@U2@@@@QAE@ABV0@@Z 1001bd40 f   DiamondBuildWorker.obj
 0001:0001ad60       __unwindfunclet$??0DiamondBuildTaskSettings@U2@@QAE@XZ$0 1001bd60 f   DiamondBuildWorker.obj
 0001:0001ad69       __unwindfunclet$??0DiamondBuildTaskSettings@U2@@QAE@XZ$1 1001bd69 f   DiamondBuildWorker.obj
 0001:0001ad74       __unwindfunclet$??0DiamondBuildTaskSettings@U2@@QAE@XZ$2 1001bd74 f   DiamondBuildWorker.obj
 0001:0001ad80       __unwindfunclet$??0DiamondBuildTaskSettings@U2@@QAE@XZ$3 1001bd80 f   DiamondBuildWorker.obj
 0001:0001ad8c       __ehhandler$??0DiamondBuildTaskSettings@U2@@QAE@XZ 1001bd8c f   DiamondBuildWorker.obj
 0001:0001adb0       __unwindfunclet$??0QStringList@@QAE@ABVQString@@@Z$0 1001bdb0 f   DiamondBuildWorker.obj
 0001:0001adb8       __ehhandler$??0QStringList@@QAE@ABVQString@@@Z 1001bdb8 f   DiamondBuildWorker.obj
 0001:0001ade0       __unwindfunclet$??A?$QMap@VQString@@VQScriptValue@@@@QAEAAVQScriptValue@@ABVQString@@@Z$0 1001bde0 f   DiamondBuildWorker.obj
 0001:0001ade9       __ehhandler$??A?$QMap@VQString@@VQScriptValue@@@@QAEAAVQScriptValue@@ABVQString@@@Z 1001bde9 f   DiamondBuildWorker.obj
 0001:0001ae10       __unwindfunclet$??A?$QMap@VQString@@VQVariant@@@@QAEAAVQVariant@@ABVQString@@@Z$0 1001be10 f   DiamondBuildWorker.obj
 0001:0001ae19       __ehhandler$??A?$QMap@VQString@@VQVariant@@@@QAEAAVQVariant@@ABVQString@@@Z 1001be19 f   DiamondBuildWorker.obj
 0001:0001ae40       __unwindfunclet$??H@YA?BVQString@@ABV0@0@Z$0 1001be40 f   DiamondBuildWorker.obj
 0001:0001ae5a       __ehhandler$??H@YA?BVQString@@ABV0@0@Z 1001be5a f   DiamondBuildWorker.obj
 0001:0001ae80       __unwindfunclet$??__EalgoLog@U2@@YAXXZ$0 1001be80 f   DiamondBuildWorker.obj
 0001:0001ae89       __ehhandler$??__EalgoLog@U2@@YAXXZ 1001be89 f   DiamondBuildWorker.obj
 0001:0001aeb0       __unwindfunclet$??__EcmdLog@U2@@YAXXZ$0 1001beb0 f   DiamondBuildWorker.obj
 0001:0001aeb9       __ehhandler$??__EcmdLog@U2@@YAXXZ 1001beb9 f   DiamondBuildWorker.obj
 0001:0001aee0       __unwindfunclet$??__EcoreLog@U2@@YAXXZ$0 1001bee0 f   DiamondBuildWorker.obj
 0001:0001aee9       __ehhandler$??__EcoreLog@U2@@YAXXZ 1001bee9 f   DiamondBuildWorker.obj
 0001:0001af10       __unwindfunclet$??__EioLog@U2@@YAXXZ$0 1001bf10 f   DiamondBuildWorker.obj
 0001:0001af19       __ehhandler$??__EioLog@U2@@YAXXZ 1001bf19 f   DiamondBuildWorker.obj
 0001:0001af40       __unwindfunclet$??__EperfLog@U2@@YAXXZ$0 1001bf40 f   DiamondBuildWorker.obj
 0001:0001af49       __ehhandler$??__EperfLog@U2@@YAXXZ 1001bf49 f   DiamondBuildWorker.obj
 0001:0001af70       __unwindfunclet$??__EscriptLog@U2@@YAXXZ$0 1001bf70 f   DiamondBuildWorker.obj
 0001:0001af79       __ehhandler$??__EscriptLog@U2@@YAXXZ 1001bf79 f   DiamondBuildWorker.obj
 0001:0001afa0       __unwindfunclet$??__EtaskLog@U2@@YAXXZ$0 1001bfa0 f   DiamondBuildWorker.obj
 0001:0001afa9       __ehhandler$??__EtaskLog@U2@@YAXXZ 1001bfa9 f   DiamondBuildWorker.obj
 0001:0001afd0       __unwindfunclet$??__EuiLog@U2@@YAXXZ$0 1001bfd0 f   DiamondBuildWorker.obj
 0001:0001afd9       __ehhandler$??__EuiLog@U2@@YAXXZ 1001bfd9 f   DiamondBuildWorker.obj
 0001:0001b000       __unwindfunclet$??__EuserActLog@U2@@YAXXZ$0 1001c000 f   DiamondBuildWorker.obj
 0001:0001b009       __ehhandler$??__EuserActLog@U2@@YAXXZ 1001c009 f   DiamondBuildWorker.obj
 0001:0001b030       __unwindfunclet$?Construct@?$QMetaTypeFunctionHelper@V?$QList@VDataset@U2@@@@$00@QtMetaTypePrivate@@SAPAXPAXPBX@Z$0 1001c030 f   DiamondBuildWorker.obj
 0001:0001b041       __ehhandler$?Construct@?$QMetaTypeFunctionHelper@V?$QList@VDataset@U2@@@@$00@QtMetaTypePrivate@@SAPAXPAXPBX@Z 1001c041 f   DiamondBuildWorker.obj
 0001:0001b060       __unwindfunclet$?Create@?$QMetaTypeFunctionHelper@V?$QList@VDataset@U2@@@@$00@QtMetaTypePrivate@@SAPAXPBX@Z$0 1001c060 f   DiamondBuildWorker.obj
 0001:0001b06b       __ehhandler$?Create@?$QMetaTypeFunctionHelper@V?$QList@VDataset@U2@@@@$00@QtMetaTypePrivate@@SAPAXPBX@Z 1001c06b f   DiamondBuildWorker.obj
 0001:0001b090       __unwindfunclet$?append@?$QList@VDescriptor@U2@@@@QAEXABVDescriptor@U2@@@Z$6 1001c090 f   DiamondBuildWorker.obj
 0001:0001b09b       __ehhandler$?append@?$QList@VDescriptor@U2@@@@QAEXABVDescriptor@U2@@@Z 1001c09b f   DiamondBuildWorker.obj
 0001:0001b0c0       __unwindfunclet$?createNode@?$QMapData@VQString@@VQScriptValue@@@@QAEPAU?$QMapNode@VQString@@VQScriptValue@@@@ABVQString@@ABVQScriptValue@@PAU2@_N@Z$4 1001c0c0 f   DiamondBuildWorker.obj
 0001:0001b0d4       __unwindfunclet$?createNode@?$QMapData@VQString@@VQScriptValue@@@@QAEPAU?$QMapNode@VQString@@VQScriptValue@@@@ABVQString@@ABVQScriptValue@@PAU2@_N@Z$5 1001c0d4 f   DiamondBuildWorker.obj
 0001:0001b0e8       __ehhandler$?createNode@?$QMapData@VQString@@VQScriptValue@@@@QAEPAU?$QMapNode@VQString@@VQScriptValue@@@@ABVQString@@ABVQScriptValue@@PAU2@_N@Z 1001c0e8 f   DiamondBuildWorker.obj
 0001:0001b110       __unwindfunclet$?createNode@?$QMapData@VQString@@VQVariant@@@@QAEPAU?$QMapNode@VQString@@VQVariant@@@@ABVQString@@ABVQVariant@@PAU2@_N@Z$4 1001c110 f   DiamondBuildWorker.obj
 0001:0001b124       __unwindfunclet$?createNode@?$QMapData@VQString@@VQVariant@@@@QAEPAU?$QMapNode@VQString@@VQVariant@@@@ABVQString@@ABVQVariant@@PAU2@_N@Z$5 1001c124 f   DiamondBuildWorker.obj
 0001:0001b138       __ehhandler$?createNode@?$QMapData@VQString@@VQVariant@@@@QAEPAU?$QMapNode@VQString@@VQVariant@@@@ABVQString@@ABVQVariant@@PAU2@_N@Z 1001c138 f   DiamondBuildWorker.obj
 0001:0001b160       __ehhandler$?detach_helper@?$QList@VDescriptor@U2@@@@AAEXH@Z 1001c160 f   DiamondBuildWorker.obj
 0001:0001b180       __ehhandler$?detach_helper_grow@?$QList@VDescriptor@U2@@@@AAEPAUNode@1@HH@Z 1001c180 f   DiamondBuildWorker.obj
 0001:0001b1a0       __unwindfunclet$?getSettings@DiamondBuildWorker@LocalWorkflow@U2@@AAE?AUDiamondBuildTaskSettings@3@AAVU2OpStatus@3@@Z$25 1001c1a0 f   DiamondBuildWorker.obj
 0001:0001b1a9       __unwindfunclet$?getSettings@DiamondBuildWorker@LocalWorkflow@U2@@AAE?AUDiamondBuildTaskSettings@3@AAVU2OpStatus@3@@Z$26 1001c1a9 f   DiamondBuildWorker.obj
 0001:0001b1b1       __unwindfunclet$?getSettings@DiamondBuildWorker@LocalWorkflow@U2@@AAE?AUDiamondBuildTaskSettings@3@AAVU2OpStatus@3@@Z$27 1001c1b1 f   DiamondBuildWorker.obj
 0001:0001b1ba       __unwindfunclet$?getSettings@DiamondBuildWorker@LocalWorkflow@U2@@AAE?AUDiamondBuildTaskSettings@3@AAVU2OpStatus@3@@Z$28 1001c1ba f   DiamondBuildWorker.obj
 0001:0001b1c3       __unwindfunclet$?getSettings@DiamondBuildWorker@LocalWorkflow@U2@@AAE?AUDiamondBuildTaskSettings@3@AAVU2OpStatus@3@@Z$0 1001c1c3 f   DiamondBuildWorker.obj
 0001:0001b1cb       __unwindfunclet$?getSettings@DiamondBuildWorker@LocalWorkflow@U2@@AAE?AUDiamondBuildTaskSettings@3@AAVU2OpStatus@3@@Z$1 1001c1cb f   DiamondBuildWorker.obj
 0001:0001b1d4       __unwindfunclet$?getSettings@DiamondBuildWorker@LocalWorkflow@U2@@AAE?AUDiamondBuildTaskSettings@3@AAVU2OpStatus@3@@Z$2 1001c1d4 f   DiamondBuildWorker.obj
 0001:0001b1dd       __unwindfunclet$?getSettings@DiamondBuildWorker@LocalWorkflow@U2@@AAE?AUDiamondBuildTaskSettings@3@AAVU2OpStatus@3@@Z$3 1001c1dd f   DiamondBuildWorker.obj
 0001:0001b1e6       __unwindfunclet$?getSettings@DiamondBuildWorker@LocalWorkflow@U2@@AAE?AUDiamondBuildTaskSettings@3@AAVU2OpStatus@3@@Z$30 1001c1e6 f   DiamondBuildWorker.obj
 0001:0001b1ee       __unwindfunclet$?getSettings@DiamondBuildWorker@LocalWorkflow@U2@@AAE?AUDiamondBuildTaskSettings@3@AAVU2OpStatus@3@@Z$4 1001c1ee f   DiamondBuildWorker.obj
 0001:0001b1f6       __unwindfunclet$?getSettings@DiamondBuildWorker@LocalWorkflow@U2@@AAE?AUDiamondBuildTaskSettings@3@AAVU2OpStatus@3@@Z$5 1001c1f6 f   DiamondBuildWorker.obj
 0001:0001b1ff       __unwindfunclet$?getSettings@DiamondBuildWorker@LocalWorkflow@U2@@AAE?AUDiamondBuildTaskSettings@3@AAVU2OpStatus@3@@Z$6 1001c1ff f   DiamondBuildWorker.obj
 0001:0001b208       __unwindfunclet$?getSettings@DiamondBuildWorker@LocalWorkflow@U2@@AAE?AUDiamondBuildTaskSettings@3@AAVU2OpStatus@3@@Z$7 1001c208 f   DiamondBuildWorker.obj
 0001:0001b210       __unwindfunclet$?getSettings@DiamondBuildWorker@LocalWorkflow@U2@@AAE?AUDiamondBuildTaskSettings@3@AAVU2OpStatus@3@@Z$8 1001c210 f   DiamondBuildWorker.obj
 0001:0001b219       __unwindfunclet$?getSettings@DiamondBuildWorker@LocalWorkflow@U2@@AAE?AUDiamondBuildTaskSettings@3@AAVU2OpStatus@3@@Z$9 1001c219 f   DiamondBuildWorker.obj
 0001:0001b221       __unwindfunclet$?getSettings@DiamondBuildWorker@LocalWorkflow@U2@@AAE?AUDiamondBuildTaskSettings@3@AAVU2OpStatus@3@@Z$10 1001c221 f   DiamondBuildWorker.obj
 0001:0001b229       __unwindfunclet$?getSettings@DiamondBuildWorker@LocalWorkflow@U2@@AAE?AUDiamondBuildTaskSettings@3@AAVU2OpStatus@3@@Z$11 1001c229 f   DiamondBuildWorker.obj
 0001:0001b231       __unwindfunclet$?getSettings@DiamondBuildWorker@LocalWorkflow@U2@@AAE?AUDiamondBuildTaskSettings@3@AAVU2OpStatus@3@@Z$12 1001c231 f   DiamondBuildWorker.obj
 0001:0001b23a       __unwindfunclet$?getSettings@DiamondBuildWorker@LocalWorkflow@U2@@AAE?AUDiamondBuildTaskSettings@3@AAVU2OpStatus@3@@Z$13 1001c23a f   DiamondBuildWorker.obj
 0001:0001b243       __unwindfunclet$?getSettings@DiamondBuildWorker@LocalWorkflow@U2@@AAE?AUDiamondBuildTaskSettings@3@AAVU2OpStatus@3@@Z$14 1001c243 f   DiamondBuildWorker.obj
 0001:0001b24c       __unwindfunclet$?getSettings@DiamondBuildWorker@LocalWorkflow@U2@@AAE?AUDiamondBuildTaskSettings@3@AAVU2OpStatus@3@@Z$15 1001c24c f   DiamondBuildWorker.obj
 0001:0001b255       __unwindfunclet$?getSettings@DiamondBuildWorker@LocalWorkflow@U2@@AAE?AUDiamondBuildTaskSettings@3@AAVU2OpStatus@3@@Z$16 1001c255 f   DiamondBuildWorker.obj
 0001:0001b25e       __unwindfunclet$?getSettings@DiamondBuildWorker@LocalWorkflow@U2@@AAE?AUDiamondBuildTaskSettings@3@AAVU2OpStatus@3@@Z$17 1001c25e f   DiamondBuildWorker.obj
 0001:0001b267       __unwindfunclet$?getSettings@DiamondBuildWorker@LocalWorkflow@U2@@AAE?AUDiamondBuildTaskSettings@3@AAVU2OpStatus@3@@Z$18 1001c267 f   DiamondBuildWorker.obj
 0001:0001b270       __unwindfunclet$?getSettings@DiamondBuildWorker@LocalWorkflow@U2@@AAE?AUDiamondBuildTaskSettings@3@AAVU2OpStatus@3@@Z$19 1001c270 f   DiamondBuildWorker.obj
 0001:0001b279       __unwindfunclet$?getSettings@DiamondBuildWorker@LocalWorkflow@U2@@AAE?AUDiamondBuildTaskSettings@3@AAVU2OpStatus@3@@Z$35 1001c279 f   DiamondBuildWorker.obj
 0001:0001b282       __unwindfunclet$?getSettings@DiamondBuildWorker@LocalWorkflow@U2@@AAE?AUDiamondBuildTaskSettings@3@AAVU2OpStatus@3@@Z$36 1001c282 f   DiamondBuildWorker.obj
 0001:0001b28d       __unwindfunclet$?getSettings@DiamondBuildWorker@LocalWorkflow@U2@@AAE?AUDiamondBuildTaskSettings@3@AAVU2OpStatus@3@@Z$37 1001c28d f   DiamondBuildWorker.obj
 0001:0001b299       __unwindfunclet$?getSettings@DiamondBuildWorker@LocalWorkflow@U2@@AAE?AUDiamondBuildTaskSettings@3@AAVU2OpStatus@3@@Z$38 1001c299 f   DiamondBuildWorker.obj
 0001:0001b2a5       __unwindfunclet$?getSettings@DiamondBuildWorker@LocalWorkflow@U2@@AAE?AUDiamondBuildTaskSettings@3@AAVU2OpStatus@3@@Z$20 1001c2a5 f   DiamondBuildWorker.obj
 0001:0001b2be       __unwindfunclet$?getSettings@DiamondBuildWorker@LocalWorkflow@U2@@AAE?AUDiamondBuildTaskSettings@3@AAVU2OpStatus@3@@Z$41 1001c2be f   DiamondBuildWorker.obj
 0001:0001b2c7       __unwindfunclet$?getSettings@DiamondBuildWorker@LocalWorkflow@U2@@AAE?AUDiamondBuildTaskSettings@3@AAVU2OpStatus@3@@Z$42 1001c2c7 f   DiamondBuildWorker.obj
 0001:0001b2cf       __unwindfunclet$?getSettings@DiamondBuildWorker@LocalWorkflow@U2@@AAE?AUDiamondBuildTaskSettings@3@AAVU2OpStatus@3@@Z$43 1001c2cf f   DiamondBuildWorker.obj
 0001:0001b2d8       __unwindfunclet$?getSettings@DiamondBuildWorker@LocalWorkflow@U2@@AAE?AUDiamondBuildTaskSettings@3@AAVU2OpStatus@3@@Z$44 1001c2d8 f   DiamondBuildWorker.obj
 0001:0001b2e1       __unwindfunclet$?getSettings@DiamondBuildWorker@LocalWorkflow@U2@@AAE?AUDiamondBuildTaskSettings@3@AAVU2OpStatus@3@@Z$21 1001c2e1 f   DiamondBuildWorker.obj
 0001:0001b2ea       __unwindfunclet$?getSettings@DiamondBuildWorker@LocalWorkflow@U2@@AAE?AUDiamondBuildTaskSettings@3@AAVU2OpStatus@3@@Z$47 1001c2ea f   DiamondBuildWorker.obj
 0001:0001b2f3       __unwindfunclet$?getSettings@DiamondBuildWorker@LocalWorkflow@U2@@AAE?AUDiamondBuildTaskSettings@3@AAVU2OpStatus@3@@Z$48 1001c2f3 f   DiamondBuildWorker.obj
 0001:0001b2fe       __unwindfunclet$?getSettings@DiamondBuildWorker@LocalWorkflow@U2@@AAE?AUDiamondBuildTaskSettings@3@AAVU2OpStatus@3@@Z$49 1001c2fe f   DiamondBuildWorker.obj
 0001:0001b30a       __unwindfunclet$?getSettings@DiamondBuildWorker@LocalWorkflow@U2@@AAE?AUDiamondBuildTaskSettings@3@AAVU2OpStatus@3@@Z$50 1001c30a f   DiamondBuildWorker.obj
 0001:0001b316       __unwindfunclet$?getSettings@DiamondBuildWorker@LocalWorkflow@U2@@AAE?AUDiamondBuildTaskSettings@3@AAVU2OpStatus@3@@Z$53 1001c316 f   DiamondBuildWorker.obj
 0001:0001b31f       __unwindfunclet$?getSettings@DiamondBuildWorker@LocalWorkflow@U2@@AAE?AUDiamondBuildTaskSettings@3@AAVU2OpStatus@3@@Z$54 1001c31f f   DiamondBuildWorker.obj
 0001:0001b327       __unwindfunclet$?getSettings@DiamondBuildWorker@LocalWorkflow@U2@@AAE?AUDiamondBuildTaskSettings@3@AAVU2OpStatus@3@@Z$55 1001c327 f   DiamondBuildWorker.obj
 0001:0001b330       __unwindfunclet$?getSettings@DiamondBuildWorker@LocalWorkflow@U2@@AAE?AUDiamondBuildTaskSettings@3@AAVU2OpStatus@3@@Z$56 1001c330 f   DiamondBuildWorker.obj
 0001:0001b339       __unwindfunclet$?getSettings@DiamondBuildWorker@LocalWorkflow@U2@@AAE?AUDiamondBuildTaskSettings@3@AAVU2OpStatus@3@@Z$23 1001c339 f   DiamondBuildWorker.obj
 0001:0001b342       __unwindfunclet$?getSettings@DiamondBuildWorker@LocalWorkflow@U2@@AAE?AUDiamondBuildTaskSettings@3@AAVU2OpStatus@3@@Z$24 1001c342 f   DiamondBuildWorker.obj
 0001:0001b34b       __unwindfunclet$?getSettings@DiamondBuildWorker@LocalWorkflow@U2@@AAE?AUDiamondBuildTaskSettings@3@AAVU2OpStatus@3@@Z$22 1001c34b f   DiamondBuildWorker.obj
 0001:0001b354       __unwindfunclet$?getSettings@DiamondBuildWorker@LocalWorkflow@U2@@AAE?AUDiamondBuildTaskSettings@3@AAVU2OpStatus@3@@Z$59 1001c354 f   DiamondBuildWorker.obj
 0001:0001b35d       __unwindfunclet$?getSettings@DiamondBuildWorker@LocalWorkflow@U2@@AAE?AUDiamondBuildTaskSettings@3@AAVU2OpStatus@3@@Z$60 1001c35d f   DiamondBuildWorker.obj
 0001:0001b368       __unwindfunclet$?getSettings@DiamondBuildWorker@LocalWorkflow@U2@@AAE?AUDiamondBuildTaskSettings@3@AAVU2OpStatus@3@@Z$61 1001c368 f   DiamondBuildWorker.obj
 0001:0001b374       __unwindfunclet$?getSettings@DiamondBuildWorker@LocalWorkflow@U2@@AAE?AUDiamondBuildTaskSettings@3@AAVU2OpStatus@3@@Z$62 1001c374 f   DiamondBuildWorker.obj
 0001:0001b380       __unwindfunclet$?getSettings@DiamondBuildWorker@LocalWorkflow@U2@@AAE?AUDiamondBuildTaskSettings@3@AAVU2OpStatus@3@@Z$65 1001c380 f   DiamondBuildWorker.obj
 0001:0001b389       __unwindfunclet$?getSettings@DiamondBuildWorker@LocalWorkflow@U2@@AAE?AUDiamondBuildTaskSettings@3@AAVU2OpStatus@3@@Z$66 1001c389 f   DiamondBuildWorker.obj
 0001:0001b391       __unwindfunclet$?getSettings@DiamondBuildWorker@LocalWorkflow@U2@@AAE?AUDiamondBuildTaskSettings@3@AAVU2OpStatus@3@@Z$67 1001c391 f   DiamondBuildWorker.obj
 0001:0001b39a       __unwindfunclet$?getSettings@DiamondBuildWorker@LocalWorkflow@U2@@AAE?AUDiamondBuildTaskSettings@3@AAVU2OpStatus@3@@Z$68 1001c39a f   DiamondBuildWorker.obj
 0001:0001b3a3       __ehhandler$?getSettings@DiamondBuildWorker@LocalWorkflow@U2@@AAE?AUDiamondBuildTaskSettings@3@AAVU2OpStatus@3@@Z 1001c3a3 f   DiamondBuildWorker.obj
 0001:0001b3c0       __unwindfunclet$?init@DiamondBuildWorker@LocalWorkflow@U2@@UAEXXZ$0 1001c3c0 f   DiamondBuildWorker.obj
 0001:0001b3c9       __unwindfunclet$?init@DiamondBuildWorker@LocalWorkflow@U2@@UAEXXZ$1 1001c3c9 f   DiamondBuildWorker.obj
 0001:0001b3d2       __unwindfunclet$?init@DiamondBuildWorker@LocalWorkflow@U2@@UAEXXZ$2 1001c3d2 f   DiamondBuildWorker.obj
 0001:0001b3db       __unwindfunclet$?init@DiamondBuildWorker@LocalWorkflow@U2@@UAEXXZ$3 1001c3db f   DiamondBuildWorker.obj
 0001:0001b3e4       __unwindfunclet$?init@DiamondBuildWorker@LocalWorkflow@U2@@UAEXXZ$4 1001c3e4 f   DiamondBuildWorker.obj
 0001:0001b3ed       __unwindfunclet$?init@DiamondBuildWorker@LocalWorkflow@U2@@UAEXXZ$5 1001c3ed f   DiamondBuildWorker.obj
 0001:0001b3f6       __unwindfunclet$?init@DiamondBuildWorker@LocalWorkflow@U2@@UAEXXZ$6 1001c3f6 f   DiamondBuildWorker.obj
 0001:0001b3ff       __ehhandler$?init@DiamondBuildWorker@LocalWorkflow@U2@@UAEXXZ 1001c3ff f   DiamondBuildWorker.obj
 0001:0001b420       __unwindfunclet$?metaType@?$QVariantValueHelper@V?$QList@VDataset@U2@@@@@QtPrivate@@SA?AV?$QList@VDataset@U2@@@@ABVQVariant@@@Z$0 1001c420 f   DiamondBuildWorker.obj
 0001:0001b439       __unwindfunclet$?metaType@?$QVariantValueHelper@V?$QList@VDataset@U2@@@@@QtPrivate@@SA?AV?$QList@VDataset@U2@@@@ABVQVariant@@@Z$1 1001c439 f   DiamondBuildWorker.obj
 0001:0001b441       __ehhandler$?metaType@?$QVariantValueHelper@V?$QList@VDataset@U2@@@@@QtPrivate@@SA?AV?$QList@VDataset@U2@@@@ABVQVariant@@@Z 1001c441 f   DiamondBuildWorker.obj
 0001:0001b460       __unwindfunclet$?metaType@?$QVariantValueHelper@VQString@@@QtPrivate@@SA?AVQString@@ABVQVariant@@@Z$0 1001c460 f   DiamondBuildWorker.obj
 0001:0001b47a       __unwindfunclet$?metaType@?$QVariantValueHelper@VQString@@@QtPrivate@@SA?AVQString@@ABVQVariant@@@Z$1 1001c47a f   DiamondBuildWorker.obj
 0001:0001b483       __ehhandler$?metaType@?$QVariantValueHelper@VQString@@@QtPrivate@@SA?AVQString@@ABVQVariant@@@Z 1001c483 f   DiamondBuildWorker.obj
 0001:0001b4a0       __unwindfunclet$?node_construct@?$QList@VDescriptor@U2@@@@AAEXPAUNode@1@ABVDescriptor@U2@@@Z$0 1001c4a0 f   DiamondBuildWorker.obj
 0001:0001b4ab       __ehhandler$?node_construct@?$QList@VDescriptor@U2@@@@AAEXPAUNode@1@ABVDescriptor@U2@@@Z 1001c4ab f   DiamondBuildWorker.obj
 0001:0001b4d0       __unwindfunclet$?node_copy@?$QList@VDataset@U2@@@@AAEXPAUNode@1@00@Z$4 1001c4d0 f   DiamondBuildWorker.obj
 0001:0001b4db       __ehhandler$?node_copy@?$QList@VDataset@U2@@@@AAEXPAUNode@1@00@Z 1001c4db f   DiamondBuildWorker.obj
 0001:0001b500       __unwindfunclet$?node_copy@?$QList@VDescriptor@U2@@@@AAEXPAUNode@1@00@Z$4 1001c500 f   DiamondBuildWorker.obj
 0001:0001b50b       __ehhandler$?node_copy@?$QList@VDescriptor@U2@@@@AAEXPAUNode@1@00@Z 1001c50b f   DiamondBuildWorker.obj
 0001:0001b530       __unwindfunclet$?qt_metatype_id@?$QMetaTypeId@V?$QList@VDataset@U2@@@@@@SAHXZ$0 1001c530 f   DiamondBuildWorker.obj
 0001:0001b539       __ehhandler$?qt_metatype_id@?$QMetaTypeId@V?$QList@VDataset@U2@@@@@@SAHXZ 1001c539 f   DiamondBuildWorker.obj
 0001:0001b560       __unwindfunclet$?sl_taskFinished@DiamondBuildWorker@LocalWorkflow@U2@@AAEXPAVTask@3@@Z$0 1001c560 f   DiamondBuildWorker.obj
 0001:0001b569       __unwindfunclet$?sl_taskFinished@DiamondBuildWorker@LocalWorkflow@U2@@AAEXPAVTask@3@@Z$1 1001c569 f   DiamondBuildWorker.obj
 0001:0001b572       __unwindfunclet$?sl_taskFinished@DiamondBuildWorker@LocalWorkflow@U2@@AAEXPAVTask@3@@Z$2 1001c572 f   DiamondBuildWorker.obj
 0001:0001b57b       __unwindfunclet$?sl_taskFinished@DiamondBuildWorker@LocalWorkflow@U2@@AAEXPAVTask@3@@Z$3 1001c57b f   DiamondBuildWorker.obj
 0001:0001b583       __unwindfunclet$?sl_taskFinished@DiamondBuildWorker@LocalWorkflow@U2@@AAEXPAVTask@3@@Z$4 1001c583 f   DiamondBuildWorker.obj
 0001:0001b58c       __unwindfunclet$?sl_taskFinished@DiamondBuildWorker@LocalWorkflow@U2@@AAEXPAVTask@3@@Z$5 1001c58c f   DiamondBuildWorker.obj
 0001:0001b595       __unwindfunclet$?sl_taskFinished@DiamondBuildWorker@LocalWorkflow@U2@@AAEXPAVTask@3@@Z$6 1001c595 f   DiamondBuildWorker.obj
 0001:0001b59e       __unwindfunclet$?sl_taskFinished@DiamondBuildWorker@LocalWorkflow@U2@@AAEXPAVTask@3@@Z$7 1001c59e f   DiamondBuildWorker.obj
 0001:0001b5a7       __unwindfunclet$?sl_taskFinished@DiamondBuildWorker@LocalWorkflow@U2@@AAEXPAVTask@3@@Z$9 1001c5a7 f   DiamondBuildWorker.obj
 0001:0001b5b0       __unwindfunclet$?sl_taskFinished@DiamondBuildWorker@LocalWorkflow@U2@@AAEXPAVTask@3@@Z$10 1001c5b0 f   DiamondBuildWorker.obj
 0001:0001b5b9       __ehhandler$?sl_taskFinished@DiamondBuildWorker@LocalWorkflow@U2@@AAEXPAVTask@3@@Z 1001c5b9 f   DiamondBuildWorker.obj
 0001:0001b5e0       __unwindfunclet$?tick@DiamondBuildWorker@LocalWorkflow@U2@@UAEPAVTask@3@XZ$0 1001c5e0 f   DiamondBuildWorker.obj
 0001:0001b5e9       __unwindfunclet$?tick@DiamondBuildWorker@LocalWorkflow@U2@@UAEPAVTask@3@XZ$1 1001c5e9 f   DiamondBuildWorker.obj
 0001:0001b5f1       __unwindfunclet$?tick@DiamondBuildWorker@LocalWorkflow@U2@@UAEPAVTask@3@XZ$2 1001c5f1 f   DiamondBuildWorker.obj
 0001:0001b5fc       __unwindfunclet$?tick@DiamondBuildWorker@LocalWorkflow@U2@@UAEPAVTask@3@XZ$3 1001c5fc f   DiamondBuildWorker.obj
 0001:0001b616       __unwindfunclet$?tick@DiamondBuildWorker@LocalWorkflow@U2@@UAEPAVTask@3@XZ$4 1001c616 f   DiamondBuildWorker.obj
 0001:0001b621       __unwindfunclet$?tick@DiamondBuildWorker@LocalWorkflow@U2@@UAEPAVTask@3@XZ$5 1001c621 f   DiamondBuildWorker.obj
 0001:0001b629       __unwindfunclet$?tick@DiamondBuildWorker@LocalWorkflow@U2@@UAEPAVTask@3@XZ$6 1001c629 f   DiamondBuildWorker.obj
 0001:0001b634       __unwindfunclet$?tick@DiamondBuildWorker@LocalWorkflow@U2@@UAEPAVTask@3@XZ$8 1001c634 f   DiamondBuildWorker.obj
 0001:0001b63d       __unwindfunclet$?tick@DiamondBuildWorker@LocalWorkflow@U2@@UAEPAVTask@3@XZ$9 1001c63d f   DiamondBuildWorker.obj
 0001:0001b645       __unwindfunclet$?tick@DiamondBuildWorker@LocalWorkflow@U2@@UAEPAVTask@3@XZ$10 1001c645 f   DiamondBuildWorker.obj
 0001:0001b64e       __unwindfunclet$?tick@DiamondBuildWorker@LocalWorkflow@U2@@UAEPAVTask@3@XZ$11 1001c64e f   DiamondBuildWorker.obj
 0001:0001b657       __ehhandler$?tick@DiamondBuildWorker@LocalWorkflow@U2@@UAEPAVTask@3@XZ 1001c657 f   DiamondBuildWorker.obj
 0001:0001b680       __unwindfunclet$?uniqueKeys@?$QMap@VDescriptor@U2@@VQVariant@@@@QBE?AV?$QList@VDescriptor@U2@@@@XZ$1 1001c680 f   DiamondBuildWorker.obj
 0001:0001b699       __ehhandler$?uniqueKeys@?$QMap@VDescriptor@U2@@VQVariant@@@@QBE?AV?$QList@VDescriptor@U2@@@@XZ 1001c699 f   DiamondBuildWorker.obj
 0001:0001b6c0       __unwindfunclet$??A?$QMap@VDescriptor@U2@@V?$QExplicitlySharedDataPointer@VDataType@U2@@@@@@QAEAAV?$QExplicitlySharedDataPointer@VDataType@U2@@@@ABVDescriptor@U2@@@Z$0 1001c6c0 f   DiamondBuildWorkerFactory.obj
 0001:0001b6c8       __ehhandler$??A?$QMap@VDescriptor@U2@@V?$QExplicitlySharedDataPointer@VDataType@U2@@@@@@QAEAAV?$QExplicitlySharedDataPointer@VDataType@U2@@@@ABVDescriptor@U2@@@Z 1001c6c8 f   DiamondBuildWorkerFactory.obj
 0001:0001b6f0       __unwindfunclet$??__EalgoLog@U2@@YAXXZ$0 1001c6f0 f   DiamondBuildWorkerFactory.obj
 0001:0001b6f9       __ehhandler$??__EalgoLog@U2@@YAXXZ 1001c6f9 f   DiamondBuildWorkerFactory.obj
 0001:0001b720       __unwindfunclet$??__EcmdLog@U2@@YAXXZ$0 1001c720 f   DiamondBuildWorkerFactory.obj
 0001:0001b729       __ehhandler$??__EcmdLog@U2@@YAXXZ 1001c729 f   DiamondBuildWorkerFactory.obj
 0001:0001b750       __unwindfunclet$??__EcoreLog@U2@@YAXXZ$0 1001c750 f   DiamondBuildWorkerFactory.obj
 0001:0001b759       __ehhandler$??__EcoreLog@U2@@YAXXZ 1001c759 f   DiamondBuildWorkerFactory.obj
 0001:0001b780       __unwindfunclet$??__EioLog@U2@@YAXXZ$0 1001c780 f   DiamondBuildWorkerFactory.obj
 0001:0001b789       __ehhandler$??__EioLog@U2@@YAXXZ 1001c789 f   DiamondBuildWorkerFactory.obj
 0001:0001b7b0       __unwindfunclet$??__EperfLog@U2@@YAXXZ$0 1001c7b0 f   DiamondBuildWorkerFactory.obj
 0001:0001b7b9       __ehhandler$??__EperfLog@U2@@YAXXZ 1001c7b9 f   DiamondBuildWorkerFactory.obj
 0001:0001b7e0       __unwindfunclet$??__EscriptLog@U2@@YAXXZ$0 1001c7e0 f   DiamondBuildWorkerFactory.obj
 0001:0001b7e9       __ehhandler$??__EscriptLog@U2@@YAXXZ 1001c7e9 f   DiamondBuildWorkerFactory.obj
 0001:0001b810       __unwindfunclet$??__EtaskLog@U2@@YAXXZ$0 1001c810 f   DiamondBuildWorkerFactory.obj
 0001:0001b819       __ehhandler$??__EtaskLog@U2@@YAXXZ 1001c819 f   DiamondBuildWorkerFactory.obj
 0001:0001b840       __unwindfunclet$??__EuiLog@U2@@YAXXZ$0 1001c840 f   DiamondBuildWorkerFactory.obj
 0001:0001b849       __ehhandler$??__EuiLog@U2@@YAXXZ 1001c849 f   DiamondBuildWorkerFactory.obj
 0001:0001b870       __unwindfunclet$??__EuserActLog@U2@@YAXXZ$0 1001c870 f   DiamondBuildWorkerFactory.obj
 0001:0001b879       __ehhandler$??__EuserActLog@U2@@YAXXZ 1001c879 f   DiamondBuildWorkerFactory.obj
 0001:0001b8a0       __ehhandler$?append@?$QList@PAVAttribute@U2@@@@QAEXABQAVAttribute@U2@@@Z 1001c8a0 f   DiamondBuildWorkerFactory.obj
 0001:0001b8c0       __ehhandler$?append@?$QList@PAVPortDescriptor@Workflow@U2@@@@QAEXABQAVPortDescriptor@Workflow@U2@@@Z 1001c8c0 f   DiamondBuildWorkerFactory.obj
 0001:0001b8e0       __unwindfunclet$?createNode@?$QMapData@VDescriptor@U2@@V?$QExplicitlySharedDataPointer@VDataType@U2@@@@@@QAEPAU?$QMapNode@VDescriptor@U2@@V?$QExplicitlySharedDataPointer@VDataType@U2@@@@@@ABVDescriptor@U2@@ABV?$QExplicitlySharedDataPointer@VDataType@U2@@@@PAU2@_N@Z$4 1001c8e0 f   DiamondBuildWorkerFactory.obj
 0001:0001b8f4       __ehhandler$?createNode@?$QMapData@VDescriptor@U2@@V?$QExplicitlySharedDataPointer@VDataType@U2@@@@@@QAEPAU?$QMapNode@VDescriptor@U2@@V?$QExplicitlySharedDataPointer@VDataType@U2@@@@@@ABVDescriptor@U2@@ABV?$QExplicitlySharedDataPointer@VDataType@U2@@@@PAU2@_N@Z 1001c8f4 f   DiamondBuildWorkerFactory.obj
 0001:0001b910       __unwindfunclet$?createNode@?$QMapData@VQString@@PAVPropertyDelegate@U2@@@@QAEPAU?$QMapNode@VQString@@PAVPropertyDelegate@U2@@@@ABVQString@@ABQAVPropertyDelegate@U2@@PAU2@_N@Z$4 1001c910 f   DiamondBuildWorkerFactory.obj
 0001:0001b924       __ehhandler$?createNode@?$QMapData@VQString@@PAVPropertyDelegate@U2@@@@QAEPAU?$QMapNode@VQString@@PAVPropertyDelegate@U2@@@@ABVQString@@ABQAVPropertyDelegate@U2@@PAU2@_N@Z 1001c924 f   DiamondBuildWorkerFactory.obj
 0001:0001b940       __unwindfunclet$?createWorker@DiamondBuildWorkerFactory@LocalWorkflow@U2@@UAEPAVWorker@Workflow@3@PAVActor@53@@Z$0 1001c940 f   DiamondBuildWorkerFactory.obj
 0001:0001b94b       __ehhandler$?createWorker@DiamondBuildWorkerFactory@LocalWorkflow@U2@@UAEPAVWorker@Workflow@3@PAVActor@53@@Z 1001c94b f   DiamondBuildWorkerFactory.obj
 0001:0001b970       __ehhandler$?detach_helper_grow@?$QList@PAVAttribute@U2@@@@AAEPAUNode@1@HH@Z 1001c970 f   DiamondBuildWorkerFactory.obj
 0001:0001b990       __ehhandler$?detach_helper_grow@?$QList@PAVPortDescriptor@Workflow@U2@@@@AAEPAUNode@1@HH@Z 1001c990 f   DiamondBuildWorkerFactory.obj
 0001:0001b9b0       __unwindfunclet$?init@DiamondBuildWorkerFactory@LocalWorkflow@U2@@SAXXZ$0 1001c9b0 f   DiamondBuildWorkerFactory.obj
 0001:0001b9b8       __unwindfunclet$?init@DiamondBuildWorkerFactory@LocalWorkflow@U2@@SAXXZ$1 1001c9b8 f   DiamondBuildWorkerFactory.obj
 0001:0001b9c1       __unwindfunclet$?init@DiamondBuildWorkerFactory@LocalWorkflow@U2@@SAXXZ$2 1001c9c1 f   DiamondBuildWorkerFactory.obj
 0001:0001b9ca       __unwindfunclet$?init@DiamondBuildWorkerFactory@LocalWorkflow@U2@@SAXXZ$3 1001c9ca f   DiamondBuildWorkerFactory.obj
 0001:0001b9d3       __unwindfunclet$?init@DiamondBuildWorkerFactory@LocalWorkflow@U2@@SAXXZ$4 1001c9d3 f   DiamondBuildWorkerFactory.obj
 0001:0001b9dc       __unwindfunclet$?init@DiamondBuildWorkerFactory@LocalWorkflow@U2@@SAXXZ$5 1001c9dc f   DiamondBuildWorkerFactory.obj
 0001:0001b9e5       __unwindfunclet$?init@DiamondBuildWorkerFactory@LocalWorkflow@U2@@SAXXZ$6 1001c9e5 f   DiamondBuildWorkerFactory.obj
 0001:0001b9ed       __unwindfunclet$?init@DiamondBuildWorkerFactory@LocalWorkflow@U2@@SAXXZ$7 1001c9ed f   DiamondBuildWorkerFactory.obj
 0001:0001b9f5       __unwindfunclet$?init@DiamondBuildWorkerFactory@LocalWorkflow@U2@@SAXXZ$8 1001c9f5 f   DiamondBuildWorkerFactory.obj
 0001:0001b9fe       __unwindfunclet$?init@DiamondBuildWorkerFactory@LocalWorkflow@U2@@SAXXZ$9 1001c9fe f   DiamondBuildWorkerFactory.obj
 0001:0001ba07       __unwindfunclet$?init@DiamondBuildWorkerFactory@LocalWorkflow@U2@@SAXXZ$10 1001ca07 f   DiamondBuildWorkerFactory.obj
 0001:0001ba10       __unwindfunclet$?init@DiamondBuildWorkerFactory@LocalWorkflow@U2@@SAXXZ$11 1001ca10 f   DiamondBuildWorkerFactory.obj
 0001:0001ba1b       __unwindfunclet$?init@DiamondBuildWorkerFactory@LocalWorkflow@U2@@SAXXZ$12 1001ca1b f   DiamondBuildWorkerFactory.obj
 0001:0001ba26       __unwindfunclet$?init@DiamondBuildWorkerFactory@LocalWorkflow@U2@@SAXXZ$13 1001ca26 f   DiamondBuildWorkerFactory.obj
 0001:0001ba40       __unwindfunclet$?init@DiamondBuildWorkerFactory@LocalWorkflow@U2@@SAXXZ$14 1001ca40 f   DiamondBuildWorkerFactory.obj
 0001:0001ba5a       __unwindfunclet$?init@DiamondBuildWorkerFactory@LocalWorkflow@U2@@SAXXZ$16 1001ca5a f   DiamondBuildWorkerFactory.obj
 0001:0001ba62       __unwindfunclet$?init@DiamondBuildWorkerFactory@LocalWorkflow@U2@@SAXXZ$17 1001ca62 f   DiamondBuildWorkerFactory.obj
 0001:0001ba6b       __unwindfunclet$?init@DiamondBuildWorkerFactory@LocalWorkflow@U2@@SAXXZ$18 1001ca6b f   DiamondBuildWorkerFactory.obj
 0001:0001ba74       __unwindfunclet$?init@DiamondBuildWorkerFactory@LocalWorkflow@U2@@SAXXZ$19 1001ca74 f   DiamondBuildWorkerFactory.obj
 0001:0001ba7d       __unwindfunclet$?init@DiamondBuildWorkerFactory@LocalWorkflow@U2@@SAXXZ$20 1001ca7d f   DiamondBuildWorkerFactory.obj
 0001:0001ba86       __unwindfunclet$?init@DiamondBuildWorkerFactory@LocalWorkflow@U2@@SAXXZ$21 1001ca86 f   DiamondBuildWorkerFactory.obj
 0001:0001ba8f       __unwindfunclet$?init@DiamondBuildWorkerFactory@LocalWorkflow@U2@@SAXXZ$22 1001ca8f f   DiamondBuildWorkerFactory.obj
 0001:0001ba98       __unwindfunclet$?init@DiamondBuildWorkerFactory@LocalWorkflow@U2@@SAXXZ$23 1001ca98 f   DiamondBuildWorkerFactory.obj
 0001:0001baa3       __unwindfunclet$?init@DiamondBuildWorkerFactory@LocalWorkflow@U2@@SAXXZ$24 1001caa3 f   DiamondBuildWorkerFactory.obj
 0001:0001babd       __unwindfunclet$?init@DiamondBuildWorkerFactory@LocalWorkflow@U2@@SAXXZ$26 1001cabd f   DiamondBuildWorkerFactory.obj
 0001:0001bac8       __unwindfunclet$?init@DiamondBuildWorkerFactory@LocalWorkflow@U2@@SAXXZ$27 1001cac8 f   DiamondBuildWorkerFactory.obj
 0001:0001bae2       __unwindfunclet$?init@DiamondBuildWorkerFactory@LocalWorkflow@U2@@SAXXZ$29 1001cae2 f   DiamondBuildWorkerFactory.obj
 0001:0001baea       __unwindfunclet$?init@DiamondBuildWorkerFactory@LocalWorkflow@U2@@SAXXZ$30 1001caea f   DiamondBuildWorkerFactory.obj
 0001:0001baf3       __unwindfunclet$?init@DiamondBuildWorkerFactory@LocalWorkflow@U2@@SAXXZ$31 1001caf3 f   DiamondBuildWorkerFactory.obj
 0001:0001bafc       __unwindfunclet$?init@DiamondBuildWorkerFactory@LocalWorkflow@U2@@SAXXZ$32 1001cafc f   DiamondBuildWorkerFactory.obj
 0001:0001bb05       __unwindfunclet$?init@DiamondBuildWorkerFactory@LocalWorkflow@U2@@SAXXZ$33 1001cb05 f   DiamondBuildWorkerFactory.obj
 0001:0001bb0d       __unwindfunclet$?init@DiamondBuildWorkerFactory@LocalWorkflow@U2@@SAXXZ$49 1001cb0d f   DiamondBuildWorkerFactory.obj
 0001:0001bb15       __unwindfunclet$?init@DiamondBuildWorkerFactory@LocalWorkflow@U2@@SAXXZ$34 1001cb15 f   DiamondBuildWorkerFactory.obj
 0001:0001bb1d       __unwindfunclet$?init@DiamondBuildWorkerFactory@LocalWorkflow@U2@@SAXXZ$35 1001cb1d f   DiamondBuildWorkerFactory.obj
 0001:0001bb26       __unwindfunclet$?init@DiamondBuildWorkerFactory@LocalWorkflow@U2@@SAXXZ$36 1001cb26 f   DiamondBuildWorkerFactory.obj
 0001:0001bb2f       __unwindfunclet$?init@DiamondBuildWorkerFactory@LocalWorkflow@U2@@SAXXZ$37 1001cb2f f   DiamondBuildWorkerFactory.obj
 0001:0001bb3a       __unwindfunclet$?init@DiamondBuildWorkerFactory@LocalWorkflow@U2@@SAXXZ$38 1001cb3a f   DiamondBuildWorkerFactory.obj
 0001:0001bb54       __unwindfunclet$?init@DiamondBuildWorkerFactory@LocalWorkflow@U2@@SAXXZ$39 1001cb54 f   DiamondBuildWorkerFactory.obj
 0001:0001bb5f       __unwindfunclet$?init@DiamondBuildWorkerFactory@LocalWorkflow@U2@@SAXXZ$40 1001cb5f f   DiamondBuildWorkerFactory.obj
 0001:0001bb68       __unwindfunclet$?init@DiamondBuildWorkerFactory@LocalWorkflow@U2@@SAXXZ$41 1001cb68 f   DiamondBuildWorkerFactory.obj
 0001:0001bb71       __unwindfunclet$?init@DiamondBuildWorkerFactory@LocalWorkflow@U2@@SAXXZ$42 1001cb71 f   DiamondBuildWorkerFactory.obj
 0001:0001bb7d       __unwindfunclet$?init@DiamondBuildWorkerFactory@LocalWorkflow@U2@@SAXXZ$43 1001cb7d f   DiamondBuildWorkerFactory.obj
 0001:0001bb88       __unwindfunclet$?init@DiamondBuildWorkerFactory@LocalWorkflow@U2@@SAXXZ$44 1001cb88 f   DiamondBuildWorkerFactory.obj
 0001:0001bb93       __unwindfunclet$?init@DiamondBuildWorkerFactory@LocalWorkflow@U2@@SAXXZ$45 1001cb93 f   DiamondBuildWorkerFactory.obj
 0001:0001bb9e       __unwindfunclet$?init@DiamondBuildWorkerFactory@LocalWorkflow@U2@@SAXXZ$46 1001cb9e f   DiamondBuildWorkerFactory.obj
 0001:0001bba7       __unwindfunclet$?init@DiamondBuildWorkerFactory@LocalWorkflow@U2@@SAXXZ$47 1001cba7 f   DiamondBuildWorkerFactory.obj
 0001:0001bbb0       __unwindfunclet$?init@DiamondBuildWorkerFactory@LocalWorkflow@U2@@SAXXZ$48 1001cbb0 f   DiamondBuildWorkerFactory.obj
 0001:0001bbbb       __ehhandler$?init@DiamondBuildWorkerFactory@LocalWorkflow@U2@@SAXXZ 1001cbbb f   DiamondBuildWorkerFactory.obj
 0001:0001bbe0       __unwindfunclet$??__EalgoLog@U2@@YAXXZ$0 1001cbe0 f   DiamondClassifyPrompter.obj
 0001:0001bbe9       __ehhandler$??__EalgoLog@U2@@YAXXZ 1001cbe9 f   DiamondClassifyPrompter.obj
 0001:0001bc10       __unwindfunclet$??__EcmdLog@U2@@YAXXZ$0 1001cc10 f   DiamondClassifyPrompter.obj
 0001:0001bc19       __ehhandler$??__EcmdLog@U2@@YAXXZ 1001cc19 f   DiamondClassifyPrompter.obj
 0001:0001bc40       __unwindfunclet$??__EcoreLog@U2@@YAXXZ$0 1001cc40 f   DiamondClassifyPrompter.obj
 0001:0001bc49       __ehhandler$??__EcoreLog@U2@@YAXXZ 1001cc49 f   DiamondClassifyPrompter.obj
 0001:0001bc70       __unwindfunclet$??__EioLog@U2@@YAXXZ$0 1001cc70 f   DiamondClassifyPrompter.obj
 0001:0001bc79       __ehhandler$??__EioLog@U2@@YAXXZ 1001cc79 f   DiamondClassifyPrompter.obj
 0001:0001bca0       __unwindfunclet$??__EperfLog@U2@@YAXXZ$0 1001cca0 f   DiamondClassifyPrompter.obj
 0001:0001bca9       __ehhandler$??__EperfLog@U2@@YAXXZ 1001cca9 f   DiamondClassifyPrompter.obj
 0001:0001bcd0       __unwindfunclet$??__EscriptLog@U2@@YAXXZ$0 1001ccd0 f   DiamondClassifyPrompter.obj
 0001:0001bcd9       __ehhandler$??__EscriptLog@U2@@YAXXZ 1001ccd9 f   DiamondClassifyPrompter.obj
 0001:0001bd00       __unwindfunclet$??__EtaskLog@U2@@YAXXZ$0 1001cd00 f   DiamondClassifyPrompter.obj
 0001:0001bd09       __ehhandler$??__EtaskLog@U2@@YAXXZ 1001cd09 f   DiamondClassifyPrompter.obj
 0001:0001bd30       __unwindfunclet$??__EuiLog@U2@@YAXXZ$0 1001cd30 f   DiamondClassifyPrompter.obj
 0001:0001bd39       __ehhandler$??__EuiLog@U2@@YAXXZ 1001cd39 f   DiamondClassifyPrompter.obj
 0001:0001bd60       __unwindfunclet$??__EuserActLog@U2@@YAXXZ$0 1001cd60 f   DiamondClassifyPrompter.obj
 0001:0001bd69       __ehhandler$??__EuserActLog@U2@@YAXXZ 1001cd69 f   DiamondClassifyPrompter.obj
 0001:0001bd90       __unwindfunclet$?composeRichDoc@DiamondClassifyPrompter@LocalWorkflow@U2@@EAE?AVQString@@XZ$0 1001cd90 f   DiamondClassifyPrompter.obj
 0001:0001bd99       __unwindfunclet$?composeRichDoc@DiamondClassifyPrompter@LocalWorkflow@U2@@EAE?AVQString@@XZ$1 1001cd99 f   DiamondClassifyPrompter.obj
 0001:0001bda2       __unwindfunclet$?composeRichDoc@DiamondClassifyPrompter@LocalWorkflow@U2@@EAE?AVQString@@XZ$2 1001cda2 f   DiamondClassifyPrompter.obj
 0001:0001bdab       __unwindfunclet$?composeRichDoc@DiamondClassifyPrompter@LocalWorkflow@U2@@EAE?AVQString@@XZ$3 1001cdab f   DiamondClassifyPrompter.obj
 0001:0001bdb4       __unwindfunclet$?composeRichDoc@DiamondClassifyPrompter@LocalWorkflow@U2@@EAE?AVQString@@XZ$4 1001cdb4 f   DiamondClassifyPrompter.obj
 0001:0001bdbd       __unwindfunclet$?composeRichDoc@DiamondClassifyPrompter@LocalWorkflow@U2@@EAE?AVQString@@XZ$5 1001cdbd f   DiamondClassifyPrompter.obj
 0001:0001bdc6       __unwindfunclet$?composeRichDoc@DiamondClassifyPrompter@LocalWorkflow@U2@@EAE?AVQString@@XZ$6 1001cdc6 f   DiamondClassifyPrompter.obj
 0001:0001bdcf       __unwindfunclet$?composeRichDoc@DiamondClassifyPrompter@LocalWorkflow@U2@@EAE?AVQString@@XZ$7 1001cdcf f   DiamondClassifyPrompter.obj
 0001:0001bde9       __ehhandler$?composeRichDoc@DiamondClassifyPrompter@LocalWorkflow@U2@@EAE?AVQString@@XZ 1001cde9 f   DiamondClassifyPrompter.obj
 0001:0001be10       __unwindfunclet$?createDescription@?$PrompterBase@VDiamondClassifyPrompter@LocalWorkflow@U2@@@U2@@UAEPAVActorDocument@Workflow@2@PAVActor@42@@Z$0 1001ce10 f   DiamondClassifyPrompter.obj
 0001:0001be1b       __unwindfunclet$?createDescription@?$PrompterBase@VDiamondClassifyPrompter@LocalWorkflow@U2@@@U2@@UAEPAVActorDocument@Workflow@2@PAVActor@42@@Z$3 1001ce1b f   DiamondClassifyPrompter.obj
 0001:0001be23       __unwindfunclet$?createDescription@?$PrompterBase@VDiamondClassifyPrompter@LocalWorkflow@U2@@@U2@@UAEPAVActorDocument@Workflow@2@PAVActor@42@@Z$4 1001ce23 f   DiamondClassifyPrompter.obj
 0001:0001be2b       __unwindfunclet$?createDescription@?$PrompterBase@VDiamondClassifyPrompter@LocalWorkflow@U2@@@U2@@UAEPAVActorDocument@Workflow@2@PAVActor@42@@Z$6 1001ce2b f   DiamondClassifyPrompter.obj
 0001:0001be33       __unwindfunclet$?createDescription@?$PrompterBase@VDiamondClassifyPrompter@LocalWorkflow@U2@@@U2@@UAEPAVActorDocument@Workflow@2@PAVActor@42@@Z$7 1001ce33 f   DiamondClassifyPrompter.obj
 0001:0001be3b       __ehhandler$?createDescription@?$PrompterBase@VDiamondClassifyPrompter@LocalWorkflow@U2@@@U2@@UAEPAVActorDocument@Workflow@2@PAVActor@42@@Z 1001ce3b f   DiamondClassifyPrompter.obj
 0001:0001be60       __unwindfunclet$??0DiamondClassifyTask@U2@@QAE@ABUDiamondClassifyTaskSettings@1@@Z$0 1001ce60 f   DiamondClassifyTask.obj
 0001:0001be69       __unwindfunclet$??0DiamondClassifyTask@U2@@QAE@ABUDiamondClassifyTaskSettings@1@@Z$1 1001ce69 f   DiamondClassifyTask.obj
 0001:0001be72       __unwindfunclet$??0DiamondClassifyTask@U2@@QAE@ABUDiamondClassifyTaskSettings@1@@Z$2 1001ce72 f   DiamondClassifyTask.obj
 0001:0001be80       __unwindfunclet$??0DiamondClassifyTask@U2@@QAE@ABUDiamondClassifyTaskSettings@1@@Z$3 1001ce80 f   DiamondClassifyTask.obj
 0001:0001be8e       __unwindfunclet$??0DiamondClassifyTask@U2@@QAE@ABUDiamondClassifyTaskSettings@1@@Z$4 1001ce8e f   DiamondClassifyTask.obj
 0001:0001be9c       __unwindfunclet$??0DiamondClassifyTask@U2@@QAE@ABUDiamondClassifyTaskSettings@1@@Z$5 1001ce9c f   DiamondClassifyTask.obj
 0001:0001bea5       __unwindfunclet$??0DiamondClassifyTask@U2@@QAE@ABUDiamondClassifyTaskSettings@1@@Z$6 1001cea5 f   DiamondClassifyTask.obj
 0001:0001beae       __unwindfunclet$??0DiamondClassifyTask@U2@@QAE@ABUDiamondClassifyTaskSettings@1@@Z$7 1001ceae f   DiamondClassifyTask.obj
 0001:0001beb7       __ehhandler$??0DiamondClassifyTask@U2@@QAE@ABUDiamondClassifyTaskSettings@1@@Z 1001ceb7 f   DiamondClassifyTask.obj
 0001:0001bee0       __unwindfunclet$??0DiamondClassifyTaskSettings@U2@@QAE@ABU01@@Z$0 1001cee0 f   DiamondClassifyTask.obj
 0001:0001bee9       __unwindfunclet$??0DiamondClassifyTaskSettings@U2@@QAE@ABU01@@Z$1 1001cee9 f   DiamondClassifyTask.obj
 0001:0001bef5       __unwindfunclet$??0DiamondClassifyTaskSettings@U2@@QAE@ABU01@@Z$2 1001cef5 f   DiamondClassifyTask.obj
 0001:0001bf01       __unwindfunclet$??0DiamondClassifyTaskSettings@U2@@QAE@ABU01@@Z$3 1001cf01 f   DiamondClassifyTask.obj
 0001:0001bf0d       __unwindfunclet$??0DiamondClassifyTaskSettings@U2@@QAE@ABU01@@Z$4 1001cf0d f   DiamondClassifyTask.obj
 0001:0001bf19       __unwindfunclet$??0DiamondClassifyTaskSettings@U2@@QAE@ABU01@@Z$5 1001cf19 f   DiamondClassifyTask.obj
 0001:0001bf25       __unwindfunclet$??0DiamondClassifyTaskSettings@U2@@QAE@ABU01@@Z$6 1001cf25 f   DiamondClassifyTask.obj
 0001:0001bf31       __ehhandler$??0DiamondClassifyTaskSettings@U2@@QAE@ABU01@@Z 1001cf31 f   DiamondClassifyTask.obj
 0001:0001bf50       __unwindfunclet$??0DiamondClassifyTaskSettings@U2@@QAE@XZ$0 1001cf50 f   DiamondClassifyTask.obj
 0001:0001bf59       __unwindfunclet$??0DiamondClassifyTaskSettings@U2@@QAE@XZ$1 1001cf59 f   DiamondClassifyTask.obj
 0001:0001bf65       __unwindfunclet$??0DiamondClassifyTaskSettings@U2@@QAE@XZ$2 1001cf65 f   DiamondClassifyTask.obj
 0001:0001bf71       __unwindfunclet$??0DiamondClassifyTaskSettings@U2@@QAE@XZ$3 1001cf71 f   DiamondClassifyTask.obj
 0001:0001bf7d       __unwindfunclet$??0DiamondClassifyTaskSettings@U2@@QAE@XZ$4 1001cf7d f   DiamondClassifyTask.obj
 0001:0001bf89       __unwindfunclet$??0DiamondClassifyTaskSettings@U2@@QAE@XZ$5 1001cf89 f   DiamondClassifyTask.obj
 0001:0001bf95       __unwindfunclet$??0DiamondClassifyTaskSettings@U2@@QAE@XZ$6 1001cf95 f   DiamondClassifyTask.obj
 0001:0001bfa1       __ehhandler$??0DiamondClassifyTaskSettings@U2@@QAE@XZ 1001cfa1 f   DiamondClassifyTask.obj
 0001:0001bfc0       __unwindfunclet$??1DiamondClassifyTask@U2@@UAE@XZ$0 1001cfc0 f   DiamondClassifyTask.obj
 0001:0001bfc9       __unwindfunclet$??1DiamondClassifyTask@U2@@UAE@XZ$1 1001cfc9 f   DiamondClassifyTask.obj
 0001:0001bfd7       __ehhandler$??1DiamondClassifyTask@U2@@UAE@XZ 1001cfd7 f   DiamondClassifyTask.obj
 0001:0001c000       __unwindfunclet$??1DiamondClassifyTaskSettings@U2@@QAE@XZ$0 1001d000 f   DiamondClassifyTask.obj
 0001:0001c009       __unwindfunclet$??1DiamondClassifyTaskSettings@U2@@QAE@XZ$1 1001d009 f   DiamondClassifyTask.obj
 0001:0001c015       __unwindfunclet$??1DiamondClassifyTaskSettings@U2@@QAE@XZ$2 1001d015 f   DiamondClassifyTask.obj
 0001:0001c021       __unwindfunclet$??1DiamondClassifyTaskSettings@U2@@QAE@XZ$3 1001d021 f   DiamondClassifyTask.obj
 0001:0001c02d       __unwindfunclet$??1DiamondClassifyTaskSettings@U2@@QAE@XZ$4 1001d02d f   DiamondClassifyTask.obj
 0001:0001c039       __unwindfunclet$??1DiamondClassifyTaskSettings@U2@@QAE@XZ$5 1001d039 f   DiamondClassifyTask.obj
 0001:0001c045       __unwindfunclet$??1DiamondClassifyTaskSettings@U2@@QAE@XZ$6 1001d045 f   DiamondClassifyTask.obj
 0001:0001c051       __ehhandler$??1DiamondClassifyTaskSettings@U2@@QAE@XZ 1001d051 f   DiamondClassifyTask.obj
 0001:0001c070       __unwindfunclet$??_GDiamondClassifyTask@U2@@UAEPAXI@Z$0 1001d070 f   DiamondClassifyTask.obj
 0001:0001c079       __unwindfunclet$??_GDiamondClassifyTask@U2@@UAEPAXI@Z$1 1001d079 f   DiamondClassifyTask.obj
 0001:0001c087       __ehhandler$??_GDiamondClassifyTask@U2@@UAEPAXI@Z 1001d087 f   DiamondClassifyTask.obj
 0001:0001c0b0       __unwindfunclet$??__EalgoLog@U2@@YAXXZ$0 1001d0b0 f   DiamondClassifyTask.obj
 0001:0001c0b9       __ehhandler$??__EalgoLog@U2@@YAXXZ 1001d0b9 f   DiamondClassifyTask.obj
 0001:0001c0e0       __unwindfunclet$??__EcmdLog@U2@@YAXXZ$0 1001d0e0 f   DiamondClassifyTask.obj
 0001:0001c0e9       __ehhandler$??__EcmdLog@U2@@YAXXZ 1001d0e9 f   DiamondClassifyTask.obj
 0001:0001c110       __unwindfunclet$??__EcoreLog@U2@@YAXXZ$0 1001d110 f   DiamondClassifyTask.obj
 0001:0001c119       __ehhandler$??__EcoreLog@U2@@YAXXZ 1001d119 f   DiamondClassifyTask.obj
 0001:0001c140       __unwindfunclet$??__EioLog@U2@@YAXXZ$0 1001d140 f   DiamondClassifyTask.obj
 0001:0001c149       __ehhandler$??__EioLog@U2@@YAXXZ 1001d149 f   DiamondClassifyTask.obj
 0001:0001c170       __unwindfunclet$??__EperfLog@U2@@YAXXZ$0 1001d170 f   DiamondClassifyTask.obj
 0001:0001c179       __ehhandler$??__EperfLog@U2@@YAXXZ 1001d179 f   DiamondClassifyTask.obj
 0001:0001c1a0       __unwindfunclet$??__EscriptLog@U2@@YAXXZ$0 1001d1a0 f   DiamondClassifyTask.obj
 0001:0001c1a9       __ehhandler$??__EscriptLog@U2@@YAXXZ 1001d1a9 f   DiamondClassifyTask.obj
 0001:0001c1d0       __unwindfunclet$??__EtaskLog@U2@@YAXXZ$0 1001d1d0 f   DiamondClassifyTask.obj
 0001:0001c1d9       __ehhandler$??__EtaskLog@U2@@YAXXZ 1001d1d9 f   DiamondClassifyTask.obj
 0001:0001c200       __unwindfunclet$??__EuiLog@U2@@YAXXZ$0 1001d200 f   DiamondClassifyTask.obj
 0001:0001c209       __ehhandler$??__EuiLog@U2@@YAXXZ 1001d209 f   DiamondClassifyTask.obj
 0001:0001c230       __unwindfunclet$??__EuserActLog@U2@@YAXXZ$0 1001d230 f   DiamondClassifyTask.obj
 0001:0001c239       __ehhandler$??__EuserActLog@U2@@YAXXZ 1001d239 f   DiamondClassifyTask.obj
 0001:0001c260       __unwindfunclet$?checkSettings@DiamondClassifyTask@U2@@AAEXXZ$0 1001d260 f   DiamondClassifyTask.obj
 0001:0001c269       __unwindfunclet$?checkSettings@DiamondClassifyTask@U2@@AAEXXZ$1 1001d269 f   DiamondClassifyTask.obj
 0001:0001c272       __unwindfunclet$?checkSettings@DiamondClassifyTask@U2@@AAEXXZ$2 1001d272 f   DiamondClassifyTask.obj
 0001:0001c27b       __unwindfunclet$?checkSettings@DiamondClassifyTask@U2@@AAEXXZ$3 1001d27b f   DiamondClassifyTask.obj
 0001:0001c284       __unwindfunclet$?checkSettings@DiamondClassifyTask@U2@@AAEXXZ$4 1001d284 f   DiamondClassifyTask.obj
 0001:0001c28d       __unwindfunclet$?checkSettings@DiamondClassifyTask@U2@@AAEXXZ$5 1001d28d f   DiamondClassifyTask.obj
 0001:0001c296       __unwindfunclet$?checkSettings@DiamondClassifyTask@U2@@AAEXXZ$6 1001d296 f   DiamondClassifyTask.obj
 0001:0001c29f       __ehhandler$?checkSettings@DiamondClassifyTask@U2@@AAEXXZ 1001d29f f   DiamondClassifyTask.obj
 0001:0001c2c0       __unwindfunclet$?createNode@?$QMapData@VQString@@I@@QAEPAU?$QMapNode@VQString@@I@@ABVQString@@ABIPAU2@_N@Z$4 1001d2c0 f   DiamondClassifyTask.obj
 0001:0001c2d4       __ehhandler$?createNode@?$QMapData@VQString@@I@@QAEPAU?$QMapNode@VQString@@I@@ABVQString@@ABIPAU2@_N@Z 1001d2d4 f   DiamondClassifyTask.obj
 0001:0001c2f0       __ehhandler$?detach_helper@?$QList@VQByteArray@@@@AAEXH@Z 1001d2f0 f   DiamondClassifyTask.obj
 0001:0001c310       __unwindfunclet$?getArguments@DiamondClassifyTask@U2@@ABE?AVQStringList@@XZ$0 1001d310 f   DiamondClassifyTask.obj
 0001:0001c329       __unwindfunclet$?getArguments@DiamondClassifyTask@U2@@ABE?AVQStringList@@XZ$1 1001d329 f   DiamondClassifyTask.obj
 0001:0001c332       __unwindfunclet$?getArguments@DiamondClassifyTask@U2@@ABE?AVQStringList@@XZ$2 1001d332 f   DiamondClassifyTask.obj
 0001:0001c33b       __unwindfunclet$?getArguments@DiamondClassifyTask@U2@@ABE?AVQStringList@@XZ$3 1001d33b f   DiamondClassifyTask.obj
 0001:0001c344       __unwindfunclet$?getArguments@DiamondClassifyTask@U2@@ABE?AVQStringList@@XZ$4 1001d344 f   DiamondClassifyTask.obj
 0001:0001c34d       __unwindfunclet$?getArguments@DiamondClassifyTask@U2@@ABE?AVQStringList@@XZ$5 1001d34d f   DiamondClassifyTask.obj
 0001:0001c356       __unwindfunclet$?getArguments@DiamondClassifyTask@U2@@ABE?AVQStringList@@XZ$6 1001d356 f   DiamondClassifyTask.obj
 0001:0001c35f       __unwindfunclet$?getArguments@DiamondClassifyTask@U2@@ABE?AVQStringList@@XZ$7 1001d35f f   DiamondClassifyTask.obj
 0001:0001c368       __unwindfunclet$?getArguments@DiamondClassifyTask@U2@@ABE?AVQStringList@@XZ$8 1001d368 f   DiamondClassifyTask.obj
 0001:0001c371       __unwindfunclet$?getArguments@DiamondClassifyTask@U2@@ABE?AVQStringList@@XZ$9 1001d371 f   DiamondClassifyTask.obj
 0001:0001c37a       __unwindfunclet$?getArguments@DiamondClassifyTask@U2@@ABE?AVQStringList@@XZ$10 1001d37a f   DiamondClassifyTask.obj
 0001:0001c383       __unwindfunclet$?getArguments@DiamondClassifyTask@U2@@ABE?AVQStringList@@XZ$11 1001d383 f   DiamondClassifyTask.obj
 0001:0001c38c       __unwindfunclet$?getArguments@DiamondClassifyTask@U2@@ABE?AVQStringList@@XZ$12 1001d38c f   DiamondClassifyTask.obj
 0001:0001c395       __unwindfunclet$?getArguments@DiamondClassifyTask@U2@@ABE?AVQStringList@@XZ$13 1001d395 f   DiamondClassifyTask.obj
 0001:0001c39e       __unwindfunclet$?getArguments@DiamondClassifyTask@U2@@ABE?AVQStringList@@XZ$14 1001d39e f   DiamondClassifyTask.obj
 0001:0001c3a7       __unwindfunclet$?getArguments@DiamondClassifyTask@U2@@ABE?AVQStringList@@XZ$15 1001d3a7 f   DiamondClassifyTask.obj
 0001:0001c3b0       __unwindfunclet$?getArguments@DiamondClassifyTask@U2@@ABE?AVQStringList@@XZ$16 1001d3b0 f   DiamondClassifyTask.obj
 0001:0001c3b9       __unwindfunclet$?getArguments@DiamondClassifyTask@U2@@ABE?AVQStringList@@XZ$17 1001d3b9 f   DiamondClassifyTask.obj
 0001:0001c3c2       __unwindfunclet$?getArguments@DiamondClassifyTask@U2@@ABE?AVQStringList@@XZ$18 1001d3c2 f   DiamondClassifyTask.obj
 0001:0001c3cb       __unwindfunclet$?getArguments@DiamondClassifyTask@U2@@ABE?AVQStringList@@XZ$19 1001d3cb f   DiamondClassifyTask.obj
 0001:0001c3d4       __unwindfunclet$?getArguments@DiamondClassifyTask@U2@@ABE?AVQStringList@@XZ$20 1001d3d4 f   DiamondClassifyTask.obj
 0001:0001c3dd       __unwindfunclet$?getArguments@DiamondClassifyTask@U2@@ABE?AVQStringList@@XZ$21 1001d3dd f   DiamondClassifyTask.obj
 0001:0001c3e6       __unwindfunclet$?getArguments@DiamondClassifyTask@U2@@ABE?AVQStringList@@XZ$22 1001d3e6 f   DiamondClassifyTask.obj
 0001:0001c3ef       __unwindfunclet$?getArguments@DiamondClassifyTask@U2@@ABE?AVQStringList@@XZ$23 1001d3ef f   DiamondClassifyTask.obj
 0001:0001c3f8       __unwindfunclet$?getArguments@DiamondClassifyTask@U2@@ABE?AVQStringList@@XZ$24 1001d3f8 f   DiamondClassifyTask.obj
 0001:0001c401       __unwindfunclet$?getArguments@DiamondClassifyTask@U2@@ABE?AVQStringList@@XZ$25 1001d401 f   DiamondClassifyTask.obj
 0001:0001c40a       __unwindfunclet$?getArguments@DiamondClassifyTask@U2@@ABE?AVQStringList@@XZ$26 1001d40a f   DiamondClassifyTask.obj
 0001:0001c413       __unwindfunclet$?getArguments@DiamondClassifyTask@U2@@ABE?AVQStringList@@XZ$27 1001d413 f   DiamondClassifyTask.obj
 0001:0001c41c       __unwindfunclet$?getArguments@DiamondClassifyTask@U2@@ABE?AVQStringList@@XZ$28 1001d41c f   DiamondClassifyTask.obj
 0001:0001c425       __ehhandler$?getArguments@DiamondClassifyTask@U2@@ABE?AVQStringList@@XZ 1001d425 f   DiamondClassifyTask.obj
 0001:0001c440       __unwindfunclet$?node_copy@?$QList@VQByteArray@@@@AAEXPAUNode@1@00@Z$5 1001d440 f   DiamondClassifyTask.obj
 0001:0001c451       __ehhandler$?node_copy@?$QList@VQByteArray@@@@AAEXPAUNode@1@00@Z 1001d451 f   DiamondClassifyTask.obj
 0001:0001c470       __unwindfunclet$?prepare@DiamondClassifyTask@U2@@EAEXXZ$0 1001d470 f   DiamondClassifyTask.obj
 0001:0001c47b       __unwindfunclet$?prepare@DiamondClassifyTask@U2@@EAEXXZ$1 1001d47b f   DiamondClassifyTask.obj
 0001:0001c495       __unwindfunclet$?prepare@DiamondClassifyTask@U2@@EAEXXZ$2 1001d495 f   DiamondClassifyTask.obj
 0001:0001c4a0       __unwindfunclet$?prepare@DiamondClassifyTask@U2@@EAEXXZ$3 1001d4a0 f   DiamondClassifyTask.obj
 0001:0001c4ba       __unwindfunclet$?prepare@DiamondClassifyTask@U2@@EAEXXZ$4 1001d4ba f   DiamondClassifyTask.obj
 0001:0001c4d3       __unwindfunclet$?prepare@DiamondClassifyTask@U2@@EAEXXZ$5 1001d4d3 f   DiamondClassifyTask.obj
 0001:0001c4ec       __ehhandler$?prepare@DiamondClassifyTask@U2@@EAEXXZ 1001d4ec f   DiamondClassifyTask.obj
 0001:0001c510       __unwindfunclet$?run@DiamondClassifyTask@U2@@EAEXXZ$0 1001d510 f   DiamondClassifyTask.obj
 0001:0001c519       __unwindfunclet$?run@DiamondClassifyTask@U2@@EAEXXZ$1 1001d519 f   DiamondClassifyTask.obj
 0001:0001c522       __unwindfunclet$?run@DiamondClassifyTask@U2@@EAEXXZ$2 1001d522 f   DiamondClassifyTask.obj
 0001:0001c52b       __unwindfunclet$?run@DiamondClassifyTask@U2@@EAEXXZ$3 1001d52b f   DiamondClassifyTask.obj
 0001:0001c534       __unwindfunclet$?run@DiamondClassifyTask@U2@@EAEXXZ$4 1001d534 f   DiamondClassifyTask.obj
 0001:0001c53d       __unwindfunclet$?run@DiamondClassifyTask@U2@@EAEXXZ$5 1001d53d f   DiamondClassifyTask.obj
 0001:0001c545       __unwindfunclet$?run@DiamondClassifyTask@U2@@EAEXXZ$6 1001d545 f   DiamondClassifyTask.obj
 0001:0001c54e       __unwindfunclet$?run@DiamondClassifyTask@U2@@EAEXXZ$7 1001d54e f   DiamondClassifyTask.obj
 0001:0001c557       __unwindfunclet$?run@DiamondClassifyTask@U2@@EAEXXZ$8 1001d557 f   DiamondClassifyTask.obj
 0001:0001c560       __unwindfunclet$?run@DiamondClassifyTask@U2@@EAEXXZ$9 1001d560 f   DiamondClassifyTask.obj
 0001:0001c569       __unwindfunclet$?run@DiamondClassifyTask@U2@@EAEXXZ$10 1001d569 f   DiamondClassifyTask.obj
 0001:0001c572       __unwindfunclet$?run@DiamondClassifyTask@U2@@EAEXXZ$11 1001d572 f   DiamondClassifyTask.obj
 0001:0001c57b       __unwindfunclet$?run@DiamondClassifyTask@U2@@EAEXXZ$12 1001d57b f   DiamondClassifyTask.obj
 0001:0001c584       __unwindfunclet$?run@DiamondClassifyTask@U2@@EAEXXZ$13 1001d584 f   DiamondClassifyTask.obj
 0001:0001c58d       __unwindfunclet$?run@DiamondClassifyTask@U2@@EAEXXZ$14 1001d58d f   DiamondClassifyTask.obj
 0001:0001c596       __ehhandler$?run@DiamondClassifyTask@U2@@EAEXXZ 1001d596 f   DiamondClassifyTask.obj
 0001:0001c5c0       __unwindfunclet$??$getAttributeValue@H@Attribute@U2@@QBEHPAVWorkflowContext@Workflow@1@@Z$0 1001d5c0 f   DiamondClassifyWorker.obj
 0001:0001c5c9       __unwindfunclet$??$getAttributeValue@H@Attribute@U2@@QBEHPAVWorkflowContext@Workflow@1@@Z$1 1001d5c9 f   DiamondClassifyWorker.obj
 0001:0001c5d1       __unwindfunclet$??$getAttributeValue@H@Attribute@U2@@QBEHPAVWorkflowContext@Workflow@1@@Z$2 1001d5d1 f   DiamondClassifyWorker.obj
 0001:0001c5d9       __unwindfunclet$??$getAttributeValue@H@Attribute@U2@@QBEHPAVWorkflowContext@Workflow@1@@Z$3 1001d5d9 f   DiamondClassifyWorker.obj
 0001:0001c5e1       __unwindfunclet$??$getAttributeValue@H@Attribute@U2@@QBEHPAVWorkflowContext@Workflow@1@@Z$4 1001d5e1 f   DiamondClassifyWorker.obj
 0001:0001c5ea       __unwindfunclet$??$getAttributeValue@H@Attribute@U2@@QBEHPAVWorkflowContext@Workflow@1@@Z$5 1001d5ea f   DiamondClassifyWorker.obj
 0001:0001c5f3       __unwindfunclet$??$getAttributeValue@H@Attribute@U2@@QBEHPAVWorkflowContext@Workflow@1@@Z$6 1001d5f3 f   DiamondClassifyWorker.obj
 0001:0001c5fc       __unwindfunclet$??$getAttributeValue@H@Attribute@U2@@QBEHPAVWorkflowContext@Workflow@1@@Z$7 1001d5fc f   DiamondClassifyWorker.obj
 0001:0001c605       __unwindfunclet$??$getAttributeValue@H@Attribute@U2@@QBEHPAVWorkflowContext@Workflow@1@@Z$8 1001d605 f   DiamondClassifyWorker.obj
 0001:0001c60e       __unwindfunclet$??$getAttributeValue@H@Attribute@U2@@QBEHPAVWorkflowContext@Workflow@1@@Z$9 1001d60e f   DiamondClassifyWorker.obj
 0001:0001c617       __unwindfunclet$??$getAttributeValue@H@Attribute@U2@@QBEHPAVWorkflowContext@Workflow@1@@Z$10 1001d617 f   DiamondClassifyWorker.obj
 0001:0001c620       __unwindfunclet$??$getAttributeValue@H@Attribute@U2@@QBEHPAVWorkflowContext@Workflow@1@@Z$11 1001d620 f   DiamondClassifyWorker.obj
 0001:0001c629       __ehhandler$??$getAttributeValue@H@Attribute@U2@@QBEHPAVWorkflowContext@Workflow@1@@Z 1001d629 f   DiamondClassifyWorker.obj
 0001:0001c650       __unwindfunclet$??$qRegisterMetaType@V?$QMap@VQString@@I@@@@YAHPBDPAV?$QMap@VQString@@I@@W4DefinedType@?$MetaTypeDefinedHelper@V?$QMap@VQString@@I@@$00@QtPrivate@@@Z$0 1001d650 f   DiamondClassifyWorker.obj
 0001:0001c659       __ehhandler$??$qRegisterMetaType@V?$QMap@VQString@@I@@@@YAHPBDPAV?$QMap@VQString@@I@@W4DefinedType@?$MetaTypeDefinedHelper@V?$QMap@VQString@@I@@$00@QtPrivate@@@Z 1001d659 f   DiamondClassifyWorker.obj
 0001:0001c680       __unwindfunclet$??$qRegisterMetaType@VQAssociativeIterableImpl@QtMetaTypePrivate@@@@YAHPBDPAVQAssociativeIterableImpl@QtMetaTypePrivate@@W4DefinedType@?$MetaTypeDefinedHelper@VQAssociativeIterableImpl@QtMetaTypePrivate@@$00@QtPrivate@@@Z$0 1001d680 f   DiamondClassifyWorker.obj
 0001:0001c689       __ehhandler$??$qRegisterMetaType@VQAssociativeIterableImpl@QtMetaTypePrivate@@@@YAHPBDPAVQAssociativeIterableImpl@QtMetaTypePrivate@@W4DefinedType@?$MetaTypeDefinedHelper@VQAssociativeIterableImpl@QtMetaTypePrivate@@$00@QtPrivate@@@Z 1001d689 f   DiamondClassifyWorker.obj
 0001:0001c6b0       __unwindfunclet$??__EalgoLog@U2@@YAXXZ$0 1001d6b0 f   DiamondClassifyWorker.obj
 0001:0001c6b9       __ehhandler$??__EalgoLog@U2@@YAXXZ 1001d6b9 f   DiamondClassifyWorker.obj
 0001:0001c6e0       __unwindfunclet$??__EcmdLog@U2@@YAXXZ$0 1001d6e0 f   DiamondClassifyWorker.obj
 0001:0001c6e9       __ehhandler$??__EcmdLog@U2@@YAXXZ 1001d6e9 f   DiamondClassifyWorker.obj
 0001:0001c710       __unwindfunclet$??__EcoreLog@U2@@YAXXZ$0 1001d710 f   DiamondClassifyWorker.obj
 0001:0001c719       __ehhandler$??__EcoreLog@U2@@YAXXZ 1001d719 f   DiamondClassifyWorker.obj
 0001:0001c740       __unwindfunclet$??__EioLog@U2@@YAXXZ$0 1001d740 f   DiamondClassifyWorker.obj
 0001:0001c749       __ehhandler$??__EioLog@U2@@YAXXZ 1001d749 f   DiamondClassifyWorker.obj
 0001:0001c770       __unwindfunclet$??__EperfLog@U2@@YAXXZ$0 1001d770 f   DiamondClassifyWorker.obj
 0001:0001c779       __ehhandler$??__EperfLog@U2@@YAXXZ 1001d779 f   DiamondClassifyWorker.obj
 0001:0001c7a0       __unwindfunclet$??__EscriptLog@U2@@YAXXZ$0 1001d7a0 f   DiamondClassifyWorker.obj
 0001:0001c7a9       __ehhandler$??__EscriptLog@U2@@YAXXZ 1001d7a9 f   DiamondClassifyWorker.obj
 0001:0001c7d0       __unwindfunclet$??__EtaskLog@U2@@YAXXZ$0 1001d7d0 f   DiamondClassifyWorker.obj
 0001:0001c7d9       __ehhandler$??__EtaskLog@U2@@YAXXZ 1001d7d9 f   DiamondClassifyWorker.obj
 0001:0001c800       __unwindfunclet$??__EuiLog@U2@@YAXXZ$0 1001d800 f   DiamondClassifyWorker.obj
 0001:0001c809       __ehhandler$??__EuiLog@U2@@YAXXZ 1001d809 f   DiamondClassifyWorker.obj
 0001:0001c830       __unwindfunclet$??__EuserActLog@U2@@YAXXZ$0 1001d830 f   DiamondClassifyWorker.obj
 0001:0001c839       __ehhandler$??__EuserActLog@U2@@YAXXZ 1001d839 f   DiamondClassifyWorker.obj
 0001:0001c860       __unwindfunclet$?Construct@?$QMetaTypeFunctionHelper@V?$QMap@VQString@@I@@$00@QtMetaTypePrivate@@SAPAXPAXPBX@Z$0 1001d860 f   DiamondClassifyWorker.obj
 0001:0001c871       __ehhandler$?Construct@?$QMetaTypeFunctionHelper@V?$QMap@VQString@@I@@$00@QtMetaTypePrivate@@SAPAXPAXPBX@Z 1001d871 f   DiamondClassifyWorker.obj
 0001:0001c890       __unwindfunclet$?Create@?$QMetaTypeFunctionHelper@V?$QMap@VQString@@I@@$00@QtMetaTypePrivate@@SAPAXPBX@Z$0 1001d890 f   DiamondClassifyWorker.obj
 0001:0001c89b       __ehhandler$?Create@?$QMetaTypeFunctionHelper@V?$QMap@VQString@@I@@$00@QtMetaTypePrivate@@SAPAXPBX@Z 1001d89b f   DiamondClassifyWorker.obj
 0001:0001c8c0       __unwindfunclet$?getSettings@DiamondClassifyWorker@LocalWorkflow@U2@@AAE?AUDiamondClassifyTaskSettings@3@AAVU2OpStatus@3@@Z$0 1001d8c0 f   DiamondClassifyWorker.obj
 0001:0001c8d9       __unwindfunclet$?getSettings@DiamondClassifyWorker@LocalWorkflow@U2@@AAE?AUDiamondClassifyTaskSettings@3@AAVU2OpStatus@3@@Z$1 1001d8d9 f   DiamondClassifyWorker.obj
 0001:0001c8e2       __unwindfunclet$?getSettings@DiamondClassifyWorker@LocalWorkflow@U2@@AAE?AUDiamondClassifyTaskSettings@3@AAVU2OpStatus@3@@Z$2 1001d8e2 f   DiamondClassifyWorker.obj
 0001:0001c8eb       __unwindfunclet$?getSettings@DiamondClassifyWorker@LocalWorkflow@U2@@AAE?AUDiamondClassifyTaskSettings@3@AAVU2OpStatus@3@@Z$3 1001d8eb f   DiamondClassifyWorker.obj
 0001:0001c8f4       __unwindfunclet$?getSettings@DiamondClassifyWorker@LocalWorkflow@U2@@AAE?AUDiamondClassifyTaskSettings@3@AAVU2OpStatus@3@@Z$4 1001d8f4 f   DiamondClassifyWorker.obj
 0001:0001c8fc       __unwindfunclet$?getSettings@DiamondClassifyWorker@LocalWorkflow@U2@@AAE?AUDiamondClassifyTaskSettings@3@AAVU2OpStatus@3@@Z$5 1001d8fc f   DiamondClassifyWorker.obj
 0001:0001c905       __unwindfunclet$?getSettings@DiamondClassifyWorker@LocalWorkflow@U2@@AAE?AUDiamondClassifyTaskSettings@3@AAVU2OpStatus@3@@Z$6 1001d905 f   DiamondClassifyWorker.obj
 0001:0001c90e       __unwindfunclet$?getSettings@DiamondClassifyWorker@LocalWorkflow@U2@@AAE?AUDiamondClassifyTaskSettings@3@AAVU2OpStatus@3@@Z$7 1001d90e f   DiamondClassifyWorker.obj
 0001:0001c917       __unwindfunclet$?getSettings@DiamondClassifyWorker@LocalWorkflow@U2@@AAE?AUDiamondClassifyTaskSettings@3@AAVU2OpStatus@3@@Z$8 1001d917 f   DiamondClassifyWorker.obj
 0001:0001c920       __unwindfunclet$?getSettings@DiamondClassifyWorker@LocalWorkflow@U2@@AAE?AUDiamondClassifyTaskSettings@3@AAVU2OpStatus@3@@Z$9 1001d920 f   DiamondClassifyWorker.obj
 0001:0001c929       __unwindfunclet$?getSettings@DiamondClassifyWorker@LocalWorkflow@U2@@AAE?AUDiamondClassifyTaskSettings@3@AAVU2OpStatus@3@@Z$10 1001d929 f   DiamondClassifyWorker.obj
 0001:0001c932       __unwindfunclet$?getSettings@DiamondClassifyWorker@LocalWorkflow@U2@@AAE?AUDiamondClassifyTaskSettings@3@AAVU2OpStatus@3@@Z$11 1001d932 f   DiamondClassifyWorker.obj
 0001:0001c93b       __unwindfunclet$?getSettings@DiamondClassifyWorker@LocalWorkflow@U2@@AAE?AUDiamondClassifyTaskSettings@3@AAVU2OpStatus@3@@Z$12 1001d93b f   DiamondClassifyWorker.obj
 0001:0001c944       __unwindfunclet$?getSettings@DiamondClassifyWorker@LocalWorkflow@U2@@AAE?AUDiamondClassifyTaskSettings@3@AAVU2OpStatus@3@@Z$13 1001d944 f   DiamondClassifyWorker.obj
 0001:0001c94d       __unwindfunclet$?getSettings@DiamondClassifyWorker@LocalWorkflow@U2@@AAE?AUDiamondClassifyTaskSettings@3@AAVU2OpStatus@3@@Z$14 1001d94d f   DiamondClassifyWorker.obj
 0001:0001c956       __unwindfunclet$?getSettings@DiamondClassifyWorker@LocalWorkflow@U2@@AAE?AUDiamondClassifyTaskSettings@3@AAVU2OpStatus@3@@Z$15 1001d956 f   DiamondClassifyWorker.obj
 0001:0001c95f       __unwindfunclet$?getSettings@DiamondClassifyWorker@LocalWorkflow@U2@@AAE?AUDiamondClassifyTaskSettings@3@AAVU2OpStatus@3@@Z$16 1001d95f f   DiamondClassifyWorker.obj
 0001:0001c979       __unwindfunclet$?getSettings@DiamondClassifyWorker@LocalWorkflow@U2@@AAE?AUDiamondClassifyTaskSettings@3@AAVU2OpStatus@3@@Z$17 1001d979 f   DiamondClassifyWorker.obj
 0001:0001c993       __unwindfunclet$?getSettings@DiamondClassifyWorker@LocalWorkflow@U2@@AAE?AUDiamondClassifyTaskSettings@3@AAVU2OpStatus@3@@Z$18 1001d993 f   DiamondClassifyWorker.obj
 0001:0001c9ad       __unwindfunclet$?getSettings@DiamondClassifyWorker@LocalWorkflow@U2@@AAE?AUDiamondClassifyTaskSettings@3@AAVU2OpStatus@3@@Z$19 1001d9ad f   DiamondClassifyWorker.obj
 0001:0001c9c7       __unwindfunclet$?getSettings@DiamondClassifyWorker@LocalWorkflow@U2@@AAE?AUDiamondClassifyTaskSettings@3@AAVU2OpStatus@3@@Z$20 1001d9c7 f   DiamondClassifyWorker.obj
 0001:0001c9e0       __unwindfunclet$?getSettings@DiamondClassifyWorker@LocalWorkflow@U2@@AAE?AUDiamondClassifyTaskSettings@3@AAVU2OpStatus@3@@Z$21 1001d9e0 f   DiamondClassifyWorker.obj
 0001:0001c9fa       __unwindfunclet$?getSettings@DiamondClassifyWorker@LocalWorkflow@U2@@AAE?AUDiamondClassifyTaskSettings@3@AAVU2OpStatus@3@@Z$22 1001d9fa f   DiamondClassifyWorker.obj
 0001:0001ca03       __unwindfunclet$?getSettings@DiamondClassifyWorker@LocalWorkflow@U2@@AAE?AUDiamondClassifyTaskSettings@3@AAVU2OpStatus@3@@Z$23 1001da03 f   DiamondClassifyWorker.obj
 0001:0001ca0c       __unwindfunclet$?getSettings@DiamondClassifyWorker@LocalWorkflow@U2@@AAE?AUDiamondClassifyTaskSettings@3@AAVU2OpStatus@3@@Z$24 1001da0c f   DiamondClassifyWorker.obj
 0001:0001ca15       __unwindfunclet$?getSettings@DiamondClassifyWorker@LocalWorkflow@U2@@AAE?AUDiamondClassifyTaskSettings@3@AAVU2OpStatus@3@@Z$25 1001da15 f   DiamondClassifyWorker.obj
 0001:0001ca1d       __unwindfunclet$?getSettings@DiamondClassifyWorker@LocalWorkflow@U2@@AAE?AUDiamondClassifyTaskSettings@3@AAVU2OpStatus@3@@Z$26 1001da1d f   DiamondClassifyWorker.obj
 0001:0001ca26       __unwindfunclet$?getSettings@DiamondClassifyWorker@LocalWorkflow@U2@@AAE?AUDiamondClassifyTaskSettings@3@AAVU2OpStatus@3@@Z$27 1001da26 f   DiamondClassifyWorker.obj
 0001:0001ca2f       __unwindfunclet$?getSettings@DiamondClassifyWorker@LocalWorkflow@U2@@AAE?AUDiamondClassifyTaskSettings@3@AAVU2OpStatus@3@@Z$28 1001da2f f   DiamondClassifyWorker.obj
 0001:0001ca38       __ehhandler$?getSettings@DiamondClassifyWorker@LocalWorkflow@U2@@AAE?AUDiamondClassifyTaskSettings@3@AAVU2OpStatus@3@@Z 1001da38 f   DiamondClassifyWorker.obj
 0001:0001ca60       __unwindfunclet$?init@DiamondClassifyWorker@LocalWorkflow@U2@@UAEXXZ$0 1001da60 f   DiamondClassifyWorker.obj
 0001:0001ca69       __unwindfunclet$?init@DiamondClassifyWorker@LocalWorkflow@U2@@UAEXXZ$1 1001da69 f   DiamondClassifyWorker.obj
 0001:0001ca72       __unwindfunclet$?init@DiamondClassifyWorker@LocalWorkflow@U2@@UAEXXZ$2 1001da72 f   DiamondClassifyWorker.obj
 0001:0001ca7b       __unwindfunclet$?init@DiamondClassifyWorker@LocalWorkflow@U2@@UAEXXZ$3 1001da7b f   DiamondClassifyWorker.obj
 0001:0001ca84       __unwindfunclet$?init@DiamondClassifyWorker@LocalWorkflow@U2@@UAEXXZ$4 1001da84 f   DiamondClassifyWorker.obj
 0001:0001ca8d       __unwindfunclet$?init@DiamondClassifyWorker@LocalWorkflow@U2@@UAEXXZ$5 1001da8d f   DiamondClassifyWorker.obj
 0001:0001ca96       __unwindfunclet$?init@DiamondClassifyWorker@LocalWorkflow@U2@@UAEXXZ$6 1001da96 f   DiamondClassifyWorker.obj
 0001:0001ca9f       __unwindfunclet$?init@DiamondClassifyWorker@LocalWorkflow@U2@@UAEXXZ$7 1001da9f f   DiamondClassifyWorker.obj
 0001:0001caa8       __unwindfunclet$?init@DiamondClassifyWorker@LocalWorkflow@U2@@UAEXXZ$8 1001daa8 f   DiamondClassifyWorker.obj
 0001:0001cab1       __unwindfunclet$?init@DiamondClassifyWorker@LocalWorkflow@U2@@UAEXXZ$9 1001dab1 f   DiamondClassifyWorker.obj
 0001:0001caba       __unwindfunclet$?init@DiamondClassifyWorker@LocalWorkflow@U2@@UAEXXZ$10 1001daba f   DiamondClassifyWorker.obj
 0001:0001cac3       __unwindfunclet$?init@DiamondClassifyWorker@LocalWorkflow@U2@@UAEXXZ$11 1001dac3 f   DiamondClassifyWorker.obj
 0001:0001cacc       __unwindfunclet$?init@DiamondClassifyWorker@LocalWorkflow@U2@@UAEXXZ$12 1001dacc f   DiamondClassifyWorker.obj
 0001:0001cad5       __unwindfunclet$?init@DiamondClassifyWorker@LocalWorkflow@U2@@UAEXXZ$13 1001dad5 f   DiamondClassifyWorker.obj
 0001:0001cade       __ehhandler$?init@DiamondClassifyWorker@LocalWorkflow@U2@@UAEXXZ 1001dade f   DiamondClassifyWorker.obj
 0001:0001cb00       __unwindfunclet$?qt_metatype_id@?$QMetaTypeId@V?$QMap@VQString@@I@@@@SAHXZ$0 1001db00 f   DiamondClassifyWorker.obj
 0001:0001cb09       __ehhandler$?qt_metatype_id@?$QMetaTypeId@V?$QMap@VQString@@I@@@@SAHXZ 1001db09 f   DiamondClassifyWorker.obj
 0001:0001cb30       __unwindfunclet$?qt_metatype_id@?$QMetaTypeId@VQAssociativeIterableImpl@QtMetaTypePrivate@@@@SAHXZ$0 1001db30 f   DiamondClassifyWorker.obj
 0001:0001cb39       __ehhandler$?qt_metatype_id@?$QMetaTypeId@VQAssociativeIterableImpl@QtMetaTypePrivate@@@@SAHXZ 1001db39 f   DiamondClassifyWorker.obj
 0001:0001cb60       __unwindfunclet$?sl_taskFinished@DiamondClassifyWorker@LocalWorkflow@U2@@AAEXPAVTask@3@@Z$0 1001db60 f   DiamondClassifyWorker.obj
 0001:0001cb69       __unwindfunclet$?sl_taskFinished@DiamondClassifyWorker@LocalWorkflow@U2@@AAEXPAVTask@3@@Z$1 1001db69 f   DiamondClassifyWorker.obj
 0001:0001cb71       __unwindfunclet$?sl_taskFinished@DiamondClassifyWorker@LocalWorkflow@U2@@AAEXPAVTask@3@@Z$2 1001db71 f   DiamondClassifyWorker.obj
 0001:0001cb7a       __unwindfunclet$?sl_taskFinished@DiamondClassifyWorker@LocalWorkflow@U2@@AAEXPAVTask@3@@Z$3 1001db7a f   DiamondClassifyWorker.obj
 0001:0001cb83       __unwindfunclet$?sl_taskFinished@DiamondClassifyWorker@LocalWorkflow@U2@@AAEXPAVTask@3@@Z$5 1001db83 f   DiamondClassifyWorker.obj
 0001:0001cb8c       __unwindfunclet$?sl_taskFinished@DiamondClassifyWorker@LocalWorkflow@U2@@AAEXPAVTask@3@@Z$6 1001db8c f   DiamondClassifyWorker.obj
 0001:0001cb95       __unwindfunclet$?sl_taskFinished@DiamondClassifyWorker@LocalWorkflow@U2@@AAEXPAVTask@3@@Z$7 1001db95 f   DiamondClassifyWorker.obj
 0001:0001cb9e       __unwindfunclet$?sl_taskFinished@DiamondClassifyWorker@LocalWorkflow@U2@@AAEXPAVTask@3@@Z$8 1001db9e f   DiamondClassifyWorker.obj
 0001:0001cba7       __unwindfunclet$?sl_taskFinished@DiamondClassifyWorker@LocalWorkflow@U2@@AAEXPAVTask@3@@Z$9 1001dba7 f   DiamondClassifyWorker.obj
 0001:0001cbb0       __unwindfunclet$?sl_taskFinished@DiamondClassifyWorker@LocalWorkflow@U2@@AAEXPAVTask@3@@Z$10 1001dbb0 f   DiamondClassifyWorker.obj
 0001:0001cbb9       __unwindfunclet$?sl_taskFinished@DiamondClassifyWorker@LocalWorkflow@U2@@AAEXPAVTask@3@@Z$11 1001dbb9 f   DiamondClassifyWorker.obj
 0001:0001cbc2       __unwindfunclet$?sl_taskFinished@DiamondClassifyWorker@LocalWorkflow@U2@@AAEXPAVTask@3@@Z$12 1001dbc2 f   DiamondClassifyWorker.obj
 0001:0001cbcb       __ehhandler$?sl_taskFinished@DiamondClassifyWorker@LocalWorkflow@U2@@AAEXPAVTask@3@@Z 1001dbcb f   DiamondClassifyWorker.obj
 0001:0001cbf0       __unwindfunclet$?tick@DiamondClassifyWorker@LocalWorkflow@U2@@UAEPAVTask@3@XZ$0 1001dbf0 f   DiamondClassifyWorker.obj
 0001:0001cbf9       __unwindfunclet$?tick@DiamondClassifyWorker@LocalWorkflow@U2@@UAEPAVTask@3@XZ$1 1001dbf9 f   DiamondClassifyWorker.obj
 0001:0001cc04       __unwindfunclet$?tick@DiamondClassifyWorker@LocalWorkflow@U2@@UAEPAVTask@3@XZ$2 1001dc04 f   DiamondClassifyWorker.obj
 0001:0001cc0f       __unwindfunclet$?tick@DiamondClassifyWorker@LocalWorkflow@U2@@UAEPAVTask@3@XZ$3 1001dc0f f   DiamondClassifyWorker.obj
 0001:0001cc29       __unwindfunclet$?tick@DiamondClassifyWorker@LocalWorkflow@U2@@UAEPAVTask@3@XZ$4 1001dc29 f   DiamondClassifyWorker.obj
 0001:0001cc34       __unwindfunclet$?tick@DiamondClassifyWorker@LocalWorkflow@U2@@UAEPAVTask@3@XZ$5 1001dc34 f   DiamondClassifyWorker.obj
 0001:0001cc3c       __unwindfunclet$?tick@DiamondClassifyWorker@LocalWorkflow@U2@@UAEPAVTask@3@XZ$6 1001dc3c f   DiamondClassifyWorker.obj
 0001:0001cc47       __ehhandler$?tick@DiamondClassifyWorker@LocalWorkflow@U2@@UAEPAVTask@3@XZ 1001dc47 f   DiamondClassifyWorker.obj
 0001:0001cc70       __unwindfunclet$??$?0VQString@@H@?$QPair@VQString@@VQVariant@@@@QAE@$$QAU?$QPair@VQString@@H@@@Z$0 1001dc70 f   DiamondClassifyWorkerFactory.obj
 0001:0001cc79       __ehhandler$??$?0VQString@@H@?$QPair@VQString@@VQVariant@@@@QAE@$$QAU?$QPair@VQString@@H@@@Z 1001dc79 f   DiamondClassifyWorkerFactory.obj
 0001:0001cca0       __unwindfunclet$??$?0VQString@@V0@@?$QPair@VQString@@VQVariant@@@@QAE@$$QAU?$QPair@VQString@@V1@@@@Z$0 1001dca0 f   DiamondClassifyWorkerFactory.obj
 0001:0001cca9       __ehhandler$??$?0VQString@@V0@@?$QPair@VQString@@VQVariant@@@@QAE@$$QAU?$QPair@VQString@@V1@@@@Z 1001dca9 f   DiamondClassifyWorkerFactory.obj
 0001:0001ccd0       __unwindfunclet$??$qMakePair@VQString@@V1@@@YA?AU?$QPair@VQString@@V1@@@ABVQString@@0@Z$1 1001dcd0 f   DiamondClassifyWorkerFactory.obj
 0001:0001ccd9       __ehhandler$??$qMakePair@VQString@@V1@@@YA?AU?$QPair@VQString@@V1@@@ABVQString@@0@Z 1001dcd9 f   DiamondClassifyWorkerFactory.obj
 0001:0001cd00       __ehhandler$??0?$QList@PAVDNATranslation@U2@@@@QAE@ABV0@@Z 1001dd00 f   DiamondClassifyWorkerFactory.obj
 0001:0001cd20       __unwindfunclet$??0?$QPair@VQString@@V1@@@QAE@ABU0@@Z$0 1001dd20 f   DiamondClassifyWorkerFactory.obj
 0001:0001cd29       __ehhandler$??0?$QPair@VQString@@V1@@@QAE@ABU0@@Z 1001dd29 f   DiamondClassifyWorkerFactory.obj
 0001:0001cd50       __unwindfunclet$??0?$QPair@VQString@@V1@@@QAE@ABVQString@@0@Z$0 1001dd50 f   DiamondClassifyWorkerFactory.obj
 0001:0001cd59       __ehhandler$??0?$QPair@VQString@@V1@@@QAE@ABVQString@@0@Z 1001dd59 f   DiamondClassifyWorkerFactory.obj
 0001:0001cd80       __unwindfunclet$??0?$QPair@VQString@@VQVariant@@@@QAE@ABU0@@Z$0 1001dd80 f   DiamondClassifyWorkerFactory.obj
 0001:0001cd89       __ehhandler$??0?$QPair@VQString@@VQVariant@@@@QAE@ABU0@@Z 1001dd89 f   DiamondClassifyWorkerFactory.obj
 0001:0001cdb0       __unwindfunclet$??1?$QPair@VQString@@V1@@@QAE@XZ$0 1001ddb0 f   DiamondClassifyWorkerFactory.obj
 0001:0001cdb9       __ehhandler$??1?$QPair@VQString@@V1@@@QAE@XZ 1001ddb9 f   DiamondClassifyWorkerFactory.obj
 0001:0001cde0       __unwindfunclet$??1?$QPair@VQString@@VQVariant@@@@QAE@XZ$0 1001dde0 f   DiamondClassifyWorkerFactory.obj
 0001:0001cde9       __ehhandler$??1?$QPair@VQString@@VQVariant@@@@QAE@XZ 1001dde9 f   DiamondClassifyWorkerFactory.obj
 0001:0001ce10       __unwindfunclet$??_G?$QPair@VQString@@V1@@@QAEPAXI@Z$0 1001de10 f   DiamondClassifyWorkerFactory.obj
 0001:0001ce19       __ehhandler$??_G?$QPair@VQString@@V1@@@QAEPAXI@Z 1001de19 f   DiamondClassifyWorkerFactory.obj
 0001:0001ce40       __unwindfunclet$??_G?$QPair@VQString@@VQVariant@@@@QAEPAXI@Z$0 1001de40 f   DiamondClassifyWorkerFactory.obj
 0001:0001ce49       __ehhandler$??_G?$QPair@VQString@@VQVariant@@@@QAEPAXI@Z 1001de49 f   DiamondClassifyWorkerFactory.obj
 0001:0001ce70       __unwindfunclet$??__EalgoLog@U2@@YAXXZ$0 1001de70 f   DiamondClassifyWorkerFactory.obj
 0001:0001ce79       __ehhandler$??__EalgoLog@U2@@YAXXZ 1001de79 f   DiamondClassifyWorkerFactory.obj
 0001:0001cea0       __unwindfunclet$??__EcmdLog@U2@@YAXXZ$0 1001dea0 f   DiamondClassifyWorkerFactory.obj
 0001:0001cea9       __ehhandler$??__EcmdLog@U2@@YAXXZ 1001dea9 f   DiamondClassifyWorkerFactory.obj
 0001:0001ced0       __unwindfunclet$??__EcoreLog@U2@@YAXXZ$0 1001ded0 f   DiamondClassifyWorkerFactory.obj
 0001:0001ced9       __ehhandler$??__EcoreLog@U2@@YAXXZ 1001ded9 f   DiamondClassifyWorkerFactory.obj
 0001:0001cf00       __unwindfunclet$??__EioLog@U2@@YAXXZ$0 1001df00 f   DiamondClassifyWorkerFactory.obj
 0001:0001cf09       __ehhandler$??__EioLog@U2@@YAXXZ 1001df09 f   DiamondClassifyWorkerFactory.obj
 0001:0001cf30       __unwindfunclet$??__EperfLog@U2@@YAXXZ$0 1001df30 f   DiamondClassifyWorkerFactory.obj
 0001:0001cf39       __ehhandler$??__EperfLog@U2@@YAXXZ 1001df39 f   DiamondClassifyWorkerFactory.obj
 0001:0001cf60       __unwindfunclet$??__EscriptLog@U2@@YAXXZ$0 1001df60 f   DiamondClassifyWorkerFactory.obj
 0001:0001cf69       __ehhandler$??__EscriptLog@U2@@YAXXZ 1001df69 f   DiamondClassifyWorkerFactory.obj
 0001:0001cf90       __unwindfunclet$??__EtaskLog@U2@@YAXXZ$0 1001df90 f   DiamondClassifyWorkerFactory.obj
 0001:0001cf99       __ehhandler$??__EtaskLog@U2@@YAXXZ 1001df99 f   DiamondClassifyWorkerFactory.obj
 0001:0001cfc0       __unwindfunclet$??__EuiLog@U2@@YAXXZ$0 1001dfc0 f   DiamondClassifyWorkerFactory.obj
 0001:0001cfc9       __ehhandler$??__EuiLog@U2@@YAXXZ 1001dfc9 f   DiamondClassifyWorkerFactory.obj
 0001:0001cff0       __unwindfunclet$??__EuserActLog@U2@@YAXXZ$0 1001dff0 f   DiamondClassifyWorkerFactory.obj
 0001:0001cff9       __ehhandler$??__EuserActLog@U2@@YAXXZ 1001dff9 f   DiamondClassifyWorkerFactory.obj
 0001:0001d020       __ehhandler$?append@?$QList@U?$QPair@VQString@@V1@@@@@QAEXABU?$QPair@VQString@@V1@@@@Z 1001e020 f   DiamondClassifyWorkerFactory.obj
 0001:0001d040       __ehhandler$?append@?$QList@U?$QPair@VQString@@VQVariant@@@@@@QAEXABU?$QPair@VQString@@VQVariant@@@@@Z 1001e040 f   DiamondClassifyWorkerFactory.obj
 0001:0001d060       __unwindfunclet$?createWorker@DiamondClassifyWorkerFactory@LocalWorkflow@U2@@UAEPAVWorker@Workflow@3@PAVActor@53@@Z$0 1001e060 f   DiamondClassifyWorkerFactory.obj
 0001:0001d06b       __ehhandler$?createWorker@DiamondClassifyWorkerFactory@LocalWorkflow@U2@@UAEPAVWorker@Workflow@3@PAVActor@53@@Z 1001e06b f   DiamondClassifyWorkerFactory.obj
 0001:0001d090       __ehhandler$?detach_helper_grow@?$QList@U?$QPair@VQString@@V1@@@@@AAEPAUNode@1@HH@Z 1001e090 f   DiamondClassifyWorkerFactory.obj
 0001:0001d0b0       __ehhandler$?detach_helper_grow@?$QList@U?$QPair@VQString@@VQVariant@@@@@@AAEPAUNode@1@HH@Z 1001e0b0 f   DiamondClassifyWorkerFactory.obj
 0001:0001d0d0       __unwindfunclet$?init@DiamondClassifyWorkerFactory@LocalWorkflow@U2@@SAXXZ$0 1001e0d0 f   DiamondClassifyWorkerFactory.obj
 0001:0001d0db       __unwindfunclet$?init@DiamondClassifyWorkerFactory@LocalWorkflow@U2@@SAXXZ$1 1001e0db f   DiamondClassifyWorkerFactory.obj
 0001:0001d0e4       __unwindfunclet$?init@DiamondClassifyWorkerFactory@LocalWorkflow@U2@@SAXXZ$2 1001e0e4 f   DiamondClassifyWorkerFactory.obj
 0001:0001d0ed       __unwindfunclet$?init@DiamondClassifyWorkerFactory@LocalWorkflow@U2@@SAXXZ$3 1001e0ed f   DiamondClassifyWorkerFactory.obj
 0001:0001d0f6       __unwindfunclet$?init@DiamondClassifyWorkerFactory@LocalWorkflow@U2@@SAXXZ$4 1001e0f6 f   DiamondClassifyWorkerFactory.obj
 0001:0001d0fe       __unwindfunclet$?init@DiamondClassifyWorkerFactory@LocalWorkflow@U2@@SAXXZ$5 1001e0fe f   DiamondClassifyWorkerFactory.obj
 0001:0001d106       __unwindfunclet$?init@DiamondClassifyWorkerFactory@LocalWorkflow@U2@@SAXXZ$6 1001e106 f   DiamondClassifyWorkerFactory.obj
 0001:0001d10e       __unwindfunclet$?init@DiamondClassifyWorkerFactory@LocalWorkflow@U2@@SAXXZ$7 1001e10e f   DiamondClassifyWorkerFactory.obj
 0001:0001d116       __unwindfunclet$?init@DiamondClassifyWorkerFactory@LocalWorkflow@U2@@SAXXZ$8 1001e116 f   DiamondClassifyWorkerFactory.obj
 0001:0001d11f       __unwindfunclet$?init@DiamondClassifyWorkerFactory@LocalWorkflow@U2@@SAXXZ$9 1001e11f f   DiamondClassifyWorkerFactory.obj
 0001:0001d12b       __unwindfunclet$?init@DiamondClassifyWorkerFactory@LocalWorkflow@U2@@SAXXZ$10 1001e12b f   DiamondClassifyWorkerFactory.obj
 0001:0001d134       __unwindfunclet$?init@DiamondClassifyWorkerFactory@LocalWorkflow@U2@@SAXXZ$11 1001e134 f   DiamondClassifyWorkerFactory.obj
 0001:0001d13d       __unwindfunclet$?init@DiamondClassifyWorkerFactory@LocalWorkflow@U2@@SAXXZ$12 1001e13d f   DiamondClassifyWorkerFactory.obj
 0001:0001d149       __unwindfunclet$?init@DiamondClassifyWorkerFactory@LocalWorkflow@U2@@SAXXZ$13 1001e149 f   DiamondClassifyWorkerFactory.obj
 0001:0001d155       __unwindfunclet$?init@DiamondClassifyWorkerFactory@LocalWorkflow@U2@@SAXXZ$14 1001e155 f   DiamondClassifyWorkerFactory.obj
 0001:0001d161       __unwindfunclet$?init@DiamondClassifyWorkerFactory@LocalWorkflow@U2@@SAXXZ$15 1001e161 f   DiamondClassifyWorkerFactory.obj
 0001:0001d16c       __unwindfunclet$?init@DiamondClassifyWorkerFactory@LocalWorkflow@U2@@SAXXZ$16 1001e16c f   DiamondClassifyWorkerFactory.obj
 0001:0001d177       __unwindfunclet$?init@DiamondClassifyWorkerFactory@LocalWorkflow@U2@@SAXXZ$17 1001e177 f   DiamondClassifyWorkerFactory.obj
 0001:0001d191       __unwindfunclet$?init@DiamondClassifyWorkerFactory@LocalWorkflow@U2@@SAXXZ$18 1001e191 f   DiamondClassifyWorkerFactory.obj
 0001:0001d1ae       __unwindfunclet$?init@DiamondClassifyWorkerFactory@LocalWorkflow@U2@@SAXXZ$20 1001e1ae f   DiamondClassifyWorkerFactory.obj
 0001:0001d1b9       __unwindfunclet$?init@DiamondClassifyWorkerFactory@LocalWorkflow@U2@@SAXXZ$21 1001e1b9 f   DiamondClassifyWorkerFactory.obj
 0001:0001d1c4       __unwindfunclet$?init@DiamondClassifyWorkerFactory@LocalWorkflow@U2@@SAXXZ$22 1001e1c4 f   DiamondClassifyWorkerFactory.obj
 0001:0001d1de       __unwindfunclet$?init@DiamondClassifyWorkerFactory@LocalWorkflow@U2@@SAXXZ$23 1001e1de f   DiamondClassifyWorkerFactory.obj
 0001:0001d1fb       __unwindfunclet$?init@DiamondClassifyWorkerFactory@LocalWorkflow@U2@@SAXXZ$25 1001e1fb f   DiamondClassifyWorkerFactory.obj
 0001:0001d203       __unwindfunclet$?init@DiamondClassifyWorkerFactory@LocalWorkflow@U2@@SAXXZ$26 1001e203 f   DiamondClassifyWorkerFactory.obj
 0001:0001d20c       __unwindfunclet$?init@DiamondClassifyWorkerFactory@LocalWorkflow@U2@@SAXXZ$27 1001e20c f   DiamondClassifyWorkerFactory.obj
 0001:0001d215       __unwindfunclet$?init@DiamondClassifyWorkerFactory@LocalWorkflow@U2@@SAXXZ$28 1001e215 f   DiamondClassifyWorkerFactory.obj
 0001:0001d21e       __unwindfunclet$?init@DiamondClassifyWorkerFactory@LocalWorkflow@U2@@SAXXZ$29 1001e21e f   DiamondClassifyWorkerFactory.obj
 0001:0001d22a       __unwindfunclet$?init@DiamondClassifyWorkerFactory@LocalWorkflow@U2@@SAXXZ$30 1001e22a f   DiamondClassifyWorkerFactory.obj
 0001:0001d236       __unwindfunclet$?init@DiamondClassifyWorkerFactory@LocalWorkflow@U2@@SAXXZ$31 1001e236 f   DiamondClassifyWorkerFactory.obj
 0001:0001d242       __unwindfunclet$?init@DiamondClassifyWorkerFactory@LocalWorkflow@U2@@SAXXZ$32 1001e242 f   DiamondClassifyWorkerFactory.obj
 0001:0001d24b       __unwindfunclet$?init@DiamondClassifyWorkerFactory@LocalWorkflow@U2@@SAXXZ$33 1001e24b f   DiamondClassifyWorkerFactory.obj
 0001:0001d257       __unwindfunclet$?init@DiamondClassifyWorkerFactory@LocalWorkflow@U2@@SAXXZ$34 1001e257 f   DiamondClassifyWorkerFactory.obj
 0001:0001d263       __unwindfunclet$?init@DiamondClassifyWorkerFactory@LocalWorkflow@U2@@SAXXZ$35 1001e263 f   DiamondClassifyWorkerFactory.obj
 0001:0001d26f       __unwindfunclet$?init@DiamondClassifyWorkerFactory@LocalWorkflow@U2@@SAXXZ$36 1001e26f f   DiamondClassifyWorkerFactory.obj
 0001:0001d278       __unwindfunclet$?init@DiamondClassifyWorkerFactory@LocalWorkflow@U2@@SAXXZ$37 1001e278 f   DiamondClassifyWorkerFactory.obj
 0001:0001d284       __unwindfunclet$?init@DiamondClassifyWorkerFactory@LocalWorkflow@U2@@SAXXZ$38 1001e284 f   DiamondClassifyWorkerFactory.obj
 0001:0001d290       __unwindfunclet$?init@DiamondClassifyWorkerFactory@LocalWorkflow@U2@@SAXXZ$39 1001e290 f   DiamondClassifyWorkerFactory.obj
 0001:0001d29c       __unwindfunclet$?init@DiamondClassifyWorkerFactory@LocalWorkflow@U2@@SAXXZ$40 1001e29c f   DiamondClassifyWorkerFactory.obj
 0001:0001d2a8       __unwindfunclet$?init@DiamondClassifyWorkerFactory@LocalWorkflow@U2@@SAXXZ$41 1001e2a8 f   DiamondClassifyWorkerFactory.obj
 0001:0001d2b4       __unwindfunclet$?init@DiamondClassifyWorkerFactory@LocalWorkflow@U2@@SAXXZ$42 1001e2b4 f   DiamondClassifyWorkerFactory.obj
 0001:0001d2c0       __unwindfunclet$?init@DiamondClassifyWorkerFactory@LocalWorkflow@U2@@SAXXZ$43 1001e2c0 f   DiamondClassifyWorkerFactory.obj
 0001:0001d2cc       __unwindfunclet$?init@DiamondClassifyWorkerFactory@LocalWorkflow@U2@@SAXXZ$44 1001e2cc f   DiamondClassifyWorkerFactory.obj
 0001:0001d2d8       __unwindfunclet$?init@DiamondClassifyWorkerFactory@LocalWorkflow@U2@@SAXXZ$45 1001e2d8 f   DiamondClassifyWorkerFactory.obj
 0001:0001d2e4       __unwindfunclet$?init@DiamondClassifyWorkerFactory@LocalWorkflow@U2@@SAXXZ$46 1001e2e4 f   DiamondClassifyWorkerFactory.obj
 0001:0001d2f0       __unwindfunclet$?init@DiamondClassifyWorkerFactory@LocalWorkflow@U2@@SAXXZ$47 1001e2f0 f   DiamondClassifyWorkerFactory.obj
 0001:0001d2fc       __unwindfunclet$?init@DiamondClassifyWorkerFactory@LocalWorkflow@U2@@SAXXZ$48 1001e2fc f   DiamondClassifyWorkerFactory.obj
 0001:0001d308       __unwindfunclet$?init@DiamondClassifyWorkerFactory@LocalWorkflow@U2@@SAXXZ$49 1001e308 f   DiamondClassifyWorkerFactory.obj
 0001:0001d314       __unwindfunclet$?init@DiamondClassifyWorkerFactory@LocalWorkflow@U2@@SAXXZ$50 1001e314 f   DiamondClassifyWorkerFactory.obj
 0001:0001d320       __unwindfunclet$?init@DiamondClassifyWorkerFactory@LocalWorkflow@U2@@SAXXZ$51 1001e320 f   DiamondClassifyWorkerFactory.obj
 0001:0001d32c       __unwindfunclet$?init@DiamondClassifyWorkerFactory@LocalWorkflow@U2@@SAXXZ$52 1001e32c f   DiamondClassifyWorkerFactory.obj
 0001:0001d338       __unwindfunclet$?init@DiamondClassifyWorkerFactory@LocalWorkflow@U2@@SAXXZ$53 1001e338 f   DiamondClassifyWorkerFactory.obj
 0001:0001d344       __unwindfunclet$?init@DiamondClassifyWorkerFactory@LocalWorkflow@U2@@SAXXZ$54 1001e344 f   DiamondClassifyWorkerFactory.obj
 0001:0001d350       __unwindfunclet$?init@DiamondClassifyWorkerFactory@LocalWorkflow@U2@@SAXXZ$55 1001e350 f   DiamondClassifyWorkerFactory.obj
 0001:0001d35c       __unwindfunclet$?init@DiamondClassifyWorkerFactory@LocalWorkflow@U2@@SAXXZ$56 1001e35c f   DiamondClassifyWorkerFactory.obj
 0001:0001d368       __unwindfunclet$?init@DiamondClassifyWorkerFactory@LocalWorkflow@U2@@SAXXZ$57 1001e368 f   DiamondClassifyWorkerFactory.obj
 0001:0001d374       __unwindfunclet$?init@DiamondClassifyWorkerFactory@LocalWorkflow@U2@@SAXXZ$58 1001e374 f   DiamondClassifyWorkerFactory.obj
 0001:0001d380       __unwindfunclet$?init@DiamondClassifyWorkerFactory@LocalWorkflow@U2@@SAXXZ$59 1001e380 f   DiamondClassifyWorkerFactory.obj
 0001:0001d389       __unwindfunclet$?init@DiamondClassifyWorkerFactory@LocalWorkflow@U2@@SAXXZ$60 1001e389 f   DiamondClassifyWorkerFactory.obj
 0001:0001d395       __unwindfunclet$?init@DiamondClassifyWorkerFactory@LocalWorkflow@U2@@SAXXZ$61 1001e395 f   DiamondClassifyWorkerFactory.obj
 0001:0001d3a1       __unwindfunclet$?init@DiamondClassifyWorkerFactory@LocalWorkflow@U2@@SAXXZ$62 1001e3a1 f   DiamondClassifyWorkerFactory.obj
 0001:0001d3aa       __unwindfunclet$?init@DiamondClassifyWorkerFactory@LocalWorkflow@U2@@SAXXZ$63 1001e3aa f   DiamondClassifyWorkerFactory.obj
 0001:0001d3b3       __unwindfunclet$?init@DiamondClassifyWorkerFactory@LocalWorkflow@U2@@SAXXZ$64 1001e3b3 f   DiamondClassifyWorkerFactory.obj
 0001:0001d3bf       __unwindfunclet$?init@DiamondClassifyWorkerFactory@LocalWorkflow@U2@@SAXXZ$65 1001e3bf f   DiamondClassifyWorkerFactory.obj
 0001:0001d3c8       __unwindfunclet$?init@DiamondClassifyWorkerFactory@LocalWorkflow@U2@@SAXXZ$66 1001e3c8 f   DiamondClassifyWorkerFactory.obj
 0001:0001d3d4       __unwindfunclet$?init@DiamondClassifyWorkerFactory@LocalWorkflow@U2@@SAXXZ$67 1001e3d4 f   DiamondClassifyWorkerFactory.obj
 0001:0001d3dd       __unwindfunclet$?init@DiamondClassifyWorkerFactory@LocalWorkflow@U2@@SAXXZ$68 1001e3dd f   DiamondClassifyWorkerFactory.obj
 0001:0001d3e6       __unwindfunclet$?init@DiamondClassifyWorkerFactory@LocalWorkflow@U2@@SAXXZ$69 1001e3e6 f   DiamondClassifyWorkerFactory.obj
 0001:0001d3ef       __unwindfunclet$?init@DiamondClassifyWorkerFactory@LocalWorkflow@U2@@SAXXZ$70 1001e3ef f   DiamondClassifyWorkerFactory.obj
 0001:0001d3fa       __unwindfunclet$?init@DiamondClassifyWorkerFactory@LocalWorkflow@U2@@SAXXZ$71 1001e3fa f   DiamondClassifyWorkerFactory.obj
 0001:0001d414       __unwindfunclet$?init@DiamondClassifyWorkerFactory@LocalWorkflow@U2@@SAXXZ$73 1001e414 f   DiamondClassifyWorkerFactory.obj
 0001:0001d41f       __unwindfunclet$?init@DiamondClassifyWorkerFactory@LocalWorkflow@U2@@SAXXZ$74 1001e41f f   DiamondClassifyWorkerFactory.obj
 0001:0001d439       __unwindfunclet$?init@DiamondClassifyWorkerFactory@LocalWorkflow@U2@@SAXXZ$76 1001e439 f   DiamondClassifyWorkerFactory.obj
 0001:0001d444       __unwindfunclet$?init@DiamondClassifyWorkerFactory@LocalWorkflow@U2@@SAXXZ$77 1001e444 f   DiamondClassifyWorkerFactory.obj
 0001:0001d45e       __unwindfunclet$?init@DiamondClassifyWorkerFactory@LocalWorkflow@U2@@SAXXZ$79 1001e45e f   DiamondClassifyWorkerFactory.obj
 0001:0001d469       __unwindfunclet$?init@DiamondClassifyWorkerFactory@LocalWorkflow@U2@@SAXXZ$80 1001e469 f   DiamondClassifyWorkerFactory.obj
 0001:0001d488       __unwindfunclet$?init@DiamondClassifyWorkerFactory@LocalWorkflow@U2@@SAXXZ$82 1001e488 f   DiamondClassifyWorkerFactory.obj
 0001:0001d493       __unwindfunclet$?init@DiamondClassifyWorkerFactory@LocalWorkflow@U2@@SAXXZ$83 1001e493 f   DiamondClassifyWorkerFactory.obj
 0001:0001d4b2       __unwindfunclet$?init@DiamondClassifyWorkerFactory@LocalWorkflow@U2@@SAXXZ$85 1001e4b2 f   DiamondClassifyWorkerFactory.obj
 0001:0001d4bd       __unwindfunclet$?init@DiamondClassifyWorkerFactory@LocalWorkflow@U2@@SAXXZ$86 1001e4bd f   DiamondClassifyWorkerFactory.obj
 0001:0001d4dc       __unwindfunclet$?init@DiamondClassifyWorkerFactory@LocalWorkflow@U2@@SAXXZ$88 1001e4dc f   DiamondClassifyWorkerFactory.obj
 0001:0001d4e7       __unwindfunclet$?init@DiamondClassifyWorkerFactory@LocalWorkflow@U2@@SAXXZ$89 1001e4e7 f   DiamondClassifyWorkerFactory.obj
 0001:0001d506       __unwindfunclet$?init@DiamondClassifyWorkerFactory@LocalWorkflow@U2@@SAXXZ$91 1001e506 f   DiamondClassifyWorkerFactory.obj
 0001:0001d511       __unwindfunclet$?init@DiamondClassifyWorkerFactory@LocalWorkflow@U2@@SAXXZ$92 1001e511 f   DiamondClassifyWorkerFactory.obj
 0001:0001d530       __unwindfunclet$?init@DiamondClassifyWorkerFactory@LocalWorkflow@U2@@SAXXZ$94 1001e530 f   DiamondClassifyWorkerFactory.obj
 0001:0001d53b       __unwindfunclet$?init@DiamondClassifyWorkerFactory@LocalWorkflow@U2@@SAXXZ$95 1001e53b f   DiamondClassifyWorkerFactory.obj
 0001:0001d55a       __unwindfunclet$?init@DiamondClassifyWorkerFactory@LocalWorkflow@U2@@SAXXZ$97 1001e55a f   DiamondClassifyWorkerFactory.obj
 0001:0001d565       __unwindfunclet$?init@DiamondClassifyWorkerFactory@LocalWorkflow@U2@@SAXXZ$98 1001e565 f   DiamondClassifyWorkerFactory.obj
 0001:0001d584       __unwindfunclet$?init@DiamondClassifyWorkerFactory@LocalWorkflow@U2@@SAXXZ$100 1001e584 f   DiamondClassifyWorkerFactory.obj
 0001:0001d58f       __unwindfunclet$?init@DiamondClassifyWorkerFactory@LocalWorkflow@U2@@SAXXZ$101 1001e58f f   DiamondClassifyWorkerFactory.obj
 0001:0001d5ae       __unwindfunclet$?init@DiamondClassifyWorkerFactory@LocalWorkflow@U2@@SAXXZ$103 1001e5ae f   DiamondClassifyWorkerFactory.obj
 0001:0001d5b9       __unwindfunclet$?init@DiamondClassifyWorkerFactory@LocalWorkflow@U2@@SAXXZ$104 1001e5b9 f   DiamondClassifyWorkerFactory.obj
 0001:0001d5d8       __unwindfunclet$?init@DiamondClassifyWorkerFactory@LocalWorkflow@U2@@SAXXZ$106 1001e5d8 f   DiamondClassifyWorkerFactory.obj
 0001:0001d5e3       __unwindfunclet$?init@DiamondClassifyWorkerFactory@LocalWorkflow@U2@@SAXXZ$107 1001e5e3 f   DiamondClassifyWorkerFactory.obj
 0001:0001d602       __unwindfunclet$?init@DiamondClassifyWorkerFactory@LocalWorkflow@U2@@SAXXZ$109 1001e602 f   DiamondClassifyWorkerFactory.obj
 0001:0001d60d       __unwindfunclet$?init@DiamondClassifyWorkerFactory@LocalWorkflow@U2@@SAXXZ$110 1001e60d f   DiamondClassifyWorkerFactory.obj
 0001:0001d62c       __unwindfunclet$?init@DiamondClassifyWorkerFactory@LocalWorkflow@U2@@SAXXZ$112 1001e62c f   DiamondClassifyWorkerFactory.obj
 0001:0001d634       __unwindfunclet$?init@DiamondClassifyWorkerFactory@LocalWorkflow@U2@@SAXXZ$113 1001e634 f   DiamondClassifyWorkerFactory.obj
 0001:0001d63c       __unwindfunclet$?init@DiamondClassifyWorkerFactory@LocalWorkflow@U2@@SAXXZ$235 1001e63c f   DiamondClassifyWorkerFactory.obj
 0001:0001d645       __unwindfunclet$?init@DiamondClassifyWorkerFactory@LocalWorkflow@U2@@SAXXZ$114 1001e645 f   DiamondClassifyWorkerFactory.obj
 0001:0001d64d       __unwindfunclet$?init@DiamondClassifyWorkerFactory@LocalWorkflow@U2@@SAXXZ$237 1001e64d f   DiamondClassifyWorkerFactory.obj
 0001:0001d656       __unwindfunclet$?init@DiamondClassifyWorkerFactory@LocalWorkflow@U2@@SAXXZ$239 1001e656 f   DiamondClassifyWorkerFactory.obj
 0001:0001d65f       __unwindfunclet$?init@DiamondClassifyWorkerFactory@LocalWorkflow@U2@@SAXXZ$115 1001e65f f   DiamondClassifyWorkerFactory.obj
 0001:0001d667       __unwindfunclet$?init@DiamondClassifyWorkerFactory@LocalWorkflow@U2@@SAXXZ$241 1001e667 f   DiamondClassifyWorkerFactory.obj
 0001:0001d670       __unwindfunclet$?init@DiamondClassifyWorkerFactory@LocalWorkflow@U2@@SAXXZ$116 1001e670 f   DiamondClassifyWorkerFactory.obj
 0001:0001d67b       __unwindfunclet$?init@DiamondClassifyWorkerFactory@LocalWorkflow@U2@@SAXXZ$117 1001e67b f   DiamondClassifyWorkerFactory.obj
 0001:0001d69a       __unwindfunclet$?init@DiamondClassifyWorkerFactory@LocalWorkflow@U2@@SAXXZ$118 1001e69a f   DiamondClassifyWorkerFactory.obj
 0001:0001d6a2       __unwindfunclet$?init@DiamondClassifyWorkerFactory@LocalWorkflow@U2@@SAXXZ$119 1001e6a2 f   DiamondClassifyWorkerFactory.obj
 0001:0001d6ab       __unwindfunclet$?init@DiamondClassifyWorkerFactory@LocalWorkflow@U2@@SAXXZ$120 1001e6ab f   DiamondClassifyWorkerFactory.obj
 0001:0001d6b3       __unwindfunclet$?init@DiamondClassifyWorkerFactory@LocalWorkflow@U2@@SAXXZ$122 1001e6b3 f   DiamondClassifyWorkerFactory.obj
 0001:0001d6be       __unwindfunclet$?init@DiamondClassifyWorkerFactory@LocalWorkflow@U2@@SAXXZ$123 1001e6be f   DiamondClassifyWorkerFactory.obj
 0001:0001d6c7       __unwindfunclet$?init@DiamondClassifyWorkerFactory@LocalWorkflow@U2@@SAXXZ$124 1001e6c7 f   DiamondClassifyWorkerFactory.obj
 0001:0001d6d0       __unwindfunclet$?init@DiamondClassifyWorkerFactory@LocalWorkflow@U2@@SAXXZ$125 1001e6d0 f   DiamondClassifyWorkerFactory.obj
 0001:0001d6d8       __unwindfunclet$?init@DiamondClassifyWorkerFactory@LocalWorkflow@U2@@SAXXZ$244 1001e6d8 f   DiamondClassifyWorkerFactory.obj
 0001:0001d6e1       __unwindfunclet$?init@DiamondClassifyWorkerFactory@LocalWorkflow@U2@@SAXXZ$126 1001e6e1 f   DiamondClassifyWorkerFactory.obj
 0001:0001d6e9       __unwindfunclet$?init@DiamondClassifyWorkerFactory@LocalWorkflow@U2@@SAXXZ$246 1001e6e9 f   DiamondClassifyWorkerFactory.obj
 0001:0001d6f2       __unwindfunclet$?init@DiamondClassifyWorkerFactory@LocalWorkflow@U2@@SAXXZ$127 1001e6f2 f   DiamondClassifyWorkerFactory.obj
 0001:0001d6fd       __unwindfunclet$?init@DiamondClassifyWorkerFactory@LocalWorkflow@U2@@SAXXZ$128 1001e6fd f   DiamondClassifyWorkerFactory.obj
 0001:0001d705       __unwindfunclet$?init@DiamondClassifyWorkerFactory@LocalWorkflow@U2@@SAXXZ$129 1001e705 f   DiamondClassifyWorkerFactory.obj
 0001:0001d70e       __unwindfunclet$?init@DiamondClassifyWorkerFactory@LocalWorkflow@U2@@SAXXZ$130 1001e70e f   DiamondClassifyWorkerFactory.obj
 0001:0001d716       __unwindfunclet$?init@DiamondClassifyWorkerFactory@LocalWorkflow@U2@@SAXXZ$250 1001e716 f   DiamondClassifyWorkerFactory.obj
 0001:0001d71f       __unwindfunclet$?init@DiamondClassifyWorkerFactory@LocalWorkflow@U2@@SAXXZ$131 1001e71f f   DiamondClassifyWorkerFactory.obj
 0001:0001d727       __unwindfunclet$?init@DiamondClassifyWorkerFactory@LocalWorkflow@U2@@SAXXZ$252 1001e727 f   DiamondClassifyWorkerFactory.obj
 0001:0001d730       __unwindfunclet$?init@DiamondClassifyWorkerFactory@LocalWorkflow@U2@@SAXXZ$254 1001e730 f   DiamondClassifyWorkerFactory.obj
 0001:0001d739       __unwindfunclet$?init@DiamondClassifyWorkerFactory@LocalWorkflow@U2@@SAXXZ$132 1001e739 f   DiamondClassifyWorkerFactory.obj
 0001:0001d742       __unwindfunclet$?init@DiamondClassifyWorkerFactory@LocalWorkflow@U2@@SAXXZ$133 1001e742 f   DiamondClassifyWorkerFactory.obj
 0001:0001d74a       __unwindfunclet$?init@DiamondClassifyWorkerFactory@LocalWorkflow@U2@@SAXXZ$256 1001e74a f   DiamondClassifyWorkerFactory.obj
 0001:0001d753       __unwindfunclet$?init@DiamondClassifyWorkerFactory@LocalWorkflow@U2@@SAXXZ$134 1001e753 f   DiamondClassifyWorkerFactory.obj
 0001:0001d75b       __unwindfunclet$?init@DiamondClassifyWorkerFactory@LocalWorkflow@U2@@SAXXZ$258 1001e75b f   DiamondClassifyWorkerFactory.obj
 0001:0001d764       __unwindfunclet$?init@DiamondClassifyWorkerFactory@LocalWorkflow@U2@@SAXXZ$260 1001e764 f   DiamondClassifyWorkerFactory.obj
 0001:0001d76d       __unwindfunclet$?init@DiamondClassifyWorkerFactory@LocalWorkflow@U2@@SAXXZ$135 1001e76d f   DiamondClassifyWorkerFactory.obj
 0001:0001d776       __unwindfunclet$?init@DiamondClassifyWorkerFactory@LocalWorkflow@U2@@SAXXZ$136 1001e776 f   DiamondClassifyWorkerFactory.obj
 0001:0001d77e       __unwindfunclet$?init@DiamondClassifyWorkerFactory@LocalWorkflow@U2@@SAXXZ$262 1001e77e f   DiamondClassifyWorkerFactory.obj
 0001:0001d787       __unwindfunclet$?init@DiamondClassifyWorkerFactory@LocalWorkflow@U2@@SAXXZ$137 1001e787 f   DiamondClassifyWorkerFactory.obj
 0001:0001d78f       __unwindfunclet$?init@DiamondClassifyWorkerFactory@LocalWorkflow@U2@@SAXXZ$264 1001e78f f   DiamondClassifyWorkerFactory.obj
 0001:0001d798       __unwindfunclet$?init@DiamondClassifyWorkerFactory@LocalWorkflow@U2@@SAXXZ$266 1001e798 f   DiamondClassifyWorkerFactory.obj
 0001:0001d7a1       __unwindfunclet$?init@DiamondClassifyWorkerFactory@LocalWorkflow@U2@@SAXXZ$138 1001e7a1 f   DiamondClassifyWorkerFactory.obj
 0001:0001d7ac       __unwindfunclet$?init@DiamondClassifyWorkerFactory@LocalWorkflow@U2@@SAXXZ$139 1001e7ac f   DiamondClassifyWorkerFactory.obj
 0001:0001d7b4       __unwindfunclet$?init@DiamondClassifyWorkerFactory@LocalWorkflow@U2@@SAXXZ$140 1001e7b4 f   DiamondClassifyWorkerFactory.obj
 0001:0001d7bd       __unwindfunclet$?init@DiamondClassifyWorkerFactory@LocalWorkflow@U2@@SAXXZ$141 1001e7bd f   DiamondClassifyWorkerFactory.obj
 0001:0001d7c6       __unwindfunclet$?init@DiamondClassifyWorkerFactory@LocalWorkflow@U2@@SAXXZ$142 1001e7c6 f   DiamondClassifyWorkerFactory.obj
 0001:0001d7d2       __unwindfunclet$?init@DiamondClassifyWorkerFactory@LocalWorkflow@U2@@SAXXZ$143 1001e7d2 f   DiamondClassifyWorkerFactory.obj
 0001:0001d7db       __unwindfunclet$?init@DiamondClassifyWorkerFactory@LocalWorkflow@U2@@SAXXZ$144 1001e7db f   DiamondClassifyWorkerFactory.obj
 0001:0001d7e7       __unwindfunclet$?init@DiamondClassifyWorkerFactory@LocalWorkflow@U2@@SAXXZ$145 1001e7e7 f   DiamondClassifyWorkerFactory.obj
 0001:0001d7f0       __unwindfunclet$?init@DiamondClassifyWorkerFactory@LocalWorkflow@U2@@SAXXZ$146 1001e7f0 f   DiamondClassifyWorkerFactory.obj
 0001:0001d7fb       __unwindfunclet$?init@DiamondClassifyWorkerFactory@LocalWorkflow@U2@@SAXXZ$147 1001e7fb f   DiamondClassifyWorkerFactory.obj
 0001:0001d803       __unwindfunclet$?init@DiamondClassifyWorkerFactory@LocalWorkflow@U2@@SAXXZ$148 1001e803 f   DiamondClassifyWorkerFactory.obj
 0001:0001d80c       __unwindfunclet$?init@DiamondClassifyWorkerFactory@LocalWorkflow@U2@@SAXXZ$149 1001e80c f   DiamondClassifyWorkerFactory.obj
 0001:0001d818       __unwindfunclet$?init@DiamondClassifyWorkerFactory@LocalWorkflow@U2@@SAXXZ$150 1001e818 f   DiamondClassifyWorkerFactory.obj
 0001:0001d824       __unwindfunclet$?init@DiamondClassifyWorkerFactory@LocalWorkflow@U2@@SAXXZ$151 1001e824 f   DiamondClassifyWorkerFactory.obj
 0001:0001d830       __unwindfunclet$?init@DiamondClassifyWorkerFactory@LocalWorkflow@U2@@SAXXZ$152 1001e830 f   DiamondClassifyWorkerFactory.obj
 0001:0001d83c       __unwindfunclet$?init@DiamondClassifyWorkerFactory@LocalWorkflow@U2@@SAXXZ$153 1001e83c f   DiamondClassifyWorkerFactory.obj
 0001:0001d848       __unwindfunclet$?init@DiamondClassifyWorkerFactory@LocalWorkflow@U2@@SAXXZ$154 1001e848 f   DiamondClassifyWorkerFactory.obj
 0001:0001d854       __unwindfunclet$?init@DiamondClassifyWorkerFactory@LocalWorkflow@U2@@SAXXZ$155 1001e854 f   DiamondClassifyWorkerFactory.obj
 0001:0001d860       __unwindfunclet$?init@DiamondClassifyWorkerFactory@LocalWorkflow@U2@@SAXXZ$156 1001e860 f   DiamondClassifyWorkerFactory.obj
 0001:0001d86b       __unwindfunclet$?init@DiamondClassifyWorkerFactory@LocalWorkflow@U2@@SAXXZ$157 1001e86b f   DiamondClassifyWorkerFactory.obj
 0001:0001d873       __unwindfunclet$?init@DiamondClassifyWorkerFactory@LocalWorkflow@U2@@SAXXZ$158 1001e873 f   DiamondClassifyWorkerFactory.obj
 0001:0001d87c       __unwindfunclet$?init@DiamondClassifyWorkerFactory@LocalWorkflow@U2@@SAXXZ$159 1001e87c f   DiamondClassifyWorkerFactory.obj
 0001:0001d885       __unwindfunclet$?init@DiamondClassifyWorkerFactory@LocalWorkflow@U2@@SAXXZ$160 1001e885 f   DiamondClassifyWorkerFactory.obj
 0001:0001d891       __unwindfunclet$?init@DiamondClassifyWorkerFactory@LocalWorkflow@U2@@SAXXZ$161 1001e891 f   DiamondClassifyWorkerFactory.obj
 0001:0001d89a       __unwindfunclet$?init@DiamondClassifyWorkerFactory@LocalWorkflow@U2@@SAXXZ$162 1001e89a f   DiamondClassifyWorkerFactory.obj
 0001:0001d8a3       __unwindfunclet$?init@DiamondClassifyWorkerFactory@LocalWorkflow@U2@@SAXXZ$163 1001e8a3 f   DiamondClassifyWorkerFactory.obj
 0001:0001d8ac       __unwindfunclet$?init@DiamondClassifyWorkerFactory@LocalWorkflow@U2@@SAXXZ$164 1001e8ac f   DiamondClassifyWorkerFactory.obj
 0001:0001d8b5       __unwindfunclet$?init@DiamondClassifyWorkerFactory@LocalWorkflow@U2@@SAXXZ$165 1001e8b5 f   DiamondClassifyWorkerFactory.obj
 0001:0001d8c0       __unwindfunclet$?init@DiamondClassifyWorkerFactory@LocalWorkflow@U2@@SAXXZ$166 1001e8c0 f   DiamondClassifyWorkerFactory.obj
 0001:0001d8c8       __unwindfunclet$?init@DiamondClassifyWorkerFactory@LocalWorkflow@U2@@SAXXZ$167 1001e8c8 f   DiamondClassifyWorkerFactory.obj
 0001:0001d8d1       __unwindfunclet$?init@DiamondClassifyWorkerFactory@LocalWorkflow@U2@@SAXXZ$168 1001e8d1 f   DiamondClassifyWorkerFactory.obj
 0001:0001d8da       __unwindfunclet$?init@DiamondClassifyWorkerFactory@LocalWorkflow@U2@@SAXXZ$169 1001e8da f   DiamondClassifyWorkerFactory.obj
 0001:0001d8e6       __unwindfunclet$?init@DiamondClassifyWorkerFactory@LocalWorkflow@U2@@SAXXZ$170 1001e8e6 f   DiamondClassifyWorkerFactory.obj
 0001:0001d8ef       __unwindfunclet$?init@DiamondClassifyWorkerFactory@LocalWorkflow@U2@@SAXXZ$171 1001e8ef f   DiamondClassifyWorkerFactory.obj
 0001:0001d8f8       __unwindfunclet$?init@DiamondClassifyWorkerFactory@LocalWorkflow@U2@@SAXXZ$172 1001e8f8 f   DiamondClassifyWorkerFactory.obj
 0001:0001d901       __unwindfunclet$?init@DiamondClassifyWorkerFactory@LocalWorkflow@U2@@SAXXZ$173 1001e901 f   DiamondClassifyWorkerFactory.obj
 0001:0001d90a       __unwindfunclet$?init@DiamondClassifyWorkerFactory@LocalWorkflow@U2@@SAXXZ$174 1001e90a f   DiamondClassifyWorkerFactory.obj
 0001:0001d915       __unwindfunclet$?init@DiamondClassifyWorkerFactory@LocalWorkflow@U2@@SAXXZ$175 1001e915 f   DiamondClassifyWorkerFactory.obj
 0001:0001d91d       __unwindfunclet$?init@DiamondClassifyWorkerFactory@LocalWorkflow@U2@@SAXXZ$176 1001e91d f   DiamondClassifyWorkerFactory.obj
 0001:0001d926       __unwindfunclet$?init@DiamondClassifyWorkerFactory@LocalWorkflow@U2@@SAXXZ$177 1001e926 f   DiamondClassifyWorkerFactory.obj
 0001:0001d92f       __unwindfunclet$?init@DiamondClassifyWorkerFactory@LocalWorkflow@U2@@SAXXZ$178 1001e92f f   DiamondClassifyWorkerFactory.obj
 0001:0001d93b       __unwindfunclet$?init@DiamondClassifyWorkerFactory@LocalWorkflow@U2@@SAXXZ$179 1001e93b f   DiamondClassifyWorkerFactory.obj
 0001:0001d944       __unwindfunclet$?init@DiamondClassifyWorkerFactory@LocalWorkflow@U2@@SAXXZ$180 1001e944 f   DiamondClassifyWorkerFactory.obj
 0001:0001d94d       __unwindfunclet$?init@DiamondClassifyWorkerFactory@LocalWorkflow@U2@@SAXXZ$181 1001e94d f   DiamondClassifyWorkerFactory.obj
 0001:0001d956       __unwindfunclet$?init@DiamondClassifyWorkerFactory@LocalWorkflow@U2@@SAXXZ$182 1001e956 f   DiamondClassifyWorkerFactory.obj
 0001:0001d95f       __unwindfunclet$?init@DiamondClassifyWorkerFactory@LocalWorkflow@U2@@SAXXZ$183 1001e95f f   DiamondClassifyWorkerFactory.obj
 0001:0001d96a       __unwindfunclet$?init@DiamondClassifyWorkerFactory@LocalWorkflow@U2@@SAXXZ$184 1001e96a f   DiamondClassifyWorkerFactory.obj
 0001:0001d972       __unwindfunclet$?init@DiamondClassifyWorkerFactory@LocalWorkflow@U2@@SAXXZ$185 1001e972 f   DiamondClassifyWorkerFactory.obj
 0001:0001d97b       __unwindfunclet$?init@DiamondClassifyWorkerFactory@LocalWorkflow@U2@@SAXXZ$186 1001e97b f   DiamondClassifyWorkerFactory.obj
 0001:0001d984       __unwindfunclet$?init@DiamondClassifyWorkerFactory@LocalWorkflow@U2@@SAXXZ$187 1001e984 f   DiamondClassifyWorkerFactory.obj
 0001:0001d990       __unwindfunclet$?init@DiamondClassifyWorkerFactory@LocalWorkflow@U2@@SAXXZ$188 1001e990 f   DiamondClassifyWorkerFactory.obj
 0001:0001d999       __unwindfunclet$?init@DiamondClassifyWorkerFactory@LocalWorkflow@U2@@SAXXZ$189 1001e999 f   DiamondClassifyWorkerFactory.obj
 0001:0001d9a2       __unwindfunclet$?init@DiamondClassifyWorkerFactory@LocalWorkflow@U2@@SAXXZ$190 1001e9a2 f   DiamondClassifyWorkerFactory.obj
 0001:0001d9ab       __unwindfunclet$?init@DiamondClassifyWorkerFactory@LocalWorkflow@U2@@SAXXZ$191 1001e9ab f   DiamondClassifyWorkerFactory.obj
 0001:0001d9b4       __unwindfunclet$?init@DiamondClassifyWorkerFactory@LocalWorkflow@U2@@SAXXZ$192 1001e9b4 f   DiamondClassifyWorkerFactory.obj
 0001:0001d9bf       __unwindfunclet$?init@DiamondClassifyWorkerFactory@LocalWorkflow@U2@@SAXXZ$193 1001e9bf f   DiamondClassifyWorkerFactory.obj
 0001:0001d9c7       __unwindfunclet$?init@DiamondClassifyWorkerFactory@LocalWorkflow@U2@@SAXXZ$194 1001e9c7 f   DiamondClassifyWorkerFactory.obj
 0001:0001d9d0       __unwindfunclet$?init@DiamondClassifyWorkerFactory@LocalWorkflow@U2@@SAXXZ$195 1001e9d0 f   DiamondClassifyWorkerFactory.obj
 0001:0001d9d9       __unwindfunclet$?init@DiamondClassifyWorkerFactory@LocalWorkflow@U2@@SAXXZ$196 1001e9d9 f   DiamondClassifyWorkerFactory.obj
 0001:0001d9e5       __unwindfunclet$?init@DiamondClassifyWorkerFactory@LocalWorkflow@U2@@SAXXZ$197 1001e9e5 f   DiamondClassifyWorkerFactory.obj
 0001:0001d9ee       __unwindfunclet$?init@DiamondClassifyWorkerFactory@LocalWorkflow@U2@@SAXXZ$198 1001e9ee f   DiamondClassifyWorkerFactory.obj
 0001:0001d9fa       __unwindfunclet$?init@DiamondClassifyWorkerFactory@LocalWorkflow@U2@@SAXXZ$199 1001e9fa f   DiamondClassifyWorkerFactory.obj
 0001:0001da03       __unwindfunclet$?init@DiamondClassifyWorkerFactory@LocalWorkflow@U2@@SAXXZ$200 1001ea03 f   DiamondClassifyWorkerFactory.obj
 0001:0001da0e       __unwindfunclet$?init@DiamondClassifyWorkerFactory@LocalWorkflow@U2@@SAXXZ$201 1001ea0e f   DiamondClassifyWorkerFactory.obj
 0001:0001da16       __unwindfunclet$?init@DiamondClassifyWorkerFactory@LocalWorkflow@U2@@SAXXZ$202 1001ea16 f   DiamondClassifyWorkerFactory.obj
 0001:0001da1f       __unwindfunclet$?init@DiamondClassifyWorkerFactory@LocalWorkflow@U2@@SAXXZ$203 1001ea1f f   DiamondClassifyWorkerFactory.obj
 0001:0001da28       __unwindfunclet$?init@DiamondClassifyWorkerFactory@LocalWorkflow@U2@@SAXXZ$204 1001ea28 f   DiamondClassifyWorkerFactory.obj
 0001:0001da34       __unwindfunclet$?init@DiamondClassifyWorkerFactory@LocalWorkflow@U2@@SAXXZ$205 1001ea34 f   DiamondClassifyWorkerFactory.obj
 0001:0001da3d       __unwindfunclet$?init@DiamondClassifyWorkerFactory@LocalWorkflow@U2@@SAXXZ$206 1001ea3d f   DiamondClassifyWorkerFactory.obj
 0001:0001da49       __unwindfunclet$?init@DiamondClassifyWorkerFactory@LocalWorkflow@U2@@SAXXZ$207 1001ea49 f   DiamondClassifyWorkerFactory.obj
 0001:0001da52       __unwindfunclet$?init@DiamondClassifyWorkerFactory@LocalWorkflow@U2@@SAXXZ$208 1001ea52 f   DiamondClassifyWorkerFactory.obj
 0001:0001da5b       __unwindfunclet$?init@DiamondClassifyWorkerFactory@LocalWorkflow@U2@@SAXXZ$209 1001ea5b f   DiamondClassifyWorkerFactory.obj
 0001:0001da64       __unwindfunclet$?init@DiamondClassifyWorkerFactory@LocalWorkflow@U2@@SAXXZ$210 1001ea64 f   DiamondClassifyWorkerFactory.obj
 0001:0001da6d       __unwindfunclet$?init@DiamondClassifyWorkerFactory@LocalWorkflow@U2@@SAXXZ$211 1001ea6d f   DiamondClassifyWorkerFactory.obj
 0001:0001da78       __unwindfunclet$?init@DiamondClassifyWorkerFactory@LocalWorkflow@U2@@SAXXZ$212 1001ea78 f   DiamondClassifyWorkerFactory.obj
 0001:0001da80       __unwindfunclet$?init@DiamondClassifyWorkerFactory@LocalWorkflow@U2@@SAXXZ$213 1001ea80 f   DiamondClassifyWorkerFactory.obj
 0001:0001da89       __unwindfunclet$?init@DiamondClassifyWorkerFactory@LocalWorkflow@U2@@SAXXZ$214 1001ea89 f   DiamondClassifyWorkerFactory.obj
 0001:0001da92       __unwindfunclet$?init@DiamondClassifyWorkerFactory@LocalWorkflow@U2@@SAXXZ$215 1001ea92 f   DiamondClassifyWorkerFactory.obj
 0001:0001da9b       __unwindfunclet$?init@DiamondClassifyWorkerFactory@LocalWorkflow@U2@@SAXXZ$216 1001ea9b f   DiamondClassifyWorkerFactory.obj
 0001:0001daa4       __unwindfunclet$?init@DiamondClassifyWorkerFactory@LocalWorkflow@U2@@SAXXZ$217 1001eaa4 f   DiamondClassifyWorkerFactory.obj
 0001:0001daaf       __unwindfunclet$?init@DiamondClassifyWorkerFactory@LocalWorkflow@U2@@SAXXZ$218 1001eaaf f   DiamondClassifyWorkerFactory.obj
 0001:0001dabb       __unwindfunclet$?init@DiamondClassifyWorkerFactory@LocalWorkflow@U2@@SAXXZ$219 1001eabb f   DiamondClassifyWorkerFactory.obj
 0001:0001dac4       __unwindfunclet$?init@DiamondClassifyWorkerFactory@LocalWorkflow@U2@@SAXXZ$220 1001eac4 f   DiamondClassifyWorkerFactory.obj
 0001:0001dacc       __unwindfunclet$?init@DiamondClassifyWorkerFactory@LocalWorkflow@U2@@SAXXZ$221 1001eacc f   DiamondClassifyWorkerFactory.obj
 0001:0001dad5       __unwindfunclet$?init@DiamondClassifyWorkerFactory@LocalWorkflow@U2@@SAXXZ$222 1001ead5 f   DiamondClassifyWorkerFactory.obj
 0001:0001dade       __unwindfunclet$?init@DiamondClassifyWorkerFactory@LocalWorkflow@U2@@SAXXZ$223 1001eade f   DiamondClassifyWorkerFactory.obj
 0001:0001daea       __unwindfunclet$?init@DiamondClassifyWorkerFactory@LocalWorkflow@U2@@SAXXZ$224 1001eaea f   DiamondClassifyWorkerFactory.obj
 0001:0001daf5       __unwindfunclet$?init@DiamondClassifyWorkerFactory@LocalWorkflow@U2@@SAXXZ$225 1001eaf5 f   DiamondClassifyWorkerFactory.obj
 0001:0001db14       __unwindfunclet$?init@DiamondClassifyWorkerFactory@LocalWorkflow@U2@@SAXXZ$226 1001eb14 f   DiamondClassifyWorkerFactory.obj
 0001:0001db1d       __unwindfunclet$?init@DiamondClassifyWorkerFactory@LocalWorkflow@U2@@SAXXZ$227 1001eb1d f   DiamondClassifyWorkerFactory.obj
 0001:0001db26       __unwindfunclet$?init@DiamondClassifyWorkerFactory@LocalWorkflow@U2@@SAXXZ$228 1001eb26 f   DiamondClassifyWorkerFactory.obj
 0001:0001db32       __unwindfunclet$?init@DiamondClassifyWorkerFactory@LocalWorkflow@U2@@SAXXZ$229 1001eb32 f   DiamondClassifyWorkerFactory.obj
 0001:0001db3d       __unwindfunclet$?init@DiamondClassifyWorkerFactory@LocalWorkflow@U2@@SAXXZ$230 1001eb3d f   DiamondClassifyWorkerFactory.obj
 0001:0001db48       __unwindfunclet$?init@DiamondClassifyWorkerFactory@LocalWorkflow@U2@@SAXXZ$231 1001eb48 f   DiamondClassifyWorkerFactory.obj
 0001:0001db53       __unwindfunclet$?init@DiamondClassifyWorkerFactory@LocalWorkflow@U2@@SAXXZ$232 1001eb53 f   DiamondClassifyWorkerFactory.obj
 0001:0001db5c       __unwindfunclet$?init@DiamondClassifyWorkerFactory@LocalWorkflow@U2@@SAXXZ$233 1001eb5c f   DiamondClassifyWorkerFactory.obj
 0001:0001db65       __unwindfunclet$?init@DiamondClassifyWorkerFactory@LocalWorkflow@U2@@SAXXZ$234 1001eb65 f   DiamondClassifyWorkerFactory.obj
 0001:0001db70       __ehhandler$?init@DiamondClassifyWorkerFactory@LocalWorkflow@U2@@SAXXZ 1001eb70 f   DiamondClassifyWorkerFactory.obj
 0001:0001db90       __unwindfunclet$?node_construct@?$QList@U?$QPair@VQString@@V1@@@@@AAEXPAUNode@1@ABU?$QPair@VQString@@V1@@@@Z$0 1001eb90 f   DiamondClassifyWorkerFactory.obj
 0001:0001db9b       __unwindfunclet$?node_construct@?$QList@U?$QPair@VQString@@V1@@@@@AAEXPAUNode@1@ABU?$QPair@VQString@@V1@@@@Z$2 1001eb9b f   DiamondClassifyWorkerFactory.obj
 0001:0001dba4       __ehhandler$?node_construct@?$QList@U?$QPair@VQString@@V1@@@@@AAEXPAUNode@1@ABU?$QPair@VQString@@V1@@@@Z 1001eba4 f   DiamondClassifyWorkerFactory.obj
 0001:0001dbc0       __unwindfunclet$?node_construct@?$QList@U?$QPair@VQString@@VQVariant@@@@@@AAEXPAUNode@1@ABU?$QPair@VQString@@VQVariant@@@@@Z$0 1001ebc0 f   DiamondClassifyWorkerFactory.obj
 0001:0001dbcb       __unwindfunclet$?node_construct@?$QList@U?$QPair@VQString@@VQVariant@@@@@@AAEXPAUNode@1@ABU?$QPair@VQString@@VQVariant@@@@@Z$2 1001ebcb f   DiamondClassifyWorkerFactory.obj
 0001:0001dbd4       __ehhandler$?node_construct@?$QList@U?$QPair@VQString@@VQVariant@@@@@@AAEXPAUNode@1@ABU?$QPair@VQString@@VQVariant@@@@@Z 1001ebd4 f   DiamondClassifyWorkerFactory.obj
 0001:0001dbf0       __unwindfunclet$?node_copy@?$QList@U?$QPair@VQString@@V1@@@@@AAEXPAUNode@1@00@Z$4 1001ebf0 f   DiamondClassifyWorkerFactory.obj
 0001:0001dbfb       __unwindfunclet$?node_copy@?$QList@U?$QPair@VQString@@V1@@@@@AAEXPAUNode@1@00@Z$6 1001ebfb f   DiamondClassifyWorkerFactory.obj
 0001:0001dc04       __unwindfunclet$?node_copy@?$QList@U?$QPair@VQString@@V1@@@@@AAEXPAUNode@1@00@Z$8 1001ec04 f   DiamondClassifyWorkerFactory.obj
 0001:0001dc0d       __ehhandler$?node_copy@?$QList@U?$QPair@VQString@@V1@@@@@AAEXPAUNode@1@00@Z 1001ec0d f   DiamondClassifyWorkerFactory.obj
 0001:0001dc30       __unwindfunclet$?node_copy@?$QList@U?$QPair@VQString@@VQVariant@@@@@@AAEXPAUNode@1@00@Z$4 1001ec30 f   DiamondClassifyWorkerFactory.obj
 0001:0001dc3b       __unwindfunclet$?node_copy@?$QList@U?$QPair@VQString@@VQVariant@@@@@@AAEXPAUNode@1@00@Z$6 1001ec3b f   DiamondClassifyWorkerFactory.obj
 0001:0001dc44       __unwindfunclet$?node_copy@?$QList@U?$QPair@VQString@@VQVariant@@@@@@AAEXPAUNode@1@00@Z$8 1001ec44 f   DiamondClassifyWorkerFactory.obj
 0001:0001dc4d       __ehhandler$?node_copy@?$QList@U?$QPair@VQString@@VQVariant@@@@@@AAEXPAUNode@1@00@Z 1001ec4d f   DiamondClassifyWorkerFactory.obj
 0001:0001dc70       __unwindfunclet$?node_destruct@?$QList@U?$QPair@VQString@@V1@@@@@AAEXPAUNode@1@0@Z$0 1001ec70 f   DiamondClassifyWorkerFactory.obj
 0001:0001dc79       __ehhandler$?node_destruct@?$QList@U?$QPair@VQString@@V1@@@@@AAEXPAUNode@1@0@Z 1001ec79 f   DiamondClassifyWorkerFactory.obj
 0001:0001dca0       __unwindfunclet$?node_destruct@?$QList@U?$QPair@VQString@@V1@@@@@AAEXPAUNode@1@@Z$0 1001eca0 f   DiamondClassifyWorkerFactory.obj
 0001:0001dca9       __ehhandler$?node_destruct@?$QList@U?$QPair@VQString@@V1@@@@@AAEXPAUNode@1@@Z 1001eca9 f   DiamondClassifyWorkerFactory.obj
 0001:0001dcd0       __unwindfunclet$?node_destruct@?$QList@U?$QPair@VQString@@VQVariant@@@@@@AAEXPAUNode@1@0@Z$0 1001ecd0 f   DiamondClassifyWorkerFactory.obj
 0001:0001dcd9       __ehhandler$?node_destruct@?$QList@U?$QPair@VQString@@VQVariant@@@@@@AAEXPAUNode@1@0@Z 1001ecd9 f   DiamondClassifyWorkerFactory.obj
 0001:0001dd00       __unwindfunclet$?node_destruct@?$QList@U?$QPair@VQString@@VQVariant@@@@@@AAEXPAUNode@1@@Z$0 1001ed00 f   DiamondClassifyWorkerFactory.obj
 0001:0001dd09       __ehhandler$?node_destruct@?$QList@U?$QPair@VQString@@VQVariant@@@@@@AAEXPAUNode@1@@Z 1001ed09 f   DiamondClassifyWorkerFactory.obj
 0001:0001dd30       __unwindfunclet$??0DiamondSupport@U2@@QAE@ABVQString@@@Z$0 1001ed30 f   DiamondSupport.obj
 0001:0001dd39       __unwindfunclet$??0DiamondSupport@U2@@QAE@ABVQString@@@Z$2 1001ed39 f   DiamondSupport.obj
 0001:0001dd42       __unwindfunclet$??0DiamondSupport@U2@@QAE@ABVQString@@@Z$3 1001ed42 f   DiamondSupport.obj
 0001:0001dd4b       __unwindfunclet$??0DiamondSupport@U2@@QAE@ABVQString@@@Z$4 1001ed4b f   DiamondSupport.obj
 0001:0001dd54       __unwindfunclet$??0DiamondSupport@U2@@QAE@ABVQString@@@Z$5 1001ed54 f   DiamondSupport.obj
 0001:0001dd5d       __unwindfunclet$??0DiamondSupport@U2@@QAE@ABVQString@@@Z$6 1001ed5d f   DiamondSupport.obj
 0001:0001dd66       __ehhandler$??0DiamondSupport@U2@@QAE@ABVQString@@@Z 1001ed66 f   DiamondSupport.obj
 0001:0001dd90       __unwindfunclet$??0DiamondSupportPlugin@U2@@QAE@XZ$0 1001ed90 f   DiamondSupportPlugin.obj
 0001:0001dd99       __unwindfunclet$??0DiamondSupportPlugin@U2@@QAE@XZ$1 1001ed99 f   DiamondSupportPlugin.obj
 0001:0001dda4       __ehhandler$??0DiamondSupportPlugin@U2@@QAE@XZ 1001eda4 f   DiamondSupportPlugin.obj
 0001:0001ddc0       __unwindfunclet$??1DiamondSupportPlugin@U2@@UAE@XZ$0 1001edc0 f   DiamondSupportPlugin.obj
 0001:0001ddc9       __ehhandler$??1DiamondSupportPlugin@U2@@UAE@XZ 1001edc9 f   DiamondSupportPlugin.obj
 0001:0001ddf0       __unwindfunclet$??_GDiamondSupportPlugin@U2@@UAEPAXI@Z$0 1001edf0 f   DiamondSupportPlugin.obj
 0001:0001ddf9       __ehhandler$??_GDiamondSupportPlugin@U2@@UAEPAXI@Z 1001edf9 f   DiamondSupportPlugin.obj
 0001:0001de20       __unwindfunclet$??__EalgoLog@U2@@YAXXZ$0 1001ee20 f   DiamondSupportPlugin.obj
 0001:0001de29       __ehhandler$??__EalgoLog@U2@@YAXXZ 1001ee29 f   DiamondSupportPlugin.obj
 0001:0001de50       __unwindfunclet$??__EcmdLog@U2@@YAXXZ$0 1001ee50 f   DiamondSupportPlugin.obj
 0001:0001de59       __ehhandler$??__EcmdLog@U2@@YAXXZ 1001ee59 f   DiamondSupportPlugin.obj
 0001:0001de80       __unwindfunclet$??__EcoreLog@U2@@YAXXZ$0 1001ee80 f   DiamondSupportPlugin.obj
 0001:0001de89       __ehhandler$??__EcoreLog@U2@@YAXXZ 1001ee89 f   DiamondSupportPlugin.obj
 0001:0001deb0       __unwindfunclet$??__EioLog@U2@@YAXXZ$0 1001eeb0 f   DiamondSupportPlugin.obj
 0001:0001deb9       __ehhandler$??__EioLog@U2@@YAXXZ 1001eeb9 f   DiamondSupportPlugin.obj
 0001:0001dee0       __unwindfunclet$??__EperfLog@U2@@YAXXZ$0 1001eee0 f   DiamondSupportPlugin.obj
 0001:0001dee9       __ehhandler$??__EperfLog@U2@@YAXXZ 1001eee9 f   DiamondSupportPlugin.obj
 0001:0001df10       __unwindfunclet$??__EscriptLog@U2@@YAXXZ$0 1001ef10 f   DiamondSupportPlugin.obj
 0001:0001df19       __ehhandler$??__EscriptLog@U2@@YAXXZ 1001ef19 f   DiamondSupportPlugin.obj
 0001:0001df40       __unwindfunclet$??__EtaskLog@U2@@YAXXZ$0 1001ef40 f   DiamondSupportPlugin.obj
 0001:0001df49       __ehhandler$??__EtaskLog@U2@@YAXXZ 1001ef49 f   DiamondSupportPlugin.obj
 0001:0001df70       __unwindfunclet$??__EuiLog@U2@@YAXXZ$0 1001ef70 f   DiamondSupportPlugin.obj
 0001:0001df79       __ehhandler$??__EuiLog@U2@@YAXXZ 1001ef79 f   DiamondSupportPlugin.obj
 0001:0001dfa0       __unwindfunclet$??__EuserActLog@U2@@YAXXZ$0 1001efa0 f   DiamondSupportPlugin.obj
 0001:0001dfa9       __ehhandler$??__EuserActLog@U2@@YAXXZ 1001efa9 f   DiamondSupportPlugin.obj
 0001:0001dfd0       __unwindfunclet$??0GenomesPreparationTask@U2@@QAE@ABVQStringList@@ABVQString@@@Z$0 1001efd0 f   GenomesPreparationTask.obj
 0001:0001dfd9       __unwindfunclet$??0GenomesPreparationTask@U2@@QAE@ABVQStringList@@ABVQString@@@Z$1 1001efd9 f   GenomesPreparationTask.obj
 0001:0001dfe2       __unwindfunclet$??0GenomesPreparationTask@U2@@QAE@ABVQStringList@@ABVQString@@@Z$2 1001efe2 f   GenomesPreparationTask.obj
 0001:0001dff0       __unwindfunclet$??0GenomesPreparationTask@U2@@QAE@ABVQStringList@@ABVQString@@@Z$3 1001eff0 f   GenomesPreparationTask.obj
 0001:0001dfff       __unwindfunclet$??0GenomesPreparationTask@U2@@QAE@ABVQStringList@@ABVQString@@@Z$4 1001efff f   GenomesPreparationTask.obj
 0001:0001e008       __unwindfunclet$??0GenomesPreparationTask@U2@@QAE@ABVQStringList@@ABVQString@@@Z$5 1001f008 f   GenomesPreparationTask.obj
 0001:0001e011       __ehhandler$??0GenomesPreparationTask@U2@@QAE@ABVQStringList@@ABVQString@@@Z 1001f011 f   GenomesPreparationTask.obj
 0001:0001e030       __unwindfunclet$??1GenomesPreparationTask@U2@@UAE@XZ$0 1001f030 f   GenomesPreparationTask.obj
 0001:0001e039       __unwindfunclet$??1GenomesPreparationTask@U2@@UAE@XZ$1 1001f039 f   GenomesPreparationTask.obj
 0001:0001e047       __ehhandler$??1GenomesPreparationTask@U2@@UAE@XZ 1001f047 f   GenomesPreparationTask.obj
 0001:0001e070       __unwindfunclet$??_GGenomesPreparationTask@U2@@UAEPAXI@Z$0 1001f070 f   GenomesPreparationTask.obj
 0001:0001e079       __unwindfunclet$??_GGenomesPreparationTask@U2@@UAEPAXI@Z$1 1001f079 f   GenomesPreparationTask.obj
 0001:0001e087       __ehhandler$??_GGenomesPreparationTask@U2@@UAEPAXI@Z 1001f087 f   GenomesPreparationTask.obj
 0001:0001e0b0       __unwindfunclet$??__EalgoLog@U2@@YAXXZ$0 1001f0b0 f   GenomesPreparationTask.obj
 0001:0001e0b9       __ehhandler$??__EalgoLog@U2@@YAXXZ 1001f0b9 f   GenomesPreparationTask.obj
 0001:0001e0e0       __unwindfunclet$??__EcmdLog@U2@@YAXXZ$0 1001f0e0 f   GenomesPreparationTask.obj
 0001:0001e0e9       __ehhandler$??__EcmdLog@U2@@YAXXZ 1001f0e9 f   GenomesPreparationTask.obj
 0001:0001e110       __unwindfunclet$??__EcoreLog@U2@@YAXXZ$0 1001f110 f   GenomesPreparationTask.obj
 0001:0001e119       __ehhandler$??__EcoreLog@U2@@YAXXZ 1001f119 f   GenomesPreparationTask.obj
 0001:0001e140       __unwindfunclet$??__EioLog@U2@@YAXXZ$0 1001f140 f   GenomesPreparationTask.obj
 0001:0001e149       __ehhandler$??__EioLog@U2@@YAXXZ 1001f149 f   GenomesPreparationTask.obj
 0001:0001e170       __unwindfunclet$??__EperfLog@U2@@YAXXZ$0 1001f170 f   GenomesPreparationTask.obj
 0001:0001e179       __ehhandler$??__EperfLog@U2@@YAXXZ 1001f179 f   GenomesPreparationTask.obj
 0001:0001e1a0       __unwindfunclet$??__EscriptLog@U2@@YAXXZ$0 1001f1a0 f   GenomesPreparationTask.obj
 0001:0001e1a9       __ehhandler$??__EscriptLog@U2@@YAXXZ 1001f1a9 f   GenomesPreparationTask.obj
 0001:0001e1d0       __unwindfunclet$??__EtaskLog@U2@@YAXXZ$0 1001f1d0 f   GenomesPreparationTask.obj
 0001:0001e1d9       __ehhandler$??__EtaskLog@U2@@YAXXZ 1001f1d9 f   GenomesPreparationTask.obj
 0001:0001e200       __unwindfunclet$??__EuiLog@U2@@YAXXZ$0 1001f200 f   GenomesPreparationTask.obj
 0001:0001e209       __ehhandler$??__EuiLog@U2@@YAXXZ 1001f209 f   GenomesPreparationTask.obj
 0001:0001e230       __unwindfunclet$??__EuserActLog@U2@@YAXXZ$0 1001f230 f   GenomesPreparationTask.obj
 0001:0001e239       __ehhandler$??__EuserActLog@U2@@YAXXZ 1001f239 f   GenomesPreparationTask.obj
 0001:0001e260       __unwindfunclet$?run@GenomesPreparationTask@U2@@EAEXXZ$0 1001f260 f   GenomesPreparationTask.obj
 0001:0001e269       __unwindfunclet$?run@GenomesPreparationTask@U2@@EAEXXZ$1 1001f269 f   GenomesPreparationTask.obj
 0001:0001e272       __unwindfunclet$?run@GenomesPreparationTask@U2@@EAEXXZ$2 1001f272 f   GenomesPreparationTask.obj
 0001:0001e27b       __unwindfunclet$?run@GenomesPreparationTask@U2@@EAEXXZ$3 1001f27b f   GenomesPreparationTask.obj
 0001:0001e284       __unwindfunclet$?run@GenomesPreparationTask@U2@@EAEXXZ$4 1001f284 f   GenomesPreparationTask.obj
 0001:0001e28d       __unwindfunclet$?run@GenomesPreparationTask@U2@@EAEXXZ$5 1001f28d f   GenomesPreparationTask.obj
 0001:0001e296       __unwindfunclet$?run@GenomesPreparationTask@U2@@EAEXXZ$7 1001f296 f   GenomesPreparationTask.obj
 0001:0001e29f       __unwindfunclet$?run@GenomesPreparationTask@U2@@EAEXXZ$8 1001f29f f   GenomesPreparationTask.obj
 0001:0001e2a8       __unwindfunclet$?run@GenomesPreparationTask@U2@@EAEXXZ$6 1001f2a8 f   GenomesPreparationTask.obj
 0001:0001e2b1       __ehhandler$?run@GenomesPreparationTask@U2@@EAEXXZ 1001f2b1 f   GenomesPreparationTask.obj
 0001:0001e2d0       __unwindfunclet$??__EalgoLog@U2@@YAXXZ$0 1001f2d0 f   moc_DiamondBuildPrompter.obj
 0001:0001e2d9       __ehhandler$??__EalgoLog@U2@@YAXXZ 1001f2d9 f   moc_DiamondBuildPrompter.obj
 0001:0001e300       __unwindfunclet$??__EcmdLog@U2@@YAXXZ$0 1001f300 f   moc_DiamondBuildPrompter.obj
 0001:0001e309       __ehhandler$??__EcmdLog@U2@@YAXXZ 1001f309 f   moc_DiamondBuildPrompter.obj
 0001:0001e330       __unwindfunclet$??__EcoreLog@U2@@YAXXZ$0 1001f330 f   moc_DiamondBuildPrompter.obj
 0001:0001e339       __ehhandler$??__EcoreLog@U2@@YAXXZ 1001f339 f   moc_DiamondBuildPrompter.obj
 0001:0001e360       __unwindfunclet$??__EioLog@U2@@YAXXZ$0 1001f360 f   moc_DiamondBuildPrompter.obj
 0001:0001e369       __ehhandler$??__EioLog@U2@@YAXXZ 1001f369 f   moc_DiamondBuildPrompter.obj
 0001:0001e390       __unwindfunclet$??__EperfLog@U2@@YAXXZ$0 1001f390 f   moc_DiamondBuildPrompter.obj
 0001:0001e399       __ehhandler$??__EperfLog@U2@@YAXXZ 1001f399 f   moc_DiamondBuildPrompter.obj
 0001:0001e3c0       __unwindfunclet$??__EscriptLog@U2@@YAXXZ$0 1001f3c0 f   moc_DiamondBuildPrompter.obj
 0001:0001e3c9       __ehhandler$??__EscriptLog@U2@@YAXXZ 1001f3c9 f   moc_DiamondBuildPrompter.obj
 0001:0001e3f0       __unwindfunclet$??__EtaskLog@U2@@YAXXZ$0 1001f3f0 f   moc_DiamondBuildPrompter.obj
 0001:0001e3f9       __ehhandler$??__EtaskLog@U2@@YAXXZ 1001f3f9 f   moc_DiamondBuildPrompter.obj
 0001:0001e420       __unwindfunclet$??__EuiLog@U2@@YAXXZ$0 1001f420 f   moc_DiamondBuildPrompter.obj
 0001:0001e429       __ehhandler$??__EuiLog@U2@@YAXXZ 1001f429 f   moc_DiamondBuildPrompter.obj
 0001:0001e450       __unwindfunclet$??__EuserActLog@U2@@YAXXZ$0 1001f450 f   moc_DiamondBuildPrompter.obj
 0001:0001e459       __ehhandler$??__EuserActLog@U2@@YAXXZ 1001f459 f   moc_DiamondBuildPrompter.obj
 0001:0001e480       __unwindfunclet$??__EalgoLog@U2@@YAXXZ$0 1001f480 f   moc_DiamondBuildTask.obj
 0001:0001e489       __ehhandler$??__EalgoLog@U2@@YAXXZ 1001f489 f   moc_DiamondBuildTask.obj
 0001:0001e4b0       __unwindfunclet$??__EcmdLog@U2@@YAXXZ$0 1001f4b0 f   moc_DiamondBuildTask.obj
 0001:0001e4b9       __ehhandler$??__EcmdLog@U2@@YAXXZ 1001f4b9 f   moc_DiamondBuildTask.obj
 0001:0001e4e0       __unwindfunclet$??__EcoreLog@U2@@YAXXZ$0 1001f4e0 f   moc_DiamondBuildTask.obj
 0001:0001e4e9       __ehhandler$??__EcoreLog@U2@@YAXXZ 1001f4e9 f   moc_DiamondBuildTask.obj
 0001:0001e510       __unwindfunclet$??__EioLog@U2@@YAXXZ$0 1001f510 f   moc_DiamondBuildTask.obj
 0001:0001e519       __ehhandler$??__EioLog@U2@@YAXXZ 1001f519 f   moc_DiamondBuildTask.obj
 0001:0001e540       __unwindfunclet$??__EperfLog@U2@@YAXXZ$0 1001f540 f   moc_DiamondBuildTask.obj
 0001:0001e549       __ehhandler$??__EperfLog@U2@@YAXXZ 1001f549 f   moc_DiamondBuildTask.obj
 0001:0001e570       __unwindfunclet$??__EscriptLog@U2@@YAXXZ$0 1001f570 f   moc_DiamondBuildTask.obj
 0001:0001e579       __ehhandler$??__EscriptLog@U2@@YAXXZ 1001f579 f   moc_DiamondBuildTask.obj
 0001:0001e5a0       __unwindfunclet$??__EtaskLog@U2@@YAXXZ$0 1001f5a0 f   moc_DiamondBuildTask.obj
 0001:0001e5a9       __ehhandler$??__EtaskLog@U2@@YAXXZ 1001f5a9 f   moc_DiamondBuildTask.obj
 0001:0001e5d0       __unwindfunclet$??__EuiLog@U2@@YAXXZ$0 1001f5d0 f   moc_DiamondBuildTask.obj
 0001:0001e5d9       __ehhandler$??__EuiLog@U2@@YAXXZ 1001f5d9 f   moc_DiamondBuildTask.obj
 0001:0001e600       __unwindfunclet$??__EuserActLog@U2@@YAXXZ$0 1001f600 f   moc_DiamondBuildTask.obj
 0001:0001e609       __ehhandler$??__EuserActLog@U2@@YAXXZ 1001f609 f   moc_DiamondBuildTask.obj
 0001:0001e630       __unwindfunclet$??__EalgoLog@U2@@YAXXZ$0 1001f630 f   moc_DiamondBuildWorker.obj
 0001:0001e639       __ehhandler$??__EalgoLog@U2@@YAXXZ 1001f639 f   moc_DiamondBuildWorker.obj
 0001:0001e660       __unwindfunclet$??__EcmdLog@U2@@YAXXZ$0 1001f660 f   moc_DiamondBuildWorker.obj
 0001:0001e669       __ehhandler$??__EcmdLog@U2@@YAXXZ 1001f669 f   moc_DiamondBuildWorker.obj
 0001:0001e690       __unwindfunclet$??__EcoreLog@U2@@YAXXZ$0 1001f690 f   moc_DiamondBuildWorker.obj
 0001:0001e699       __ehhandler$??__EcoreLog@U2@@YAXXZ 1001f699 f   moc_DiamondBuildWorker.obj
 0001:0001e6c0       __unwindfunclet$??__EioLog@U2@@YAXXZ$0 1001f6c0 f   moc_DiamondBuildWorker.obj
 0001:0001e6c9       __ehhandler$??__EioLog@U2@@YAXXZ 1001f6c9 f   moc_DiamondBuildWorker.obj
 0001:0001e6f0       __unwindfunclet$??__EperfLog@U2@@YAXXZ$0 1001f6f0 f   moc_DiamondBuildWorker.obj
 0001:0001e6f9       __ehhandler$??__EperfLog@U2@@YAXXZ 1001f6f9 f   moc_DiamondBuildWorker.obj
 0001:0001e720       __unwindfunclet$??__EscriptLog@U2@@YAXXZ$0 1001f720 f   moc_DiamondBuildWorker.obj
 0001:0001e729       __ehhandler$??__EscriptLog@U2@@YAXXZ 1001f729 f   moc_DiamondBuildWorker.obj
 0001:0001e750       __unwindfunclet$??__EtaskLog@U2@@YAXXZ$0 1001f750 f   moc_DiamondBuildWorker.obj
 0001:0001e759       __ehhandler$??__EtaskLog@U2@@YAXXZ 1001f759 f   moc_DiamondBuildWorker.obj
 0001:0001e780       __unwindfunclet$??__EuiLog@U2@@YAXXZ$0 1001f780 f   moc_DiamondBuildWorker.obj
 0001:0001e789       __ehhandler$??__EuiLog@U2@@YAXXZ 1001f789 f   moc_DiamondBuildWorker.obj
 0001:0001e7b0       __unwindfunclet$??__EuserActLog@U2@@YAXXZ$0 1001f7b0 f   moc_DiamondBuildWorker.obj
 0001:0001e7b9       __ehhandler$??__EuserActLog@U2@@YAXXZ 1001f7b9 f   moc_DiamondBuildWorker.obj
 0001:0001e7e0       __unwindfunclet$?qt_metatype_id@?$QMetaTypeIdQObject@PAVTask@U2@@$00@@SAHXZ$0 1001f7e0 f   moc_DiamondBuildWorker.obj
 0001:0001e7e9       __ehhandler$?qt_metatype_id@?$QMetaTypeIdQObject@PAVTask@U2@@$00@@SAHXZ 1001f7e9 f   moc_DiamondBuildWorker.obj
 0001:0001e810       __unwindfunclet$??__EalgoLog@U2@@YAXXZ$0 1001f810 f   moc_DiamondClassifyPrompter.obj
 0001:0001e819       __ehhandler$??__EalgoLog@U2@@YAXXZ 1001f819 f   moc_DiamondClassifyPrompter.obj
 0001:0001e840       __unwindfunclet$??__EcmdLog@U2@@YAXXZ$0 1001f840 f   moc_DiamondClassifyPrompter.obj
 0001:0001e849       __ehhandler$??__EcmdLog@U2@@YAXXZ 1001f849 f   moc_DiamondClassifyPrompter.obj
 0001:0001e870       __unwindfunclet$??__EcoreLog@U2@@YAXXZ$0 1001f870 f   moc_DiamondClassifyPrompter.obj
 0001:0001e879       __ehhandler$??__EcoreLog@U2@@YAXXZ 1001f879 f   moc_DiamondClassifyPrompter.obj
 0001:0001e8a0       __unwindfunclet$??__EioLog@U2@@YAXXZ$0 1001f8a0 f   moc_DiamondClassifyPrompter.obj
 0001:0001e8a9       __ehhandler$??__EioLog@U2@@YAXXZ 1001f8a9 f   moc_DiamondClassifyPrompter.obj
 0001:0001e8d0       __unwindfunclet$??__EperfLog@U2@@YAXXZ$0 1001f8d0 f   moc_DiamondClassifyPrompter.obj
 0001:0001e8d9       __ehhandler$??__EperfLog@U2@@YAXXZ 1001f8d9 f   moc_DiamondClassifyPrompter.obj
 0001:0001e900       __unwindfunclet$??__EscriptLog@U2@@YAXXZ$0 1001f900 f   moc_DiamondClassifyPrompter.obj
 0001:0001e909       __ehhandler$??__EscriptLog@U2@@YAXXZ 1001f909 f   moc_DiamondClassifyPrompter.obj
 0001:0001e930       __unwindfunclet$??__EtaskLog@U2@@YAXXZ$0 1001f930 f   moc_DiamondClassifyPrompter.obj
 0001:0001e939       __ehhandler$??__EtaskLog@U2@@YAXXZ 1001f939 f   moc_DiamondClassifyPrompter.obj
 0001:0001e960       __unwindfunclet$??__EuiLog@U2@@YAXXZ$0 1001f960 f   moc_DiamondClassifyPrompter.obj
 0001:0001e969       __ehhandler$??__EuiLog@U2@@YAXXZ 1001f969 f   moc_DiamondClassifyPrompter.obj
 0001:0001e990       __unwindfunclet$??__EuserActLog@U2@@YAXXZ$0 1001f990 f   moc_DiamondClassifyPrompter.obj
 0001:0001e999       __ehhandler$??__EuserActLog@U2@@YAXXZ 1001f999 f   moc_DiamondClassifyPrompter.obj
 0001:0001e9c0       __unwindfunclet$??__EalgoLog@U2@@YAXXZ$0 1001f9c0 f   moc_DiamondClassifyTask.obj
 0001:0001e9c9       __ehhandler$??__EalgoLog@U2@@YAXXZ 1001f9c9 f   moc_DiamondClassifyTask.obj
 0001:0001e9f0       __unwindfunclet$??__EcmdLog@U2@@YAXXZ$0 1001f9f0 f   moc_DiamondClassifyTask.obj
 0001:0001e9f9       __ehhandler$??__EcmdLog@U2@@YAXXZ 1001f9f9 f   moc_DiamondClassifyTask.obj
 0001:0001ea20       __unwindfunclet$??__EcoreLog@U2@@YAXXZ$0 1001fa20 f   moc_DiamondClassifyTask.obj
 0001:0001ea29       __ehhandler$??__EcoreLog@U2@@YAXXZ 1001fa29 f   moc_DiamondClassifyTask.obj
 0001:0001ea50       __unwindfunclet$??__EioLog@U2@@YAXXZ$0 1001fa50 f   moc_DiamondClassifyTask.obj
 0001:0001ea59       __ehhandler$??__EioLog@U2@@YAXXZ 1001fa59 f   moc_DiamondClassifyTask.obj
 0001:0001ea80       __unwindfunclet$??__EperfLog@U2@@YAXXZ$0 1001fa80 f   moc_DiamondClassifyTask.obj
 0001:0001ea89       __ehhandler$??__EperfLog@U2@@YAXXZ 1001fa89 f   moc_DiamondClassifyTask.obj
 0001:0001eab0       __unwindfunclet$??__EscriptLog@U2@@YAXXZ$0 1001fab0 f   moc_DiamondClassifyTask.obj
 0001:0001eab9       __ehhandler$??__EscriptLog@U2@@YAXXZ 1001fab9 f   moc_DiamondClassifyTask.obj
 0001:0001eae0       __unwindfunclet$??__EtaskLog@U2@@YAXXZ$0 1001fae0 f   moc_DiamondClassifyTask.obj
 0001:0001eae9       __ehhandler$??__EtaskLog@U2@@YAXXZ 1001fae9 f   moc_DiamondClassifyTask.obj
 0001:0001eb10       __unwindfunclet$??__EuiLog@U2@@YAXXZ$0 1001fb10 f   moc_DiamondClassifyTask.obj
 0001:0001eb19       __ehhandler$??__EuiLog@U2@@YAXXZ 1001fb19 f   moc_DiamondClassifyTask.obj
 0001:0001eb40       __unwindfunclet$??__EuserActLog@U2@@YAXXZ$0 1001fb40 f   moc_DiamondClassifyTask.obj
 0001:0001eb49       __ehhandler$??__EuserActLog@U2@@YAXXZ 1001fb49 f   moc_DiamondClassifyTask.obj
 0001:0001eb70       __unwindfunclet$??__EalgoLog@U2@@YAXXZ$0 1001fb70 f   moc_DiamondClassifyWorker.obj
 0001:0001eb79       __ehhandler$??__EalgoLog@U2@@YAXXZ 1001fb79 f   moc_DiamondClassifyWorker.obj
 0001:0001eba0       __unwindfunclet$??__EcmdLog@U2@@YAXXZ$0 1001fba0 f   moc_DiamondClassifyWorker.obj
 0001:0001eba9       __ehhandler$??__EcmdLog@U2@@YAXXZ 1001fba9 f   moc_DiamondClassifyWorker.obj
 0001:0001ebd0       __unwindfunclet$??__EcoreLog@U2@@YAXXZ$0 1001fbd0 f   moc_DiamondClassifyWorker.obj
 0001:0001ebd9       __ehhandler$??__EcoreLog@U2@@YAXXZ 1001fbd9 f   moc_DiamondClassifyWorker.obj
 0001:0001ec00       __unwindfunclet$??__EioLog@U2@@YAXXZ$0 1001fc00 f   moc_DiamondClassifyWorker.obj
 0001:0001ec09       __ehhandler$??__EioLog@U2@@YAXXZ 1001fc09 f   moc_DiamondClassifyWorker.obj
 0001:0001ec30       __unwindfunclet$??__EperfLog@U2@@YAXXZ$0 1001fc30 f   moc_DiamondClassifyWorker.obj
 0001:0001ec39       __ehhandler$??__EperfLog@U2@@YAXXZ 1001fc39 f   moc_DiamondClassifyWorker.obj
 0001:0001ec60       __unwindfunclet$??__EscriptLog@U2@@YAXXZ$0 1001fc60 f   moc_DiamondClassifyWorker.obj
 0001:0001ec69       __ehhandler$??__EscriptLog@U2@@YAXXZ 1001fc69 f   moc_DiamondClassifyWorker.obj
 0001:0001ec90       __unwindfunclet$??__EtaskLog@U2@@YAXXZ$0 1001fc90 f   moc_DiamondClassifyWorker.obj
 0001:0001ec99       __ehhandler$??__EtaskLog@U2@@YAXXZ 1001fc99 f   moc_DiamondClassifyWorker.obj
 0001:0001ecc0       __unwindfunclet$??__EuiLog@U2@@YAXXZ$0 1001fcc0 f   moc_DiamondClassifyWorker.obj
 0001:0001ecc9       __ehhandler$??__EuiLog@U2@@YAXXZ 1001fcc9 f   moc_DiamondClassifyWorker.obj
 0001:0001ecf0       __unwindfunclet$??__EuserActLog@U2@@YAXXZ$0 1001fcf0 f   moc_DiamondClassifyWorker.obj
 0001:0001ecf9       __ehhandler$??__EuserActLog@U2@@YAXXZ 1001fcf9 f   moc_DiamondClassifyWorker.obj
 0001:0001ed20       __unwindfunclet$??__EalgoLog@U2@@YAXXZ$0 1001fd20 f   moc_GenomesPreparationTask.obj
 0001:0001ed29       __ehhandler$??__EalgoLog@U2@@YAXXZ 1001fd29 f   moc_GenomesPreparationTask.obj
 0001:0001ed50       __unwindfunclet$??__EcmdLog@U2@@YAXXZ$0 1001fd50 f   moc_GenomesPreparationTask.obj
 0001:0001ed59       __ehhandler$??__EcmdLog@U2@@YAXXZ 1001fd59 f   moc_GenomesPreparationTask.obj
 0001:0001ed80       __unwindfunclet$??__EcoreLog@U2@@YAXXZ$0 1001fd80 f   moc_GenomesPreparationTask.obj
 0001:0001ed89       __ehhandler$??__EcoreLog@U2@@YAXXZ 1001fd89 f   moc_GenomesPreparationTask.obj
 0001:0001edb0       __unwindfunclet$??__EioLog@U2@@YAXXZ$0 1001fdb0 f   moc_GenomesPreparationTask.obj
 0001:0001edb9       __ehhandler$??__EioLog@U2@@YAXXZ 1001fdb9 f   moc_GenomesPreparationTask.obj
 0001:0001ede0       __unwindfunclet$??__EperfLog@U2@@YAXXZ$0 1001fde0 f   moc_GenomesPreparationTask.obj
 0001:0001ede9       __ehhandler$??__EperfLog@U2@@YAXXZ 1001fde9 f   moc_GenomesPreparationTask.obj
 0001:0001ee10       __unwindfunclet$??__EscriptLog@U2@@YAXXZ$0 1001fe10 f   moc_GenomesPreparationTask.obj
 0001:0001ee19       __ehhandler$??__EscriptLog@U2@@YAXXZ 1001fe19 f   moc_GenomesPreparationTask.obj
 0001:0001ee40       __unwindfunclet$??__EtaskLog@U2@@YAXXZ$0 1001fe40 f   moc_GenomesPreparationTask.obj
 0001:0001ee49       __ehhandler$??__EtaskLog@U2@@YAXXZ 1001fe49 f   moc_GenomesPreparationTask.obj
 0001:0001ee70       __unwindfunclet$??__EuiLog@U2@@YAXXZ$0 1001fe70 f   moc_GenomesPreparationTask.obj
 0001:0001ee79       __ehhandler$??__EuiLog@U2@@YAXXZ 1001fe79 f   moc_GenomesPreparationTask.obj
 0001:0001eea0       __unwindfunclet$??__EuserActLog@U2@@YAXXZ$0 1001fea0 f   moc_GenomesPreparationTask.obj
 0001:0001eea9       __ehhandler$??__EuserActLog@U2@@YAXXZ 1001fea9 f   moc_GenomesPreparationTask.obj
 0001:0001eed0       ??__F?_Generic_object@?$_Error_objects@H@std@@2V_Generic_error_category@2@A@@YAXXZ 1001fed0 f   DiamondBuildPrompter.obj
 0001:0001eee0       ??__F?_Iostream_object@?$_Error_objects@H@std@@2V_Iostream_error_category@2@A@@YAXXZ 1001fee0 f   DiamondBuildPrompter.obj
 0001:0001eef0       ??__F?_System_object@?$_Error_objects@H@std@@2V_System_error_category@2@A@@YAXXZ 1001fef0 f   DiamondBuildPrompter.obj
 0001:0001ef00       ??__FalgoLog@U2@@YAXXZ     1001ff00 f   DiamondBuildPrompter.obj
 0001:0001ef10       ??__FcmdLog@U2@@YAXXZ      1001ff10 f   DiamondBuildPrompter.obj
 0001:0001ef20       ??__FcoreLog@U2@@YAXXZ     1001ff20 f   DiamondBuildPrompter.obj
 0001:0001ef30       ??__FioLog@U2@@YAXXZ       1001ff30 f   DiamondBuildPrompter.obj
 0001:0001ef40       ??__FperfLog@U2@@YAXXZ     1001ff40 f   DiamondBuildPrompter.obj
 0001:0001ef50       ??__FscriptLog@U2@@YAXXZ   1001ff50 f   DiamondBuildPrompter.obj
 0001:0001ef60       ??__FtaskLog@U2@@YAXXZ     1001ff60 f   DiamondBuildPrompter.obj
 0001:0001ef70       ??__FuiLog@U2@@YAXXZ       1001ff70 f   DiamondBuildPrompter.obj
 0001:0001ef80       ??__FuserActLog@U2@@YAXXZ  1001ff80 f   DiamondBuildPrompter.obj
 0001:0001ef90       ??__F?_Generic_object@?$_Error_objects@H@std@@2V_Generic_error_category@2@A@@YAXXZ 1001ff90 f   DiamondBuildTask.obj
 0001:0001efa0       ??__F?_Iostream_object@?$_Error_objects@H@std@@2V_Iostream_error_category@2@A@@YAXXZ 1001ffa0 f   DiamondBuildTask.obj
 0001:0001efb0       ??__F?_System_object@?$_Error_objects@H@std@@2V_System_error_category@2@A@@YAXXZ 1001ffb0 f   DiamondBuildTask.obj
 0001:0001efc0       ??__FalgoLog@U2@@YAXXZ     1001ffc0 f   DiamondBuildTask.obj
 0001:0001efd0       ??__FcmdLog@U2@@YAXXZ      1001ffd0 f   DiamondBuildTask.obj
 0001:0001efe0       ??__FcoreLog@U2@@YAXXZ     1001ffe0 f   DiamondBuildTask.obj
 0001:0001eff0       ??__Fcvar@?1???0DiamondBuildTask@U2@@QAE@ABUDiamondBuildTaskSettings@1@@Z@YAXXZ 1001fff0 f   DiamondBuildTask.obj
 0001:0001f000       ??__FioLog@U2@@YAXXZ       10020000 f   DiamondBuildTask.obj
 0001:0001f010       ??__FperfLog@U2@@YAXXZ     10020010 f   DiamondBuildTask.obj
 0001:0001f020       ??__FscriptLog@U2@@YAXXZ   10020020 f   DiamondBuildTask.obj
 0001:0001f030       ??__FtaskLog@U2@@YAXXZ     10020030 f   DiamondBuildTask.obj
 0001:0001f040       ??__FuiLog@U2@@YAXXZ       10020040 f   DiamondBuildTask.obj
 0001:0001f050       ??__FuserActLog@U2@@YAXXZ  10020050 f   DiamondBuildTask.obj
 0001:0001f060       ??__F?_Generic_object@?$_Error_objects@H@std@@2V_Generic_error_category@2@A@@YAXXZ 10020060 f   DiamondBuildValidator.obj
 0001:0001f070       ??__F?_Iostream_object@?$_Error_objects@H@std@@2V_Iostream_error_category@2@A@@YAXXZ 10020070 f   DiamondBuildValidator.obj
 0001:0001f080       ??__F?_System_object@?$_Error_objects@H@std@@2V_System_error_category@2@A@@YAXXZ 10020080 f   DiamondBuildValidator.obj
 0001:0001f090       ??__FalgoLog@U2@@YAXXZ     10020090 f   DiamondBuildValidator.obj
 0001:0001f0a0       ??__FcmdLog@U2@@YAXXZ      100200a0 f   DiamondBuildValidator.obj
 0001:0001f0b0       ??__FcoreLog@U2@@YAXXZ     100200b0 f   DiamondBuildValidator.obj
 0001:0001f0c0       ??__FioLog@U2@@YAXXZ       100200c0 f   DiamondBuildValidator.obj
 0001:0001f0d0       ??__FperfLog@U2@@YAXXZ     100200d0 f   DiamondBuildValidator.obj
 0001:0001f0e0       ??__FscriptLog@U2@@YAXXZ   100200e0 f   DiamondBuildValidator.obj
 0001:0001f0f0       ??__FtaskLog@U2@@YAXXZ     100200f0 f   DiamondBuildValidator.obj
 0001:0001f100       ??__FuiLog@U2@@YAXXZ       10020100 f   DiamondBuildValidator.obj
 0001:0001f110       ??__FuserActLog@U2@@YAXXZ  10020110 f   DiamondBuildValidator.obj
 0001:0001f120       ??__F?DIAMOND_BUILD_DIR@DiamondBuildWorker@LocalWorkflow@U2@@0VQString@@B@@YAXXZ 10020120 f   DiamondBuildWorker.obj
 0001:0001f130       ??__F?_Generic_object@?$_Error_objects@H@std@@2V_Generic_error_category@2@A@@YAXXZ 10020130 f   DiamondBuildWorker.obj
 0001:0001f140       ??__F?_Iostream_object@?$_Error_objects@H@std@@2V_Iostream_error_category@2@A@@YAXXZ 10020140 f   DiamondBuildWorker.obj
 0001:0001f150       ??__F?_System_object@?$_Error_objects@H@std@@2V_System_error_category@2@A@@YAXXZ 10020150 f   DiamondBuildWorker.obj
 0001:0001f160       ??__FalgoLog@U2@@YAXXZ     10020160 f   DiamondBuildWorker.obj
 0001:0001f170       ??__FcmdLog@U2@@YAXXZ      10020170 f   DiamondBuildWorker.obj
 0001:0001f180       ??__FcoreLog@U2@@YAXXZ     10020180 f   DiamondBuildWorker.obj
 0001:0001f190       ??__FioLog@U2@@YAXXZ       10020190 f   DiamondBuildWorker.obj
 0001:0001f1a0       ??__FperfLog@U2@@YAXXZ     100201a0 f   DiamondBuildWorker.obj
 0001:0001f1b0       ??__FscriptLog@U2@@YAXXZ   100201b0 f   DiamondBuildWorker.obj
 0001:0001f1c0       ??__FtaskLog@U2@@YAXXZ     100201c0 f   DiamondBuildWorker.obj
 0001:0001f1d0       ??__FuiLog@U2@@YAXXZ       100201d0 f   DiamondBuildWorker.obj
 0001:0001f1e0       ??__FuserActLog@U2@@YAXXZ  100201e0 f   DiamondBuildWorker.obj
 0001:0001f1f0       ??__F?ACTOR_ID@DiamondBuildWorkerFactory@LocalWorkflow@U2@@2VQString@@B@@YAXXZ 100201f0 f   DiamondBuildWorkerFactory.obj
 0001:0001f200       ??__F?DATABASE_ATTR_ID@DiamondBuildWorkerFactory@LocalWorkflow@U2@@2VQString@@B@@YAXXZ 10020200 f   DiamondBuildWorkerFactory.obj
 0001:0001f210       ??__F?GENOMIC_LIBRARY_ATTR_ID@DiamondBuildWorkerFactory@LocalWorkflow@U2@@2VQString@@B@@YAXXZ 10020210 f   DiamondBuildWorkerFactory.obj
 0001:0001f220       ??__F?OUTPUT_PORT_ID@DiamondBuildWorkerFactory@LocalWorkflow@U2@@2VQString@@B@@YAXXZ 10020220 f   DiamondBuildWorkerFactory.obj
 0001:0001f230       ??__F?_Generic_object@?$_Error_objects@H@std@@2V_Generic_error_category@2@A@@YAXXZ 10020230 f   DiamondBuildWorkerFactory.obj
 0001:0001f240       ??__F?_Iostream_object@?$_Error_objects@H@std@@2V_Iostream_error_category@2@A@@YAXXZ 10020240 f   DiamondBuildWorkerFactory.obj
 0001:0001f250       ??__F?_System_object@?$_Error_objects@H@std@@2V_System_error_category@2@A@@YAXXZ 10020250 f   DiamondBuildWorkerFactory.obj
 0001:0001f260       ??__FalgoLog@U2@@YAXXZ     10020260 f   DiamondBuildWorkerFactory.obj
 0001:0001f270       ??__FcmdLog@U2@@YAXXZ      10020270 f   DiamondBuildWorkerFactory.obj
 0001:0001f280       ??__FcoreLog@U2@@YAXXZ     10020280 f   DiamondBuildWorkerFactory.obj
 0001:0001f290       ??__FioLog@U2@@YAXXZ       10020290 f   DiamondBuildWorkerFactory.obj
 0001:0001f2a0       ??__FperfLog@U2@@YAXXZ     100202a0 f   DiamondBuildWorkerFactory.obj
 0001:0001f2b0       ??__FscriptLog@U2@@YAXXZ   100202b0 f   DiamondBuildWorkerFactory.obj
 0001:0001f2c0       ??__FtaskLog@U2@@YAXXZ     100202c0 f   DiamondBuildWorkerFactory.obj
 0001:0001f2d0       ??__FuiLog@U2@@YAXXZ       100202d0 f   DiamondBuildWorkerFactory.obj
 0001:0001f2e0       ??__FuserActLog@U2@@YAXXZ  100202e0 f   DiamondBuildWorkerFactory.obj
 0001:0001f2f0       ??__F?_Generic_object@?$_Error_objects@H@std@@2V_Generic_error_category@2@A@@YAXXZ 100202f0 f   DiamondClassifyPrompter.obj
 0001:0001f300       ??__F?_Iostream_object@?$_Error_objects@H@std@@2V_Iostream_error_category@2@A@@YAXXZ 10020300 f   DiamondClassifyPrompter.obj
 0001:0001f310       ??__F?_System_object@?$_Error_objects@H@std@@2V_System_error_category@2@A@@YAXXZ 10020310 f   DiamondClassifyPrompter.obj
 0001:0001f320       ??__FalgoLog@U2@@YAXXZ     10020320 f   DiamondClassifyPrompter.obj
 0001:0001f330       ??__FcmdLog@U2@@YAXXZ      10020330 f   DiamondClassifyPrompter.obj
 0001:0001f340       ??__FcoreLog@U2@@YAXXZ     10020340 f   DiamondClassifyPrompter.obj
 0001:0001f350       ??__FioLog@U2@@YAXXZ       10020350 f   DiamondClassifyPrompter.obj
 0001:0001f360       ??__FperfLog@U2@@YAXXZ     10020360 f   DiamondClassifyPrompter.obj
 0001:0001f370       ??__FscriptLog@U2@@YAXXZ   10020370 f   DiamondClassifyPrompter.obj
 0001:0001f380       ??__FtaskLog@U2@@YAXXZ     10020380 f   DiamondClassifyPrompter.obj
 0001:0001f390       ??__FuiLog@U2@@YAXXZ       10020390 f   DiamondClassifyPrompter.obj
 0001:0001f3a0       ??__FuserActLog@U2@@YAXXZ  100203a0 f   DiamondClassifyPrompter.obj
 0001:0001f3b0       ??__F?BLOSUM45@DiamondClassifyTaskSettings@U2@@2VQString@@B@@YAXXZ 100203b0 f   DiamondClassifyTask.obj
 0001:0001f3c0       ??__F?BLOSUM50@DiamondClassifyTaskSettings@U2@@2VQString@@B@@YAXXZ 100203c0 f   DiamondClassifyTask.obj
 0001:0001f3d0       ??__F?BLOSUM62@DiamondClassifyTaskSettings@U2@@2VQString@@B@@YAXXZ 100203d0 f   DiamondClassifyTask.obj
 0001:0001f3e0       ??__F?BLOSUM80@DiamondClassifyTaskSettings@U2@@2VQString@@B@@YAXXZ 100203e0 f   DiamondClassifyTask.obj
 0001:0001f3f0       ??__F?BLOSUM90@DiamondClassifyTaskSettings@U2@@2VQString@@B@@YAXXZ 100203f0 f   DiamondClassifyTask.obj
 0001:0001f400       ??__F?PAM250@DiamondClassifyTaskSettings@U2@@2VQString@@B@@YAXXZ 10020400 f   DiamondClassifyTask.obj
 0001:0001f410       ??__F?PAM30@DiamondClassifyTaskSettings@U2@@2VQString@@B@@YAXXZ 10020410 f   DiamondClassifyTask.obj
 0001:0001f420       ??__F?PAM70@DiamondClassifyTaskSettings@U2@@2VQString@@B@@YAXXZ 10020420 f   DiamondClassifyTask.obj
 0001:0001f430       ??__F?SENSITIVE_DEFAULT@DiamondClassifyTaskSettings@U2@@2VQString@@B@@YAXXZ 10020430 f   DiamondClassifyTask.obj
 0001:0001f440       ??__F?SENSITIVE_HIGH@DiamondClassifyTaskSettings@U2@@2VQString@@B@@YAXXZ 10020440 f   DiamondClassifyTask.obj
 0001:0001f450       ??__F?SENSITIVE_ULTRA@DiamondClassifyTaskSettings@U2@@2VQString@@B@@YAXXZ 10020450 f   DiamondClassifyTask.obj
 0001:0001f460       ??__F?TAXONOMIC_CLASSIFICATION_OUTPUT_FORMAT@DiamondClassifyTask@U2@@0VQString@@B@@YAXXZ 10020460 f   DiamondClassifyTask.obj
 0001:0001f470       ??__F?_Generic_object@?$_Error_objects@H@std@@2V_Generic_error_category@2@A@@YAXXZ 10020470 f   DiamondClassifyTask.obj
 0001:0001f480       ??__F?_Iostream_object@?$_Error_objects@H@std@@2V_Iostream_error_category@2@A@@YAXXZ 10020480 f   DiamondClassifyTask.obj
 0001:0001f490       ??__F?_System_object@?$_Error_objects@H@std@@2V_System_error_category@2@A@@YAXXZ 10020490 f   DiamondClassifyTask.obj
 0001:0001f4a0       ??__FalgoLog@U2@@YAXXZ     100204a0 f   DiamondClassifyTask.obj
 0001:0001f4b0       ??__FcmdLog@U2@@YAXXZ      100204b0 f   DiamondClassifyTask.obj
 0001:0001f4c0       ??__FcoreLog@U2@@YAXXZ     100204c0 f   DiamondClassifyTask.obj
 0001:0001f4d0       ??__Fcvar@?1???0DiamondClassifyTask@U2@@QAE@ABUDiamondClassifyTaskSettings@1@@Z@YAXXZ 100204d0 f   DiamondClassifyTask.obj
 0001:0001f4e0       ??__FioLog@U2@@YAXXZ       100204e0 f   DiamondClassifyTask.obj
 0001:0001f4f0       ??__FperfLog@U2@@YAXXZ     100204f0 f   DiamondClassifyTask.obj
 0001:0001f500       ??__FscriptLog@U2@@YAXXZ   10020500 f   DiamondClassifyTask.obj
 0001:0001f510       ??__FtaskLog@U2@@YAXXZ     10020510 f   DiamondClassifyTask.obj
 0001:0001f520       ??__FuiLog@U2@@YAXXZ       10020520 f   DiamondClassifyTask.obj
 0001:0001f530       ??__FuserActLog@U2@@YAXXZ  10020530 f   DiamondClassifyTask.obj
 0001:0001f540       ??__F?DIAMOND_DIR@DiamondClassifyWorker@LocalWorkflow@U2@@0VQString@@B@@YAXXZ 10020540 f   DiamondClassifyWorker.obj
 0001:0001f550       ??__F?_Generic_object@?$_Error_objects@H@std@@2V_Generic_error_category@2@A@@YAXXZ 10020550 f   DiamondClassifyWorker.obj
 0001:0001f560       ??__F?_Iostream_object@?$_Error_objects@H@std@@2V_Iostream_error_category@2@A@@YAXXZ 10020560 f   DiamondClassifyWorker.obj
 0001:0001f570       ??__F?_System_object@?$_Error_objects@H@std@@2V_System_error_category@2@A@@YAXXZ 10020570 f   DiamondClassifyWorker.obj
 0001:0001f580       ??__FalgoLog@U2@@YAXXZ     10020580 f   DiamondClassifyWorker.obj
 0001:0001f590       ??__FcmdLog@U2@@YAXXZ      10020590 f   DiamondClassifyWorker.obj
 0001:0001f5a0       ??__FcoreLog@U2@@YAXXZ     100205a0 f   DiamondClassifyWorker.obj
 0001:0001f5d0       ??__FioLog@U2@@YAXXZ       100205d0 f   DiamondClassifyWorker.obj
 0001:0001f5e0       ??__FperfLog@U2@@YAXXZ     100205e0 f   DiamondClassifyWorker.obj
 0001:0001f5f0       ??__FscriptLog@U2@@YAXXZ   100205f0 f   DiamondClassifyWorker.obj
 0001:0001f600       ??__FtaskLog@U2@@YAXXZ     10020600 f   DiamondClassifyWorker.obj
 0001:0001f610       ??__FuiLog@U2@@YAXXZ       10020610 f   DiamondClassifyWorker.obj
 0001:0001f620       ??__FuserActLog@U2@@YAXXZ  10020620 f   DiamondClassifyWorker.obj
 0001:0001f630       ??__F?ACTOR_ID@DiamondClassifyWorkerFactory@LocalWorkflow@U2@@2VQString@@B@@YAXXZ 10020630 f   DiamondClassifyWorkerFactory.obj
 0001:0001f640       ??__F?BSIZE_ATTR_ID@DiamondClassifyWorkerFactory@LocalWorkflow@U2@@2VQString@@B@@YAXXZ 10020640 f   DiamondClassifyWorkerFactory.obj
 0001:0001f650       ??__F?CHUNKS_ATTR_ID@DiamondClassifyWorkerFactory@LocalWorkflow@U2@@2VQString@@B@@YAXXZ 10020650 f   DiamondClassifyWorkerFactory.obj
 0001:0001f660       ??__F?DATABASE_ATTR_ID@DiamondClassifyWorkerFactory@LocalWorkflow@U2@@2VQString@@B@@YAXXZ 10020660 f   DiamondClassifyWorkerFactory.obj
 0001:0001f670       ??__F?EVALUE_ATTR_ID@DiamondClassifyWorkerFactory@LocalWorkflow@U2@@2VQString@@B@@YAXXZ 10020670 f   DiamondClassifyWorkerFactory.obj
 0001:0001f680       ??__F?FSHIFT_ATTR_ID@DiamondClassifyWorkerFactory@LocalWorkflow@U2@@2VQString@@B@@YAXXZ 10020680 f   DiamondClassifyWorkerFactory.obj
 0001:0001f690       ??__F?GENCODE_ATTR_ID@DiamondClassifyWorkerFactory@LocalWorkflow@U2@@2VQString@@B@@YAXXZ 10020690 f   DiamondClassifyWorkerFactory.obj
 0001:0001f6a0       ??__F?GE_PEN_ATTR_ID@DiamondClassifyWorkerFactory@LocalWorkflow@U2@@2VQString@@B@@YAXXZ 100206a0 f   DiamondClassifyWorkerFactory.obj
 0001:0001f6b0       ??__F?GO_PEN_ATTR_ID@DiamondClassifyWorkerFactory@LocalWorkflow@U2@@2VQString@@B@@YAXXZ 100206b0 f   DiamondClassifyWorkerFactory.obj
 0001:0001f6c0       ??__F?INPUT_DATA_ATTR_ID@DiamondClassifyWorkerFactory@LocalWorkflow@U2@@2VQString@@B@@YAXXZ 100206c0 f   DiamondClassifyWorkerFactory.obj
 0001:0001f6d0       ??__F?INPUT_PORT_ID@DiamondClassifyWorkerFactory@LocalWorkflow@U2@@2VQString@@B@@YAXXZ 100206d0 f   DiamondClassifyWorkerFactory.obj
 0001:0001f6e0       ??__F?INPUT_SLOT@DiamondClassifyWorkerFactory@LocalWorkflow@U2@@2VQString@@B@@YAXXZ 100206e0 f   DiamondClassifyWorkerFactory.obj
 0001:0001f6f0       ??__F?MATRIX_ATTR_ID@DiamondClassifyWorkerFactory@LocalWorkflow@U2@@2VQString@@B@@YAXXZ 100206f0 f   DiamondClassifyWorkerFactory.obj
 0001:0001f700       ??__F?OUTPUT_PORT_ID@DiamondClassifyWorkerFactory@LocalWorkflow@U2@@2VQString@@B@@YAXXZ 10020700 f   DiamondClassifyWorkerFactory.obj
 0001:0001f710       ??__F?OUTPUT_URL_ATTR_ID@DiamondClassifyWorkerFactory@LocalWorkflow@U2@@2VQString@@B@@YAXXZ 10020710 f   DiamondClassifyWorkerFactory.obj
 0001:0001f720       ??__F?SENSITIVE_ATTR_ID@DiamondClassifyWorkerFactory@LocalWorkflow@U2@@2VQString@@B@@YAXXZ 10020720 f   DiamondClassifyWorkerFactory.obj
 0001:0001f730       ??__F?THREADS_ATTR_ID@DiamondClassifyWorkerFactory@LocalWorkflow@U2@@2VQString@@B@@YAXXZ 10020730 f   DiamondClassifyWorkerFactory.obj
 0001:0001f740       ??__F?TOP_ALIGNMENTS_PERCENTAGE_ATTR_ID@DiamondClassifyWorkerFactory@LocalWorkflow@U2@@2VQString@@B@@YAXXZ 10020740 f   DiamondClassifyWorkerFactory.obj
 0001:0001f750       ??__F?WORKFLOW_CLASSIFY_TOOL_DIAMOND@DiamondClassifyWorkerFactory@LocalWorkflow@U2@@2VQString@@B@@YAXXZ 10020750 f   DiamondClassifyWorkerFactory.obj
 0001:0001f760       ??__F?_Generic_object@?$_Error_objects@H@std@@2V_Generic_error_category@2@A@@YAXXZ 10020760 f   DiamondClassifyWorkerFactory.obj
 0001:0001f770       ??__F?_Iostream_object@?$_Error_objects@H@std@@2V_Iostream_error_category@2@A@@YAXXZ 10020770 f   DiamondClassifyWorkerFactory.obj
 0001:0001f780       ??__F?_System_object@?$_Error_objects@H@std@@2V_System_error_category@2@A@@YAXXZ 10020780 f   DiamondClassifyWorkerFactory.obj
 0001:0001f790       ??__FalgoLog@U2@@YAXXZ     10020790 f   DiamondClassifyWorkerFactory.obj
 0001:0001f7a0       ??__FcmdLog@U2@@YAXXZ      100207a0 f   DiamondClassifyWorkerFactory.obj
 0001:0001f7b0       ??__FcoreLog@U2@@YAXXZ     100207b0 f   DiamondClassifyWorkerFactory.obj
 0001:0001f7c0       ??__FioLog@U2@@YAXXZ       100207c0 f   DiamondClassifyWorkerFactory.obj
 0001:0001f7d0       ??__FperfLog@U2@@YAXXZ     100207d0 f   DiamondClassifyWorkerFactory.obj
 0001:0001f7e0       ??__FscriptLog@U2@@YAXXZ   100207e0 f   DiamondClassifyWorkerFactory.obj
 0001:0001f7f0       ??__FtaskLog@U2@@YAXXZ     100207f0 f   DiamondClassifyWorkerFactory.obj
 0001:0001f800       ??__FuiLog@U2@@YAXXZ       10020800 f   DiamondClassifyWorkerFactory.obj
 0001:0001f810       ??__FuserActLog@U2@@YAXXZ  10020810 f   DiamondClassifyWorkerFactory.obj
 0001:0001f820       ??__F?TOOL_NAME@DiamondSupport@U2@@2VQString@@B@@YAXXZ 10020820 f   DiamondSupport.obj
 0001:0001f830       ??__F?_Generic_object@?$_Error_objects@H@std@@2V_Generic_error_category@2@A@@YAXXZ 10020830 f   DiamondSupport.obj
 0001:0001f840       ??__F?_Iostream_object@?$_Error_objects@H@std@@2V_Iostream_error_category@2@A@@YAXXZ 10020840 f   DiamondSupport.obj
 0001:0001f850       ??__F?_System_object@?$_Error_objects@H@std@@2V_System_error_category@2@A@@YAXXZ 10020850 f   DiamondSupport.obj
 0001:0001f860       ??__F?PLUGIN_DESCRIPRION@DiamondSupportPlugin@U2@@2VQString@@B@@YAXXZ 10020860 f   DiamondSupportPlugin.obj
 0001:0001f870       ??__F?PLUGIN_NAME@DiamondSupportPlugin@U2@@2VQString@@B@@YAXXZ 10020870 f   DiamondSupportPlugin.obj
 0001:0001f880       ??__F?_Generic_object@?$_Error_objects@H@std@@2V_Generic_error_category@2@A@@YAXXZ 10020880 f   DiamondSupportPlugin.obj
 0001:0001f890       ??__F?_Iostream_object@?$_Error_objects@H@std@@2V_Iostream_error_category@2@A@@YAXXZ 10020890 f   DiamondSupportPlugin.obj
 0001:0001f8a0       ??__F?_System_object@?$_Error_objects@H@std@@2V_System_error_category@2@A@@YAXXZ 100208a0 f   DiamondSupportPlugin.obj
 0001:0001f8b0       ??__FalgoLog@U2@@YAXXZ     100208b0 f   DiamondSupportPlugin.obj
 0001:0001f8c0       ??__FcmdLog@U2@@YAXXZ      100208c0 f   DiamondSupportPlugin.obj
 0001:0001f8d0       ??__FcoreLog@U2@@YAXXZ     100208d0 f   DiamondSupportPlugin.obj
 0001:0001f8e0       ??__FioLog@U2@@YAXXZ       100208e0 f   DiamondSupportPlugin.obj
 0001:0001f8f0       ??__FperfLog@U2@@YAXXZ     100208f0 f   DiamondSupportPlugin.obj
 0001:0001f900       ??__FscriptLog@U2@@YAXXZ   10020900 f   DiamondSupportPlugin.obj
 0001:0001f910       ??__FtaskLog@U2@@YAXXZ     10020910 f   DiamondSupportPlugin.obj
 0001:0001f920       ??__FuiLog@U2@@YAXXZ       10020920 f   DiamondSupportPlugin.obj
 0001:0001f930       ??__FuserActLog@U2@@YAXXZ  10020930 f   DiamondSupportPlugin.obj
 0001:0001f940       ??__F?_Generic_object@?$_Error_objects@H@std@@2V_Generic_error_category@2@A@@YAXXZ 10020940 f   GenomesPreparationTask.obj
 0001:0001f950       ??__F?_Iostream_object@?$_Error_objects@H@std@@2V_Iostream_error_category@2@A@@YAXXZ 10020950 f   GenomesPreparationTask.obj
 0001:0001f960       ??__F?_System_object@?$_Error_objects@H@std@@2V_System_error_category@2@A@@YAXXZ 10020960 f   GenomesPreparationTask.obj
 0001:0001f970       ??__FalgoLog@U2@@YAXXZ     10020970 f   GenomesPreparationTask.obj
 0001:0001f980       ??__FcmdLog@U2@@YAXXZ      10020980 f   GenomesPreparationTask.obj
 0001:0001f990       ??__FcoreLog@U2@@YAXXZ     10020990 f   GenomesPreparationTask.obj
 0001:0001f9a0       ??__FioLog@U2@@YAXXZ       100209a0 f   GenomesPreparationTask.obj
 0001:0001f9b0       ??__FperfLog@U2@@YAXXZ     100209b0 f   GenomesPreparationTask.obj
 0001:0001f9c0       ??__FscriptLog@U2@@YAXXZ   100209c0 f   GenomesPreparationTask.obj
 0001:0001f9d0       ??__FtaskLog@U2@@YAXXZ     100209d0 f   GenomesPreparationTask.obj
 0001:0001f9e0       ??__FuiLog@U2@@YAXXZ       100209e0 f   GenomesPreparationTask.obj
 0001:0001f9f0       ??__FuserActLog@U2@@YAXXZ  100209f0 f   GenomesPreparationTask.obj
 0001:0001fa00       ??__F?_Generic_object@?$_Error_objects@H@std@@2V_Generic_error_category@2@A@@YAXXZ 10020a00 f   moc_DiamondBuildPrompter.obj
 0001:0001fa10       ??__F?_Iostream_object@?$_Error_objects@H@std@@2V_Iostream_error_category@2@A@@YAXXZ 10020a10 f   moc_DiamondBuildPrompter.obj
 0001:0001fa20       ??__F?_System_object@?$_Error_objects@H@std@@2V_System_error_category@2@A@@YAXXZ 10020a20 f   moc_DiamondBuildPrompter.obj
 0001:0001fa30       ??__FalgoLog@U2@@YAXXZ     10020a30 f   moc_DiamondBuildPrompter.obj
 0001:0001fa40       ??__FcmdLog@U2@@YAXXZ      10020a40 f   moc_DiamondBuildPrompter.obj
 0001:0001fa50       ??__FcoreLog@U2@@YAXXZ     10020a50 f   moc_DiamondBuildPrompter.obj
 0001:0001fa60       ??__FioLog@U2@@YAXXZ       10020a60 f   moc_DiamondBuildPrompter.obj
 0001:0001fa70       ??__FperfLog@U2@@YAXXZ     10020a70 f   moc_DiamondBuildPrompter.obj
 0001:0001fa80       ??__FscriptLog@U2@@YAXXZ   10020a80 f   moc_DiamondBuildPrompter.obj
 0001:0001fa90       ??__FtaskLog@U2@@YAXXZ     10020a90 f   moc_DiamondBuildPrompter.obj
 0001:0001faa0       ??__FuiLog@U2@@YAXXZ       10020aa0 f   moc_DiamondBuildPrompter.obj
 0001:0001fab0       ??__FuserActLog@U2@@YAXXZ  10020ab0 f   moc_DiamondBuildPrompter.obj
 0001:0001fac0       ??__F?_Generic_object@?$_Error_objects@H@std@@2V_Generic_error_category@2@A@@YAXXZ 10020ac0 f   moc_DiamondBuildTask.obj
 0001:0001fad0       ??__F?_Iostream_object@?$_Error_objects@H@std@@2V_Iostream_error_category@2@A@@YAXXZ 10020ad0 f   moc_DiamondBuildTask.obj
 0001:0001fae0       ??__F?_System_object@?$_Error_objects@H@std@@2V_System_error_category@2@A@@YAXXZ 10020ae0 f   moc_DiamondBuildTask.obj
 0001:0001faf0       ??__FalgoLog@U2@@YAXXZ     10020af0 f   moc_DiamondBuildTask.obj
 0001:0001fb00       ??__FcmdLog@U2@@YAXXZ      10020b00 f   moc_DiamondBuildTask.obj
 0001:0001fb10       ??__FcoreLog@U2@@YAXXZ     10020b10 f   moc_DiamondBuildTask.obj
 0001:0001fb20       ??__FioLog@U2@@YAXXZ       10020b20 f   moc_DiamondBuildTask.obj
 0001:0001fb30       ??__FperfLog@U2@@YAXXZ     10020b30 f   moc_DiamondBuildTask.obj
 0001:0001fb40       ??__FscriptLog@U2@@YAXXZ   10020b40 f   moc_DiamondBuildTask.obj
 0001:0001fb50       ??__FtaskLog@U2@@YAXXZ     10020b50 f   moc_DiamondBuildTask.obj
 0001:0001fb60       ??__FuiLog@U2@@YAXXZ       10020b60 f   moc_DiamondBuildTask.obj
 0001:0001fb70       ??__FuserActLog@U2@@YAXXZ  10020b70 f   moc_DiamondBuildTask.obj
 0001:0001fb80       ??__F?_Generic_object@?$_Error_objects@H@std@@2V_Generic_error_category@2@A@@YAXXZ 10020b80 f   moc_DiamondBuildWorker.obj
 0001:0001fb90       ??__F?_Iostream_object@?$_Error_objects@H@std@@2V_Iostream_error_category@2@A@@YAXXZ 10020b90 f   moc_DiamondBuildWorker.obj
 0001:0001fba0       ??__F?_System_object@?$_Error_objects@H@std@@2V_System_error_category@2@A@@YAXXZ 10020ba0 f   moc_DiamondBuildWorker.obj
 0001:0001fbb0       ??__FalgoLog@U2@@YAXXZ     10020bb0 f   moc_DiamondBuildWorker.obj
 0001:0001fbc0       ??__FcmdLog@U2@@YAXXZ      10020bc0 f   moc_DiamondBuildWorker.obj
 0001:0001fbd0       ??__FcoreLog@U2@@YAXXZ     10020bd0 f   moc_DiamondBuildWorker.obj
 0001:0001fbe0       ??__FioLog@U2@@YAXXZ       10020be0 f   moc_DiamondBuildWorker.obj
 0001:0001fbf0       ??__FperfLog@U2@@YAXXZ     10020bf0 f   moc_DiamondBuildWorker.obj
 0001:0001fc00       ??__FscriptLog@U2@@YAXXZ   10020c00 f   moc_DiamondBuildWorker.obj
 0001:0001fc10       ??__FtaskLog@U2@@YAXXZ     10020c10 f   moc_DiamondBuildWorker.obj
 0001:0001fc20       ??__FuiLog@U2@@YAXXZ       10020c20 f   moc_DiamondBuildWorker.obj
 0001:0001fc30       ??__FuserActLog@U2@@YAXXZ  10020c30 f   moc_DiamondBuildWorker.obj
 0001:0001fc40       ??__F?_Generic_object@?$_Error_objects@H@std@@2V_Generic_error_category@2@A@@YAXXZ 10020c40 f   moc_DiamondClassifyPrompter.obj
 0001:0001fc50       ??__F?_Iostream_object@?$_Error_objects@H@std@@2V_Iostream_error_category@2@A@@YAXXZ 10020c50 f   moc_DiamondClassifyPrompter.obj
 0001:0001fc60       ??__F?_System_object@?$_Error_objects@H@std@@2V_System_error_category@2@A@@YAXXZ 10020c60 f   moc_DiamondClassifyPrompter.obj
 0001:0001fc70       ??__FalgoLog@U2@@YAXXZ     10020c70 f   moc_DiamondClassifyPrompter.obj
 0001:0001fc80       ??__FcmdLog@U2@@YAXXZ      10020c80 f   moc_DiamondClassifyPrompter.obj
 0001:0001fc90       ??__FcoreLog@U2@@YAXXZ     10020c90 f   moc_DiamondClassifyPrompter.obj
 0001:0001fca0       ??__FioLog@U2@@YAXXZ       10020ca0 f   moc_DiamondClassifyPrompter.obj
 0001:0001fcb0       ??__FperfLog@U2@@YAXXZ     10020cb0 f   moc_DiamondClassifyPrompter.obj
 0001:0001fcc0       ??__FscriptLog@U2@@YAXXZ   10020cc0 f   moc_DiamondClassifyPrompter.obj
 0001:0001fcd0       ??__FtaskLog@U2@@YAXXZ     10020cd0 f   moc_DiamondClassifyPrompter.obj
 0001:0001fce0       ??__FuiLog@U2@@YAXXZ       10020ce0 f   moc_DiamondClassifyPrompter.obj
 0001:0001fcf0       ??__FuserActLog@U2@@YAXXZ  10020cf0 f   moc_DiamondClassifyPrompter.obj
 0001:0001fd00       ??__F?_Generic_object@?$_Error_objects@H@std@@2V_Generic_error_category@2@A@@YAXXZ 10020d00 f   moc_DiamondClassifyTask.obj
 0001:0001fd10       ??__F?_Iostream_object@?$_Error_objects@H@std@@2V_Iostream_error_category@2@A@@YAXXZ 10020d10 f   moc_DiamondClassifyTask.obj
 0001:0001fd20       ??__F?_System_object@?$_Error_objects@H@std@@2V_System_error_category@2@A@@YAXXZ 10020d20 f   moc_DiamondClassifyTask.obj
 0001:0001fd30       ??__FalgoLog@U2@@YAXXZ     10020d30 f   moc_DiamondClassifyTask.obj
 0001:0001fd40       ??__FcmdLog@U2@@YAXXZ      10020d40 f   moc_DiamondClassifyTask.obj
 0001:0001fd50       ??__FcoreLog@U2@@YAXXZ     10020d50 f   moc_DiamondClassifyTask.obj
 0001:0001fd60       ??__FioLog@U2@@YAXXZ       10020d60 f   moc_DiamondClassifyTask.obj
 0001:0001fd70       ??__FperfLog@U2@@YAXXZ     10020d70 f   moc_DiamondClassifyTask.obj
 0001:0001fd80       ??__FscriptLog@U2@@YAXXZ   10020d80 f   moc_DiamondClassifyTask.obj
 0001:0001fd90       ??__FtaskLog@U2@@YAXXZ     10020d90 f   moc_DiamondClassifyTask.obj
 0001:0001fda0       ??__FuiLog@U2@@YAXXZ       10020da0 f   moc_DiamondClassifyTask.obj
 0001:0001fdb0       ??__FuserActLog@U2@@YAXXZ  10020db0 f   moc_DiamondClassifyTask.obj
 0001:0001fdc0       ??__F?_Generic_object@?$_Error_objects@H@std@@2V_Generic_error_category@2@A@@YAXXZ 10020dc0 f   moc_DiamondClassifyWorker.obj
 0001:0001fdd0       ??__F?_Iostream_object@?$_Error_objects@H@std@@2V_Iostream_error_category@2@A@@YAXXZ 10020dd0 f   moc_DiamondClassifyWorker.obj
 0001:0001fde0       ??__F?_System_object@?$_Error_objects@H@std@@2V_System_error_category@2@A@@YAXXZ 10020de0 f   moc_DiamondClassifyWorker.obj
 0001:0001fdf0       ??__FalgoLog@U2@@YAXXZ     10020df0 f   moc_DiamondClassifyWorker.obj
 0001:0001fe00       ??__FcmdLog@U2@@YAXXZ      10020e00 f   moc_DiamondClassifyWorker.obj
 0001:0001fe10       ??__FcoreLog@U2@@YAXXZ     10020e10 f   moc_DiamondClassifyWorker.obj
 0001:0001fe20       ??__FioLog@U2@@YAXXZ       10020e20 f   moc_DiamondClassifyWorker.obj
 0001:0001fe30       ??__FperfLog@U2@@YAXXZ     10020e30 f   moc_DiamondClassifyWorker.obj
 0001:0001fe40       ??__FscriptLog@U2@@YAXXZ   10020e40 f   moc_DiamondClassifyWorker.obj
 0001:0001fe50       ??__FtaskLog@U2@@YAXXZ     10020e50 f   moc_DiamondClassifyWorker.obj
 0001:0001fe60       ??__FuiLog@U2@@YAXXZ       10020e60 f   moc_DiamondClassifyWorker.obj
 0001:0001fe70       ??__FuserActLog@U2@@YAXXZ  10020e70 f   moc_DiamondClassifyWorker.obj
 0001:0001fe80       ??__F?_Generic_object@?$_Error_objects@H@std@@2V_Generic_error_category@2@A@@YAXXZ 10020e80 f   moc_DiamondSupport.obj
 0001:0001fe90       ??__F?_Iostream_object@?$_Error_objects@H@std@@2V_Iostream_error_category@2@A@@YAXXZ 10020e90 f   moc_DiamondSupport.obj
 0001:0001fea0       ??__F?_System_object@?$_Error_objects@H@std@@2V_System_error_category@2@A@@YAXXZ 10020ea0 f   moc_DiamondSupport.obj
 0001:0001feb0       ??__F?_Generic_object@?$_Error_objects@H@std@@2V_Generic_error_category@2@A@@YAXXZ 10020eb0 f   moc_DiamondSupportPlugin.obj
 0001:0001fec0       ??__F?_Iostream_object@?$_Error_objects@H@std@@2V_Iostream_error_category@2@A@@YAXXZ 10020ec0 f   moc_DiamondSupportPlugin.obj
 0001:0001fed0       ??__F?_System_object@?$_Error_objects@H@std@@2V_System_error_category@2@A@@YAXXZ 10020ed0 f   moc_DiamondSupportPlugin.obj
 0001:0001fee0       ??__F?_Generic_object@?$_Error_objects@H@std@@2V_Generic_error_category@2@A@@YAXXZ 10020ee0 f   moc_GenomesPreparationTask.obj
 0001:0001fef0       ??__F?_Iostream_object@?$_Error_objects@H@std@@2V_Iostream_error_category@2@A@@YAXXZ 10020ef0 f   moc_GenomesPreparationTask.obj
 0001:0001ff00       ??__F?_System_object@?$_Error_objects@H@std@@2V_System_error_category@2@A@@YAXXZ 10020f00 f   moc_GenomesPreparationTask.obj
 0001:0001ff10       ??__FalgoLog@U2@@YAXXZ     10020f10 f   moc_GenomesPreparationTask.obj
 0001:0001ff20       ??__FcmdLog@U2@@YAXXZ      10020f20 f   moc_GenomesPreparationTask.obj
 0001:0001ff30       ??__FcoreLog@U2@@YAXXZ     10020f30 f   moc_GenomesPreparationTask.obj
 0001:0001ff40       ??__FioLog@U2@@YAXXZ       10020f40 f   moc_GenomesPreparationTask.obj
 0001:0001ff50       ??__FperfLog@U2@@YAXXZ     10020f50 f   moc_GenomesPreparationTask.obj
 0001:0001ff60       ??__FscriptLog@U2@@YAXXZ   10020f60 f   moc_GenomesPreparationTask.obj
 0001:0001ff70       ??__FtaskLog@U2@@YAXXZ     10020f70 f   moc_GenomesPreparationTask.obj
 0001:0001ff80       ??__FuiLog@U2@@YAXXZ       10020f80 f   moc_GenomesPreparationTask.obj
 0001:0001ff90       ??__FuserActLog@U2@@YAXXZ  10020f90 f   moc_GenomesPreparationTask.obj
 0002:00000838       _algoLog$initializer$      10021838     DiamondBuildPrompter.obj
 0002:0000083c       _cmdLog$initializer$       1002183c     DiamondBuildPrompter.obj
 0002:00000840       _coreLog$initializer$      10021840     DiamondBuildPrompter.obj
 0002:00000844       _ioLog$initializer$        10021844     DiamondBuildPrompter.obj
 0002:00000848       _perfLog$initializer$      10021848     DiamondBuildPrompter.obj
 0002:0000084c       _scriptLog$initializer$    1002184c     DiamondBuildPrompter.obj
 0002:00000850       _taskLog$initializer$      10021850     DiamondBuildPrompter.obj
 0002:00000854       _uiLog$initializer$        10021854     DiamondBuildPrompter.obj
 0002:00000858       _userActLog$initializer$   10021858     DiamondBuildPrompter.obj
 0002:0000085c       ?_Generic_object$initializer$@?$_Error_objects@H@std@@2P6AXXZA 1002185c     DiamondBuildPrompter.obj
 0002:00000860       ?_Iostream_object$initializer$@?$_Error_objects@H@std@@2P6AXXZA 10021860     DiamondBuildPrompter.obj
 0002:00000864       ?_System_object$initializer$@?$_Error_objects@H@std@@2P6AXXZA 10021864     DiamondBuildPrompter.obj
 0002:00000868       _algoLog$initializer$      10021868     DiamondBuildTask.obj
 0002:0000086c       _cmdLog$initializer$       1002186c     DiamondBuildTask.obj
 0002:00000870       _coreLog$initializer$      10021870     DiamondBuildTask.obj
 0002:00000874       _ioLog$initializer$        10021874     DiamondBuildTask.obj
 0002:00000878       _perfLog$initializer$      10021878     DiamondBuildTask.obj
 0002:0000087c       _scriptLog$initializer$    1002187c     DiamondBuildTask.obj
 0002:00000880       _taskLog$initializer$      10021880     DiamondBuildTask.obj
 0002:00000884       _uiLog$initializer$        10021884     DiamondBuildTask.obj
 0002:00000888       _userActLog$initializer$   10021888     DiamondBuildTask.obj
 0002:0000088c       _algoLog$initializer$      1002188c     DiamondBuildValidator.obj
 0002:00000890       _cmdLog$initializer$       10021890     DiamondBuildValidator.obj
 0002:00000894       _coreLog$initializer$      10021894     DiamondBuildValidator.obj
 0002:00000898       _ioLog$initializer$        10021898     DiamondBuildValidator.obj
 0002:0000089c       _perfLog$initializer$      1002189c     DiamondBuildValidator.obj
 0002:000008a0       _scriptLog$initializer$    100218a0     DiamondBuildValidator.obj
 0002:000008a4       _taskLog$initializer$      100218a4     DiamondBuildValidator.obj
 0002:000008a8       _uiLog$initializer$        100218a8     DiamondBuildValidator.obj
 0002:000008ac       _userActLog$initializer$   100218ac     DiamondBuildValidator.obj
 0002:000008b0       _algoLog$initializer$      100218b0     DiamondBuildWorker.obj
 0002:000008b4       _cmdLog$initializer$       100218b4     DiamondBuildWorker.obj
 0002:000008b8       _coreLog$initializer$      100218b8     DiamondBuildWorker.obj
 0002:000008bc       _ioLog$initializer$        100218bc     DiamondBuildWorker.obj
 0002:000008c0       _perfLog$initializer$      100218c0     DiamondBuildWorker.obj
 0002:000008c4       _scriptLog$initializer$    100218c4     DiamondBuildWorker.obj
 0002:000008c8       _taskLog$initializer$      100218c8     DiamondBuildWorker.obj
 0002:000008cc       _uiLog$initializer$        100218cc     DiamondBuildWorker.obj
 0002:000008d0       _userActLog$initializer$   100218d0     DiamondBuildWorker.obj
 0002:000008d4       ?DIAMOND_BUILD_DIR$initializer$@DiamondBuildWorker@LocalWorkflow@U2@@0P6AXXZA 100218d4     DiamondBuildWorker.obj
 0002:000008d8       _algoLog$initializer$      100218d8     DiamondBuildWorkerFactory.obj
 0002:000008dc       _cmdLog$initializer$       100218dc     DiamondBuildWorkerFactory.obj
 0002:000008e0       _coreLog$initializer$      100218e0     DiamondBuildWorkerFactory.obj
 0002:000008e4       _ioLog$initializer$        100218e4     DiamondBuildWorkerFactory.obj
 0002:000008e8       _perfLog$initializer$      100218e8     DiamondBuildWorkerFactory.obj
 0002:000008ec       _scriptLog$initializer$    100218ec     DiamondBuildWorkerFactory.obj
 0002:000008f0       _taskLog$initializer$      100218f0     DiamondBuildWorkerFactory.obj
 0002:000008f4       _uiLog$initializer$        100218f4     DiamondBuildWorkerFactory.obj
 0002:000008f8       _userActLog$initializer$   100218f8     DiamondBuildWorkerFactory.obj
 0002:000008fc       ?ACTOR_ID$initializer$@DiamondBuildWorkerFactory@LocalWorkflow@U2@@2P6AXXZA 100218fc     DiamondBuildWorkerFactory.obj
 0002:00000900       ?OUTPUT_PORT_ID$initializer$@DiamondBuildWorkerFactory@LocalWorkflow@U2@@2P6AXXZA 10021900     DiamondBuildWorkerFactory.obj
 0002:00000904       ?DATABASE_ATTR_ID$initializer$@DiamondBuildWorkerFactory@LocalWorkflow@U2@@2P6AXXZA 10021904     DiamondBuildWorkerFactory.obj
 0002:00000908       ?GENOMIC_LIBRARY_ATTR_ID$initializer$@DiamondBuildWorkerFactory@LocalWorkflow@U2@@2P6AXXZA 10021908     DiamondBuildWorkerFactory.obj
 0002:0000090c       _algoLog$initializer$      1002190c     DiamondClassifyPrompter.obj
 0002:00000910       _cmdLog$initializer$       10021910     DiamondClassifyPrompter.obj
 0002:00000914       _coreLog$initializer$      10021914     DiamondClassifyPrompter.obj
 0002:00000918       _ioLog$initializer$        10021918     DiamondClassifyPrompter.obj
 0002:0000091c       _perfLog$initializer$      1002191c     DiamondClassifyPrompter.obj
 0002:00000920       _scriptLog$initializer$    10021920     DiamondClassifyPrompter.obj
 0002:00000924       _taskLog$initializer$      10021924     DiamondClassifyPrompter.obj
 0002:00000928       _uiLog$initializer$        10021928     DiamondClassifyPrompter.obj
 0002:0000092c       _userActLog$initializer$   1002192c     DiamondClassifyPrompter.obj
 0002:00000930       _algoLog$initializer$      10021930     DiamondClassifyTask.obj
 0002:00000934       _cmdLog$initializer$       10021934     DiamondClassifyTask.obj
 0002:00000938       _coreLog$initializer$      10021938     DiamondClassifyTask.obj
 0002:0000093c       _ioLog$initializer$        1002193c     DiamondClassifyTask.obj
 0002:00000940       _perfLog$initializer$      10021940     DiamondClassifyTask.obj
 0002:00000944       _scriptLog$initializer$    10021944     DiamondClassifyTask.obj
 0002:00000948       _taskLog$initializer$      10021948     DiamondClassifyTask.obj
 0002:0000094c       _uiLog$initializer$        1002194c     DiamondClassifyTask.obj
 0002:00000950       _userActLog$initializer$   10021950     DiamondClassifyTask.obj
 0002:00000954       ?SENSITIVE_DEFAULT$initializer$@DiamondClassifyTaskSettings@U2@@2P6AXXZA 10021954     DiamondClassifyTask.obj
 0002:00000958       ?SENSITIVE_ULTRA$initializer$@DiamondClassifyTaskSettings@U2@@2P6AXXZA 10021958     DiamondClassifyTask.obj
 0002:0000095c       ?SENSITIVE_HIGH$initializer$@DiamondClassifyTaskSettings@U2@@2P6AXXZA 1002195c     DiamondClassifyTask.obj
 0002:00000960       ?BLOSUM45$initializer$@DiamondClassifyTaskSettings@U2@@2P6AXXZA 10021960     DiamondClassifyTask.obj
 0002:00000964       ?BLOSUM50$initializer$@DiamondClassifyTaskSettings@U2@@2P6AXXZA 10021964     DiamondClassifyTask.obj
 0002:00000968       ?BLOSUM62$initializer$@DiamondClassifyTaskSettings@U2@@2P6AXXZA 10021968     DiamondClassifyTask.obj
 0002:0000096c       ?BLOSUM80$initializer$@DiamondClassifyTaskSettings@U2@@2P6AXXZA 1002196c     DiamondClassifyTask.obj
 0002:00000970       ?BLOSUM90$initializer$@DiamondClassifyTaskSettings@U2@@2P6AXXZA 10021970     DiamondClassifyTask.obj
 0002:00000974       ?PAM250$initializer$@DiamondClassifyTaskSettings@U2@@2P6AXXZA 10021974     DiamondClassifyTask.obj
 0002:00000978       ?PAM70$initializer$@DiamondClassifyTaskSettings@U2@@2P6AXXZA 10021978     DiamondClassifyTask.obj
 0002:0000097c       ?PAM30$initializer$@DiamondClassifyTaskSettings@U2@@2P6AXXZA 1002197c     DiamondClassifyTask.obj
 0002:00000980       ?TAXONOMIC_CLASSIFICATION_OUTPUT_FORMAT$initializer$@DiamondClassifyTask@U2@@0P6AXXZA 10021980     DiamondClassifyTask.obj
 0002:00000984       _algoLog$initializer$      10021984     DiamondClassifyWorker.obj
 0002:00000988       _cmdLog$initializer$       10021988     DiamondClassifyWorker.obj
 0002:0000098c       _coreLog$initializer$      1002198c     DiamondClassifyWorker.obj
 0002:00000990       _ioLog$initializer$        10021990     DiamondClassifyWorker.obj
 0002:00000994       _perfLog$initializer$      10021994     DiamondClassifyWorker.obj
 0002:00000998       _scriptLog$initializer$    10021998     DiamondClassifyWorker.obj
 0002:0000099c       _taskLog$initializer$      1002199c     DiamondClassifyWorker.obj
 0002:000009a0       _uiLog$initializer$        100219a0     DiamondClassifyWorker.obj
 0002:000009a4       _userActLog$initializer$   100219a4     DiamondClassifyWorker.obj
 0002:000009a8       ?DIAMOND_DIR$initializer$@DiamondClassifyWorker@LocalWorkflow@U2@@0P6AXXZA 100219a8     DiamondClassifyWorker.obj
 0002:000009ac       _algoLog$initializer$      100219ac     DiamondClassifyWorkerFactory.obj
 0002:000009b0       _cmdLog$initializer$       100219b0     DiamondClassifyWorkerFactory.obj
 0002:000009b4       _coreLog$initializer$      100219b4     DiamondClassifyWorkerFactory.obj
 0002:000009b8       _ioLog$initializer$        100219b8     DiamondClassifyWorkerFactory.obj
 0002:000009bc       _perfLog$initializer$      100219bc     DiamondClassifyWorkerFactory.obj
 0002:000009c0       _scriptLog$initializer$    100219c0     DiamondClassifyWorkerFactory.obj
 0002:000009c4       _taskLog$initializer$      100219c4     DiamondClassifyWorkerFactory.obj
 0002:000009c8       _uiLog$initializer$        100219c8     DiamondClassifyWorkerFactory.obj
 0002:000009cc       _userActLog$initializer$   100219cc     DiamondClassifyWorkerFactory.obj
 0002:000009d0       ?ACTOR_ID$initializer$@DiamondClassifyWorkerFactory@LocalWorkflow@U2@@2P6AXXZA 100219d0     DiamondClassifyWorkerFactory.obj
 0002:000009d4       ?INPUT_PORT_ID$initializer$@DiamondClassifyWorkerFactory@LocalWorkflow@U2@@2P6AXXZA 100219d4     DiamondClassifyWorkerFactory.obj
 0002:000009d8       ?OUTPUT_PORT_ID$initializer$@DiamondClassifyWorkerFactory@LocalWorkflow@U2@@2P6AXXZA 100219d8     DiamondClassifyWorkerFactory.obj
 0002:000009dc       ?INPUT_SLOT$initializer$@DiamondClassifyWorkerFactory@LocalWorkflow@U2@@2P6AXXZA 100219dc     DiamondClassifyWorkerFactory.obj
 0002:000009e0       ?INPUT_DATA_ATTR_ID$initializer$@DiamondClassifyWorkerFactory@LocalWorkflow@U2@@2P6AXXZA 100219e0     DiamondClassifyWorkerFactory.obj
 0002:000009e4       ?DATABASE_ATTR_ID$initializer$@DiamondClassifyWorkerFactory@LocalWorkflow@U2@@2P6AXXZA 100219e4     DiamondClassifyWorkerFactory.obj
 0002:000009e8       ?GENCODE_ATTR_ID$initializer$@DiamondClassifyWorkerFactory@LocalWorkflow@U2@@2P6AXXZA 100219e8     DiamondClassifyWorkerFactory.obj
 0002:000009ec       ?SENSITIVE_ATTR_ID$initializer$@DiamondClassifyWorkerFactory@LocalWorkflow@U2@@2P6AXXZA 100219ec     DiamondClassifyWorkerFactory.obj
 0002:000009f0       ?TOP_ALIGNMENTS_PERCENTAGE_ATTR_ID$initializer$@DiamondClassifyWorkerFactory@LocalWorkflow@U2@@2P6AXXZA 100219f0     DiamondClassifyWorkerFactory.obj
 0002:000009f4       ?FSHIFT_ATTR_ID$initializer$@DiamondClassifyWorkerFactory@LocalWorkflow@U2@@2P6AXXZA 100219f4     DiamondClassifyWorkerFactory.obj
 0002:000009f8       ?EVALUE_ATTR_ID$initializer$@DiamondClassifyWorkerFactory@LocalWorkflow@U2@@2P6AXXZA 100219f8     DiamondClassifyWorkerFactory.obj
 0002:000009fc       ?MATRIX_ATTR_ID$initializer$@DiamondClassifyWorkerFactory@LocalWorkflow@U2@@2P6AXXZA 100219fc     DiamondClassifyWorkerFactory.obj
 0002:00000a00       ?GO_PEN_ATTR_ID$initializer$@DiamondClassifyWorkerFactory@LocalWorkflow@U2@@2P6AXXZA 10021a00     DiamondClassifyWorkerFactory.obj
 0002:00000a04       ?GE_PEN_ATTR_ID$initializer$@DiamondClassifyWorkerFactory@LocalWorkflow@U2@@2P6AXXZA 10021a04     DiamondClassifyWorkerFactory.obj
 0002:00000a08       ?THREADS_ATTR_ID$initializer$@DiamondClassifyWorkerFactory@LocalWorkflow@U2@@2P6AXXZA 10021a08     DiamondClassifyWorkerFactory.obj
 0002:00000a0c       ?BSIZE_ATTR_ID$initializer$@DiamondClassifyWorkerFactory@LocalWorkflow@U2@@2P6AXXZA 10021a0c     DiamondClassifyWorkerFactory.obj
 0002:00000a10       ?CHUNKS_ATTR_ID$initializer$@DiamondClassifyWorkerFactory@LocalWorkflow@U2@@2P6AXXZA 10021a10     DiamondClassifyWorkerFactory.obj
 0002:00000a14       ?OUTPUT_URL_ATTR_ID$initializer$@DiamondClassifyWorkerFactory@LocalWorkflow@U2@@2P6AXXZA 10021a14     DiamondClassifyWorkerFactory.obj
 0002:00000a18       ?WORKFLOW_CLASSIFY_TOOL_DIAMOND$initializer$@DiamondClassifyWorkerFactory@LocalWorkflow@U2@@2P6AXXZA 10021a18     DiamondClassifyWorkerFactory.obj
 0002:00000a1c       ?TOOL_NAME$initializer$@DiamondSupport@U2@@2P6AXXZA 10021a1c     DiamondSupport.obj
 0002:00000a20       _algoLog$initializer$      10021a20     DiamondSupportPlugin.obj
 0002:00000a24       _cmdLog$initializer$       10021a24     DiamondSupportPlugin.obj
 0002:00000a28       _coreLog$initializer$      10021a28     DiamondSupportPlugin.obj
 0002:00000a2c       _ioLog$initializer$        10021a2c     DiamondSupportPlugin.obj
 0002:00000a30       _perfLog$initializer$      10021a30     DiamondSupportPlugin.obj
 0002:00000a34       _scriptLog$initializer$    10021a34     DiamondSupportPlugin.obj
 0002:00000a38       _taskLog$initializer$      10021a38     DiamondSupportPlugin.obj
 0002:00000a3c       _uiLog$initializer$        10021a3c     DiamondSupportPlugin.obj
 0002:00000a40       _userActLog$initializer$   10021a40     DiamondSupportPlugin.obj
 0002:00000a44       ?PLUGIN_NAME$initializer$@DiamondSupportPlugin@U2@@2P6AXXZA 10021a44     DiamondSupportPlugin.obj
 0002:00000a48       ?PLUGIN_DESCRIPRION$initializer$@DiamondSupportPlugin@U2@@2P6AXXZA 10021a48     DiamondSupportPlugin.obj
 0002:00000a4c       _algoLog$initializer$      10021a4c     GenomesPreparationTask.obj
 0002:00000a50       _cmdLog$initializer$       10021a50     GenomesPreparationTask.obj
 0002:00000a54       _coreLog$initializer$      10021a54     GenomesPreparationTask.obj
 0002:00000a58       _ioLog$initializer$        10021a58     GenomesPreparationTask.obj
 0002:00000a5c       _perfLog$initializer$      10021a5c     GenomesPreparationTask.obj
 0002:00000a60       _scriptLog$initializer$    10021a60     GenomesPreparationTask.obj
 0002:00000a64       _taskLog$initializer$      10021a64     GenomesPreparationTask.obj
 0002:00000a68       _uiLog$initializer$        10021a68     GenomesPreparationTask.obj
 0002:00000a6c       _userActLog$initializer$   10021a6c     GenomesPreparationTask.obj
 0002:00000a70       _algoLog$initializer$      10021a70     moc_DiamondBuildPrompter.obj
 0002:00000a74       _cmdLog$initializer$       10021a74     moc_DiamondBuildPrompter.obj
 0002:00000a78       _coreLog$initializer$      10021a78     moc_DiamondBuildPrompter.obj
 0002:00000a7c       _ioLog$initializer$        10021a7c     moc_DiamondBuildPrompter.obj
 0002:00000a80       _perfLog$initializer$      10021a80     moc_DiamondBuildPrompter.obj
 0002:00000a84       _scriptLog$initializer$    10021a84     moc_DiamondBuildPrompter.obj
 0002:00000a88       _taskLog$initializer$      10021a88     moc_DiamondBuildPrompter.obj
 0002:00000a8c       _uiLog$initializer$        10021a8c     moc_DiamondBuildPrompter.obj
 0002:00000a90       _userActLog$initializer$   10021a90     moc_DiamondBuildPrompter.obj
 0002:00000a94       ?staticMetaObject$initializer$@DiamondBuildPrompter@LocalWorkflow@U2@@2P6AXXZA 10021a94     moc_DiamondBuildPrompter.obj
 0002:00000a98       _algoLog$initializer$      10021a98     moc_DiamondBuildTask.obj
 0002:00000a9c       _cmdLog$initializer$       10021a9c     moc_DiamondBuildTask.obj
 0002:00000aa0       _coreLog$initializer$      10021aa0     moc_DiamondBuildTask.obj
 0002:00000aa4       _ioLog$initializer$        10021aa4     moc_DiamondBuildTask.obj
 0002:00000aa8       _perfLog$initializer$      10021aa8     moc_DiamondBuildTask.obj
 0002:00000aac       _scriptLog$initializer$    10021aac     moc_DiamondBuildTask.obj
 0002:00000ab0       _taskLog$initializer$      10021ab0     moc_DiamondBuildTask.obj
 0002:00000ab4       _uiLog$initializer$        10021ab4     moc_DiamondBuildTask.obj
 0002:00000ab8       _userActLog$initializer$   10021ab8     moc_DiamondBuildTask.obj
 0002:00000abc       ?staticMetaObject$initializer$@DiamondBuildTask@U2@@2P6AXXZA 10021abc     moc_DiamondBuildTask.obj
 0002:00000ac0       _algoLog$initializer$      10021ac0     moc_DiamondBuildWorker.obj
 0002:00000ac4       _cmdLog$initializer$       10021ac4     moc_DiamondBuildWorker.obj
 0002:00000ac8       _coreLog$initializer$      10021ac8     moc_DiamondBuildWorker.obj
 0002:00000acc       _ioLog$initializer$        10021acc     moc_DiamondBuildWorker.obj
 0002:00000ad0       _perfLog$initializer$      10021ad0     moc_DiamondBuildWorker.obj
 0002:00000ad4       _scriptLog$initializer$    10021ad4     moc_DiamondBuildWorker.obj
 0002:00000ad8       _taskLog$initializer$      10021ad8     moc_DiamondBuildWorker.obj
 0002:00000adc       _uiLog$initializer$        10021adc     moc_DiamondBuildWorker.obj
 0002:00000ae0       _userActLog$initializer$   10021ae0     moc_DiamondBuildWorker.obj
 0002:00000ae4       ?staticMetaObject$initializer$@DiamondBuildWorker@LocalWorkflow@U2@@2P6AXXZA 10021ae4     moc_DiamondBuildWorker.obj
 0002:00000ae8       _algoLog$initializer$      10021ae8     moc_DiamondClassifyPrompter.obj
 0002:00000aec       _cmdLog$initializer$       10021aec     moc_DiamondClassifyPrompter.obj
 0002:00000af0       _coreLog$initializer$      10021af0     moc_DiamondClassifyPrompter.obj
 0002:00000af4       _ioLog$initializer$        10021af4     moc_DiamondClassifyPrompter.obj
 0002:00000af8       _perfLog$initializer$      10021af8     moc_DiamondClassifyPrompter.obj
 0002:00000afc       _scriptLog$initializer$    10021afc     moc_DiamondClassifyPrompter.obj
 0002:00000b00       _taskLog$initializer$      10021b00     moc_DiamondClassifyPrompter.obj
 0002:00000b04       _uiLog$initializer$        10021b04     moc_DiamondClassifyPrompter.obj
 0002:00000b08       _userActLog$initializer$   10021b08     moc_DiamondClassifyPrompter.obj
 0002:00000b0c       ?staticMetaObject$initializer$@DiamondClassifyPrompter@LocalWorkflow@U2@@2P6AXXZA 10021b0c     moc_DiamondClassifyPrompter.obj
 0002:00000b10       _algoLog$initializer$      10021b10     moc_DiamondClassifyTask.obj
 0002:00000b14       _cmdLog$initializer$       10021b14     moc_DiamondClassifyTask.obj
 0002:00000b18       _coreLog$initializer$      10021b18     moc_DiamondClassifyTask.obj
 0002:00000b1c       _ioLog$initializer$        10021b1c     moc_DiamondClassifyTask.obj
 0002:00000b20       _perfLog$initializer$      10021b20     moc_DiamondClassifyTask.obj
 0002:00000b24       _scriptLog$initializer$    10021b24     moc_DiamondClassifyTask.obj
 0002:00000b28       _taskLog$initializer$      10021b28     moc_DiamondClassifyTask.obj
 0002:00000b2c       _uiLog$initializer$        10021b2c     moc_DiamondClassifyTask.obj
 0002:00000b30       _userActLog$initializer$   10021b30     moc_DiamondClassifyTask.obj
 0002:00000b34       ?staticMetaObject$initializer$@DiamondClassifyTask@U2@@2P6AXXZA 10021b34     moc_DiamondClassifyTask.obj
 0002:00000b38       _algoLog$initializer$      10021b38     moc_DiamondClassifyWorker.obj
 0002:00000b3c       _cmdLog$initializer$       10021b3c     moc_DiamondClassifyWorker.obj
 0002:00000b40       _coreLog$initializer$      10021b40     moc_DiamondClassifyWorker.obj
 0002:00000b44       _ioLog$initializer$        10021b44     moc_DiamondClassifyWorker.obj
 0002:00000b48       _perfLog$initializer$      10021b48     moc_DiamondClassifyWorker.obj
 0002:00000b4c       _scriptLog$initializer$    10021b4c     moc_DiamondClassifyWorker.obj
 0002:00000b50       _taskLog$initializer$      10021b50     moc_DiamondClassifyWorker.obj
 0002:00000b54       _uiLog$initializer$        10021b54     moc_DiamondClassifyWorker.obj
 0002:00000b58       _userActLog$initializer$   10021b58     moc_DiamondClassifyWorker.obj
 0002:00000b5c       ?staticMetaObject$initializer$@DiamondClassifyWorker@LocalWorkflow@U2@@2P6AXXZA 10021b5c     moc_DiamondClassifyWorker.obj
 0002:00000b60       ?staticMetaObject$initializer$@DiamondSupport@U2@@2P6AXXZA 10021b60     moc_DiamondSupport.obj
 0002:00000b64       ?staticMetaObject$initializer$@DiamondSupportPlugin@U2@@2P6AXXZA 10021b64     moc_DiamondSupportPlugin.obj
 0002:00000b68       _algoLog$initializer$      10021b68     moc_GenomesPreparationTask.obj
 0002:00000b6c       _cmdLog$initializer$       10021b6c     moc_GenomesPreparationTask.obj
 0002:00000b70       _coreLog$initializer$      10021b70     moc_GenomesPreparationTask.obj
 0002:00000b74       _ioLog$initializer$        10021b74     moc_GenomesPreparationTask.obj
 0002:00000b78       _perfLog$initializer$      10021b78     moc_GenomesPreparationTask.obj
 0002:00000b7c       _scriptLog$initializer$    10021b7c     moc_GenomesPreparationTask.obj
 0002:00000b80       _taskLog$initializer$      10021b80     moc_GenomesPreparationTask.obj
 0002:00000b84       _uiLog$initializer$        10021b84     moc_GenomesPreparationTask.obj
 0002:00000b88       _userActLog$initializer$   10021b88     moc_GenomesPreparationTask.obj
 0002:00000b8c       ?staticMetaObject$initializer$@GenomesPreparationTask@U2@@2P6AXXZA 10021b8c     moc_GenomesPreparationTask.obj
 0002:00000b98       _pcinit                    10021b98     MSVCRT:crtdll.obj
 0002:00000b9c       _pinit                     10021b9c     MSVCRT:atonexit.obj
 0002:00003080       _qt_meta_stringdata_U2__LocalWorkflow__DiamondBuildPrompter 10024080     moc_DiamondBuildPrompter.obj
 0002:000030b8       _qt_meta_data_U2__LocalWorkflow__DiamondBuildPrompter 100240b8     moc_DiamondBuildPrompter.obj
 0002:000030f4       _qt_meta_stringdata_U2__DiamondBuildTask 100240f4     moc_DiamondBuildTask.obj
 0002:0000311c       _qt_meta_data_U2__DiamondBuildTask 1002411c     moc_DiamondBuildTask.obj
 0002:00003158       _qt_meta_stringdata_U2__LocalWorkflow__DiamondBuildWorker 10024158     moc_DiamondBuildWorker.obj
 0002:000031f0       _qt_meta_data_U2__LocalWorkflow__DiamondBuildWorker 100241f0     moc_DiamondBuildWorker.obj
 0002:0000324c       _qt_meta_stringdata_U2__LocalWorkflow__DiamondClassifyPrompter 1002424c     moc_DiamondClassifyPrompter.obj
 0002:00003288       _qt_meta_data_U2__LocalWorkflow__DiamondClassifyPrompter 10024288     moc_DiamondClassifyPrompter.obj
 0002:000032c4       _qt_meta_stringdata_U2__DiamondClassifyTask 100242c4     moc_DiamondClassifyTask.obj
 0002:000032ec       _qt_meta_data_U2__DiamondClassifyTask 100242ec     moc_DiamondClassifyTask.obj
 0002:00003328       _qt_meta_stringdata_U2__LocalWorkflow__DiamondClassifyWorker 10024328     moc_DiamondClassifyWorker.obj
 0002:000033c0       _qt_meta_data_U2__LocalWorkflow__DiamondClassifyWorker 100243c0     moc_DiamondClassifyWorker.obj
 0002:0000341c       _qt_meta_stringdata_U2__DiamondSupport 1002441c     moc_DiamondSupport.obj
 0002:00003440       _qt_meta_data_U2__DiamondSupport 10024440     moc_DiamondSupport.obj
 0002:0000347c       _qt_meta_stringdata_U2__DiamondSupportPlugin 1002447c     moc_DiamondSupportPlugin.obj
 0002:000034a8       _qt_meta_data_U2__DiamondSupportPlugin 100244a8     moc_DiamondSupportPlugin.obj
 0002:000034e4       _qt_meta_stringdata_U2__GenomesPreparationTask 100244e4     moc_GenomesPreparationTask.obj
 0002:00003510       _qt_meta_data_U2__GenomesPreparationTask 10024510     moc_GenomesPreparationTask.obj
 0002:0000355c       _GS_ExceptionPointers      1002455c     MSVCRT:gs_report.obj
 0002:00004cc8       __catchsym$?_Copy@?$basic_string@DU?$char_traits@D@std@@V?$allocator@D@2@@std@@QAEXII@Z$5 10025cc8     DiamondBuildPrompter.obj
 0002:00004cd8       __catchsym$?_Copy@?$basic_string@DU?$char_traits@D@std@@V?$allocator@D@2@@std@@QAEXII@Z$4 10025cd8     DiamondBuildPrompter.obj
 0002:00004ce8       __unwindtable$?_Copy@?$basic_string@DU?$char_traits@D@std@@V?$allocator@D@2@@std@@QAEXII@Z 10025ce8     DiamondBuildPrompter.obj
 0002:00004d08       __ehfuncinfo$?_Copy@?$basic_string@DU?$char_traits@D@std@@V?$allocator@D@2@@std@@QAEXII@Z 10025d08     DiamondBuildPrompter.obj
 0002:00004d2c       __tryblocktable$?_Copy@?$basic_string@DU?$char_traits@D@std@@V?$allocator@D@2@@std@@QAEXII@Z 10025d2c     DiamondBuildPrompter.obj
 0002:00004d54       __unwindtable$??__EalgoLog@U2@@YAXXZ 10025d54     DiamondBuildPrompter.obj
 0002:00004d5c       __ehfuncinfo$??__EalgoLog@U2@@YAXXZ 10025d5c     DiamondBuildPrompter.obj
 0002:00004d80       __unwindtable$??__EcmdLog@U2@@YAXXZ 10025d80     DiamondBuildPrompter.obj
 0002:00004d88       __ehfuncinfo$??__EcmdLog@U2@@YAXXZ 10025d88     DiamondBuildPrompter.obj
 0002:00004dac       __unwindtable$??__EcoreLog@U2@@YAXXZ 10025dac     DiamondBuildPrompter.obj
 0002:00004db4       __ehfuncinfo$??__EcoreLog@U2@@YAXXZ 10025db4     DiamondBuildPrompter.obj
 0002:00004dd8       __unwindtable$??__EioLog@U2@@YAXXZ 10025dd8     DiamondBuildPrompter.obj
 0002:00004de0       __ehfuncinfo$??__EioLog@U2@@YAXXZ 10025de0     DiamondBuildPrompter.obj
 0002:00004e04       __unwindtable$??__EperfLog@U2@@YAXXZ 10025e04     DiamondBuildPrompter.obj
 0002:00004e0c       __ehfuncinfo$??__EperfLog@U2@@YAXXZ 10025e0c     DiamondBuildPrompter.obj
 0002:00004e30       __unwindtable$??__EscriptLog@U2@@YAXXZ 10025e30     DiamondBuildPrompter.obj
 0002:00004e38       __ehfuncinfo$??__EscriptLog@U2@@YAXXZ 10025e38     DiamondBuildPrompter.obj
 0002:00004e5c       __unwindtable$??__EtaskLog@U2@@YAXXZ 10025e5c     DiamondBuildPrompter.obj
 0002:00004e64       __ehfuncinfo$??__EtaskLog@U2@@YAXXZ 10025e64     DiamondBuildPrompter.obj
 0002:00004e88       __unwindtable$??__EuiLog@U2@@YAXXZ 10025e88     DiamondBuildPrompter.obj
 0002:00004e90       __ehfuncinfo$??__EuiLog@U2@@YAXXZ 10025e90     DiamondBuildPrompter.obj
 0002:00004eb4       __unwindtable$??__EuserActLog@U2@@YAXXZ 10025eb4     DiamondBuildPrompter.obj
 0002:00004ebc       __ehfuncinfo$??__EuserActLog@U2@@YAXXZ 10025ebc     DiamondBuildPrompter.obj
 0002:00004ee0       __ehfuncinfo$?createDescription@?$PrompterBase@VDiamondBuildPrompter@LocalWorkflow@U2@@@U2@@UAEPAVActorDocument@Workflow@2@PAVActor@42@@Z 10025ee0     DiamondBuildPrompter.obj
 0002:00004f04       __unwindtable$?createDescription@?$PrompterBase@VDiamondBuildPrompter@LocalWorkflow@U2@@@U2@@UAEPAVActorDocument@Workflow@2@PAVActor@42@@Z 10025f04     DiamondBuildPrompter.obj
 0002:00004f3c       __ehfuncinfo$?composeRichDoc@DiamondBuildPrompter@LocalWorkflow@U2@@EAE?AVQString@@XZ 10025f3c     DiamondBuildPrompter.obj
 0002:00004f60       __unwindtable$?composeRichDoc@DiamondBuildPrompter@LocalWorkflow@U2@@EAE?AVQString@@XZ 10025f60     DiamondBuildPrompter.obj
 0002:00004fa8       __catchsym$??0?$QList@PAVPort@Workflow@U2@@@@QAE@ABV0@@Z$2 10025fa8     DiamondBuildPrompter.obj
 0002:00004fb8       __unwindtable$??0?$QList@PAVPort@Workflow@U2@@@@QAE@ABV0@@Z 10025fb8     DiamondBuildPrompter.obj
 0002:00004fc8       __tryblocktable$??0?$QList@PAVPort@Workflow@U2@@@@QAE@ABV0@@Z 10025fc8     DiamondBuildPrompter.obj
 0002:00004fdc       __ehfuncinfo$??0?$QList@PAVPort@Workflow@U2@@@@QAE@ABV0@@Z 10025fdc     DiamondBuildPrompter.obj
 0002:00005000       __unwindtable$??H@YA?BVQString@@ABV0@PBD@Z 10026000     DiamondBuildTask.obj
 0002:00005010       __ehfuncinfo$??H@YA?BVQString@@ABV0@PBD@Z 10026010     DiamondBuildTask.obj
 0002:00005034       __catchsym$??0?$QList@VQString@@@@QAE@ABV0@@Z$2 10026034     DiamondBuildTask.obj
 0002:00005044       __unwindtable$??0?$QList@VQString@@@@QAE@ABV0@@Z 10026044     DiamondBuildTask.obj
 0002:00005054       __tryblocktable$??0?$QList@VQString@@@@QAE@ABV0@@Z 10026054     DiamondBuildTask.obj
 0002:00005068       __ehfuncinfo$??0?$QList@VQString@@@@QAE@ABV0@@Z 10026068     DiamondBuildTask.obj
 0002:0000508c       __catchsym$?append@?$QList@VQString@@@@QAEXABVQString@@@Z$13 1002608c     DiamondBuildTask.obj
 0002:0000509c       __catchsym$?append@?$QList@VQString@@@@QAEXABVQString@@@Z$12 1002609c     DiamondBuildTask.obj
 0002:000050ac       __ehfuncinfo$?append@?$QList@VQString@@@@QAEXABVQString@@@Z 100260ac     DiamondBuildTask.obj
 0002:000050d0       __tryblocktable$?append@?$QList@VQString@@@@QAEXABVQString@@@Z 100260d0     DiamondBuildTask.obj
 0002:000050f8       __unwindtable$?append@?$QList@VQString@@@@QAEXABVQString@@@Z 100260f8     DiamondBuildTask.obj
 0002:00005158       __catchsym$?detach_helper_grow@?$QList@VQString@@@@AAEPAUNode@1@HH@Z$5 10026158     DiamondBuildTask.obj
 0002:00005168       __catchsym$?detach_helper_grow@?$QList@VQString@@@@AAEPAUNode@1@HH@Z$4 10026168     DiamondBuildTask.obj
 0002:00005178       __unwindtable$?detach_helper_grow@?$QList@VQString@@@@AAEPAUNode@1@HH@Z 10026178     DiamondBuildTask.obj
 0002:00005198       __ehfuncinfo$?detach_helper_grow@?$QList@VQString@@@@AAEPAUNode@1@HH@Z 10026198     DiamondBuildTask.obj
 0002:000051bc       __tryblocktable$?detach_helper_grow@?$QList@VQString@@@@AAEPAUNode@1@HH@Z 100261bc     DiamondBuildTask.obj
 0002:000051e4       __unwindtable$?node_construct@?$QList@VQString@@@@AAEXPAUNode@1@ABVQString@@@Z 100261e4     DiamondBuildTask.obj
 0002:000051f4       __ehfuncinfo$?node_construct@?$QList@VQString@@@@AAEXPAUNode@1@ABVQString@@@Z 100261f4     DiamondBuildTask.obj
 0002:00005218       __catchsym$?node_copy@?$QList@VQString@@@@AAEXPAUNode@1@00@Z$6 10026218     DiamondBuildTask.obj
 0002:00005228       __tryblocktable$?node_copy@?$QList@VQString@@@@AAEXPAUNode@1@00@Z 10026228     DiamondBuildTask.obj
 0002:0000523c       __ehfuncinfo$?node_copy@?$QList@VQString@@@@AAEXPAUNode@1@00@Z 1002623c     DiamondBuildTask.obj
 0002:00005260       __unwindtable$?node_copy@?$QList@VQString@@@@AAEXPAUNode@1@00@Z 10026260     DiamondBuildTask.obj
 0002:00005290       __unwindtable$??__EalgoLog@U2@@YAXXZ 10026290     DiamondBuildTask.obj
 0002:00005298       __ehfuncinfo$??__EalgoLog@U2@@YAXXZ 10026298     DiamondBuildTask.obj
 0002:000052bc       __unwindtable$??__EcmdLog@U2@@YAXXZ 100262bc     DiamondBuildTask.obj
 0002:000052c4       __ehfuncinfo$??__EcmdLog@U2@@YAXXZ 100262c4     DiamondBuildTask.obj
 0002:000052e8       __unwindtable$??__EcoreLog@U2@@YAXXZ 100262e8     DiamondBuildTask.obj
 0002:000052f0       __ehfuncinfo$??__EcoreLog@U2@@YAXXZ 100262f0     DiamondBuildTask.obj
 0002:00005314       __unwindtable$??__EioLog@U2@@YAXXZ 10026314     DiamondBuildTask.obj
 0002:0000531c       __ehfuncinfo$??__EioLog@U2@@YAXXZ 1002631c     DiamondBuildTask.obj
 0002:00005340       __unwindtable$??__EperfLog@U2@@YAXXZ 10026340     DiamondBuildTask.obj
 0002:00005348       __ehfuncinfo$??__EperfLog@U2@@YAXXZ 10026348     DiamondBuildTask.obj
 0002:0000536c       __unwindtable$??__EscriptLog@U2@@YAXXZ 1002636c     DiamondBuildTask.obj
 0002:00005374       __ehfuncinfo$??__EscriptLog@U2@@YAXXZ 10026374     DiamondBuildTask.obj
 0002:00005398       __unwindtable$??__EtaskLog@U2@@YAXXZ 10026398     DiamondBuildTask.obj
 0002:000053a0       __ehfuncinfo$??__EtaskLog@U2@@YAXXZ 100263a0     DiamondBuildTask.obj
 0002:000053c4       __unwindtable$??__EuiLog@U2@@YAXXZ 100263c4     DiamondBuildTask.obj
 0002:000053cc       __ehfuncinfo$??__EuiLog@U2@@YAXXZ 100263cc     DiamondBuildTask.obj
 0002:000053f0       __unwindtable$??__EuserActLog@U2@@YAXXZ 100263f0     DiamondBuildTask.obj
 0002:000053f8       __ehfuncinfo$??__EuserActLog@U2@@YAXXZ 100263f8     DiamondBuildTask.obj
 0002:0000541c       __catchsym$?append@?$QList@PAVTask@U2@@@@QAEXABQAVTask@U2@@@Z$6 1002641c     DiamondBuildTask.obj
 0002:0000542c       __tryblocktable$?append@?$QList@PAVTask@U2@@@@QAEXABQAVTask@U2@@@Z 1002642c     DiamondBuildTask.obj
 0002:00005440       __ehfuncinfo$?append@?$QList@PAVTask@U2@@@@QAEXABQAVTask@U2@@@Z 10026440     DiamondBuildTask.obj
 0002:00005464       __unwindtable$?append@?$QList@PAVTask@U2@@@@QAEXABQAVTask@U2@@@Z 10026464     DiamondBuildTask.obj
 0002:00005494       __catchsym$?detach_helper_grow@?$QList@PAVTask@U2@@@@AAEPAUNode@1@HH@Z$5 10026494     DiamondBuildTask.obj
 0002:000054a4       __catchsym$?detach_helper_grow@?$QList@PAVTask@U2@@@@AAEPAUNode@1@HH@Z$4 100264a4     DiamondBuildTask.obj
 0002:000054b4       __unwindtable$?detach_helper_grow@?$QList@PAVTask@U2@@@@AAEPAUNode@1@HH@Z 100264b4     DiamondBuildTask.obj
 0002:000054d4       __ehfuncinfo$?detach_helper_grow@?$QList@PAVTask@U2@@@@AAEPAUNode@1@HH@Z 100264d4     DiamondBuildTask.obj
 0002:000054f8       __tryblocktable$?detach_helper_grow@?$QList@PAVTask@U2@@@@AAEPAUNode@1@HH@Z 100264f8     DiamondBuildTask.obj
 0002:00005520       __unwindtable$??1DiamondBuildTaskSettings@U2@@QAE@XZ 10026520     DiamondBuildTask.obj
 0002:00005540       __ehfuncinfo$??1DiamondBuildTaskSettings@U2@@QAE@XZ 10026540     DiamondBuildTask.obj
 0002:00005564       __unwindtable$??0DiamondBuildTaskSettings@U2@@QAE@ABU01@@Z 10026564     DiamondBuildTask.obj
 0002:00005584       __ehfuncinfo$??0DiamondBuildTaskSettings@U2@@QAE@ABU01@@Z 10026584     DiamondBuildTask.obj
 0002:000055a8       __ehfuncinfo$??0DiamondBuildTask@U2@@QAE@ABUDiamondBuildTaskSettings@1@@Z 100265a8     DiamondBuildTask.obj
 0002:000055cc       __unwindtable$??0DiamondBuildTask@U2@@QAE@ABUDiamondBuildTaskSettings@1@@Z 100265cc     DiamondBuildTask.obj
 0002:0000562c       __ehfuncinfo$?prepare@DiamondBuildTask@U2@@EAEXXZ 1002662c     DiamondBuildTask.obj
 0002:00005650       __unwindtable$?prepare@DiamondBuildTask@U2@@EAEXXZ 10026650     DiamondBuildTask.obj
 0002:00005688       __ehfuncinfo$?onSubTaskFinished@DiamondBuildTask@U2@@EAE?AV?$QList@PAVTask@U2@@@@PAVTask@2@@Z 10026688     DiamondBuildTask.obj
 0002:000056ac       __unwindtable$?onSubTaskFinished@DiamondBuildTask@U2@@EAE?AV?$QList@PAVTask@U2@@@@PAVTask@2@@Z 100266ac     DiamondBuildTask.obj
 0002:0000570c       __unwindtable$?checkSettings@DiamondBuildTask@U2@@AAEXXZ 1002670c     DiamondBuildTask.obj
 0002:0000572c       __ehfuncinfo$?checkSettings@DiamondBuildTask@U2@@AAEXXZ 1002672c     DiamondBuildTask.obj
 0002:00005750       __ehfuncinfo$?getArguments@DiamondBuildTask@U2@@ABE?AVQStringList@@ABVQString@@@Z 10026750     DiamondBuildTask.obj
 0002:00005774       __unwindtable$?getArguments@DiamondBuildTask@U2@@ABE?AVQStringList@@ABVQString@@@Z 10026774     DiamondBuildTask.obj
 0002:000057a4       __ehfuncinfo$??1DiamondBuildTask@U2@@UAE@XZ 100267a4     DiamondBuildTask.obj
 0002:000057c8       __unwindtable$??1DiamondBuildTask@U2@@UAE@XZ 100267c8     DiamondBuildTask.obj
 0002:000057f0       __unwindtable$??__EalgoLog@U2@@YAXXZ 100267f0     DiamondBuildValidator.obj
 0002:000057f8       __ehfuncinfo$??__EalgoLog@U2@@YAXXZ 100267f8     DiamondBuildValidator.obj
 0002:0000581c       __unwindtable$??__EcmdLog@U2@@YAXXZ 1002681c     DiamondBuildValidator.obj
 0002:00005824       __ehfuncinfo$??__EcmdLog@U2@@YAXXZ 10026824     DiamondBuildValidator.obj
 0002:00005848       __unwindtable$??__EcoreLog@U2@@YAXXZ 10026848     DiamondBuildValidator.obj
 0002:00005850       __ehfuncinfo$??__EcoreLog@U2@@YAXXZ 10026850     DiamondBuildValidator.obj
 0002:00005874       __unwindtable$??__EioLog@U2@@YAXXZ 10026874     DiamondBuildValidator.obj
 0002:0000587c       __ehfuncinfo$??__EioLog@U2@@YAXXZ 1002687c     DiamondBuildValidator.obj
 0002:000058a0       __unwindtable$??__EperfLog@U2@@YAXXZ 100268a0     DiamondBuildValidator.obj
 0002:000058a8       __ehfuncinfo$??__EperfLog@U2@@YAXXZ 100268a8     DiamondBuildValidator.obj
 0002:000058cc       __unwindtable$??__EscriptLog@U2@@YAXXZ 100268cc     DiamondBuildValidator.obj
 0002:000058d4       __ehfuncinfo$??__EscriptLog@U2@@YAXXZ 100268d4     DiamondBuildValidator.obj
 0002:000058f8       __unwindtable$??__EtaskLog@U2@@YAXXZ 100268f8     DiamondBuildValidator.obj
 0002:00005900       __ehfuncinfo$??__EtaskLog@U2@@YAXXZ 10026900     DiamondBuildValidator.obj
 0002:00005924       __unwindtable$??__EuiLog@U2@@YAXXZ 10026924     DiamondBuildValidator.obj
 0002:0000592c       __ehfuncinfo$??__EuiLog@U2@@YAXXZ 1002692c     DiamondBuildValidator.obj
 0002:00005950       __unwindtable$??__EuserActLog@U2@@YAXXZ 10026950     DiamondBuildValidator.obj
 0002:00005958       __ehfuncinfo$??__EuserActLog@U2@@YAXXZ 10026958     DiamondBuildValidator.obj
 0002:0000597c       __ehfuncinfo$?validateTaxonomy@DiamondBuildValidator@Workflow@U2@@ABE_NPBVActor@23@AAV?$QList@VWorkflowNotification@U2@@@@@Z 1002697c     DiamondBuildValidator.obj
 0002:000059a0       __unwindtable$?validateTaxonomy@DiamondBuildValidator@Workflow@U2@@ABE_NPBVActor@23@AAV?$QList@VWorkflowNotification@U2@@@@@Z 100269a0     DiamondBuildValidator.obj
 0002:00005a08       __catchsym$?append@?$QList@VWorkflowNotification@U2@@@@QAEXABVWorkflowNotification@U2@@@Z$11 10026a08     DiamondBuildValidator.obj
 0002:00005a18       __catchsym$?append@?$QList@VWorkflowNotification@U2@@@@QAEXABVWorkflowNotification@U2@@@Z$10 10026a18     DiamondBuildValidator.obj
 0002:00005a28       __ehfuncinfo$?append@?$QList@VWorkflowNotification@U2@@@@QAEXABVWorkflowNotification@U2@@@Z 10026a28     DiamondBuildValidator.obj
 0002:00005a4c       __tryblocktable$?append@?$QList@VWorkflowNotification@U2@@@@QAEXABVWorkflowNotification@U2@@@Z 10026a4c     DiamondBuildValidator.obj
 0002:00005a74       __unwindtable$?append@?$QList@VWorkflowNotification@U2@@@@QAEXABVWorkflowNotification@U2@@@Z 10026a74     DiamondBuildValidator.obj
 0002:00005ac4       __catchsym$?detach_helper_grow@?$QList@VWorkflowNotification@U2@@@@AAEPAUNode@1@HH@Z$5 10026ac4     DiamondBuildValidator.obj
 0002:00005ad4       __catchsym$?detach_helper_grow@?$QList@VWorkflowNotification@U2@@@@AAEPAUNode@1@HH@Z$4 10026ad4     DiamondBuildValidator.obj
 0002:00005ae4       __unwindtable$?detach_helper_grow@?$QList@VWorkflowNotification@U2@@@@AAEPAUNode@1@HH@Z 10026ae4     DiamondBuildValidator.obj
 0002:00005b04       __ehfuncinfo$?detach_helper_grow@?$QList@VWorkflowNotification@U2@@@@AAEPAUNode@1@HH@Z 10026b04     DiamondBuildValidator.obj
 0002:00005b28       __tryblocktable$?detach_helper_grow@?$QList@VWorkflowNotification@U2@@@@AAEPAUNode@1@HH@Z 10026b28     DiamondBuildValidator.obj
 0002:00005b50       __unwindtable$?node_construct@?$QList@VWorkflowNotification@U2@@@@AAEXPAUNode@1@ABVWorkflowNotification@U2@@@Z 10026b50     DiamondBuildValidator.obj
 0002:00005b60       __ehfuncinfo$?node_construct@?$QList@VWorkflowNotification@U2@@@@AAEXPAUNode@1@ABVWorkflowNotification@U2@@@Z 10026b60     DiamondBuildValidator.obj
 0002:00005b84       __catchsym$?node_copy@?$QList@VWorkflowNotification@U2@@@@AAEXPAUNode@1@00@Z$6 10026b84     DiamondBuildValidator.obj
 0002:00005b94       __tryblocktable$?node_copy@?$QList@VWorkflowNotification@U2@@@@AAEXPAUNode@1@00@Z 10026b94     DiamondBuildValidator.obj
 0002:00005ba8       __ehfuncinfo$?node_copy@?$QList@VWorkflowNotification@U2@@@@AAEXPAUNode@1@00@Z 10026ba8     DiamondBuildValidator.obj
 0002:00005bcc       __unwindtable$?node_copy@?$QList@VWorkflowNotification@U2@@@@AAEXPAUNode@1@00@Z 10026bcc     DiamondBuildValidator.obj
 0002:00005bfc       __unwindtable$??H@YA?BVQString@@ABV0@0@Z 10026bfc     DiamondBuildWorker.obj
 0002:00005c04       __ehfuncinfo$??H@YA?BVQString@@ABV0@0@Z 10026c04     DiamondBuildWorker.obj
 0002:00005c28       __unwindtable$??0QStringList@@QAE@ABVQString@@@Z 10026c28     DiamondBuildWorker.obj
 0002:00005c30       __ehfuncinfo$??0QStringList@@QAE@ABVQString@@@Z 10026c30     DiamondBuildWorker.obj
 0002:00005c54       __unwindtable$??A?$QMap@VQString@@VQVariant@@@@QAEAAVQVariant@@ABVQString@@@Z 10026c54     DiamondBuildWorker.obj
 0002:00005c5c       __ehfuncinfo$??A?$QMap@VQString@@VQVariant@@@@QAEAAVQVariant@@ABVQString@@@Z 10026c5c     DiamondBuildWorker.obj
 0002:00005c80       __unwindtable$??__EalgoLog@U2@@YAXXZ 10026c80     DiamondBuildWorker.obj
 0002:00005c88       __ehfuncinfo$??__EalgoLog@U2@@YAXXZ 10026c88     DiamondBuildWorker.obj
 0002:00005cac       __unwindtable$??__EcmdLog@U2@@YAXXZ 10026cac     DiamondBuildWorker.obj
 0002:00005cb4       __ehfuncinfo$??__EcmdLog@U2@@YAXXZ 10026cb4     DiamondBuildWorker.obj
 0002:00005cd8       __unwindtable$??__EcoreLog@U2@@YAXXZ 10026cd8     DiamondBuildWorker.obj
 0002:00005ce0       __ehfuncinfo$??__EcoreLog@U2@@YAXXZ 10026ce0     DiamondBuildWorker.obj
 0002:00005d04       __unwindtable$??__EioLog@U2@@YAXXZ 10026d04     DiamondBuildWorker.obj
 0002:00005d0c       __ehfuncinfo$??__EioLog@U2@@YAXXZ 10026d0c     DiamondBuildWorker.obj
 0002:00005d30       __unwindtable$??__EperfLog@U2@@YAXXZ 10026d30     DiamondBuildWorker.obj
 0002:00005d38       __ehfuncinfo$??__EperfLog@U2@@YAXXZ 10026d38     DiamondBuildWorker.obj
 0002:00005d5c       __unwindtable$??__EscriptLog@U2@@YAXXZ 10026d5c     DiamondBuildWorker.obj
 0002:00005d64       __ehfuncinfo$??__EscriptLog@U2@@YAXXZ 10026d64     DiamondBuildWorker.obj
 0002:00005d88       __unwindtable$??__EtaskLog@U2@@YAXXZ 10026d88     DiamondBuildWorker.obj
 0002:00005d90       __ehfuncinfo$??__EtaskLog@U2@@YAXXZ 10026d90     DiamondBuildWorker.obj
 0002:00005db4       __unwindtable$??__EuiLog@U2@@YAXXZ 10026db4     DiamondBuildWorker.obj
 0002:00005dbc       __ehfuncinfo$??__EuiLog@U2@@YAXXZ 10026dbc     DiamondBuildWorker.obj
 0002:00005de0       __unwindtable$??__EuserActLog@U2@@YAXXZ 10026de0     DiamondBuildWorker.obj
 0002:00005de8       __ehfuncinfo$??__EuserActLog@U2@@YAXXZ 10026de8     DiamondBuildWorker.obj
 0002:00005e0c       __catchsym$??0?$QList@VDescriptor@U2@@@@QAE@ABV0@@Z$2 10026e0c     DiamondBuildWorker.obj
 0002:00005e1c       __unwindtable$??0?$QList@VDescriptor@U2@@@@QAE@ABV0@@Z 10026e1c     DiamondBuildWorker.obj
 0002:00005e2c       __tryblocktable$??0?$QList@VDescriptor@U2@@@@QAE@ABV0@@Z 10026e2c     DiamondBuildWorker.obj
 0002:00005e40       __ehfuncinfo$??0?$QList@VDescriptor@U2@@@@QAE@ABV0@@Z 10026e40     DiamondBuildWorker.obj
 0002:00005e64       __catchsym$?append@?$QList@VDescriptor@U2@@@@QAEXABVDescriptor@U2@@@Z$9 10026e64     DiamondBuildWorker.obj
 0002:00005e74       __catchsym$?append@?$QList@VDescriptor@U2@@@@QAEXABVDescriptor@U2@@@Z$8 10026e74     DiamondBuildWorker.obj
 0002:00005e84       __ehfuncinfo$?append@?$QList@VDescriptor@U2@@@@QAEXABVDescriptor@U2@@@Z 10026e84     DiamondBuildWorker.obj
 0002:00005ea8       __tryblocktable$?append@?$QList@VDescriptor@U2@@@@QAEXABVDescriptor@U2@@@Z 10026ea8     DiamondBuildWorker.obj
 0002:00005ed0       __unwindtable$?append@?$QList@VDescriptor@U2@@@@QAEXABVDescriptor@U2@@@Z 10026ed0     DiamondBuildWorker.obj
 0002:00005f10       __catchsym$?detach_helper_grow@?$QList@VDescriptor@U2@@@@AAEPAUNode@1@HH@Z$5 10026f10     DiamondBuildWorker.obj
 0002:00005f20       __catchsym$?detach_helper_grow@?$QList@VDescriptor@U2@@@@AAEPAUNode@1@HH@Z$4 10026f20     DiamondBuildWorker.obj
 0002:00005f30       __unwindtable$?detach_helper_grow@?$QList@VDescriptor@U2@@@@AAEPAUNode@1@HH@Z 10026f30     DiamondBuildWorker.obj
 0002:00005f50       __ehfuncinfo$?detach_helper_grow@?$QList@VDescriptor@U2@@@@AAEPAUNode@1@HH@Z 10026f50     DiamondBuildWorker.obj
 0002:00005f74       __tryblocktable$?detach_helper_grow@?$QList@VDescriptor@U2@@@@AAEPAUNode@1@HH@Z 10026f74     DiamondBuildWorker.obj
 0002:00005f9c       __catchsym$?detach_helper@?$QList@VDescriptor@U2@@@@AAEXH@Z$2 10026f9c     DiamondBuildWorker.obj
 0002:00005fac       __unwindtable$?detach_helper@?$QList@VDescriptor@U2@@@@AAEXH@Z 10026fac     DiamondBuildWorker.obj
 0002:00005fbc       __tryblocktable$?detach_helper@?$QList@VDescriptor@U2@@@@AAEXH@Z 10026fbc     DiamondBuildWorker.obj
 0002:00005fd0       __ehfuncinfo$?detach_helper@?$QList@VDescriptor@U2@@@@AAEXH@Z 10026fd0     DiamondBuildWorker.obj
 0002:00005ff4       __unwindtable$?node_construct@?$QList@VDescriptor@U2@@@@AAEXPAUNode@1@ABVDescriptor@U2@@@Z 10026ff4     DiamondBuildWorker.obj
 0002:00006004       __ehfuncinfo$?node_construct@?$QList@VDescriptor@U2@@@@AAEXPAUNode@1@ABVDescriptor@U2@@@Z 10027004     DiamondBuildWorker.obj
 0002:00006028       __catchsym$?node_copy@?$QList@VDescriptor@U2@@@@AAEXPAUNode@1@00@Z$6 10027028     DiamondBuildWorker.obj
 0002:00006038       __tryblocktable$?node_copy@?$QList@VDescriptor@U2@@@@AAEXPAUNode@1@00@Z 10027038     DiamondBuildWorker.obj
 0002:0000604c       __ehfuncinfo$?node_copy@?$QList@VDescriptor@U2@@@@AAEXPAUNode@1@00@Z 1002704c     DiamondBuildWorker.obj
 0002:00006070       __unwindtable$?node_copy@?$QList@VDescriptor@U2@@@@AAEXPAUNode@1@00@Z 10027070     DiamondBuildWorker.obj
 0002:000060a0       __catchsym$??0?$QList@PAVURLContainer@U2@@@@QAE@ABV0@@Z$2 100270a0     DiamondBuildWorker.obj
 0002:000060b0       __unwindtable$??0?$QList@PAVURLContainer@U2@@@@QAE@ABV0@@Z 100270b0     DiamondBuildWorker.obj
 0002:000060c0       __tryblocktable$??0?$QList@PAVURLContainer@U2@@@@QAE@ABV0@@Z 100270c0     DiamondBuildWorker.obj
 0002:000060d4       __ehfuncinfo$??0?$QList@PAVURLContainer@U2@@@@QAE@ABV0@@Z 100270d4     DiamondBuildWorker.obj
 0002:000060f8       __catchsym$??0?$QList@VDataset@U2@@@@QAE@ABV0@@Z$2 100270f8     DiamondBuildWorker.obj
 0002:00006108       __unwindtable$??0?$QList@VDataset@U2@@@@QAE@ABV0@@Z 10027108     DiamondBuildWorker.obj
 0002:00006118       __tryblocktable$??0?$QList@VDataset@U2@@@@QAE@ABV0@@Z 10027118     DiamondBuildWorker.obj
 0002:0000612c       __ehfuncinfo$??0?$QList@VDataset@U2@@@@QAE@ABV0@@Z 1002712c     DiamondBuildWorker.obj
 0002:00006150       __catchsym$?node_copy@?$QList@VDataset@U2@@@@AAEXPAUNode@1@00@Z$6 10027150     DiamondBuildWorker.obj
 0002:00006160       __tryblocktable$?node_copy@?$QList@VDataset@U2@@@@AAEXPAUNode@1@00@Z 10027160     DiamondBuildWorker.obj
 0002:00006174       __ehfuncinfo$?node_copy@?$QList@VDataset@U2@@@@AAEXPAUNode@1@00@Z 10027174     DiamondBuildWorker.obj
 0002:00006198       __unwindtable$?node_copy@?$QList@VDataset@U2@@@@AAEXPAUNode@1@00@Z 10027198     DiamondBuildWorker.obj
 0002:000061c8       __unwindtable$?qt_metatype_id@?$QMetaTypeId@V?$QList@VDataset@U2@@@@@@SAHXZ 100271c8     DiamondBuildWorker.obj
 0002:000061d0       __ehfuncinfo$?qt_metatype_id@?$QMetaTypeId@V?$QList@VDataset@U2@@@@@@SAHXZ 100271d0     DiamondBuildWorker.obj
 0002:000061f4       __unwindtable$??$qRegisterMetaType@V?$QList@VDataset@U2@@@@@@YAHPBDPAV?$QList@VDataset@U2@@@@W4DefinedType@?$MetaTypeDefinedHelper@V?$QList@VDataset@U2@@@@$00@QtPrivate@@@Z 100271f4     DiamondBuildWorker.obj
 0002:000061fc       __ehfuncinfo$??$qRegisterMetaType@V?$QList@VDataset@U2@@@@@@YAHPBDPAV?$QList@VDataset@U2@@@@W4DefinedType@?$MetaTypeDefinedHelper@V?$QList@VDataset@U2@@@@$00@QtPrivate@@@Z 100271fc     DiamondBuildWorker.obj
 0002:00006220       __unwindtable$??A?$QMap@VQString@@VQScriptValue@@@@QAEAAVQScriptValue@@ABVQString@@@Z 10027220     DiamondBuildWorker.obj
 0002:00006228       __ehfuncinfo$??A?$QMap@VQString@@VQScriptValue@@@@QAEAAVQScriptValue@@ABVQString@@@Z 10027228     DiamondBuildWorker.obj
 0002:0000624c       __unwindtable$?uniqueKeys@?$QMap@VDescriptor@U2@@VQVariant@@@@QBE?AV?$QList@VDescriptor@U2@@@@XZ 1002724c     DiamondBuildWorker.obj
 0002:00006254       __ehfuncinfo$?uniqueKeys@?$QMap@VDescriptor@U2@@VQVariant@@@@QBE?AV?$QList@VDescriptor@U2@@@@XZ 10027254     DiamondBuildWorker.obj
 0002:00006278       __ehfuncinfo$??$getAttributeValue@VQString@@@Attribute@U2@@QBE?AVQString@@PAVWorkflowContext@Workflow@1@@Z 10027278     DiamondBuildWorker.obj
 0002:0000629c       __unwindtable$??$getAttributeValue@VQString@@@Attribute@U2@@QBE?AVQString@@PAVWorkflowContext@Workflow@1@@Z 1002729c     DiamondBuildWorker.obj
 0002:0000630c       __unwindtable$??$getValue@VQString@@@BaseWorker@LocalWorkflow@U2@@IBE?AVQString@@ABV3@@Z 1002730c     DiamondBuildWorker.obj
 0002:0000631c       __ehfuncinfo$??$getValue@VQString@@@BaseWorker@LocalWorkflow@U2@@IBE?AVQString@@ABV3@@Z 1002731c     DiamondBuildWorker.obj
 0002:00006340       __unwindtable$??0DiamondBuildTaskSettings@U2@@QAE@XZ 10027340     DiamondBuildWorker.obj
 0002:00006360       __ehfuncinfo$??0DiamondBuildTaskSettings@U2@@QAE@XZ 10027360     DiamondBuildWorker.obj
 0002:00006384       __ehfuncinfo$?init@DiamondBuildWorker@LocalWorkflow@U2@@UAEXXZ 10027384     DiamondBuildWorker.obj
 0002:000063a8       __unwindtable$?init@DiamondBuildWorker@LocalWorkflow@U2@@UAEXXZ 100273a8     DiamondBuildWorker.obj
 0002:000063e0       __ehfuncinfo$?tick@DiamondBuildWorker@LocalWorkflow@U2@@UAEPAVTask@3@XZ 100273e0     DiamondBuildWorker.obj
 0002:00006404       __unwindtable$?tick@DiamondBuildWorker@LocalWorkflow@U2@@UAEPAVTask@3@XZ 10027404     DiamondBuildWorker.obj
 0002:00006464       __ehfuncinfo$?sl_taskFinished@DiamondBuildWorker@LocalWorkflow@U2@@AAEXPAVTask@3@@Z 10027464     DiamondBuildWorker.obj
 0002:00006488       __unwindtable$?sl_taskFinished@DiamondBuildWorker@LocalWorkflow@U2@@AAEXPAVTask@3@@Z 10027488     DiamondBuildWorker.obj
 0002:000064e0       __ehfuncinfo$?getSettings@DiamondBuildWorker@LocalWorkflow@U2@@AAE?AUDiamondBuildTaskSettings@3@AAVU2OpStatus@3@@Z 100274e0     DiamondBuildWorker.obj
 0002:00006504       __unwindtable$?getSettings@DiamondBuildWorker@LocalWorkflow@U2@@AAE?AUDiamondBuildTaskSettings@3@AAVU2OpStatus@3@@Z 10027504     DiamondBuildWorker.obj
 0002:000066bc       __catchsym$?createNode@?$QMapData@VQString@@VQVariant@@@@QAEPAU?$QMapNode@VQString@@VQVariant@@@@ABVQString@@ABVQVariant@@PAU2@_N@Z$7 100276bc     DiamondBuildWorker.obj
 0002:000066cc       __catchsym$?createNode@?$QMapData@VQString@@VQVariant@@@@QAEPAU?$QMapNode@VQString@@VQVariant@@@@ABVQString@@ABVQVariant@@PAU2@_N@Z$6 100276cc     DiamondBuildWorker.obj
 0002:000066dc       __ehfuncinfo$?createNode@?$QMapData@VQString@@VQVariant@@@@QAEPAU?$QMapNode@VQString@@VQVariant@@@@ABVQString@@ABVQVariant@@PAU2@_N@Z 100276dc     DiamondBuildWorker.obj
 0002:00006700       __tryblocktable$?createNode@?$QMapData@VQString@@VQVariant@@@@QAEPAU?$QMapNode@VQString@@VQVariant@@@@ABVQString@@ABVQVariant@@PAU2@_N@Z 10027700     DiamondBuildWorker.obj
 0002:00006728       __unwindtable$?createNode@?$QMapData@VQString@@VQVariant@@@@QAEPAU?$QMapNode@VQString@@VQVariant@@@@ABVQString@@ABVQVariant@@PAU2@_N@Z 10027728     DiamondBuildWorker.obj
 0002:00006758       __catchsym$?createNode@?$QMapData@VQString@@VQScriptValue@@@@QAEPAU?$QMapNode@VQString@@VQScriptValue@@@@ABVQString@@ABVQScriptValue@@PAU2@_N@Z$7 10027758     DiamondBuildWorker.obj
 0002:00006768       __catchsym$?createNode@?$QMapData@VQString@@VQScriptValue@@@@QAEPAU?$QMapNode@VQString@@VQScriptValue@@@@ABVQString@@ABVQScriptValue@@PAU2@_N@Z$6 10027768     DiamondBuildWorker.obj
 0002:00006778       __ehfuncinfo$?createNode@?$QMapData@VQString@@VQScriptValue@@@@QAEPAU?$QMapNode@VQString@@VQScriptValue@@@@ABVQString@@ABVQScriptValue@@PAU2@_N@Z 10027778     DiamondBuildWorker.obj
 0002:0000679c       __tryblocktable$?createNode@?$QMapData@VQString@@VQScriptValue@@@@QAEPAU?$QMapNode@VQString@@VQScriptValue@@@@ABVQString@@ABVQScriptValue@@PAU2@_N@Z 1002779c     DiamondBuildWorker.obj
 0002:000067c4       __unwindtable$?createNode@?$QMapData@VQString@@VQScriptValue@@@@QAEPAU?$QMapNode@VQString@@VQScriptValue@@@@ABVQString@@ABVQScriptValue@@PAU2@_N@Z 100277c4     DiamondBuildWorker.obj
 0002:000067f4       __unwindtable$?metaType@?$QVariantValueHelper@VQString@@@QtPrivate@@SA?AVQString@@ABVQVariant@@@Z 100277f4     DiamondBuildWorker.obj
 0002:00006804       __ehfuncinfo$?metaType@?$QVariantValueHelper@VQString@@@QtPrivate@@SA?AVQString@@ABVQVariant@@@Z 10027804     DiamondBuildWorker.obj
 0002:00006828       __unwindtable$?Create@?$QMetaTypeFunctionHelper@V?$QList@VDataset@U2@@@@$00@QtMetaTypePrivate@@SAPAXPBX@Z 10027828     DiamondBuildWorker.obj
 0002:00006830       __ehfuncinfo$?Create@?$QMetaTypeFunctionHelper@V?$QList@VDataset@U2@@@@$00@QtMetaTypePrivate@@SAPAXPBX@Z 10027830     DiamondBuildWorker.obj
 0002:00006854       __unwindtable$?Construct@?$QMetaTypeFunctionHelper@V?$QList@VDataset@U2@@@@$00@QtMetaTypePrivate@@SAPAXPAXPBX@Z 10027854     DiamondBuildWorker.obj
 0002:0000685c       __ehfuncinfo$?Construct@?$QMetaTypeFunctionHelper@V?$QList@VDataset@U2@@@@$00@QtMetaTypePrivate@@SAPAXPAXPBX@Z 1002785c     DiamondBuildWorker.obj
 0002:00006880       __unwindtable$?metaType@?$QVariantValueHelper@V?$QList@VDataset@U2@@@@@QtPrivate@@SA?AV?$QList@VDataset@U2@@@@ABVQVariant@@@Z 10027880     DiamondBuildWorker.obj
 0002:00006890       __ehfuncinfo$?metaType@?$QVariantValueHelper@V?$QList@VDataset@U2@@@@@QtPrivate@@SA?AV?$QList@VDataset@U2@@@@ABVQVariant@@@Z 10027890     DiamondBuildWorker.obj
 0002:000068b4       __unwindtable$??__EalgoLog@U2@@YAXXZ 100278b4     DiamondBuildWorkerFactory.obj
 0002:000068bc       __ehfuncinfo$??__EalgoLog@U2@@YAXXZ 100278bc     DiamondBuildWorkerFactory.obj
 0002:000068e0       __unwindtable$??__EcmdLog@U2@@YAXXZ 100278e0     DiamondBuildWorkerFactory.obj
 0002:000068e8       __ehfuncinfo$??__EcmdLog@U2@@YAXXZ 100278e8     DiamondBuildWorkerFactory.obj
 0002:0000690c       __unwindtable$??__EcoreLog@U2@@YAXXZ 1002790c     DiamondBuildWorkerFactory.obj
 0002:00006914       __ehfuncinfo$??__EcoreLog@U2@@YAXXZ 10027914     DiamondBuildWorkerFactory.obj
 0002:00006938       __unwindtable$??__EioLog@U2@@YAXXZ 10027938     DiamondBuildWorkerFactory.obj
 0002:00006940       __ehfuncinfo$??__EioLog@U2@@YAXXZ 10027940     DiamondBuildWorkerFactory.obj
 0002:00006964       __unwindtable$??__EperfLog@U2@@YAXXZ 10027964     DiamondBuildWorkerFactory.obj
 0002:0000696c       __ehfuncinfo$??__EperfLog@U2@@YAXXZ 1002796c     DiamondBuildWorkerFactory.obj
 0002:00006990       __unwindtable$??__EscriptLog@U2@@YAXXZ 10027990     DiamondBuildWorkerFactory.obj
 0002:00006998       __ehfuncinfo$??__EscriptLog@U2@@YAXXZ 10027998     DiamondBuildWorkerFactory.obj
 0002:000069bc       __unwindtable$??__EtaskLog@U2@@YAXXZ 100279bc     DiamondBuildWorkerFactory.obj
 0002:000069c4       __ehfuncinfo$??__EtaskLog@U2@@YAXXZ 100279c4     DiamondBuildWorkerFactory.obj
 0002:000069e8       __unwindtable$??__EuiLog@U2@@YAXXZ 100279e8     DiamondBuildWorkerFactory.obj
 0002:000069f0       __ehfuncinfo$??__EuiLog@U2@@YAXXZ 100279f0     DiamondBuildWorkerFactory.obj
 0002:00006a14       __unwindtable$??__EuserActLog@U2@@YAXXZ 10027a14     DiamondBuildWorkerFactory.obj
 0002:00006a1c       __ehfuncinfo$??__EuserActLog@U2@@YAXXZ 10027a1c     DiamondBuildWorkerFactory.obj
 0002:00006a40       __unwindtable$??A?$QMap@VDescriptor@U2@@V?$QExplicitlySharedDataPointer@VDataType@U2@@@@@@QAEAAV?$QExplicitlySharedDataPointer@VDataType@U2@@@@ABVDescriptor@U2@@@Z 10027a40     DiamondBuildWorkerFactory.obj
 0002:00006a48       __ehfuncinfo$??A?$QMap@VDescriptor@U2@@V?$QExplicitlySharedDataPointer@VDataType@U2@@@@@@QAEAAV?$QExplicitlySharedDataPointer@VDataType@U2@@@@ABVDescriptor@U2@@@Z 10027a48     DiamondBuildWorkerFactory.obj
 0002:00006a6c       __catchsym$?append@?$QList@PAVAttribute@U2@@@@QAEXABQAVAttribute@U2@@@Z$6 10027a6c     DiamondBuildWorkerFactory.obj
 0002:00006a7c       __tryblocktable$?append@?$QList@PAVAttribute@U2@@@@QAEXABQAVAttribute@U2@@@Z 10027a7c     DiamondBuildWorkerFactory.obj
 0002:00006a90       __ehfuncinfo$?append@?$QList@PAVAttribute@U2@@@@QAEXABQAVAttribute@U2@@@Z 10027a90     DiamondBuildWorkerFactory.obj
 0002:00006ab4       __unwindtable$?append@?$QList@PAVAttribute@U2@@@@QAEXABQAVAttribute@U2@@@Z 10027ab4     DiamondBuildWorkerFactory.obj
 0002:00006ae4       __catchsym$?detach_helper_grow@?$QList@PAVAttribute@U2@@@@AAEPAUNode@1@HH@Z$5 10027ae4     DiamondBuildWorkerFactory.obj
 0002:00006af4       __catchsym$?detach_helper_grow@?$QList@PAVAttribute@U2@@@@AAEPAUNode@1@HH@Z$4 10027af4     DiamondBuildWorkerFactory.obj
 0002:00006b04       __unwindtable$?detach_helper_grow@?$QList@PAVAttribute@U2@@@@AAEPAUNode@1@HH@Z 10027b04     DiamondBuildWorkerFactory.obj
 0002:00006b24       __ehfuncinfo$?detach_helper_grow@?$QList@PAVAttribute@U2@@@@AAEPAUNode@1@HH@Z 10027b24     DiamondBuildWorkerFactory.obj
 0002:00006b48       __tryblocktable$?detach_helper_grow@?$QList@PAVAttribute@U2@@@@AAEPAUNode@1@HH@Z 10027b48     DiamondBuildWorkerFactory.obj
 0002:00006b70       __catchsym$?append@?$QList@PAVPortDescriptor@Workflow@U2@@@@QAEXABQAVPortDescriptor@Workflow@U2@@@Z$6 10027b70     DiamondBuildWorkerFactory.obj
 0002:00006b80       __tryblocktable$?append@?$QList@PAVPortDescriptor@Workflow@U2@@@@QAEXABQAVPortDescriptor@Workflow@U2@@@Z 10027b80     DiamondBuildWorkerFactory.obj
 0002:00006b94       __ehfuncinfo$?append@?$QList@PAVPortDescriptor@Workflow@U2@@@@QAEXABQAVPortDescriptor@Workflow@U2@@@Z 10027b94     DiamondBuildWorkerFactory.obj
 0002:00006bb8       __unwindtable$?append@?$QList@PAVPortDescriptor@Workflow@U2@@@@QAEXABQAVPortDescriptor@Workflow@U2@@@Z 10027bb8     DiamondBuildWorkerFactory.obj
 0002:00006be8       __catchsym$?detach_helper_grow@?$QList@PAVPortDescriptor@Workflow@U2@@@@AAEPAUNode@1@HH@Z$5 10027be8     DiamondBuildWorkerFactory.obj
 0002:00006bf8       __catchsym$?detach_helper_grow@?$QList@PAVPortDescriptor@Workflow@U2@@@@AAEPAUNode@1@HH@Z$4 10027bf8     DiamondBuildWorkerFactory.obj
 0002:00006c08       __unwindtable$?detach_helper_grow@?$QList@PAVPortDescriptor@Workflow@U2@@@@AAEPAUNode@1@HH@Z 10027c08     DiamondBuildWorkerFactory.obj
 0002:00006c28       __ehfuncinfo$?detach_helper_grow@?$QList@PAVPortDescriptor@Workflow@U2@@@@AAEPAUNode@1@HH@Z 10027c28     DiamondBuildWorkerFactory.obj
 0002:00006c4c       __tryblocktable$?detach_helper_grow@?$QList@PAVPortDescriptor@Workflow@U2@@@@AAEPAUNode@1@HH@Z 10027c4c     DiamondBuildWorkerFactory.obj
 0002:00006c74       __unwindtable$?createWorker@DiamondBuildWorkerFactory@LocalWorkflow@U2@@UAEPAVWorker@Workflow@3@PAVActor@53@@Z 10027c74     DiamondBuildWorkerFactory.obj
 0002:00006c7c       __ehfuncinfo$?createWorker@DiamondBuildWorkerFactory@LocalWorkflow@U2@@UAEPAVWorker@Workflow@3@PAVActor@53@@Z 10027c7c     DiamondBuildWorkerFactory.obj
 0002:00006ca0       __ehfuncinfo$?init@DiamondBuildWorkerFactory@LocalWorkflow@U2@@SAXXZ 10027ca0     DiamondBuildWorkerFactory.obj
 0002:00006cc4       __unwindtable$?init@DiamondBuildWorkerFactory@LocalWorkflow@U2@@SAXXZ 10027cc4     DiamondBuildWorkerFactory.obj
 0002:00006ed4       __catchsym$?createNode@?$QMapData@VDescriptor@U2@@V?$QExplicitlySharedDataPointer@VDataType@U2@@@@@@QAEPAU?$QMapNode@VDescriptor@U2@@V?$QExplicitlySharedDataPointer@VDataType@U2@@@@@@ABVDescriptor@U2@@ABV?$QExplicitlySharedDataPointer@VDataType@U2@@@@PAU2@_N@Z$6 10027ed4     DiamondBuildWorkerFactory.obj
 0002:00006ee4       __tryblocktable$?createNode@?$QMapData@VDescriptor@U2@@V?$QExplicitlySharedDataPointer@VDataType@U2@@@@@@QAEPAU?$QMapNode@VDescriptor@U2@@V?$QExplicitlySharedDataPointer@VDataType@U2@@@@@@ABVDescriptor@U2@@ABV?$QExplicitlySharedDataPointer@VDataType@U2@@@@PAU2@_N@Z 10027ee4     DiamondBuildWorkerFactory.obj
 0002:00006ef8       __ehfuncinfo$?createNode@?$QMapData@VDescriptor@U2@@V?$QExplicitlySharedDataPointer@VDataType@U2@@@@@@QAEPAU?$QMapNode@VDescriptor@U2@@V?$QExplicitlySharedDataPointer@VDataType@U2@@@@@@ABVDescriptor@U2@@ABV?$QExplicitlySharedDataPointer@VDataType@U2@@@@PAU2@_N@Z 10027ef8     DiamondBuildWorkerFactory.obj
 0002:00006f1c       __unwindtable$?createNode@?$QMapData@VDescriptor@U2@@V?$QExplicitlySharedDataPointer@VDataType@U2@@@@@@QAEPAU?$QMapNode@VDescriptor@U2@@V?$QExplicitlySharedDataPointer@VDataType@U2@@@@@@ABVDescriptor@U2@@ABV?$QExplicitlySharedDataPointer@VDataType@U2@@@@PAU2@_N@Z 10027f1c     DiamondBuildWorkerFactory.obj
 0002:00006f44       __catchsym$?createNode@?$QMapData@VQString@@PAVPropertyDelegate@U2@@@@QAEPAU?$QMapNode@VQString@@PAVPropertyDelegate@U2@@@@ABVQString@@ABQAVPropertyDelegate@U2@@PAU2@_N@Z$5 10027f44     DiamondBuildWorkerFactory.obj
 0002:00006f54       __tryblocktable$?createNode@?$QMapData@VQString@@PAVPropertyDelegate@U2@@@@QAEPAU?$QMapNode@VQString@@PAVPropertyDelegate@U2@@@@ABVQString@@ABQAVPropertyDelegate@U2@@PAU2@_N@Z 10027f54     DiamondBuildWorkerFactory.obj
 0002:00006f68       __ehfuncinfo$?createNode@?$QMapData@VQString@@PAVPropertyDelegate@U2@@@@QAEPAU?$QMapNode@VQString@@PAVPropertyDelegate@U2@@@@ABVQString@@ABQAVPropertyDelegate@U2@@PAU2@_N@Z 10027f68     DiamondBuildWorkerFactory.obj
 0002:00006f8c       __unwindtable$?createNode@?$QMapData@VQString@@PAVPropertyDelegate@U2@@@@QAEPAU?$QMapNode@VQString@@PAVPropertyDelegate@U2@@@@ABVQString@@ABQAVPropertyDelegate@U2@@PAU2@_N@Z 10027f8c     DiamondBuildWorkerFactory.obj
 0002:00006fb4       __unwindtable$??__EalgoLog@U2@@YAXXZ 10027fb4     DiamondClassifyPrompter.obj
 0002:00006fbc       __ehfuncinfo$??__EalgoLog@U2@@YAXXZ 10027fbc     DiamondClassifyPrompter.obj
 0002:00006fe0       __unwindtable$??__EcmdLog@U2@@YAXXZ 10027fe0     DiamondClassifyPrompter.obj
 0002:00006fe8       __ehfuncinfo$??__EcmdLog@U2@@YAXXZ 10027fe8     DiamondClassifyPrompter.obj
 0002:0000700c       __unwindtable$??__EcoreLog@U2@@YAXXZ 1002800c     DiamondClassifyPrompter.obj
 0002:00007014       __ehfuncinfo$??__EcoreLog@U2@@YAXXZ 10028014     DiamondClassifyPrompter.obj
 0002:00007038       __unwindtable$??__EioLog@U2@@YAXXZ 10028038     DiamondClassifyPrompter.obj
 0002:00007040       __ehfuncinfo$??__EioLog@U2@@YAXXZ 10028040     DiamondClassifyPrompter.obj
 0002:00007064       __unwindtable$??__EperfLog@U2@@YAXXZ 10028064     DiamondClassifyPrompter.obj
 0002:0000706c       __ehfuncinfo$??__EperfLog@U2@@YAXXZ 1002806c     DiamondClassifyPrompter.obj
 0002:00007090       __unwindtable$??__EscriptLog@U2@@YAXXZ 10028090     DiamondClassifyPrompter.obj
 0002:00007098       __ehfuncinfo$??__EscriptLog@U2@@YAXXZ 10028098     DiamondClassifyPrompter.obj
 0002:000070bc       __unwindtable$??__EtaskLog@U2@@YAXXZ 100280bc     DiamondClassifyPrompter.obj
 0002:000070c4       __ehfuncinfo$??__EtaskLog@U2@@YAXXZ 100280c4     DiamondClassifyPrompter.obj
 0002:000070e8       __unwindtable$??__EuiLog@U2@@YAXXZ 100280e8     DiamondClassifyPrompter.obj
 0002:000070f0       __ehfuncinfo$??__EuiLog@U2@@YAXXZ 100280f0     DiamondClassifyPrompter.obj
 0002:00007114       __unwindtable$??__EuserActLog@U2@@YAXXZ 10028114     DiamondClassifyPrompter.obj
 0002:0000711c       __ehfuncinfo$??__EuserActLog@U2@@YAXXZ 1002811c     DiamondClassifyPrompter.obj
 0002:00007140       __ehfuncinfo$?createDescription@?$PrompterBase@VDiamondClassifyPrompter@LocalWorkflow@U2@@@U2@@UAEPAVActorDocument@Workflow@2@PAVActor@42@@Z 10028140     DiamondClassifyPrompter.obj
 0002:00007164       __unwindtable$?createDescription@?$PrompterBase@VDiamondClassifyPrompter@LocalWorkflow@U2@@@U2@@UAEPAVActorDocument@Workflow@2@PAVActor@42@@Z 10028164     DiamondClassifyPrompter.obj
 0002:0000719c       __ehfuncinfo$?composeRichDoc@DiamondClassifyPrompter@LocalWorkflow@U2@@EAE?AVQString@@XZ 1002819c     DiamondClassifyPrompter.obj
 0002:000071c0       __unwindtable$?composeRichDoc@DiamondClassifyPrompter@LocalWorkflow@U2@@EAE?AVQString@@XZ 100281c0     DiamondClassifyPrompter.obj
 0002:00007218       __catchsym$?detach_helper@?$QList@VQByteArray@@@@AAEXH@Z$2 10028218     DiamondClassifyTask.obj
 0002:00007228       __unwindtable$?detach_helper@?$QList@VQByteArray@@@@AAEXH@Z 10028228     DiamondClassifyTask.obj
 0002:00007238       __tryblocktable$?detach_helper@?$QList@VQByteArray@@@@AAEXH@Z 10028238     DiamondClassifyTask.obj
 0002:0000724c       __ehfuncinfo$?detach_helper@?$QList@VQByteArray@@@@AAEXH@Z 1002824c     DiamondClassifyTask.obj
 0002:00007270       __catchsym$?node_copy@?$QList@VQByteArray@@@@AAEXPAUNode@1@00@Z$6 10028270     DiamondClassifyTask.obj
 0002:00007280       __tryblocktable$?node_copy@?$QList@VQByteArray@@@@AAEXPAUNode@1@00@Z 10028280     DiamondClassifyTask.obj
 0002:00007294       __ehfuncinfo$?node_copy@?$QList@VQByteArray@@@@AAEXPAUNode@1@00@Z 10028294     DiamondClassifyTask.obj
 0002:000072b8       __unwindtable$?node_copy@?$QList@VQByteArray@@@@AAEXPAUNode@1@00@Z 100282b8     DiamondClassifyTask.obj
 0002:000072e8       __unwindtable$??__EalgoLog@U2@@YAXXZ 100282e8     DiamondClassifyTask.obj
 0002:000072f0       __ehfuncinfo$??__EalgoLog@U2@@YAXXZ 100282f0     DiamondClassifyTask.obj
 0002:00007314       __unwindtable$??__EcmdLog@U2@@YAXXZ 10028314     DiamondClassifyTask.obj
 0002:0000731c       __ehfuncinfo$??__EcmdLog@U2@@YAXXZ 1002831c     DiamondClassifyTask.obj
 0002:00007340       __unwindtable$??__EcoreLog@U2@@YAXXZ 10028340     DiamondClassifyTask.obj
 0002:00007348       __ehfuncinfo$??__EcoreLog@U2@@YAXXZ 10028348     DiamondClassifyTask.obj
 0002:0000736c       __unwindtable$??__EioLog@U2@@YAXXZ 1002836c     DiamondClassifyTask.obj
 0002:00007374       __ehfuncinfo$??__EioLog@U2@@YAXXZ 10028374     DiamondClassifyTask.obj
 0002:00007398       __unwindtable$??__EperfLog@U2@@YAXXZ 10028398     DiamondClassifyTask.obj
 0002:000073a0       __ehfuncinfo$??__EperfLog@U2@@YAXXZ 100283a0     DiamondClassifyTask.obj
 0002:000073c4       __unwindtable$??__EscriptLog@U2@@YAXXZ 100283c4     DiamondClassifyTask.obj
 0002:000073cc       __ehfuncinfo$??__EscriptLog@U2@@YAXXZ 100283cc     DiamondClassifyTask.obj
 0002:000073f0       __unwindtable$??__EtaskLog@U2@@YAXXZ 100283f0     DiamondClassifyTask.obj
 0002:000073f8       __ehfuncinfo$??__EtaskLog@U2@@YAXXZ 100283f8     DiamondClassifyTask.obj
 0002:0000741c       __unwindtable$??__EuiLog@U2@@YAXXZ 1002841c     DiamondClassifyTask.obj
 0002:00007424       __ehfuncinfo$??__EuiLog@U2@@YAXXZ 10028424     DiamondClassifyTask.obj
 0002:00007448       __unwindtable$??__EuserActLog@U2@@YAXXZ 10028448     DiamondClassifyTask.obj
 0002:00007450       __ehfuncinfo$??__EuserActLog@U2@@YAXXZ 10028450     DiamondClassifyTask.obj
 0002:00007474       __ehfuncinfo$??0DiamondClassifyTaskSettings@U2@@QAE@XZ 10028474     DiamondClassifyTask.obj
 0002:00007498       __unwindtable$??0DiamondClassifyTaskSettings@U2@@QAE@XZ 10028498     DiamondClassifyTask.obj
 0002:000074d0       __ehfuncinfo$??1DiamondClassifyTaskSettings@U2@@QAE@XZ 100284d0     DiamondClassifyTask.obj
 0002:000074f4       __unwindtable$??1DiamondClassifyTaskSettings@U2@@QAE@XZ 100284f4     DiamondClassifyTask.obj
 0002:0000752c       __ehfuncinfo$??0DiamondClassifyTaskSettings@U2@@QAE@ABU01@@Z 1002852c     DiamondClassifyTask.obj
 0002:00007550       __unwindtable$??0DiamondClassifyTaskSettings@U2@@QAE@ABU01@@Z 10028550     DiamondClassifyTask.obj
 0002:00007588       __ehfuncinfo$??0DiamondClassifyTask@U2@@QAE@ABUDiamondClassifyTaskSettings@1@@Z 10028588     DiamondClassifyTask.obj
 0002:000075ac       __unwindtable$??0DiamondClassifyTask@U2@@QAE@ABUDiamondClassifyTaskSettings@1@@Z 100285ac     DiamondClassifyTask.obj
 0002:000075f4       __ehfuncinfo$?prepare@DiamondClassifyTask@U2@@EAEXXZ 100285f4     DiamondClassifyTask.obj
 0002:00007618       __unwindtable$?prepare@DiamondClassifyTask@U2@@EAEXXZ 10028618     DiamondClassifyTask.obj
 0002:00007668       __ehfuncinfo$?run@DiamondClassifyTask@U2@@EAEXXZ 10028668     DiamondClassifyTask.obj
 0002:0000768c       __unwindtable$?run@DiamondClassifyTask@U2@@EAEXXZ 1002868c     DiamondClassifyTask.obj
 0002:0000770c       __ehfuncinfo$?checkSettings@DiamondClassifyTask@U2@@AAEXXZ 1002870c     DiamondClassifyTask.obj
 0002:00007730       __unwindtable$?checkSettings@DiamondClassifyTask@U2@@AAEXXZ 10028730     DiamondClassifyTask.obj
 0002:00007768       __ehfuncinfo$?getArguments@DiamondClassifyTask@U2@@ABE?AVQStringList@@XZ 10028768     DiamondClassifyTask.obj
 0002:0000778c       __unwindtable$?getArguments@DiamondClassifyTask@U2@@ABE?AVQStringList@@XZ 1002878c     DiamondClassifyTask.obj
 0002:00007874       __unwindtable$??1DiamondClassifyTask@U2@@UAE@XZ 10028874     DiamondClassifyTask.obj
 0002:00007884       __ehfuncinfo$??1DiamondClassifyTask@U2@@UAE@XZ 10028884     DiamondClassifyTask.obj
 0002:000078a8       __unwindtable$??_GDiamondClassifyTask@U2@@UAEPAXI@Z 100288a8     DiamondClassifyTask.obj
 0002:000078b8       __ehfuncinfo$??_GDiamondClassifyTask@U2@@UAEPAXI@Z 100288b8     DiamondClassifyTask.obj
 0002:000078dc       __catchsym$?createNode@?$QMapData@VQString@@I@@QAEPAU?$QMapNode@VQString@@I@@ABVQString@@ABIPAU2@_N@Z$5 100288dc     DiamondClassifyTask.obj
 0002:000078ec       __tryblocktable$?createNode@?$QMapData@VQString@@I@@QAEPAU?$QMapNode@VQString@@I@@ABVQString@@ABIPAU2@_N@Z 100288ec     DiamondClassifyTask.obj
 0002:00007900       __ehfuncinfo$?createNode@?$QMapData@VQString@@I@@QAEPAU?$QMapNode@VQString@@I@@ABVQString@@ABIPAU2@_N@Z 10028900     DiamondClassifyTask.obj
 0002:00007924       __unwindtable$?createNode@?$QMapData@VQString@@I@@QAEPAU?$QMapNode@VQString@@I@@ABVQString@@ABIPAU2@_N@Z 10028924     DiamondClassifyTask.obj
 0002:0000794c       __unwindtable$?qt_metatype_id@?$QMetaTypeId@VQAssociativeIterableImpl@QtMetaTypePrivate@@@@SAHXZ 1002894c     DiamondClassifyWorker.obj
 0002:00007954       __ehfuncinfo$?qt_metatype_id@?$QMetaTypeId@VQAssociativeIterableImpl@QtMetaTypePrivate@@@@SAHXZ 10028954     DiamondClassifyWorker.obj
 0002:00007978       __unwindtable$??$qRegisterMetaType@VQAssociativeIterableImpl@QtMetaTypePrivate@@@@YAHPBDPAVQAssociativeIterableImpl@QtMetaTypePrivate@@W4DefinedType@?$MetaTypeDefinedHelper@VQAssociativeIterableImpl@QtMetaTypePrivate@@$00@QtPrivate@@@Z 10028978     DiamondClassifyWorker.obj
 0002:00007980       __ehfuncinfo$??$qRegisterMetaType@VQAssociativeIterableImpl@QtMetaTypePrivate@@@@YAHPBDPAVQAssociativeIterableImpl@QtMetaTypePrivate@@W4DefinedType@?$MetaTypeDefinedHelper@VQAssociativeIterableImpl@QtMetaTypePrivate@@$00@QtPrivate@@@Z 10028980     DiamondClassifyWorker.obj
 0002:000079a4       __unwindtable$??__EalgoLog@U2@@YAXXZ 100289a4     DiamondClassifyWorker.obj
 0002:000079ac       __ehfuncinfo$??__EalgoLog@U2@@YAXXZ 100289ac     DiamondClassifyWorker.obj
 0002:000079d0       __unwindtable$??__EcmdLog@U2@@YAXXZ 100289d0     DiamondClassifyWorker.obj
 0002:000079d8       __ehfuncinfo$??__EcmdLog@U2@@YAXXZ 100289d8     DiamondClassifyWorker.obj
 0002:000079fc       __unwindtable$??__EcoreLog@U2@@YAXXZ 100289fc     DiamondClassifyWorker.obj
 0002:00007a04       __ehfuncinfo$??__EcoreLog@U2@@YAXXZ 10028a04     DiamondClassifyWorker.obj
 0002:00007a28       __unwindtable$??__EioLog@U2@@YAXXZ 10028a28     DiamondClassifyWorker.obj
 0002:00007a30       __ehfuncinfo$??__EioLog@U2@@YAXXZ 10028a30     DiamondClassifyWorker.obj
 0002:00007a54       __unwindtable$??__EperfLog@U2@@YAXXZ 10028a54     DiamondClassifyWorker.obj
 0002:00007a5c       __ehfuncinfo$??__EperfLog@U2@@YAXXZ 10028a5c     DiamondClassifyWorker.obj
 0002:00007a80       __unwindtable$??__EscriptLog@U2@@YAXXZ 10028a80     DiamondClassifyWorker.obj
 0002:00007a88       __ehfuncinfo$??__EscriptLog@U2@@YAXXZ 10028a88     DiamondClassifyWorker.obj
 0002:00007aac       __unwindtable$??__EtaskLog@U2@@YAXXZ 10028aac     DiamondClassifyWorker.obj
 0002:00007ab4       __ehfuncinfo$??__EtaskLog@U2@@YAXXZ 10028ab4     DiamondClassifyWorker.obj
 0002:00007ad8       __unwindtable$??__EuiLog@U2@@YAXXZ 10028ad8     DiamondClassifyWorker.obj
 0002:00007ae0       __ehfuncinfo$??__EuiLog@U2@@YAXXZ 10028ae0     DiamondClassifyWorker.obj
 0002:00007b04       __unwindtable$??__EuserActLog@U2@@YAXXZ 10028b04     DiamondClassifyWorker.obj
 0002:00007b0c       __ehfuncinfo$??__EuserActLog@U2@@YAXXZ 10028b0c     DiamondClassifyWorker.obj
 0002:00007b30       __ehfuncinfo$??$getAttributeValue@H@Attribute@U2@@QBEHPAVWorkflowContext@Workflow@1@@Z 10028b30     DiamondClassifyWorker.obj
 0002:00007b54       __unwindtable$??$getAttributeValue@H@Attribute@U2@@QBEHPAVWorkflowContext@Workflow@1@@Z 10028b54     DiamondClassifyWorker.obj
 0002:00007bbc       __unwindtable$?qt_metatype_id@?$QMetaTypeId@V?$QMap@VQString@@I@@@@SAHXZ 10028bbc     DiamondClassifyWorker.obj
 0002:00007bc4       __ehfuncinfo$?qt_metatype_id@?$QMetaTypeId@V?$QMap@VQString@@I@@@@SAHXZ 10028bc4     DiamondClassifyWorker.obj
 0002:00007be8       __unwindtable$??$qRegisterMetaType@V?$QMap@VQString@@I@@@@YAHPBDPAV?$QMap@VQString@@I@@W4DefinedType@?$MetaTypeDefinedHelper@V?$QMap@VQString@@I@@$00@QtPrivate@@@Z 10028be8     DiamondClassifyWorker.obj
 0002:00007bf0       __ehfuncinfo$??$qRegisterMetaType@V?$QMap@VQString@@I@@@@YAHPBDPAV?$QMap@VQString@@I@@W4DefinedType@?$MetaTypeDefinedHelper@V?$QMap@VQString@@I@@$00@QtPrivate@@@Z 10028bf0     DiamondClassifyWorker.obj
 0002:00007c14       __ehfuncinfo$?init@DiamondClassifyWorker@LocalWorkflow@U2@@UAEXXZ 10028c14     DiamondClassifyWorker.obj
 0002:00007c38       __unwindtable$?init@DiamondClassifyWorker@LocalWorkflow@U2@@UAEXXZ 10028c38     DiamondClassifyWorker.obj
 0002:00007ca8       __ehfuncinfo$?tick@DiamondClassifyWorker@LocalWorkflow@U2@@UAEPAVTask@3@XZ 10028ca8     DiamondClassifyWorker.obj
 0002:00007ccc       __unwindtable$?tick@DiamondClassifyWorker@LocalWorkflow@U2@@UAEPAVTask@3@XZ 10028ccc     DiamondClassifyWorker.obj
 0002:00007d0c       __ehfuncinfo$?sl_taskFinished@DiamondClassifyWorker@LocalWorkflow@U2@@AAEXPAVTask@3@@Z 10028d0c     DiamondClassifyWorker.obj
 0002:00007d30       __unwindtable$?sl_taskFinished@DiamondClassifyWorker@LocalWorkflow@U2@@AAEXPAVTask@3@@Z 10028d30     DiamondClassifyWorker.obj
 0002:00007d90       __ehfuncinfo$?getSettings@DiamondClassifyWorker@LocalWorkflow@U2@@AAE?AUDiamondClassifyTaskSettings@3@AAVU2OpStatus@3@@Z 10028d90     DiamondClassifyWorker.obj
 0002:00007db4       __unwindtable$?getSettings@DiamondClassifyWorker@LocalWorkflow@U2@@AAE?AUDiamondClassifyTaskSettings@3@AAVU2OpStatus@3@@Z 10028db4     DiamondClassifyWorker.obj
 0002:00007eb4       __unwindtable$?Create@?$QMetaTypeFunctionHelper@V?$QMap@VQString@@I@@$00@QtMetaTypePrivate@@SAPAXPBX@Z 10028eb4     DiamondClassifyWorker.obj
 0002:00007ebc       __ehfuncinfo$?Create@?$QMetaTypeFunctionHelper@V?$QMap@VQString@@I@@$00@QtMetaTypePrivate@@SAPAXPBX@Z 10028ebc     DiamondClassifyWorker.obj
 0002:00007ee0       __unwindtable$?Construct@?$QMetaTypeFunctionHelper@V?$QMap@VQString@@I@@$00@QtMetaTypePrivate@@SAPAXPAXPBX@Z 10028ee0     DiamondClassifyWorker.obj
 0002:00007ee8       __ehfuncinfo$?Construct@?$QMetaTypeFunctionHelper@V?$QMap@VQString@@I@@$00@QtMetaTypePrivate@@SAPAXPAXPBX@Z 10028ee8     DiamondClassifyWorker.obj
 0002:00007f0c       __unwindtable$??__EalgoLog@U2@@YAXXZ 10028f0c     DiamondClassifyWorkerFactory.obj
 0002:00007f14       __ehfuncinfo$??__EalgoLog@U2@@YAXXZ 10028f14     DiamondClassifyWorkerFactory.obj
 0002:00007f38       __unwindtable$??__EcmdLog@U2@@YAXXZ 10028f38     DiamondClassifyWorkerFactory.obj
 0002:00007f40       __ehfuncinfo$??__EcmdLog@U2@@YAXXZ 10028f40     DiamondClassifyWorkerFactory.obj
 0002:00007f64       __unwindtable$??__EcoreLog@U2@@YAXXZ 10028f64     DiamondClassifyWorkerFactory.obj
 0002:00007f6c       __ehfuncinfo$??__EcoreLog@U2@@YAXXZ 10028f6c     DiamondClassifyWorkerFactory.obj
 0002:00007f90       __unwindtable$??__EioLog@U2@@YAXXZ 10028f90     DiamondClassifyWorkerFactory.obj
 0002:00007f98       __ehfuncinfo$??__EioLog@U2@@YAXXZ 10028f98     DiamondClassifyWorkerFactory.obj
 0002:00007fbc       __unwindtable$??__EperfLog@U2@@YAXXZ 10028fbc     DiamondClassifyWorkerFactory.obj
 0002:00007fc4       __ehfuncinfo$??__EperfLog@U2@@YAXXZ 10028fc4     DiamondClassifyWorkerFactory.obj
 0002:00007fe8       __unwindtable$??__EscriptLog@U2@@YAXXZ 10028fe8     DiamondClassifyWorkerFactory.obj
 0002:00007ff0       __ehfuncinfo$??__EscriptLog@U2@@YAXXZ 10028ff0     DiamondClassifyWorkerFactory.obj
 0002:00008014       __unwindtable$??__EtaskLog@U2@@YAXXZ 10029014     DiamondClassifyWorkerFactory.obj
 0002:0000801c       __ehfuncinfo$??__EtaskLog@U2@@YAXXZ 1002901c     DiamondClassifyWorkerFactory.obj
 0002:00008040       __unwindtable$??__EuiLog@U2@@YAXXZ 10029040     DiamondClassifyWorkerFactory.obj
 0002:00008048       __ehfuncinfo$??__EuiLog@U2@@YAXXZ 10029048     DiamondClassifyWorkerFactory.obj
 0002:0000806c       __unwindtable$??__EuserActLog@U2@@YAXXZ 1002906c     DiamondClassifyWorkerFactory.obj
 0002:00008074       __ehfuncinfo$??__EuserActLog@U2@@YAXXZ 10029074     DiamondClassifyWorkerFactory.obj
 0002:00008098       __catchsym$??0?$QList@PAVDNATranslation@U2@@@@QAE@ABV0@@Z$2 10029098     DiamondClassifyWorkerFactory.obj
 0002:000080a8       __unwindtable$??0?$QList@PAVDNATranslation@U2@@@@QAE@ABV0@@Z 100290a8     DiamondClassifyWorkerFactory.obj
 0002:000080b8       __tryblocktable$??0?$QList@PAVDNATranslation@U2@@@@QAE@ABV0@@Z 100290b8     DiamondClassifyWorkerFactory.obj
 0002:000080cc       __ehfuncinfo$??0?$QList@PAVDNATranslation@U2@@@@QAE@ABV0@@Z 100290cc     DiamondClassifyWorkerFactory.obj
 0002:000080f0       __catchsym$?append@?$QList@U?$QPair@VQString@@VQVariant@@@@@@QAEXABU?$QPair@VQString@@VQVariant@@@@@Z$7 100290f0     DiamondClassifyWorkerFactory.obj
 0002:00008100       __catchsym$?append@?$QList@U?$QPair@VQString@@VQVariant@@@@@@QAEXABU?$QPair@VQString@@VQVariant@@@@@Z$6 10029100     DiamondClassifyWorkerFactory.obj
 0002:00008110       __ehfuncinfo$?append@?$QList@U?$QPair@VQString@@VQVariant@@@@@@QAEXABU?$QPair@VQString@@VQVariant@@@@@Z 10029110     DiamondClassifyWorkerFactory.obj
 0002:00008134       __tryblocktable$?append@?$QList@U?$QPair@VQString@@VQVariant@@@@@@QAEXABU?$QPair@VQString@@VQVariant@@@@@Z 10029134     DiamondClassifyWorkerFactory.obj
 0002:0000815c       __unwindtable$?append@?$QList@U?$QPair@VQString@@VQVariant@@@@@@QAEXABU?$QPair@VQString@@VQVariant@@@@@Z 1002915c     DiamondClassifyWorkerFactory.obj
 0002:0000818c       __catchsym$?detach_helper_grow@?$QList@U?$QPair@VQString@@VQVariant@@@@@@AAEPAUNode@1@HH@Z$5 1002918c     DiamondClassifyWorkerFactory.obj
 0002:0000819c       __catchsym$?detach_helper_grow@?$QList@U?$QPair@VQString@@VQVariant@@@@@@AAEPAUNode@1@HH@Z$4 1002919c     DiamondClassifyWorkerFactory.obj
 0002:000081ac       __unwindtable$?detach_helper_grow@?$QList@U?$QPair@VQString@@VQVariant@@@@@@AAEPAUNode@1@HH@Z 100291ac     DiamondClassifyWorkerFactory.obj
 0002:000081cc       __ehfuncinfo$?detach_helper_grow@?$QList@U?$QPair@VQString@@VQVariant@@@@@@AAEPAUNode@1@HH@Z 100291cc     DiamondClassifyWorkerFactory.obj
 0002:000081f0       __tryblocktable$?detach_helper_grow@?$QList@U?$QPair@VQString@@VQVariant@@@@@@AAEPAUNode@1@HH@Z 100291f0     DiamondClassifyWorkerFactory.obj
 0002:00008218       __unwindtable$?node_construct@?$QList@U?$QPair@VQString@@VQVariant@@@@@@AAEXPAUNode@1@ABU?$QPair@VQString@@VQVariant@@@@@Z 10029218     DiamondClassifyWorkerFactory.obj
 0002:00008238       __ehfuncinfo$?node_construct@?$QList@U?$QPair@VQString@@VQVariant@@@@@@AAEXPAUNode@1@ABU?$QPair@VQString@@VQVariant@@@@@Z 10029238     DiamondClassifyWorkerFactory.obj
 0002:0000825c       __unwindtable$?node_destruct@?$QList@U?$QPair@VQString@@VQVariant@@@@@@AAEXPAUNode@1@@Z 1002925c     DiamondClassifyWorkerFactory.obj
 0002:0000826c       __ehfuncinfo$?node_destruct@?$QList@U?$QPair@VQString@@VQVariant@@@@@@AAEXPAUNode@1@@Z 1002926c     DiamondClassifyWorkerFactory.obj
 0002:00008290       __catchsym$?node_copy@?$QList@U?$QPair@VQString@@VQVariant@@@@@@AAEXPAUNode@1@00@Z$14 10029290     DiamondClassifyWorkerFactory.obj
 0002:000082a0       __tryblocktable$?node_copy@?$QList@U?$QPair@VQString@@VQVariant@@@@@@AAEXPAUNode@1@00@Z 100292a0     DiamondClassifyWorkerFactory.obj
 0002:000082b4       __ehfuncinfo$?node_copy@?$QList@U?$QPair@VQString@@VQVariant@@@@@@AAEXPAUNode@1@00@Z 100292b4     DiamondClassifyWorkerFactory.obj
 0002:000082d8       __unwindtable$?node_copy@?$QList@U?$QPair@VQString@@VQVariant@@@@@@AAEXPAUNode@1@00@Z 100292d8     DiamondClassifyWorkerFactory.obj
 0002:00008328       __unwindtable$?node_destruct@?$QList@U?$QPair@VQString@@VQVariant@@@@@@AAEXPAUNode@1@0@Z 10029328     DiamondClassifyWorkerFactory.obj
 0002:00008338       __ehfuncinfo$?node_destruct@?$QList@U?$QPair@VQString@@VQVariant@@@@@@AAEXPAUNode@1@0@Z 10029338     DiamondClassifyWorkerFactory.obj
 0002:0000835c       __unwindtable$??0?$QPair@VQString@@V1@@@QAE@ABVQString@@0@Z 1002935c     DiamondClassifyWorkerFactory.obj
 0002:00008364       __ehfuncinfo$??0?$QPair@VQString@@V1@@@QAE@ABVQString@@0@Z 10029364     DiamondClassifyWorkerFactory.obj
 0002:00008388       __unwindtable$??1?$QPair@VQString@@V1@@@QAE@XZ 10029388     DiamondClassifyWorkerFactory.obj
 0002:00008390       __ehfuncinfo$??1?$QPair@VQString@@V1@@@QAE@XZ 10029390     DiamondClassifyWorkerFactory.obj
 0002:000083b4       __unwindtable$??0?$QPair@VQString@@V1@@@QAE@ABU0@@Z 100293b4     DiamondClassifyWorkerFactory.obj
 0002:000083bc       __ehfuncinfo$??0?$QPair@VQString@@V1@@@QAE@ABU0@@Z 100293bc     DiamondClassifyWorkerFactory.obj
 0002:000083e0       __unwindtable$??_G?$QPair@VQString@@V1@@@QAEPAXI@Z 100293e0     DiamondClassifyWorkerFactory.obj
 0002:000083e8       __ehfuncinfo$??_G?$QPair@VQString@@V1@@@QAEPAXI@Z 100293e8     DiamondClassifyWorkerFactory.obj
 0002:0000840c       __unwindtable$?createWorker@DiamondClassifyWorkerFactory@LocalWorkflow@U2@@UAEPAVWorker@Workflow@3@PAVActor@53@@Z 1002940c     DiamondClassifyWorkerFactory.obj
 0002:00008414       __ehfuncinfo$?createWorker@DiamondClassifyWorkerFactory@LocalWorkflow@U2@@UAEPAVWorker@Workflow@3@PAVActor@53@@Z 10029414     DiamondClassifyWorkerFactory.obj
 0002:00008438       __ehfuncinfo$?init@DiamondClassifyWorkerFactory@LocalWorkflow@U2@@SAXXZ 10029438     DiamondClassifyWorkerFactory.obj
 0002:0000845c       __unwindtable$?init@DiamondClassifyWorkerFactory@LocalWorkflow@U2@@SAXXZ 1002945c     DiamondClassifyWorkerFactory.obj
 0002:00008d84       __catchsym$?append@?$QList@U?$QPair@VQString@@V1@@@@@QAEXABU?$QPair@VQString@@V1@@@@Z$7 10029d84     DiamondClassifyWorkerFactory.obj
 0002:00008d94       __catchsym$?append@?$QList@U?$QPair@VQString@@V1@@@@@QAEXABU?$QPair@VQString@@V1@@@@Z$6 10029d94     DiamondClassifyWorkerFactory.obj
 0002:00008da4       __ehfuncinfo$?append@?$QList@U?$QPair@VQString@@V1@@@@@QAEXABU?$QPair@VQString@@V1@@@@Z 10029da4     DiamondClassifyWorkerFactory.obj
 0002:00008dc8       __tryblocktable$?append@?$QList@U?$QPair@VQString@@V1@@@@@QAEXABU?$QPair@VQString@@V1@@@@Z 10029dc8     DiamondClassifyWorkerFactory.obj
 0002:00008df0       __unwindtable$?append@?$QList@U?$QPair@VQString@@V1@@@@@QAEXABU?$QPair@VQString@@V1@@@@Z 10029df0     DiamondClassifyWorkerFactory.obj
 0002:00008e20       __catchsym$?detach_helper_grow@?$QList@U?$QPair@VQString@@V1@@@@@AAEPAUNode@1@HH@Z$5 10029e20     DiamondClassifyWorkerFactory.obj
 0002:00008e30       __catchsym$?detach_helper_grow@?$QList@U?$QPair@VQString@@V1@@@@@AAEPAUNode@1@HH@Z$4 10029e30     DiamondClassifyWorkerFactory.obj
 0002:00008e40       __unwindtable$?detach_helper_grow@?$QList@U?$QPair@VQString@@V1@@@@@AAEPAUNode@1@HH@Z 10029e40     DiamondClassifyWorkerFactory.obj
 0002:00008e60       __ehfuncinfo$?detach_helper_grow@?$QList@U?$QPair@VQString@@V1@@@@@AAEPAUNode@1@HH@Z 10029e60     DiamondClassifyWorkerFactory.obj
 0002:00008e84       __tryblocktable$?detach_helper_grow@?$QList@U?$QPair@VQString@@V1@@@@@AAEPAUNode@1@HH@Z 10029e84     DiamondClassifyWorkerFactory.obj
 0002:00008eac       __unwindtable$?node_construct@?$QList@U?$QPair@VQString@@V1@@@@@AAEXPAUNode@1@ABU?$QPair@VQString@@V1@@@@Z 10029eac     DiamondClassifyWorkerFactory.obj
 0002:00008ecc       __ehfuncinfo$?node_construct@?$QList@U?$QPair@VQString@@V1@@@@@AAEXPAUNode@1@ABU?$QPair@VQString@@V1@@@@Z 10029ecc     DiamondClassifyWorkerFactory.obj
 0002:00008ef0       __unwindtable$?node_destruct@?$QList@U?$QPair@VQString@@V1@@@@@AAEXPAUNode@1@@Z 10029ef0     DiamondClassifyWorkerFactory.obj
 0002:00008f00       __ehfuncinfo$?node_destruct@?$QList@U?$QPair@VQString@@V1@@@@@AAEXPAUNode@1@@Z 10029f00     DiamondClassifyWorkerFactory.obj
 0002:00008f24       __catchsym$?node_copy@?$QList@U?$QPair@VQString@@V1@@@@@AAEXPAUNode@1@00@Z$14 10029f24     DiamondClassifyWorkerFactory.obj
 0002:00008f34       __tryblocktable$?node_copy@?$QList@U?$QPair@VQString@@V1@@@@@AAEXPAUNode@1@00@Z 10029f34     DiamondClassifyWorkerFactory.obj
 0002:00008f48       __ehfuncinfo$?node_copy@?$QList@U?$QPair@VQString@@V1@@@@@AAEXPAUNode@1@00@Z 10029f48     DiamondClassifyWorkerFactory.obj
 0002:00008f6c       __unwindtable$?node_copy@?$QList@U?$QPair@VQString@@V1@@@@@AAEXPAUNode@1@00@Z 10029f6c     DiamondClassifyWorkerFactory.obj
 0002:00008fbc       __unwindtable$?node_destruct@?$QList@U?$QPair@VQString@@V1@@@@@AAEXPAUNode@1@0@Z 10029fbc     DiamondClassifyWorkerFactory.obj
 0002:00008fcc       __ehfuncinfo$?node_destruct@?$QList@U?$QPair@VQString@@V1@@@@@AAEXPAUNode@1@0@Z 10029fcc     DiamondClassifyWorkerFactory.obj
 0002:00008ff0       __unwindtable$??1?$QPair@VQString@@VQVariant@@@@QAE@XZ 10029ff0     DiamondClassifyWorkerFactory.obj
 0002:00008ff8       __ehfuncinfo$??1?$QPair@VQString@@VQVariant@@@@QAE@XZ 10029ff8     DiamondClassifyWorkerFactory.obj
 0002:0000901c       __unwindtable$??0?$QPair@VQString@@VQVariant@@@@QAE@ABU0@@Z 1002a01c     DiamondClassifyWorkerFactory.obj
 0002:00009024       __ehfuncinfo$??0?$QPair@VQString@@VQVariant@@@@QAE@ABU0@@Z 1002a024     DiamondClassifyWorkerFactory.obj
 0002:00009048       __unwindtable$??_G?$QPair@VQString@@VQVariant@@@@QAEPAXI@Z 1002a048     DiamondClassifyWorkerFactory.obj
 0002:00009050       __ehfuncinfo$??_G?$QPair@VQString@@VQVariant@@@@QAEPAXI@Z 1002a050     DiamondClassifyWorkerFactory.obj
 0002:00009074       __unwindtable$??$?0VQString@@H@?$QPair@VQString@@VQVariant@@@@QAE@$$QAU?$QPair@VQString@@H@@@Z 1002a074     DiamondClassifyWorkerFactory.obj
 0002:0000907c       __ehfuncinfo$??$?0VQString@@H@?$QPair@VQString@@VQVariant@@@@QAE@$$QAU?$QPair@VQString@@H@@@Z 1002a07c     DiamondClassifyWorkerFactory.obj
 0002:000090a0       __unwindtable$??$qMakePair@VQString@@V1@@@YA?AU?$QPair@VQString@@V1@@@ABVQString@@0@Z 1002a0a0     DiamondClassifyWorkerFactory.obj
 0002:000090a8       __ehfuncinfo$??$qMakePair@VQString@@V1@@@YA?AU?$QPair@VQString@@V1@@@ABVQString@@0@Z 1002a0a8     DiamondClassifyWorkerFactory.obj
 0002:000090cc       __unwindtable$??$?0VQString@@V0@@?$QPair@VQString@@VQVariant@@@@QAE@$$QAU?$QPair@VQString@@V1@@@@Z 1002a0cc     DiamondClassifyWorkerFactory.obj
 0002:000090d4       __ehfuncinfo$??$?0VQString@@V0@@?$QPair@VQString@@VQVariant@@@@QAE@$$QAU?$QPair@VQString@@V1@@@@Z 1002a0d4     DiamondClassifyWorkerFactory.obj
 0002:000090f8       __ehfuncinfo$??0DiamondSupport@U2@@QAE@ABVQString@@@Z 1002a0f8     DiamondSupport.obj
 0002:0000911c       __unwindtable$??0DiamondSupport@U2@@QAE@ABVQString@@@Z 1002a11c     DiamondSupport.obj
 0002:0000914c       __unwindtable$??__EalgoLog@U2@@YAXXZ 1002a14c     DiamondSupportPlugin.obj
 0002:00009154       __ehfuncinfo$??__EalgoLog@U2@@YAXXZ 1002a154     DiamondSupportPlugin.obj
 0002:00009178       __unwindtable$??__EcmdLog@U2@@YAXXZ 1002a178     DiamondSupportPlugin.obj
 0002:00009180       __ehfuncinfo$??__EcmdLog@U2@@YAXXZ 1002a180     DiamondSupportPlugin.obj
 0002:000091a4       __unwindtable$??__EcoreLog@U2@@YAXXZ 1002a1a4     DiamondSupportPlugin.obj
 0002:000091ac       __ehfuncinfo$??__EcoreLog@U2@@YAXXZ 1002a1ac     DiamondSupportPlugin.obj
 0002:000091d0       __unwindtable$??__EioLog@U2@@YAXXZ 1002a1d0     DiamondSupportPlugin.obj
 0002:000091d8       __ehfuncinfo$??__EioLog@U2@@YAXXZ 1002a1d8     DiamondSupportPlugin.obj
 0002:000091fc       __unwindtable$??__EperfLog@U2@@YAXXZ 1002a1fc     DiamondSupportPlugin.obj
 0002:00009204       __ehfuncinfo$??__EperfLog@U2@@YAXXZ 1002a204     DiamondSupportPlugin.obj
 0002:00009228       __unwindtable$??__EscriptLog@U2@@YAXXZ 1002a228     DiamondSupportPlugin.obj
 0002:00009230       __ehfuncinfo$??__EscriptLog@U2@@YAXXZ 1002a230     DiamondSupportPlugin.obj
 0002:00009254       __unwindtable$??__EtaskLog@U2@@YAXXZ 1002a254     DiamondSupportPlugin.obj
 0002:0000925c       __ehfuncinfo$??__EtaskLog@U2@@YAXXZ 1002a25c     DiamondSupportPlugin.obj
 0002:00009280       __unwindtable$??__EuiLog@U2@@YAXXZ 1002a280     DiamondSupportPlugin.obj
 0002:00009288       __ehfuncinfo$??__EuiLog@U2@@YAXXZ 1002a288     DiamondSupportPlugin.obj
 0002:000092ac       __unwindtable$??__EuserActLog@U2@@YAXXZ 1002a2ac     DiamondSupportPlugin.obj
 0002:000092b4       __ehfuncinfo$??__EuserActLog@U2@@YAXXZ 1002a2b4     DiamondSupportPlugin.obj
 0002:000092d8       __unwindtable$??0DiamondSupportPlugin@U2@@QAE@XZ 1002a2d8     DiamondSupportPlugin.obj
 0002:000092e8       __ehfuncinfo$??0DiamondSupportPlugin@U2@@QAE@XZ 1002a2e8     DiamondSupportPlugin.obj
 0002:0000930c       __unwindtable$??1DiamondSupportPlugin@U2@@UAE@XZ 1002a30c     DiamondSupportPlugin.obj
 0002:00009314       __ehfuncinfo$??1DiamondSupportPlugin@U2@@UAE@XZ 1002a314     DiamondSupportPlugin.obj
 0002:00009338       __unwindtable$??_GDiamondSupportPlugin@U2@@UAEPAXI@Z 1002a338     DiamondSupportPlugin.obj
 0002:00009340       __ehfuncinfo$??_GDiamondSupportPlugin@U2@@UAEPAXI@Z 1002a340     DiamondSupportPlugin.obj
 0002:00009364       __unwindtable$??__EalgoLog@U2@@YAXXZ 1002a364     GenomesPreparationTask.obj
 0002:0000936c       __ehfuncinfo$??__EalgoLog@U2@@YAXXZ 1002a36c     GenomesPreparationTask.obj
 0002:00009390       __unwindtable$??__EcmdLog@U2@@YAXXZ 1002a390     GenomesPreparationTask.obj
 0002:00009398       __ehfuncinfo$??__EcmdLog@U2@@YAXXZ 1002a398     GenomesPreparationTask.obj
 0002:000093bc       __unwindtable$??__EcoreLog@U2@@YAXXZ 1002a3bc     GenomesPreparationTask.obj
 0002:000093c4       __ehfuncinfo$??__EcoreLog@U2@@YAXXZ 1002a3c4     GenomesPreparationTask.obj
 0002:000093e8       __unwindtable$??__EioLog@U2@@YAXXZ 1002a3e8     GenomesPreparationTask.obj
 0002:000093f0       __ehfuncinfo$??__EioLog@U2@@YAXXZ 1002a3f0     GenomesPreparationTask.obj
 0002:00009414       __unwindtable$??__EperfLog@U2@@YAXXZ 1002a414     GenomesPreparationTask.obj
 0002:0000941c       __ehfuncinfo$??__EperfLog@U2@@YAXXZ 1002a41c     GenomesPreparationTask.obj
 0002:00009440       __unwindtable$??__EscriptLog@U2@@YAXXZ 1002a440     GenomesPreparationTask.obj
 0002:00009448       __ehfuncinfo$??__EscriptLog@U2@@YAXXZ 1002a448     GenomesPreparationTask.obj
 0002:0000946c       __unwindtable$??__EtaskLog@U2@@YAXXZ 1002a46c     GenomesPreparationTask.obj
 0002:00009474       __ehfuncinfo$??__EtaskLog@U2@@YAXXZ 1002a474     GenomesPreparationTask.obj
 0002:00009498       __unwindtable$??__EuiLog@U2@@YAXXZ 1002a498     GenomesPreparationTask.obj
 0002:000094a0       __ehfuncinfo$??__EuiLog@U2@@YAXXZ 1002a4a0     GenomesPreparationTask.obj
 0002:000094c4       __unwindtable$??__EuserActLog@U2@@YAXXZ 1002a4c4     GenomesPreparationTask.obj
 0002:000094cc       __ehfuncinfo$??__EuserActLog@U2@@YAXXZ 1002a4cc     GenomesPreparationTask.obj
 0002:000094f0       __ehfuncinfo$??0GenomesPreparationTask@U2@@QAE@ABVQStringList@@ABVQString@@@Z 1002a4f0     GenomesPreparationTask.obj
 0002:00009514       __unwindtable$??0GenomesPreparationTask@U2@@QAE@ABVQStringList@@ABVQString@@@Z 1002a514     GenomesPreparationTask.obj
 0002:0000954c       __ehfuncinfo$?run@GenomesPreparationTask@U2@@EAEXXZ 1002a54c     GenomesPreparationTask.obj
 0002:00009570       __unwindtable$?run@GenomesPreparationTask@U2@@EAEXXZ 1002a570     GenomesPreparationTask.obj
 0002:000095b8       __unwindtable$??1GenomesPreparationTask@U2@@UAE@XZ 1002a5b8     GenomesPreparationTask.obj
 0002:000095c8       __ehfuncinfo$??1GenomesPreparationTask@U2@@UAE@XZ 1002a5c8     GenomesPreparationTask.obj
 0002:000095ec       __unwindtable$??_GGenomesPreparationTask@U2@@UAEPAXI@Z 1002a5ec     GenomesPreparationTask.obj
 0002:000095fc       __ehfuncinfo$??_GGenomesPreparationTask@U2@@UAEPAXI@Z 1002a5fc     GenomesPreparationTask.obj
 0002:00009620       __unwindtable$??__EalgoLog@U2@@YAXXZ 1002a620     moc_DiamondBuildPrompter.obj
 0002:00009628       __ehfuncinfo$??__EalgoLog@U2@@YAXXZ 1002a628     moc_DiamondBuildPrompter.obj
 0002:0000964c       __unwindtable$??__EcmdLog@U2@@YAXXZ 1002a64c     moc_DiamondBuildPrompter.obj
 0002:00009654       __ehfuncinfo$??__EcmdLog@U2@@YAXXZ 1002a654     moc_DiamondBuildPrompter.obj
 0002:00009678       __unwindtable$??__EcoreLog@U2@@YAXXZ 1002a678     moc_DiamondBuildPrompter.obj
 0002:00009680       __ehfuncinfo$??__EcoreLog@U2@@YAXXZ 1002a680     moc_DiamondBuildPrompter.obj
 0002:000096a4       __unwindtable$??__EioLog@U2@@YAXXZ 1002a6a4     moc_DiamondBuildPrompter.obj
 0002:000096ac       __ehfuncinfo$??__EioLog@U2@@YAXXZ 1002a6ac     moc_DiamondBuildPrompter.obj
 0002:000096d0       __unwindtable$??__EperfLog@U2@@YAXXZ 1002a6d0     moc_DiamondBuildPrompter.obj
 0002:000096d8       __ehfuncinfo$??__EperfLog@U2@@YAXXZ 1002a6d8     moc_DiamondBuildPrompter.obj
 0002:000096fc       __unwindtable$??__EscriptLog@U2@@YAXXZ 1002a6fc     moc_DiamondBuildPrompter.obj
 0002:00009704       __ehfuncinfo$??__EscriptLog@U2@@YAXXZ 1002a704     moc_DiamondBuildPrompter.obj
 0002:00009728       __unwindtable$??__EtaskLog@U2@@YAXXZ 1002a728     moc_DiamondBuildPrompter.obj
 0002:00009730       __ehfuncinfo$??__EtaskLog@U2@@YAXXZ 1002a730     moc_DiamondBuildPrompter.obj
 0002:00009754       __unwindtable$??__EuiLog@U2@@YAXXZ 1002a754     moc_DiamondBuildPrompter.obj
 0002:0000975c       __ehfuncinfo$??__EuiLog@U2@@YAXXZ 1002a75c     moc_DiamondBuildPrompter.obj
 0002:00009780       __unwindtable$??__EuserActLog@U2@@YAXXZ 1002a780     moc_DiamondBuildPrompter.obj
 0002:00009788       __ehfuncinfo$??__EuserActLog@U2@@YAXXZ 1002a788     moc_DiamondBuildPrompter.obj
 0002:000097ac       __unwindtable$??__EalgoLog@U2@@YAXXZ 1002a7ac     moc_DiamondBuildTask.obj
 0002:000097b4       __ehfuncinfo$??__EalgoLog@U2@@YAXXZ 1002a7b4     moc_DiamondBuildTask.obj
 0002:000097d8       __unwindtable$??__EcmdLog@U2@@YAXXZ 1002a7d8     moc_DiamondBuildTask.obj
 0002:000097e0       __ehfuncinfo$??__EcmdLog@U2@@YAXXZ 1002a7e0     moc_DiamondBuildTask.obj
 0002:00009804       __unwindtable$??__EcoreLog@U2@@YAXXZ 1002a804     moc_DiamondBuildTask.obj
 0002:0000980c       __ehfuncinfo$??__EcoreLog@U2@@YAXXZ 1002a80c     moc_DiamondBuildTask.obj
 0002:00009830       __unwindtable$??__EioLog@U2@@YAXXZ 1002a830     moc_DiamondBuildTask.obj
 0002:00009838       __ehfuncinfo$??__EioLog@U2@@YAXXZ 1002a838     moc_DiamondBuildTask.obj
 0002:0000985c       __unwindtable$??__EperfLog@U2@@YAXXZ 1002a85c     moc_DiamondBuildTask.obj
 0002:00009864       __ehfuncinfo$??__EperfLog@U2@@YAXXZ 1002a864     moc_DiamondBuildTask.obj
 0002:00009888       __unwindtable$??__EscriptLog@U2@@YAXXZ 1002a888     moc_DiamondBuildTask.obj
 0002:00009890       __ehfuncinfo$??__EscriptLog@U2@@YAXXZ 1002a890     moc_DiamondBuildTask.obj
 0002:000098b4       __unwindtable$??__EtaskLog@U2@@YAXXZ 1002a8b4     moc_DiamondBuildTask.obj
 0002:000098bc       __ehfuncinfo$??__EtaskLog@U2@@YAXXZ 1002a8bc     moc_DiamondBuildTask.obj
 0002:000098e0       __unwindtable$??__EuiLog@U2@@YAXXZ 1002a8e0     moc_DiamondBuildTask.obj
 0002:000098e8       __ehfuncinfo$??__EuiLog@U2@@YAXXZ 1002a8e8     moc_DiamondBuildTask.obj
 0002:0000990c       __unwindtable$??__EuserActLog@U2@@YAXXZ 1002a90c     moc_DiamondBuildTask.obj
 0002:00009914       __ehfuncinfo$??__EuserActLog@U2@@YAXXZ 1002a914     moc_DiamondBuildTask.obj
 0002:00009938       __unwindtable$??__EalgoLog@U2@@YAXXZ 1002a938     moc_DiamondBuildWorker.obj
 0002:00009940       __ehfuncinfo$??__EalgoLog@U2@@YAXXZ 1002a940     moc_DiamondBuildWorker.obj
 0002:00009964       __unwindtable$??__EcmdLog@U2@@YAXXZ 1002a964     moc_DiamondBuildWorker.obj
 0002:0000996c       __ehfuncinfo$??__EcmdLog@U2@@YAXXZ 1002a96c     moc_DiamondBuildWorker.obj
 0002:00009990       __unwindtable$??__EcoreLog@U2@@YAXXZ 1002a990     moc_DiamondBuildWorker.obj
 0002:00009998       __ehfuncinfo$??__EcoreLog@U2@@YAXXZ 1002a998     moc_DiamondBuildWorker.obj
 0002:000099bc       __unwindtable$??__EioLog@U2@@YAXXZ 1002a9bc     moc_DiamondBuildWorker.obj
 0002:000099c4       __ehfuncinfo$??__EioLog@U2@@YAXXZ 1002a9c4     moc_DiamondBuildWorker.obj
 0002:000099e8       __unwindtable$??__EperfLog@U2@@YAXXZ 1002a9e8     moc_DiamondBuildWorker.obj
 0002:000099f0       __ehfuncinfo$??__EperfLog@U2@@YAXXZ 1002a9f0     moc_DiamondBuildWorker.obj
 0002:00009a14       __unwindtable$??__EscriptLog@U2@@YAXXZ 1002aa14     moc_DiamondBuildWorker.obj
 0002:00009a1c       __ehfuncinfo$??__EscriptLog@U2@@YAXXZ 1002aa1c     moc_DiamondBuildWorker.obj
 0002:00009a40       __unwindtable$??__EtaskLog@U2@@YAXXZ 1002aa40     moc_DiamondBuildWorker.obj
 0002:00009a48       __ehfuncinfo$??__EtaskLog@U2@@YAXXZ 1002aa48     moc_DiamondBuildWorker.obj
 0002:00009a6c       __unwindtable$??__EuiLog@U2@@YAXXZ 1002aa6c     moc_DiamondBuildWorker.obj
 0002:00009a74       __ehfuncinfo$??__EuiLog@U2@@YAXXZ 1002aa74     moc_DiamondBuildWorker.obj
 0002:00009a98       __unwindtable$??__EuserActLog@U2@@YAXXZ 1002aa98     moc_DiamondBuildWorker.obj
 0002:00009aa0       __ehfuncinfo$??__EuserActLog@U2@@YAXXZ 1002aaa0     moc_DiamondBuildWorker.obj
 0002:00009ac4       __unwindtable$?qt_metatype_id@?$QMetaTypeIdQObject@PAVTask@U2@@$00@@SAHXZ 1002aac4     moc_DiamondBuildWorker.obj
 0002:00009acc       __ehfuncinfo$?qt_metatype_id@?$QMetaTypeIdQObject@PAVTask@U2@@$00@@SAHXZ 1002aacc     moc_DiamondBuildWorker.obj
 0002:00009af0       __unwindtable$??__EalgoLog@U2@@YAXXZ 1002aaf0     moc_DiamondClassifyPrompter.obj
 0002:00009af8       __ehfuncinfo$??__EalgoLog@U2@@YAXXZ 1002aaf8     moc_DiamondClassifyPrompter.obj
 0002:00009b1c       __unwindtable$??__EcmdLog@U2@@YAXXZ 1002ab1c     moc_DiamondClassifyPrompter.obj
 0002:00009b24       __ehfuncinfo$??__EcmdLog@U2@@YAXXZ 1002ab24     moc_DiamondClassifyPrompter.obj
 0002:00009b48       __unwindtable$??__EcoreLog@U2@@YAXXZ 1002ab48     moc_DiamondClassifyPrompter.obj
 0002:00009b50       __ehfuncinfo$??__EcoreLog@U2@@YAXXZ 1002ab50     moc_DiamondClassifyPrompter.obj
 0002:00009b74       __unwindtable$??__EioLog@U2@@YAXXZ 1002ab74     moc_DiamondClassifyPrompter.obj
 0002:00009b7c       __ehfuncinfo$??__EioLog@U2@@YAXXZ 1002ab7c     moc_DiamondClassifyPrompter.obj
 0002:00009ba0       __unwindtable$??__EperfLog@U2@@YAXXZ 1002aba0     moc_DiamondClassifyPrompter.obj
 0002:00009ba8       __ehfuncinfo$??__EperfLog@U2@@YAXXZ 1002aba8     moc_DiamondClassifyPrompter.obj
 0002:00009bcc       __unwindtable$??__EscriptLog@U2@@YAXXZ 1002abcc     moc_DiamondClassifyPrompter.obj
 0002:00009bd4       __ehfuncinfo$??__EscriptLog@U2@@YAXXZ 1002abd4     moc_DiamondClassifyPrompter.obj
 0002:00009bf8       __unwindtable$??__EtaskLog@U2@@YAXXZ 1002abf8     moc_DiamondClassifyPrompter.obj
 0002:00009c00       __ehfuncinfo$??__EtaskLog@U2@@YAXXZ 1002ac00     moc_DiamondClassifyPrompter.obj
 0002:00009c24       __unwindtable$??__EuiLog@U2@@YAXXZ 1002ac24     moc_DiamondClassifyPrompter.obj
 0002:00009c2c       __ehfuncinfo$??__EuiLog@U2@@YAXXZ 1002ac2c     moc_DiamondClassifyPrompter.obj
 0002:00009c50       __unwindtable$??__EuserActLog@U2@@YAXXZ 1002ac50     moc_DiamondClassifyPrompter.obj
 0002:00009c58       __ehfuncinfo$??__EuserActLog@U2@@YAXXZ 1002ac58     moc_DiamondClassifyPrompter.obj
 0002:00009c7c       __unwindtable$??__EalgoLog@U2@@YAXXZ 1002ac7c     moc_DiamondClassifyTask.obj
 0002:00009c84       __ehfuncinfo$??__EalgoLog@U2@@YAXXZ 1002ac84     moc_DiamondClassifyTask.obj
 0002:00009ca8       __unwindtable$??__EcmdLog@U2@@YAXXZ 1002aca8     moc_DiamondClassifyTask.obj
 0002:00009cb0       __ehfuncinfo$??__EcmdLog@U2@@YAXXZ 1002acb0     moc_DiamondClassifyTask.obj
 0002:00009cd4       __unwindtable$??__EcoreLog@U2@@YAXXZ 1002acd4     moc_DiamondClassifyTask.obj
 0002:00009cdc       __ehfuncinfo$??__EcoreLog@U2@@YAXXZ 1002acdc     moc_DiamondClassifyTask.obj
 0002:00009d00       __unwindtable$??__EioLog@U2@@YAXXZ 1002ad00     moc_DiamondClassifyTask.obj
 0002:00009d08       __ehfuncinfo$??__EioLog@U2@@YAXXZ 1002ad08     moc_DiamondClassifyTask.obj
 0002:00009d2c       __unwindtable$??__EperfLog@U2@@YAXXZ 1002ad2c     moc_DiamondClassifyTask.obj
 0002:00009d34       __ehfuncinfo$??__EperfLog@U2@@YAXXZ 1002ad34     moc_DiamondClassifyTask.obj
 0002:00009d58       __unwindtable$??__EscriptLog@U2@@YAXXZ 1002ad58     moc_DiamondClassifyTask.obj
 0002:00009d60       __ehfuncinfo$??__EscriptLog@U2@@YAXXZ 1002ad60     moc_DiamondClassifyTask.obj
 0002:00009d84       __unwindtable$??__EtaskLog@U2@@YAXXZ 1002ad84     moc_DiamondClassifyTask.obj
 0002:00009d8c       __ehfuncinfo$??__EtaskLog@U2@@YAXXZ 1002ad8c     moc_DiamondClassifyTask.obj
 0002:00009db0       __unwindtable$??__EuiLog@U2@@YAXXZ 1002adb0     moc_DiamondClassifyTask.obj
 0002:00009db8       __ehfuncinfo$??__EuiLog@U2@@YAXXZ 1002adb8     moc_DiamondClassifyTask.obj
 0002:00009ddc       __unwindtable$??__EuserActLog@U2@@YAXXZ 1002addc     moc_DiamondClassifyTask.obj
 0002:00009de4       __ehfuncinfo$??__EuserActLog@U2@@YAXXZ 1002ade4     moc_DiamondClassifyTask.obj
 0002:00009e08       __unwindtable$??__EalgoLog@U2@@YAXXZ 1002ae08     moc_DiamondClassifyWorker.obj
 0002:00009e10       __ehfuncinfo$??__EalgoLog@U2@@YAXXZ 1002ae10     moc_DiamondClassifyWorker.obj
 0002:00009e34       __unwindtable$??__EcmdLog@U2@@YAXXZ 1002ae34     moc_DiamondClassifyWorker.obj
 0002:00009e3c       __ehfuncinfo$??__EcmdLog@U2@@YAXXZ 1002ae3c     moc_DiamondClassifyWorker.obj
 0002:00009e60       __unwindtable$??__EcoreLog@U2@@YAXXZ 1002ae60     moc_DiamondClassifyWorker.obj
 0002:00009e68       __ehfuncinfo$??__EcoreLog@U2@@YAXXZ 1002ae68     moc_DiamondClassifyWorker.obj
 0002:00009e8c       __unwindtable$??__EioLog@U2@@YAXXZ 1002ae8c     moc_DiamondClassifyWorker.obj
 0002:00009e94       __ehfuncinfo$??__EioLog@U2@@YAXXZ 1002ae94     moc_DiamondClassifyWorker.obj
 0002:00009eb8       __unwindtable$??__EperfLog@U2@@YAXXZ 1002aeb8     moc_DiamondClassifyWorker.obj
 0002:00009ec0       __ehfuncinfo$??__EperfLog@U2@@YAXXZ 1002aec0     moc_DiamondClassifyWorker.obj
 0002:00009ee4       __unwindtable$??__EscriptLog@U2@@YAXXZ 1002aee4     moc_DiamondClassifyWorker.obj
 0002:00009eec       __ehfuncinfo$??__EscriptLog@U2@@YAXXZ 1002aeec     moc_DiamondClassifyWorker.obj
 0002:00009f10       __unwindtable$??__EtaskLog@U2@@YAXXZ 1002af10     moc_DiamondClassifyWorker.obj
 0002:00009f18       __ehfuncinfo$??__EtaskLog@U2@@YAXXZ 1002af18     moc_DiamondClassifyWorker.obj
 0002:00009f3c       __unwindtable$??__EuiLog@U2@@YAXXZ 1002af3c     moc_DiamondClassifyWorker.obj
 0002:00009f44       __ehfuncinfo$??__EuiLog@U2@@YAXXZ 1002af44     moc_DiamondClassifyWorker.obj
 0002:00009f68       __unwindtable$??__EuserActLog@U2@@YAXXZ 1002af68     moc_DiamondClassifyWorker.obj
 0002:00009f70       __ehfuncinfo$??__EuserActLog@U2@@YAXXZ 1002af70     moc_DiamondClassifyWorker.obj
 0002:00009f94       __unwindtable$??__EalgoLog@U2@@YAXXZ 1002af94     moc_GenomesPreparationTask.obj
 0002:00009f9c       __ehfuncinfo$??__EalgoLog@U2@@YAXXZ 1002af9c     moc_GenomesPreparationTask.obj
 0002:00009fc0       __unwindtable$??__EcmdLog@U2@@YAXXZ 1002afc0     moc_GenomesPreparationTask.obj
 0002:00009fc8       __ehfuncinfo$??__EcmdLog@U2@@YAXXZ 1002afc8     moc_GenomesPreparationTask.obj
 0002:00009fec       __unwindtable$??__EcoreLog@U2@@YAXXZ 1002afec     moc_GenomesPreparationTask.obj
 0002:00009ff4       __ehfuncinfo$??__EcoreLog@U2@@YAXXZ 1002aff4     moc_GenomesPreparationTask.obj
 0002:0000a018       __unwindtable$??__EioLog@U2@@YAXXZ 1002b018     moc_GenomesPreparationTask.obj
 0002:0000a020       __ehfuncinfo$??__EioLog@U2@@YAXXZ 1002b020     moc_GenomesPreparationTask.obj
 0002:0000a044       __unwindtable$??__EperfLog@U2@@YAXXZ 1002b044     moc_GenomesPreparationTask.obj
 0002:0000a04c       __ehfuncinfo$??__EperfLog@U2@@YAXXZ 1002b04c     moc_GenomesPreparationTask.obj
 0002:0000a070       __unwindtable$??__EscriptLog@U2@@YAXXZ 1002b070     moc_GenomesPreparationTask.obj
 0002:0000a078       __ehfuncinfo$??__EscriptLog@U2@@YAXXZ 1002b078     moc_GenomesPreparationTask.obj
 0002:0000a09c       __unwindtable$??__EtaskLog@U2@@YAXXZ 1002b09c     moc_GenomesPreparationTask.obj
 0002:0000a0a4       __ehfuncinfo$??__EtaskLog@U2@@YAXXZ 1002b0a4     moc_GenomesPreparationTask.obj
 0002:0000a0c8       __unwindtable$??__EuiLog@U2@@YAXXZ 1002b0c8     moc_GenomesPreparationTask.obj
 0002:0000a0d0       __ehfuncinfo$??__EuiLog@U2@@YAXXZ 1002b0d0     moc_GenomesPreparationTask.obj
 0002:0000a0f4       __unwindtable$??__EuserActLog@U2@@YAXXZ 1002b0f4     moc_GenomesPreparationTask.obj
 0002:0000a0fc       __ehfuncinfo$??__EuserActLog@U2@@YAXXZ 1002b0fc     moc_GenomesPreparationTask.obj
 0002:0000a120       __sehtable$__onexit        1002b120     MSVCRT:atonexit.obj
 0002:0000a140       __sehtable$___DllMainCRTStartup 1002b140     MSVCRT:crtdll.obj
 0002:0000a168       __sehtable$??_M@YGXPAXIHP6EX0@Z@Z 1002b168     MSVCRT:ehvecdtr.obj
 0002:0000a188       __sehtable$?__ArrayUnwind@@YGXPAXIHP6EX0@Z@Z 1002b188     MSVCRT:ehvecdtr.obj
 0002:0000a1a8       __sehtable$__IsNonwritableInCurrentImage 1002b1a8     MSVCRT:pesect.obj
 0002:0000a1d0       .edata                     1002b1d0     diamond_support.exp
 0002:0000a1f8       rgpv                       1002b1f8     diamond_support.exp
 0002:0000a1fc       rgszName                   1002b1fc     diamond_support.exp
 0002:0000a200       rgwOrd                     1002b200     diamond_support.exp
 0002:0000a202       szName                     1002b202     diamond_support.exp
 0002:0000a216       $N00001                    1002b216     diamond_support.exp
 0002:0000b4bc       .idata$6                   1002c4bc     ngs_reads_classification:ngs_reads_classification.dll
 0002:0000cd02       .idata$6                   1002dd02     U2Core:U2Core.dll
 0002:0000cf46       .idata$6                   1002df46     U2Formats:U2Formats.dll
 0002:0000cff8       .idata$6                   1002dff8     U2Gui:U2Gui.dll
 0002:0000f10e       .idata$6                   1003010e     U2Lang:U2Lang.dll
 0002:000101dc       .idata$6                   100311dc     U2Designer:U2Designer.dll
 0002:0001062c       .idata$6                   1003162c     Qt5Widgets:Qt5Widgets.dll
 0002:000106de       .idata$6                   100316de     Qt5Gui:Qt5Gui.dll
 0002:00010850       .idata$6                   10031850     Qt5Script:Qt5Script.dll
 0002:00011750       .idata$6                   10032750     Qt5Core:Qt5Core.dll
 0002:000117f6       .idata$6                   100327f6     msvcprt:MSVCP120.dll
 0002:0001187a       .idata$6                   1003287a     MSVCRT:MSVCR120.dll
 0002:00011a8e       .idata$6                   10032a8e     kernel32:KERNEL32.dll
 0003:00000a60       __Tuple_alloc              10033a60     DiamondBuildPrompter.obj
 0003:00000a61       _ignore                    10033a61     DiamondBuildPrompter.obj
 0003:00000a62       _allocator_arg             10033a62     DiamondBuildPrompter.obj
 0003:00000a63       _piecewise_construct       10033a63     DiamondBuildPrompter.obj
 0003:00000a64       _taskLog                   10033a64     DiamondBuildPrompter.obj
 0003:00000a6c       _algoLog                   10033a6c     DiamondBuildPrompter.obj
 0003:00000a74       _userActLog                10033a74     DiamondBuildPrompter.obj
 0003:00000a7c       _ioLog                     10033a7c     DiamondBuildPrompter.obj
 0003:00000a84       _coreLog                   10033a84     DiamondBuildPrompter.obj
 0003:00000a8c       _uiLog                     10033a8c     DiamondBuildPrompter.obj
 0003:00000a94       _scriptLog                 10033a94     DiamondBuildPrompter.obj
 0003:00000a9c       _perfLog                   10033a9c     DiamondBuildPrompter.obj
 0003:00000aa4       _cmdLog                    10033aa4     DiamondBuildPrompter.obj
 0003:00000ab4       __Tuple_alloc              10033ab4     DiamondBuildTask.obj
 0003:00000ab5       _ignore                    10033ab5     DiamondBuildTask.obj
 0003:00000ab6       _allocator_arg             10033ab6     DiamondBuildTask.obj
 0003:00000ab7       _piecewise_construct       10033ab7     DiamondBuildTask.obj
 0003:00000ab8       _taskLog                   10033ab8     DiamondBuildTask.obj
 0003:00000ac0       _algoLog                   10033ac0     DiamondBuildTask.obj
 0003:00000ac8       _userActLog                10033ac8     DiamondBuildTask.obj
 0003:00000ad0       _ioLog                     10033ad0     DiamondBuildTask.obj
 0003:00000ad8       _coreLog                   10033ad8     DiamondBuildTask.obj
 0003:00000ae0       _uiLog                     10033ae0     DiamondBuildTask.obj
 0003:00000ae8       _scriptLog                 10033ae8     DiamondBuildTask.obj
 0003:00000af0       _perfLog                   10033af0     DiamondBuildTask.obj
 0003:00000af8       _cmdLog                    10033af8     DiamondBuildTask.obj
 0003:00000b00       ?cvar@?1???0DiamondBuildTask@U2@@QAE@ABUDiamondBuildTaskSettings@2@@Z@4VGReportableCounter@2@A 10033b00     DiamondBuildTask.obj
 0003:00000b28       ?$S1@?1???0DiamondBuildTask@U2@@QAE@ABUDiamondBuildTaskSettings@2@@Z@4IA 10033b28     DiamondBuildTask.obj
 0003:00000b2c       __Tuple_alloc              10033b2c     DiamondBuildValidator.obj
 0003:00000b2d       _ignore                    10033b2d     DiamondBuildValidator.obj
 0003:00000b2e       _allocator_arg             10033b2e     DiamondBuildValidator.obj
 0003:00000b2f       _piecewise_construct       10033b2f     DiamondBuildValidator.obj
 0003:00000b30       _taskLog                   10033b30     DiamondBuildValidator.obj
 0003:00000b38       _algoLog                   10033b38     DiamondBuildValidator.obj
 0003:00000b40       _userActLog                10033b40     DiamondBuildValidator.obj
 0003:00000b48       _ioLog                     10033b48     DiamondBuildValidator.obj
 0003:00000b50       _coreLog                   10033b50     DiamondBuildValidator.obj
 0003:00000b58       _uiLog                     10033b58     DiamondBuildValidator.obj
 0003:00000b60       _scriptLog                 10033b60     DiamondBuildValidator.obj
 0003:00000b68       _perfLog                   10033b68     DiamondBuildValidator.obj
 0003:00000b70       _cmdLog                    10033b70     DiamondBuildValidator.obj
 0003:00000b78       __Tuple_alloc              10033b78     DiamondBuildWorker.obj
 0003:00000b79       _ignore                    10033b79     DiamondBuildWorker.obj
 0003:00000b7a       _allocator_arg             10033b7a     DiamondBuildWorker.obj
 0003:00000b7b       _piecewise_construct       10033b7b     DiamondBuildWorker.obj
 0003:00000b7c       _taskLog                   10033b7c     DiamondBuildWorker.obj
 0003:00000b84       _algoLog                   10033b84     DiamondBuildWorker.obj
 0003:00000b8c       _userActLog                10033b8c     DiamondBuildWorker.obj
 0003:00000b94       _ioLog                     10033b94     DiamondBuildWorker.obj
 0003:00000b9c       _coreLog                   10033b9c     DiamondBuildWorker.obj
 0003:00000ba8       _uiLog                     10033ba8     DiamondBuildWorker.obj
 0003:00000bb0       _scriptLog                 10033bb0     DiamondBuildWorker.obj
 0003:00000bb8       _perfLog                   10033bb8     DiamondBuildWorker.obj
 0003:00000bc0       _cmdLog                    10033bc0     DiamondBuildWorker.obj
 0003:00000bcc       __Tuple_alloc              10033bcc     DiamondBuildWorkerFactory.obj
 0003:00000bcd       _ignore                    10033bcd     DiamondBuildWorkerFactory.obj
 0003:00000bce       _allocator_arg             10033bce     DiamondBuildWorkerFactory.obj
 0003:00000bcf       _piecewise_construct       10033bcf     DiamondBuildWorkerFactory.obj
 0003:00000bd0       _taskLog                   10033bd0     DiamondBuildWorkerFactory.obj
 0003:00000bd8       _algoLog                   10033bd8     DiamondBuildWorkerFactory.obj
 0003:00000be0       _userActLog                10033be0     DiamondBuildWorkerFactory.obj
 0003:00000be8       _ioLog                     10033be8     DiamondBuildWorkerFactory.obj
 0003:00000bf0       _coreLog                   10033bf0     DiamondBuildWorkerFactory.obj
 0003:00000c00       _uiLog                     10033c00     DiamondBuildWorkerFactory.obj
 0003:00000c08       _scriptLog                 10033c08     DiamondBuildWorkerFactory.obj
 0003:00000c10       _perfLog                   10033c10     DiamondBuildWorkerFactory.obj
 0003:00000c1c       _cmdLog                    10033c1c     DiamondBuildWorkerFactory.obj
 0003:00000c28       __Tuple_alloc              10033c28     DiamondClassifyPrompter.obj
 0003:00000c29       _ignore                    10033c29     DiamondClassifyPrompter.obj
 0003:00000c2a       _allocator_arg             10033c2a     DiamondClassifyPrompter.obj
 0003:00000c2b       _piecewise_construct       10033c2b     DiamondClassifyPrompter.obj
 0003:00000c2c       _taskLog                   10033c2c     DiamondClassifyPrompter.obj
 0003:00000c34       _algoLog                   10033c34     DiamondClassifyPrompter.obj
 0003:00000c3c       _userActLog                10033c3c     DiamondClassifyPrompter.obj
 0003:00000c44       _ioLog                     10033c44     DiamondClassifyPrompter.obj
 0003:00000c4c       _coreLog                   10033c4c     DiamondClassifyPrompter.obj
 0003:00000c54       _uiLog                     10033c54     DiamondClassifyPrompter.obj
 0003:00000c5c       _scriptLog                 10033c5c     DiamondClassifyPrompter.obj
 0003:00000c64       _perfLog                   10033c64     DiamondClassifyPrompter.obj
 0003:00000c6c       _cmdLog                    10033c6c     DiamondClassifyPrompter.obj
 0003:00000c74       __Tuple_alloc              10033c74     DiamondClassifyTask.obj
 0003:00000c75       _ignore                    10033c75     DiamondClassifyTask.obj
 0003:00000c76       _allocator_arg             10033c76     DiamondClassifyTask.obj
 0003:00000c77       _piecewise_construct       10033c77     DiamondClassifyTask.obj
 0003:00000c78       _taskLog                   10033c78     DiamondClassifyTask.obj
 0003:00000c84       _algoLog                   10033c84     DiamondClassifyTask.obj
 0003:00000c90       _userActLog                10033c90     DiamondClassifyTask.obj
 0003:00000c98       _ioLog                     10033c98     DiamondClassifyTask.obj
 0003:00000ca0       _coreLog                   10033ca0     DiamondClassifyTask.obj
 0003:00000cac       _uiLog                     10033cac     DiamondClassifyTask.obj
 0003:00000cb4       _scriptLog                 10033cb4     DiamondClassifyTask.obj
 0003:00000cc8       _perfLog                   10033cc8     DiamondClassifyTask.obj
 0003:00000cd8       _cmdLog                    10033cd8     DiamondClassifyTask.obj
 0003:00000cf0       ?cvar@?1???0DiamondClassifyTask@U2@@QAE@ABUDiamondClassifyTaskSettings@2@@Z@4VGReportableCounter@2@A 10033cf0     DiamondClassifyTask.obj
 0003:00000d18       ?$S1@?1???0DiamondClassifyTask@U2@@QAE@ABUDiamondClassifyTaskSettings@2@@Z@4IA 10033d18     DiamondClassifyTask.obj
 0003:00000d1c       __Tuple_alloc              10033d1c     DiamondClassifyWorker.obj
 0003:00000d1d       _ignore                    10033d1d     DiamondClassifyWorker.obj
 0003:00000d1e       _allocator_arg             10033d1e     DiamondClassifyWorker.obj
 0003:00000d1f       _piecewise_construct       10033d1f     DiamondClassifyWorker.obj
 0003:00000d20       _taskLog                   10033d20     DiamondClassifyWorker.obj
 0003:00000d28       _algoLog                   10033d28     DiamondClassifyWorker.obj
 0003:00000d30       _userActLog                10033d30     DiamondClassifyWorker.obj
 0003:00000d38       _ioLog                     10033d38     DiamondClassifyWorker.obj
 0003:00000d40       _coreLog                   10033d40     DiamondClassifyWorker.obj
 0003:00000d48       _uiLog                     10033d48     DiamondClassifyWorker.obj
 0003:00000d50       _scriptLog                 10033d50     DiamondClassifyWorker.obj
 0003:00000d58       _perfLog                   10033d58     DiamondClassifyWorker.obj
 0003:00000d60       _cmdLog                    10033d60     DiamondClassifyWorker.obj
 0003:00000d80       __Tuple_alloc              10033d80     DiamondClassifyWorkerFactory.obj
 0003:00000d81       _ignore                    10033d81     DiamondClassifyWorkerFactory.obj
 0003:00000d82       _allocator_arg             10033d82     DiamondClassifyWorkerFactory.obj
 0003:00000d83       _piecewise_construct       10033d83     DiamondClassifyWorkerFactory.obj
 0003:00000d98       _taskLog                   10033d98     DiamondClassifyWorkerFactory.obj
 0003:00000da0       _algoLog                   10033da0     DiamondClassifyWorkerFactory.obj
 0003:00000da8       _userActLog                10033da8     DiamondClassifyWorkerFactory.obj
 0003:00000db0       _ioLog                     10033db0     DiamondClassifyWorkerFactory.obj
 0003:00000db8       _coreLog                   10033db8     DiamondClassifyWorkerFactory.obj
 0003:00000dd4       _uiLog                     10033dd4     DiamondClassifyWorkerFactory.obj
 0003:00000ddc       _scriptLog                 10033ddc     DiamondClassifyWorkerFactory.obj
 0003:00000de8       _perfLog                   10033de8     DiamondClassifyWorkerFactory.obj
 0003:00000df4       _cmdLog                    10033df4     DiamondClassifyWorkerFactory.obj
 0003:00000e18       __Tuple_alloc              10033e18     DiamondSupport.obj
 0003:00000e19       _ignore                    10033e19     DiamondSupport.obj
 0003:00000e1a       _allocator_arg             10033e1a     DiamondSupport.obj
 0003:00000e1b       _piecewise_construct       10033e1b     DiamondSupport.obj
 0003:00000e20       __Tuple_alloc              10033e20     DiamondSupportPlugin.obj
 0003:00000e21       _ignore                    10033e21     DiamondSupportPlugin.obj
 0003:00000e22       _allocator_arg             10033e22     DiamondSupportPlugin.obj
 0003:00000e23       _piecewise_construct       10033e23     DiamondSupportPlugin.obj
 0003:00000e24       _taskLog                   10033e24     DiamondSupportPlugin.obj
 0003:00000e2c       _algoLog                   10033e2c     DiamondSupportPlugin.obj
 0003:00000e34       _userActLog                10033e34     DiamondSupportPlugin.obj
 0003:00000e3c       _ioLog                     10033e3c     DiamondSupportPlugin.obj
 0003:00000e44       _coreLog                   10033e44     DiamondSupportPlugin.obj
 0003:00000e4c       _uiLog                     10033e4c     DiamondSupportPlugin.obj
 0003:00000e54       _scriptLog                 10033e54     DiamondSupportPlugin.obj
 0003:00000e60       _perfLog                   10033e60     DiamondSupportPlugin.obj
 0003:00000e68       _cmdLog                    10033e68     DiamondSupportPlugin.obj
 0003:00000e74       __Tuple_alloc              10033e74     GenomesPreparationTask.obj
 0003:00000e75       _ignore                    10033e75     GenomesPreparationTask.obj
 0003:00000e76       _allocator_arg             10033e76     GenomesPreparationTask.obj
 0003:00000e77       _piecewise_construct       10033e77     GenomesPreparationTask.obj
 0003:00000e78       _taskLog                   10033e78     GenomesPreparationTask.obj
 0003:00000e80       _algoLog                   10033e80     GenomesPreparationTask.obj
 0003:00000e88       _userActLog                10033e88     GenomesPreparationTask.obj
 0003:00000e90       _ioLog                     10033e90     GenomesPreparationTask.obj
 0003:00000e98       _coreLog                   10033e98     GenomesPreparationTask.obj
 0003:00000ea0       _uiLog                     10033ea0     GenomesPreparationTask.obj
 0003:00000ea8       _scriptLog                 10033ea8     GenomesPreparationTask.obj
 0003:00000eb0       _perfLog                   10033eb0     GenomesPreparationTask.obj
 0003:00000eb8       _cmdLog                    10033eb8     GenomesPreparationTask.obj
 0003:00000ec0       __Tuple_alloc              10033ec0     moc_DiamondBuildPrompter.obj
 0003:00000ec1       _ignore                    10033ec1     moc_DiamondBuildPrompter.obj
 0003:00000ec2       _allocator_arg             10033ec2     moc_DiamondBuildPrompter.obj
 0003:00000ec3       _piecewise_construct       10033ec3     moc_DiamondBuildPrompter.obj
 0003:00000ec4       _taskLog                   10033ec4     moc_DiamondBuildPrompter.obj
 0003:00000ecc       _algoLog                   10033ecc     moc_DiamondBuildPrompter.obj
 0003:00000ed4       _userActLog                10033ed4     moc_DiamondBuildPrompter.obj
 0003:00000edc       _ioLog                     10033edc     moc_DiamondBuildPrompter.obj
 0003:00000ee4       _coreLog                   10033ee4     moc_DiamondBuildPrompter.obj
 0003:00000eec       _uiLog                     10033eec     moc_DiamondBuildPrompter.obj
 0003:00000ef4       _scriptLog                 10033ef4     moc_DiamondBuildPrompter.obj
 0003:00000efc       _perfLog                   10033efc     moc_DiamondBuildPrompter.obj
 0003:00000f04       _cmdLog                    10033f04     moc_DiamondBuildPrompter.obj
 0003:00000f0c       __Tuple_alloc              10033f0c     moc_DiamondBuildTask.obj
 0003:00000f0d       _ignore                    10033f0d     moc_DiamondBuildTask.obj
 0003:00000f0e       _allocator_arg             10033f0e     moc_DiamondBuildTask.obj
 0003:00000f0f       _piecewise_construct       10033f0f     moc_DiamondBuildTask.obj
 0003:00000f10       _taskLog                   10033f10     moc_DiamondBuildTask.obj
 0003:00000f18       _algoLog                   10033f18     moc_DiamondBuildTask.obj
 0003:00000f20       _userActLog                10033f20     moc_DiamondBuildTask.obj
 0003:00000f28       _ioLog                     10033f28     moc_DiamondBuildTask.obj
 0003:00000f30       _coreLog                   10033f30     moc_DiamondBuildTask.obj
 0003:00000f38       _uiLog                     10033f38     moc_DiamondBuildTask.obj
 0003:00000f40       _scriptLog                 10033f40     moc_DiamondBuildTask.obj
 0003:00000f48       _perfLog                   10033f48     moc_DiamondBuildTask.obj
 0003:00000f50       _cmdLog                    10033f50     moc_DiamondBuildTask.obj
 0003:00000f58       __Tuple_alloc              10033f58     moc_DiamondBuildWorker.obj
 0003:00000f59       _ignore                    10033f59     moc_DiamondBuildWorker.obj
 0003:00000f5a       _allocator_arg             10033f5a     moc_DiamondBuildWorker.obj
 0003:00000f5b       _piecewise_construct       10033f5b     moc_DiamondBuildWorker.obj
 0003:00000f5c       _taskLog                   10033f5c     moc_DiamondBuildWorker.obj
 0003:00000f64       _algoLog                   10033f64     moc_DiamondBuildWorker.obj
 0003:00000f6c       _userActLog                10033f6c     moc_DiamondBuildWorker.obj
 0003:00000f74       _ioLog                     10033f74     moc_DiamondBuildWorker.obj
 0003:00000f7c       _coreLog                   10033f7c     moc_DiamondBuildWorker.obj
 0003:00000f84       _uiLog                     10033f84     moc_DiamondBuildWorker.obj
 0003:00000f8c       _scriptLog                 10033f8c     moc_DiamondBuildWorker.obj
 0003:00000f94       _perfLog                   10033f94     moc_DiamondBuildWorker.obj
 0003:00000f9c       _cmdLog                    10033f9c     moc_DiamondBuildWorker.obj
 0003:00000fa8       __Tuple_alloc              10033fa8     moc_DiamondClassifyPrompter.obj
 0003:00000fa9       _ignore                    10033fa9     moc_DiamondClassifyPrompter.obj
 0003:00000faa       _allocator_arg             10033faa     moc_DiamondClassifyPrompter.obj
 0003:00000fab       _piecewise_construct       10033fab     moc_DiamondClassifyPrompter.obj
 0003:00000fac       _taskLog                   10033fac     moc_DiamondClassifyPrompter.obj
 0003:00000fb4       _algoLog                   10033fb4     moc_DiamondClassifyPrompter.obj
 0003:00000fbc       _userActLog                10033fbc     moc_DiamondClassifyPrompter.obj
 0003:00000fc4       _ioLog                     10033fc4     moc_DiamondClassifyPrompter.obj
 0003:00000fcc       _coreLog                   10033fcc     moc_DiamondClassifyPrompter.obj
 0003:00000fd4       _uiLog                     10033fd4     moc_DiamondClassifyPrompter.obj
 0003:00000fdc       _scriptLog                 10033fdc     moc_DiamondClassifyPrompter.obj
 0003:00000fe4       _perfLog                   10033fe4     moc_DiamondClassifyPrompter.obj
 0003:00000fec       _cmdLog                    10033fec     moc_DiamondClassifyPrompter.obj
 0003:00000ff4       __Tuple_alloc              10033ff4     moc_DiamondClassifyTask.obj
 0003:00000ff5       _ignore                    10033ff5     moc_DiamondClassifyTask.obj
 0003:00000ff6       _allocator_arg             10033ff6     moc_DiamondClassifyTask.obj
 0003:00000ff7       _piecewise_construct       10033ff7     moc_DiamondClassifyTask.obj
 0003:00000ff8       _taskLog                   10033ff8     moc_DiamondClassifyTask.obj
 0003:00001000       _algoLog                   10034000     moc_DiamondClassifyTask.obj
 0003:00001008       _userActLog                10034008     moc_DiamondClassifyTask.obj
 0003:00001010       _ioLog                     10034010     moc_DiamondClassifyTask.obj
 0003:00001018       _coreLog                   10034018     moc_DiamondClassifyTask.obj
 0003:00001020       _uiLog                     10034020     moc_DiamondClassifyTask.obj
 0003:00001028       _scriptLog                 10034028     moc_DiamondClassifyTask.obj
 0003:00001030       _perfLog                   10034030     moc_DiamondClassifyTask.obj
 0003:00001038       _cmdLog                    10034038     moc_DiamondClassifyTask.obj
 0003:00001040       __Tuple_alloc              10034040     moc_DiamondClassifyWorker.obj
 0003:00001041       _ignore                    10034041     moc_DiamondClassifyWorker.obj
 0003:00001042       _allocator_arg             10034042     moc_DiamondClassifyWorker.obj
 0003:00001043       _piecewise_construct       10034043     moc_DiamondClassifyWorker.obj
 0003:00001044       _taskLog                   10034044     moc_DiamondClassifyWorker.obj
 0003:0000104c       _algoLog                   1003404c     moc_DiamondClassifyWorker.obj
 0003:00001054       _userActLog                10034054     moc_DiamondClassifyWorker.obj
 0003:0000105c       _ioLog                     1003405c     moc_DiamondClassifyWorker.obj
 0003:00001064       _coreLog                   10034064     moc_DiamondClassifyWorker.obj
 0003:0000106c       _uiLog                     1003406c     moc_DiamondClassifyWorker.obj
 0003:00001074       _scriptLog                 10034074     moc_DiamondClassifyWorker.obj
 0003:0000107c       _perfLog                   1003407c     moc_DiamondClassifyWorker.obj
 0003:00001084       _cmdLog                    10034084     moc_DiamondClassifyWorker.obj
 0003:0000108c       __Tuple_alloc              1003408c     moc_DiamondSupport.obj
 0003:0000108d       _ignore                    1003408d     moc_DiamondSupport.obj
 0003:0000108e       _allocator_arg             1003408e     moc_DiamondSupport.obj
 0003:0000108f       _piecewise_construct       1003408f     moc_DiamondSupport.obj
 0003:00001090       __Tuple_alloc              10034090     moc_DiamondSupportPlugin.obj
 0003:00001091       _ignore                    10034091     moc_DiamondSupportPlugin.obj
 0003:00001092       _allocator_arg             10034092     moc_DiamondSupportPlugin.obj
 0003:00001093       _piecewise_construct       10034093     moc_DiamondSupportPlugin.obj
 0003:00001094       __Tuple_alloc              10034094     moc_GenomesPreparationTask.obj
 0003:00001095       _ignore                    10034095     moc_GenomesPreparationTask.obj
 0003:00001096       _allocator_arg             10034096     moc_GenomesPreparationTask.obj
 0003:00001097       _piecewise_construct       10034097     moc_GenomesPreparationTask.obj
 0003:00001098       _taskLog                   10034098     moc_GenomesPreparationTask.obj
 0003:000010a0       _algoLog                   100340a0     moc_GenomesPreparationTask.obj
 0003:000010a8       _userActLog                100340a8     moc_GenomesPreparationTask.obj
 0003:000010b0       _ioLog                     100340b0     moc_GenomesPreparationTask.obj
 0003:000010b8       _coreLog                   100340b8     moc_GenomesPreparationTask.obj
 0003:000010c0       _uiLog                     100340c0     moc_GenomesPreparationTask.obj
 0003:000010c8       _scriptLog                 100340c8     moc_GenomesPreparationTask.obj
 0003:000010d0       _perfLog                   100340d0     moc_GenomesPreparationTask.obj
 0003:000010d8       _cmdLog                    100340d8     moc_GenomesPreparationTask.obj
 0003:000010e0       ___proc_attached           100340e0     MSVCRT:crtdll.obj
 0003:000010e8       _GS_ExceptionRecord        100340e8     MSVCRT:gs_report.obj
 0003:00001138       _GS_ContextRecord          10034138     MSVCRT:gs_report.obj
 0003:00001404       _DebuggerWasPresent        10034404     MSVCRT:gs_report.obj
 0004:00000060       $R000000                   10035060     * linker generated manifest res *

 Exports

  ordinal    name

        1    _ugene_plugin_init
               exported name: ugene_plugin_init
